 LenRCServer

 Timestamp is 54265c01 (Sat Sep 27 14:41:05 2014)

 Preferred load address is 00400000

 Start         Length     Name                   Class
 0001:00000000 00076c1eH .text                   CODE
 0001:00076c20 00009431H .text$x                 CODE
 0001:00080060 0000024eH .text$yc                CODE
 0001:000802b0 0000011cH .text$yd                CODE
 0002:00000000 000013b0H .idata$5                DATA
 0002:000013b0 00000004H .CRT$XCA                DATA
 0002:000013b4 00000004H .CRT$XCAA               DATA
 0002:000013b8 00000004H .CRT$XCL                DATA
 0002:000013bc 00000048H .CRT$XCU                DATA
 0002:00001404 00000004H .CRT$XCZ                DATA
 0002:00001408 00000004H .CRT$XIA                DATA
 0002:0000140c 00000004H .CRT$XIAA               DATA
 0002:00001410 00000004H .CRT$XIC                DATA
 0002:00001414 00000004H .CRT$XIY                DATA
 0002:00001418 00000004H .CRT$XIZ                DATA
 0002:00001420 000165e8H .rdata                  DATA
 0002:00017a08 0000004aH .rdata$debug            DATA
 0002:00017a54 00002964H .rdata$r                DATA
 0002:0001a3c0 00000560H .rdata$sxdata           DATA
 0002:0001a920 00000004H .rtc$IAA                DATA
 0002:0001a924 00000004H .rtc$IZZ                DATA
 0002:0001a928 00000004H .rtc$TAA                DATA
 0002:0001a92c 00000004H .rtc$TZZ                DATA
 0002:0001a930 00007d88H .xdata$x                DATA
 0002:000226b8 00000000H ATL$__a                 DATA
 0002:000226b8 00000000H ATL$__z                 DATA
 0002:000226b8 00000020H .didat$2                DATA
 0002:000226d8 00000020H .didat$3                DATA
 0002:000226f8 00000008H .didat$4                DATA
 0002:00022700 00000008H .didat$7                DATA
 0002:00022708 000001b8H .idata$2                DATA
 0002:000228c0 00000014H .idata$3                DATA
 0002:000228d4 000013b0H .idata$4                DATA
 0002:00023c84 000012faH .idata$6                DATA
 0002:00024f7e 00000000H .edata                  DATA
 0003:00000000 000014e4H .data                   DATA
 0003:000014e4 00000008H .didat$5                DATA
 0003:000014f0 000019c0H .bss                    DATA
 0004:00000000 00002c08H .rsrc$01                DATA
 0004:00002c10 0011fa40H .rsrc$02                DATA

  Address         Publics by Value              Rva+Base       Lib:Object

 0000:00000000       __except_list              00000000     <absolute>
 0000:00000158       ___safe_se_handler_count   00000158     <absolute>
 0000:00009876       __fltused                  00009876     <absolute>
 0000:00009876       __ldused                   00009876     <absolute>
 0000:00000000       ___ImageBase               00400000     <linker-defined>
 0001:00000000       ?GetRuntimeClass@CAboutDlg@@UBEPAUCRuntimeClass@@XZ 00401000 f   AboutDlg.obj
 0001:00000010       ??0CAboutDlg@@QAE@PAVCWnd@@@Z 00401010 f   AboutDlg.obj
 0001:000000d0       ??_ECAboutDlg@@UAEPAXI@Z   004010d0 f i AboutDlg.obj
 0001:000000d0       ??_GCAboutDlg@@UAEPAXI@Z   004010d0 f i AboutDlg.obj
 0001:00000100       ??1CAboutDlg@@UAE@XZ       00401100 f   AboutDlg.obj
 0001:000001b0       ?DoDataExchange@CAboutDlg@@MAEXPAVCDataExchange@@@Z 004011b0 f   AboutDlg.obj
 0001:00000240       ?GetMessageMap@CAboutDlg@@MBEPBUAFX_MSGMAP@@XZ 00401240 f   AboutDlg.obj
 0001:00000250       ?GetThisMessageMap@CAboutDlg@@KGPBUAFX_MSGMAP@@XZ 00401250 f   AboutDlg.obj
 0001:00000260       ?OnInitDialog@CAboutDlg@@MAEHXZ 00401260 f   AboutDlg.obj
 0001:00000730       ?SetTitle@CAboutDlg@@QAEXXZ 00401730 f   AboutDlg.obj
 0001:00000910       ?OnBnClickedButton1@CAboutDlg@@QAEXXZ 00401910 f   AboutDlg.obj
 0001:00000b10       ??3CObject@@SGXPAX@Z       00401b10 f i AboutDlg.obj
 0001:00000b30       ?BeginModalState@CWnd@@UAEXXZ 00401b30 f i AboutDlg.obj
 0001:00000b50       ?EndModalState@CWnd@@UAEXXZ 00401b50 f i AboutDlg.obj
 0001:00000b70       ?Create@CDialog@@UAEHIPAVCWnd@@@Z 00401b70 f i AboutDlg.obj
 0001:00000b90       ??0CStatic@@QAE@XZ         00401b90 f i AboutDlg.obj
 0001:00000bb0       ??_GCStatic@@UAEPAXI@Z     00401bb0 f i AboutDlg.obj
 0001:00000bb0       ??_ECStatic@@UAEPAXI@Z     00401bb0 f i AboutDlg.obj
 0001:00000be0       ??HATL@@YA?AV?$CStringT@DV?$StrTraitMFC_DLL@DV?$ChTraitsCRT@D@ATL@@@@@0@ABV10@PBD@Z 00401be0 f i AboutDlg.obj
 0001:00000ca0       ??HATL@@YA?AV?$CStringT@DV?$StrTraitMFC_DLL@DV?$ChTraitsCRT@D@ATL@@@@@0@PBDABV10@@Z 00401ca0 f i AboutDlg.obj
 0001:00000d60       ??0CAddToGroup@@QAE@PAVCWnd@@@Z 00401d60 f   AddToGroup.obj
 0001:00000e00       ??_ECAddToGroup@@UAEPAXI@Z 00401e00 f i AddToGroup.obj
 0001:00000e00       ??_GCAddToGroup@@UAEPAXI@Z 00401e00 f i AddToGroup.obj
 0001:00000e30       ??1CAddToGroup@@UAE@XZ     00401e30 f i AddToGroup.obj
 0001:00000ea0       ?DoDataExchange@CAddToGroup@@MAEXPAVCDataExchange@@@Z 00401ea0 f   AddToGroup.obj
 0001:00000ef0       ?OnOK@CAddToGroup@@MAEXXZ  00401ef0 f   AddToGroup.obj
 0001:00000f10       ?OnInitDialog@CAddToGroup@@MAEHXZ 00401f10 f   AddToGroup.obj
 0001:00001220       ?SortGroup@CAddToGroup@@QAEHAAVCStringList@@@Z 00402220 f   AddToGroup.obj
 0001:000013b0       ?GetHeadPosition@?$CList@PAVCFtpdPi@@PAV1@@@QBEPAU__POSITION@@XZ 004023b0 f i CFtpd.obj
 0001:000013b0       ??BCBlockingSocket@@QAEIXZ 004023b0 f i blocksock.obj
 0001:000013b0       ?GetHeadPosition@CStringList@@QBEPAU__POSITION@@XZ 004023b0 f i AddToGroup.obj
 0001:000013d0       ?GetNext@CStringList@@QAEAAV?$CStringT@DV?$StrTraitMFC_DLL@DV?$ChTraitsCRT@D@ATL@@@@@ATL@@AAPAU__POSITION@@@Z 004023d0 f i AddToGroup.obj
 0001:00001410       ?GetAt@CStringList@@QAEAAV?$CStringT@DV?$StrTraitMFC_DLL@DV?$ChTraitsCRT@D@ATL@@@@@ATL@@PAU__POSITION@@@Z 00402410 f i AddToGroup.obj
 0001:00001440       ?SetAt@CStringList@@QAEXPAU__POSITION@@ABV?$CStringT@DV?$StrTraitMFC_DLL@DV?$ChTraitsCRT@D@ATL@@@@@ATL@@@Z 00402440 f i AddToGroup.obj
 0001:00001470       ?GetStartPosition@CMapStringToString@@QBEPAU__POSITION@@XZ 00402470 f i PropertyViewDlg.obj
 0001:00001470       ?GetStartPosition@CMapPtrToPtr@@QBEPAU__POSITION@@XZ 00402470 f i IOCPImplement.obj
 0001:00001470       ?GetStartPosition@CMapStringToPtr@@QBEPAU__POSITION@@XZ 00402470 f i AddToGroup.obj
 0001:00001490       ??0CComboBox@@QAE@XZ       00402490 f i AddToGroup.obj
 0001:000014b0       ??_GCComboBox@@UAEPAXI@Z   004024b0 f i AddToGroup.obj
 0001:000014b0       ??_ECComboBox@@UAEPAXI@Z   004024b0 f i AddToGroup.obj
 0001:000014e0       ?SetCurSel@CComboBox@@QAEHH@Z 004024e0 f i AddToGroup.obj
 0001:00001510       ?AddString@CComboBox@@QAEHPBD@Z 00402510 f i AddToGroup.obj
 0001:00001540       ??8ATL@@YA_NABV?$CStringT@DV?$StrTraitMFC_DLL@DV?$ChTraitsCRT@D@ATL@@@@@0@0@Z 00402540 f i AddToGroup.obj
 0001:00001560       ??0CBlackListDlg@@QAE@PAVCWnd@@@Z 00402560 f   BlackListDlg.obj
 0001:000015d0       ??_GCBlackListDlg@@UAEPAXI@Z 004025d0 f i BlackListDlg.obj
 0001:000015d0       ??_ECBlackListDlg@@UAEPAXI@Z 004025d0 f i BlackListDlg.obj
 0001:00001600       ?DoDataExchange@CBlackListDlg@@MAEXPAVCDataExchange@@@Z 00402600 f   BlackListDlg.obj
 0001:00001630       ?GetMessageMap@CBlackListDlg@@MBEPBUAFX_MSGMAP@@XZ 00402630 f   BlackListDlg.obj
 0001:00001640       ?GetThisMessageMap@CBlackListDlg@@KGPBUAFX_MSGMAP@@XZ 00402640 f   BlackListDlg.obj
 0001:00001650       ?OnInitDialog@CBlackListDlg@@MAEHXZ 00402650 f   BlackListDlg.obj
 0001:000019f0       ?OnOK@CBlackListDlg@@MAEXXZ 004029f0 f   BlackListDlg.obj
 0001:00001c80       ??1CBlackListDlg@@UAE@XZ   00402c80 f   BlackListDlg.obj
 0001:00001ce0       ?OnBnClickedSelall@CBlackListDlg@@QAEXXZ 00402ce0 f   BlackListDlg.obj
 0001:00001d40       ??0CListCtrl@@QAE@XZ       00402d40 f i BlackListDlg.obj
 0001:00001d60       ??_GCListCtrl@@UAEPAXI@Z   00402d60 f i BlackListDlg.obj
 0001:00001d60       ??_ECListCtrl@@UAEPAXI@Z   00402d60 f i BlackListDlg.obj
 0001:00001d90       ?GetItemCount@CListCtrl@@QBEHXZ 00402d90 f i BlackListDlg.obj
 0001:00001dc0       ?InsertItem@CListCtrl@@QAEHHPBDH@Z 00402dc0 f i BlackListDlg.obj
 0001:00001df0       ?DeleteItem@CListCtrl@@QAEHH@Z 00402df0 f i BlackListDlg.obj
 0001:00001e20       ?GetFirstSelectedItemPosition@CListCtrl@@QBEPAU__POSITION@@XZ 00402e20 f i BlackListDlg.obj
 0001:00001e40       ?GetNextItem@CListCtrl@@QBEHHH@Z 00402e40 f i BlackListDlg.obj
 0001:00001e70       ?GetNextSelectedItem@CListCtrl@@QBEHAAPAU__POSITION@@@Z 00402e70 f i BlackListDlg.obj
 0001:00001eb0       ?SetExtendedStyle@CListCtrl@@QAEKK@Z 00402eb0 f i BlackListDlg.obj
 0001:00001ee0       ?GetExtendedStyle@CListCtrl@@QBEKXZ 00402ee0 f i BlackListDlg.obj
 0001:00001f10       ?_GetBaseClass@CBlockingSocketException@@KGPAUCRuntimeClass@@XZ 00402f10 f   blocksock.obj
 0001:00001f20       ?GetRuntimeClass@CBlockingSocketException@@UBEPAUCRuntimeClass@@XZ 00402f20 f   blocksock.obj
 0001:00001f30       ??0CBlockingSocketException@@QAE@PAD@Z 00402f30 f   blocksock.obj
 0001:00001fc0       ??_ECBlockingSocketException@@UAEPAXI@Z 00402fc0 f i blocksock.obj
 0001:00001fc0       ??_GCBlockingSocketException@@UAEPAXI@Z 00402fc0 f i blocksock.obj
 0001:00001ff0       ??1CBlockingSocketException@@UAE@XZ 00402ff0 f i blocksock.obj
 0001:00002020       ?GetErrorMessage@CBlockingSocketException@@UAEHPADIPAI@Z 00403020 f   blocksock.obj
 0001:000020d0       ?_GetBaseClass@CBlockingSocket@@KGPAUCRuntimeClass@@XZ 004030d0 f   blocksock.obj
 0001:000020e0       ?GetRuntimeClass@CBlockingSocket@@UBEPAUCRuntimeClass@@XZ 004030e0 f   blocksock.obj
 0001:000020f0       ?Create@CBlockingSocket@@QAE_NH@Z 004030f0 f   blocksock.obj
 0001:00002130       ?Bind@CBlockingSocket@@QAE_NPBUsockaddr@@@Z 00403130 f   blocksock.obj
 0001:00002160       ?Listen@CBlockingSocket@@QAE_NXZ 00403160 f   blocksock.obj
 0001:00002190       ?Accept@CBlockingSocket@@QAEHAAV1@PAUsockaddr@@@Z 00403190 f   blocksock.obj
 0001:00002260       ?Close@CBlockingSocket@@QAEXXZ 00403260 f   blocksock.obj
 0001:00002310       ?Connect@CBlockingSocket@@QAE_NPBUsockaddr@@@Z 00403310 f   blocksock.obj
 0001:00002340       ?Send@CBlockingSocket@@QAEHPBDHH@Z 00403340 f   blocksock.obj
 0001:000024e0       ?Receive@CBlockingSocket@@QAEHPADHH@Z 004034e0 f   blocksock.obj
 0001:00002680       ??0CBlockingSocket@@QAE@XZ 00403680 f i blocksock.obj
 0001:000026b0       ??_ECBlockingSocket@@UAEPAXI@Z 004036b0 f i blocksock.obj
 0001:000026b0       ??_GCBlockingSocket@@UAEPAXI@Z 004036b0 f i blocksock.obj
 0001:000026e0       ?OnMsgEdit@CMainFrame@@QAEXXZ 004036e0 f i MainFrm.obj
 0001:000026e0       ?OnAppAbout@CKiboManagerApp@@QAEXXZ 004036e0 f i KiboManager.obj
 0001:000026e0       ?SaveCustomState@CKiboManagerApp@@UAEXXZ 004036e0 f i KiboManager.obj
 0001:000026e0       ?OnContinueMoving@CDockablePane@@MAEXXZ 004036e0 f i MainFrm.obj
 0001:000026e0       ?OnScheduleset@CMainFrame@@QAEXXZ 004036e0 f i MainFrm.obj
 0001:000026e0       ?PreSaveState@CWinAppEx@@MAEXXZ 004036e0 f i KiboManager.obj
 0001:000026e0       ?ToggleAutoHide@CPane@@UAEXXZ 004036e0 f i MFCRibbonBarNew.obj
 0001:000026e0       ?AdjustLayout@CBasePane@@UAEXXZ 004036e0 f i MainFrm.obj
 0001:000026e0       ?AssertValid@CObject@@UBEXXZ 004036e0 f i AboutDlg.obj
 0001:000026e0       ?DestroyCtrl@CMFCRibbonBaseElement@@UAEXXZ 004036e0 f i MainFrm.obj
 0001:000026e0       ?OnEnChangeEditDelaysec@CClientSettingsDlg@@QAEXXZ 004036e0 f i ClientSettingsDlg.obj
 0001:000026e0       ?OnSettings@CMainFrame@@QAEXXZ 004036e0 f i MainFrm.obj
 0001:000026e0       ?OnMsginteract@CMainFrame@@QAEXXZ 004036e0 f i MainFrm.obj
 0001:000026e0       ?OnRemoteoperation@CMainFrame@@QAEXXZ 004036e0 f i MainFrm.obj
 0001:000026e0       ?OnStnClickedStaticInfo@CProgressDlg@@QAEXXZ 004036e0 f i ProgressDlg.obj
 0001:000026e0       ??1CObject@@UAE@XZ         004036e0 f i blocksock.obj
 0001:000026e0       ?OnProtectandtrans@CMainFrame@@QAEXXZ 004036e0 f i MainFrm.obj
 0001:000026e0       ?OnPropertymanagement@CMainFrame@@QAEXXZ 004036e0 f i MainFrm.obj
 0001:000026e0       ??1_Container_base_aux@std@@QAE@XZ 004036e0 f i KiboManagerView.obj
 0001:000026e0       ?OnDrawCaption@CBasePane@@UAEXXZ 004036e0 f i MainFrm.obj
 0001:000026e0       ?StretchHorizontally@CMFCRibbonBaseElement@@UAEXXZ 004036e0 f i MainFrm.obj
 0001:000026e0       ?LoadCustomState@CKiboManagerApp@@UAEXXZ 004036e0 f i KiboManager.obj
 0001:000026f0       ??2CObject@@SGPAXI@Z       004036f0 f i blocksock.obj
 0001:00002710       ??1CException@@UAE@XZ      00403710 f i blocksock.obj
 0001:00002710       ??1CBlockingSocket@@UAE@XZ 00403710 f i blocksock.obj
 0001:00002730       ??0CBootModuleManager@@QAE@XZ 00403730 f   BootModuleManager.obj
 0001:000027c0       ??_ECBootModuleManager@@UAEPAXI@Z 004037c0 f i BootModuleManager.obj
 0001:000027c0       ??_GCBootModuleManager@@UAEPAXI@Z 004037c0 f i BootModuleManager.obj
 0001:000027f0       ??1?$CTypedPtrList@VCPtrList@@PAUPartitionTransInfo@@@@UAE@XZ 004037f0 f i MainFrm.obj
 0001:000027f0       ??1?$CTypedPtrList@VCPtrList@@PAUtagRECVREQUEST@@@@UAE@XZ 004037f0 f i MainFrm.obj
 0001:000027f0       ??1?$CTypedPtrList@VCPtrList@@PAK@@UAE@XZ 004037f0 f i BootModuleManager.obj
 0001:00002810       ??1CBootModuleManager@@UAE@XZ 00403810 f   BootModuleManager.obj
 0001:000028a0       ?GetBootParamInfo@CBootModuleManager@@QAEHXZ 004038a0 f   BootModuleManager.obj
 0001:00002a00       ?ClearCommand@CBootModuleManager@@QAEXXZ 00403a00 f   BootModuleManager.obj
 0001:00002a50       ?GetPartitionProtectType@CBootModuleManager@@QAEEE@Z 00403a50 f   BootModuleManager.obj
 0001:00002b00       ??0?$CTypedPtrList@VCPtrList@@PAK@@QAE@H@Z 00403b00 f i BootModuleManager.obj
 0001:00002b30       ??_G?$CTypedPtrList@VCPtrList@@PAK@@UAEPAXI@Z 00403b30 f i BootModuleManager.obj
 0001:00002b30       ??_G?$CTypedPtrList@VCPtrList@@PAUtagRECVREQUEST@@@@UAEPAXI@Z 00403b30 f i MainFrm.obj
 0001:00002b30       ??_E?$CTypedPtrList@VCPtrList@@PAUtagRECVREQUEST@@@@UAEPAXI@Z 00403b30 f i MainFrm.obj
 0001:00002b30       ??_E?$CTypedPtrList@VCPtrList@@PAK@@UAEPAXI@Z 00403b30 f i BootModuleManager.obj
 0001:00002b30       ??_G?$CTypedPtrList@VCPtrList@@PAUPartitionTransInfo@@@@UAEPAXI@Z 00403b30 f i MainFrm.obj
 0001:00002b30       ??_E?$CTypedPtrList@VCPtrList@@PAUPartitionTransInfo@@@@UAEPAXI@Z 00403b30 f i MainFrm.obj
 0001:00002b60       ??0?$_CTypedPtrList@VCPtrList@@PAK@@QAE@H@Z 00403b60 f i BootModuleManager.obj
 0001:00002b90       ??_G?$_CTypedPtrList@VCPtrList@@PAUtagRECVREQUEST@@@@UAEPAXI@Z 00403b90 f i MainFrm.obj
 0001:00002b90       ??_G?$_CTypedPtrList@VCPtrList@@PAK@@UAEPAXI@Z 00403b90 f i BootModuleManager.obj
 0001:00002b90       ??_E?$_CTypedPtrList@VCPtrList@@PAUtagRECVREQUEST@@@@UAEPAXI@Z 00403b90 f i MainFrm.obj
 0001:00002b90       ??_E?$_CTypedPtrList@VCPtrList@@PAK@@UAEPAXI@Z 00403b90 f i BootModuleManager.obj
 0001:00002b90       ??_E?$_CTypedPtrList@VCPtrList@@PAUPartitionTransInfo@@@@UAEPAXI@Z 00403b90 f i MainFrm.obj
 0001:00002b90       ??_G?$_CTypedPtrList@VCPtrList@@PAUPartitionTransInfo@@@@UAEPAXI@Z 00403b90 f i MainFrm.obj
 0001:00002bc0       ??0CCriticalSection@@QAE@XZ 00403bc0 f i BootModuleManager.obj
 0001:00002c40       ?OnTearOffMenu@CFrameWndEx@@UAEHPAVCMFCPopupMenu@@PAVCPane@@@Z 00403c40 f i MainFrm.obj
 0001:00002c40       ?Unlock@CSyncObject@@UAEHJPAJ@Z 00403c40 f i BootModuleManager.obj
 0001:00002c60       ?Init@CCriticalSection@@AAEHXZ 00403c60 f i BootModuleManager.obj
 0001:00002d00       ??_GCCriticalSection@@UAEPAXI@Z 00403d00 f i BootModuleManager.obj
 0001:00002d00       ??_ECCriticalSection@@UAEPAXI@Z 00403d00 f i BootModuleManager.obj
 0001:00002d30       ??1CCriticalSection@@UAE@XZ 00403d30 f i BootModuleManager.obj
 0001:00002d60       ?Lock@CCriticalSection@@UAEHK@Z 00403d60 f i BootModuleManager.obj
 0001:00002d80       ?Lock@CCriticalSection@@QAEHXZ 00403d80 f i BootModuleManager.obj
 0001:00002e20       ?Unlock@CCriticalSection@@UAEHXZ 00403e20 f i BootModuleManager.obj
 0001:00002e40       ?_GetBaseClass@CSetDrfaultNICDlg@@KGPAUCRuntimeClass@@XZ 00403e40 f   SetDrfaultNICDlg.obj
 0001:00002e40       ?_GetBaseClass@CSetClientchancelDLg@@KGPAUCRuntimeClass@@XZ 00403e40 f   SetClientchancelDLg.obj
 0001:00002e40       ?_GetBaseClass@CLoginPasswordDlg@@KGPAUCRuntimeClass@@XZ 00403e40 f   LoginPasswordDlg.obj
 0001:00002e40       ?_GetBaseClass@CGroupExt@@KGPAUCRuntimeClass@@XZ 00403e40 f   GroupExt.obj
 0001:00002e40       ?_GetBaseClass@CPortChannelDlg@@KGPAUCRuntimeClass@@XZ 00403e40 f   PortChannelDlg.obj
 0001:00002e40       ?_GetBaseClass@CMsgDlg@@KGPAUCRuntimeClass@@XZ 00403e40 f   MsgDlg.obj
 0001:00002e40       ?_GetBaseClass@CPortCtrlDlg@@KGPAUCRuntimeClass@@XZ 00403e40 f   PortCtrlDlg.obj
 0001:00002e40       ?_GetBaseClass@CBroadIE@@KGPAUCRuntimeClass@@XZ 00403e40 f   BroadIE.obj
 0001:00002e40       ?_GetBaseClass@CAboutDlg@@KGPAUCRuntimeClass@@XZ 00403e40 f   AboutDlg.obj
 0001:00002e40       ?_GetBaseClass@CBroadWaitDlg@@KGPAUCRuntimeClass@@XZ 00403e40 f   BroadWaitDlg.obj
 0001:00002e40       ?_GetBaseClass@CSpecialPartitionRS@@KGPAUCRuntimeClass@@XZ 00403e40 f   SpecialPartitionRS.obj
 0001:00002e40       ?_GetBaseClass@CExecuteProcedure@@KGPAUCRuntimeClass@@XZ 00403e40 f   ExecuteProcedure.obj
 0001:00002e50       ?GetRuntimeClass@CBroadIE@@UBEPAUCRuntimeClass@@XZ 00403e50 f   BroadIE.obj
 0001:00002e60       ??0CBroadIE@@QAE@PAVCWnd@@@Z 00403e60 f   BroadIE.obj
 0001:00002f20       ??_ECBroadIE@@UAEPAXI@Z    00403f20 f i BroadIE.obj
 0001:00002f20       ??_GCBroadIE@@UAEPAXI@Z    00403f20 f i BroadIE.obj
 0001:00002f50       ??1CBroadIE@@UAE@XZ        00403f50 f   BroadIE.obj
 0001:00002fd0       ?DoDataExchange@CBroadIE@@MAEXPAVCDataExchange@@@Z 00403fd0 f   BroadIE.obj
 0001:00003050       ?GetMessageMap@CBroadIE@@MBEPBUAFX_MSGMAP@@XZ 00404050 f   BroadIE.obj
 0001:00003060       ?GetThisMessageMap@CBroadIE@@KGPBUAFX_MSGMAP@@XZ 00404060 f   BroadIE.obj
 0001:00003070       ?OnInitDialog@CBroadIE@@MAEHXZ 00404070 f   BroadIE.obj
 0001:000033f0       ?OnBnClickedOk@CBroadIE@@QAEXXZ 004043f0 f   BroadIE.obj
 0001:00003b50       ?OnBnClickedClear@CBroadIE@@QAEXXZ 00404b50 f   BroadIE.obj
 0001:00003c00       ?OnBnClickedCheckStart@CBroadIE@@QAEXXZ 00404c00 f   BroadIE.obj
 0001:00003c60       ?GetRuntimeClass@CBroadWaitDlg@@UBEPAUCRuntimeClass@@XZ 00404c60 f   BroadWaitDlg.obj
 0001:00003c70       ??0CBroadWaitDlg@@QAE@PAVCWnd@@@Z 00404c70 f   BroadWaitDlg.obj
 0001:00003d00       ??_ECBroadWaitDlg@@UAEPAXI@Z 00404d00 f i BroadWaitDlg.obj
 0001:00003d00       ??_GCBroadWaitDlg@@UAEPAXI@Z 00404d00 f i BroadWaitDlg.obj
 0001:00003d30       ??1CBroadWaitDlg@@UAE@XZ   00404d30 f   BroadWaitDlg.obj
 0001:00003dc0       ?DoDataExchange@CBroadWaitDlg@@MAEXPAVCDataExchange@@@Z 00404dc0 f   BroadWaitDlg.obj
 0001:00003e00       ?GetMessageMap@CBroadWaitDlg@@MBEPBUAFX_MSGMAP@@XZ 00404e00 f   BroadWaitDlg.obj
 0001:00003e10       ?GetThisMessageMap@CBroadWaitDlg@@KGPBUAFX_MSGMAP@@XZ 00404e10 f   BroadWaitDlg.obj
 0001:00003e20       ?ReEnableParent@CBroadWaitDlg@@QAEXXZ 00404e20 f   BroadWaitDlg.obj
 0001:00003e60       ?OnInitDialog@CBroadWaitDlg@@UAEHXZ 00404e60 f   BroadWaitDlg.obj
 0001:00003f20       ?OnClose@CBroadWaitDlg@@QAEXXZ 00404f20 f   BroadWaitDlg.obj
 0001:00003f40       ?Create@CBroadWaitDlg@@QAEHPAVCWnd@@@Z 00404f40 f   BroadWaitDlg.obj
 0001:00003fc0       ?DestroyWindow@CBroadWaitDlg@@UAEHXZ 00404fc0 f   BroadWaitDlg.obj
 0001:00003fe0       ?WaitStart@CBroadWaitDlg@@QAEHV?$CStringT@DV?$StrTraitMFC_DLL@DV?$ChTraitsCRT@D@ATL@@@@@ATL@@0HPAVCWnd@@@Z 00404fe0 f   BroadWaitDlg.obj
 0001:00004150       ?OnTimer@CBroadWaitDlg@@QAEXI@Z 00405150 f   BroadWaitDlg.obj
 0001:00004170       ?PreTranslateMessage@CBroadWaitDlg@@UAEHPAUtagMSG@@@Z 00405170 f   BroadWaitDlg.obj
 0001:000041d0       ?UpdateWindow@CWnd@@QAEXXZ 004051d0 f i BroadWaitDlg.obj
 0001:000041f0       ?OnClose@CWnd@@IAEXXZ      004051f0 f i BroadWaitDlg.obj
 0001:00004210       ??0CCalendarBar@@QAE@XZ    00405210 f   CalendarBar.obj
 0001:000042a0       ??_GCCalendarBar@@UAEPAXI@Z 004052a0 f i CalendarBar.obj
 0001:000042a0       ??_ECCalendarBar@@UAEPAXI@Z 004052a0 f i CalendarBar.obj
 0001:000042d0       ??1CCalendarBar@@UAE@XZ    004052d0 f   CalendarBar.obj
 0001:00004350       ?GetMessageMap@CCalendarBar@@MBEPBUAFX_MSGMAP@@XZ 00405350 f   CalendarBar.obj
 0001:00004360       ?GetThisMessageMap@CCalendarBar@@KGPBUAFX_MSGMAP@@XZ 00405360 f   CalendarBar.obj
 0001:00004370       ?OnCreate@CCalendarBar@@IAEHPAUtagCREATESTRUCTA@@@Z 00405370 f   CalendarBar.obj
 0001:00004460       ?OnSize@CCalendarBar@@IAEXIHH@Z 00405460 f   CalendarBar.obj
 0001:000044d0       ?Create@CCalendarBar@@UAEHABUtagRECT@@PAVCWnd@@I@Z 004054d0 f   CalendarBar.obj
 0001:00004500       ?OnPaint@CCalendarBar@@IAEXXZ 00405500 f   CalendarBar.obj
 0001:00004920       ??0CRect@@QAE@HHHH@Z       00405920 f i CalendarBar.obj
 0001:00004960       ?DeflateRect@CRect@@QAEXHH@Z 00405960 f i CalendarBar.obj
 0001:00004990       ??0CBitmap@@QAE@XZ         00405990 f i CalendarBar.obj
 0001:000049b0       ??0CGdiObject@@QAE@XZ      004059b0 f i CalendarBar.obj
 0001:000049e0       ??_ECGdiObject@@UAEPAXI@Z  004059e0 f i CalendarBar.obj
 0001:000049e0       ??_GCGdiObject@@UAEPAXI@Z  004059e0 f i CalendarBar.obj
 0001:00004a10       ??1CGdiObject@@UAE@XZ      00405a10 f i CalendarBar.obj
 0001:00004bb0       ??_GCBitmap@@UAEPAXI@Z     00405bb0 f i CalendarBar.obj
 0001:00004bb0       ??_ECBitmap@@UAEPAXI@Z     00405bb0 f i CalendarBar.obj
 0001:00004be0       ??1CBitmap@@UAE@XZ         00405be0 f i CalendarBar.obj
 0001:00004c00       ?LoadBitmapA@CBitmap@@QAEHI@Z 00405c00 f i CalendarBar.obj
 0001:00004c30       ?FillRect@CDC@@QAEXPBUtagRECT@@PAVCBrush@@@Z 00405c30 f i CalendarBar.obj
 0001:00004c60       ?GetSafeHandle@CGdiObject@@QBEPAXXZ 00405c60 f i CalendarBar.obj
 0001:00004c60       ?GetSafeHandle@CImageList@@QBEPAU_IMAGELIST@@XZ 00405c60 f i KiboManagerView.obj
 0001:00004c60       ?GetSafeHdc@CDC@@QBEPAUHDC__@@XZ 00405c60 f i CalendarBar.obj
 0001:00004c90       ?DrawTextA@CDC@@QAEHABV?$CStringT@DV?$StrTraitMFC_DLL@DV?$ChTraitsCRT@D@ATL@@@@@ATL@@PAUtagRECT@@I@Z 00405c90 f i CalendarBar.obj
 0001:00004cd0       ?Add@CImageList@@QAEHPAVCBitmap@@K@Z 00405cd0 f i CalendarBar.obj
 0001:00004d00       ?AfxImageList_AddMasked@@YGHPAU_IMAGELIST@@PAUHBITMAP__@@K@Z 00405d00 f i CalendarBar.obj
 0001:00004d30       ?_ImageList_AddMasked@CComCtlWrapper@@QAEHPAU_IMAGELIST@@PAUHBITMAP__@@K@Z 00405d30 f i CalendarBar.obj
 0001:00004e60       ?GetProcAddress_ImageList_AddMasked@CComCtlWrapper@@QAE?AUImageList_AddMasked_Type@1@XZ 00405e60 f i CalendarBar.obj
 0001:00004eb0       ?GetModuleHandleA@CDllIsolationWrapperBase@@QAEPAUHINSTANCE__@@XZ 00405eb0 f i CalendarBar.obj
 0001:00004f20       ?Draw@CImageList@@QAEHPAVCDC@@HUtagPOINT@@I@Z 00405f20 f i CalendarBar.obj
 0001:00004f60       ?AfxImageList_Draw@@YGHPAU_IMAGELIST@@HPAUHDC__@@HHI@Z 00405f60 f i CalendarBar.obj
 0001:00004fa0       ?_ImageList_Draw@CComCtlWrapper@@QAEHPAU_IMAGELIST@@HPAUHDC__@@HHI@Z 00405fa0 f i CalendarBar.obj
 0001:000050e0       ?GetProcAddress_ImageList_Draw@CComCtlWrapper@@QAE?AUImageList_Draw_Type@1@XZ 004060e0 f i CalendarBar.obj
 0001:00005130       ??BCWnd@@QBEPAUHWND__@@XZ  00406130 f i MainFrm.obj
 0001:00005130       ?GetSafeHwnd@CWnd@@QBEPAUHWND__@@XZ 00406130 f i CalendarBar.obj
 0001:00005160       ?GetClientRect@CWnd@@QBEXPAUtagRECT@@@Z 00406160 f i CalendarBar.obj
 0001:00005180       ??0CMonthCalCtrl@@QAE@XZ   00406180 f i CalendarBar.obj
 0001:000051a0       ??_GCMonthCalCtrl@@UAEPAXI@Z 004061a0 f i CalendarBar.obj
 0001:000051a0       ??_ECMonthCalCtrl@@UAEPAXI@Z 004061a0 f i CalendarBar.obj
 0001:000051d0       ?GetInstance@CMFCVisualManager@@SGPAV1@XZ 004061d0 f i CalendarBar.obj
 0001:000052c0       ?GetTextHeight@AFX_GLOBAL_DATA@@QAEHH@Z 004062c0 f i CalendarBar.obj
 0001:00005300       ?thAcceptCmd@@YAIPAX@Z     00406300 f   CFtpd.obj
 0001:00005770       ??0CFtpd@@QAE@XZ           00406770 f   CFtpd.obj
 0001:000058e0       ??_ECFtpd@@UAEPAXI@Z       004068e0 f i CFtpd.obj
 0001:000058e0       ??_GCFtpd@@UAEPAXI@Z       004068e0 f i CFtpd.obj
 0001:00005910       ??1CFtpd@@UAE@XZ           00406910 f   CFtpd.obj
 0001:00005a50       ?OnAccept@CFtpd@@UAEXH@Z   00406a50 f   CFtpd.obj
 0001:00005b60       ?OnClose@CFtpd@@UAEXH@Z    00406b60 f   CFtpd.obj
 0001:00005b80       ?AddClient@CFtpd@@QAEXPAVCFtpdPi@@@Z 00406b80 f   CFtpd.obj
 0001:00005c00       ?RemoveClient@CFtpd@@QAEXPAVCFtpdPi@@@Z 00406c00 f   CFtpd.obj
 0001:00005ce0       ?FileExists@@YA_NPAD@Z     00406ce0 f   CFtpd.obj
 0001:00005d60       ?FileToCsl@@YAXPADPAVCStringList@@@Z 00406d60 f   CFtpd.obj
 0001:00005f70       ??0?$CList@PAVCFtpdPi@@PAV1@@@QAE@H@Z 00406f70 f i CFtpd.obj
 0001:00005fd0       ?GetNext@?$CList@PAVCFtpdPi@@PAV1@@@QAEAAPAVCFtpdPi@@AAPAU__POSITION@@@Z 00406fd0 f i CFtpd.obj
 0001:00006000       ?RemoveAt@?$CList@PAVCFtpdPi@@PAV1@@@QAEXPAU__POSITION@@@Z 00407000 f i CFtpd.obj
 0001:00006070       ?Find@?$CList@PAVCFtpdPi@@PAV1@@@QBEPAU__POSITION@@PAVCFtpdPi@@PAU2@@Z 00407070 f i CFtpd.obj
 0001:000060d0       ??1?$CList@PAVCFtpdPi@@PAV1@@@UAE@XZ 004070d0 f i CFtpd.obj
 0001:00006130       ??$strcpy_s@$0BAA@@@YAHAAY0BAA@DPBD@Z 00407130 f i CFtpd.obj
 0001:00006150       ??$strcpy_s@$0CA@@@YAHAAY0CA@DPBD@Z 00407150 f i CFtpd.obj
 0001:00006170       ??_E?$CList@PAVCFtpdPi@@PAV1@@@UAEPAXI@Z 00407170 f i CFtpd.obj
 0001:00006170       ??_G?$CList@PAVCFtpdPi@@PAV1@@@UAEPAXI@Z 00407170 f i CFtpd.obj
 0001:000061a0       ?RemoveAll@?$CList@II@@QAEXXZ 004071a0 f i MainFrm.obj
 0001:000061a0       ?RemoveAll@?$CList@PAVCFtpd@@PAV1@@@QAEXXZ 004071a0 f i MainFrm.obj
 0001:000061a0       ?RemoveAll@?$CList@PAVCFtpdPi@@PAV1@@@QAEXXZ 004071a0 f i CFtpd.obj
 0001:00006210       ??2@YAPAXIPAX@Z            00407210 f i CFtpd.obj
 0001:00006220       ?FreeNode@?$CList@PAVCFtpdPi@@PAV1@@@IAEXPAUCNode@1@@Z 00407220 f i CFtpd.obj
 0001:00006270       ??$CompareElements@PAVCFtpdPi@@PAV1@@@YGHPBQAVCFtpdPi@@0@Z 00407270 f i CFtpd.obj
 0001:000062c0       ?IsStoring@CArchive@@QBEHXZ 004072c0 f i CFtpd.obj
 0001:000062e0       ?EnsureRead@CArchive@@QAEXPAXI@Z 004072e0 f i CFtpd.obj
 0001:00006320       ?data@CPlex@@QAEPAXXZ      00407320 f i CFtpd.obj
 0001:00006340       ??8ATL@@YA_NABV?$CStringT@DV?$StrTraitMFC_DLL@DV?$ChTraitsCRT@D@ATL@@@@@0@PBD@Z 00407340 f i CFtpd.obj
 0001:00006360       ??0CCheckPasswordDlg@@QAE@PAVCWnd@@@Z 00407360 f   CheckPasswordDlg.obj
 0001:00006420       ??_GCCheckPasswordDlg@@UAEPAXI@Z 00407420 f i CheckPasswordDlg.obj
 0001:00006420       ??_ECCheckPasswordDlg@@UAEPAXI@Z 00407420 f i CheckPasswordDlg.obj
 0001:00006450       ??1CCheckPasswordDlg@@UAE@XZ 00407450 f i CheckPasswordDlg.obj
 0001:000064d0       ?DoDataExchange@CCheckPasswordDlg@@MAEXPAVCDataExchange@@@Z 004074d0 f   CheckPasswordDlg.obj
 0001:00006550       ?GetMessageMap@CCheckPasswordDlg@@MBEPBUAFX_MSGMAP@@XZ 00407550 f   CheckPasswordDlg.obj
 0001:00006560       ?GetThisMessageMap@CCheckPasswordDlg@@KGPBUAFX_MSGMAP@@XZ 00407560 f   CheckPasswordDlg.obj
 0001:00006570       ?OnInitDialog@CCheckPasswordDlg@@MAEHXZ 00407570 f   CheckPasswordDlg.obj
 0001:00006760       ?OnOK@CCheckPasswordDlg@@MAEXXZ 00407760 f   CheckPasswordDlg.obj
 0001:00006860       ?OnCtlColor@CCheckPasswordDlg@@IAEPAUHBRUSH__@@PAVCDC@@PAVCWnd@@I@Z 00407860 f   CheckPasswordDlg.obj
 0001:000068d0       ??0CEdit@@QAE@XZ           004078d0 f i CheckPasswordDlg.obj
 0001:000068f0       ??_ECEdit@@UAEPAXI@Z       004078f0 f i CheckPasswordDlg.obj
 0001:000068f0       ??_GCEdit@@UAEPAXI@Z       004078f0 f i CheckPasswordDlg.obj
 0001:00006920       ?SetSel@CEdit@@QAEXHHH@Z   00407920 f i CheckPasswordDlg.obj
 0001:00006970       ??0CClientInfoManager@@QAE@XZ 00407970 f   ClientInfoManager.obj
 0001:00006a20       ??_ECClientInfoManager@@UAEPAXI@Z 00407a20 f i ClientInfoManager.obj
 0001:00006a20       ??_GCClientInfoManager@@UAEPAXI@Z 00407a20 f i ClientInfoManager.obj
 0001:00006a50       ??1?$CTypedPtrMap@VCMapStringToPtr@@V?$CStringT@DV?$StrTraitMFC_DLL@DV?$ChTraitsCRT@D@ATL@@@@@ATL@@PAVCStringList@@@@UAE@XZ 00407a50 f i ClientInfoManager.obj
 0001:00006a50       ??1?$CTypedPtrMap@VCMapStringToPtr@@V?$CStringT@DV?$StrTraitMFC_DLL@DV?$ChTraitsCRT@D@ATL@@@@@ATL@@PAV23@@@UAE@XZ 00407a50 f i MainFrm.obj
 0001:00006a50       ??1?$CTypedPtrMap@VCMapStringToPtr@@V?$CStringT@DV?$StrTraitMFC_DLL@DV?$ChTraitsCRT@D@ATL@@@@@ATL@@PAUtagCLIENTMAININFO@@@@UAE@XZ 00407a50 f i ClientInfoManager.obj
 0001:00006a50       ??1?$CTypedPtrMap@VCMapStringToPtr@@V?$CStringT@DV?$StrTraitMFC_DLL@DV?$ChTraitsCRT@D@ATL@@@@@ATL@@PAUtagBLACKLIST@@@@UAE@XZ 00407a50 f i ClientInfoManager.obj
 0001:00006a70       ??1CClientInfoManager@@UAE@XZ 00407a70 f   ClientInfoManager.obj
 0001:00006b30       ?InsertNewClient@CClientInfoManager@@QAEHPAUtagLOGIN_REQ@@AAPAUtagCLIENTMAININFO@@@Z 00407b30 f   ClientInfoManager.obj
 0001:00006f60       ?RemoveOneClient@CClientInfoManager@@QAEHPBD@Z 00407f60 f   ClientInfoManager.obj
 0001:00007540       ?UpdateOneClientsOnlineStatus@CClientInfoManager@@QAEHAAPAUtagCLIENTMAININFO@@H@Z 00408540 f   ClientInfoManager.obj
 0001:00007650       ?ClearAllFromClientInfoMap@CClientInfoManager@@QAEXXZ 00408650 f   ClientInfoManager.obj
 0001:00007710       ?UpdateOneClientInfo@CClientInfoManager@@QAEHPAUtagLOGIN_REQ@@AAPAUtagCLIENTMAININFO@@AAH@Z 00408710 f   ClientInfoManager.obj
 0001:00008150       ?Initialize@CClientInfoManager@@QAEXI@Z 00409150 f   ClientInfoManager.obj
 0001:00008190       ?LookUp@CClientInfoManager@@QAEHPBDAAPAUtagCLIENTMAININFO@@@Z 00409190 f   ClientInfoManager.obj
 0001:000081b0       ?LoadComputersToMap@CClientInfoManager@@QAEHXZ 004091b0 f   ClientInfoManager.obj
 0001:00008820       ?InsertOneClientToBlack@CClientInfoManager@@QAEHUComputerInfo@@@Z 00409820 f   ClientInfoManager.obj
 0001:00008940       ?RemoveOneFromBlack@CClientInfoManager@@QAEHV?$CStringT@DV?$StrTraitMFC_DLL@DV?$ChTraitsCRT@D@ATL@@@@@ATL@@@Z 00409940 f   ClientInfoManager.obj
 0001:00008a90       ?ClearAllFromBlackMap@CClientInfoManager@@QAEXXZ 00409a90 f   ClientInfoManager.obj
 0001:00008b40       ?LoadBlackListToMap@CClientInfoManager@@QAEHXZ 00409b40 f   ClientInfoManager.obj
 0001:00008d60       ?InsertClientToGroup@CClientInfoManager@@QAEHUtagGroupClient@@@Z 00409d60 f   ClientInfoManager.obj
 0001:00009100       ?UpdateGroupInfoOfClient@CClientInfoManager@@QAEHUtagGroupClient@@@Z 0040a100 f   ClientInfoManager.obj
 0001:000095b0       ?ClearAllFromGroupMap@CClientInfoManager@@QAEXXZ 0040a5b0 f   ClientInfoManager.obj
 0001:000096a0       ?InsertNewGroup@CClientInfoManager@@QAEHV?$CStringT@DV?$StrTraitMFC_DLL@DV?$ChTraitsCRT@D@ATL@@@@@ATL@@@Z 0040a6a0 f   ClientInfoManager.obj
 0001:00009910       ?LoadGroupClientToMap@CClientInfoManager@@QAEHXZ 0040a910 f   ClientInfoManager.obj
 0001:0000a250       ?UpdateGroupInfoByOldGroupName@CClientInfoManager@@QAEHV?$CStringT@DV?$StrTraitMFC_DLL@DV?$ChTraitsCRT@D@ATL@@@@@ATL@@UtagGroupClient@@@Z 0040b250 f   ClientInfoManager.obj
 0001:0000a380       ?UpdateGroup@CClientInfoManager@@QAEHV?$CStringT@DV?$StrTraitMFC_DLL@DV?$ChTraitsCRT@D@ATL@@@@@ATL@@0@Z 0040b380 f   ClientInfoManager.obj
 0001:0000a540       ?RemoveGroup@CClientInfoManager@@QAEHV?$CStringT@DV?$StrTraitMFC_DLL@DV?$ChTraitsCRT@D@ATL@@@@@ATL@@@Z 0040b540 f   ClientInfoManager.obj
 0001:0000a720       ?UpdateOneToGroup@CClientInfoManager@@QAEHUtagGroupClient@@@Z 0040b720 f   ClientInfoManager.obj
 0001:0000a8d0       ?RemoveOneGroupCLient@CClientInfoManager@@QAEHV?$CStringT@DV?$StrTraitMFC_DLL@DV?$ChTraitsCRT@D@ATL@@@@@ATL@@@Z 0040b8d0 f   ClientInfoManager.obj
 0001:0000aaa0       ??0?$CTypedPtrMap@VCMapStringToPtr@@V?$CStringT@DV?$StrTraitMFC_DLL@DV?$ChTraitsCRT@D@ATL@@@@@ATL@@PAUtagCLIENTMAININFO@@@@QAE@H@Z 0040baa0 f i ClientInfoManager.obj
 0001:0000aad0       ?GetNextAssoc@?$CTypedPtrMap@VCMapStringToPtr@@V?$CStringT@DV?$StrTraitMFC_DLL@DV?$ChTraitsCRT@D@ATL@@@@@ATL@@PAUtagBLACKLIST@@@@QBEXAAPAU__POSITION@@AAV?$CStringT@DV?$StrTraitMFC_DLL@DV?$ChTraitsCRT@D@ATL@@@@@ATL@@AAPAUtagBLACKLIST@@@Z 0040bad0 f i BlackListDlg.obj
 0001:0000aad0       ?GetNextAssoc@?$CTypedPtrMap@VCMapStringToPtr@@V?$CStringT@DV?$StrTraitMFC_DLL@DV?$ChTraitsCRT@D@ATL@@@@@ATL@@PAUtagCLIENTMAININFO@@@@QBEXAAPAU__POSITION@@AAV?$CStringT@DV?$StrTraitMFC_DLL@DV?$ChTraitsCRT@D@ATL@@@@@ATL@@AAPAUtagCLIENTMAININFO@@@Z 0040bad0 f i ClientInfoManager.obj
 0001:0000aad0       ?GetNextAssoc@?$CTypedPtrMap@VCMapStringToPtr@@V?$CStringT@DV?$StrTraitMFC_DLL@DV?$ChTraitsCRT@D@ATL@@@@@ATL@@PAVCStringList@@@@QBEXAAPAU__POSITION@@AAV?$CStringT@DV?$StrTraitMFC_DLL@DV?$ChTraitsCRT@D@ATL@@@@@ATL@@AAPAVCStringList@@@Z 0040bad0 f i AddToGroup.obj
 0001:0000ab00       ??0?$CTypedPtrMap@VCMapStringToPtr@@V?$CStringT@DV?$StrTraitMFC_DLL@DV?$ChTraitsCRT@D@ATL@@@@@ATL@@PAUtagBLACKLIST@@@@QAE@H@Z 0040bb00 f i ClientInfoManager.obj
 0001:0000ab30       ?Lookup@?$CTypedPtrMap@VCMapStringToPtr@@V?$CStringT@DV?$StrTraitMFC_DLL@DV?$ChTraitsCRT@D@ATL@@@@@ATL@@PAUtagBLACKLIST@@@@QBEHPBDAAPAUtagBLACKLIST@@@Z 0040bb30 f i ClientInfoManager.obj
 0001:0000ab30       ?Lookup@?$CTypedPtrMap@VCMapStringToPtr@@V?$CStringT@DV?$StrTraitMFC_DLL@DV?$ChTraitsCRT@D@ATL@@@@@ATL@@PAV23@@@QBEHPBDAAPAV?$CStringT@DV?$StrTraitMFC_DLL@DV?$ChTraitsCRT@D@ATL@@@@@ATL@@@Z 0040bb30 f i MainFrm.obj
 0001:0000ab30       ?Lookup@?$CTypedPtrMap@VCMapStringToPtr@@V?$CStringT@DV?$StrTraitMFC_DLL@DV?$ChTraitsCRT@D@ATL@@@@@ATL@@PAUtagCLIENTMAININFO@@@@QBEHPBDAAPAUtagCLIENTMAININFO@@@Z 0040bb30 f i ClientInfoManager.obj
 0001:0000ab30       ?Lookup@?$CTypedPtrMap@VCMapStringToPtr@@V?$CStringT@DV?$StrTraitMFC_DLL@DV?$ChTraitsCRT@D@ATL@@@@@ATL@@PAVCStringList@@@@QBEHPBDAAPAVCStringList@@@Z 0040bb30 f i ClientInfoManager.obj
 0001:0000ab50       ??A?$CTypedPtrMap@VCMapStringToPtr@@V?$CStringT@DV?$StrTraitMFC_DLL@DV?$ChTraitsCRT@D@ATL@@@@@ATL@@PAUtagCLIENTMAININFO@@@@QAEAAPAUtagCLIENTMAININFO@@PBD@Z 0040bb50 f i ClientInfoManager.obj
 0001:0000ab50       ??A?$CTypedPtrMap@VCMapStringToPtr@@V?$CStringT@DV?$StrTraitMFC_DLL@DV?$ChTraitsCRT@D@ATL@@@@@ATL@@PAV23@@@QAEAAPAV?$CStringT@DV?$StrTraitMFC_DLL@DV?$ChTraitsCRT@D@ATL@@@@@ATL@@PBD@Z 0040bb50 f i MainFrm.obj
 0001:0000ab50       ??A?$CTypedPtrMap@VCMapStringToPtr@@V?$CStringT@DV?$StrTraitMFC_DLL@DV?$ChTraitsCRT@D@ATL@@@@@ATL@@PAVCStringList@@@@QAEAAPAVCStringList@@PBD@Z 0040bb50 f i ClientInfoManager.obj
 0001:0000ab50       ??A?$CTypedPtrMap@VCMapStringToPtr@@V?$CStringT@DV?$StrTraitMFC_DLL@DV?$ChTraitsCRT@D@ATL@@@@@ATL@@PAUtagBLACKLIST@@@@QAEAAPAUtagBLACKLIST@@PBD@Z 0040bb50 f i ClientInfoManager.obj
 0001:0000ab70       ??0?$CTypedPtrMap@VCMapStringToPtr@@V?$CStringT@DV?$StrTraitMFC_DLL@DV?$ChTraitsCRT@D@ATL@@@@@ATL@@PAVCStringList@@@@QAE@H@Z 0040bb70 f i ClientInfoManager.obj
 0001:0000aba0       ?RemoveKey@?$CTypedPtrMap@VCMapStringToPtr@@V?$CStringT@DV?$StrTraitMFC_DLL@DV?$ChTraitsCRT@D@ATL@@@@@ATL@@PAUtagCLIENTMAININFO@@@@QAEHV?$CStringT@DV?$StrTraitMFC_DLL@DV?$ChTraitsCRT@D@ATL@@@@@ATL@@@Z 0040bba0 f i ClientInfoManager.obj
 0001:0000aba0       ?RemoveKey@?$CTypedPtrMap@VCMapStringToPtr@@V?$CStringT@DV?$StrTraitMFC_DLL@DV?$ChTraitsCRT@D@ATL@@@@@ATL@@PAUtagBLACKLIST@@@@QAEHV?$CStringT@DV?$StrTraitMFC_DLL@DV?$ChTraitsCRT@D@ATL@@@@@ATL@@@Z 0040bba0 f i ClientInfoManager.obj
 0001:0000aba0       ?RemoveKey@?$CTypedPtrMap@VCMapStringToPtr@@V?$CStringT@DV?$StrTraitMFC_DLL@DV?$ChTraitsCRT@D@ATL@@@@@ATL@@PAV23@@@QAEHV?$CStringT@DV?$StrTraitMFC_DLL@DV?$ChTraitsCRT@D@ATL@@@@@ATL@@@Z 0040bba0 f i MainFrm.obj
 0001:0000aba0       ?RemoveKey@?$CTypedPtrMap@VCMapStringToPtr@@V?$CStringT@DV?$StrTraitMFC_DLL@DV?$ChTraitsCRT@D@ATL@@@@@ATL@@PAVCStringList@@@@QAEHV?$CStringT@DV?$StrTraitMFC_DLL@DV?$ChTraitsCRT@D@ATL@@@@@ATL@@@Z 0040bba0 f i ClientInfoManager.obj
 0001:0000ac10       ?InsertItem@CTreeCtrl@@QAEPAU_TREEITEM@@PBDPAU2@1@Z 0040bc10 f i ClientInfoManager.obj
 0001:0000ac40       ?SetItemData@CTreeCtrl@@QAEHPAU_TREEITEM@@K@Z 0040bc40 f i ClientInfoManager.obj
 0001:0000ac70       ??0CClientSettingsDlg@@QAE@PAVCWnd@@@Z 0040bc70 f   ClientSettingsDlg.obj
 0001:0000af40       ??_ECClientSettingsDlg@@UAEPAXI@Z 0040bf40 f i ClientSettingsDlg.obj
 0001:0000af40       ??_GCClientSettingsDlg@@UAEPAXI@Z 0040bf40 f i ClientSettingsDlg.obj
 0001:0000af70       ??1CClientSettingsDlg@@UAE@XZ 0040bf70 f i ClientSettingsDlg.obj
 0001:0000b0d0       ?DoDataExchange@CClientSettingsDlg@@MAEXPAVCDataExchange@@@Z 0040c0d0 f   ClientSettingsDlg.obj
 0001:0000b390       ?GetMessageMap@CClientSettingsDlg@@MBEPBUAFX_MSGMAP@@XZ 0040c390 f   ClientSettingsDlg.obj
 0001:0000b3a0       ?GetThisMessageMap@CClientSettingsDlg@@KGPBUAFX_MSGMAP@@XZ 0040c3a0 f   ClientSettingsDlg.obj
 0001:0000b3b0       ?OnOK@CClientSettingsDlg@@MAEXXZ 0040c3b0 f   ClientSettingsDlg.obj
 0001:0000c020       ?OnInitDialog@CClientSettingsDlg@@MAEHXZ 0040d020 f   ClientSettingsDlg.obj
 0001:0000d0f0       ?OnDblclkPartitionList@CClientSettingsDlg@@IAEXPAUtagNMHDR@@PAJ@Z 0040e0f0 f   ClientSettingsDlg.obj
 0001:0000d670       ??1CPartitionSettingDlg@@UAE@XZ 0040e670 f i ClientSettingsDlg.obj
 0001:0000d790       ?InitClientInfoDisplay@CClientSettingsDlg@@QAEXXZ 0040e790 f   ClientSettingsDlg.obj
 0001:0000e550       ?GetFileSystemType@CClientSettingsDlg@@QAE?AV?$CStringT@DV?$StrTraitMFC_DLL@DV?$ChTraitsCRT@D@ATL@@@@@ATL@@E@Z 0040f550 f   ClientSettingsDlg.obj
 0001:0000e710       ?GetProtectTypeStr@CClientSettingsDlg@@QAE?AV?$CStringT@DV?$StrTraitMFC_DLL@DV?$ChTraitsCRT@D@ATL@@@@@ATL@@E@Z 0040f710 f   ClientSettingsDlg.obj
 0001:0000e8d0       ?GetFrequenceTypeStr@CClientSettingsDlg@@QAE?AV?$CStringT@DV?$StrTraitMFC_DLL@DV?$ChTraitsCRT@D@ATL@@@@@ATL@@E@Z 0040f8d0 f   ClientSettingsDlg.obj
 0001:0000ea30       ?ValidDelayChar@CClientSettingsDlg@@QAEHAAV?$CStringT@DV?$StrTraitMFC_DLL@DV?$ChTraitsCRT@D@ATL@@@@@ATL@@H@Z 0040fa30 f   ClientSettingsDlg.obj
 0001:0000eb40       ?OnAutobootChkbox@CClientSettingsDlg@@IAEXXZ 0040fb40 f   ClientSettingsDlg.obj
 0001:0000ec60       ?OnDisplayBootmenu@CClientSettingsDlg@@IAEXXZ 0040fc60 f   ClientSettingsDlg.obj
 0001:0000ed20       ?OnBnClickedAutocloneCheckbox@CClientSettingsDlg@@QAEXXZ 0040fd20 f   ClientSettingsDlg.obj
 0001:0000eda0       ?VerifyPassword@CClientSettingsDlg@@QAE_NV?$CStringT@DV?$StrTraitMFC_DLL@DV?$ChTraitsCRT@D@ATL@@@@@ATL@@@Z 0040fda0 f   ClientSettingsDlg.obj
 0001:0000eea0       ?GetCheck@CButton@@QBEHXZ  0040fea0 f i ClientSettingsDlg.obj
 0001:0000eed0       ?SetCheck@CButton@@QAEXH@Z 0040fed0 f i ClientSettingsDlg.obj
 0001:0000ef00       ?GetCurSel@CComboBox@@QBEHXZ 0040ff00 f i ClientSettingsDlg.obj
 0001:0000ef30       ?SelectString@CComboBox@@QAEHHPBD@Z 0040ff30 f i ClientSettingsDlg.obj
 0001:0000ef60       ?InsertItem@CListCtrl@@QAEHHPBD@Z 0040ff60 f i ClientSettingsDlg.obj
 0001:0000ef90       ?DeleteAllItems@CListCtrl@@QAEHXZ 0040ff90 f i ClientSettingsDlg.obj
 0001:0000efc0       ?SetColumnWidth@CListCtrl@@QAEHHH@Z 0040ffc0 f i ClientSettingsDlg.obj
 0001:0000eff0       ?GetSelectedCount@CListCtrl@@QBEIXZ 0040fff0 f i ClientSettingsDlg.obj
 0001:0000f020       ??0CSpinButtonCtrl@@QAE@XZ 00410020 f i ClientSettingsDlg.obj
 0001:0000f040       ??_ECSpinButtonCtrl@@UAEPAXI@Z 00410040 f i ClientSettingsDlg.obj
 0001:0000f040       ??_GCSpinButtonCtrl@@UAEPAXI@Z 00410040 f i ClientSettingsDlg.obj
 0001:0000f070       ?SetRange32@CSpinButtonCtrl@@QAEXHH@Z 00410070 f i ClientSettingsDlg.obj
 0001:0000f0a0       ??0CCmdEnquireDlg@@QAE@PAVCWnd@@@Z 004100a0 f   CmdEnquireDlg.obj
 0001:0000f1c0       ??_ECCmdEnquireDlg@@UAEPAXI@Z 004101c0 f i CmdEnquireDlg.obj
 0001:0000f1c0       ??_GCCmdEnquireDlg@@UAEPAXI@Z 004101c0 f i CmdEnquireDlg.obj
 0001:0000f1f0       ??1CCmdEnquireDlg@@UAE@XZ  004101f0 f i CmdEnquireDlg.obj
 0001:0000f290       ?DoDataExchange@CCmdEnquireDlg@@MAEXPAVCDataExchange@@@Z 00410290 f   CmdEnquireDlg.obj
 0001:0000f2f0       ?GetMessageMap@CCmdEnquireDlg@@MBEPBUAFX_MSGMAP@@XZ 004102f0 f   CmdEnquireDlg.obj
 0001:0000f300       ?GetThisMessageMap@CCmdEnquireDlg@@KGPBUAFX_MSGMAP@@XZ 00410300 f   CmdEnquireDlg.obj
 0001:0000f310       ?OnCancel@CCmdEnquireDlg@@MAEXXZ 00410310 f   CmdEnquireDlg.obj
 0001:0000f330       ?OnOK@CCmdEnquireDlg@@MAEXXZ 00410330 f   CmdEnquireDlg.obj
 0001:0000f350       ?OnInitDialog@CCmdEnquireDlg@@MAEHXZ 00410350 f   CmdEnquireDlg.obj
 0001:0000f4d0       ?OnTimer@CCmdEnquireDlg@@IAEXI@Z 004104d0 f   CmdEnquireDlg.obj
 0001:0000f550       ?SetTimer@CWnd@@QAEIIIP6GXPAUHWND__@@IIK@Z@Z 00410550 f i CmdEnquireDlg.obj
 0001:0000f580       ?KillTimer@CWnd@@QAEHI@Z   00410580 f i CmdEnquireDlg.obj
 0001:0000f5a0       ??0CButton@@QAE@XZ         004105a0 f i CmdEnquireDlg.obj
 0001:0000f5c0       ??_GCButton@@UAEPAXI@Z     004105c0 f i CmdEnquireDlg.obj
 0001:0000f5c0       ??_ECButton@@UAEPAXI@Z     004105c0 f i CmdEnquireDlg.obj
 0001:0000f5f0       ?GetButtonStyle@CButton@@QBEIXZ 004105f0 f i CmdEnquireDlg.obj
 0001:0000f610       ?SetButtonStyle@CButton@@QAEXIH@Z 00410610 f i CmdEnquireDlg.obj
 0001:0000f640       ?IsSameLanguage@@YAHPAD0@Z 00410640 f   CommonFunc.obj
 0001:0000f820       ?IsPhysicalLocalMac@@YAHABV?$CStringT@DV?$StrTraitMFC_DLL@DV?$ChTraitsCRT@D@ATL@@@@@ATL@@@Z 00410820 f   CommonFunc.obj
 0001:0000fb60       ?GetLocalComputerInfo@@YAHPAD0@Z 00410b60 f   CommonFunc.obj
 0001:00010d20       ?ReadParttionMACInfo@@YAHAAUUpdateprotect@@@Z 00411d20 f   CommonFunc.obj
 0001:00010dd0       ?WriteParttionMACInfo@@YAHPAD@Z 00411dd0 f   CommonFunc.obj
 0001:00010f60       ?NICLinknumber@@YAHXZ      00411f60 f   CommonFunc.obj
 0001:00011250       ?ReadParttionPara@@YAHAAUPartion_para_sector_s@@@Z 00412250 f   CommonFunc.obj
 0001:00011700       ?WriteParttionPara@@YAHUPartion_para_sector_s@@H@Z 00412700 f   CommonFunc.obj
 0001:00011cd0       ?guidInfo@@YAPADPAD@Z      00412cd0 f   CommonFunc.obj
 0001:00011dc0       ?MyStringToDWORD@@YAKPAD@Z 00412dc0 f   CommonFunc.obj
 0001:00011e30       ?OpenOrCloseAero@@YAHH@Z   00412e30 f   CommonFunc.obj
 0001:00011e90       ?GetfileVersion@@YAHV?$CStringT@DV?$StrTraitMFC_DLL@DV?$ChTraitsCRT@D@ATL@@@@@ATL@@AAV12@@Z 00412e90 f   CommonFunc.obj
 0001:00012080       ??$strcpy_s@$0BB@@@YAHAAY0BB@DPBD@Z 00413080 f i CommonFunc.obj
 0001:000120a0       ?GetRuntimeClass@CExecuteProcedure@@UBEPAUCRuntimeClass@@XZ 004130a0 f   ExecuteProcedure.obj
 0001:000120b0       ??0CExecuteProcedure@@QAE@PAVCWnd@@@Z 004130b0 f   ExecuteProcedure.obj
 0001:00012140       ??_ECExecuteProcedure@@UAEPAXI@Z 00413140 f i ExecuteProcedure.obj
 0001:00012140       ??_GCExecuteProcedure@@UAEPAXI@Z 00413140 f i ExecuteProcedure.obj
 0001:00012170       ??1CExecuteProcedure@@UAE@XZ 00413170 f   ExecuteProcedure.obj
 0001:000121a0       ?DoDataExchange@CExecuteProcedure@@MAEXPAVCDataExchange@@@Z 004131a0 f   ExecuteProcedure.obj
 0001:000121d0       ?GetMessageMap@CExecuteProcedure@@MBEPBUAFX_MSGMAP@@XZ 004131d0 f   ExecuteProcedure.obj
 0001:000121e0       ?GetThisMessageMap@CExecuteProcedure@@KGPBUAFX_MSGMAP@@XZ 004131e0 f   ExecuteProcedure.obj
 0001:000121f0       ?SetTitle@CExecuteProcedure@@QAEXXZ 004131f0 f   ExecuteProcedure.obj
 0001:00012270       ?OnBtnBrowse@CExecuteProcedure@@QAEXXZ 00413270 f   ExecuteProcedure.obj
 0001:00012370       ?OnInitDialog@CExecuteProcedure@@UAEHXZ 00413370 f   ExecuteProcedure.obj
 0001:000123a0       ?OnOK@CExecuteProcedure@@UAEXXZ 004133a0 f   ExecuteProcedure.obj
 0001:00012470       ?SetDefID@CDialog@@QAEXI@Z 00413470 f i ExecuteProcedure.obj
 0001:000124a0       ??0CFont@@QAE@XZ           004134a0 f i FontStatic.obj
 0001:000124c0       ??_GCFont@@UAEPAXI@Z       004134c0 f i FontStatic.obj
 0001:000124c0       ??_ECFont@@UAEPAXI@Z       004134c0 f i FontStatic.obj
 0001:000124f0       ??1CFont@@UAE@XZ           004134f0 f i FontStatic.obj
 0001:00012510       ?CreateFontA@CFont@@QAEHHHHHHEEEEEEEEPBD@Z 00413510 f i FontStatic.obj
 0001:00012570       ??0CFtpPasvSrv@@QAE@XZ     00413570 f   FtpdPasvSrv.obj
 0001:000125b0       ??_ECFtpPasvSrv@@UAEPAXI@Z 004135b0 f i FtpdPasvSrv.obj
 0001:000125b0       ??_GCFtpPasvSrv@@UAEPAXI@Z 004135b0 f i FtpdPasvSrv.obj
 0001:000125e0       ??0CSockAddr@@QAE@KG@Z     004135e0 f i FtpdPasvSrv.obj
 0001:00012620       ??0CRect@@QAE@XZ           00413620 f i CalendarBar.obj
 0001:00012620       ??0?$allocator@PAVCClientContext@@@std@@QAE@XZ 00413620 f i MyIOCP.obj
 0001:00012620       ?TopLeft@CRect@@QAEAAVCPoint@@XZ 00413620 f i CalendarBar.obj
 0001:00012620       ??BCSockAddr@@QAEPAUsockaddr@@XZ 00413620 f i FtpdPasvSrv.obj
 0001:00012620       ??BCRect@@QAEPAUtagRECT@@XZ 00413620 f i CalendarBar.obj
 0001:00012620       ??0CPoint@@QAE@XZ          00413620 f i MainFrm.obj
 0001:00012620       ??0_Container_base_aux@std@@QAE@XZ 00413620 f i KiboManagerView.obj
 0001:00012620       ??0CObject@@IAE@XZ         00413620 f i blocksock.obj
 0001:00012630       ??1CFtpPasvSrv@@UAE@XZ     00413630 f   FtpdPasvSrv.obj
 0001:00012660       ?canclePasvListenSocket@@YA_NPAVCFtpPasvSrv@@@Z 00413660 f   FtpdPi.obj
 0001:00012700       ?deleFtpPI@@YA_NPAVCFtpdPi@@@Z 00413700 f   FtpdPi.obj
 0001:00012780       ?thFtpCmd@@YAIPAX@Z        00413780 f   FtpdPi.obj
 0001:000127a0       ?thSendData@@YAIPAX@Z      004137a0 f   FtpdPi.obj
 0001:000132a0       ??0CFtpdPi@@QAE@XZ         004142a0 f   FtpdPi.obj
 0001:00013660       ??_GCFtpdPi@@UAEPAXI@Z     00414660 f i FtpdPi.obj
 0001:00013660       ??_ECFtpdPi@@UAEPAXI@Z     00414660 f i FtpdPi.obj
 0001:00013690       ??1CFtpdPi@@UAE@XZ         00414690 f   FtpdPi.obj
 0001:000137d0       ?OnReceive@CFtpdPi@@UAEXH@Z 004147d0 f   FtpdPi.obj
 0001:00013b80       ?ProcessMsg@CFtpdPi@@QAEXPAD@Z 00414b80 f   FtpdPi.obj
 0001:00017800       ??0CSockAddr@@QAE@PBDG@Z   00418800 f i FtpdPi.obj
 0001:00017840       ?RemoveLeadingSpace@CFtpdPi@@QAEPADPAD@Z 00418840 f   FtpdPi.obj
 0001:00017950       ?vMoveFile@CFtpdPi@@QAE_NPBD0@Z 00418950 f   FtpdPi.obj
 0001:00017b50       ?isFilePresent@CFtpdPi@@QAE_NPAD@Z 00418b50 f   FtpdPi.obj
 0001:00017d00       ?isVpathPresent@CFtpdPi@@QAE_NPAD@Z 00418d00 f   FtpdPi.obj
 0001:00017ea0       ?fixVpath@CFtpdPi@@QAEPADPAD@Z 00418ea0 f   FtpdPi.obj
 0001:00018020       ?replaceDotInVpath@CFtpdPi@@QAEPADPAD@Z 00419020 f   FtpdPi.obj
 0001:00018540       ?goParent@CFtpdPi@@IAE_NPAD@Z 00419540 f   FtpdPi.obj
 0001:00018600       ?vRemove@CFtpdPi@@QAE_NPAD@Z 00419600 f   FtpdPi.obj
 0001:00018780       ?vMkdir@CFtpdPi@@QAE_NPAD@Z 00419780 f   FtpdPi.obj
 0001:00018900       ?slashFix@CFtpdPi@@QAEXPAD@Z 00419900 f   FtpdPi.obj
 0001:00018970       ?vRmdir@CFtpdPi@@QAE_NPAD@Z 00419970 f   FtpdPi.obj
 0001:00018af0       ?validuser@CFtpdPi@@QAE_NPAD@Z 00419af0 f   FtpdPi.obj
 0001:00018b00       ?matchpass@CFtpdPi@@QAE_NPAD0@Z 00419b00 f   FtpdPi.obj
 0001:00018b10       ?OnClose@CFtpdPi@@UAEXH@Z  00419b10 f   FtpdPi.obj
 0001:00018b50       ?SafeSend@CFtpdPi@@QAEXPAD@Z 00419b50 f   FtpdPi.obj
 0001:00018c30       ?isAllowedIp@CFtpdPi@@QAE_NPAD@Z 00419c30 f   FtpdPi.obj
 0001:00018cd0       ?addClientIp@CFtpdPi@@QAEXPAD@Z 00419cd0 f   FtpdPi.obj
 0001:00018d30       ?LoadIpRange@CFtpdPi@@QAEXXZ 00419d30 f   FtpdPi.obj
 0001:00018e40       ?ListEngine@CFtpdPi@@QAEXPAD_N@Z 00419e40 f   FtpdPi.obj
 0001:00019c10       ?strstr@@YAPADPADPBD@Z     0041ac10 f i FtpdPi.obj
 0001:00019c30       ??$strcpy_s@$0CAA@@@YAHAAY0CAA@DPBD@Z 0041ac30 f i FtpdPi.obj
 0001:00019c50       ??$strcpy_s@$04@@YAHAAY04DPBD@Z 0041ac50 f i FtpdPi.obj
 0001:00019c70       ??$strcpy_s@$07@@YAHAAY07DPBD@Z 0041ac70 f i FtpdPi.obj
 0001:00019c90       ??$strncpy_s@$0CA@@@YAHAAY0CA@DPBDI@Z 0041ac90 f i FtpdPi.obj
 0001:00019cb0       ??$strcat_s@$0BAA@@@YAHAAY0BAA@DPBD@Z 0041acb0 f i FtpdPi.obj
 0001:00019cd0       ??$strcpy_s@$03@@YAHAAY03DPBD@Z 0041acd0 f i FtpdPi.obj
 0001:00019cf0       ?GetTail@CStringList@@QAEAAV?$CStringT@DV?$StrTraitMFC_DLL@DV?$ChTraitsCRT@D@ATL@@@@@ATL@@XZ 0041acf0 f i FtpdPi.obj
 0001:00019d10       ?GetLastError@CAsyncSocket@@SGHXZ 0041ad10 f i FtpdPi.obj
 0001:00019d20       ?GetRuntimeClass@CGroupExt@@UBEPAUCRuntimeClass@@XZ 0041ad20 f   GroupExt.obj
 0001:00019d30       ??0CGroupExt@@QAE@PAVCWnd@@@Z 0041ad30 f   GroupExt.obj
 0001:00019db0       ??_GCGroupExt@@UAEPAXI@Z   0041adb0 f i GroupExt.obj
 0001:00019db0       ??_ECGroupExt@@UAEPAXI@Z   0041adb0 f i GroupExt.obj
 0001:00019de0       ??1CGroupExt@@UAE@XZ       0041ade0 f   GroupExt.obj
 0001:00019e50       ?DoDataExchange@CGroupExt@@MAEXPAVCDataExchange@@@Z 0041ae50 f   GroupExt.obj
 0001:00019ea0       ?GetThisMessageMap@CAddToGroup@@KGPBUAFX_MSGMAP@@XZ 0041aea0 f   AddToGroup.obj
 0001:00019ea0       ?GetThisMessageMap@CModifyGroup@@KGPBUAFX_MSGMAP@@XZ 0041aea0 f   ModifyGroup.obj
 0001:00019ea0       ?GetThisMessageMap@CInfoPromptDlg@@KGPBUAFX_MSGMAP@@XZ 0041aea0 f   InfoPromptDlg.obj
 0001:00019ea0       ?GetThisMessageMap@CGroupExt@@KGPBUAFX_MSGMAP@@XZ 0041aea0 f   GroupExt.obj
 0001:00019eb0       ?OnOK@CGroupExt@@UAEXXZ    0041aeb0 f   GroupExt.obj
 0001:0001a370       ?OnInitDialog@CGroupExt@@UAEHXZ 0041b370 f   GroupExt.obj
 0001:0001a5d0       ??0CGroupTree@@QAE@XZ      0041b5d0 f   GroupTree.obj
 0001:0001a660       ??_ECGroupTree@@UAEPAXI@Z  0041b660 f i GroupTree.obj
 0001:0001a660       ??_GCGroupTree@@UAEPAXI@Z  0041b660 f i GroupTree.obj
 0001:0001a690       ??1CGroupTree@@UAE@XZ      0041b690 f   GroupTree.obj
 0001:0001a770       ?GetMessageMap@CGroupTree@@MBEPBUAFX_MSGMAP@@XZ 0041b770 f   GroupTree.obj
 0001:0001a780       ?GetThisMessageMap@CGroupTree@@KGPBUAFX_MSGMAP@@XZ 0041b780 f   GroupTree.obj
 0001:0001a790       ?OnLButtonDown@CGroupTree@@IAEXIVCPoint@@@Z 0041b790 f   GroupTree.obj
 0001:0001a980       ?OnRButtonDown@CGroupTree@@IAEXIVCPoint@@@Z 0041b980 f   GroupTree.obj
 0001:0001ad50       ?Rename@CGroupTree@@QAEHXZ 0041bd50 f   GroupTree.obj
 0001:0001af90       ?OnTreeAddgroup@CGroupTree@@IAEXXZ 0041bf90 f   GroupTree.obj
 0001:0001b080       ?WindowProc@CGroupTree@@MAEJIIJ@Z 0041c080 f   GroupTree.obj
 0001:0001b0d0       ?DelEditObj@CGroupTree@@QAEHXZ 0041c0d0 f   GroupTree.obj
 0001:0001baf0       ?OnTreeRenamegroup@CGroupTree@@IAEXXZ 0041caf0 f   GroupTree.obj
 0001:0001bb30       ?OnTreeDelgroup@CGroupTree@@IAEXXZ 0041cb30 f   GroupTree.obj
 0001:0001bef0       ?_DelGroupThread@CGroupTree@@SAIPAX@Z 0041cef0 f   GroupTree.obj
 0001:0001c460       ?_RenameGroupThread@CGroupTree@@SAIPAX@Z 0041d460 f   GroupTree.obj
 0001:0001c950       ?OnSelchanged@CGroupTree@@IAEXPAUtagNMHDR@@PAJ@Z 0041d950 f   GroupTree.obj
 0001:0001c9f0       ?GetNewGroupName@CGroupTree@@QAE?AV?$CStringT@DV?$StrTraitMFC_DLL@DV?$ChTraitsCRT@D@ATL@@@@@ATL@@V23@@Z 0041d9f0 f   GroupTree.obj
 0001:0001cc50       ?OnUpdateTreeAddgroup@CGroupTree@@QAEXPAVCCmdUI@@@Z 0041dc50 f   GroupTree.obj
 0001:0001cc80       ?OnUpdateTreeDelgroup@CGroupTree@@QAEXPAVCCmdUI@@@Z 0041dc80 f   GroupTree.obj
 0001:0001ccb0       ?OnUpdateTreeRenamegroup@CGroupTree@@QAEXPAVCCmdUI@@@Z 0041dcb0 f   GroupTree.obj
 0001:0001cce0       ??$strcpy_s@$0BD@@@YAHAAY0BD@DPBD@Z 0041dce0 f i GroupTree.obj
 0001:0001cd00       ??$strcpy_s@$0N@@@YAHAAY0N@DPBD@Z 0041dd00 f i GroupTree.obj
 0001:0001cd20       ?Offset@CPoint@@QAEXHH@Z   0041dd20 f i GroupTree.obj
 0001:0001cd50       ?AfxGetMainWnd@@YGPAVCWnd@@XZ 0041dd50 f i GroupTree.obj
 0001:0001cd90       ??0CMenu@@QAE@XZ           0041dd90 f i GroupTree.obj
 0001:0001cdc0       ??_GCMenu@@UAEPAXI@Z       0041ddc0 f i GroupTree.obj
 0001:0001cdc0       ??_ECMenu@@UAEPAXI@Z       0041ddc0 f i GroupTree.obj
 0001:0001cdf0       ??1CMenu@@UAE@XZ           0041ddf0 f i GroupTree.obj
 0001:0001ce50       ?EnableMenuItem@CMenu@@QAEIII@Z 0041de50 f i GroupTree.obj
 0001:0001ce80       ?GetSubMenu@CMenu@@QBEPAV1@H@Z 0041de80 f i GroupTree.obj
 0001:0001ceb0       ?LoadMenuA@CMenu@@QAEHI@Z  0041deb0 f i GroupTree.obj
 0001:0001cee0       ?SendMessageA@CWnd@@QBEJIIJ@Z 0041dee0 f i GroupTree.obj
 0001:0001cf10       ?PostMessageA@CWnd@@QAEHIIJ@Z 0041df10 f i GroupTree.obj
 0001:0001cf40       ?SetLimitText@CEdit@@QAEXI@Z 0041df40 f i GroupTree.obj
 0001:0001cf70       ??0CTreeCtrl@@QAE@XZ       0041df70 f i GroupTree.obj
 0001:0001cf90       ??_GCTreeCtrl@@UAEPAXI@Z   0041df90 f i GroupTree.obj
 0001:0001cf90       ??_ECTreeCtrl@@UAEPAXI@Z   0041df90 f i GroupTree.obj
 0001:0001cfc0       ?DeleteItem@CTreeCtrl@@QAEHPAU_TREEITEM@@@Z 0041dfc0 f i GroupTree.obj
 0001:0001cff0       ?GetChildItem@CTreeCtrl@@QBEPAU_TREEITEM@@PAU2@@Z 0041dff0 f i GroupTree.obj
 0001:0001d020       ?GetNextSiblingItem@CTreeCtrl@@QBEPAU_TREEITEM@@PAU2@@Z 0041e020 f i GroupTree.obj
 0001:0001d050       ?GetSelectedItem@CTreeCtrl@@QBEPAU_TREEITEM@@XZ 0041e050 f i GroupTree.obj
 0001:0001d080       ?SelectItem@CTreeCtrl@@QAEHPAU_TREEITEM@@@Z 0041e080 f i GroupTree.obj
 0001:0001d0b0       ?SetItemText@CTreeCtrl@@QAEHPAU_TREEITEM@@PBD@Z 0041e0b0 f i GroupTree.obj
 0001:0001d0e0       ?EnsureVisible@CTreeCtrl@@QAEHPAU_TREEITEM@@@Z 0041e0e0 f i GroupTree.obj
 0001:0001d110       ??0CInfoPromptDlg@@QAE@PAVCWnd@@@Z 0041e110 f   InfoPromptDlg.obj
 0001:0001d1b0       ??_ECInfoPromptDlg@@UAEPAXI@Z 0041e1b0 f i InfoPromptDlg.obj
 0001:0001d1b0       ??_GCInfoPromptDlg@@UAEPAXI@Z 0041e1b0 f i InfoPromptDlg.obj
 0001:0001d1e0       ??1CInfoPromptDlg@@UAE@XZ  0041e1e0 f i InfoPromptDlg.obj
 0001:0001d210       ?DoDataExchange@CInfoPromptDlg@@MAEXPAVCDataExchange@@@Z 0041e210 f   InfoPromptDlg.obj
 0001:0001d240       ?OnInitDialog@CInfoPromptDlg@@MAEHXZ 0041e240 f   InfoPromptDlg.obj
 0001:0001d2f0       ??0CIOCPImplement@@QAE@XZ  0041e2f0 f   IOCPImplement.obj
 0001:0001d360       ??_ECIOCPImplement@@UAEPAXI@Z 0041e360 f i IOCPImplement.obj
 0001:0001d360       ??_GCIOCPImplement@@UAEPAXI@Z 0041e360 f i IOCPImplement.obj
 0001:0001d390       ??1CIOCPImplement@@UAE@XZ  0041e390 f   IOCPImplement.obj
 0001:0001d450       ??1?$CTypedPtrMap@VCMapPtrToPtr@@PAVCClientContext@@PAUIOCP_DataRecvBuffer@@@@UAE@XZ 0041e450 f i IOCPImplement.obj
 0001:0001d470       ?WriteToConsole@CIOCPImplement@@UAEXPAD@Z 0041e470 f   IOCPImplement.obj
 0001:0001d4a0       ?OnRecvComplete@CIOCPImplement@@UAEHPAVCClientContext@@@Z 0041e4a0 f   IOCPImplement.obj
 0001:0001d910       ?GetSocket@CClientContext@@QAEIXZ 0041e910 f i IOCPImplement.obj
 0001:0001d930       ?GetBuffer@CClientContext@@QAEHPADAAI@Z 0041e930 f i IOCPImplement.obj
 0001:0001d990       ?OnSendComplete@CIOCPImplement@@UAEHPAVCClientContext@@@Z 0041e990 f   IOCPImplement.obj
 0001:0001da00       ?SendAck@CIOCPImplement@@UAEHPAVCClientContext@@@Z 0041ea00 f   IOCPImplement.obj
 0001:0001dbd0       ?SetOpCode@CClientContext@@QAEXH@Z 0041ebd0 f i IOCPImplement.obj
 0001:0001dbf0       ?SetBuffer@CClientContext@@QAEHPADAAI@Z 0041ebf0 f i IOCPImplement.obj
 0001:0001dc40       ?OnConnectionEstablished@CIOCPImplement@@UAEXPAVCClientContext@@@Z 0041ec40 f   IOCPImplement.obj
 0001:0001dcc0       ?OnConnectionClosing@CIOCPImplement@@UAEXPAVCClientContext@@@Z 0041ecc0 f   IOCPImplement.obj
 0001:0001dd10       ??0?$CTypedPtrMap@VCMapPtrToPtr@@PAVCClientContext@@PAUIOCP_DataRecvBuffer@@@@QAE@H@Z 0041ed10 f i IOCPImplement.obj
 0001:0001dd40       ?Lookup@?$CTypedPtrMap@VCMapPtrToPtr@@PAVCClientContext@@PAUIOCP_DataRecvBuffer@@@@QBEHPAXAAPAUIOCP_DataRecvBuffer@@@Z 0041ed40 f i IOCPImplement.obj
 0001:0001dd60       ??A?$CTypedPtrMap@VCMapPtrToPtr@@PAVCClientContext@@PAUIOCP_DataRecvBuffer@@@@QAEAAPAUIOCP_DataRecvBuffer@@PAX@Z 0041ed60 f i IOCPImplement.obj
 0001:0001dd80       ?RemoveKey@?$CTypedPtrMap@VCMapPtrToPtr@@PAVCClientContext@@PAUIOCP_DataRecvBuffer@@@@QAEHPAVCClientContext@@@Z 0041ed80 f i IOCPImplement.obj
 0001:0001dda0       ?GetNextAssoc@?$CTypedPtrMap@VCMapPtrToPtr@@PAVCClientContext@@PAUIOCP_DataRecvBuffer@@@@QBEXAAPAU__POSITION@@AAPAVCClientContext@@AAPAUIOCP_DataRecvBuffer@@@Z 0041eda0 f i IOCPImplement.obj
 0001:0001ddd0       ??_G?$CTypedPtrMap@VCMapPtrToPtr@@PAVCClientContext@@PAUIOCP_DataRecvBuffer@@@@UAEPAXI@Z 0041edd0 f i IOCPImplement.obj
 0001:0001ddd0       ??_E?$CTypedPtrMap@VCMapPtrToPtr@@PAVCClientContext@@PAUIOCP_DataRecvBuffer@@@@UAEPAXI@Z 0041edd0 f i IOCPImplement.obj
 0001:0001de00       ??$sprintf_s@$0PP@@@YAHAAY0PP@DPBDZZ 0041ee00 f i IOCPImplement.obj
 0001:0001de30       ?GetMessageMap@CKiboManagerApp@@MBEPBUAFX_MSGMAP@@XZ 0041ee30 f   KiboManager.obj
 0001:0001de40       ?GetThisMessageMap@CKiboManagerApp@@KGPBUAFX_MSGMAP@@XZ 0041ee40 f   KiboManager.obj
 0001:0001de50       ??0CKiboManagerApp@@QAE@XZ 0041ee50 f   KiboManager.obj
 0001:0001de80       ??_ECKiboManagerApp@@UAEPAXI@Z 0041ee80 f i KiboManager.obj
 0001:0001de80       ??_GCKiboManagerApp@@UAEPAXI@Z 0041ee80 f i KiboManager.obj
 0001:0001deb0       ??1CKiboManagerApp@@UAE@XZ 0041eeb0 f i KiboManager.obj
 0001:0001ded0       ?InitInstance@CKiboManagerApp@@UAEHXZ 0041eed0 f   KiboManager.obj
 0001:0001e3f0       ?ExitInstance@CKiboManagerApp@@UAEHXZ 0041f3f0 f   KiboManager.obj
 0001:0001e4a0       ?PreLoadState@CKiboManagerApp@@UAEXXZ 0041f4a0 f   KiboManager.obj
 0001:0001e530       ?GetParent@CWnd@@QBEPAV1@XZ 0041f530 f i KiboManager.obj
 0001:0001e550       ??0GdiplusStartupInput@Gdiplus@@QAE@P6GXW4DebugEventLevel@1@PAD@ZHH@Z 0041f550 f i KiboManager.obj
 0001:0001e590       ??0CMFCToolTipInfo@@QAE@XZ 0041f590 f i KiboManager.obj
 0001:0001e620       ?CreateObject@CKiboManagerDoc@@SGPAVCObject@@XZ 0041f620 f   KiboManagerDoc.obj
 0001:0001e690       ?_GetBaseClass@CKiboManagerDoc@@KGPAUCRuntimeClass@@XZ 0041f690 f   KiboManagerDoc.obj
 0001:0001e6a0       ?GetThisClass@CKiboManagerDoc@@SGPAUCRuntimeClass@@XZ 0041f6a0 f   KiboManagerDoc.obj
 0001:0001e6b0       ?GetRuntimeClass@CKiboManagerDoc@@UBEPAUCRuntimeClass@@XZ 0041f6b0 f   KiboManagerDoc.obj
 0001:0001e6c0       ?GetMessageMap@CKiboManagerDoc@@MBEPBUAFX_MSGMAP@@XZ 0041f6c0 f   KiboManagerDoc.obj
 0001:0001e6d0       ?GetThisMessageMap@CKiboManagerDoc@@KGPBUAFX_MSGMAP@@XZ 0041f6d0 f   KiboManagerDoc.obj
 0001:0001e6e0       ??0CKiboManagerDoc@@IAE@XZ 0041f6e0 f   KiboManagerDoc.obj
 0001:0001e700       ??_GCKiboManagerDoc@@UAEPAXI@Z 0041f700 f i KiboManagerDoc.obj
 0001:0001e700       ??_ECKiboManagerDoc@@UAEPAXI@Z 0041f700 f i KiboManagerDoc.obj
 0001:0001e730       ??1CKiboManagerDoc@@UAE@XZ 0041f730 f   KiboManagerDoc.obj
 0001:0001e750       ?OnNewDocument@CKiboManagerDoc@@UAEHXZ 0041f750 f   KiboManagerDoc.obj
 0001:0001e8b0       ?Serialize@CKiboManagerDoc@@UAEXAAVCArchive@@@Z 0041f8b0 f   KiboManagerDoc.obj
 0001:0001e8d0       ?GetNotifyID@CMFCRibbonBaseElement@@UAEIXZ 0041f8d0 f i MainFrm.obj
 0001:0001e8d0       ?GetQuickAccessToolBarID@CMFCRibbonBaseElement@@UBEIXZ 0041f8d0 f i MainFrm.obj
 0001:0001e8d0       ?IsModified@CDocument@@UAEHXZ 0041f8d0 f i KiboManagerDoc.obj
 0001:0001e8f0       ?SetModifiedFlag@CDocument@@UAEXH@Z 0041f8f0 f i KiboManagerDoc.obj
 0001:0001e910       ?CreateObject@CKiboManagerView@@SGPAVCObject@@XZ 0041f910 f   KiboManagerView.obj
 0001:0001e990       ?_GetBaseClass@CKiboManagerView@@KGPAUCRuntimeClass@@XZ 0041f990 f   KiboManagerView.obj
 0001:0001e9a0       ?GetThisClass@CKiboManagerView@@SGPAUCRuntimeClass@@XZ 0041f9a0 f   KiboManagerView.obj
 0001:0001e9b0       ?GetRuntimeClass@CKiboManagerView@@UBEPAUCRuntimeClass@@XZ 0041f9b0 f   KiboManagerView.obj
 0001:0001e9c0       ?GetMessageMap@CKiboManagerView@@MBEPBUAFX_MSGMAP@@XZ 0041f9c0 f   KiboManagerView.obj
 0001:0001e9d0       ?GetThisMessageMap@CKiboManagerView@@KGPBUAFX_MSGMAP@@XZ 0041f9d0 f   KiboManagerView.obj
 0001:0001e9e0       ??0CKiboManagerView@@IAE@XZ 0041f9e0 f   KiboManagerView.obj
 0001:0001eb10       ??_ECKiboManagerView@@UAEPAXI@Z 0041fb10 f i KiboManagerView.obj
 0001:0001eb10       ??_GCKiboManagerView@@UAEPAXI@Z 0041fb10 f i KiboManagerView.obj
 0001:0001eb40       ??1CKiboManagerView@@UAE@XZ 0041fb40 f   KiboManagerView.obj
 0001:0001ebf0       ?DoDataExchange@CKiboManagerView@@MAEXPAVCDataExchange@@@Z 0041fbf0 f   KiboManagerView.obj
 0001:0001ec30       ?PreCreateWindow@CKiboManagerView@@UAEHAAUtagCREATESTRUCTA@@@Z 0041fc30 f   KiboManagerView.obj
 0001:0001ec50       ?OnInitialUpdate@CKiboManagerView@@MAEXXZ 0041fc50 f   KiboManagerView.obj
 0001:0001f200       ?OnContextMenu@CKiboManagerView@@IAEXPAVCWnd@@VCPoint@@@Z 00420200 f   KiboManagerView.obj
 0001:0001f840       ?OnSize@CKiboManagerView@@QAEXIHH@Z 00420840 f   KiboManagerView.obj
 0001:0001f980       ?CheckSelectionForCmd@CKiboManagerView@@QAEHH@Z 00420980 f   KiboManagerView.obj
 0001:0001fc50       ?CheckOnlineAndHasSysForCmd@CKiboManagerView@@QAEHXZ 00420c50 f   KiboManagerView.obj
 0001:0001feb0       ?CheckDriverAndStatus@CKiboManagerView@@QAEHH@Z 00420eb0 f   KiboManagerView.obj
 0001:00020260       ?CheckAllSelOnline@CKiboManagerView@@QAEHXZ 00421260 f   KiboManagerView.obj
 0001:000204a0       ?_SortListItemThread@CKiboManagerView@@SAIPAX@Z 004214a0 f   KiboManagerView.obj
 0001:000206f0       ?OnLvnItemchangedList1@CKiboManagerView@@QAEXPAUtagNMHDR@@PAJ@Z 004216f0 f   KiboManagerView.obj
 0001:00020c80       ?_DeleteListItemThread@CKiboManagerView@@SAIPAX@Z 00421c80 f   KiboManagerView.obj
 0001:00021190       ?LoadComputerView@CKiboManagerView@@QAEXXZ 00422190 f   KiboManagerView.obj
 0001:000216a0       ?LoadGroupView@CKiboManagerView@@QAEXXZ 004226a0 f   KiboManagerView.obj
 0001:00021800       ?OnLvnColumnclickList1@CKiboManagerView@@QAEXPAUtagNMHDR@@PAJ@Z 00422800 f   KiboManagerView.obj
 0001:000218c0       ?OnSetItemTextList1@CKiboManagerView@@QAEXPAUtagNMHDR@@PAJ@Z 004228c0 f   KiboManagerView.obj
 0001:00021be0       ?OnNMDblclkList1@CKiboManagerView@@QAEXPAUtagNMHDR@@PAJ@Z 00422be0 f   KiboManagerView.obj
 0001:00021d40       ?OnViewproperty@CKiboManagerView@@QAEXXZ 00422d40 f   KiboManagerView.obj
 0001:00021f60       ?OnNMSetfocusList1@CKiboManagerView@@QAEXPAUtagNMHDR@@PAJ@Z 00422f60 f   KiboManagerView.obj
 0001:00021fc0       ?OnShutdown@CKiboManagerView@@QAEXXZ 00422fc0 f   KiboManagerView.obj
 0001:00021fe0       ?OnRestart@CKiboManagerView@@QAEXXZ 00422fe0 f   KiboManagerView.obj
 0001:00022000       ?OnWol@CKiboManagerView@@QAEXXZ 00423000 f   KiboManagerView.obj
 0001:00022020       ?OnClientsettings@CKiboManagerView@@QAEXXZ 00423020 f   KiboManagerView.obj
 0001:00022040       ?OnIpsettings@CKiboManagerView@@QAEXXZ 00423040 f   KiboManagerView.obj
 0001:00022060       ?OnMenuDelfromgroup@CKiboManagerView@@QAEXXZ 00423060 f   KiboManagerView.obj
 0001:00022440       ?_DelFromGroupThread@CKiboManagerView@@SAIPAX@Z 00423440 f   KiboManagerView.obj
 0001:00022a20       ?OnMenuAddtogroup@CKiboManagerView@@QAEXXZ 00423a20 f   KiboManagerView.obj
 0001:00023090       ?_AddClientToGroupThread@CKiboManagerView@@SAIPAX@Z 00424090 f   KiboManagerView.obj
 0001:00023530       ?OnDellist@CKiboManagerView@@QAEXXZ 00424530 f   KiboManagerView.obj
 0001:00023550       ?OnLvnGetInfoTipList1@CKiboManagerView@@QAEXPAUtagNMHDR@@PAJ@Z 00424550 f   KiboManagerView.obj
 0001:00023920       ?OnNMKillfocusList1@CKiboManagerView@@QAEXPAUtagNMHDR@@PAJ@Z 00424920 f   KiboManagerView.obj
 0001:00023940       ?OnMenuRemovehand@CKiboManagerView@@QAEXXZ 00424940 f   KiboManagerView.obj
 0001:00023960       ?CheckMode@CKiboManagerView@@QAEHH@Z 00424960 f   KiboManagerView.obj
 0001:000244e0       ?PreTranslateMessage@CKiboManagerView@@UAEHPAUtagMSG@@@Z 004254e0 f   KiboManagerView.obj
 0001:00024500       ?OnUpdateShutdown@CKiboManagerView@@QAEXPAVCCmdUI@@@Z 00425500 f   KiboManagerView.obj
 0001:00024530       ?OnUpdateRestart@CKiboManagerView@@QAEXPAVCCmdUI@@@Z 00425530 f   KiboManagerView.obj
 0001:00024560       ?OnUpdateWol@CKiboManagerView@@QAEXPAVCCmdUI@@@Z 00425560 f   KiboManagerView.obj
 0001:00024590       ?OnUpdateViewproperty@CKiboManagerView@@QAEXPAVCCmdUI@@@Z 00425590 f   KiboManagerView.obj
 0001:000245c0       ?OnUpdateClientsettings@CKiboManagerView@@QAEXPAVCCmdUI@@@Z 004255c0 f   KiboManagerView.obj
 0001:000245f0       ?OnUpdateIpsettings@CKiboManagerView@@QAEXPAVCCmdUI@@@Z 004255f0 f   KiboManagerView.obj
 0001:00024620       ?OnUpdateMenuDelfromgroup@CKiboManagerView@@QAEXPAVCCmdUI@@@Z 00425620 f   KiboManagerView.obj
 0001:00024650       ?OnUpdateMenuAddtogroup@CKiboManagerView@@QAEXPAVCCmdUI@@@Z 00425650 f   KiboManagerView.obj
 0001:00024680       ?OnUpdateMenuRemovehand@CKiboManagerView@@QAEXPAVCCmdUI@@@Z 00425680 f   KiboManagerView.obj
 0001:000246b0       ?CheckSelectionNum@CKiboManagerView@@QAEHHH@Z 004256b0 f   KiboManagerView.obj
 0001:00024980       ?OnNMRClickList1@CKiboManagerView@@QAEXPAUtagNMHDR@@PAJ@Z 00425980 f   KiboManagerView.obj
 0001:00024a50       ?OnSpecialSave@CKiboManagerView@@QAEXXZ 00425a50 f   KiboManagerView.obj
 0001:00024a70       ?OnSpecialRecovery@CKiboManagerView@@QAEXXZ 00425a70 f   KiboManagerView.obj
 0001:00024a90       ?CheckOnlineAndRegistered@CKiboManagerView@@QAEHXZ 00425a90 f   KiboManagerView.obj
 0001:00024ce0       ?OnAddRadom@CKiboManagerView@@QAEXXZ 00425ce0 f   KiboManagerView.obj
 0001:00024d10       ?OnUpdateAddRadom@CKiboManagerView@@QAEXPAVCCmdUI@@@Z 00425d10 f   KiboManagerView.obj
 0001:00024d10       ?OnUpdateDellist@CKiboManagerView@@QAEXPAVCCmdUI@@@Z 00425d10 f   KiboManagerView.obj
 0001:00024d40       ?OnOnLinePC@CKiboManagerView@@QAEXXZ 00425d40 f   KiboManagerView.obj
 0001:00024d90       ?OnUpdateOnLinePC@CKiboManagerView@@QAEXPAVCCmdUI@@@Z 00425d90 f   KiboManagerView.obj
 0001:00024dc0       ??9ATL@@YA_NABV?$CStringT@DV?$StrTraitMFC_DLL@DV?$ChTraitsCRT@D@ATL@@@@@0@0@Z 00425dc0 f i KiboManagerView.obj
 0001:00024de0       ??0logic_error@std@@QAE@ABV?$basic_string@DU?$char_traits@D@std@@V?$allocator@D@2@@1@@Z 00425de0 f i KiboManagerView.obj
 0001:00024e50       ?what@logic_error@std@@UBEPBDXZ 00425e50 f i KiboManagerView.obj
 0001:00024e70       ??_Elogic_error@std@@UAEPAXI@Z 00425e70 f i KiboManagerView.obj
 0001:00024e70       ??_Glogic_error@std@@UAEPAXI@Z 00425e70 f i KiboManagerView.obj
 0001:00024ea0       ??1logic_error@std@@UAE@XZ 00425ea0 f i KiboManagerView.obj
 0001:00024ed0       ??0logic_error@std@@QAE@ABV01@@Z 00425ed0 f i KiboManagerView.obj
 0001:00024f50       ??0length_error@std@@QAE@ABV?$basic_string@DU?$char_traits@D@std@@V?$allocator@D@2@@1@@Z 00425f50 f i KiboManagerView.obj
 0001:00024f80       ??1length_error@std@@UAE@XZ 00425f80 f i KiboManagerView.obj
 0001:00024fa0       ??_Elength_error@std@@UAEPAXI@Z 00425fa0 f i KiboManagerView.obj
 0001:00024fa0       ??_Glength_error@std@@UAEPAXI@Z 00425fa0 f i KiboManagerView.obj
 0001:00024fd0       ??0length_error@std@@QAE@ABV01@@Z 00425fd0 f i KiboManagerView.obj
 0001:00025000       ??0bad_alloc@std@@QAE@ABV01@@Z 00426000 f i KiboManagerView.obj
 0001:00025030       ??0CSize@@QAE@HH@Z         00426030 f i MainFrm.obj
 0001:00025030       ??0CPoint@@QAE@HH@Z        00426030 f i KiboManagerView.obj
 0001:00025060       ?Width@CRect@@QBEHXZ       00426060 f i KiboManagerView.obj
 0001:00025080       ?Height@CRect@@QBEHXZ      00426080 f i KiboManagerView.obj
 0001:000250a0       ?ModifyMenuA@CMenu@@QAEHIIIPBD@Z 004260a0 f i KiboManagerView.obj
 0001:000250d0       ?SetRedraw@CWnd@@QAEXH@Z   004260d0 f i KiboManagerView.obj
 0001:00025100       ?get_accChild@CFormView@@UAEJUtagVARIANT@@PAPAUIDispatch@@@Z 00426100 f i KiboManagerView.obj
 0001:00025140       ?get_accChildCount@CFormView@@UAEJPAJ@Z 00426140 f i KiboManagerView.obj
 0001:00025160       ?get_accName@CFormView@@UAEJUtagVARIANT@@PAPA_W@Z 00426160 f i KiboManagerView.obj
 0001:000251a0       ?accLocation@CFormView@@UAEJPAJ000UtagVARIANT@@@Z 004261a0 f i KiboManagerView.obj
 0001:000251f0       ?accHitTest@CFormView@@UAEJJJPAUtagVARIANT@@@Z 004261f0 f i KiboManagerView.obj
 0001:00025220       ?SetImageList@CListCtrl@@QAEPAVCImageList@@PAV2@H@Z 00426220 f i KiboManagerView.obj
 0001:00025260       ?DeleteColumn@CListCtrl@@QAEHH@Z 00426260 f i KiboManagerView.obj
 0001:00025290       ??0_Aux_cont@std@@QAE@QBV_Container_base_aux@1@@Z 00426290 f i KiboManagerView.obj
 0001:000252b0       ?_Set_container@_Iterator_base_aux@std@@QAEXQBV_Container_base_aux@2@@Z 004262b0 f i KiboManagerView.obj
 0001:000252d0       ?_Getmycont@_Iterator_base_aux@std@@QBEPBV_Container_base_aux@2@XZ 004262d0 f i KiboManagerView.obj
 0001:00025300       ?_Same_container@_Iterator_base_aux@std@@QBE_NABV12@@Z 00426300 f i KiboManagerView.obj
 0001:00025320       ?_Has_container@_Iterator_base_aux@std@@QBE_NXZ 00426320 f i KiboManagerView.obj
 0001:00025340       ??0bad_alloc@std@@QAE@PBD@Z 00426340 f i KiboManagerView.obj
 0001:00025370       ??1bad_alloc@std@@UAE@XZ   00426370 f i KiboManagerView.obj
 0001:00025390       ??_Gbad_alloc@std@@UAEPAXI@Z 00426390 f i KiboManagerView.obj
 0001:00025390       ??_Ebad_alloc@std@@UAEPAXI@Z 00426390 f i KiboManagerView.obj
 0001:000253c0       ??0CLenPropertyODBC@@QAE@XZ 004263c0 f   LenPropertyODBC.obj
 0001:000253f0       ??_GCLenPropertyODBC@@UAEPAXI@Z 004263f0 f i LenPropertyODBC.obj
 0001:000253f0       ??_ECLenPropertyODBC@@UAEPAXI@Z 004263f0 f i LenPropertyODBC.obj
 0001:00025420       ??1CLenPropertyODBC@@UAE@XZ 00426420 f   LenPropertyODBC.obj
 0001:00025450       ?InsertOnePropertyMainInfo@CLenPropertyODBC@@QAE?AV?$CStringT@DV?$StrTraitMFC_DLL@DV?$ChTraitsCRT@D@ATL@@@@@ATL@@PAUPropertyInfo@@H@Z 00426450 f   LenPropertyODBC.obj
 0001:00025620       ?UpdateOnePropertyMainInfo@CLenPropertyODBC@@QAE?AV?$CStringT@DV?$StrTraitMFC_DLL@DV?$ChTraitsCRT@D@ATL@@@@@ATL@@PAUPropertyInfo@@H@Z 00426620 f   LenPropertyODBC.obj
 0001:000257f0       ?DeleteOnePropertyMainInfo@CLenPropertyODBC@@QAE?AV?$CStringT@DV?$StrTraitMFC_DLL@DV?$ChTraitsCRT@D@ATL@@@@@ATL@@PBDH@Z 004267f0 f   LenPropertyODBC.obj
 0001:000258d0       ?InsertOneComputerInfo@CLenPropertyODBC@@QAE?AV?$CStringT@DV?$StrTraitMFC_DLL@DV?$ChTraitsCRT@D@ATL@@@@@ATL@@PAUComputerInfo@@@Z 004268d0 f   LenPropertyODBC.obj
 0001:000259c0       ?UpdateOneComputerInfo@CLenPropertyODBC@@QAE?AV?$CStringT@DV?$StrTraitMFC_DLL@DV?$ChTraitsCRT@D@ATL@@@@@ATL@@PAUComputerInfo@@@Z 004269c0 f   LenPropertyODBC.obj
 0001:00025ab0       ?DeleteOneComputerInfo@CLenPropertyODBC@@QAE?AV?$CStringT@DV?$StrTraitMFC_DLL@DV?$ChTraitsCRT@D@ATL@@@@@ATL@@PBD@Z 00426ab0 f   LenPropertyODBC.obj
 0001:00025b40       ?GetAllComputerInfo@CLenPropertyODBC@@QAE?AV?$CStringT@DV?$StrTraitMFC_DLL@DV?$ChTraitsCRT@D@ATL@@@@@ATL@@XZ 00426b40 f   LenPropertyODBC.obj
 0001:00025bd0       ?InsertOneSoftwareInfo@CLenPropertyODBC@@QAE?AV?$CStringT@DV?$StrTraitMFC_DLL@DV?$ChTraitsCRT@D@ATL@@@@@ATL@@PBDI0H@Z 00426bd0 f   LenPropertyODBC.obj
 0001:00025cb0       ?DeleteSoftwareInfo@CLenPropertyODBC@@QAE?AV?$CStringT@DV?$StrTraitMFC_DLL@DV?$ChTraitsCRT@D@ATL@@@@@ATL@@PBDH@Z 00426cb0 f   LenPropertyODBC.obj
 0001:00025d90       ?DeleteSoftwareInfo@CLenPropertyODBC@@QAE?AV?$CStringT@DV?$StrTraitMFC_DLL@DV?$ChTraitsCRT@D@ATL@@@@@ATL@@PBDIH@Z 00426d90 f   LenPropertyODBC.obj
 0001:00025e70       ?GetOnePropertyInfo@CLenPropertyODBC@@QAEHPBDIHPAUPropertyInfo@@@Z 00426e70 f   LenPropertyODBC.obj
 0001:000263e0       ?IfCurrentPropertyInfoChanged@CLenPropertyODBC@@QAEHPAUPropertyInfo@@AAV?$CStringT@DV?$StrTraitMFC_DLL@DV?$ChTraitsCRT@D@ATL@@@@@ATL@@@Z 004273e0 f   LenPropertyODBC.obj
 0001:00027b40       ?CompareAndGetAbstract@CLenPropertyODBC@@QAEHPAUPropertyInfo@@0AAV?$CStringT@DV?$StrTraitMFC_DLL@DV?$ChTraitsCRT@D@ATL@@@@@ATL@@@Z 00428b40 f   LenPropertyODBC.obj
 0001:00028250       ?InsertOneClientToBlack@CLenPropertyODBC@@QAE?AV?$CStringT@DV?$StrTraitMFC_DLL@DV?$ChTraitsCRT@D@ATL@@@@@ATL@@UComputerInfo@@@Z 00429250 f   LenPropertyODBC.obj
 0001:000282f0       ?RemoveOneFromBlack@CLenPropertyODBC@@QAE?AV?$CStringT@DV?$StrTraitMFC_DLL@DV?$ChTraitsCRT@D@ATL@@@@@ATL@@V23@@Z 004292f0 f   LenPropertyODBC.obj
 0001:00028390       ?GetAllBlackComputer@CLenPropertyODBC@@QAE?AV?$CStringT@DV?$StrTraitMFC_DLL@DV?$ChTraitsCRT@D@ATL@@@@@ATL@@XZ 00429390 f   LenPropertyODBC.obj
 0001:00028420       ?UpdateGroupNameOfClient@CLenPropertyODBC@@QAE?AV?$CStringT@DV?$StrTraitMFC_DLL@DV?$ChTraitsCRT@D@ATL@@@@@ATL@@UtagGroupClient@@@Z 00429420 f   LenPropertyODBC.obj
 0001:000284f0       ?InsertNewGroup@CLenPropertyODBC@@QAE?AV?$CStringT@DV?$StrTraitMFC_DLL@DV?$ChTraitsCRT@D@ATL@@@@@ATL@@V23@@Z 004294f0 f   LenPropertyODBC.obj
 0001:000285d0       ?UpdateGroupName@CLenPropertyODBC@@QAE?AV?$CStringT@DV?$StrTraitMFC_DLL@DV?$ChTraitsCRT@D@ATL@@@@@ATL@@V23@0@Z 004295d0 f   LenPropertyODBC.obj
 0001:000286f0       ?UpdateGroupInfoByOldGroupName@CLenPropertyODBC@@QAE?AV?$CStringT@DV?$StrTraitMFC_DLL@DV?$ChTraitsCRT@D@ATL@@@@@ATL@@V23@UtagGroupClient@@@Z 004296f0 f   LenPropertyODBC.obj
 0001:00028810       ?GetAllGroup@CLenPropertyODBC@@QAE?AV?$CStringT@DV?$StrTraitMFC_DLL@DV?$ChTraitsCRT@D@ATL@@@@@ATL@@XZ 00429810 f   LenPropertyODBC.obj
 0001:000288a0       ?GetAllGroupClient@CLenPropertyODBC@@QAE?AV?$CStringT@DV?$StrTraitMFC_DLL@DV?$ChTraitsCRT@D@ATL@@@@@ATL@@V23@@Z 004298a0 f   LenPropertyODBC.obj
 0001:00028980       ?RemoveGroup@CLenPropertyODBC@@QAE?AV?$CStringT@DV?$StrTraitMFC_DLL@DV?$ChTraitsCRT@D@ATL@@@@@ATL@@V23@@Z 00429980 f   LenPropertyODBC.obj
 0001:00028a60       ?UpdateOneToGroup@CLenPropertyODBC@@QAE?AV?$CStringT@DV?$StrTraitMFC_DLL@DV?$ChTraitsCRT@D@ATL@@@@@ATL@@UtagGroupClient@@@Z 00429a60 f   LenPropertyODBC.obj
 0001:00028b30       ?InsertClientToGroup@CLenPropertyODBC@@QAE?AV?$CStringT@DV?$StrTraitMFC_DLL@DV?$ChTraitsCRT@D@ATL@@@@@ATL@@UtagGroupClient@@@Z 00429b30 f   LenPropertyODBC.obj
 0001:00028c00       ?RemoveOneGroupCLient@CLenPropertyODBC@@QAE?AV?$CStringT@DV?$StrTraitMFC_DLL@DV?$ChTraitsCRT@D@ATL@@@@@ATL@@V23@@Z 00429c00 f   LenPropertyODBC.obj
 0001:00028ca0       ?TranHexToString@CLenPropertyODBC@@QAE?AV?$CStringT@DV?$StrTraitMFC_DLL@DV?$ChTraitsCRT@D@ATL@@@@@ATL@@V23@H@Z 00429ca0 f   LenPropertyODBC.obj
 0001:00028fa0       ?SortSoftwareInfo@CLenPropertyODBC@@QAE?AV?$CStringT@DV?$StrTraitMFC_DLL@DV?$ChTraitsCRT@D@ATL@@@@@ATL@@H@Z 00429fa0 f   LenPropertyODBC.obj
 0001:00029070       ??9ATL@@YA_NABV?$CStringT@DV?$StrTraitMFC_DLL@DV?$ChTraitsCRT@D@ATL@@@@@0@PBD@Z 0042a070 f i LenPropertyODBC.obj
 0001:00029090       ??$strcpy_s@$0BE@@@YAHAAY0BE@DPBD@Z 0042a090 f i LenPropertyODBC.obj
 0001:000290b0       ??$strcpy_s@$0JG@@@YAHAAY0JG@DPBD@Z 0042a0b0 f i LenPropertyODBC.obj
 0001:000290d0       ??$strcpy_s@$0PP@@@YAHAAY0PP@DPBD@Z 0042a0d0 f i LenPropertyODBC.obj
 0001:000290f0       ??$strcpy_s@$0GE@@@YAHAAY0GE@DPBD@Z 0042a0f0 f i LenPropertyODBC.obj
 0001:00029110       ??$strcpy_s@$0MI@@@YAHAAY0MI@DPBD@Z 0042a110 f i LenPropertyODBC.obj
 0001:00029130       ??$sprintf_s@$04@@YAHAAY04DPBDZZ 0042a130 f i LenPropertyODBC.obj
 0001:00029160       ?SetAt@CMapStringToString@@QAEXPBD0@Z 0042a160 f i LenPropertyODBC.obj
 0001:00029190       ?GetItem@CListCtrl@@QBEHPAUtagLVITEMA@@@Z 0042a190 f i ListCtrlEx.obj
 0001:000291c0       ?SetItem@CListCtrl@@QAEHPBUtagLVITEMA@@@Z 0042a1c0 f i ListCtrlEx.obj
 0001:000291f0       ?GetItemState@CListCtrl@@QBEIHI@Z 0042a1f0 f i ListCtrlEx.obj
 0001:00029220       ?SortItems@CListCtrl@@QAEHP6GHJJJ@ZK@Z 0042a220 f i ListCtrlEx.obj
 0001:00029250       ?GetRuntimeClass@CLoginPasswordDlg@@UBEPAUCRuntimeClass@@XZ 0042a250 f   LoginPasswordDlg.obj
 0001:00029260       ??0CLoginPasswordDlg@@QAE@PAVCWnd@@@Z 0042a260 f   LoginPasswordDlg.obj
 0001:00029300       ??_GCLoginPasswordDlg@@UAEPAXI@Z 0042a300 f i LoginPasswordDlg.obj
 0001:00029300       ??_ECLoginPasswordDlg@@UAEPAXI@Z 0042a300 f i LoginPasswordDlg.obj
 0001:00029330       ??1CLoginPasswordDlg@@UAE@XZ 0042a330 f   LoginPasswordDlg.obj
 0001:000293a0       ?DoDataExchange@CLoginPasswordDlg@@MAEXPAVCDataExchange@@@Z 0042a3a0 f   LoginPasswordDlg.obj
 0001:00029410       ?GetMessageMap@CLoginPasswordDlg@@MBEPBUAFX_MSGMAP@@XZ 0042a410 f   LoginPasswordDlg.obj
 0001:00029420       ?GetThisMessageMap@CLoginPasswordDlg@@KGPBUAFX_MSGMAP@@XZ 0042a420 f   LoginPasswordDlg.obj
 0001:00029430       ?OnOK@CLoginPasswordDlg@@MAEXXZ 0042a430 f   LoginPasswordDlg.obj
 0001:00029580       ?OnInitDialog@CLoginPasswordDlg@@MAEHXZ 0042a580 f   LoginPasswordDlg.obj
 0001:00029930       ?OnBnClickedOk@CLoginPasswordDlg@@QAEXXZ 0042a930 f   LoginPasswordDlg.obj
 0001:00029a50       ?OnEnChangeEditMainpwd@CLoginPasswordDlg@@IAEXXZ 0042aa50 f   LoginPasswordDlg.obj
 0001:00029ac0       ?ExtPwd@CLoginPasswordDlg@@AAE_NAAV?$CStringT@DV?$StrTraitMFC_DLL@DV?$ChTraitsCRT@D@ATL@@@@@ATL@@PAEH@Z 0042aac0 f   LoginPasswordDlg.obj
 0001:00029d50       ?EncodeString@@YAXPBDPAPAD0@Z 0042ad50 f   LoginPasswordDlg.obj
 0001:00029f80       ?SetIcon@CWnd@@QAEPAUHICON__@@PAU2@H@Z 0042af80 f i LoginPasswordDlg.obj
 0001:00029fb0       ?GetWindowRect@CWnd@@QBEXPAUtagRECT@@@Z 0042afb0 f i MainDlg.obj
 0001:00029fd0       ?CompareProc@@YGHJJJ@Z     0042afd0 f   MainFrm.obj
 0001:0002a840       ?CreateObject@CMainFrame@@SGPAVCObject@@XZ 0042b840 f   MainFrm.obj
 0001:0002a8c0       ?_GetBaseClass@CMainFrame@@KGPAUCRuntimeClass@@XZ 0042b8c0 f   MainFrm.obj
 0001:0002a8d0       ?GetThisClass@CMainFrame@@SGPAUCRuntimeClass@@XZ 0042b8d0 f   MainFrm.obj
 0001:0002a8e0       ?GetRuntimeClass@CMainFrame@@UBEPAUCRuntimeClass@@XZ 0042b8e0 f   MainFrm.obj
 0001:0002a8f0       ?GetMessageMap@CMainFrame@@MBEPBUAFX_MSGMAP@@XZ 0042b8f0 f   MainFrm.obj
 0001:0002a900       ?GetThisMessageMap@CMainFrame@@KGPBUAFX_MSGMAP@@XZ 0042b900 f   MainFrm.obj
 0001:0002a910       ??0CMainFrame@@IAE@XZ      0042b910 f   MainFrm.obj
 0001:0002adc0       ??_ECMainFrame@@UAEPAXI@Z  0042bdc0 f i MainFrm.obj
 0001:0002adc0       ??_GCMainFrame@@UAEPAXI@Z  0042bdc0 f i MainFrm.obj
 0001:0002adf0       ??0COutlookBar@@QAE@XZ     0042bdf0 f i MainFrm.obj
 0001:0002ae10       ?GetPaneName@COutlookBar@@EBEXAAV?$CStringT@DV?$StrTraitMFC_DLL@DV?$ChTraitsCRT@D@ATL@@@@@ATL@@@Z 0042be10 f i MainFrm.obj
 0001:0002ae30       ??1COutlookBar@@UAE@XZ     0042be30 f i MainFrm.obj
 0001:0002ae50       ??1?$_CTypedPtrList@VCPtrList@@PAK@@UAE@XZ 0042be50 f i BootModuleManager.obj
 0001:0002ae50       ??1?$_CTypedPtrList@VCPtrList@@PAUtagRECVREQUEST@@@@UAE@XZ 0042be50 f i MainFrm.obj
 0001:0002ae50       ??1?$_CTypedPtrList@VCPtrList@@PAUPartitionTransInfo@@@@UAE@XZ 0042be50 f i MainFrm.obj
 0001:0002ae70       ??_GCOutlookBar@@UAEPAXI@Z 0042be70 f i MainFrm.obj
 0001:0002ae70       ??_ECOutlookBar@@UAEPAXI@Z 0042be70 f i MainFrm.obj
 0001:0002aea0       ??1CMainFrame@@UAE@XZ      0042bea0 f   MainFrm.obj
 0001:0002b130       ?DoDataExchange@CMainFrame@@UAEXPAVCDataExchange@@@Z 0042c130 f   MainFrm.obj
 0001:0002b160       ?OnCreate@CMainFrame@@IAEHPAUtagCREATESTRUCTA@@@Z 0042c160 f   MainFrm.obj
 0001:0002c4b0       ?OnCreateClient@CMainFrame@@UAEHPAUtagCREATESTRUCTA@@PAUCCreateContext@@@Z 0042d4b0 f   MainFrm.obj
 0001:0002c520       ?PreCreateWindow@CMainFrame@@UAEHAAUtagCREATESTRUCTA@@@Z 0042d520 f   MainFrm.obj
 0001:0002c550       ?InitializeRibbon@CMainFrame@@IAEXXZ 0042d550 f   MainFrm.obj
 0001:0002ca00       ?ProductVERCheck@CMainFrame@@QAEHXZ 0042da00 f   MainFrm.obj
 0001:0002cb60       ?CreateDockingWindows@CMainFrame@@IAEHXZ 0042db60 f   MainFrm.obj
 0001:0002ccc0       ?SetDockingWindowIcons@CMainFrame@@IAEXH@Z 0042dcc0 f   MainFrm.obj
 0001:0002cd20       ?OnApplicationLook@CMainFrame@@IAEXI@Z 0042dd20 f   MainFrm.obj
 0001:0002cec0       ?OnUpdateApplicationLook@CMainFrame@@IAEXPAVCCmdUI@@@Z 0042dec0 f   MainFrm.obj
 0001:0002cef0       ?OnViewCaptionBar@CMainFrame@@IAEXXZ 0042def0 f   MainFrm.obj
 0001:0002cf50       ?OnUpdateViewCaptionBar@CMainFrame@@IAEXPAVCCmdUI@@@Z 0042df50 f   MainFrm.obj
 0001:0002cfb0       ?OnViewWorkspace@CMainFrame@@QAEXXZ 0042dfb0 f   MainFrm.obj
 0001:0002d010       ?OnUpdateViewWorkspace@CMainFrame@@QAEXPAVCCmdUI@@@Z 0042e010 f   MainFrm.obj
 0001:0002d070       ?OnViewWorkspace2@CMainFrame@@QAEXXZ 0042e070 f   MainFrm.obj
 0001:0002d0d0       ?OnUpdateViewWorkspace2@CMainFrame@@QAEXPAVCCmdUI@@@Z 0042e0d0 f   MainFrm.obj
 0001:0002d130       ?IsPrintPreviewMode@CMainFrame@@QAEHXZ 0042e130 f   MainFrm.obj
 0001:0002d150       ?OnViewOutput@CMainFrame@@QAEXXZ 0042e150 f   MainFrm.obj
 0001:0002d1b0       ?OnUpdateViewOutput@CMainFrame@@QAEXPAVCCmdUI@@@Z 0042e1b0 f   MainFrm.obj
 0001:0002d210       ?OnViewStatusBar@CMainFrame@@QAEXXZ 0042e210 f   MainFrm.obj
 0001:0002d270       ?OnUpdateViewStatusBar@CMainFrame@@QAEXPAVCCmdUI@@@Z 0042e270 f   MainFrm.obj
 0001:0002d2d0       ?OnIconView@CMainFrame@@QAEXXZ 0042e2d0 f   MainFrm.obj
 0001:0002d320       ?OnReportView@CMainFrame@@QAEXXZ 0042e320 f   MainFrm.obj
 0001:0002d430       ?OnUpdateIconView@CMainFrame@@QAEXPAVCCmdUI@@@Z 0042e430 f   MainFrm.obj
 0001:0002d470       ?OnUpdateReportView@CMainFrame@@QAEXPAVCCmdUI@@@Z 0042e470 f   MainFrm.obj
 0001:0002d4c0       ?OnTimer@CMainFrame@@QAEXI@Z 0042e4c0 f   MainFrm.obj
 0001:0002dc40       ?InitNetworkComponent@CMainFrame@@QAEHXZ 0042ec40 f   MainFrm.obj
 0001:0002dee0       ?_RequestHandleThread@CMainFrame@@SAIPAX@Z 0042eee0 f   MainFrm.obj
 0001:0002e3e0       ?_CheckOnlineThread@CMainFrame@@SAIPAX@Z 0042f3e0 f   MainFrm.obj
 0001:0002e440       ?CheckClientsOnline@CMainFrame@@QAEXXZ 0042f440 f   MainFrm.obj
 0001:0002eaf0       ?HandleLoginRequest@CMainFrame@@QAEHPAUtagRECVREQUEST@@@Z 0042faf0 f   MainFrm.obj
 0001:00032370       ?SetProtectState@CMainFrame@@QAEXHHH@Z 00433370 f   MainFrm.obj
 0001:000324d0       ?OnRecvC@CMainFrame@@QAEJIJ@Z 004334d0 f   MainFrm.obj
 0001:000325d0       ?InitListCtrlDisplay@CMainFrame@@QAEXXZ 004335d0 f   MainFrm.obj
 0001:00032ef0       ?SortTree@CMainFrame@@QAEXXZ 00433ef0 f   MainFrm.obj
 0001:00032f30       ?OnShutdown@CMainFrame@@QAEXXZ 00433f30 f   MainFrm.obj
 0001:00033540       ?OnRestart@CMainFrame@@QAEXXZ 00434540 f   MainFrm.obj
 0001:00033b60       ?OnWol@CMainFrame@@QAEXXZ  00434b60 f   MainFrm.obj
 0001:00034550       ?OnLockmonitor@CMainFrame@@QAEXXZ 00435550 f   MainFrm.obj
 0001:00034af0       ?OnUnlockmonitor@CMainFrame@@QAEXXZ 00435af0 f   MainFrm.obj
 0001:00035090       ?OnLockusb@CMainFrame@@QAEXXZ 00436090 f   MainFrm.obj
 0001:00035640       ?OnUnlockusb@CMainFrame@@QAEXXZ 00436640 f   MainFrm.obj
 0001:00035bf0       ?OnScanclient@CMainFrame@@QAEXXZ 00436bf0 f   MainFrm.obj
 0001:00035d40       ?_RefreshThread@CMainFrame@@SAIPAX@Z 00436d40 f   MainFrm.obj
 0001:00036390       ?OnSupervise@CMainFrame@@QAEXXZ 00437390 f   MainFrm.obj
 0001:00037270       ?OnRemotectrl@CMainFrame@@QAEXXZ 00438270 f   MainFrm.obj
 0001:00038160       ?OnQuicksave@CMainFrame@@QAEXXZ 00439160 f   MainFrm.obj
 0001:00038730       ?OnQuickrecovery@CMainFrame@@QAEXXZ 00439730 f   MainFrm.obj
 0001:00038d00       ?OnStarttrans@CMainFrame@@QAEXXZ 00439d00 f   MainFrm.obj
 0001:00039320       ?AddLogRecord@CMainFrame@@QAEHV?$CStringT@DV?$StrTraitMFC_DLL@DV?$ChTraitsCRT@D@ATL@@@@@ATL@@000I0@Z 0043a320 f   MainFrm.obj
 0001:00039440       ?OnClientsettings@CMainFrame@@QAEXXZ 0043a440 f   MainFrm.obj
 0001:00039690       ?_GetBootModuleInfoThread@CMainFrame@@SAIPAX@Z 0043a690 f   MainFrm.obj
 0001:00039ae0       ?HandleBootModuleInfoPacket@CMainFrame@@QAEXPAUPartitionTransInfo@@K@Z 0043aae0 f   MainFrm.obj
 0001:00039e60       ?HandlePortInfoPacket@CMainFrame@@QAEXPAUPortInfo@@K@Z 0043ae60 f   MainFrm.obj
 0001:00039ed0       ?_WaitAllThreadExited@CMainFrame@@SAIPAX@Z 0043aed0 f   MainFrm.obj
 0001:0003a390       ?OnSendmsg@CMainFrame@@QAEXXZ 0043b390 f   MainFrm.obj
 0001:0003a990       ?OnIpsettings@CMainFrame@@QAEXXZ 0043b990 f   MainFrm.obj
 0001:0003b240       ?GetHostBasicIPInfo@CMainFrame@@QAEHAAUstruct_ipsetting_param@@@Z 0043c240 f   MainFrm.obj
 0001:0003c3d0       ?OnScanproperty@CMainFrame@@QAEXXZ 0043d3d0 f   MainFrm.obj
 0001:0003c5f0       ?_PropertyCheckThread@CMainFrame@@SAIPAX@Z 0043d5f0 f   MainFrm.obj
 0001:0003cc10       ?OnUpdateproperty@CMainFrame@@QAEXXZ 0043dc10 f   MainFrm.obj
 0001:0003cfb0       ?_PropertyUpdateThread@CMainFrame@@SAIPAX@Z 0043dfb0 f   MainFrm.obj
 0001:0003d150       ?UpdateOnePropertyInfoInDatabase@CMainFrame@@QAEHV?$CStringT@DV?$StrTraitMFC_DLL@DV?$ChTraitsCRT@D@ATL@@@@@ATL@@@Z 0043e150 f   MainFrm.obj
 0001:0003e690       ?GetCount@CMapStringToPtr@@QBEHXZ 0043f690 f i KiboManagerView.obj
 0001:0003e690       ?GetCount@CStringList@@QBEHXZ 0043f690 f i AddToGroup.obj
 0001:0003e690       ?GetCount@CMapStringToString@@QBEHXZ 0043f690 f i LenPropertyODBC.obj
 0001:0003e690       ?GetCount@CPtrList@@QBEHXZ 0043f690 f i MainFrm.obj
 0001:0003e6b0       ?OnStyle@CMainFrame@@QAEXXZ 0043f6b0 f   MainFrm.obj
 0001:0003e7c0       ?OnDellist@CMainFrame@@QAEXXZ 0043f7c0 f   MainFrm.obj
 0001:0003ed80       ?OnBlacklist@CMainFrame@@QAEXXZ 0043fd80 f   MainFrm.obj
 0001:0003edf0       ?OnPropertychangeLog@CMainFrame@@QAEXXZ 0043fdf0 f   MainFrm.obj
 0001:0003ee00       ?HandlePropertyInfoPacket@CMainFrame@@QAEXPAUPropertyInfo@@HK@Z 0043fe00 f   MainFrm.obj
 0001:000413d0       ?OnSetStatuBarText@CMainFrame@@QAEHH@Z 004423d0 f   MainFrm.obj
 0001:00041600       ?UpdateGroupDisplay@CMainFrame@@QAEXV?$CStringT@DV?$StrTraitMFC_DLL@DV?$ChTraitsCRT@D@ATL@@@@@ATL@@H@Z 00442600 f   MainFrm.obj
 0001:000419c0       ?DisplayGroup@CMainFrame@@QAEXXZ 004429c0 f   MainFrm.obj
 0001:00041af0       ?DisplayAllClient@CMainFrame@@QAEXXZ 00442af0 f   MainFrm.obj
 0001:00042320       ?DisplayGroupClient@CMainFrame@@QAEXV?$CStringT@DV?$StrTraitMFC_DLL@DV?$ChTraitsCRT@D@ATL@@@@@ATL@@@Z 00443320 f   MainFrm.obj
 0001:00042c80       ?InitializeBackupPanel@CMainFrame@@QAEXXZ 00443c80 f   MainFrm.obj
 0001:00043780       ?InitializeRegisterPanel@CMainFrame@@QAEXXZ 00444780 f   MainFrm.obj
 0001:000439f0       ?InitializePropertyPanel@CMainFrame@@QAEXXZ 004449f0 f   MainFrm.obj
 0001:00043d50       ?InitializeRemoteCtrlPanel@CMainFrame@@QAEXXZ 00444d50 f   MainFrm.obj
 0001:00044ef0       ?InitializeAppPanel@CMainFrame@@QAEXXZ 00445ef0 f   MainFrm.obj
 0001:00045660       ?InitializeOwnPanel@CMainFrame@@QAEXXZ 00446660 f   MainFrm.obj
 0001:000459c0       ?OnClose@CMainFrame@@QAEXXZ 004469c0 f   MainFrm.obj
 0001:00045a60       ?WindowProc@CMainFrame@@MAEJIIJ@Z 00446a60 f   MainFrm.obj
 0001:00045b10       ?CleanUpBefClose@CMainFrame@@QAEXXZ 00446b10 f   MainFrm.obj
 0001:00045b80       ?OnOnePropertyRefreshFinished@CMainFrame@@QAEJIJ@Z 00446b80 f   MainFrm.obj
 0001:00045c00       ?OnProgressDlgClosed@CMainFrame@@QAEJIJ@Z 00446c00 f   MainFrm.obj
 0001:00047610       ?OnProgressDlgCanceled@CMainFrame@@QAEJIJ@Z 00448610 f   MainFrm.obj
 0001:000476f0       ?OnSysCommand@CMainFrame@@QAEXIJ@Z 004486f0 f   MainFrm.obj
 0001:000477d0       ?OnMyMsg@CMainFrame@@QAEJIJ@Z 004487d0 f   MainFrm.obj
 0001:000479f0       ?PreTranslateMessage@CMainFrame@@UAEHPAUtagMSG@@@Z 004489f0 f   MainFrm.obj
 0001:00047a70       ?OnTrayBackup@CMainFrame@@QAEXXZ 00448a70 f   MainFrm.obj
 0001:000481e0       ?DriverExist@CMainFrame@@QAEHXZ 004491e0 f   MainFrm.obj
 0001:00048480       ?OnTrayRecovery@CMainFrame@@QAEXXZ 00449480 f   MainFrm.obj
 0001:00048b80       ?OnTrayModifygroup@CMainFrame@@QAEXXZ 00449b80 f   MainFrm.obj
 0001:00048df0       ??1CModifyGroup@@UAE@XZ    00449df0 f i MainFrm.obj
 0001:00048e60       ?GetServerGroup@CMainFrame@@IAEHXZ 00449e60 f   MainFrm.obj
 0001:00049200       ?SetServerGroup@CMainFrame@@IAEHXZ 0044a200 f   MainFrm.obj
 0001:00049320       ?DisplayMsg@CMainFrame@@QAEXPAXHH@Z 0044a320 f   MainFrm.obj
 0001:00049a40       ?OnLockmouse@CMainFrame@@QAEXXZ 0044aa40 f   MainFrm.obj
 0001:00049ed0       ?OnUnlockmouse@CMainFrame@@QAEXXZ 0044aed0 f   MainFrm.obj
 0001:0004a360       ?OnLockkeyboard@CMainFrame@@QAEXXZ 0044b360 f   MainFrm.obj
 0001:0004a8a0       ?OnUnlockkeyboard@CMainFrame@@QAEXXZ 0044b8a0 f   MainFrm.obj
 0001:0004ade0       ?OnSynTime@CMainFrame@@QAEXXZ 0044bde0 f   MainFrm.obj
 0001:0004b500       ?OnGroupmsg@CMainFrame@@QAEXXZ 0044c500 f   MainFrm.obj
 0001:0004b540       ?OnUpdateGroupmsg@CMainFrame@@QAEXPAVCCmdUI@@@Z 0044c540 f   MainFrm.obj
 0001:0004b580       ?SetDefaultCategory@CMainFrame@@QAEHH@Z 0044c580 f   MainFrm.obj
 0001:0004b5c0       ?OnViewMaindlg@CMainFrame@@QAEXXZ 0044c5c0 f   MainFrm.obj
 0001:0004b6e0       ?OnUpdateViewMaindlg@CMainFrame@@QAEXPAVCCmdUI@@@Z 0044c6e0 f   MainFrm.obj
 0001:0004b720       ?OnTransfile@CMainFrame@@QAEXXZ 0044c720 f   MainFrm.obj
 0001:0004bd70       ?HandleRemoteControlCmd@CMainFrame@@QAEXPAUtagRECVREQUEST@@@Z 0044cd70 f   MainFrm.obj
 0001:0004c310       ?OnPortLock@CMainFrame@@QAEXXZ 0044d310 f   MainFrm.obj
 0001:0004c6d0       ?OnSaveHistorymsg@CMainFrame@@QAEXXZ 0044d6d0 f   MainFrm.obj
 0001:0004c7f0       ?OnUpdateSaveHistorymsg@CMainFrame@@QAEXPAVCCmdUI@@@Z 0044d7f0 f   MainFrm.obj
 0001:0004c830       ?_GetPortInfoThread@CMainFrame@@SAIPAX@Z 0044d830 f   MainFrm.obj
 0001:0004cc30       ?AddRemoveTray@CMainFrame@@QAEHH@Z 0044dc30 f   MainFrm.obj
 0001:0004d0e0       ?OnWM_NOTIFYICON@CMainFrame@@QAEJIJ@Z 0044e0e0 f   MainFrm.obj
 0001:0004d170       ?DisplayMenu@CMainFrame@@QAEXXZ 0044e170 f   MainFrm.obj
 0001:0004d330       ?OnTrayShow@CMainFrame@@QAEXXZ 0044e330 f   MainFrm.obj
 0001:0004d360       ?OnTrayMinimize@CMainFrame@@QAEXXZ 0044e360 f   MainFrm.obj
 0001:0004d390       ?OnTrayExit@CMainFrame@@QAEXXZ 0044e390 f   MainFrm.obj
 0001:0004d3b0       ?OnAppAbout@CMainFrame@@QAEXXZ 0044e3b0 f   MainFrm.obj
 0001:0004d420       ?OnHelp@CMainFrame@@QAEXXZ 0044e420 f   MainFrm.obj
 0001:0004d4f0       ?OnSelallcomputer@CMainFrame@@QAEXXZ 0044e4f0 f   MainFrm.obj
 0001:0004d5c0       ?OnUpdateSelallcomputer@CMainFrame@@QAEXPAVCCmdUI@@@Z 0044e5c0 f   MainFrm.obj
 0001:0004d600       ?OnBroadclass@CMainFrame@@QAEXXZ 0044e600 f   MainFrm.obj
 0001:0004e4e0       ?InitializeBroadClass@CMainFrame@@QAEXXZ 0044f4e0 f   MainFrm.obj
 0001:0004ec20       ?OnStopbroadclass@CMainFrame@@QAEXXZ 0044fc20 f   MainFrm.obj
 0001:0004f0b0       ?OnStudentdemo@CMainFrame@@QAEXXZ 004500b0 f   MainFrm.obj
 0001:00050280       ?OnStopstudentdemo@CMainFrame@@QAEXXZ 00451280 f   MainFrm.obj
 0001:00050590       ?OnUpdateBroadclass@CMainFrame@@QAEXPAVCCmdUI@@@Z 00451590 f   MainFrm.obj
 0001:00050690       ?OnUpdateStudentdemo@CMainFrame@@QAEXPAVCCmdUI@@@Z 00451690 f   MainFrm.obj
 0001:00050790       ?OnExammode@CMainFrame@@QAEXXZ 00451790 f   MainFrm.obj
 0001:00050be0       ?OnNetvideo@CMainFrame@@QAEXXZ 00451be0 f   MainFrm.obj
 0001:00051250       ?OnMenuRemovehand@CMainFrame@@QAEXXZ 00452250 f   MainFrm.obj
 0001:00051580       ?OnBroadIE@CMainFrame@@QAEXXZ 00452580 f   MainFrm.obj
 0001:00051ab0       ?InitFtpServer@CMainFrame@@QAE_NV?$CStringT@DV?$StrTraitMFC_DLL@DV?$ChTraitsCRT@D@ATL@@@@@ATL@@00I@Z 00452ab0 f   MainFrm.obj
 0001:00051e30       ?OnServersetting@CMainFrame@@QAEXXZ 00452e30 f   MainFrm.obj
 0001:00051ec0       ?InitializeCommonPanel@CMainFrame@@QAEXXZ 00452ec0 f   MainFrm.obj
 0001:000522f0       ?OnProtectmode@CMainFrame@@QAEXXZ 004532f0 f   MainFrm.obj
 0001:00052730       ?OnOpenmode@CMainFrame@@QAEXXZ 00453730 f   MainFrm.obj
 0001:00052b70       ?OnMessageUnlock@CMainFrame@@QAEXXZ 00453b70 f   MainFrm.obj
 0001:00052bb0       ?_CallRegisterProcess@CMainFrame@@SAIPAX@Z 00453bb0 f   MainFrm.obj
 0001:00052e50       ?OnRegister@CMainFrame@@QAEXXZ 00453e50 f   MainFrm.obj
 0001:00052ee0       ?CheckGroupRegister@CMainFrame@@QAEHV?$CStringT@DV?$StrTraitMFC_DLL@DV?$ChTraitsCRT@D@ATL@@@@@ATL@@AAH1@Z 00453ee0 f   MainFrm.obj
 0001:000530a0       ?OnViewproperty@CMainFrame@@QAEXXZ 004540a0 f   MainFrm.obj
 0001:000530c0       ?GetMessageMap@COutlookBar@@MBEPBUAFX_MSGMAP@@XZ 004540c0 f   MainFrm.obj
 0001:000530d0       ?GetThisMessageMap@COutlookBar@@KGPBUAFX_MSGMAP@@XZ 004540d0 f   MainFrm.obj
 0001:000530e0       ?OnRButtonDown@CWorkspaceBar@@QAEXIVCPoint@@@Z 004540e0 f   WorkspaceBar.obj
 0001:000530e0       ?OnRButtonDown@COutlookBar@@IAEXIVCPoint@@@Z 004540e0 f   MainFrm.obj
 0001:000530e0       ?OnRButtonDown@CWorkspaceBar2@@QAEXIVCPoint@@@Z 004540e0 f   WorkspaceBar2.obj
 0001:00053110       ?OnSetPort@CMainFrame@@QAEXXZ 00454110 f   MainFrm.obj
 0001:00053290       ?InitPortAndCode@CMainFrame@@QAEXXZ 00454290 f   MainFrm.obj
 0001:000533e0       ?OnSetclientPort@CMainFrame@@QAEXXZ 004543e0 f   MainFrm.obj
 0001:00053970       ?ModifyTrayTip@CMainFrame@@QAEXXZ 00454970 f   MainFrm.obj
 0001:000539e0       ?OnNetworkSet@CMainFrame@@QAEXXZ 004549e0 f   MainFrm.obj
 0001:00053a60       ?ShowBalloonTip@CMainFrame@@QAEHPBD0K@Z 00454a60 f   MainFrm.obj
 0001:00053af0       ?ReInitNetwrokComponent@CMainFrame@@QAEXXZ 00454af0 f   MainFrm.obj
 0001:00053db0       ?CheckGUID@CMainFrame@@QAEHPADH0@Z 00454db0 f   MainFrm.obj
 0001:00054430       ?OnSpecialRecovery@CMainFrame@@QAEXXZ 00455430 f   MainFrm.obj
 0001:000546a0       ?OnSpecialSave@CMainFrame@@QAEXXZ 004556a0 f   MainFrm.obj
 0001:00054910       ?OnDisablecdrom@CMainFrame@@QAEHI@Z 00455910 f   MainFrm.obj
 0001:00054e20       ?OnRegisterLocal@CMainFrame@@QAEXXZ 00455e20 f   MainFrm.obj
 0001:00054e90       ?OnGroupset@CMainFrame@@QAEXXZ 00455e90 f   MainFrm.obj
 0001:00055270       ?OnRemoteRunprocedure@CMainFrame@@QAEXXZ 00456270 f   MainFrm.obj
 0001:00055890       ??9ATL@@YA_NPBDABV?$CStringT@DV?$StrTraitMFC_DLL@DV?$ChTraitsCRT@D@ATL@@@@@0@@Z 00456890 f i MainFrm.obj
 0001:000558b0       ?RemoveHead@?$_CTypedPtrList@VCPtrList@@PAUtagUDPRECV@@@@QAEPAUtagUDPRECV@@XZ 004568b0 f i MainFrm.obj
 0001:000558b0       ?RemoveHead@?$_CTypedPtrList@VCPtrList@@PAUtagRECVREQUEST@@@@QAEPAUtagRECVREQUEST@@XZ 004568b0 f i MainFrm.obj
 0001:000558d0       ??0?$CTypedPtrList@VCPtrList@@PAUtagRECVREQUEST@@@@QAE@H@Z 004568d0 f i MainFrm.obj
 0001:00055900       ?AddTail@?$CTypedPtrList@VCPtrList@@PAUtagRECVREQUEST@@@@QAEPAU__POSITION@@PAUtagRECVREQUEST@@@Z 00456900 f i MainFrm.obj
 0001:00055900       ?AddTail@?$CTypedPtrList@VCPtrList@@PAUPartitionTransInfo@@@@QAEPAU__POSITION@@PAUPartitionTransInfo@@@Z 00456900 f i MainFrm.obj
 0001:00055920       ??0?$CTypedPtrList@VCPtrList@@PAUPartitionTransInfo@@@@QAE@H@Z 00456920 f i MainFrm.obj
 0001:00055950       ??0?$CTypedPtrMap@VCMapStringToPtr@@V?$CStringT@DV?$StrTraitMFC_DLL@DV?$ChTraitsCRT@D@ATL@@@@@ATL@@PAV23@@@QAE@H@Z 00456950 f i MainFrm.obj
 0001:00055980       ??_G?$CTypedPtrMap@VCMapStringToPtr@@V?$CStringT@DV?$StrTraitMFC_DLL@DV?$ChTraitsCRT@D@ATL@@@@@ATL@@PAV23@@@UAEPAXI@Z 00456980 f i MainFrm.obj
 0001:00055980       ??_E?$CTypedPtrMap@VCMapStringToPtr@@V?$CStringT@DV?$StrTraitMFC_DLL@DV?$ChTraitsCRT@D@ATL@@@@@ATL@@PAUtagBLACKLIST@@@@UAEPAXI@Z 00456980 f i ClientInfoManager.obj
 0001:00055980       ??_E?$CTypedPtrMap@VCMapStringToPtr@@V?$CStringT@DV?$StrTraitMFC_DLL@DV?$ChTraitsCRT@D@ATL@@@@@ATL@@PAV23@@@UAEPAXI@Z 00456980 f i MainFrm.obj
 0001:00055980       ??_E?$CTypedPtrMap@VCMapStringToPtr@@V?$CStringT@DV?$StrTraitMFC_DLL@DV?$ChTraitsCRT@D@ATL@@@@@ATL@@PAVCStringList@@@@UAEPAXI@Z 00456980 f i ClientInfoManager.obj
 0001:00055980       ??_G?$CTypedPtrMap@VCMapStringToPtr@@V?$CStringT@DV?$StrTraitMFC_DLL@DV?$ChTraitsCRT@D@ATL@@@@@ATL@@PAVCStringList@@@@UAEPAXI@Z 00456980 f i ClientInfoManager.obj
 0001:00055980       ??_G?$CTypedPtrMap@VCMapStringToPtr@@V?$CStringT@DV?$StrTraitMFC_DLL@DV?$ChTraitsCRT@D@ATL@@@@@ATL@@PAUtagCLIENTMAININFO@@@@UAEPAXI@Z 00456980 f i ClientInfoManager.obj
 0001:00055980       ??_G?$CTypedPtrMap@VCMapStringToPtr@@V?$CStringT@DV?$StrTraitMFC_DLL@DV?$ChTraitsCRT@D@ATL@@@@@ATL@@PAUtagBLACKLIST@@@@UAEPAXI@Z 00456980 f i ClientInfoManager.obj
 0001:00055980       ??_E?$CTypedPtrMap@VCMapStringToPtr@@V?$CStringT@DV?$StrTraitMFC_DLL@DV?$ChTraitsCRT@D@ATL@@@@@ATL@@PAUtagCLIENTMAININFO@@@@UAEPAXI@Z 00456980 f i ClientInfoManager.obj
 0001:000559b0       ??0?$_CTypedPtrList@VCPtrList@@PAUtagRECVREQUEST@@@@QAE@H@Z 004569b0 f i MainFrm.obj
 0001:000559e0       ??0?$_CTypedPtrList@VCPtrList@@PAUPartitionTransInfo@@@@QAE@H@Z 004569e0 f i MainFrm.obj
 0001:00055a10       ??0?$CList@II@@QAE@H@Z     00456a10 f i MainFrm.obj
 0001:00055a70       ?AfxGetInstanceHandle@@YGPAUHINSTANCE__@@XZ 00456a70 f i MainFrm.obj
 0001:00055a80       ?AfxGetResourceHandle@@YGPAUHINSTANCE__@@XZ 00456a80 f i MainFrm.obj
 0001:00055a90       ??$strcpy_s@$0FA@@@YAHAAY0FA@DPBD@Z 00456a90 f i MainFrm.obj
 0001:00055ab0       ?AfxSetResourceHandle@@YGXPAUHINSTANCE__@@@Z 00456ab0 f i MainFrm.obj
 0001:00055ad0       ??$strcpy_s@$0BK@@@YAHAAY0BK@DPBD@Z 00456ad0 f i MainFrm.obj
 0001:00055af0       ??$strcpy_s@$08@@YAHAAY08DPBD@Z 00456af0 f i MainFrm.obj
 0001:00055b10       ??$strcat_s@$0BAE@@@YAHAAY0BAE@DPBD@Z 00456b10 f i MainFrm.obj
 0001:00055b30       ??$strcpy_s@$0BA@@@YAHAAY0BA@DPBD@Z 00456b30 f i MainFrm.obj
 0001:00055b50       ??0?$CList@PAVCFtpd@@PAV1@@@QAE@H@Z 00456b50 f i MainFrm.obj
 0001:00055bb0       ??1?$CList@PAVCFtpd@@PAV1@@@UAE@XZ 00456bb0 f i MainFrm.obj
 0001:00055c10       ??$strcpy_s@$0EA@@@YAHAAY0EA@DPBD@Z 00456c10 f i MainFrm.obj
 0001:00055c30       ??_G?$CList@PAVCFtpd@@PAV1@@@UAEPAXI@Z 00456c30 f i MainFrm.obj
 0001:00055c30       ??_E?$CList@PAVCFtpd@@PAV1@@@UAEPAXI@Z 00456c30 f i MainFrm.obj
 0001:00055c60       ?SetFont@CWnd@@QAEXPAVCFont@@H@Z 00456c60 f i MainFrm.obj
 0001:00055c90       ?InvalidateRect@CWnd@@QAEXPBUtagRECT@@H@Z 00456c90 f i MainFrm.obj
 0001:00055cc0       ?RedrawWindow@CWnd@@QAEHPBUtagRECT@@PAVCRgn@@I@Z 00456cc0 f i MainFrm.obj
 0001:00055cf0       ?FindWindowA@CWnd@@SGPAV1@PBD0@Z 00456cf0 f i MainFrm.obj
 0001:00055d10       ?SetForegroundWindow@CWnd@@QAEHXZ 00456d10 f i MainFrm.obj
 0001:00055d30       ??0CWaitCursor@@QAE@XZ     00456d30 f i MainFrm.obj
 0001:00055d50       ?AfxGetApp@@YGPAVCWinApp@@XZ 00456d50 f i MainFrm.obj
 0001:00055d60       ??1CWaitCursor@@QAE@XZ     00456d60 f i MainFrm.obj
 0001:00055ef0       ?GetNextVisibleItem@CTreeCtrl@@QBEPAU_TREEITEM@@PAU2@@Z 00456ef0 f i MainFrm.obj
 0001:00055f20       ?SortChildrenCB@CTreeCtrl@@QAEHPAUtagTVSORTCB@@@Z 00456f20 f i MainFrm.obj
 0001:00055f50       ?ReplaceSel@CRichEditCtrl@@QAEXPBDH@Z 00456f50 f i MainFrm.obj
 0001:00055f80       ?SetImageSize@CMFCToolBarImages@@QAEXUtagSIZE@@H@Z 00456f80 f i MainFrm.obj
 0001:00055fc0       ??0CSize@@QAE@UtagSIZE@@@Z 00456fc0 f i MainFrm.obj
 0001:00055fe0       ?SetTransparentColor@CMFCToolBarImages@@QAEKK@Z 00456fe0 f i MainFrm.obj
 0001:00056030       ?IsFloating@CBasePane@@UBEHXZ 00457030 f i MainFrm.obj
 0001:00056060       ?IsHighlighted@CMFCRibbonBaseElement@@UBEHXZ 00457060 f i MainFrm.obj
 0001:00056060       ?GetEnabledAlignment@CBasePane@@UBEKXZ 00457060 f i MainFrm.obj
 0001:00056080       ?GetParentDockSite@CBasePane@@UBEPAVCDockSite@@XZ 00457080 f i MainFrm.obj
 0001:000560a0       ?GetRecentVisibleState@CBasePane@@UBEHXZ 004570a0 f i MainFrm.obj
 0001:000560c0       ?IsRestoredFromRegistry@CBasePane@@UBEHXZ 004570c0 f i MainFrm.obj
 0001:000560e0       ?SetRestoredFromRegistry@CBasePane@@UAEXH@Z 004570e0 f i MainFrm.obj
 0001:00056100       ?IsFocused@CMFCRibbonBaseElement@@UBEHXZ 00457100 f i MainFrm.obj
 0001:00056100       ?GetPaneStyle@CBasePane@@UBEKXZ 00457100 f i MainFrm.obj
 0001:00056120       ?IsPressed@CMFCRibbonBaseElement@@UBEHXZ 00457120 f i MainFrm.obj
 0001:00056120       ?GetControlBarStyle@CBasePane@@UBEKXZ 00457120 f i MainFrm.obj
 0001:00056140       ?CanBeClosed@CBasePane@@UBEHXZ 00457140 f i MainFrm.obj
 0001:00056160       ?CanBeResized@CBasePane@@UBEHXZ 00457160 f i MainFrm.obj
 0001:00056180       ?SetPaneAlignment@CBasePane@@UAEXK@Z 00457180 f i MainFrm.obj
 0001:000561b0       ?SetPaneStyle@CBasePane@@UAEXK@Z 004571b0 f i MainFrm.obj
 0001:000561d0       ?SetControlBarStyle@CBasePane@@UAEXK@Z 004571d0 f i MainFrm.obj
 0001:000561f0       ?EnableDocking@CBasePane@@UAEXK@Z 004571f0 f i MainFrm.obj
 0001:00056210       ?StretchPane@CBasePane@@UAE?AVCSize@@HH@Z 00457210 f i MainFrm.obj
 0001:00056230       ?IsHorizontal@CBasePane@@UBEHXZ 00457230 f i MainFrm.obj
 0001:00056250       ?IsDragMode@CPane@@UBEHXZ  00457250 f i MainFrm.obj
 0001:00056270       ?GetMinLength@CPane@@UBEHXZ 00457270 f i MainFrm.obj
 0001:000562a0       ?GetResizeStep@CPane@@UBEHXZ 004572a0 f i MainFrm.obj
 0001:000562b0       ?DoesAllowSiblingBars@CPane@@UBEHXZ 004572b0 f i MainFrm.obj
 0001:000562d0       ?SetExclusiveRowMode@CPane@@UAEXH@Z 004572d0 f i MainFrm.obj
 0001:000562f0       ?GetExclusiveRowMode@CPane@@UBEHXZ 004572f0 f i MainFrm.obj
 0001:00056310       ?CalcSize@CPane@@UAE?AVCSize@@H@Z 00457310 f i MainFrm.obj
 0001:00056330       ?CanBeDocked@CPane@@UBEHPAVCBasePane@@@Z 00457330 f i MainFrm.obj
 0001:00056370       ?IsAutoHideMode@CDockablePane@@UBEHXZ 00457370 f i MainFrm.obj
 0001:00056390       ?IsAutohideAllEnabled@CDockablePane@@UBEHXZ 00457390 f i MainFrm.obj
 0001:000563b0       ?OnAfterDockFromMiniFrame@CDockablePane@@UAEXXZ 004573b0 f i MainFrm.obj
 0001:000563e0       ?DockToRecentPos@CDockablePane@@UAEHXZ 004573e0 f i MainFrm.obj
 0001:00056410       ?IsHideInAutoHideMode@CDockablePane@@UBEHXZ 00457410 f i MainFrm.obj
 0001:00056430       ?CanAdjustLayout@CDockablePane@@UBEHXZ 00457430 f i MainFrm.obj
 0001:00056470       ?GetAHSlideMode@CDockablePane@@UBEIXZ 00457470 f i MainFrm.obj
 0001:00056490       ?GetUnderlyingWindow@CBaseTabbedPane@@UAEPAVCMFCBaseTabCtrl@@XZ 00457490 f i MainFrm.obj
 0001:000564b0       ?GetTabsNum@CBaseTabbedPane@@UBEHXZ 004574b0 f i MainFrm.obj
 0001:000564f0       ?GetVisibleTabsNum@CBaseTabbedPane@@UBEHXZ 004574f0 f i MainFrm.obj
 0001:00056530       ?IsHideSingleTab@CBaseTabbedPane@@UBEHXZ 00457530 f i MainFrm.obj
 0001:00056570       ?EnableSetCaptionTextToTabName@CBaseTabbedPane@@UAEXH@Z 00457570 f i MainFrm.obj
 0001:00056590       ?OnConnectionClosing@CMyIOCP@@UAEXPAVCClientContext@@@Z 00457590 f i MyIOCP.obj
 0001:00056590       ?OnActivateTab@CBaseTabbedPane@@MAEXH@Z 00457590 f i MainFrm.obj
 0001:00056590       ?OnRTLChanged@CMFCRibbonBaseElement@@UAEXH@Z 00457590 f i MainFrm.obj
 0001:00056590       ?OnScroll@CMFCOutlookBar@@UAEXH@Z 00457590 f i MainFrm.obj
 0001:00056590       ?OnSetFocus@CMFCRibbonBaseElement@@MAEXH@Z 00457590 f i MainFrm.obj
 0001:00056590       ?OnMovePaneDivider@CBasePane@@UAEXPAVCPaneDivider@@@Z 00457590 f i MainFrm.obj
 0001:00056590       ?Serialize@CObject@@UAEXAAVCArchive@@@Z 00457590 f i AboutDlg.obj
 0001:00056590       ?AccNotifyObjectFocusEvent@CBasePane@@UAEXH@Z 00457590 f i MainFrm.obj
 0001:00056590       ?OnDraw@CKiboManagerView@@MAEXPAVCDC@@@Z 00457590 f i KiboManagerView.obj
 0001:00056590       ?OnAfterStretch@CPane@@MAEXH@Z 00457590 f i MainFrm.obj
 0001:00056590       ?OnRemoveFromMiniFrame@CBasePane@@UAEXPAVCPaneFrameWnd@@@Z 00457590 f i MainFrm.obj
 0001:00056590       ?OnHighlight@CMFCRibbonBaseElement@@MAEXH@Z 00457590 f i MainFrm.obj
 0001:00056590       ?OnAfterAnimation@CMFCOutlookBar@@UAEXH@Z 00457590 f i MainFrm.obj
 0001:00056590       ?OnPressButtons@CDockablePane@@MAEXI@Z 00457590 f i MainFrm.obj
 0001:00056590       ?OnCheck@CMFCRibbonBaseElement@@MAEXH@Z 00457590 f i MainFrm.obj
 0001:00056590       ?OnConnectionEstablished@CMyIOCP@@UAEXPAVCClientContext@@@Z 00457590 f i MyIOCP.obj
 0001:00056590       ?DoDataExchange@CWnd@@MAEXPAVCDataExchange@@@Z 00457590 f i AboutDlg.obj
 0001:00056590       ?EnableGripper@CBasePane@@UAEXH@Z 00457590 f i MFCRibbonBarNew.obj
 0001:00056590       ?Dump@CObject@@UBEXAAVCDumpContext@@@Z 00457590 f i AboutDlg.obj
 0001:00056590       ?OnEnable@CMFCRibbonBaseElement@@MAEXH@Z 00457590 f i MainFrm.obj
 0001:00056590       ?OnShow@CMFCRibbonBaseElement@@UAEXH@Z 00457590 f i MainFrm.obj
 0001:00056590       ?OnBeforeStretch@CPane@@MAEXAAH@Z 00457590 f i MainFrm.obj
 0001:000565a0       ?DoesAllowDynInsertBefore@CBasePane@@UBEHXZ 004575a0 f i MFCRibbonBarNew.obj
 0001:000565a0       ?AllowDestroyEmptyTabbedPane@CMFCOutlookBar@@UBEHXZ 004575a0 f i MainFrm.obj
 0001:000565c0       ?CanSetCaptionTextToTabName@CMFCOutlookBar@@UBEHXZ 004575c0 f i MainFrm.obj
 0001:000565f0       ?CanSetCaptionTextToTabName@CBaseTabbedPane@@UBEHXZ 004575f0 f i MainFrm.obj
 0001:00056610       ??0CMFCRibbonApplicationButton@@QAE@XZ 00457610 f i MainFrm.obj
 0001:00056680       ?IsDisabled@CMFCRibbonBaseElement@@UBEHXZ 00457680 f i MainFrm.obj
 0001:000566a0       ?IsChecked@CMFCRibbonBaseElement@@UBEHXZ 004576a0 f i MainFrm.obj
 0001:000566c0       ?IsDroppedDown@CMFCRibbonBaseElement@@UBEHXZ 004576c0 f i MainFrm.obj
 0001:000566e0       ?SetCompactMode@CMFCRibbonBaseElement@@UAEXH@Z 004576e0 f i MainFrm.obj
 0001:000567a0       ?CanBeCompacted@CMFCRibbonBaseElement@@UBEHXZ 004577a0 f i MainFrm.obj
 0001:00056800       ?GetSize@CMFCRibbonBaseElement@@UAE?AVCSize@@PAVCDC@@@Z 00457800 f i MainFrm.obj
 0001:000568a0       ?SetInitialMode@CMFCRibbonBaseElement@@UAEXH@Z 004578a0 f i MainFrm.obj
 0001:00056950       ?IsShowGroupBorder@CMFCRibbonBar@@UBEHPAVCMFCRibbonButtonsGroup@@@Z 00457950 f i MFCRibbonBarNew.obj
 0001:00056950       ?IsAutoRepeatMode@CMFCRibbonBaseElement@@UBEHAAH@Z 00457950 f i MainFrm.obj
 0001:00056950       ?OnMenuKey@CMFCRibbonBaseElement@@UAEHI@Z 00457950 f i MainFrm.obj
 0001:00056950       ?OnProcessKey@CMFCRibbonBaseElement@@MAEHI@Z 00457950 f i MainFrm.obj
 0001:00056950       ?CanAcceptPane@CBasePane@@UBEHPBV1@@Z 00457950 f i MFCRibbonBarNew.obj
 0001:00056950       ?OnWorkspaceIdle@CWinAppEx@@UAEHPAVCWnd@@@Z 00457950 f i KiboManager.obj
 0001:00056960       ?OnDrawMenuImage@CMFCRibbonBaseElement@@UAEHPAVCDC@@VCRect@@@Z 00457960 f i MainFrm.obj
 0001:000569b0       ?HasMenu@CMFCRibbonButton@@UBEHXZ 004579b0 f i MainFrm.obj
 0001:000569f0       ?IsCommandAreaHighlighted@CMFCRibbonButton@@UBEHXZ 004579f0 f i MainFrm.obj
 0001:00056a30       ?IsMenuAreaHighlighted@CMFCRibbonButton@@UBEHXZ 00457a30 f i MainFrm.obj
 0001:00056a70       ?IsAlwaysDrawBorder@CMFCRibbonButton@@UBEHXZ 00457a70 f i MainFrm.obj
 0001:00056a90       ?IsAlwaysLargeImage@CMFCRibbonButton@@UBEHXZ 00457a90 f i MainFrm.obj
 0001:00056ae0       ?HasLargeMode@CMFCRibbonButton@@UBEHXZ 00457ae0 f i MainFrm.obj
 0001:00056b30       ??9CSize@@QBEHUtagSIZE@@@Z 00457b30 f i MainFrm.obj
 0001:00056b70       ?HasIntermediateMode@CMFCRibbonButton@@UBEHXZ 00457b70 f i MainFrm.obj
 0001:00056ba0       ?HasCompactMode@CMFCRibbonButton@@UBEHXZ 00457ba0 f i MainFrm.obj
 0001:00056bf0       ?CleanUpSizes@CMFCRibbonButton@@UAEXXZ 00457bf0 f i MainFrm.obj
 0001:00056c40       ?IsPopupDefaultMenuLook@CMFCRibbonButton@@UBEHXZ 00457c40 f i MainFrm.obj
 0001:00056c40       ?HasAutoHideMode@CDockablePane@@UBEHXZ 00457c40 f i OutputWnd.obj
 0001:00056c40       ?CanBeAttached@CDockablePane@@UBEHXZ 00457c40 f i MainFrm.obj
 0001:00056c40       ?IsAccessibilityCompatible@CBasePane@@UAEHXZ 00457c40 f i MFCRibbonBarNew.obj
 0001:00056c40       ?HideInPrintPreviewMode@CBasePane@@UBEHXZ 00457c40 f i MainFrm.obj
 0001:00056c40       ?CanFocus@CBasePane@@UBEHXZ 00457c40 f i MainFrm.obj
 0001:00056c40       ?AllowShowOnPaneMenu@CPane@@UBEHXZ 00457c40 f i OutputWnd.obj
 0001:00056c40       ?IsTabLocationBottom@CDockablePane@@UBEHXZ 00457c40 f i MainFrm.obj
 0001:00056c40       ?IsApplicationButton@CMFCRibbonApplicationButton@@MBEHXZ 00457c40 f i MainFrm.obj
 0001:00056c40       ?IsResizable@CDockablePane@@UBEHXZ 00457c40 f i MainFrm.obj
 0001:00056c40       ?AllowShowOnPaneMenu@COutlookBar@@EBEHXZ 00457c40 f i MainFrm.obj
 0001:00056c40       ?IsMainRibbonBar@CMFCRibbonBar@@UBEHXZ 00457c40 f i MFCRibbonBarNew.obj
 0001:00056c40       ?IsAlignByColumn@CMFCRibbonBaseElement@@UBEHXZ 00457c40 f i MainFrm.obj
 0001:00056c40       ?IsTabStop@CMFCRibbonBaseElement@@UBEHXZ 00457c40 f i MainFrm.obj
 0001:00056c50       ?GetTextOffset@CMFCRibbonButton@@MBEHXZ 00457c50 f i MainFrm.obj
 0001:00056c70       ?SetMargin@CMFCRibbonButton@@MAEXABVCSize@@@Z 00457c70 f i MainFrm.obj
 0001:00056ca0       ?AddToListBox@CMFCRibbonApplicationButton@@MAEHPAVCMFCRibbonCommandsListBox@@H@Z 00457ca0 f i MainFrm.obj
 0001:00056cb0       ?GetImageSize@CMFCRibbonApplicationButton@@MBE?AVCSize@@W4RibbonImageType@CMFCRibbonBaseElement@@@Z 00457cb0 f i MainFrm.obj
 0001:00056cf0       ?GetImageSize@CMFCToolBarImages@@QBE?AUtagSIZE@@H@Z 00457cf0 f i MainFrm.obj
 0001:00056d40       ?DrawImage@CMFCRibbonApplicationButton@@MAEXPAVCDC@@W4RibbonImageType@CMFCRibbonBaseElement@@VCRect@@@Z 00457d40 f i MainFrm.obj
 0001:00056dd0       ?SetACCData@CMFCRibbonApplicationButton@@MAEHPAVCWnd@@AAVCAccessibilityData@@@Z 00457dd0 f i MainFrm.obj
 0001:00056e10       ??_ECMFCRibbonApplicationButton@@UAEPAXI@Z 00457e10 f i MainFrm.obj
 0001:00056e10       ??_GCMFCRibbonApplicationButton@@UAEPAXI@Z 00457e10 f i MainFrm.obj
 0001:00056e40       ??1CMFCRibbonApplicationButton@@UAE@XZ 00457e40 f i MainFrm.obj
 0001:00056ea0       ?IsPrintPreviewValid@CDockingManager@@QBEHXZ 00457ea0 f i MainFrm.obj
 0001:00056ec0       ?GetDockingManager@CFrameWndEx@@QAEPAVCDockingManager@@XZ 00457ec0 f i MainFrm.obj
 0001:00056ee0       ?OnShowCustomizePane@CFrameWndEx@@UAEHPAVCMFCPopupMenu@@I@Z 00457ee0 f i MainFrm.obj
 0001:00056f10       ?OnMenuButtonToolHitTest@CFrameWndEx@@UAEHPAVCMFCToolBarButton@@PAUtagTOOLINFOA@@@Z 00457f10 f i MainFrm.obj
 0001:00056f10       ?OnWmHotKey@CWait@@IAEJIJ@Z 00457f10 f i Wait.obj
 0001:00056f10       ?GetToolbarButtonToolTipText@CFrameWndEx@@UAEHPAVCMFCToolBarButton@@AAV?$CStringT@DV?$StrTraitMFC_DLL@DV?$ChTraitsCRT@D@ATL@@@@@ATL@@@Z 00457f10 f i MainFrm.obj
 0001:00056f20       ?Listen@CAsyncSocket@@QAEHH@Z 00457f20 f i MainFrm.obj
 0001:00056f50       ?Create@CSocket@@QAEHIHPBD@Z 00457f50 f i MainFrm.obj
 0001:00056f80       ??1?$CList@II@@UAE@XZ      00457f80 f i MainFrm.obj
 0001:00056fe0       ?Serialize@?$CList@PAVCFtpdPi@@PAV1@@@UAEXAAVCArchive@@@Z 00457fe0 f i CFtpd.obj
 0001:00056fe0       ?Serialize@?$CList@PAVCFtpd@@PAV1@@@UAEXAAVCArchive@@@Z 00457fe0 f i MainFrm.obj
 0001:00056fe0       ?Serialize@?$CList@II@@UAEXAAVCArchive@@@Z 00457fe0 f i MainFrm.obj
 0001:00057090       ??_E?$CList@II@@UAEPAXI@Z  00458090 f i MainFrm.obj
 0001:00057090       ??_G?$CList@II@@UAEPAXI@Z  00458090 f i MainFrm.obj
 0001:000570c0       ?AddTail@?$CList@PAVCFtpd@@PAV1@@@QAEPAU__POSITION@@PAVCFtpd@@@Z 004580c0 f i MainFrm.obj
 0001:000570c0       ?AddTail@?$CList@II@@QAEPAU__POSITION@@I@Z 004580c0 f i MainFrm.obj
 0001:000570c0       ?AddTail@?$CList@PAVCFtpdPi@@PAV1@@@QAEPAU__POSITION@@PAVCFtpdPi@@@Z 004580c0 f i CFtpd.obj
 0001:00057120       ??$SerializeElements@PAVCFtpd@@@@YGXAAVCArchive@@PAPAVCFtpd@@H@Z 00458120 f i MainFrm.obj
 0001:00057120       ??$SerializeElements@H@@YGXAAVCArchive@@PAHH@Z 00458120 f i ReportCtrl.obj
 0001:00057120       ??$SerializeElements@I@@YGXAAVCArchive@@PAIH@Z 00458120 f i MainFrm.obj
 0001:00057120       ??$SerializeElements@K@@YGXAAVCArchive@@PAKH@Z 00458120 f i ReportCtrl.obj
 0001:00057120       ??$SerializeElements@PAVCFtpdPi@@@@YGXAAVCArchive@@PAPAVCFtpdPi@@H@Z 00458120 f i CFtpd.obj
 0001:00057220       ?NewNode@?$CList@II@@IAEPAUCNode@1@PAU21@0@Z 00458220 f i MainFrm.obj
 0001:00057220       ?NewNode@?$CList@PAVCFtpd@@PAV1@@@IAEPAUCNode@1@PAU21@0@Z 00458220 f i MainFrm.obj
 0001:00057220       ?NewNode@?$CList@PAVCFtpdPi@@PAV1@@@IAEPAUCNode@1@PAU21@0@Z 00458220 f i CFtpd.obj
 0001:00057320       ??0?$CMap@V?$CStringT@DV?$StrTraitMFC_DLL@DV?$ChTraitsCRT@D@ATL@@@@@ATL@@PBDUItemInfo@@AAU3@@@QAE@H@Z 00458320 f i MainFrm.obj
 0001:00057380       ?Serialize@?$CMap@V?$CStringT@DV?$StrTraitMFC_DLL@DV?$ChTraitsCRT@D@ATL@@@@@ATL@@PBDUItemInfo@@AAU3@@@UAEXAAVCArchive@@@Z 00458380 f i MainFrm.obj
 0001:00057530       ??_G?$CMap@V?$CStringT@DV?$StrTraitMFC_DLL@DV?$ChTraitsCRT@D@ATL@@@@@ATL@@PBDUItemInfo@@AAU3@@@UAEPAXI@Z 00458530 f i MainFrm.obj
 0001:00057530       ??_E?$CMap@V?$CStringT@DV?$StrTraitMFC_DLL@DV?$ChTraitsCRT@D@ATL@@@@@ATL@@PBDUItemInfo@@AAU3@@@UAEPAXI@Z 00458530 f i MainFrm.obj
 0001:00057560       ??1?$CMap@V?$CStringT@DV?$StrTraitMFC_DLL@DV?$ChTraitsCRT@D@ATL@@@@@ATL@@PBDUItemInfo@@AAU3@@@UAE@XZ 00458560 f i MainFrm.obj
 0001:000575c0       ??0ItemInfo@@QAE@XZ        004585c0 f i MainFrm.obj
 0001:000575f0       ??1ItemInfo@@QAE@XZ        004585f0 f i MainFrm.obj
 0001:00057620       ?SetAt@?$CMap@V?$CStringT@DV?$StrTraitMFC_DLL@DV?$ChTraitsCRT@D@ATL@@@@@ATL@@PBDUItemInfo@@AAU3@@@QAEXPBDAAUItemInfo@@@Z 00458620 f i MainFrm.obj
 0001:00057650       ?RemoveAll@?$CMap@V?$CStringT@DV?$StrTraitMFC_DLL@DV?$ChTraitsCRT@D@ATL@@@@@ATL@@PBDUItemInfo@@AAU3@@@QAEXXZ 00458650 f i MainFrm.obj
 0001:00057700       ??$SerializeElements@UItemInfo@@@@YGXAAVCArchive@@PAUItemInfo@@H@Z 00458700 f i MainFrm.obj
 0001:00057800       ??4ItemInfo@@QAEAAU0@ABU0@@Z 00458800 f i MainFrm.obj
 0001:00057850       ??1CAssoc@?$CMap@V?$CStringT@DV?$StrTraitMFC_DLL@DV?$ChTraitsCRT@D@ATL@@@@@ATL@@PBDUItemInfo@@AAU3@@@QAE@XZ 00458850 f i MainFrm.obj
 0001:00057870       ??1CPair@?$CMap@V?$CStringT@DV?$StrTraitMFC_DLL@DV?$ChTraitsCRT@D@ATL@@@@@ATL@@PBDUItemInfo@@AAU3@@@QAE@XZ 00458870 f i MainFrm.obj
 0001:00057890       ??A?$CMap@V?$CStringT@DV?$StrTraitMFC_DLL@DV?$ChTraitsCRT@D@ATL@@@@@ATL@@PBDUItemInfo@@AAU3@@@QAEAAUItemInfo@@PBD@Z 00458890 f i MainFrm.obj
 0001:00057940       ?InitHashTable@?$CMap@V?$CStringT@DV?$StrTraitMFC_DLL@DV?$ChTraitsCRT@D@ATL@@@@@ATL@@PBDUItemInfo@@AAU3@@@QAEXIH@Z 00458940 f i MainFrm.obj
 0001:000579f0       ?NewAssoc@?$CMap@V?$CStringT@DV?$StrTraitMFC_DLL@DV?$ChTraitsCRT@D@ATL@@@@@ATL@@PBDUItemInfo@@AAU3@@@IAEPAVCAssoc@1@PBD@Z 004589f0 f i MainFrm.obj
 0001:00057b60       ?GetAssocAt@?$CMap@V?$CStringT@DV?$StrTraitMFC_DLL@DV?$ChTraitsCRT@D@ATL@@@@@ATL@@PBDUItemInfo@@AAU3@@@IBEPAVCAssoc@1@PBDAAI1@Z 00458b60 f i MainFrm.obj
 0001:00057bf0       ??0CAssoc@?$CMap@V?$CStringT@DV?$StrTraitMFC_DLL@DV?$ChTraitsCRT@D@ATL@@@@@ATL@@PBDUItemInfo@@AAU3@@@QAE@PBD@Z 00458bf0 f i MainFrm.obj
 0001:00057c10       ??0CPair@?$CMap@V?$CStringT@DV?$StrTraitMFC_DLL@DV?$ChTraitsCRT@D@ATL@@@@@ATL@@PBDUItemInfo@@AAU3@@@IAE@PBD@Z 00458c10 f i MainFrm.obj
 0001:00057c40       ??$CompareElements@V?$CStringT@DV?$StrTraitMFC_DLL@DV?$ChTraitsCRT@D@ATL@@@@@ATL@@PBD@@YGHPBV?$CStringT@DV?$StrTraitMFC_DLL@DV?$ChTraitsCRT@D@ATL@@@@@ATL@@PBQBD@Z 00458c40 f i MainFrm.obj
 0001:00057ca0       ?_GetBaseClass@CMFCRibbonBarNew@@KGPAUCRuntimeClass@@XZ 00458ca0 f   MFCRibbonBarNew.obj
 0001:00057cb0       ?GetRuntimeClass@CMFCRibbonBarNew@@UBEPAUCRuntimeClass@@XZ 00458cb0 f   MFCRibbonBarNew.obj
 0001:00057cc0       ??0CMFCRibbonBarNew@@QAE@XZ 00458cc0 f   MFCRibbonBarNew.obj
 0001:00057cf0       ??_ECMFCRibbonBarNew@@UAEPAXI@Z 00458cf0 f i MFCRibbonBarNew.obj
 0001:00057cf0       ??_GCMFCRibbonBarNew@@UAEPAXI@Z 00458cf0 f i MFCRibbonBarNew.obj
 0001:00057d20       ??1CMFCRibbonBarNew@@UAE@XZ 00458d20 f   MFCRibbonBarNew.obj
 0001:00057d40       ?GetMessageMap@CMFCRibbonBarNew@@MBEPBUAFX_MSGMAP@@XZ 00458d40 f   MFCRibbonBarNew.obj
 0001:00057d50       ?GetThisMessageMap@CMFCRibbonBarNew@@KGPBUAFX_MSGMAP@@XZ 00458d50 f   MFCRibbonBarNew.obj
 0001:00057d60       ?OnShowRibbonContextMenu@CMFCRibbonBarNew@@UAEHPAVCWnd@@HHPAVCMFCRibbonBaseElement@@@Z 00458d60 f   MFCRibbonBarNew.obj
 0001:00057d70       ?GetPaneIcon@CBasePane@@UAEPAUHICON__@@H@Z 00458d70 f i MFCRibbonBarNew.obj
 0001:00057d90       ?GetIcon@CWnd@@QBEPAUHICON__@@H@Z 00458d90 f i MFCRibbonBarNew.obj
 0001:00057dc0       ?CanAutoHide@CBasePane@@UBEHXZ 00458dc0 f i MFCRibbonBarNew.obj
 0001:00057de0       ?GetMinSize@CPane@@UBEXAAVCSize@@@Z 00458de0 f i MFCRibbonBarNew.obj
 0001:00057e10       ?DockToFrameWindow@CPane@@UAEHKPBUtagRECT@@KPAVCBasePane@@HH@Z 00458e10 f i MFCRibbonBarNew.obj
 0001:00057e20       ?DockPaneStandard@CPane@@UAEPAV1@AAH@Z 00458e20 f i MFCRibbonBarNew.obj
 0001:00057e40       ?OnChangeMenuHighlight@CMFCRibbonBaseElement@@UAEXPAVCMFCRibbonPanelMenuBar@@PAV1@@Z 00458e40 f i MainFrm.obj
 0001:00057e40       ?OnDrawDragRect@CPane@@MAEXPBUtagRECT@@0@Z 00458e40 f i MFCRibbonBarNew.obj
 0001:00057e50       ?GetCaptionHeight@CMFCRibbonBar@@UBEHXZ 00458e50 f i MFCRibbonBarNew.obj
 0001:00057e70       ?CanBeAttached@CBasePane@@UBEHXZ 00458e70 f i MFCRibbonBarNew.obj
 0001:00057e70       ?CanBeStretchedHorizontally@CMFCRibbonBaseElement@@UAEHXZ 00458e70 f i MainFrm.obj
 0001:00057e70       ?OnAutoRepeat@CMFCRibbonBaseElement@@UAEHXZ 00458e70 f i MainFrm.obj
 0001:00057e70       ?CanBeAddedToQuickAccessToolBar@CMFCRibbonApplicationButton@@MBEHXZ 00458e70 f i MainFrm.obj
 0001:00057e70       ?IsWholeRowHeight@CMFCRibbonBaseElement@@UBEHXZ 00458e70 f i MainFrm.obj
 0001:00057e70       ?IsDefaultPanelButton@CMFCRibbonButton@@UBEHXZ 00458e70 f i MainFrm.obj
 0001:00057e70       ?HideInPrintPreviewMode@CMFCRibbonBar@@MBEHXZ 00458e70 f i MFCRibbonBarNew.obj
 0001:00057e70       ?IsSeparator@CMFCRibbonBaseElement@@UBEHXZ 00458e70 f i MainFrm.obj
 0001:00057e70       ?IsResizable@CPane@@UBEHXZ 00458e70 f i MFCRibbonBarNew.obj
 0001:00057e70       ?IsDrawTooltipImage@CMFCRibbonApplicationButton@@MBEHXZ 00458e70 f i MainFrm.obj
 0001:00057e70       ?IsAutoHideMode@CBasePane@@UBEHXZ 00458e70 f i MFCRibbonBarNew.obj
 0001:00057e70       ?AllowShowOnPaneMenu@CMFCRibbonBar@@MBEHXZ 00458e70 f i MFCRibbonBarNew.obj
 0001:00057e70       ?IsGalleryIcon@CMFCRibbonBaseElement@@UBEHXZ 00458e70 f i MainFrm.obj
 0001:00057e70       ?DoesAllowDynInsertBefore@CMFCOutlookBar@@UBEHXZ 00458e70 f i MainFrm.obj
 0001:00057e70       ?IsShowTooltipOnBottom@CMFCRibbonApplicationButton@@MBEHXZ 00458e70 f i MainFrm.obj
 0001:00057e70       ?IsAccessibilityCompatible@CDockablePane@@UAEHXZ 00458e70 f i MainFrm.obj
 0001:00057e70       ?IsInFloatingMultiPaneFrameWnd@CPane@@UBEHXZ 00458e70 f i MFCRibbonBarNew.obj
 0001:00057e70       ?HasAutoHideMode@CBaseTabbedPane@@UBEHXZ 00458e70 f i MainFrm.obj
 0001:00057e80       ??0CModifyGroup@@QAE@PAVCWnd@@@Z 00458e80 f   ModifyGroup.obj
 0001:00057f10       ??_ECModifyGroup@@UAEPAXI@Z 00458f10 f i ModifyGroup.obj
 0001:00057f10       ??_GCModifyGroup@@UAEPAXI@Z 00458f10 f i ModifyGroup.obj
 0001:00057f40       ?DoDataExchange@CModifyGroup@@MAEXPAVCDataExchange@@@Z 00458f40 f   ModifyGroup.obj
 0001:00057fa0       ?GetMessageMap@CGroupExt@@MBEPBUAFX_MSGMAP@@XZ 00458fa0 f   GroupExt.obj
 0001:00057fa0       ?GetMessageMap@CAddToGroup@@MBEPBUAFX_MSGMAP@@XZ 00458fa0 f   AddToGroup.obj
 0001:00057fa0       ?GetMessageMap@CInfoPromptDlg@@MBEPBUAFX_MSGMAP@@XZ 00458fa0 f   InfoPromptDlg.obj
 0001:00057fa0       ?GetMessageMap@CModifyGroup@@MBEPBUAFX_MSGMAP@@XZ 00458fa0 f   ModifyGroup.obj
 0001:00057fb0       ?OnInitDialog@CModifyGroup@@MAEHXZ 00458fb0 f   ModifyGroup.obj
 0001:000581c0       ?OnOK@CModifyGroup@@MAEXXZ 004591c0 f   ModifyGroup.obj
 0001:00058240       ?CheckValid@CModifyGroup@@QAEHV?$CStringT@DV?$StrTraitMFC_DLL@DV?$ChTraitsCRT@D@ATL@@@@@ATL@@@Z 00459240 f   ModifyGroup.obj
 0001:00058580       ?GetRuntimeClass@CMsgDlg@@UBEPAUCRuntimeClass@@XZ 00459580 f   MsgDlg.obj
 0001:00058590       ??0CMsgDlg@@QAE@PAVCWnd@@@Z 00459590 f   MsgDlg.obj
 0001:00058660       ??_GCMsgDlg@@UAEPAXI@Z     00459660 f i MsgDlg.obj
 0001:00058660       ??_ECMsgDlg@@UAEPAXI@Z     00459660 f i MsgDlg.obj
 0001:00058690       ??1CMsgDlg@@UAE@XZ         00459690 f   MsgDlg.obj
 0001:00058700       ?DoDataExchange@CMsgDlg@@MAEXPAVCDataExchange@@@Z 00459700 f   MsgDlg.obj
 0001:00058730       ?GetMessageMap@CMsgDlg@@MBEPBUAFX_MSGMAP@@XZ 00459730 f   MsgDlg.obj
 0001:00058740       ?GetThisMessageMap@CMsgDlg@@KGPBUAFX_MSGMAP@@XZ 00459740 f   MsgDlg.obj
 0001:00058750       ?OnInitDialog@CMsgDlg@@MAEHXZ 00459750 f   MsgDlg.obj
 0001:00058960       ?OnBnClickedOk@CMsgDlg@@QAEXXZ 00459960 f   MsgDlg.obj
 0001:00059220       ??0CMyEdit@@QAE@XZ         0045a220 f   MyEdit.obj
 0001:00059250       ??_GCMyEdit@@UAEPAXI@Z     0045a250 f i MyEdit.obj
 0001:00059250       ??_ECMyEdit@@UAEPAXI@Z     0045a250 f i MyEdit.obj
 0001:00059280       ??1CMyEdit@@UAE@XZ         0045a280 f   MyEdit.obj
 0001:000592a0       ?GetMessageMap@CMyEdit@@MBEPBUAFX_MSGMAP@@XZ 0045a2a0 f   MyEdit.obj
 0001:000592b0       ?GetThisMessageMap@CMyEdit@@KGPBUAFX_MSGMAP@@XZ 0045a2b0 f   MyEdit.obj
 0001:000592c0       ?OnChar@CMyEdit@@IAEXIII@Z 0045a2c0 f   MyEdit.obj
 0001:00059490       ?OnKillFocus@CMyEdit@@IAEXPAVCWnd@@@Z 0045a490 f   MyEdit.obj
 0001:00059500       ?PreTranslateMessage@CMyEdit@@UAEHPAUtagMSG@@@Z 0045a500 f   MyEdit.obj
 0001:00059540       ?WindowProc@CMyEdit@@MAEJIIJ@Z 0045a540 f   MyEdit.obj
 0001:00059570       ?OnChange@CMyEdit@@IAEXXZ  0045a570 f   MyEdit.obj
 0001:000595f0       ?ChangeRectSize@CMyEdit@@QAEXUtagRECT@@0V?$CStringT@DV?$StrTraitMFC_DLL@DV?$ChTraitsCRT@D@ATL@@@@@ATL@@@Z 0045a5f0 f   MyEdit.obj
 0001:00059700       ?OnClose@CMyEdit@@IAEXXZ   0045a700 f   MyEdit.obj
 0001:00059720       ?MyEidtBox@CMyEdit@@QAEXV?$CStringT@DV?$StrTraitMFC_DLL@DV?$ChTraitsCRT@D@ATL@@@@@ATL@@0IAAH@Z 0045a720 f   MyEdit.obj
 0001:00059880       ?MoveWindow@CWnd@@QAEXPBUtagRECT@@H@Z 0045a880 f i MyEdit.obj
 0001:000598c0       ??0CMyIOCP@@QAE@XZ         0045a8c0 f   MyIOCP.obj
 0001:00059910       ??_ECMyIOCP@@UAEPAXI@Z     0045a910 f i MyIOCP.obj
 0001:00059910       ??_GCMyIOCP@@UAEPAXI@Z     0045a910 f i MyIOCP.obj
 0001:00059940       ??1CMyIOCP@@UAE@XZ         0045a940 f   MyIOCP.obj
 0001:00059960       ?Initialize@CMyIOCP@@QAE_NXZ 0045a960 f   MyIOCP.obj
 0001:00059a60       ?InitializeIOCP@CMyIOCP@@QAE_NXZ 0045aa60 f   MyIOCP.obj
 0001:00059b50       ?CleanUp@CMyIOCP@@QAEXXZ   0045ab50 f   MyIOCP.obj
 0001:00059bd0       ?DeInitialize@CMyIOCP@@QAEXXZ 0045abd0 f   MyIOCP.obj
 0001:00059c20       ?AcceptThread@CMyIOCP@@SAIPAX@Z 0045ac20 f   MyIOCP.obj
 0001:00059ca0       ?AcceptConnection@CMyIOCP@@QAEXI@Z 0045aca0 f   MyIOCP.obj
 0001:00059fa0       ?SetSocket@CClientContext@@QAEXI@Z 0045afa0 f i MyIOCP.obj
 0001:00059fc0       ??0CClientContext@@QAE@XZ  0045afc0 f i MyIOCP.obj
 0001:0005a030       ?AssociateWithIOCP@CMyIOCP@@QAE_NPAVCClientContext@@@Z 0045b030 f   MyIOCP.obj
 0001:0005a0d0       ?WorkerThread@CMyIOCP@@SAIPAX@Z 0045b0d0 f   MyIOCP.obj
 0001:0005a1f0       ?GetOpCode@CClientContext@@QAEHXZ 0045b1f0 f i MyIOCP.obj
 0001:0005a210       ?WriteToConsole@CMyIOCP@@UAEXPAD@Z 0045b210 f   MyIOCP.obj
 0001:0005a250       ?AddToClientList@CMyIOCP@@QAEXPAVCClientContext@@@Z 0045b250 f   MyIOCP.obj
 0001:0005a290       ?RemoveFromClientListAndFreeMemory@CMyIOCP@@QAEXPAVCClientContext@@@Z 0045b290 f   MyIOCP.obj
 0001:0005a380       ?CleanClientList@CMyIOCP@@QAEXXZ 0045b380 f   MyIOCP.obj
 0001:0005a490       ?StartUp@CMyIOCP@@QAEHXZ   0045b490 f   MyIOCP.obj
 0001:0005a770       ?OnCloseMiniFrame@CFrameWndEx@@UAEHPAVCPaneFrameWnd@@@Z 0045b770 f   MainFrm.obj
 0001:0005a770       ?OnEraseBkgnd@CCalendarBar@@IAEHPAVCDC@@@Z 0045b770 f   CalendarBar.obj
 0001:0005a770       ?OnRecvComplete@CMyIOCP@@UAEHPAVCClientContext@@@Z 0045b770 f   MyIOCP.obj
 0001:0005a770       ?OnAfterShowPaneMenu@CPane@@MAEHH@Z 0045b770 f   MainFrm.obj
 0001:0005a770       ?OnSendComplete@CMyIOCP@@UAEHPAVCClientContext@@@Z 0045b770 f   MyIOCP.obj
 0001:0005a770       ?OnBeforeShowPaneMenu@CPane@@MAEHAAVCMenu@@@Z 0045b770 f   MainFrm.obj
 0001:0005a770       ?OnCloseDockingPane@CFrameWndEx@@UAEHPAVCDockablePane@@@Z 0045b770 f   MainFrm.obj
 0001:0005a770       ?OnBeforeAnimation@CMFCOutlookBar@@UAEHH@Z 0045b770 f   MainFrm.obj
 0001:0005a770       ?SendAck@CMyIOCP@@UAEHPAVCClientContext@@@Z 0045b770 f   MyIOCP.obj
 0001:0005a790       ??0?$vector@PAVCClientContext@@V?$allocator@PAVCClientContext@@@std@@@std@@QAE@XZ 0045b790 f i MyIOCP.obj
 0001:0005a800       ??1?$vector@PAVCClientContext@@V?$allocator@PAVCClientContext@@@std@@@std@@QAE@XZ 0045b800 f i MyIOCP.obj
 0001:0005a860       ?begin@?$vector@PAVCClientContext@@V?$allocator@PAVCClientContext@@@std@@@std@@QAE?AV?$_Vector_iterator@PAVCClientContext@@V?$allocator@PAVCClientContext@@@std@@@2@XZ 0045b860 f i MyIOCP.obj
 0001:0005a890       ?end@?$vector@PAVCClientContext@@V?$allocator@PAVCClientContext@@@std@@@std@@QAE?AV?$_Vector_iterator@PAVCClientContext@@V?$allocator@PAVCClientContext@@@std@@@2@XZ 0045b890 f i MyIOCP.obj
 0001:0005a8c0       ?push_back@?$vector@PAVCClientContext@@V?$allocator@PAVCClientContext@@@std@@@std@@QAEXABQAVCClientContext@@@Z 0045b8c0 f i MyIOCP.obj
 0001:0005a940       ?erase@?$vector@PAVCClientContext@@V?$allocator@PAVCClientContext@@@std@@@std@@QAE?AV?$_Vector_iterator@PAVCClientContext@@V?$allocator@PAVCClientContext@@@std@@@2@V?$_Vector_const_iterator@PAVCClientContext@@V?$allocator@PAVCClientContext@@@std@@@2@@Z 0045b940 f i MyIOCP.obj
 0001:0005a9b0       ?clear@?$vector@PAVCClientContext@@V?$allocator@PAVCClientContext@@@std@@@std@@QAEXXZ 0045b9b0 f i MyIOCP.obj
 0001:0005aa10       ??0?$_Vector_iterator@PAVCClientContext@@V?$allocator@PAVCClientContext@@@std@@@std@@QAE@XZ 0045ba10 f i MyIOCP.obj
 0001:0005aa30       ??D?$_Vector_iterator@PAVCClientContext@@V?$allocator@PAVCClientContext@@@std@@@std@@QBEAAPAVCClientContext@@XZ 0045ba30 f i MyIOCP.obj
 0001:0005aa50       ??E?$_Vector_iterator@PAVCClientContext@@V?$allocator@PAVCClientContext@@@std@@@std@@QAE?AV01@H@Z 0045ba50 f i MyIOCP.obj
 0001:0005aa90       ??9?$_Vector_const_iterator@PAVCClientContext@@V?$allocator@PAVCClientContext@@@std@@@std@@QBE_NABV01@@Z 0045ba90 f i MyIOCP.obj
 0001:0005aac0       ??1?$_Vector_val@PAVCClientContext@@V?$allocator@PAVCClientContext@@@std@@@std@@QAE@XZ 0045bac0 f i MyIOCP.obj
 0001:0005aae0       ?capacity@?$vector@PAVCClientContext@@V?$allocator@PAVCClientContext@@@std@@@std@@QBEIXZ 0045bae0 f i MyIOCP.obj
 0001:0005ab20       ?_Make_iter@?$vector@PAVCClientContext@@V?$allocator@PAVCClientContext@@@std@@@std@@QBE?AV?$_Vector_iterator@PAVCClientContext@@V?$allocator@PAVCClientContext@@@std@@@2@V?$_Vector_const_iterator@PAVCClientContext@@V?$allocator@PAVCClientContext@@@std@@@2@@Z 0045bb20 f i MyIOCP.obj
 0001:0005ab40       ?size@?$vector@PAVCClientContext@@V?$allocator@PAVCClientContext@@@std@@@std@@QBEIXZ 0045bb40 f i MyIOCP.obj
 0001:0005ab60       ?insert@?$vector@PAVCClientContext@@V?$allocator@PAVCClientContext@@@std@@@std@@QAE?AV?$_Vector_iterator@PAVCClientContext@@V?$allocator@PAVCClientContext@@@std@@@2@V?$_Vector_const_iterator@PAVCClientContext@@V?$allocator@PAVCClientContext@@@std@@@2@ABQAVCClientContext@@@Z 0045bb60 f i MyIOCP.obj
 0001:0005abe0       ?erase@?$vector@PAVCClientContext@@V?$allocator@PAVCClientContext@@@std@@@std@@QAE?AV?$_Vector_iterator@PAVCClientContext@@V?$allocator@PAVCClientContext@@@std@@@2@V?$_Vector_const_iterator@PAVCClientContext@@V?$allocator@PAVCClientContext@@@std@@@2@0@Z 0045bbe0 f i MyIOCP.obj
 0001:0005ac80       ?_Buy@?$vector@PAVCClientContext@@V?$allocator@PAVCClientContext@@@std@@@std@@IAE_NI@Z 0045bc80 f i MyIOCP.obj
 0001:0005ad00       ?_Destroy@?$vector@PAVCClientContext@@V?$allocator@PAVCClientContext@@@std@@@std@@IAEXPAPAVCClientContext@@0@Z 0045bd00 f i MyIOCP.obj
 0001:0005ad30       ?_Tidy@?$vector@PAVCClientContext@@V?$allocator@PAVCClientContext@@@std@@@std@@IAEXXZ 0045bd30 f i MyIOCP.obj
 0001:0005ada0       ?_Ufill@?$vector@PAVCClientContext@@V?$allocator@PAVCClientContext@@@std@@@std@@IAEPAPAVCClientContext@@PAPAV3@IABQAV3@@Z 0045bda0 f i MyIOCP.obj
 0001:0005ade0       ??0?$_Vector_val@PAVCClientContext@@V?$allocator@PAVCClientContext@@@std@@@std@@IAE@V?$allocator@PAVCClientContext@@@1@@Z 0045bde0 f i MyIOCP.obj
 0001:0005ae20       ??1?$_Container_base_aux_alloc_real@V?$allocator@PAVCClientContext@@@std@@@std@@IAE@XZ 0045be20 f i MyIOCP.obj
 0001:0005ae80       ??0?$_Vector_iterator@PAVCClientContext@@V?$allocator@PAVCClientContext@@@std@@@std@@QAE@PAPAVCClientContext@@PBV_Container_base_aux@1@@Z 0045be80 f i MyIOCP.obj
 0001:0005aea0       ??E?$_Vector_iterator@PAVCClientContext@@V?$allocator@PAVCClientContext@@@std@@@std@@QAEAAV01@XZ 0045bea0 f i MyIOCP.obj
 0001:0005aec0       ??0?$_Vector_const_iterator@PAVCClientContext@@V?$allocator@PAVCClientContext@@@std@@@std@@QAE@XZ 0045bec0 f i MyIOCP.obj
 0001:0005aee0       ??D?$_Vector_const_iterator@PAVCClientContext@@V?$allocator@PAVCClientContext@@@std@@@std@@QBEABQAVCClientContext@@XZ 0045bee0 f i MyIOCP.obj
 0001:0005af30       ??8?$_Vector_const_iterator@PAVCClientContext@@V?$allocator@PAVCClientContext@@@std@@@std@@QBE_NABV01@@Z 0045bf30 f i MyIOCP.obj
 0001:0005af80       ??0?$_Ranit@PAVCClientContext@@HPBQAV1@ABQAV1@@std@@QAE@XZ 0045bf80 f i MyIOCP.obj
 0001:0005afa0       ??0?$_Iterator_with_base@Urandom_access_iterator_tag@std@@PAVCClientContext@@HPBQAV3@ABQAV3@V_Iterator_base_aux@2@@std@@QAE@XZ 0045bfa0 f i MyIOCP.obj
 0001:0005afc0       ?max_size@?$vector@PAVCClientContext@@V?$allocator@PAVCClientContext@@@std@@@std@@QBEIXZ 0045bfc0 f i MyIOCP.obj
 0001:0005afe0       ?_Insert_n@?$vector@PAVCClientContext@@V?$allocator@PAVCClientContext@@@std@@@std@@IAEXV?$_Vector_const_iterator@PAVCClientContext@@V?$allocator@PAVCClientContext@@@std@@@2@IABQAVCClientContext@@@Z 0045bfe0 f i MyIOCP.obj
 0001:0005b390       ?_Xlen@?$vector@PAVCClientContext@@V?$allocator@PAVCClientContext@@@std@@@std@@KAXXZ 0045c390 f i MyIOCP.obj
 0001:0005b410       ??0?$_Container_base_aux_alloc_real@V?$allocator@PAVCClientContext@@@std@@@std@@IAE@V?$allocator@PAVCClientContext@@@1@@Z 0045c410 f i MyIOCP.obj
 0001:0005b4d0       ??0?$allocator@PAVCClientContext@@@std@@QAE@ABV01@@Z 0045c4d0 f i MyIOCP.obj
 0001:0005b4d0       ??$?0PAVCClientContext@@@?$allocator@V_Aux_cont@std@@@std@@QAE@ABV?$allocator@PAVCClientContext@@@1@@Z 0045c4d0 f i MyIOCP.obj
 0001:0005b4e0       ?deallocate@?$allocator@V_Aux_cont@std@@@std@@QAEXPAV_Aux_cont@2@I@Z 0045c4e0 f i KiboManagerView.obj
 0001:0005b4e0       ?deallocate@?$allocator@PAVCClientContext@@@std@@QAEXPAPAVCClientContext@@I@Z 0045c4e0 f i MyIOCP.obj
 0001:0005b500       ?allocate@?$allocator@V_Aux_cont@std@@@std@@QAEPAV_Aux_cont@2@I@Z 0045c500 f i KiboManagerView.obj
 0001:0005b500       ?allocate@?$allocator@PAVCClientContext@@@std@@QAEPAPAVCClientContext@@I@Z 0045c500 f i MyIOCP.obj
 0001:0005b520       ??H?$_Vector_iterator@PAVCClientContext@@V?$allocator@PAVCClientContext@@@std@@@std@@QBE?AV01@H@Z 0045c520 f i MyIOCP.obj
 0001:0005b560       ??0?$_Vector_const_iterator@PAVCClientContext@@V?$allocator@PAVCClientContext@@@std@@@std@@QAE@PAPAVCClientContext@@PBV_Container_base_aux@1@@Z 0045c560 f i MyIOCP.obj
 0001:0005b5c0       ??E?$_Vector_const_iterator@PAVCClientContext@@V?$allocator@PAVCClientContext@@@std@@@std@@QAEAAV01@XZ 0045c5c0 f i MyIOCP.obj
 0001:0005b620       ??G?$_Vector_const_iterator@PAVCClientContext@@V?$allocator@PAVCClientContext@@@std@@@std@@QBEHABV01@@Z 0045c620 f i MyIOCP.obj
 0001:0005b670       ?max_size@?$allocator@PAVCClientContext@@@std@@QBEIXZ 0045c670 f i MyIOCP.obj
 0001:0005b6a0       ??Y?$_Vector_iterator@PAVCClientContext@@V?$allocator@PAVCClientContext@@@std@@@std@@QAEAAV01@H@Z 0045c6a0 f i MyIOCP.obj
 0001:0005b6c0       ??Y?$_Vector_const_iterator@PAVCClientContext@@V?$allocator@PAVCClientContext@@@std@@@std@@QAEAAV01@H@Z 0045c6c0 f i MyIOCP.obj
 0001:0005b740       ??$sprintf_s@$0BAAA@@@YAHAAY0BAAA@DPBDZZ 0045c740 f i MyIOCP.obj
 0001:0005b770       ??$unchecked_copy@PAPAVCClientContext@@PAPAV1@@stdext@@YAPAPAVCClientContext@@PAPAV1@00@Z 0045c770 f i MyIOCP.obj
 0001:0005b7e0       ??$_Destroy_range@V?$allocator@PAVCClientContext@@@std@@@std@@YAXPAPAVCClientContext@@0AAV?$allocator@PAVCClientContext@@@0@@Z 0045c7e0 f i MyIOCP.obj
 0001:0005b820       ??$unchecked_uninitialized_fill_n@PAPAVCClientContext@@IPAV1@V?$allocator@PAVCClientContext@@@std@@@stdext@@YAXPAPAVCClientContext@@IABQAV1@AAV?$allocator@PAVCClientContext@@@std@@@Z 0045c820 f i MyIOCP.obj
 0001:0005b870       ??$_Umove@PAPAVCClientContext@@@?$vector@PAVCClientContext@@V?$allocator@PAVCClientContext@@@std@@@std@@IAEPAPAVCClientContext@@PAPAV2@00@Z 0045c870 f i MyIOCP.obj
 0001:0005b8a0       ??$fill@PAPAVCClientContext@@PAV1@@std@@YAXPAPAVCClientContext@@0ABQAV1@@Z 0045c8a0 f i MyIOCP.obj
 0001:0005b8d0       ??$_Unchecked_move_backward@PAPAVCClientContext@@PAPAV1@@stdext@@YAPAPAVCClientContext@@PAPAV1@00@Z 0045c8d0 f i MyIOCP.obj
 0001:0005b940       ??$_Allocate@PAVCClientContext@@@std@@YAPAPAVCClientContext@@IPAPAV1@@Z 0045c940 f i MyIOCP.obj
 0001:0005b940       ??$_Allocate@V_Aux_cont@std@@@std@@YAPAV_Aux_cont@0@IPAV10@@Z 0045c940 f i KiboManagerView.obj
 0001:0005b990       ??$_Checked_base@PAPAVCClientContext@@@std@@YAPAPAVCClientContext@@AAPAPAV1@@Z 0045c990 f i MyIOCP.obj
 0001:0005b9b0       ??$_Ptr_cat@PAPAVCClientContext@@PAPAV1@@std@@YA?AU_Scalar_ptr_iterator_tag@0@AAPAPAVCClientContext@@0@Z 0045c9b0 f i MyIOCP.obj
 0001:0005b9b0       ??$_Move_cat@PAPAVCClientContext@@@std@@YA?AU_Undefined_move_tag@0@ABQAPAVCClientContext@@@Z 0045c9b0 f i MyIOCP.obj
 0001:0005b9c0       ??$_Copy_opt@PAPAVCClientContext@@PAPAV1@Urandom_access_iterator_tag@std@@@std@@YAPAPAVCClientContext@@PAPAV1@00Urandom_access_iterator_tag@0@U_Scalar_ptr_iterator_tag@0@U_Range_checked_iterator_tag@0@@Z 0045c9c0 f i MyIOCP.obj
 0001:0005ba10       ??3@YAXPAX0@Z              0045ca10 f i KiboManagerView.obj
 0001:0005ba10       ??$_Destroy_range@V?$allocator@PAVCClientContext@@@std@@@std@@YAXPAPAVCClientContext@@0AAV?$allocator@PAVCClientContext@@@0@U_Scalar_ptr_iterator_tag@0@@Z 0045ca10 f i MyIOCP.obj
 0001:0005ba20       ??$_Uninit_fill_n@PAPAVCClientContext@@IPAV1@V?$allocator@PAVCClientContext@@@std@@@std@@YAXPAPAVCClientContext@@IABQAV1@AAV?$allocator@PAVCClientContext@@@0@U_Scalar_ptr_iterator_tag@0@U_Range_checked_iterator_tag@0@@Z 0045ca20 f i MyIOCP.obj
 0001:0005ba40       ??$_Unchecked_uninitialized_move@PAPAVCClientContext@@PAPAV1@V?$allocator@PAVCClientContext@@@std@@@stdext@@YAPAPAVCClientContext@@PAPAV1@00AAV?$allocator@PAVCClientContext@@@std@@@Z 0045ca40 f i MyIOCP.obj
 0001:0005ba90       ??$_Fill@PAPAVCClientContext@@PAV1@@std@@YAXPAPAVCClientContext@@0ABQAV1@@Z 0045ca90 f i MyIOCP.obj
 0001:0005bac0       ??$_Move_backward_opt@PAPAVCClientContext@@PAPAV1@Urandom_access_iterator_tag@std@@U_Undefined_move_tag@3@@std@@YAPAPAVCClientContext@@PAPAV1@00Urandom_access_iterator_tag@0@U_Undefined_move_tag@0@U_Range_checked_iterator_tag@0@@Z 0045cac0 f i MyIOCP.obj
 0001:0005bb10       ??$_Checked_base@PAPAVCClientContext@@@std@@YAPAPAVCClientContext@@AAPAPAV1@U_Unchanged_checked_iterator_base_type_tag@0@@Z 0045cb10 f i MyIOCP.obj
 0001:0005bb20       ??$unchecked_fill_n@PAPAVCClientContext@@IPAV1@@stdext@@YAXPAPAVCClientContext@@IABQAV1@@Z 0045cb20 f i MyIOCP.obj
 0001:0005bb60       ??$_Uninit_move@PAPAVCClientContext@@PAPAV1@V?$allocator@PAVCClientContext@@@std@@U_Undefined_move_tag@3@@std@@YAPAPAVCClientContext@@PAPAV1@00AAV?$allocator@PAVCClientContext@@@0@U_Undefined_move_tag@0@U_Range_checked_iterator_tag@0@@Z 0045cb60 f i MyIOCP.obj
 0001:0005bb80       ??$_Copy_backward_opt@PAPAVCClientContext@@PAPAV1@Urandom_access_iterator_tag@std@@@std@@YAPAPAVCClientContext@@PAPAV1@00Urandom_access_iterator_tag@0@U_Scalar_ptr_iterator_tag@0@U_Range_checked_iterator_tag@0@@Z 0045cb80 f i MyIOCP.obj
 0001:0005bbd0       ??$_Iter_random@PAPAVCClientContext@@PAPAV1@@std@@YA?AUrandom_access_iterator_tag@0@ABQAPAVCClientContext@@0@Z 0045cbd0 f i MyIOCP.obj
 0001:0005bbd0       ??$_Iter_cat@PAPAVCClientContext@@@std@@YA?AUrandom_access_iterator_tag@0@ABQAPAVCClientContext@@@Z 0045cbd0 f i MyIOCP.obj
 0001:0005bbe0       ??$_Fill_n@PAPAVCClientContext@@IPAV1@@std@@YAXPAPAVCClientContext@@IABQAV1@Urandom_access_iterator_tag@0@U_Range_checked_iterator_tag@0@@Z 0045cbe0 f i MyIOCP.obj
 0001:0005bc20       ??$unchecked_uninitialized_copy@PAPAVCClientContext@@PAPAV1@V?$allocator@PAVCClientContext@@@std@@@stdext@@YAPAPAVCClientContext@@PAPAV1@00AAV?$allocator@PAVCClientContext@@@std@@@Z 0045cc20 f i MyIOCP.obj
 0001:0005bc80       ??$_Fill_n@PAPAVCClientContext@@IPAV1@@std@@YAXPAPAVCClientContext@@IABQAV1@U_Range_checked_iterator_tag@0@@Z 0045cc80 f i MyIOCP.obj
 0001:0005bcb0       ??$_Uninit_copy@PAPAVCClientContext@@PAPAV1@V?$allocator@PAVCClientContext@@@std@@@std@@YAPAPAVCClientContext@@PAPAV1@00AAV?$allocator@PAVCClientContext@@@0@U_Scalar_ptr_iterator_tag@0@U_Range_checked_iterator_tag@0@@Z 0045ccb0 f i MyIOCP.obj
 0001:0005bd00       ?CreateObject@CMyPropertyPage1@@SGPAVCObject@@XZ 0045cd00 f   MyPropertyPage1.obj
 0001:0005bd80       ?GetRuntimeClass@CMyPropertyPage1@@UBEPAUCRuntimeClass@@XZ 0045cd80 f   MyPropertyPage1.obj
 0001:0005bd90       ?CreateObject@CMyPropertyPage2@@SGPAVCObject@@XZ 0045cd90 f   MyPropertyPage1.obj
 0001:0005be10       ?_GetBaseClass@CMyPropertyPage3@@KGPAUCRuntimeClass@@XZ 0045ce10 f   MyPropertyPage1.obj
 0001:0005be10       ?_GetBaseClass@CMyPropertyPage2@@KGPAUCRuntimeClass@@XZ 0045ce10 f   MyPropertyPage1.obj
 0001:0005be10       ?_GetBaseClass@CMyPropertyPage1@@KGPAUCRuntimeClass@@XZ 0045ce10 f   MyPropertyPage1.obj
 0001:0005be20       ?GetRuntimeClass@CMyPropertyPage2@@UBEPAUCRuntimeClass@@XZ 0045ce20 f   MyPropertyPage1.obj
 0001:0005be30       ?CreateObject@CMyPropertyPage3@@SGPAVCObject@@XZ 0045ce30 f   MyPropertyPage1.obj
 0001:0005beb0       ?GetRuntimeClass@CMyPropertyPage3@@UBEPAUCRuntimeClass@@XZ 0045ceb0 f   MyPropertyPage1.obj
 0001:0005bec0       ??0CMyPropertyPage1@@QAE@XZ 0045cec0 f   MyPropertyPage1.obj
 0001:0005bf40       ??_GCMyPropertyPage1@@UAEPAXI@Z 0045cf40 f i MyPropertyPage1.obj
 0001:0005bf40       ??_ECMyPropertyPage1@@UAEPAXI@Z 0045cf40 f i MyPropertyPage1.obj
 0001:0005bf70       ??1CMyPropertyPage1@@UAE@XZ 0045cf70 f   MyPropertyPage1.obj
 0001:0005bfa0       ?DoDataExchange@CMyPropertyPage1@@MAEXPAVCDataExchange@@@Z 0045cfa0 f   MyPropertyPage1.obj
 0001:0005bfe0       ?GetMessageMap@CMyPropertyPage1@@MBEPBUAFX_MSGMAP@@XZ 0045cfe0 f   MyPropertyPage1.obj
 0001:0005bff0       ?GetThisMessageMap@CMyPropertyPage1@@KGPBUAFX_MSGMAP@@XZ 0045cff0 f   MyPropertyPage1.obj
 0001:0005c000       ??0CMyPropertyPage2@@QAE@XZ 0045d000 f   MyPropertyPage1.obj
 0001:0005c040       ??_GCMyPropertyPage2@@UAEPAXI@Z 0045d040 f i MyPropertyPage1.obj
 0001:0005c040       ??_ECMyPropertyPage2@@UAEPAXI@Z 0045d040 f i MyPropertyPage1.obj
 0001:0005c070       ??1CMyPropertyPage2@@UAE@XZ 0045d070 f   MyPropertyPage1.obj
 0001:0005c090       ?DoDataExchange@CMyPropertyPage2@@MAEXPAVCDataExchange@@@Z 0045d090 f   MyPropertyPage1.obj
 0001:0005c0d0       ?GetMessageMap@CMyPropertyPage2@@MBEPBUAFX_MSGMAP@@XZ 0045d0d0 f   MyPropertyPage1.obj
 0001:0005c0e0       ?GetThisMessageMap@CMyPropertyPage2@@KGPBUAFX_MSGMAP@@XZ 0045d0e0 f   MyPropertyPage1.obj
 0001:0005c0f0       ??0CMyPropertyPage3@@QAE@XZ 0045d0f0 f   MyPropertyPage1.obj
 0001:0005c130       ??_ECMyPropertyPage3@@UAEPAXI@Z 0045d130 f i MyPropertyPage1.obj
 0001:0005c130       ??_GCMyPropertyPage3@@UAEPAXI@Z 0045d130 f i MyPropertyPage1.obj
 0001:0005c160       ??1CMyPropertyPage3@@UAE@XZ 0045d160 f   MyPropertyPage1.obj
 0001:0005c180       ?DoDataExchange@CMyPropertyPage3@@MAEXPAVCDataExchange@@@Z 0045d180 f   MyPropertyPage1.obj
 0001:0005c1c0       ?GetMessageMap@CMyPropertyPage3@@MBEPBUAFX_MSGMAP@@XZ 0045d1c0 f   MyPropertyPage1.obj
 0001:0005c1d0       ?GetThisMessageMap@CMyPropertyPage3@@KGPBUAFX_MSGMAP@@XZ 0045d1d0 f   MyPropertyPage1.obj
 0001:0005c1e0       ?GetOwnerDiskOfLogicDrv_Nt@CMyPropertyPage1@@QAEHDAAK0@Z 0045d1e0 f   MyPropertyPage1.obj
 0001:0005c2b0       ?OnBnClickedButtonBrowser@CMyPropertyPage1@@QAEXXZ 0045d2b0 f   MyPropertyPage1.obj
 0001:0005c3e0       ?OnUpfileSet@CMyPropertyPage1@@QAE_NXZ 0045d3e0 f   MyPropertyPage1.obj
 0001:0005cab0       ?OnInitDialog@CMyPropertyPage1@@UAEHXZ 0045dab0 f   MyPropertyPage1.obj
 0001:0005ceb0       ?OnInitDialog@CMyPropertyPage2@@UAEHXZ 0045deb0 f   MyPropertyPage1.obj
 0001:0005d020       ?EClassSet@CMyPropertyPage2@@QAE_NXZ 0045e020 f   MyPropertyPage1.obj
 0001:0005d100       ?OnInitDialog@CMyPropertyPage3@@UAEHXZ 0045e100 f   MyPropertyPage1.obj
 0001:0005d2d0       ?OnBnClickedRadGidget@CMyPropertyPage3@@QAEXXZ 0045e2d0 f   MyPropertyPage1.obj
 0001:0005d2f0       ?OnBnClickedRadDrivget@CMyPropertyPage3@@QAEXXZ 0045e2f0 f   MyPropertyPage1.obj
 0001:0005d310       ?BroTypeSel@CMyPropertyPage3@@QAE_NXZ 0045e310 f   MyPropertyPage1.obj
 0001:0005d3f0       ?_GetBaseClass@CMyPropertySheet@@KGPAUCRuntimeClass@@XZ 0045e3f0 f   MyPropertySheet.obj
 0001:0005d400       ?GetRuntimeClass@CMyPropertySheet@@UBEPAUCRuntimeClass@@XZ 0045e400 f   MyPropertySheet.obj
 0001:0005d410       ??0CMyPropertySheet@@QAE@W4PropSheetLook@CMFCPropertySheet@@IH@Z 0045e410 f   MyPropertySheet.obj
 0001:0005d590       ??_ECMyPropertySheet@@UAEPAXI@Z 0045e590 f i MyPropertySheet.obj
 0001:0005d590       ??_GCMyPropertySheet@@UAEPAXI@Z 0045e590 f i MyPropertySheet.obj
 0001:0005d5c0       ??1CMyPropertySheet@@UAE@XZ 0045e5c0 f   MyPropertySheet.obj
 0001:0005d650       ?GetMessageMap@CMyPropertySheet@@MBEPBUAFX_MSGMAP@@XZ 0045e650 f   MyPropertySheet.obj
 0001:0005d660       ?GetThisMessageMap@CMyPropertySheet@@KGPBUAFX_MSGMAP@@XZ 0045e660 f   MyPropertySheet.obj
 0001:0005d670       ?OnDrawPageHeader@CMyPropertySheet@@UAEXPAVCDC@@HVCRect@@@Z 0045e670 f   MyPropertySheet.obj
 0001:0005d820       ?OnCommand@CMyPropertySheet@@MAEHIJ@Z 0045e820 f   MyPropertySheet.obj
 0001:0005d8e0       ?OnInitDialog@CMyPropertySheet@@UAEHXZ 0045e8e0 f   MyPropertySheet.obj
 0001:0005d9d0       ??0CMyRichEdit@@QAE@XZ     0045e9d0 f   MyRichEdit.obj
 0001:0005d9f0       ??_GCMyRichEdit@@UAEPAXI@Z 0045e9f0 f i MyRichEdit.obj
 0001:0005d9f0       ??_ECMyRichEdit@@UAEPAXI@Z 0045e9f0 f i MyRichEdit.obj
 0001:0005da20       ??1CMyRichEdit@@UAE@XZ     0045ea20 f   MyRichEdit.obj
 0001:0005da40       ?GetMessageMap@CMyRichEdit@@MBEPBUAFX_MSGMAP@@XZ 0045ea40 f   MyRichEdit.obj
 0001:0005da50       ?GetThisMessageMap@CMyRichEdit@@KGPBUAFX_MSGMAP@@XZ 0045ea50 f   MyRichEdit.obj
 0001:0005da60       ?OnEditCopy@COutputList@@IAEXXZ 0045ea60 f i OutputWnd.obj
 0001:0005da60       ?OnCopy@CMyRichEdit@@IAEXXZ 0045ea60 f i MyRichEdit.obj
 0001:0005da80       ?OnCut@CMyRichEdit@@IAEXXZ 0045ea80 f i MyRichEdit.obj
 0001:0005daa0       ?OnPaste@CMyRichEdit@@IAEXXZ 0045eaa0 f i MyRichEdit.obj
 0001:0005dac0       ?OnSelectall@CMyRichEdit@@IAEXXZ 0045eac0 f i MyRichEdit.obj
 0001:0005dac0       ?OnSelall@COutputList@@QAEXXZ 0045eac0 f i OutputWnd.obj
 0001:0005dae0       ?OnUndo@CMyRichEdit@@IAEXXZ 0045eae0 f i MyRichEdit.obj
 0001:0005db00       ?OnClear@CMyRichEdit@@IAEXXZ 0045eb00 f i MyRichEdit.obj
 0001:0005db30       ?OnRButtonDown@CMyRichEdit@@IAEXIVCPoint@@@Z 0045eb30 f   MyRichEdit.obj
 0001:0005de60       ?CreatePopupMenu@CMenu@@QAEHXZ 0045ee60 f i MyRichEdit.obj
 0001:0005de80       ?AppendMenuA@CMenu@@QAEHIIPBD@Z 0045ee80 f i MyRichEdit.obj
 0001:0005deb0       ?OnMButtonDblClk@CWnd@@IAEXIVCPoint@@@Z 0045eeb0 f i ReportCtrl.obj
 0001:0005deb0       ?OnLButtonDblClk@CWnd@@IAEXIVCPoint@@@Z 0045eeb0 f i ReportCtrl.obj
 0001:0005deb0       ?OnRButtonDblClk@CWnd@@IAEXIVCPoint@@@Z 0045eeb0 f i ReportCtrl.obj
 0001:0005deb0       ?OnMButtonDown@CWnd@@IAEXIVCPoint@@@Z 0045eeb0 f i ReportCtrl.obj
 0001:0005deb0       ?OnSize@CWnd@@IAEXIHH@Z    0045eeb0 f i CalendarBar.obj
 0001:0005deb0       ?OnRButtonDown@CWnd@@IAEXIVCPoint@@@Z 0045eeb0 f i MyRichEdit.obj
 0001:0005deb0       ?OnLButtonDown@CWnd@@IAEXIVCPoint@@@Z 0045eeb0 f i GroupTree.obj
 0001:0005deb0       ?OnChar@CWnd@@IAEXIII@Z    0045eeb0 f i MyEdit.obj
 0001:0005ded0       ??0CRichEditCtrl@@QAE@XZ   0045eed0 f i MyRichEdit.obj
 0001:0005def0       ??_GCRichEditCtrl@@UAEPAXI@Z 0045eef0 f i MyRichEdit.obj
 0001:0005def0       ??_ECRichEditCtrl@@UAEPAXI@Z 0045eef0 f i MyRichEdit.obj
 0001:0005df20       ?CanUndo@CRichEditCtrl@@QBEHXZ 0045ef20 f i MyRichEdit.obj
 0001:0005df50       ?Undo@CRichEditCtrl@@QAEHXZ 0045ef50 f i MyRichEdit.obj
 0001:0005df80       ?Copy@CRichEditCtrl@@QAEXXZ 0045ef80 f i MyRichEdit.obj
 0001:0005dfb0       ?Cut@CRichEditCtrl@@QAEXXZ 0045efb0 f i MyRichEdit.obj
 0001:0005dfe0       ?Paste@CRichEditCtrl@@QAEXXZ 0045efe0 f i MyRichEdit.obj
 0001:0005e010       ?GetSelectionType@CRichEditCtrl@@QBEGXZ 0045f010 f i MyRichEdit.obj
 0001:0005e040       ?GetTextLength@CRichEditCtrl@@QBEJXZ 0045f040 f i MyRichEdit.obj
 0001:0005e060       ??0CNewListCtrl@@QAE@XZ    0045f060 f   NewListCtrl.obj
 0001:0005e0a0       ??_ECNewListCtrl@@UAEPAXI@Z 0045f0a0 f i NewListCtrl.obj
 0001:0005e0a0       ??_GCNewListCtrl@@UAEPAXI@Z 0045f0a0 f i NewListCtrl.obj
 0001:0005e0d0       ??1CNewListCtrl@@UAE@XZ    0045f0d0 f   NewListCtrl.obj
 0001:0005e0f0       ?GetMessageMap@CNewListCtrl@@MBEPBUAFX_MSGMAP@@XZ 0045f0f0 f   NewListCtrl.obj
 0001:0005e100       ?GetThisMessageMap@CNewListCtrl@@KGPBUAFX_MSGMAP@@XZ 0045f100 f   NewListCtrl.obj
 0001:0005e110       ?InsertItem@CNewListCtrl@@QAEHHPBDH@Z 0045f110 f   NewListCtrl.obj
 0001:0005e180       ?SetItemText@CNewListCtrl@@QAEHHHPBD@Z 0045f180 f   NewListCtrl.obj
 0001:0005e270       ?DeleteItem@CNewListCtrl@@QAEHH@Z 0045f270 f   NewListCtrl.obj
 0001:0005e2b0       ?DeleteAllItems@CNewListCtrl@@QAEHXZ 0045f2b0 f   NewListCtrl.obj
 0001:0005e310       ?OnCustomDraw@CNewListCtrl@@IAEXPAUtagNMHDR@@PAJ@Z 0045f310 f   NewListCtrl.obj
 0001:0005e940       ?OnEraseBkgnd@CNewListCtrl@@IAEHPAVCDC@@@Z 0045f940 f   NewListCtrl.obj
 0001:0005eac0       ?OnDestroy@CNewListCtrl@@IAEXXZ 0045fac0 f   NewListCtrl.obj
 0001:0005eae0       ?Sort@CNewListCtrl@@QAEXHH@Z 0045fae0 f   NewListCtrl.obj
 0001:0005eb20       ?CompareFunction@CNewListCtrl@@KGHJJJ@Z 0045fb20 f   NewListCtrl.obj
 0001:0005ec40       ?NameCompare@CNewListCtrl@@QAEHPBD0@Z 0045fc40 f   NewListCtrl.obj
 0001:0005f3b0       ?IPCompare@CNewListCtrl@@QAEHPBD0@Z 004603b0 f   NewListCtrl.obj
 0001:0005f400       ?ClearAllItemData@CNewListCtrl@@QAEXXZ 00460400 f   NewListCtrl.obj
 0001:0005f460       ?CenterPoint@CRect@@QBE?AVCPoint@@XZ 00460460 f i NewListCtrl.obj
 0001:0005f4a0       ??1CBrush@@UAE@XZ          004604a0 f i NewListCtrl.obj
 0001:0005f4c0       ??_GCBrush@@UAEPAXI@Z      004604c0 f i NewListCtrl.obj
 0001:0005f4c0       ??_ECBrush@@UAEPAXI@Z      004604c0 f i NewListCtrl.obj
 0001:0005f4f0       ?GetImageInfo@CImageList@@QBEHHPAU_IMAGEINFO@@@Z 004604f0 f i NewListCtrl.obj
 0001:0005f520       ?AfxImageList_GetImageInfo@@YGHPAU_IMAGELIST@@HPAU_IMAGEINFO@@@Z 00460520 f i NewListCtrl.obj
 0001:0005f550       ?_ImageList_GetImageInfo@CComCtlWrapper@@QAEHPAU_IMAGELIST@@HPAU_IMAGEINFO@@@Z 00460550 f i NewListCtrl.obj
 0001:0005f680       ??BImageList_AddMasked_Type@CComCtlWrapper@@QAEP6GHPAU_IMAGELIST@@PAUHBITMAP__@@K@ZXZ 00460680 f i CalendarBar.obj
 0001:0005f680       ??BImageList_ReplaceIcon_Type@CComCtlWrapper@@QAEP6GHPAU_IMAGELIST@@HPAUHICON__@@@ZXZ 00460680 f i PropertyViewDlg.obj
 0001:0005f680       ??BImageList_SetBkColor_Type@CComCtlWrapper@@QAEP6GKPAU_IMAGELIST@@K@ZXZ 00460680 f i WorkspaceBar.obj
 0001:0005f680       ??BImageList_Draw_Type@CComCtlWrapper@@QAEP6GHPAU_IMAGELIST@@HPAUHDC__@@HHI@ZXZ 00460680 f i CalendarBar.obj
 0001:0005f680       ??BImageList_GetImageInfo_Type@CComCtlWrapper@@QAEP6GHPAU_IMAGELIST@@HPAU_IMAGEINFO@@@ZXZ 00460680 f i NewListCtrl.obj
 0001:0005f680       ?_Getcont@_Aux_cont@std@@QBEPBV_Container_base_aux@2@XZ 00460680 f i KiboManagerView.obj
 0001:0005f690       ?GetProcAddress_ImageList_GetImageInfo@CComCtlWrapper@@QAE?AUImageList_GetImageInfo_Type@1@XZ 00460690 f i NewListCtrl.obj
 0001:0005f6f0       ?Invalidate@CWnd@@QAEXH@Z  004606f0 f i NewListCtrl.obj
 0001:0005f710       ?GetFocus@CWnd@@SGPAV1@XZ  00460710 f i NewListCtrl.obj
 0001:0005f730       ?SetBkColor@CListCtrl@@QAEHK@Z 00460730 f i NewListCtrl.obj
 0001:0005f760       ?GetImageList@CListCtrl@@QBEPAVCImageList@@H@Z 00460760 f i NewListCtrl.obj
 0001:0005f790       ?SetItemData@CListCtrl@@QAEHHK@Z 00460790 f i NewListCtrl.obj
 0001:0005f7c0       ??0COutputWnd@@QAE@XZ      004607c0 f   OutputWnd.obj
 0001:0005f880       ??_ECOutputWnd@@UAEPAXI@Z  00460880 f i OutputWnd.obj
 0001:0005f880       ??_GCOutputWnd@@UAEPAXI@Z  00460880 f i OutputWnd.obj
 0001:0005f8b0       ??1COutputWnd@@UAE@XZ      004608b0 f   OutputWnd.obj
 0001:0005f970       ?GetMessageMap@COutputWnd@@MBEPBUAFX_MSGMAP@@XZ 00460970 f   OutputWnd.obj
 0001:0005f980       ?GetThisMessageMap@COutputWnd@@KGPBUAFX_MSGMAP@@XZ 00460980 f   OutputWnd.obj
 0001:0005f990       ?OnCreate@COutputWnd@@IAEHPAUtagCREATESTRUCTA@@@Z 00460990 f   OutputWnd.obj
 0001:0005faf0       ?OnSize@COutputWnd@@IAEXIHH@Z 00460af0 f   OutputWnd.obj
 0001:0005fbe0       ??0COutputList@@QAE@XZ     00460be0 f   OutputWnd.obj
 0001:0005fc00       ??_ECOutputList@@UAEPAXI@Z 00460c00 f i OutputWnd.obj
 0001:0005fc00       ??_GCOutputList@@UAEPAXI@Z 00460c00 f i OutputWnd.obj
 0001:0005fc30       ??1COutputList@@UAE@XZ     00460c30 f   OutputWnd.obj
 0001:0005fc50       ?GetMessageMap@COutputList@@MBEPBUAFX_MSGMAP@@XZ 00460c50 f   OutputWnd.obj
 0001:0005fc60       ?GetThisMessageMap@COutputList@@KGPBUAFX_MSGMAP@@XZ 00460c60 f   OutputWnd.obj
 0001:0005fc70       ?OnContextMenu@COutputList@@IAEXPAVCWnd@@VCPoint@@@Z 00460c70 f   OutputWnd.obj
 0001:0005fdb0       ?OnEditClear@COutputList@@IAEXXZ 00460db0 f   OutputWnd.obj
 0001:0005fde0       ?OnViewOutput@COutputList@@IAEXXZ 00460de0 f   OutputWnd.obj
 0001:0005fe60       ?OnLButtonDown@COutputList@@QAEXIVCPoint@@@Z 00460e60 f   OutputWnd.obj
 0001:0005ff00       ?OnLButtonDown@CWorkspaceBar@@QAEXIVCPoint@@@Z 00460f00 f   WorkspaceBar.obj
 0001:0005ff00       ?OnLButtonDown@COutputWnd@@QAEXIVCPoint@@@Z 00460f00 f   OutputWnd.obj
 0001:0005ffa0       ?OnAfterDock@CPane@@MAEXPAVCBasePane@@PBUtagRECT@@W4AFX_DOCK_METHOD@@@Z 00460fa0 f   MFCRibbonBarNew.obj
 0001:0005ffa0       ?OnContextMenu@CWorkspaceBar@@QAEXPAVCWnd@@VCPoint@@@Z 00460fa0 f   WorkspaceBar.obj
 0001:0005ffa0       ?OnDrawMenuLogo@CFrameWndEx@@UAEXPAVCDC@@PAVCMFCPopupMenu@@ABVCRect@@@Z 00460fa0 f   MainFrm.obj
 0001:0005ffa0       ?OnContextMenu@CWorkspaceBar2@@QAEXPAVCWnd@@VCPoint@@@Z 00460fa0 f   WorkspaceBar2.obj
 0001:0005ffa0       ?OnContextMenu@CMainFrame@@QAEXPAVCWnd@@VCPoint@@@Z 00460fa0 f   MainFrm.obj
 0001:0005ffa0       ?OnContextMenu@COutputWnd@@QAEXPAVCWnd@@VCPoint@@@Z 00460fa0 f   OutputWnd.obj
 0001:0005ffb0       ?SetRectEmpty@CRect@@QAEXXZ 00460fb0 f i OutputWnd.obj
 0001:0005ffd0       ?CreateStockObject@CGdiObject@@QAEHH@Z 00460fd0 f i OutputWnd.obj
 0001:00060000       ?GetOwner@CWnd@@QBEPAV1@XZ 00461000 f i OutputWnd.obj
 0001:00060040       ?OnWindowPosChanging@CWnd@@IAEXPAUtagWINDOWPOS@@@Z 00461040 f i OutputWnd.obj
 0001:00060040       ?OnEraseBkgnd@CWnd@@IAEHPAVCDC@@@Z 00461040 f i NewListCtrl.obj
 0001:00060040       ?OnCreate@CWnd@@IAEHPAUtagCREATESTRUCTA@@@Z 00461040 f i CalendarBar.obj
 0001:00060040       ?OnKillFocus@CWnd@@IAEXPAV1@@Z 00461040 f i MyEdit.obj
 0001:00060040       ?OnTimer@CWnd@@IAEXI@Z     00461040 f i BroadWaitDlg.obj
 0001:00060060       ?GetTabArea@CDockablePane@@UBEXAAVCRect@@0@Z 00461060 f i OutputWnd.obj
 0001:00060080       ?CanAcceptPane@CDockablePane@@UBEHPBVCBasePane@@@Z 00461080 f i OutputWnd.obj
 0001:000600f0       ??0CPartitionSettingDlg@@QAE@PAVCWnd@@@Z 004610f0 f   PartitionSettingDlg.obj
 0001:000602c0       ??_ECPartitionSettingDlg@@UAEPAXI@Z 004612c0 f i PartitionSettingDlg.obj
 0001:000602c0       ??_GCPartitionSettingDlg@@UAEPAXI@Z 004612c0 f i PartitionSettingDlg.obj
 0001:000602f0       ?DoDataExchange@CPartitionSettingDlg@@MAEXPAVCDataExchange@@@Z 004612f0 f   PartitionSettingDlg.obj
 0001:00060410       ?GetMessageMap@CPartitionSettingDlg@@MBEPBUAFX_MSGMAP@@XZ 00461410 f   PartitionSettingDlg.obj
 0001:00060420       ?GetThisMessageMap@CPartitionSettingDlg@@KGPBUAFX_MSGMAP@@XZ 00461420 f   PartitionSettingDlg.obj
 0001:00060430       ?OnInitDialog@CPartitionSettingDlg@@MAEHXZ 00461430 f   PartitionSettingDlg.obj
 0001:000609b0       ?OnSelchangeComboType@CPartitionSettingDlg@@IAEXXZ 004619b0 f   PartitionSettingDlg.obj
 0001:00060f60       ?OnSelchangeComboFreq@CPartitionSettingDlg@@IAEXXZ 00461f60 f   PartitionSettingDlg.obj
 0001:000610c0       ?OnOK@CPartitionSettingDlg@@MAEXXZ 004620c0 f   PartitionSettingDlg.obj
 0001:000613f0       ?ResetContent@CComboBox@@QAEXXZ 004623f0 f i PartitionSettingDlg.obj
 0001:00061420       ?GetFont@CWnd@@QBEPAVCFont@@XZ 00462420 f i PngStatic.obj
 0001:00061450       ?FromHandle@CFont@@SGPAV1@PAUHFONT__@@@Z 00462450 f i PngStatic.obj
 0001:00061460       ?GetRuntimeClass@CPortChannelDlg@@UBEPAUCRuntimeClass@@XZ 00462460 f   PortChannelDlg.obj
 0001:00061470       ??0CPortChannelDlg@@QAE@PAVCWnd@@@Z 00462470 f   PortChannelDlg.obj
 0001:000614b0       ??_GCPortChannelDlg@@UAEPAXI@Z 004624b0 f i PortChannelDlg.obj
 0001:000614b0       ??_ECPortChannelDlg@@UAEPAXI@Z 004624b0 f i PortChannelDlg.obj
 0001:000614e0       ??1CPortChannelDlg@@UAE@XZ 004624e0 f   PortChannelDlg.obj
 0001:00061500       ?GetMessageMap@CPortChannelDlg@@MBEPBUAFX_MSGMAP@@XZ 00462500 f   PortChannelDlg.obj
 0001:00061510       ?GetThisMessageMap@CPortChannelDlg@@KGPBUAFX_MSGMAP@@XZ 00462510 f   PortChannelDlg.obj
 0001:00061520       ?OnBnClickedOk@CPortChannelDlg@@QAEXXZ 00462520 f   PortChannelDlg.obj
 0001:000615f0       ?OnInitDialog@CPortChannelDlg@@UAEHXZ 004625f0 f   PortChannelDlg.obj
 0001:00061770       ?SetTitle@CPortChannelDlg@@QAEXXZ 00462770 f   PortChannelDlg.obj
 0001:00061940       ?GetRuntimeClass@CPortCtrlDlg@@UBEPAUCRuntimeClass@@XZ 00462940 f   PortCtrlDlg.obj
 0001:00061950       ??0CPortCtrlDlg@@QAE@PAVCWnd@@@Z 00462950 f   PortCtrlDlg.obj
 0001:00061a00       ??_ECPortCtrlDlg@@UAEPAXI@Z 00462a00 f i PortCtrlDlg.obj
 0001:00061a00       ??_GCPortCtrlDlg@@UAEPAXI@Z 00462a00 f i PortCtrlDlg.obj
 0001:00061a30       ??1CPortCtrlDlg@@UAE@XZ    00462a30 f   PortCtrlDlg.obj
 0001:00061ab0       ?DoDataExchange@CPortCtrlDlg@@MAEXPAVCDataExchange@@@Z 00462ab0 f   PortCtrlDlg.obj
 0001:00061b10       ?GetMessageMap@CPortCtrlDlg@@MBEPBUAFX_MSGMAP@@XZ 00462b10 f   PortCtrlDlg.obj
 0001:00061b20       ?GetThisMessageMap@CPortCtrlDlg@@KGPBUAFX_MSGMAP@@XZ 00462b20 f   PortCtrlDlg.obj
 0001:00061b30       ?OnInitDialog@CPortCtrlDlg@@MAEHXZ 00462b30 f   PortCtrlDlg.obj
 0001:00062130       ?OnBnClickedOk@CPortCtrlDlg@@QAEXXZ 00463130 f   PortCtrlDlg.obj
 0001:000622a0       ?OnBnClickedAdd@CPortCtrlDlg@@QAEXXZ 004632a0 f   PortCtrlDlg.obj
 0001:00062440       ?OnBnClickedDel@CPortCtrlDlg@@QAEXXZ 00463440 f   PortCtrlDlg.obj
 0001:000625e0       ?OnBnClickedButton1@CPortCtrlDlg@@QAEXXZ 004635e0 f   PortCtrlDlg.obj
 0001:000626c0       ?_InitPortThread@CPortCtrlDlg@@SAIPAX@Z 004636c0 f   PortCtrlDlg.obj
 0001:00062890       ?GetCount@CComboBox@@QBEHXZ 00463890 f i PortCtrlDlg.obj
 0001:000628c0       ?DeleteString@CComboBox@@QAEHI@Z 004638c0 f i PortCtrlDlg.obj
 0001:000628f0       ?InsertString@CComboBox@@QAEHHPBD@Z 004638f0 f i PortCtrlDlg.obj
 0001:00062920       ??0CPrivateProfileFile@@QAE@XZ 00463920 f   PrivateProfileFile.obj
 0001:00062950       ??_ECPrivateProfileFile@@UAEPAXI@Z 00463950 f i PrivateProfileFile.obj
 0001:00062950       ??_GCPrivateProfileFile@@UAEPAXI@Z 00463950 f i PrivateProfileFile.obj
 0001:00062980       ??1CPrivateProfileFile@@UAE@XZ 00463980 f   PrivateProfileFile.obj
 0001:000629a0       ?GetKeyValue@CPrivateProfileFile@@QAEHV?$CStringT@DV?$StrTraitMFC_DLL@DV?$ChTraitsCRT@D@ATL@@@@@ATL@@0AAV23@@Z 004639a0 f   PrivateProfileFile.obj
 0001:00062b80       ?AttachFile@CPrivateProfileFile@@QAEXPBD@Z 00463b80 f   PrivateProfileFile.obj
 0001:00062ba0       ??0CProgressDlg@@QAE@PAVCWnd@@@Z 00463ba0 f   ProgressDlg.obj
 0001:00062ca0       ??_GCProgressDlg@@UAEPAXI@Z 00463ca0 f i ProgressDlg.obj
 0001:00062ca0       ??_ECProgressDlg@@UAEPAXI@Z 00463ca0 f i ProgressDlg.obj
 0001:00062cd0       ??1CProgressDlg@@UAE@XZ    00463cd0 f   ProgressDlg.obj
 0001:00062d80       ?DoDataExchange@CProgressDlg@@MAEXPAVCDataExchange@@@Z 00463d80 f   ProgressDlg.obj
 0001:00062de0       ?GetMessageMap@CProgressDlg@@MBEPBUAFX_MSGMAP@@XZ 00463de0 f   ProgressDlg.obj
 0001:00062df0       ?GetThisMessageMap@CProgressDlg@@KGPBUAFX_MSGMAP@@XZ 00463df0 f   ProgressDlg.obj
 0001:00062e00       ?ReEnableParent@CProgressDlg@@QAEXXZ 00463e00 f   ProgressDlg.obj
 0001:00062e40       ?Create@CProgressDlg@@QAEHPAVCWnd@@@Z 00463e40 f   ProgressDlg.obj
 0001:00062ec0       ?OnCancel@CProgressDlg@@MAEXXZ 00463ec0 f   ProgressDlg.obj
 0001:00062f10       ?OnInitDialog@CProgressDlg@@MAEHXZ 00463f10 f   ProgressDlg.obj
 0001:000630a0       ?DestroyWindow@CProgressDlg@@UAEHXZ 004640a0 f   ProgressDlg.obj
 0001:000630d0       ?WaitStart@CProgressDlg@@QAEHV?$CStringT@DV?$StrTraitMFC_DLL@DV?$ChTraitsCRT@D@ATL@@@@@ATL@@0PAVCWnd@@@Z 004640d0 f   ProgressDlg.obj
 0001:00063240       ?WaitEnd@CBroadWaitDlg@@QAEXXZ 00464240 f   BroadWaitDlg.obj
 0001:00063240       ?WaitEnd@CProgressDlg@@QAEXXZ 00464240 f   ProgressDlg.obj
 0001:00063260       ?SetRange@CProgressDlg@@QAEXHH@Z 00464260 f   ProgressDlg.obj
 0001:000632a0       ?SetPos@CProgressDlg@@QAEHH@Z 004642a0 f   ProgressDlg.obj
 0001:000632d0       ??0CProgressCtrl@@QAE@XZ   004642d0 f i ProgressDlg.obj
 0001:000632f0       ??_GCProgressCtrl@@UAEPAXI@Z 004642f0 f i ProgressDlg.obj
 0001:000632f0       ??_ECProgressCtrl@@UAEPAXI@Z 004642f0 f i ProgressDlg.obj
 0001:00063320       ?SetRange@CProgressCtrl@@QAEXFF@Z 00464320 f i ProgressDlg.obj
 0001:00063360       ?SetStep@CProgressCtrl@@QAEHH@Z 00464360 f i ProgressDlg.obj
 0001:00063390       ?SetPos@CProgressCtrl@@QAEHH@Z 00464390 f i ProgressDlg.obj
 0001:000633c0       ??0CPropertyViewDlg@@QAE@PAVCWnd@@@Z 004643c0 f   PropertyViewDlg.obj
 0001:000634f0       ??_GCPropertyViewDlg@@UAEPAXI@Z 004644f0 f i PropertyViewDlg.obj
 0001:000634f0       ??_ECPropertyViewDlg@@UAEPAXI@Z 004644f0 f i PropertyViewDlg.obj
 0001:00063520       ??1CPropertyViewDlg@@UAE@XZ 00464520 f i PropertyViewDlg.obj
 0001:00063610       ?DoDataExchange@CPropertyViewDlg@@MAEXPAVCDataExchange@@@Z 00464610 f   PropertyViewDlg.obj
 0001:000636d0       ?GetMessageMap@CPropertyViewDlg@@MBEPBUAFX_MSGMAP@@XZ 004646d0 f   PropertyViewDlg.obj
 0001:000636e0       ?GetThisMessageMap@CPropertyViewDlg@@KGPBUAFX_MSGMAP@@XZ 004646e0 f   PropertyViewDlg.obj
 0001:000636f0       ?OnBtnClose@CPropertyViewDlg@@IAEXXZ 004646f0 f   PropertyViewDlg.obj
 0001:00063740       ?OnBtnUpdate@CPropertyViewDlg@@IAEXXZ 00464740 f   PropertyViewDlg.obj
 0001:00063980       ?OnInitDialog@CPropertyViewDlg@@MAEHXZ 00464980 f   PropertyViewDlg.obj
 0001:000640c0       ?OnSelchangeTabProperty@CPropertyViewDlg@@IAEXPAUtagNMHDR@@PAJ@Z 004650c0 f   PropertyViewDlg.obj
 0001:00064160       ?InitListInfoDisplay1@CPropertyViewDlg@@QAEXXZ 00465160 f   PropertyViewDlg.obj
 0001:00065f70       ?InitListInfoDisplay@CPropertyViewDlg@@QAEXXZ 00466f70 f   PropertyViewDlg.obj
 0001:000679a0       ?RefreshPropertyInfo@CPropertyViewDlg@@QAEHXZ 004689a0 f   PropertyViewDlg.obj
 0001:00067c20       ?InsertHardwareListItem@CPropertyViewDlg@@QAEHHPBD00H@Z 00468c20 f   PropertyViewDlg.obj
 0001:00067ed0       ?InsertSoftwareListItem@CPropertyViewDlg@@QAEHHPADH@Z 00468ed0 f   PropertyViewDlg.obj
 0001:00068180       ?OnCloseProgressDlg@CPropertyViewDlg@@IAEJIJ@Z 00469180 f   PropertyViewDlg.obj
 0001:000681c0       ?OnProgressDlgCancel@CPropertyViewDlg@@IAEJIJ@Z 004691c0 f   PropertyViewDlg.obj
 0001:000681c0       ?OnPropertyHasUpdated@CPropertyViewDlg@@IAEJIJ@Z 004691c0 f   PropertyViewDlg.obj
 0001:000681e0       ?OnPropertyListRefresh@CPropertyViewDlg@@IAEJIJ@Z 004691e0 f   PropertyViewDlg.obj
 0001:00068200       ?OnCheckAuto@CPropertyViewDlg@@IAEXXZ 00469200 f   PropertyViewDlg.obj
 0001:00068250       ?OnSize@CPropertyViewDlg@@IAEXIHH@Z 00469250 f   PropertyViewDlg.obj
 0001:00068280       ?CondinateControlsPosition@CPropertyViewDlg@@QAEXXZ 00469280 f   PropertyViewDlg.obj
 0001:00068430       ?OnTimer@CPropertyViewDlg@@IAEXI@Z 00469430 f   PropertyViewDlg.obj
 0001:00068460       ?Create@CPropertyViewDlg@@QAEHPAVCWnd@@@Z 00469460 f   PropertyViewDlg.obj
 0001:000684e0       ?DestroyWindow@CPropertyViewDlg@@UAEHXZ 004694e0 f   PropertyViewDlg.obj
 0001:00068500       ?ReEnableParent@CPropertyViewDlg@@QAEXXZ 00469500 f   PropertyViewDlg.obj
 0001:00068540       ?Add@CImageList@@QAEHPAUHICON__@@@Z 00469540 f i PropertyViewDlg.obj
 0001:00068560       ?AfxImageList_ReplaceIcon@@YGHPAU_IMAGELIST@@HPAUHICON__@@@Z 00469560 f i PropertyViewDlg.obj
 0001:00068590       ?_ImageList_ReplaceIcon@CComCtlWrapper@@QAEHPAU_IMAGELIST@@HPAUHICON__@@@Z 00469590 f i PropertyViewDlg.obj
 0001:000686c0       ?GetProcAddress_ImageList_ReplaceIcon@CComCtlWrapper@@QAE?AUImageList_ReplaceIcon_Type@1@XZ 004696c0 f i PropertyViewDlg.obj
 0001:00068710       ??7ImageList_AddMasked_Type@CComCtlWrapper@@QBE_NXZ 00469710 f i CalendarBar.obj
 0001:00068710       ??7ImageList_SetBkColor_Type@CComCtlWrapper@@QBE_NXZ 00469710 f i WorkspaceBar.obj
 0001:00068710       ??7ImageList_GetImageInfo_Type@CComCtlWrapper@@QBE_NXZ 00469710 f i NewListCtrl.obj
 0001:00068710       ??7ImageList_ReplaceIcon_Type@CComCtlWrapper@@QBE_NXZ 00469710 f i PropertyViewDlg.obj
 0001:00068710       ??7ImageList_Draw_Type@CComCtlWrapper@@QBE_NXZ 00469710 f i CalendarBar.obj
 0001:00068730       ??0CTabCtrl@@QAE@XZ        00469730 f i PropertyViewDlg.obj
 0001:00068750       ??_ECTabCtrl@@UAEPAXI@Z    00469750 f i PropertyViewDlg.obj
 0001:00068750       ??_GCTabCtrl@@UAEPAXI@Z    00469750 f i PropertyViewDlg.obj
 0001:00068780       ?InsertItem@CTabCtrl@@QAEJHPBD@Z 00469780 f i PropertyViewDlg.obj
 0001:000687b0       ?GetCurSel@CTabCtrl@@QBEHXZ 004697b0 f i PropertyViewDlg.obj
 0001:000687e0       ?CreateObject@CPropertyViewUIThread@@SGPAVCObject@@XZ 004697e0 f   PropertyViewUIThread.obj
 0001:00068860       ?_GetBaseClass@CPropertyViewUIThread@@KGPAUCRuntimeClass@@XZ 00469860 f   PropertyViewUIThread.obj
 0001:00068870       ?GetThisClass@CPropertyViewUIThread@@SGPAUCRuntimeClass@@XZ 00469870 f   PropertyViewUIThread.obj
 0001:00068880       ?GetRuntimeClass@CPropertyViewUIThread@@UBEPAUCRuntimeClass@@XZ 00469880 f   PropertyViewUIThread.obj
 0001:00068890       ??0CPropertyViewUIThread@@IAE@XZ 00469890 f   PropertyViewUIThread.obj
 0001:00068900       ??_ECPropertyViewUIThread@@MAEPAXI@Z 00469900 f i PropertyViewUIThread.obj
 0001:00068900       ??_GCPropertyViewUIThread@@MAEPAXI@Z 00469900 f i PropertyViewUIThread.obj
 0001:00068930       ??1CPropertyViewUIThread@@MAE@XZ 00469930 f   PropertyViewUIThread.obj
 0001:00068990       ?InitInstance@CPropertyViewUIThread@@UAEHXZ 00469990 f   PropertyViewUIThread.obj
 0001:000689f0       ?ExitInstance@CPropertyViewUIThread@@UAEHXZ 004699f0 f   PropertyViewUIThread.obj
 0001:00068a20       ?GetMessageMap@CPropertyViewUIThread@@MBEPBUAFX_MSGMAP@@XZ 00469a20 f   PropertyViewUIThread.obj
 0001:00068a30       ?GetThisMessageMap@CPropertyViewUIThread@@KGPBUAFX_MSGMAP@@XZ 00469a30 f   PropertyViewUIThread.obj
 0001:00068a40       ?InsertColumn@CItemData@@QAEXH@Z 00469a40 f   ReportCtrl.obj
 0001:00068a90       ?DeleteColumn@CItemData@@QAEXH@Z 00469a90 f   ReportCtrl.obj
 0001:00068ac0       ?_IsDecNumber@_ITEM_COMPARE_FUNCS@@YAHABV?$CStringT@DV?$StrTraitMFC_DLL@DV?$ChTraitsCRT@D@ATL@@@@@ATL@@AAN@Z 00469ac0 f   ReportCtrl.obj
 0001:00068b30       ?_DecNumberCompare@_ITEM_COMPARE_FUNCS@@YAHNN@Z 00469b30 f   ReportCtrl.obj
 0001:00068b60       ?_IsHexNumber@_ITEM_COMPARE_FUNCS@@YAHABV?$CStringT@DV?$StrTraitMFC_DLL@DV?$ChTraitsCRT@D@ATL@@@@@ATL@@AAK@Z 00469b60 f   ReportCtrl.obj
 0001:00068bb0       ?_HexNumberCompare@_ITEM_COMPARE_FUNCS@@YAHKK@Z 00469bb0 f   ReportCtrl.obj
 0001:00068be0       ?_IsDate@_ITEM_COMPARE_FUNCS@@YAHABV?$CStringT@DV?$StrTraitMFC_DLL@DV?$ChTraitsCRT@D@ATL@@@@@ATL@@AAVCOleDateTime@3@@Z 00469be0 f   ReportCtrl.obj
 0001:00068c10       ?_DateCompare@_ITEM_COMPARE_FUNCS@@YAHABVCOleDateTime@ATL@@0@Z 00469c10 f   ReportCtrl.obj
 0001:00068c50       ??0CReportCtrl@@QAE@XZ     00469c50 f   ReportCtrl.obj
 0001:00068d70       ??_ECReportCtrl@@UAEPAXI@Z 00469d70 f i ReportCtrl.obj
 0001:00068d70       ??_GCReportCtrl@@UAEPAXI@Z 00469d70 f i ReportCtrl.obj
 0001:00068da0       ??1CReportCtrl@@UAE@XZ     00469da0 f   ReportCtrl.obj
 0001:00068e70       ?GetMessageMap@CReportCtrl@@MBEPBUAFX_MSGMAP@@XZ 00469e70 f   ReportCtrl.obj
 0001:00068e80       ?GetThisMessageMap@CReportCtrl@@KGPBUAFX_MSGMAP@@XZ 00469e80 f   ReportCtrl.obj
 0001:00068e90       ?OnCustomDraw@CReportCtrl@@IAEXPAUtagNMHDR@@PAJ@Z 00469e90 f   ReportCtrl.obj
 0001:00068f30       ?OnColumnclick@CReportCtrl@@IAEXPAUtagNMHDR@@PAJ@Z 00469f30 f   ReportCtrl.obj
 0001:00068f90       ?OnLButtonDown@CReportCtrl@@IAEXIVCPoint@@@Z 00469f90 f   ReportCtrl.obj
 0001:00068fc0       ?OnLButtonDblClk@CReportCtrl@@IAEXIVCPoint@@@Z 00469fc0 f   ReportCtrl.obj
 0001:00068ff0       ?OnMButtonDown@CReportCtrl@@IAEXIVCPoint@@@Z 00469ff0 f   ReportCtrl.obj
 0001:00069020       ?OnMButtonDblClk@CReportCtrl@@IAEXIVCPoint@@@Z 0046a020 f   ReportCtrl.obj
 0001:00069050       ?OnRButtonDown@CReportCtrl@@IAEXIVCPoint@@@Z 0046a050 f   ReportCtrl.obj
 0001:00069080       ?OnRButtonDblClk@CReportCtrl@@IAEXIVCPoint@@@Z 0046a080 f   ReportCtrl.obj
 0001:000690b0       ?OnCreate@CReportCtrl@@IAEHPAUtagCREATESTRUCTA@@@Z 0046a0b0 f   ReportCtrl.obj
 0001:00069110       ?OnDestroy@CReportCtrl@@IAEXXZ 0046a110 f   ReportCtrl.obj
 0001:00069160       ?_IsValidIndex@CReportCtrl@@IBEHH@Z 0046a160 f   ReportCtrl.obj
 0001:000691a0       ?DeleteItem@CReportCtrl@@QAEHHH@Z 0046a1a0 f   ReportCtrl.obj
 0001:00069200       ?DeleteAllItems@CReportCtrl@@QAEHK@Z 0046a200 f   ReportCtrl.obj
 0001:000692f0       ?SortItems@CReportCtrl@@QAEXHH@Z 0046a2f0 f   ReportCtrl.obj
 0001:00069400       ?SetItemText@CReportCtrl@@QAEHHHPBD@Z 0046a400 f   ReportCtrl.obj
 0001:00069440       ?GetColumnCount@CReportCtrl@@QBEHXZ 0046a440 f   ReportCtrl.obj
 0001:00069460       ?InsertItem@CReportCtrl@@QAEHHPBDH@Z 0046a460 f   ReportCtrl.obj
 0001:000694b0       ?InsertColumn@CReportCtrl@@QAEHHPBDHHH@Z 0046a4b0 f   ReportCtrl.obj
 0001:00069500       ?_IsEditVisible@CReportCtrl@@IBEHXZ 0046a500 f   ReportCtrl.obj
 0001:00069560       ?_ItemCheckMonitor@CReportCtrl@@IAEHHHHI@Z 0046a560 f   ReportCtrl.obj
 0001:00069640       ?SetExtendedStyle@CReportCtrl@@QAEKK@Z 0046a640 f   ReportCtrl.obj
 0001:00069670       ?PreCreateWindow@CReportCtrl@@MAEHAAUtagCREATESTRUCTA@@@Z 0046a670 f   ReportCtrl.obj
 0001:000696b0       ?PreTranslateMessage@CReportCtrl@@UAEHPAUtagMSG@@@Z 0046a6b0 f   ReportCtrl.obj
 0001:00069870       ?Create@CReportCtrl@@UAEHPAVCWnd@@IPBUtagRECT@@K@Z 0046a870 f   ReportCtrl.obj
 0001:000698e0       ?PreSubclassWindow@CReportCtrl@@MAEXXZ 0046a8e0 f   ReportCtrl.obj
 0001:00069940       ?IsSortable@CReportCtrl@@QBEHXZ 0046a940 f   ReportCtrl.obj
 0001:00069990       ?HasColumnHeader@CReportCtrl@@QBEHXZ 0046a990 f   ReportCtrl.obj
 0001:000699b0       ?_MouseClkMonitor@CReportCtrl@@IAEXIIVCPoint@@H@Z 0046a9b0 f   ReportCtrl.obj
 0001:00069b70       ?SetItemImage@CReportCtrl@@QAEHHHH@Z 0046ab70 f   ReportCtrl.obj
 0001:00069ba0       ?GetItemImage@CReportCtrl@@QBEHHH@Z 0046aba0 f   ReportCtrl.obj
 0001:00069bf0       ?SetImageList@CReportCtrl@@QAEPAVCImageList@@PAV2@@Z 0046abf0 f   ReportCtrl.obj
 0001:00069c10       ?GetImageList@CReportCtrl@@QBEPAVCImageList@@XZ 0046ac10 f   ReportCtrl.obj
 0001:00069c30       ?StartEdit@CReportCtrl@@QAEHHH@Z 0046ac30 f   ReportCtrl.obj
 0001:00069f00       ?EndEdit@CReportCtrl@@QAEHH@Z 0046af00 f   ReportCtrl.obj
 0001:0006a080       ?_UnsetSortedColumn@CReportCtrl@@IAEXXZ 0046b080 f   ReportCtrl.obj
 0001:0006a0b0       ?_GetHeaderTextFormat@CReportCtrl@@IBEKH@Z 0046b0b0 f   ReportCtrl.obj
 0001:0006a120       ?ExamItemStates@CReportCtrl@@QBEHHK@Z 0046b120 f   ReportCtrl.obj
 0001:0006a160       ?GetItemCount@CReportCtrl@@QBEHK@Z 0046b160 f   ReportCtrl.obj
 0001:0006a1d0       ?GetFirstItem@CReportCtrl@@QBEHKH@Z 0046b1d0 f   ReportCtrl.obj
 0001:0006a240       ?GetItemStates@CReportCtrl@@QBEKH@Z 0046b240 f   ReportCtrl.obj
 0001:0006a2d0       ?SetItemStates@CReportCtrl@@QAEHHK@Z 0046b2d0 f   ReportCtrl.obj
 0001:0006a310       ?SetAllItemStates@CReportCtrl@@QAEHKK@Z 0046b310 f   ReportCtrl.obj
 0001:0006a3b0       ?_EnsureSingleCheck@CReportCtrl@@IAEXH@Z 0046b3b0 f   ReportCtrl.obj
 0001:0006a440       ?_SetItemStatesNoVerify@CReportCtrl@@IAEHHK@Z 0046b440 f   ReportCtrl.obj
 0001:0006a520       ?GetHeaderCtrl@CReportCtrl@@QBEPBVCHeaderCtrl@@XZ 0046b520 f   ReportCtrl.obj
 0001:0006a550       ?_FreeItemMemory@CReportCtrl@@IAEXH@Z 0046b550 f   ReportCtrl.obj
 0001:0006a5b0       ??_GCItemData@@QAEPAXI@Z   0046b5b0 f i ReportCtrl.obj
 0001:0006a5e0       ??1CItemData@@QAE@XZ       0046b5e0 f i ReportCtrl.obj
 0001:0006a640       ?_AllocItemMemory@CReportCtrl@@IAEXH@Z 0046b640 f   ReportCtrl.obj
 0001:0006a760       ??0CItemData@@QAE@XZ       0046b760 f i ReportCtrl.obj
 0001:0006a7d0       ?_UpdateColumn@CReportCtrl@@IAEXHH@Z 0046b7d0 f   ReportCtrl.obj
 0001:0006a840       ?SetItemTextColor@CReportCtrl@@QAEXHHKH@Z 0046b840 f   ReportCtrl.obj
 0001:0006aa10       ?_PartialSort@CReportCtrl@@IAEHHH@Z 0046ba10 f   ReportCtrl.obj
 0001:0006adf0       ??_EROWINFO@@QAEPAXI@Z     0046bdf0 f i ReportCtrl.obj
 0001:0006ae60       ??0ROWINFO@@QAE@XZ         0046be60 f i ReportCtrl.obj
 0001:0006aec0       ??1ROWINFO@@QAE@XZ         0046bec0 f i ReportCtrl.obj
 0001:0006af20       ?_CompareItems@CReportCtrl@@IAEHHH@Z 0046bf20 f   ReportCtrl.obj
 0001:0006b110       ?_FindSeparator@CReportCtrl@@IBEHHH@Z 0046c110 f   ReportCtrl.obj
 0001:0006b1a0       ?_QuickSortRecursive@CReportCtrl@@IAEXPAHHH@Z 0046c1a0 f   ReportCtrl.obj
 0001:0006b310       ??0?$CArray@KK@@QAE@XZ     0046c310 f i ReportCtrl.obj
 0001:0006b360       ?InsertAt@?$CArray@KK@@QAEXHKH@Z 0046c360 f i ReportCtrl.obj
 0001:0006b4a0       ?memmove_s@Checked@ATL@@YAXPAXIPBXI@Z 0046c4a0 f i ReportCtrl.obj
 0001:0006b4d0       ?AfxCrtErrorCheck@@YAHH@Z  0046c4d0 f i ReportCtrl.obj
 0001:0006b580       ?RemoveAt@?$CArray@KK@@QAEXHH@Z 0046c580 f i ReportCtrl.obj
 0001:0006b640       ??0?$CArray@HH@@QAE@XZ     0046c640 f i ReportCtrl.obj
 0001:0006b690       ??A?$CArray@HH@@QAEAAHH@Z  0046c690 f i ReportCtrl.obj
 0001:0006b690       ??A?$CArray@KK@@QAEAAKH@Z  0046c690 f i ReportCtrl.obj
 0001:0006b6b0       ?ElementAt@?$CArray@KK@@QAEAAKH@Z 0046c6b0 f i ReportCtrl.obj
 0001:0006b6b0       ?ElementAt@?$CArray@HH@@QAEAAHH@Z 0046c6b0 f i ReportCtrl.obj
 0001:0006b6f0       ??4CRect@@QAEXABUtagRECT@@@Z 0046c6f0 f i ReportCtrl.obj
 0001:0006b710       ?DeflateRect@CRect@@QAEXHHHH@Z 0046c710 f i ReportCtrl.obj
 0001:0006b760       ??ACStringArray@@QAEAAV?$CStringT@DV?$StrTraitMFC_DLL@DV?$ChTraitsCRT@D@ATL@@@@@ATL@@H@Z 0046c760 f i ReportCtrl.obj
 0001:0006b780       ?ElementAt@CStringArray@@QAEAAV?$CStringT@DV?$StrTraitMFC_DLL@DV?$ChTraitsCRT@D@ATL@@@@@ATL@@H@Z 0046c780 f i ReportCtrl.obj
 0001:0006b7b0       ?LockWindowUpdate@CWnd@@QAEHXZ 0046c7b0 f i ReportCtrl.obj
 0001:0006b7d0       ?UnlockWindowUpdate@CWnd@@QAEXXZ 0046c7d0 f i ReportCtrl.obj
 0001:0006b7f0       ??0COleDateTime@ATL@@QAE@XZ 0046c7f0 f i ReportCtrl.obj
 0001:0006b810       ?GetSize@?$CArray@PAVCMFCRibbonBaseElement@@PAV1@@@QBEHXZ 0046c810 f i MainFrm.obj
 0001:0006b810       ?GetStatus@COleDateTime@ATL@@QBE?AW4DateTimeStatus@12@XZ 0046c810 f i ReportCtrl.obj
 0001:0006b830       ??MCOleDateTime@ATL@@QBE_NABV01@@Z 0046c830 f i ReportCtrl.obj
 0001:0006b8b0       ??OCOleDateTime@ATL@@QBE_NABV01@@Z 0046c8b0 f i ReportCtrl.obj
 0001:0006b930       ?DoubleFromDate@COleDateTime@ATL@@KGNN@Z 0046c930 f i ReportCtrl.obj
 0001:0006b970       ?ParseDateTime@COleDateTime@ATL@@QAE_NPBDKK@Z 0046c970 f i ReportCtrl.obj
 0001:0006bb60       ??$AtlMultiply@H@ATL@@YAJPAHHH@Z 0046cb60 f i ReportCtrl.obj
 0001:0006bbc0       ?_AtlVerifyStackAvailable@_ATL_SAFE_ALLOCA_IMPL@ATL@@YA_NK@Z 0046cbc0 f i ReportCtrl.obj
 0001:0006bca0       ?_AtlGetConversionACP@ATL@@YGIXZ 0046cca0 f i ReportCtrl.obj
 0001:0006bcb0       ?AtlA2WHelper@@YGPA_WPA_WPBDHI@Z 0046ccb0 f i ReportCtrl.obj
 0001:0006bd00       ?EnsureVisible@CListCtrl@@QAEHHH@Z 0046cd00 f i ReportCtrl.obj
 0001:0006bd30       ?GetItemCount@CHeaderCtrl@@QBEHXZ 0046cd30 f i ReportCtrl.obj
 0001:0006bd60       ?GetItem@CHeaderCtrl@@QBEHHPAU_HD_ITEMA@@@Z 0046cd60 f i ReportCtrl.obj
 0001:0006bd90       ?SubItemHitTest@CListCtrl@@QAEHPAUtagLVHITTESTINFO@@@Z 0046cd90 f i ReportCtrl.obj
 0001:0006bdc0       ??0?$CAtlSafeAllocBufferManager@VCCRTAllocator@ATL@@@_ATL_SAFE_ALLOCA_IMPL@ATL@@QAE@XZ 0046cdc0 f i ReportCtrl.obj
 0001:0006bdc0       ??0_Iterator_base_aux@std@@QAE@XZ 0046cdc0 f i KiboManagerView.obj
 0001:0006bde0       ?Allocate@?$CAtlSafeAllocBufferManager@VCCRTAllocator@ATL@@@_ATL_SAFE_ALLOCA_IMPL@ATL@@QAEPAXK@Z 0046cde0 f i ReportCtrl.obj
 0001:0006be30       ?Allocate@CCRTAllocator@ATL@@SAPAXI@Z 0046ce30 f i ReportCtrl.obj
 0001:0006be50       ??1?$CAtlSafeAllocBufferManager@VCCRTAllocator@ATL@@@_ATL_SAFE_ALLOCA_IMPL@ATL@@QAE@XZ 0046ce50 f i ReportCtrl.obj
 0001:0006be90       ?Free@CCRTAllocator@ATL@@SAXPAX@Z 0046ce90 f i ReportCtrl.obj
 0001:0006beb0       ?GetData@CAtlSafeAllocBufferNode@?$CAtlSafeAllocBufferManager@VCCRTAllocator@ATL@@@_ATL_SAFE_ALLOCA_IMPL@ATL@@QAEPAXXZ 0046ceb0 f i ReportCtrl.obj
 0001:0006beb0       ??BCCriticalSection@@QAEPAU_RTL_CRITICAL_SECTION@@XZ 0046ceb0 f i BootModuleManager.obj
 0001:0006bed0       ??$AtlAdd@K@ATL@@YAJPAKKK@Z 0046ced0 f i ReportCtrl.obj
 0001:0006bf00       ??1?$CArray@KK@@UAE@XZ     0046cf00 f i ReportCtrl.obj
 0001:0006bf60       ?Serialize@?$CArray@HH@@UAEXAAVCArchive@@@Z 0046cf60 f i ReportCtrl.obj
 0001:0006bf60       ?Serialize@?$CArray@KK@@UAEXAAVCArchive@@@Z 0046cf60 f i ReportCtrl.obj
 0001:0006bfd0       ??1?$CArray@HH@@UAE@XZ     0046cfd0 f i ReportCtrl.obj
 0001:0006c030       ??$AtlAddThrow@K@ATL@@YAKKK@Z 0046d030 f i ReportCtrl.obj
 0001:0006c070       ?AtlThrowImpl@ATL@@YGXJ@Z  0046d070 f i ReportCtrl.obj
 0001:0006c090       ??_G?$CArray@KK@@UAEPAXI@Z 0046d090 f i ReportCtrl.obj
 0001:0006c090       ??_E?$CArray@KK@@UAEPAXI@Z 0046d090 f i ReportCtrl.obj
 0001:0006c0c0       ??_E?$CArray@HH@@UAEPAXI@Z 0046d0c0 f i ReportCtrl.obj
 0001:0006c0c0       ??_G?$CArray@HH@@UAEPAXI@Z 0046d0c0 f i ReportCtrl.obj
 0001:0006c0f0       ?SetSize@?$CArray@HH@@QAEXHH@Z 0046d0f0 f i ReportCtrl.obj
 0001:0006c0f0       ?SetSize@?$CArray@KK@@QAEXHH@Z 0046d0f0 f i ReportCtrl.obj
 0001:0006c450       ?memcpy_s@Checked@ATL@@YAXPAXIPBXI@Z 0046d450 f i ReportCtrl.obj
 0001:0006c480       ?GetRuntimeClass@CSetClientchancelDLg@@UBEPAUCRuntimeClass@@XZ 0046d480 f   SetClientchancelDLg.obj
 0001:0006c490       ??0CSetClientchancelDLg@@QAE@PAVCWnd@@@Z 0046d490 f   SetClientchancelDLg.obj
 0001:0006c4d0       ??_ECSetClientchancelDLg@@UAEPAXI@Z 0046d4d0 f i SetClientchancelDLg.obj
 0001:0006c4d0       ??_GCSetClientchancelDLg@@UAEPAXI@Z 0046d4d0 f i SetClientchancelDLg.obj
 0001:0006c500       ??1CSetClientchancelDLg@@UAE@XZ 0046d500 f   SetClientchancelDLg.obj
 0001:0006c520       ?DoDataExchange@CPortChannelDlg@@MAEXPAVCDataExchange@@@Z 0046d520 f   PortChannelDlg.obj
 0001:0006c520       ?DoDataExchange@CSetClientchancelDLg@@MAEXPAVCDataExchange@@@Z 0046d520 f   SetClientchancelDLg.obj
 0001:0006c550       ?GetMessageMap@CSetClientchancelDLg@@MBEPBUAFX_MSGMAP@@XZ 0046d550 f   SetClientchancelDLg.obj
 0001:0006c560       ?GetThisMessageMap@CSetClientchancelDLg@@KGPBUAFX_MSGMAP@@XZ 0046d560 f   SetClientchancelDLg.obj
 0001:0006c570       ?OnBnClickedOk@CSetClientchancelDLg@@QAEXXZ 0046d570 f   SetClientchancelDLg.obj
 0001:0006c640       ?OnInitDialog@CSetClientchancelDLg@@UAEHXZ 0046d640 f   SetClientchancelDLg.obj
 0001:0006c760       ?GetRuntimeClass@CSetDrfaultNICDlg@@UBEPAUCRuntimeClass@@XZ 0046d760 f   SetDrfaultNICDlg.obj
 0001:0006c770       ??0CSetDrfaultNICDlg@@QAE@PAVCWnd@@@Z 0046d770 f   SetDrfaultNICDlg.obj
 0001:0006c820       ??_GCSetDrfaultNICDlg@@UAEPAXI@Z 0046d820 f i SetDrfaultNICDlg.obj
 0001:0006c820       ??_ECSetDrfaultNICDlg@@UAEPAXI@Z 0046d820 f i SetDrfaultNICDlg.obj
 0001:0006c850       ??1CSetDrfaultNICDlg@@UAE@XZ 0046d850 f   SetDrfaultNICDlg.obj
 0001:0006c8e0       ?DoDataExchange@CSetDrfaultNICDlg@@MAEXPAVCDataExchange@@@Z 0046d8e0 f   SetDrfaultNICDlg.obj
 0001:0006c940       ?GetMessageMap@CSetDrfaultNICDlg@@MBEPBUAFX_MSGMAP@@XZ 0046d940 f   SetDrfaultNICDlg.obj
 0001:0006c950       ?GetThisMessageMap@CSetDrfaultNICDlg@@KGPBUAFX_MSGMAP@@XZ 0046d950 f   SetDrfaultNICDlg.obj
 0001:0006c960       ?OnBnClickedOk@CSetDrfaultNICDlg@@QAEXXZ 0046d960 f   SetDrfaultNICDlg.obj
 0001:0006cad0       ?OnInitDialog@CSetDrfaultNICDlg@@UAEHXZ 0046dad0 f   SetDrfaultNICDlg.obj
 0001:0006cd10       ?GetLocalComputerInfo@CSetDrfaultNICDlg@@QAEHXZ 0046dd10 f   SetDrfaultNICDlg.obj
 0001:0006d010       ?SetTitle@CSetDrfaultNICDlg@@QAEXXZ 0046e010 f   SetDrfaultNICDlg.obj
 0001:0006d230       ?GetRuntimeClass@CSpecialPartitionRS@@UBEPAUCRuntimeClass@@XZ 0046e230 f   SpecialPartitionRS.obj
 0001:0006d240       ??0CSpecialPartitionRS@@QAE@PAVCWnd@@@Z 0046e240 f   SpecialPartitionRS.obj
 0001:0006d300       ??_ECSpecialPartitionRS@@UAEPAXI@Z 0046e300 f i SpecialPartitionRS.obj
 0001:0006d300       ??_GCSpecialPartitionRS@@UAEPAXI@Z 0046e300 f i SpecialPartitionRS.obj
 0001:0006d330       ??1CSpecialPartitionRS@@UAE@XZ 0046e330 f   SpecialPartitionRS.obj
 0001:0006d3a0       ?DoDataExchange@CSpecialPartitionRS@@MAEXPAVCDataExchange@@@Z 0046e3a0 f   SpecialPartitionRS.obj
 0001:0006d400       ?GetMessageMap@CSpecialPartitionRS@@MBEPBUAFX_MSGMAP@@XZ 0046e400 f   SpecialPartitionRS.obj
 0001:0006d410       ?GetThisMessageMap@CSpecialPartitionRS@@KGPBUAFX_MSGMAP@@XZ 0046e410 f   SpecialPartitionRS.obj
 0001:0006d420       ?OnInitDialog@CSpecialPartitionRS@@MAEHXZ 0046e420 f   SpecialPartitionRS.obj
 0001:0006d7f0       ?SetTitle@CSpecialPartitionRS@@QAEXXZ 0046e7f0 f   SpecialPartitionRS.obj
 0001:0006d970       ?IntiListCtrl@CSpecialPartitionRS@@QAEXXZ 0046e970 f   SpecialPartitionRS.obj
 0001:0006dec0       ?OnDblclkPartitionList@CSpecialPartitionRS@@IAEXPAUtagNMHDR@@PAJ@Z 0046eec0 f   SpecialPartitionRS.obj
 0001:0006e0e0       ?GetFileSystemType@CSpecialPartitionRS@@QAE?AV?$CStringT@DV?$StrTraitMFC_DLL@DV?$ChTraitsCRT@D@ATL@@@@@ATL@@E@Z 0046f0e0 f   SpecialPartitionRS.obj
 0001:0006e2a0       ?OnOK@CSpecialPartitionRS@@MAEXXZ 0046f2a0 f   SpecialPartitionRS.obj
 0001:0006e6a0       ?GetPartitionProtectType@CSpecialPartitionRS@@QAEEE@Z 0046f6a0 f   SpecialPartitionRS.obj
 0001:0006e750       ?OnBnClickedCancel@CSpecialPartitionRS@@QAEXXZ 0046f750 f   SpecialPartitionRS.obj
 0001:0006e750       ?OnBnClickedCancel@CClientSettingsDlg@@QAEXXZ 0046f750 f   ClientSettingsDlg.obj
 0001:0006e780       ??0CWait@@QAE@PAVCWnd@@@Z  0046f780 f   Wait.obj
 0001:0006e850       ??_ECWait@@UAEPAXI@Z       0046f850 f i Wait.obj
 0001:0006e850       ??_GCWait@@UAEPAXI@Z       0046f850 f i Wait.obj
 0001:0006e880       ??1CWait@@UAE@XZ           0046f880 f   Wait.obj
 0001:0006e920       ?DoDataExchange@CWait@@MAEXPAVCDataExchange@@@Z 0046f920 f   Wait.obj
 0001:0006e960       ?GetMessageMap@CWait@@MBEPBUAFX_MSGMAP@@XZ 0046f960 f   Wait.obj
 0001:0006e970       ?GetThisMessageMap@CWait@@KGPBUAFX_MSGMAP@@XZ 0046f970 f   Wait.obj
 0001:0006e980       ?OnInitDialog@CWait@@MAEHXZ 0046f980 f   Wait.obj
 0001:0006eaf0       ?OnTimer@CWait@@IAEXI@Z    0046faf0 f   Wait.obj
 0001:0006ee00       ?OnDestroy@CWait@@IAEXXZ   0046fe00 f   Wait.obj
 0001:0006ee50       ?PreTranslateMessage@CWait@@UAEHPAUtagMSG@@@Z 0046fe50 f   Wait.obj
 0001:0006ee90       ?GetSystemMenu@CWnd@@QBEPAVCMenu@@H@Z 0046fe90 f i Wait.obj
 0001:0006eec0       ?GetMessageMap@CWorkspaceBar@@MBEPBUAFX_MSGMAP@@XZ 0046fec0 f   WorkspaceBar.obj
 0001:0006eed0       ?GetThisMessageMap@CWorkspaceBar@@KGPBUAFX_MSGMAP@@XZ 0046fed0 f   WorkspaceBar.obj
 0001:0006eee0       ??0CWorkspaceBar@@QAE@XZ   0046fee0 f   WorkspaceBar.obj
 0001:0006ef50       ??_ECWorkspaceBar@@UAEPAXI@Z 0046ff50 f i WorkspaceBar.obj
 0001:0006ef50       ??_GCWorkspaceBar@@UAEPAXI@Z 0046ff50 f i WorkspaceBar.obj
 0001:0006ef80       ??1CWorkspaceBar@@UAE@XZ   0046ff80 f   WorkspaceBar.obj
 0001:0006eff0       ?OnCreate@CWorkspaceBar@@IAEHPAUtagCREATESTRUCTA@@@Z 0046fff0 f   WorkspaceBar.obj
 0001:0006f270       ?OnSize@CWorkspaceBar@@IAEXIHH@Z 00470270 f   WorkspaceBar.obj
 0001:0006f2d0       ?OnPaint@CWorkspaceBar2@@IAEXXZ 004702d0 f   WorkspaceBar2.obj
 0001:0006f2d0       ?OnPaint@CWorkspaceBar@@IAEXXZ 004702d0 f   WorkspaceBar.obj
 0001:0006f3a0       ?InflateRect@CRect@@QAEXHH@Z 004703a0 f i WorkspaceBar.obj
 0001:0006f3c0       ?SetBkColor@CImageList@@QAEKK@Z 004703c0 f i WorkspaceBar.obj
 0001:0006f3e0       ?AfxImageList_SetBkColor@@YGKPAU_IMAGELIST@@K@Z 004703e0 f i WorkspaceBar.obj
 0001:0006f410       ?_ImageList_SetBkColor@CComCtlWrapper@@QAEKPAU_IMAGELIST@@K@Z 00470410 f i WorkspaceBar.obj
 0001:0006f540       ?GetProcAddress_ImageList_SetBkColor@CComCtlWrapper@@QAE?AUImageList_SetBkColor_Type@1@XZ 00470540 f i WorkspaceBar.obj
 0001:0006f590       ??4ImageList_GetImageInfo_Type@CComCtlWrapper@@QAEXP6GHPAU_IMAGELIST@@HPAU_IMAGEINFO@@@Z@Z 00470590 f i NewListCtrl.obj
 0001:0006f590       ??4ImageList_Draw_Type@CComCtlWrapper@@QAEXP6GHPAU_IMAGELIST@@HPAUHDC__@@HHI@Z@Z 00470590 f i CalendarBar.obj
 0001:0006f590       ??4ImageList_SetBkColor_Type@CComCtlWrapper@@QAEXP6GKPAU_IMAGELIST@@K@Z@Z 00470590 f i WorkspaceBar.obj
 0001:0006f590       ??4ImageList_ReplaceIcon_Type@CComCtlWrapper@@QAEXP6GHPAU_IMAGELIST@@HPAUHICON__@@@Z@Z 00470590 f i PropertyViewDlg.obj
 0001:0006f590       ??4ImageList_AddMasked_Type@CComCtlWrapper@@QAEXP6GHPAU_IMAGELIST@@PAUHBITMAP__@@K@Z@Z 00470590 f i CalendarBar.obj
 0001:0006f5b0       ?LoadIconA@CWinApp@@QBEPAUHICON__@@I@Z 004705b0 f i WorkspaceBar.obj
 0001:0006f5e0       ?Expand@CTreeCtrl@@QAEHPAU_TREEITEM@@I@Z 004705e0 f i WorkspaceBar.obj
 0001:0006f610       ?SetImageList@CTreeCtrl@@QAEPAVCImageList@@PAV2@H@Z 00470610 f i WorkspaceBar.obj
 0001:0006f650       ?GetMessageMap@CWorkspaceBar2@@MBEPBUAFX_MSGMAP@@XZ 00470650 f   WorkspaceBar2.obj
 0001:0006f660       ?GetThisMessageMap@CWorkspaceBar2@@KGPBUAFX_MSGMAP@@XZ 00470660 f   WorkspaceBar2.obj
 0001:0006f670       ??0CWorkspaceBar2@@QAE@XZ  00470670 f   WorkspaceBar2.obj
 0001:0006f6e0       ??_ECWorkspaceBar2@@UAEPAXI@Z 004706e0 f i WorkspaceBar2.obj
 0001:0006f6e0       ??_GCWorkspaceBar2@@UAEPAXI@Z 004706e0 f i WorkspaceBar2.obj
 0001:0006f710       ??1CWorkspaceBar2@@UAE@XZ  00470710 f   WorkspaceBar2.obj
 0001:0006f780       ?OnCreate@CWorkspaceBar2@@IAEHPAUtagCREATESTRUCTA@@@Z 00470780 f   WorkspaceBar2.obj
 0001:0006f840       ?OnSize@CWorkspaceBar2@@IAEXIHH@Z 00470840 f   WorkspaceBar2.obj
 0001:0006f890       ?GetCurrentPath@@YAHXZ     00470890 f   comfunc:comfunc.obj
 0001:0006f960       ?SetLogFile@@YAHPBD@Z      00470960 f   comfunc:comfunc.obj
 0001:0006fa10       _AlreadyRunning            00470a10 f   comfunc:comfunc.obj
 0001:0006fa50       _ExReBoot                  00470a50 f   comfunc:comfunc.obj
 0001:0006fb40       _ExIsVista                 00470b40 f   comfunc:comfunc.obj
 0001:0006fbb0       _WriteRunLog               00470bb0 f   comfunc:comfunc.obj
 0001:0006fdd0       ?IsNtSys@@YAHXZ            00470dd0 f   comfunc:comfunc.obj
 0001:0006fe80       _InitComFunc               00470e80 f   comfunc:comfunc.obj
 0001:0006ff00       ?ExtractProcessName@@YA?AV?$CStringT@DV?$StrTraitMFC_DLL@DV?$ChTraitsCRT@D@ATL@@@@@ATL@@PAD@Z 00470f00 f   comfunc:comfunc.obj
 0001:0006ff50       _GetProcessIdFromName      00470f50 f   comfunc:comfunc.obj
 0001:00070030       ??0CRegistry@@QAE@XZ       00471030 f   comfunc:Registry.obj
 0001:00070060       ?ClearKey@CRegistry@@QAEHXZ 00471060 f   comfunc:Registry.obj
 0001:00070080       ?SetRootKey@CRegistry@@QAEHPAUHKEY__@@@Z 00471080 f   comfunc:Registry.obj
 0001:000700b0       ?DeleteValue@CRegistry@@QAEHV?$CStringT@DV?$StrTraitMFC_DLL@DV?$ChTraitsCRT@D@ATL@@@@@ATL@@@Z 004710b0 f   comfunc:Registry.obj
 0001:00070120       ?GetDataType@CRegistry@@QAEKV?$CStringT@DV?$StrTraitMFC_DLL@DV?$ChTraitsCRT@D@ATL@@@@@ATL@@@Z 00471120 f   comfunc:Registry.obj
 0001:000701b0       ?KeyExists@CRegistry@@QAEHV?$CStringT@DV?$StrTraitMFC_DLL@DV?$ChTraitsCRT@D@ATL@@@@@ATL@@PAUHKEY__@@@Z 004711b0 f   comfunc:Registry.obj
 0001:00070210       ?SetKey@CRegistry@@QAEHV?$CStringT@DV?$StrTraitMFC_DLL@DV?$ChTraitsCRT@D@ATL@@@@@ATL@@H@Z 00471210 f   comfunc:Registry.obj
 0001:00070360       ?ReadString@CRegistry@@QAE?AV?$CStringT@DV?$StrTraitMFC_DLL@DV?$ChTraitsCRT@D@ATL@@@@@ATL@@V23@0@Z 00471360 f   comfunc:Registry.obj
 0001:000704c0       ?ReadDword@CRegistry@@QAEKV?$CStringT@DV?$StrTraitMFC_DLL@DV?$ChTraitsCRT@D@ATL@@@@@ATL@@K@Z 004714c0 f   comfunc:Registry.obj
 0001:00070570       ?ReadBool@CRegistry@@QAEHV?$CStringT@DV?$StrTraitMFC_DLL@DV?$ChTraitsCRT@D@ATL@@@@@ATL@@H@Z 00471570 f   comfunc:Registry.obj
 0001:00070620       ?WriteBool@CRegistry@@QAEHV?$CStringT@DV?$StrTraitMFC_DLL@DV?$ChTraitsCRT@D@ATL@@@@@ATL@@H@Z 00471620 f   comfunc:Registry.obj
 0001:000706c0       ?WriteString@CRegistry@@QAEHV?$CStringT@DV?$StrTraitMFC_DLL@DV?$ChTraitsCRT@D@ATL@@@@@ATL@@0@Z 004716c0 f   comfunc:Registry.obj
 0001:000707e0       ?WriteDword@CRegistry@@QAEHV?$CStringT@DV?$StrTraitMFC_DLL@DV?$ChTraitsCRT@D@ATL@@@@@ATL@@K@Z 004717e0 f   comfunc:Registry.obj
 0001:00070880       ?WriteBinary@CRegistry@@QAEHV?$CStringT@DV?$StrTraitMFC_DLL@DV?$ChTraitsCRT@D@ATL@@@@@ATL@@PAEH@Z 00471880 f   comfunc:Registry.obj
 0001:00070920       ?ReadBinary@CRegistry@@QAEHV?$CStringT@DV?$StrTraitMFC_DLL@DV?$ChTraitsCRT@D@ATL@@@@@ATL@@PAEK@Z 00471920 f   comfunc:Registry.obj
 0001:000709c0       ?ReadMSZString@CRegistry@@QAEHV?$CStringT@DV?$StrTraitMFC_DLL@DV?$ChTraitsCRT@D@ATL@@@@@ATL@@PAD@Z 004719c0 f   comfunc:Registry.obj
 0001:00070b10       ??1CRegistry@@QAE@XZ       00471b10 f   comfunc:Registry.obj
 0001:00070b30       ?DeleteKey@CRegistry@@QAEHV?$CStringT@DV?$StrTraitMFC_DLL@DV?$ChTraitsCRT@D@ATL@@@@@ATL@@@Z 00471b30 f   comfunc:Registry.obj
 0001:00070be0       ?TranStrToNode@@YAHPAE0@Z  00471be0 f   helpful:helpful.obj
 0001:00070d10       ?TranNodeToStr@@YAHPAE0@Z  00471d10 f   helpful:helpful.obj
 0001:00070d50       ?SetTTL@CMulticastSocket@@QAEHI@Z 00471d50 f   commod2:MulticastSocket.obj
 0001:00070d80       ?SetLoopBack@CMulticastSocket@@QAEHH@Z 00471d80 f   commod2:MulticastSocket.obj
 0001:00070db0       ?JoinGroup@CMulticastSocket@@QAEHV?$CStringT@DV?$StrTraitMFC_DLL@DV?$ChTraitsCRT@D@ATL@@@@@ATL@@PBD@Z 00471db0 f   commod2:MulticastSocket.obj
 0001:00070e20       ?LeaveGroup@CMulticastSocket@@QAEHXZ 00471e20 f   commod2:MulticastSocket.obj
 0001:00070e40       ?CommSecrect@CMulticastSocket@@QAEXPAEG@Z 00471e40 f   commod2:MulticastSocket.obj
 0001:00070e60       ?SendToSingle@CMulticastSocket@@QAEHPAD0GK@Z 00471e60 f   commod2:MulticastSocket.obj
 0001:00070f30       ??1?$CTypedPtrList@VCPtrList@@PAUtagUDPRECV@@@@UAE@XZ 00471f30 f i commod2:MulticastSocket.obj
 0001:00070f30       ??1?$CTypedPtrList@VCPtrList@@PAUSTRUCT_PROTECTITEM@@@@UAE@XZ 00471f30 f i kibokern:kibokern.obj
 0001:00070f40       ?CreateReceivingSocket@CMulticastSocket@@QAEHPAVCWnd@@PBDG1@Z 00471f40 f   commod2:MulticastSocket.obj
 0001:000710a0       ?CreateSendingSocket@CMulticastSocket@@QAEHIHPBD@Z 004720a0 f   commod2:MulticastSocket.obj
 0001:000711c0       ?Receive@CMulticastSocket@@QAEHXZ 004721c0 f   commod2:MulticastSocket.obj
 0001:00071270       ?SendToGroup@CMulticastSocket@@QAEHPADH@Z 00472270 f   commod2:MulticastSocket.obj
 0001:00071340       ?Initial@CMulticastSocket@@QAEHPAVCWnd@@V?$CStringT@DV?$StrTraitMFC_DLL@DV?$ChTraitsCRT@D@ATL@@@@@ATL@@GPBDIHH@Z 00472340 f   commod2:MulticastSocket.obj
 0001:00071400       ??_E?$CTypedPtrList@VCPtrList@@PAUSTRUCT_PROTECTITEM@@@@UAEPAXI@Z 00472400 f i kibokern:kibokern.obj
 0001:00071400       ??_E?$CTypedPtrList@VCPtrList@@PAUtagUDPRECV@@@@UAEPAXI@Z 00472400 f i commod2:MulticastSocket.obj
 0001:00071400       ??_G?$CTypedPtrList@VCPtrList@@PAUSTRUCT_PROTECTITEM@@@@UAEPAXI@Z 00472400 f i kibokern:kibokern.obj
 0001:00071400       ??_G?$CTypedPtrList@VCPtrList@@PAUtagUDPRECV@@@@UAEPAXI@Z 00472400 f i commod2:MulticastSocket.obj
 0001:00071420       ??0CMulticastSocket@@QAE@XZ 00472420 f   commod2:MulticastSocket.obj
 0001:000714e0       ?CloseSocket@CMulticastSocket@@QAEXXZ 004724e0 f   commod2:MulticastSocket.obj
 0001:00071540       ??1CMulticastSocket@@UAE@XZ 00472540 f   commod2:MulticastSocket.obj
 0001:000715b0       ??_ECMulticastSocket@@UAEPAXI@Z 004725b0 f i commod2:MulticastSocket.obj
 0001:000715b0       ??_GCMulticastSocket@@UAEPAXI@Z 004725b0 f i commod2:MulticastSocket.obj
 0001:000715d0       ??0CODBCSet@@QAE@XZ        004725d0 f   dbmod2:MyODBC.obj
 0001:000715f0       ??1CODBCSet@@UAE@XZ        004725f0 f   dbmod2:MyODBC.obj
 0001:00071600       ?IsEmpty@CODBCSet@@QAEHXZ  00472600 f   dbmod2:MyODBC.obj
 0001:00071610       ?Empty@CODBCSet@@QAEXXZ    00472610 f   dbmod2:MyODBC.obj
 0001:00071680       ?GetCols@CODBCSet@@QAE?BHXZ 00472680 f   dbmod2:MyODBC.obj
 0001:00071690       ??0CMyODBC@@QAE@XZ         00472690 f   dbmod2:MyODBC.obj
 0001:000716b0       ?DisConnect@CMyODBC@@QAEHXZ 004726b0 f   dbmod2:MyODBC.obj
 0001:00071710       ?GetDefaultCType@CMyODBC@@QAEFJ@Z 00472710 f   dbmod2:MyODBC.obj
 0001:000717d0       ?GetColLength@CMyODBC@@QAEJAAPAXHH@Z 004727d0 f   dbmod2:MyODBC.obj
 0001:00071940       ?ReportError@CMyODBC@@QAEXAAPAXHV?$CStringT@DV?$StrTraitMFC_DLL@DV?$ChTraitsCRT@D@ATL@@@@@ATL@@@Z 00472940 f   dbmod2:MyODBC.obj
 0001:00071a80       ?ConvertDataToChar@CMyODBC@@QAEHXZ 00472a80 f   dbmod2:MyODBC.obj
 0001:00071b90       ?SetODBCSource@CMyODBC@@QAEHPAD0@Z 00472b90 f   dbmod2:MyODBC.obj
 0001:00071cc0       ??_GCODBCSet@@UAEPAXI@Z    00472cc0 f i dbmod2:MyODBC.obj
 0001:00071cc0       ??_ECODBCSet@@UAEPAXI@Z    00472cc0 f i dbmod2:MyODBC.obj
 0001:00071ce0       ??1CMyODBC@@UAE@XZ         00472ce0 f   dbmod2:MyODBC.obj
 0001:00071cf0       ?ConnectDB@CMyODBC@@QAEHPBD00@Z 00472cf0 f   dbmod2:MyODBC.obj
 0001:00071e00       ?ExeSqlDirect@CMyODBC@@QAEHPBD@Z 00472e00 f   dbmod2:MyODBC.obj
 0001:00071ea0       ?PrepareSql@CMyODBC@@QAEHPBDAAVCODBCSet@@@Z 00472ea0 f   dbmod2:MyODBC.obj
 0001:000723d0       ?FetchData@CMyODBC@@QAEHXZ 004733d0 f   dbmod2:MyODBC.obj
 0001:00072410       ?ExecTrans@CMyODBC@@QAEHAAVCStringList@@@Z 00473410 f   dbmod2:MyODBC.obj
 0001:000725e0       ??_GCMyODBC@@UAEPAXI@Z     004735e0 f i dbmod2:MyODBC.obj
 0001:000725e0       ??_ECMyODBC@@UAEPAXI@Z     004735e0 f i dbmod2:MyODBC.obj
 0001:000725fe       _InitLogSystem             004735fe f   RCLogSystem:RCLogSystem.dll
 0001:00072604       _AddOneLogRecord           00473604 f   RCLogSystem:RCLogSystem.dll
 0001:0007260a       _EndLogSystem              0047360a f   RCLogSystem:RCLogSystem.dll
 0001:00072610       _ShowLogManager            00473610 f   RCLogSystem:RCLogSystem.dll
 0001:00072620       ?descryptparasector@CKiboKern@@AAEXXZ 00473620 f   kibokern:kibokern.obj
 0001:000726e0       ?encryptparasector@CKiboKern@@AAEXXZ 004736e0 f   kibokern:kibokern.obj
 0001:000727a0       ?WriteParaSector@CKiboKern@@QAEXXZ 004737a0 f   kibokern:kibokern.obj
 0001:00072820       ?LoadParaSector@CKiboKern@@QAEHXZ 00473820 f   kibokern:kibokern.obj
 0001:00072900       ?InitKern@CKiboKern@@QAEHXZ 00473900 f   kibokern:kibokern.obj
 0001:00072b80       ??0CKiboKern@@QAE@XZ       00473b80 f   kibokern:kibokern.obj
 0001:00072bb0       ??1CKiboKern@@UAE@XZ       00473bb0 f   kibokern:kibokern.obj
 0001:00072c60       ??_GCKiboKern@@UAEPAXI@Z   00473c60 f i kibokern:kibokern.obj
 0001:00072c60       ??_ECKiboKern@@UAEPAXI@Z   00473c60 f i kibokern:kibokern.obj
 0001:00072c7e       _WTSRegisterSessionNotification@8 00473c7e f   WtsApi32:WTSAPI32.dll
 0001:00072c84       _WTSUnRegisterSessionNotification@4 00473c84 f   WtsApi32:WTSAPI32.dll
 0001:00072c90       ?SetBasicPath@@YAXPBD@Z    00473c90 f   loadres:exloadres.obj
 0001:00072cb0       ?ExGetResString@@YA?AV?$CStringT@DV?$StrTraitMFC_DLL@DV?$ChTraitsCRT@D@ATL@@@@@ATL@@PAD0@Z 00473cb0 f   loadres:exloadres.obj
 0001:00072dc0       ?ExGetResBmp@@YA?AV?$CStringT@DV?$StrTraitMFC_DLL@DV?$ChTraitsCRT@D@ATL@@@@@ATL@@PAD0@Z 00473dc0 f   loadres:exloadres.obj
 0001:00072f50       ?ExCheckAllRes@@YAHPBD@Z   00473f50 f   loadres:exloadres.obj
 0001:00073480       ??0CIniStruct@@QAE@XZ      00474480 f   loadres:initwork.obj
 0001:00073490       ?addsection@CIniStruct@@QAEHPAD@Z 00474490 f   loadres:initwork.obj
 0001:000735c0       ?sectionkey@CIniStruct@@QAEPADH@Z 004745c0 f   loadres:initwork.obj
 0001:000735d0       ?sectionvalue@CIniStruct@@QAEPADH@Z 004745d0 f   loadres:initwork.obj
 0001:000735e0       ?GetCount@CIniStruct@@QAEHXZ 004745e0 f   loadres:initwork.obj
 0001:000735f0       ?Release@CIniStruct@@QAEHXZ 004745f0 f   loadres:initwork.obj
 0001:00073650       ??1CIniStruct@@QAE@XZ      00474650 f   loadres:initwork.obj
 0001:00073660       ?ReadProfileSection@@YAKPBD0AAVCIniStruct@@@Z 00474660 f   loadres:initwork.obj
 0001:00073790       ??HATL@@YA?AV?$CStringT@DV?$StrTraitMFC_DLL@DV?$ChTraitsCRT@D@ATL@@@@@0@ABV10@0@Z 00474790 f i loadres:initwork.obj
 0001:00073830       ?replacestr@@YAXPAD00@Z    00474830 f   loadres:initwork.obj
 0001:000739b0       ?ReadProfileReplace@@YAKPBDAAVCIniStruct@@@Z 004749b0 f   loadres:initwork.obj
 0001:00073af0       ?ReadIniFileKey@@YAAAV?$CStringT@DV?$StrTraitMFC_DLL@DV?$ChTraitsCRT@D@ATL@@@@@ATL@@PBD0PADAAV12@@Z 00474af0 f   loadres:initwork.obj
 0001:00073ceb       __imp_load__DwmEnableComposition@4 00474ceb     dwmapi:dwmapi.dll
 0001:00073cf5       __tailMerge_dwmapi_dll     00474cf5     dwmapi:dwmapi.dll
 0001:00073d06       ___delayLoadHelper2@8      00474d06 f   DelayImp:delayhlp.obj
 0001:00073f44       ??3@YAXPAX@Z               00474f44 f   mfc90:mfc90.dll
 0001:00073f4a       ?GetThisClass@CDialog@@SGPAUCRuntimeClass@@XZ 00474f4a f   mfc90:mfc90.dll
 0001:00073f50       ??1CStatic@@UAE@XZ         00474f50 f   mfc90:mfc90.dll
 0001:00073f56       ??1CDialog@@UAE@XZ         00474f56 f   mfc90:mfc90.dll
 0001:00073f5c       ??0CDialog@@QAE@IPAVCWnd@@@Z 00474f5c f   mfc90:mfc90.dll
 0001:00073f62       ?OnCmdMsg@CDialog@@UAEHIHPAXPAUAFX_CMDHANDLERINFO@@@Z 00474f62 f   mfc90:mfc90.dll
 0001:00073f68       ?OnFinalRelease@CWnd@@UAEXXZ 00474f68 f   mfc90:mfc90.dll
 0001:00073f6e       ?IsInvokeAllowed@CCmdTarget@@UAEHJ@Z 00474f6e f   mfc90:mfc90.dll
 0001:00073f74       ?GetDispatchIID@CCmdTarget@@UAEHPAU_GUID@@@Z 00474f74 f   mfc90:mfc90.dll
 0001:00073f7a       ?GetTypeInfoCount@CCmdTarget@@UAEIXZ 00474f7a f   mfc90:mfc90.dll
 0001:00073f80       ?GetTypeLibCache@CCmdTarget@@UAEPAVCTypeLibCache@@XZ 00474f80 f   mfc90:mfc90.dll
 0001:00073f86       ?GetTypeLib@CCmdTarget@@UAEJKPAPAUITypeLib@@@Z 00474f86 f   mfc90:mfc90.dll
 0001:00073f8c       ?GetCommandMap@CCmdTarget@@MBEPBUAFX_OLECMDMAP@@XZ 00474f8c f   mfc90:mfc90.dll
 0001:00073f92       ?GetDispatchMap@CCmdTarget@@MBEPBUAFX_DISPMAP@@XZ 00474f92 f   mfc90:mfc90.dll
 0001:00073f98       ?GetConnectionMap@CCmdTarget@@MBEPBUAFX_CONNECTIONMAP@@XZ 00474f98 f   mfc90:mfc90.dll
 0001:00073f9e       ?GetInterfaceMap@CWnd@@MBEPBUAFX_INTERFACEMAP@@XZ 00474f9e f   mfc90:mfc90.dll
 0001:00073fa4       ?GetEventSinkMap@CCmdTarget@@MBEPBUAFX_EVENTSINKMAP@@XZ 00474fa4 f   mfc90:mfc90.dll
 0001:00073faa       ?OnCreateAggregates@CCmdTarget@@UAEHXZ 00474faa f   mfc90:mfc90.dll
 0001:00073fb0       ?GetInterfaceHook@CCmdTarget@@UAEPAUIUnknown@@PBX@Z 00474fb0 f   mfc90:mfc90.dll
 0001:00073fb6       ?GetExtraConnectionPoints@CCmdTarget@@MAEHPAVCPtrArray@@@Z 00474fb6 f   mfc90:mfc90.dll
 0001:00073fbc       ?GetConnectionHook@CCmdTarget@@MAEPAUIConnectionPoint@@ABU_GUID@@@Z 00474fbc f   mfc90:mfc90.dll
 0001:00073fc2       ?PreSubclassWindow@CWnd@@UAEXXZ 00474fc2 f   mfc90:mfc90.dll
 0001:00073fc8       ?Create@CWnd@@UAEHPBD0KABUtagRECT@@PAV1@IPAUCCreateContext@@@Z 00474fc8 f   mfc90:mfc90.dll
 0001:00073fce       ?CreateEx@CWnd@@UAEHKPBD0KABUtagRECT@@PAV1@IPAX@Z 00474fce f   mfc90:mfc90.dll
 0001:00073fd4       ?CreateEx@CWnd@@UAEHKPBD0KHHHHPAUHWND__@@PAUHMENU__@@PAX@Z 00474fd4 f   mfc90:mfc90.dll
 0001:00073fda       ?DestroyWindow@CWnd@@UAEHXZ 00474fda f   mfc90:mfc90.dll
 0001:00073fe0       ?PreCreateWindow@CWnd@@UAEHAAUtagCREATESTRUCTA@@@Z 00474fe0 f   mfc90:mfc90.dll
 0001:00073fe6       ?CalcWindowRect@CWnd@@UAEXPAUtagRECT@@I@Z 00474fe6 f   mfc90:mfc90.dll
 0001:00073fec       ?GetMenu@CWnd@@UBEPAVCMenu@@XZ 00474fec f   mfc90:mfc90.dll
 0001:00073ff2       ?SetMenu@CWnd@@UAEHPAVCMenu@@@Z 00474ff2 f   mfc90:mfc90.dll
 0001:00073ff8       ?OnToolHitTest@CWnd@@UBEHVCPoint@@PAUtagTOOLINFOA@@@Z 00474ff8 f   mfc90:mfc90.dll
 0001:00073ffe       ?GetScrollBarCtrl@CWnd@@UBEPAVCScrollBar@@H@Z 00474ffe f   mfc90:mfc90.dll
 0001:00074004       ?WinHelpA@CWnd@@UAEXKI@Z   00475004 f   mfc90:mfc90.dll
 0001:0007400a       ?HtmlHelpA@CWnd@@UAEXKI@Z  0047500a f   mfc90:mfc90.dll
 0001:00074010       ?WinHelpInternal@CWnd@@UAEXKI@Z 00475010 f   mfc90:mfc90.dll
 0001:00074016       ?ContinueModal@CWnd@@UAEHXZ 00475016 f   mfc90:mfc90.dll
 0001:0007401c       ?EndModalLoop@CWnd@@UAEXH@Z 0047501c f   mfc90:mfc90.dll
 0001:00074022       ?EnsureStdObj@CWnd@@UAEJXZ 00475022 f   mfc90:mfc90.dll
 0001:00074028       ?get_accParent@CWnd@@UAEJPAPAUIDispatch@@@Z 00475028 f   mfc90:mfc90.dll
 0001:0007402e       ?get_accChildCount@CWnd@@UAEJPAJ@Z 0047502e f   mfc90:mfc90.dll
 0001:00074034       ?get_accChild@CWnd@@UAEJUtagVARIANT@@PAPAUIDispatch@@@Z 00475034 f   mfc90:mfc90.dll
 0001:0007403a       ?get_accName@CWnd@@UAEJUtagVARIANT@@PAPA_W@Z 0047503a f   mfc90:mfc90.dll
 0001:00074040       ?get_accValue@CWnd@@UAEJUtagVARIANT@@PAPA_W@Z 00475040 f   mfc90:mfc90.dll
 0001:00074046       ?get_accDescription@CWnd@@UAEJUtagVARIANT@@PAPA_W@Z 00475046 f   mfc90:mfc90.dll
 0001:0007404c       ?get_accRole@CWnd@@UAEJUtagVARIANT@@PAU2@@Z 0047504c f   mfc90:mfc90.dll
 0001:00074052       ?get_accState@CWnd@@UAEJUtagVARIANT@@PAU2@@Z 00475052 f   mfc90:mfc90.dll
 0001:00074058       ?get_accHelp@CWnd@@UAEJUtagVARIANT@@PAPA_W@Z 00475058 f   mfc90:mfc90.dll
 0001:0007405e       ?get_accHelpTopic@CWnd@@UAEJPAPA_WUtagVARIANT@@PAJ@Z 0047505e f   mfc90:mfc90.dll
 0001:00074064       ?get_accKeyboardShortcut@CWnd@@UAEJUtagVARIANT@@PAPA_W@Z 00475064 f   mfc90:mfc90.dll
 0001:0007406a       ?get_accFocus@CWnd@@UAEJPAUtagVARIANT@@@Z 0047506a f   mfc90:mfc90.dll
 0001:00074070       ?get_accSelection@CWnd@@UAEJPAUtagVARIANT@@@Z 00475070 f   mfc90:mfc90.dll
 0001:00074076       ?get_accDefaultAction@CWnd@@UAEJUtagVARIANT@@PAPA_W@Z 00475076 f   mfc90:mfc90.dll
 0001:0007407c       ?accSelect@CWnd@@UAEJJUtagVARIANT@@@Z 0047507c f   mfc90:mfc90.dll
 0001:00074082       ?accLocation@CWnd@@UAEJPAJ000UtagVARIANT@@@Z 00475082 f   mfc90:mfc90.dll
 0001:00074088       ?accNavigate@CWnd@@UAEJJUtagVARIANT@@PAU2@@Z 00475088 f   mfc90:mfc90.dll
 0001:0007408e       ?accHitTest@CWnd@@UAEJJJPAUtagVARIANT@@@Z 0047508e f   mfc90:mfc90.dll
 0001:00074094       ?accDoDefaultAction@CWnd@@UAEJUtagVARIANT@@@Z 00475094 f   mfc90:mfc90.dll
 0001:0007409a       ?put_accName@CWnd@@UAEJUtagVARIANT@@PA_W@Z 0047509a f   mfc90:mfc90.dll
 0001:000740a0       ?put_accValue@CWnd@@UAEJUtagVARIANT@@PA_W@Z 004750a0 f   mfc90:mfc90.dll
 0001:000740a6       ?SetProxy@CWnd@@UAEJPAUIAccessibleProxy@@@Z 004750a6 f   mfc90:mfc90.dll
 0001:000740ac       ?CreateAccessibleProxy@CWnd@@UAEJIJPAJ@Z 004750ac f   mfc90:mfc90.dll
 0001:000740b2       ?OnCommand@CWnd@@MAEHIJ@Z  004750b2 f   mfc90:mfc90.dll
 0001:000740b8       ?OnNotify@CWnd@@MAEHIJPAJ@Z 004750b8 f   mfc90:mfc90.dll
 0001:000740be       ?GetSuperWndProcAddr@CWnd@@MAEPAP6GJPAUHWND__@@IIJ@ZXZ 004750be f   mfc90:mfc90.dll
 0001:000740c4       ?PreTranslateMessage@CDialog@@UAEHPAUtagMSG@@@Z 004750c4 f   mfc90:mfc90.dll
 0001:000740ca       ?OnAmbientProperty@CWnd@@UAEHPAVCOleControlSite@@JPAUtagVARIANT@@@Z 004750ca f   mfc90:mfc90.dll
 0001:000740d0       ?WindowProc@CWnd@@MAEJIIJ@Z 004750d0 f   mfc90:mfc90.dll
 0001:000740d6       ?OnWndMsg@CWnd@@MAEHIIJPAJ@Z 004750d6 f   mfc90:mfc90.dll
 0001:000740dc       ?DefWindowProcA@CWnd@@MAEJIIJ@Z 004750dc f   mfc90:mfc90.dll
 0001:000740e2       ?PostNcDestroy@CWnd@@MAEXXZ 004750e2 f   mfc90:mfc90.dll
 0001:000740e8       ?OnChildNotify@CWnd@@MAEHIIJPAJ@Z 004750e8 f   mfc90:mfc90.dll
 0001:000740ee       ?CheckAutoCenter@CDialog@@UAEHXZ 004750ee f   mfc90:mfc90.dll
 0001:000740f4       ?IsFrameWnd@CWnd@@UBEHXZ   004750f4 f   mfc90:mfc90.dll
 0001:000740fa       ?CreateControlContainer@CWnd@@MAEHPAPAVCOleControlContainer@@@Z 004750fa f   mfc90:mfc90.dll
 0001:00074100       ?CreateControlSite@CWnd@@MAEHPAVCOleControlContainer@@PAPAVCOleControlSite@@IABU_GUID@@@Z 00475100 f   mfc90:mfc90.dll
 0001:00074106       ?SetOccDialogInfo@CDialog@@MAEHPAU_AFX_OCC_DIALOG_INFO@@@Z 00475106 f   mfc90:mfc90.dll
 0001:0007410c       ?GetOccDialogInfo@CDialog@@MAEPAU_AFX_OCC_DIALOG_INFO@@XZ 0047510c f   mfc90:mfc90.dll
 0001:00074112       ?Create@CDialog@@UAEHPBDPAVCWnd@@@Z 00475112 f   mfc90:mfc90.dll
 0001:00074118       ?CreateIndirect@CDialog@@UAEHPAXPAVCWnd@@@Z 00475118 f   mfc90:mfc90.dll
 0001:0007411e       ?CreateIndirect@CDialog@@UAEHPBUDLGTEMPLATE@@PAVCWnd@@PAX@Z 0047511e f   mfc90:mfc90.dll
 0001:00074124       ?DoModal@CDialog@@UAEHXZ   00475124 f   mfc90:mfc90.dll
 0001:0007412a       ?OnSetFont@CDialog@@UAEXPAVCFont@@@Z 0047512a f   mfc90:mfc90.dll
 0001:00074130       ?OnOK@CDialog@@MAEXXZ      00475130 f   mfc90:mfc90.dll
 0001:00074136       ?OnCancel@CDialog@@MAEXXZ  00475136 f   mfc90:mfc90.dll
 0001:0007413c       ?PreInitDialog@CDialog@@MAEXXZ 0047513c f   mfc90:mfc90.dll
 0001:00074142       ?DDX_Text@@YGXPAVCDataExchange@@HAAV?$CStringT@DV?$StrTraitMFC_DLL@DV?$ChTraitsCRT@D@ATL@@@@@ATL@@@Z 00475142 f   mfc90:mfc90.dll
 0001:00074148       ?DDX_Control@@YGXPAVCDataExchange@@HAAVCWnd@@@Z 00475148 f   mfc90:mfc90.dll
 0001:0007414e       ?GetThisMessageMap@CDialog@@KGPBUAFX_MSGMAP@@XZ 0047514e f   mfc90:mfc90.dll
 0001:00074154       ?UpdateData@CWnd@@QAEHH@Z  00475154 f   mfc90:mfc90.dll
 0001:0007415a       ?ShowWindow@CWnd@@QAEHH@Z  0047515a f   mfc90:mfc90.dll
 0001:00074160       ?GetDlgItem@CWnd@@QBEPAV1@H@Z 00475160 f   mfc90:mfc90.dll
 0001:00074166       ?SetWindowTextA@CWnd@@QAEXPBD@Z 00475166 f   mfc90:mfc90.dll
 0001:0007416c       ?OnInitDialog@CDialog@@UAEHXZ 0047516c f   mfc90:mfc90.dll
 0001:00074172       ?EnableWindow@CWnd@@QAEHH@Z 00475172 f   mfc90:mfc90.dll
 0001:00074178       ?AfxMessageBox@@YGHPBDII@Z 00475178 f   mfc90:mfc90.dll
 0001:0007417e       ??0CWnd@@QAE@XZ            0047517e f   mfc90:mfc90.dll
 0001:00074184       ?GetRuntimeClass@CStatic@@UBEPAUCRuntimeClass@@XZ 00475184 f   mfc90:mfc90.dll
 0001:0007418a       ?OnCmdMsg@CCmdTarget@@UAEHIHPAXPAUAFX_CMDHANDLERINFO@@@Z 0047518a f   mfc90:mfc90.dll
 0001:00074190       ?GetMessageMap@CWnd@@MBEPBUAFX_MSGMAP@@XZ 00475190 f   mfc90:mfc90.dll
 0001:00074196       ?PreTranslateMessage@CWnd@@UAEHPAUtagMSG@@@Z 00475196 f   mfc90:mfc90.dll
 0001:0007419c       ?OnChildNotify@CStatic@@MAEHIIJPAJ@Z 0047519c f   mfc90:mfc90.dll
 0001:000741a2       ?CheckAutoCenter@CWnd@@UAEHXZ 004751a2 f   mfc90:mfc90.dll
 0001:000741a8       ?SetOccDialogInfo@CWnd@@MAEHPAU_AFX_OCC_DIALOG_INFO@@@Z 004751a8 f   mfc90:mfc90.dll
 0001:000741ae       ?GetOccDialogInfo@CWnd@@MAEPAU_AFX_OCC_DIALOG_INFO@@XZ 004751ae f   mfc90:mfc90.dll
 0001:000741b4       ?Create@CStatic@@UAEHPBDKABUtagRECT@@PAVCWnd@@I@Z 004751b4 f   mfc90:mfc90.dll
 0001:000741ba       ?DrawItem@CStatic@@UAEXPAUtagDRAWITEMSTRUCT@@@Z 004751ba f   mfc90:mfc90.dll
 0001:000741c0       ??1CComboBox@@UAE@XZ       004751c0 f   mfc90:mfc90.dll
 0001:000741c6       ?GetRuntimeClass@CDialog@@UBEPAUCRuntimeClass@@XZ 004751c6 f   mfc90:mfc90.dll
 0001:000741cc       ?DDX_CBString@@YGXPAVCDataExchange@@HAAV?$CStringT@DV?$StrTraitMFC_DLL@DV?$ChTraitsCRT@D@ATL@@@@@ATL@@@Z 004751cc f   mfc90:mfc90.dll
 0001:000741d2       ??1CStringList@@UAE@XZ     004751d2 f   mfc90:mfc90.dll
 0001:000741d8       ?AddTail@CStringList@@QAEPAU__POSITION@@ABV?$CStringT@DV?$StrTraitMFC_DLL@DV?$ChTraitsCRT@D@ATL@@@@@ATL@@@Z 004751d8 f   mfc90:mfc90.dll
 0001:000741de       ??0CStringList@@QAE@H@Z    004751de f   mfc90:mfc90.dll
 0001:000741e4       ?FindIndex@CStringList@@QBEPAU__POSITION@@H@Z 004751e4 f   mfc90:mfc90.dll
 0001:000741ea       ?GetNextAssoc@CMapStringToPtr@@QBEXAAPAU__POSITION@@AAV?$CStringT@DV?$StrTraitMFC_DLL@DV?$ChTraitsCRT@D@ATL@@@@@ATL@@AAPAX@Z 004751ea f   mfc90:mfc90.dll
 0001:000741f0       ?AfxThrowInvalidArgException@@YGXXZ 004751f0 f   mfc90:mfc90.dll
 0001:000741f6       ?GetRuntimeClass@CComboBox@@UBEPAUCRuntimeClass@@XZ 004751f6 f   mfc90:mfc90.dll
 0001:000741fc       ?OnChildNotify@CComboBox@@MAEHIIJPAJ@Z 004751fc f   mfc90:mfc90.dll
 0001:00074202       ?Create@CComboBox@@UAEHKABUtagRECT@@PAVCWnd@@I@Z 00475202 f   mfc90:mfc90.dll
 0001:00074208       ?DrawItem@CComboBox@@UAEXPAUtagDRAWITEMSTRUCT@@@Z 00475208 f   mfc90:mfc90.dll
 0001:0007420e       ?MeasureItem@CComboBox@@UAEXPAUtagMEASUREITEMSTRUCT@@@Z 0047520e f   mfc90:mfc90.dll
 0001:00074214       ?CompareItem@CComboBox@@UAEHPAUtagCOMPAREITEMSTRUCT@@@Z 00475214 f   mfc90:mfc90.dll
 0001:0007421a       ?DeleteItem@CComboBox@@UAEXPAUtagDELETEITEMSTRUCT@@@Z 0047521a f   mfc90:mfc90.dll
 0001:00074220       ?SetItemText@CListCtrl@@QAEHHHPBD@Z 00475220 f   mfc90:mfc90.dll
 0001:00074226       ?InsertColumn@CListCtrl@@QAEHHPBDHHH@Z 00475226 f   mfc90:mfc90.dll
 0001:0007422c       ?GetItemText@CListCtrl@@QBE?AV?$CStringT@DV?$StrTraitMFC_DLL@DV?$ChTraitsCRT@D@ATL@@@@@ATL@@HH@Z 0047522c f   mfc90:mfc90.dll
 0001:00074232       ?MessageBoxA@CWnd@@QAEHPBD0I@Z 00475232 f   mfc90:mfc90.dll
 0001:00074238       ??1CListCtrl@@UAE@XZ       00475238 f   mfc90:mfc90.dll
 0001:0007423e       ?SetFocus@CWnd@@QAEPAV1@XZ 0047523e f   mfc90:mfc90.dll
 0001:00074244       ?SetItemState@CListCtrl@@QAEHHII@Z 00475244 f   mfc90:mfc90.dll
 0001:0007424a       ?GetRuntimeClass@CListCtrl@@UBEPAUCRuntimeClass@@XZ 0047524a f   mfc90:mfc90.dll
 0001:00074250       ?GetMessageMap@CListCtrl@@MBEPBUAFX_MSGMAP@@XZ 00475250 f   mfc90:mfc90.dll
 0001:00074256       ?OnChildNotify@CListCtrl@@MAEHIIJPAJ@Z 00475256 f   mfc90:mfc90.dll
 0001:0007425c       ?DrawItem@CListCtrl@@UAEXPAUtagDRAWITEMSTRUCT@@@Z 0047525c f   mfc90:mfc90.dll
 0001:00074262       ?InsertItem@CListCtrl@@QAEHIHPBDIIHJ@Z 00475262 f   mfc90:mfc90.dll
 0001:00074268       ?GetThisClass@CException@@SGPAUCRuntimeClass@@XZ 00475268 f   mfc90:mfc90.dll
 0001:0007426e       ??0CException@@QAE@XZ      0047526e f   mfc90:mfc90.dll
 0001:00074274       ?GetErrorMessage@CException@@UBEHPADIPAI@Z 00475274 f   mfc90:mfc90.dll
 0001:0007427a       ?ReportError@CException@@UAEHII@Z 0047527a f   mfc90:mfc90.dll
 0001:00074280       ?GetThisClass@CObject@@SGPAUCRuntimeClass@@XZ 00475280 f   mfc90:mfc90.dll
 0001:00074286       ??_U@YAPAXI@Z              00475286 f   mfc90:mfc90.dll
 0001:0007428c       ??_V@YAXPAX@Z              0047528c f   mfc90:mfc90.dll
 0001:00074292       ??2@YAPAXI@Z               00475292 f   mfc90:mfc90.dll
 0001:00074298       ??1CPtrList@@UAE@XZ        00475298 f   mfc90:mfc90.dll
 0001:0007429e       ?GetRuntimeClass@CPtrList@@UBEPAUCRuntimeClass@@XZ 0047529e f   mfc90:mfc90.dll
 0001:000742a4       ??0CPtrList@@QAE@H@Z       004752a4 f   mfc90:mfc90.dll
 0001:000742aa       ??1CSyncObject@@UAE@XZ     004752aa f   mfc90:mfc90.dll
 0001:000742b0       ?AfxThrowMemoryException@@YGXXZ 004752b0 f   mfc90:mfc90.dll
 0001:000742b6       ??0CSyncObject@@QAE@PBD@Z  004752b6 f   mfc90:mfc90.dll
 0001:000742bc       ?GetRuntimeClass@CCriticalSection@@UBEPAUCRuntimeClass@@XZ 004752bc f   mfc90:mfc90.dll
 0001:000742c2       ?DDX_Check@@YGXPAVCDataExchange@@HAAH@Z 004752c2 f   mfc90:mfc90.dll
 0001:000742c8       ?IsWindowEnabled@CWnd@@QBEHXZ 004752c8 f   mfc90:mfc90.dll
 0001:000742ce       ?GetSafeOwner@CWnd@@SGPAV1@PAV1@PAPAUHWND__@@@Z 004752ce f   mfc90:mfc90.dll
 0001:000742d4       ?Default@CWnd@@IAEJXZ      004752d4 f   mfc90:mfc90.dll
 0001:000742da       ??1CMonthCalCtrl@@UAE@XZ   004752da f   mfc90:mfc90.dll
 0001:000742e0       ??1CWnd@@UAE@XZ            004752e0 f   mfc90:mfc90.dll
 0001:000742e6       ??0CImageList@@QAE@XZ      004752e6 f   mfc90:mfc90.dll
 0001:000742ec       ?GetRuntimeClass@CWnd@@UBEPAUCRuntimeClass@@XZ 004752ec f   mfc90:mfc90.dll
 0001:000742f2       ??1CImageList@@UAE@XZ      004752f2 f   mfc90:mfc90.dll
 0001:000742f8       ?GetThisMessageMap@CWnd@@KGPBUAFX_MSGMAP@@XZ 004752f8 f   mfc90:mfc90.dll
 0001:000742fe       ?OnSettingChange@CWnd@@IAEXIPBD@Z 004752fe f   mfc90:mfc90.dll
 0001:00074304       ?Create@CImageList@@QAEHHHIHH@Z 00475304 f   mfc90:mfc90.dll
 0001:0007430a       ?SetWindowPos@CWnd@@QAEHPBV1@HHHHI@Z 0047530a f   mfc90:mfc90.dll
 0001:00074310       ??1CPaintDC@@UAE@XZ        00475310 f   mfc90:mfc90.dll
 0001:00074316       ?FillSolidRect@CDC@@QAEXPBUtagRECT@@K@Z 00475316 f   mfc90:mfc90.dll
 0001:0007431c       ?SelectObject@CDC@@UAEPAVCFont@@PAV2@@Z 0047531c f   mfc90:mfc90.dll
 0001:00074322       ?SetTextColor@CDC@@UAEKK@Z 00475322 f   mfc90:mfc90.dll
 0001:00074328       ?SetBkMode@CDC@@QAEHH@Z    00475328 f   mfc90:mfc90.dll
 0001:0007432e       ?SelectStockObject@CDC@@UAEPAVCGdiObject@@H@Z 0047532e f   mfc90:mfc90.dll
 0001:00074334       ?LineTo@CDC@@QAEHHH@Z      00475334 f   mfc90:mfc90.dll
 0001:0007433a       ?MoveTo@CDC@@QAE?AVCPoint@@HH@Z 0047533a f   mfc90:mfc90.dll
 0001:00074340       ?SelectObject@CDC@@QAEPAVCPen@@PAV2@@Z 00475340 f   mfc90:mfc90.dll
 0001:00074346       ??0CPaintDC@@QAE@PAVCWnd@@@Z 00475346 f   mfc90:mfc90.dll
 0001:0007434c       ?GetRuntimeClass@CBitmap@@UBEPAUCRuntimeClass@@XZ 0047534c f   mfc90:mfc90.dll
 0001:00074352       ?GetRuntimeClass@CGdiObject@@UBEPAUCRuntimeClass@@XZ 00475352 f   mfc90:mfc90.dll
 0001:00074358       ?DeleteObject@CGdiObject@@QAEHXZ 00475358 f   mfc90:mfc90.dll
 0001:0007435e       ?Attach@CGdiObject@@QAEHPAX@Z 0047535e f   mfc90:mfc90.dll
 0001:00074364       ?AfxFindResourceHandle@@YGPAUHINSTANCE__@@PBD0@Z 00475364 f   mfc90:mfc90.dll
 0001:0007436a       ?AfxGetModuleState@@YGPAVAFX_MODULE_STATE@@XZ 0047536a f   mfc90:mfc90.dll
 0001:00074370       ?AfxDeactivateActCtx@@YGHKK@Z 00475370 f   mfc90:mfc90.dll
 0001:00074376       ?AfxActivateActCtxWrapper@@YG?AW4eActCtxResult@@PAXPAK@Z 00475376 f   mfc90:mfc90.dll
 0001:0007437c       ?GetRuntimeClass@CMonthCalCtrl@@UBEPAUCRuntimeClass@@XZ 0047537c f   mfc90:mfc90.dll
 0001:00074382       ?Create@CMonthCalCtrl@@UAEHKABUtagPOINT@@PAVCWnd@@I@Z 00475382 f   mfc90:mfc90.dll
 0001:00074388       ?Create@CMonthCalCtrl@@UAEHKABUtagRECT@@PAVCWnd@@I@Z 00475388 f   mfc90:mfc90.dll
 0001:0007438e       ?CreateObject@CRuntimeClass@@QAEPAVCObject@@XZ 0047538e f   mfc90:mfc90.dll
 0001:00074394       ??0CMFCVisualManager@@QAE@H@Z 00475394 f   mfc90:mfc90.dll
 0001:0007439a       ?AddTail@CStringList@@QAEPAU__POSITION@@PBD@Z 0047539a f   mfc90:mfc90.dll
 0001:000743a0       ??1CSocket@@UAE@XZ         004753a0 f   mfc90:mfc90.dll
 0001:000743a6       ??0CSocket@@QAE@XZ         004753a6 f   mfc90:mfc90.dll
 0001:000743ac       ?GetRuntimeClass@CSocket@@UBEPAUCRuntimeClass@@XZ 004753ac f   mfc90:mfc90.dll
 0001:000743b2       ?Accept@CSocket@@UAEHAAVCAsyncSocket@@PAUsockaddr@@PAH@Z 004753b2 f   mfc90:mfc90.dll
 0001:000743b8       ?Close@CSocket@@UAEXXZ     004753b8 f   mfc90:mfc90.dll
 0001:000743be       ?Receive@CSocket@@UAEHPAXHH@Z 004753be f   mfc90:mfc90.dll
 0001:000743c4       ?Send@CSocket@@UAEHPBXHH@Z 004753c4 f   mfc90:mfc90.dll
 0001:000743ca       ?OnReceive@CAsyncSocket@@MAEXH@Z 004753ca f   mfc90:mfc90.dll
 0001:000743d0       ?OnSend@CAsyncSocket@@MAEXH@Z 004753d0 f   mfc90:mfc90.dll
 0001:000743d6       ?OnOutOfBandData@CAsyncSocket@@MAEXH@Z 004753d6 f   mfc90:mfc90.dll
 0001:000743dc       ?OnConnect@CAsyncSocket@@MAEXH@Z 004753dc f   mfc90:mfc90.dll
 0001:000743e2       ?ConnectHelper@CSocket@@MAEHPBUsockaddr@@H@Z 004753e2 f   mfc90:mfc90.dll
 0001:000743e8       ?ReceiveFromHelper@CSocket@@MAEHPAXHPAUsockaddr@@PAHH@Z 004753e8 f   mfc90:mfc90.dll
 0001:000743ee       ?SendToHelper@CSocket@@MAEHPBXHPBUsockaddr@@HH@Z 004753ee f   mfc90:mfc90.dll
 0001:000743f4       ?OnMessagePending@CSocket@@MAEHXZ 004753f4 f   mfc90:mfc90.dll
 0001:000743fa       ?PumpMessages@CSocket@@MAEHI@Z 004753fa f   mfc90:mfc90.dll
 0001:00074400       ?OnAccept@CAsyncSocket@@MAEXH@Z 00475400 f   mfc90:mfc90.dll
 0001:00074406       ?AfxBeginThread@@YGPAVCWinThread@@P6AIPAX@Z0HIKPAU_SECURITY_ATTRIBUTES@@@Z 00475406 f   mfc90:mfc90.dll
 0001:0007440c       ?OnClose@CAsyncSocket@@MAEXH@Z 0047540c f   mfc90:mfc90.dll
 0001:00074412       ??1CStdioFile@@UAE@XZ      00475412 f   mfc90:mfc90.dll
 0001:00074418       ?Close@CStdioFile@@UAEXXZ  00475418 f   mfc90:mfc90.dll
 0001:0007441e       ?AddHead@CStringList@@QAEPAU__POSITION@@ABV?$CStringT@DV?$StrTraitMFC_DLL@DV?$ChTraitsCRT@D@ATL@@@@@ATL@@@Z 0047541e f   mfc90:mfc90.dll
 0001:00074424       ?InsertAfter@CStringList@@QAEPAU__POSITION@@PAU2@ABV?$CStringT@DV?$StrTraitMFC_DLL@DV?$ChTraitsCRT@D@ATL@@@@@ATL@@@Z 00475424 f   mfc90:mfc90.dll
 0001:0007442a       ?Find@CStringList@@QBEPAU__POSITION@@PBDPAU2@@Z 0047542a f   mfc90:mfc90.dll
 0001:00074430       ?ReadString@CStdioFile@@UAEPADPADI@Z 00475430 f   mfc90:mfc90.dll
 0001:00074436       ??0CStdioFile@@QAE@PBDI@Z  00475436 f   mfc90:mfc90.dll
 0001:0007443c       ?GetRuntimeClass@CObject@@UBEPAUCRuntimeClass@@XZ 0047543c f   mfc90:mfc90.dll
 0001:00074442       ?ReadCount@CArchive@@QAEKXZ 00475442 f   mfc90:mfc90.dll
 0001:00074448       ?WriteCount@CArchive@@QAEXK@Z 00475448 f   mfc90:mfc90.dll
 0001:0007444e       ?FreeDataChain@CPlex@@QAEXXZ 0047544e f   mfc90:mfc90.dll
 0001:00074454       ?Create@CPlex@@SGPAU1@AAPAU1@II@Z 00475454 f   mfc90:mfc90.dll
 0001:0007445a       ?Write@CArchive@@QAEXPBXI@Z 0047545a f   mfc90:mfc90.dll
 0001:00074460       ?AfxThrowArchiveException@@YGXHPBD@Z 00475460 f   mfc90:mfc90.dll
 0001:00074466       ?Read@CArchive@@QAEIPAXI@Z 00475466 f   mfc90:mfc90.dll
 0001:0007446c       ??1CEdit@@UAE@XZ           0047546c f   mfc90:mfc90.dll
 0001:00074472       ?DDV_MaxChars@@YGXPAVCDataExchange@@ABV?$CStringT@DV?$StrTraitMFC_DLL@DV?$ChTraitsCRT@D@ATL@@@@@ATL@@H@Z 00475472 f   mfc90:mfc90.dll
 0001:00074478       ?GetDlgCtrlID@CWnd@@QBEHXZ 00475478 f   mfc90:mfc90.dll
 0001:0007447e       ?OnCtlColor@CWnd@@IAEPAUHBRUSH__@@PAVCDC@@PAV1@I@Z 0047547e f   mfc90:mfc90.dll
 0001:00074484       ?GetRuntimeClass@CEdit@@UBEPAUCRuntimeClass@@XZ 00475484 f   mfc90:mfc90.dll
 0001:0007448a       ??1CMapStringToPtr@@UAE@XZ 0047548a f   mfc90:mfc90.dll
 0001:00074490       ?RemoveAll@CMapStringToPtr@@QAEXXZ 00475490 f   mfc90:mfc90.dll
 0001:00074496       ?InitHashTable@CMapStringToPtr@@QAEXIH@Z 00475496 f   mfc90:mfc90.dll
 0001:0007449c       ?RemoveAt@CStringList@@QAEXPAU__POSITION@@@Z 0047549c f   mfc90:mfc90.dll
 0001:000744a2       ??0CMapStringToPtr@@QAE@H@Z 004754a2 f   mfc90:mfc90.dll
 0001:000744a8       ?GetRuntimeClass@CMapStringToPtr@@UBEPAUCRuntimeClass@@XZ 004754a8 f   mfc90:mfc90.dll
 0001:000744ae       ?Lookup@CMapStringToPtr@@QBEHPBDAAPAX@Z 004754ae f   mfc90:mfc90.dll
 0001:000744b4       ??ACMapStringToPtr@@QAEAAPAXPBD@Z 004754b4 f   mfc90:mfc90.dll
 0001:000744ba       ?RemoveKey@CMapStringToPtr@@QAEHPBD@Z 004754ba f   mfc90:mfc90.dll
 0001:000744c0       ?InsertItem@CTreeCtrl@@QAEPAU_TREEITEM@@IPBDHHIIJPAU2@1@Z 004754c0 f   mfc90:mfc90.dll
 0001:000744c6       ?SetItem@CTreeCtrl@@QAEHPAU_TREEITEM@@IPBDHHIIJ@Z 004754c6 f   mfc90:mfc90.dll
 0001:000744cc       ??1CSpinButtonCtrl@@UAE@XZ 004754cc f   mfc90:mfc90.dll
 0001:000744d2       ?RemoveAll@CPtrList@@QAEXXZ 004754d2 f   mfc90:mfc90.dll
 0001:000744d8       ?GetLBText@CComboBox@@QBEXHAAV?$CStringT@DV?$StrTraitMFC_DLL@DV?$ChTraitsCRT@D@ATL@@@@@ATL@@@Z 004754d8 f   mfc90:mfc90.dll
 0001:000744de       ?GetRuntimeClass@CSpinButtonCtrl@@UBEPAUCRuntimeClass@@XZ 004754de f   mfc90:mfc90.dll
 0001:000744e4       ?Create@CSpinButtonCtrl@@UAEHKABUtagRECT@@PAVCWnd@@I@Z 004754e4 f   mfc90:mfc90.dll
 0001:000744ea       ?CreateEx@CSpinButtonCtrl@@UAEHKKABUtagRECT@@PAVCWnd@@I@Z 004754ea f   mfc90:mfc90.dll
 0001:000744f0       ??1CButton@@UAE@XZ         004754f0 f   mfc90:mfc90.dll
 0001:000744f6       ?GetRuntimeClass@CButton@@UBEPAUCRuntimeClass@@XZ 004754f6 f   mfc90:mfc90.dll
 0001:000744fc       ?OnChildNotify@CButton@@MAEHIIJPAJ@Z 004754fc f   mfc90:mfc90.dll
 0001:00074502       ?Create@CButton@@UAEHPBDKABUtagRECT@@PAVCWnd@@I@Z 00475502 f   mfc90:mfc90.dll
 0001:00074508       ?DrawItem@CButton@@UAEXPAUtagDRAWITEMSTRUCT@@@Z 00475508 f   mfc90:mfc90.dll
 0001:0007450e       ??1CFileDialog@@UAE@XZ     0047550e f   mfc90:mfc90.dll
 0001:00074514       ?GetPathName@CFileDialog@@QBE?AV?$CStringT@DV?$StrTraitMFC_DLL@DV?$ChTraitsCRT@D@ATL@@@@@ATL@@XZ 00475514 f   mfc90:mfc90.dll
 0001:0007451a       ?DoModal@CFileDialog@@UAEHXZ 0047551a f   mfc90:mfc90.dll
 0001:00074520       ??0CFileDialog@@QAE@HPBD0K0PAVCWnd@@KH@Z 00475520 f   mfc90:mfc90.dll
 0001:00074526       ?ModifyStyle@CWnd@@QAEHKKI@Z 00475526 f   mfc90:mfc90.dll
 0001:0007452c       ?Detach@CGdiObject@@QAEPAXXZ 0047552c f   mfc90:mfc90.dll
 0001:00074532       ?GetWindowTextA@CWnd@@QBEXAAV?$CStringT@DV?$StrTraitMFC_DLL@DV?$ChTraitsCRT@D@ATL@@@@@ATL@@@Z 00475532 f   mfc90:mfc90.dll
 0001:00074538       ?GetRuntimeClass@CFont@@UBEPAUCRuntimeClass@@XZ 00475538 f   mfc90:mfc90.dll
 0001:0007453e       ??0CFile@@QAE@PBDI@Z       0047553e f   mfc90:mfc90.dll
 0001:00074544       ?WriteString@CStdioFile@@UAEXPBD@Z 00475544 f   mfc90:mfc90.dll
 0001:0007454a       ?GetRuntimeClass@CTreeCtrl@@UBEPAUCRuntimeClass@@XZ 0047554a f   mfc90:mfc90.dll
 0001:00074550       ??1CTreeCtrl@@UAE@XZ       00475550 f   mfc90:mfc90.dll
 0001:00074556       ?GetThisMessageMap@CTreeCtrl@@KGPBUAFX_MSGMAP@@XZ 00475556 f   mfc90:mfc90.dll
 0001:0007455c       ?GetItemText@CTreeCtrl@@QBE?AV?$CStringT@DV?$StrTraitMFC_DLL@DV?$ChTraitsCRT@D@ATL@@@@@ATL@@PAU_TREEITEM@@@Z 0047555c f   mfc90:mfc90.dll
 0001:00074562       ?HitTest@CTreeCtrl@@QBEPAU_TREEITEM@@VCPoint@@PAI@Z 00475562 f   mfc90:mfc90.dll
 0001:00074568       ?UpdateDialogControls@CWnd@@QAEXPAVCCmdTarget@@H@Z 00475568 f   mfc90:mfc90.dll
 0001:0007456e       ??0CMFCPopupMenu@@QAE@XZ   0047556e f   mfc90:mfc90.dll
 0001:00074574       ?IsKindOf@CObject@@QBEHPBUCRuntimeClass@@@Z 00475574 f   mfc90:mfc90.dll
 0001:0007457a       ?GetThisClass@CFrameWndEx@@SGPAUCRuntimeClass@@XZ 0047557a f   mfc90:mfc90.dll
 0001:00074580       ?ClientToScreen@CWnd@@QBEXPAUtagRECT@@@Z 00475580 f   mfc90:mfc90.dll
 0001:00074586       ?Create@CEdit@@QAEHKABUtagRECT@@PAVCWnd@@I@Z 00475586 f   mfc90:mfc90.dll
 0001:0007458c       ?GetItemRect@CTreeCtrl@@QBEHPAU_TREEITEM@@PAUtagRECT@@H@Z 0047558c f   mfc90:mfc90.dll
 0001:00074592       ?AfxGetThread@@YGPAVCWinThread@@XZ 00475592 f   mfc90:mfc90.dll
 0001:00074598       ?GetRuntimeClass@CMenu@@UBEPAUCRuntimeClass@@XZ 00475598 f   mfc90:mfc90.dll
 0001:0007459e       ?DrawItem@CMenu@@UAEXPAUtagDRAWITEMSTRUCT@@@Z 0047559e f   mfc90:mfc90.dll
 0001:000745a4       ?MeasureItem@CMenu@@UAEXPAUtagMEASUREITEMSTRUCT@@@Z 004755a4 f   mfc90:mfc90.dll
 0001:000745aa       ?DestroyMenu@CMenu@@QAEHXZ 004755aa f   mfc90:mfc90.dll
 0001:000745b0       ?FromHandle@CMenu@@SGPAV1@PAUHMENU__@@@Z 004755b0 f   mfc90:mfc90.dll
 0001:000745b6       ?Attach@CMenu@@QAEHPAUHMENU__@@@Z 004755b6 f   mfc90:mfc90.dll
 0001:000745bc       ?GetMessageMap@CTreeCtrl@@MBEPBUAFX_MSGMAP@@XZ 004755bc f   mfc90:mfc90.dll
 0001:000745c2       ?RemoveAll@CMapPtrToPtr@@QAEXXZ 004755c2 f   mfc90:mfc90.dll
 0001:000745c8       ??1CMapPtrToPtr@@UAE@XZ    004755c8 f   mfc90:mfc90.dll
 0001:000745ce       ??0CMapPtrToPtr@@QAE@H@Z   004755ce f   mfc90:mfc90.dll
 0001:000745d4       ?GetRuntimeClass@CMapPtrToPtr@@UBEPAUCRuntimeClass@@XZ 004755d4 f   mfc90:mfc90.dll
 0001:000745da       ?Lookup@CMapPtrToPtr@@QBEHPAXAAPAX@Z 004755da f   mfc90:mfc90.dll
 0001:000745e0       ??ACMapPtrToPtr@@QAEAAPAXPAX@Z 004755e0 f   mfc90:mfc90.dll
 0001:000745e6       ?RemoveKey@CMapPtrToPtr@@QAEHPAX@Z 004755e6 f   mfc90:mfc90.dll
 0001:000745ec       ?GetNextAssoc@CMapPtrToPtr@@QBEXAAPAU__POSITION@@AAPAX1@Z 004755ec f   mfc90:mfc90.dll
 0001:000745f2       ?GetThisMessageMap@CWinApp@@KGPBUAFX_MSGMAP@@XZ 004755f2 f   mfc90:mfc90.dll
 0001:000745f8       ?OnFileNew@CWinApp@@IAEXXZ 004755f8 f   mfc90:mfc90.dll
 0001:000745fe       ?OnFileOpen@CWinApp@@IAEXXZ 004755fe f   mfc90:mfc90.dll
 0001:00074604       ??0CWinAppEx@@QAE@H@Z      00475604 f   mfc90:mfc90.dll
 0001:0007460a       ?GetRuntimeClass@CWinAppEx@@UBEPAUCRuntimeClass@@XZ 0047560a f   mfc90:mfc90.dll
 0001:00074610       ?OnFinalRelease@CCmdTarget@@UAEXXZ 00475610 f   mfc90:mfc90.dll
 0001:00074616       ?GetInterfaceMap@CCmdTarget@@MBEPBUAFX_INTERFACEMAP@@XZ 00475616 f   mfc90:mfc90.dll
 0001:0007461c       ?Run@CWinApp@@UAEHXZ       0047561c f   mfc90:mfc90.dll
 0001:00074622       ?PreTranslateMessage@CWinThread@@UAEHPAUtagMSG@@@Z 00475622 f   mfc90:mfc90.dll
 0001:00074628       ?PumpMessage@CWinThread@@UAEHXZ 00475628 f   mfc90:mfc90.dll
 0001:0007462e       ?OnIdle@CWinApp@@UAEHJ@Z   0047562e f   mfc90:mfc90.dll
 0001:00074634       ?IsIdleMessage@CWinThread@@UAEHPAUtagMSG@@@Z 00475634 f   mfc90:mfc90.dll
 0001:0007463a       ?ProcessWndProcException@CWinApp@@UAEJPAVCException@@PBUtagMSG@@@Z 0047563a f   mfc90:mfc90.dll
 0001:00074640       ?ProcessMessageFilter@CWinThread@@UAEHHPAUtagMSG@@@Z 00475640 f   mfc90:mfc90.dll
 0001:00074646       ?GetMainWnd@CWinThread@@UAEPAVCWnd@@XZ 00475646 f   mfc90:mfc90.dll
 0001:0007464c       ?Delete@CWinThread@@UAEXXZ 0047564c f   mfc90:mfc90.dll
 0001:00074652       ?InitLibId@CWinApp@@UAEXXZ 00475652 f   mfc90:mfc90.dll
 0001:00074658       ?Register@CWinApp@@UAEHXZ  00475658 f   mfc90:mfc90.dll
 0001:0007465e       ?Unregister@CWinApp@@UAEHXZ 0047565e f   mfc90:mfc90.dll
 0001:00074664       ?OpenDocumentFile@CWinApp@@UAEPAVCDocument@@PBD@Z 00475664 f   mfc90:mfc90.dll
 0001:0007466a       ?AddToRecentFileList@CWinApp@@UAEXPBD@Z 0047566a f   mfc90:mfc90.dll
 0001:00074670       ?InitApplication@CWinApp@@UAEHXZ 00475670 f   mfc90:mfc90.dll
 0001:00074676       ?SaveAllModified@CWinApp@@UAEHXZ 00475676 f   mfc90:mfc90.dll
 0001:0007467c       ?DoMessageBox@CWinApp@@UAEHPBDII@Z 0047567c f   mfc90:mfc90.dll
 0001:00074682       ?DoWaitCursor@CWinApp@@UAEXH@Z 00475682 f   mfc90:mfc90.dll
 0001:00074688       ?OnDDECommand@CWinApp@@UAEHPAD@Z 00475688 f   mfc90:mfc90.dll
 0001:0007468e       ?WinHelpA@CWinApp@@UAEXKI@Z 0047568e f   mfc90:mfc90.dll
 0001:00074694       ?HtmlHelpA@CWinApp@@UAEXKI@Z 00475694 f   mfc90:mfc90.dll
 0001:0007469a       ?WinHelpInternal@CWinApp@@UAEXKI@Z 0047569a f   mfc90:mfc90.dll
 0001:000746a0       ?LoadAppLangResourceDLL@CWinApp@@UAEPAUHINSTANCE__@@XZ 004756a0 f   mfc90:mfc90.dll
 0001:000746a6       ?LoadSysPolicies@CWinApp@@UAEHXZ 004756a6 f   mfc90:mfc90.dll
 0001:000746ac       ?LoadState@CWinAppEx@@UAEHPBDPAVCFrameImpl@@@Z 004756ac f   mfc90:mfc90.dll
 0001:000746b2       ?CleanState@CWinAppEx@@UAEHPBD@Z 004756b2 f   mfc90:mfc90.dll
 0001:000746b8       ?SaveState@CWinAppEx@@UAEHPBDPAVCFrameImpl@@@Z 004756b8 f   mfc90:mfc90.dll
 0001:000746be       ?OnViewDoubleClick@CWinAppEx@@UAEHPAVCWnd@@H@Z 004756be f   mfc90:mfc90.dll
 0001:000746c4       ?ShowPopupMenu@CWinAppEx@@UAEHIABVCPoint@@PAVCWnd@@@Z 004756c4 f   mfc90:mfc90.dll
 0001:000746ca       ?OnAppContextHelp@CWinAppEx@@UAEXPAVCWnd@@QBK@Z 004756ca f   mfc90:mfc90.dll
 0001:000746d0       ?OnClosingMainFrame@CWinAppEx@@MAEXPAVCFrameImpl@@@Z 004756d0 f   mfc90:mfc90.dll
 0001:000746d6       ?LoadWindowPlacement@CWinAppEx@@MAEHAAVCRect@@AAH1@Z 004756d6 f   mfc90:mfc90.dll
 0001:000746dc       ?StoreWindowPlacement@CWinAppEx@@MAEHABVCRect@@HH@Z 004756dc f   mfc90:mfc90.dll
 0001:000746e2       ?ReloadWindowPlacement@CWinAppEx@@MAEHPAVCFrameWnd@@@Z 004756e2 f   mfc90:mfc90.dll
 0001:000746e8       ??1CWinAppEx@@UAE@XZ       004756e8 f   mfc90:mfc90.dll
 0001:000746ee       ?GetActiveView@CFrameWnd@@QBEPAVCView@@XZ 004756ee f   mfc90:mfc90.dll
 0001:000746f4       ??1CCommandLineInfo@@UAE@XZ 004756f4 f   mfc90:mfc90.dll
 0001:000746fa       ?ProcessShellCommand@CWinApp@@QAEHAAVCCommandLineInfo@@@Z 004756fa f   mfc90:mfc90.dll
 0001:00074700       ?ParseCommandLine@CWinApp@@QAEXAAVCCommandLineInfo@@@Z 00475700 f   mfc90:mfc90.dll
 0001:00074706       ??0CCommandLineInfo@@QAE@XZ 00475706 f   mfc90:mfc90.dll
 0001:0007470c       ?AddDocTemplate@CWinApp@@QAEXPAVCDocTemplate@@@Z 0047570c f   mfc90:mfc90.dll
 0001:00074712       ??0CSingleDocTemplate@@QAE@IPAUCRuntimeClass@@00@Z 00475712 f   mfc90:mfc90.dll
 0001:00074718       ?SetTooltipParams@CTooltipManager@@QAEXIPAUCRuntimeClass@@PAVCMFCToolTipInfo@@@Z 00475718 f   mfc90:mfc90.dll
 0001:0007471e       ?GetTooltipManager@CWinAppEx@@QAEPAVCTooltipManager@@XZ 0047571e f   mfc90:mfc90.dll
 0001:00074724       ?GetThisClass@CMFCToolTipCtrl@@SGPAUCRuntimeClass@@XZ 00475724 f   mfc90:mfc90.dll
 0001:0007472a       ?InitTooltipManager@CWinAppEx@@QAEHXZ 0047572a f   mfc90:mfc90.dll
 0001:00074730       ?InitKeyboardManager@CWinAppEx@@QAEHXZ 00475730 f   mfc90:mfc90.dll
 0001:00074736       ?InitShellManager@CWinAppEx@@QAEHXZ 00475736 f   mfc90:mfc90.dll
 0001:0007473c       ?InitContextMenuManager@CWinAppEx@@QAEHXZ 0047573c f   mfc90:mfc90.dll
 0001:00074742       ?LoadStdProfileSettings@CWinApp@@IAEXI@Z 00475742 f   mfc90:mfc90.dll
 0001:00074748       ?SetRegistryKey@CWinApp@@IAEXPBD@Z 00475748 f   mfc90:mfc90.dll
 0001:0007474e       ?AfxEnableControlContainer@@YAXPAVCOccManager@@@Z 0047574e f   mfc90:mfc90.dll
 0001:00074754       ?AfxMessageBox@@YGHIII@Z   00475754 f   mfc90:mfc90.dll
 0001:0007475a       ?AfxOleInit@@YGHXZ         0047575a f   mfc90:mfc90.dll
 0001:00074760       ?InitInstance@CWinApp@@UAEHXZ 00475760 f   mfc90:mfc90.dll
 0001:00074766       ?AfxInitRichEdit2@@YGHXZ   00475766 f   mfc90:mfc90.dll
 0001:0007476c       ?ExitInstance@CWinApp@@UAEHXZ 0047576c f   mfc90:mfc90.dll
 0001:00074772       ?AddMenu@CContextMenuManager@@QAEHPBDI@Z 00475772 f   mfc90:mfc90.dll
 0001:00074778       ?GetContextMenuManager@CWinAppEx@@QAEPAVCContextMenuManager@@XZ 00475778 f   mfc90:mfc90.dll
 0001:0007477e       ??1CFileFind@@UAE@XZ       0047577e f   mfc90:mfc90.dll
 0001:00074784       ?Close@CFileFind@@QAEXXZ   00475784 f   mfc90:mfc90.dll
 0001:0007478a       ?FindFile@CFileFind@@UAEHPBDK@Z 0047578a f   mfc90:mfc90.dll
 0001:00074790       ??0CFileFind@@QAE@XZ       00475790 f   mfc90:mfc90.dll
 0001:00074796       ?FromHandle@CWnd@@SGPAV1@PAUHWND__@@@Z 00475796 f   mfc90:mfc90.dll
 0001:0007479c       ?GetThisClass@CDocument@@SGPAUCRuntimeClass@@XZ 0047579c f   mfc90:mfc90.dll
 0001:000747a2       ?GetThisMessageMap@CDocument@@KGPBUAFX_MSGMAP@@XZ 004757a2 f   mfc90:mfc90.dll
 0001:000747a8       ??0CDocument@@QAE@XZ       004757a8 f   mfc90:mfc90.dll
 0001:000747ae       ?OnCmdMsg@CDocument@@UAEHIHPAXPAUAFX_CMDHANDLERINFO@@@Z 004757ae f   mfc90:mfc90.dll
 0001:000747b4       ?OnFinalRelease@CDocument@@UAEXXZ 004757b4 f   mfc90:mfc90.dll
 0001:000747ba       ?SetTitle@CDocument@@UAEXPBD@Z 004757ba f   mfc90:mfc90.dll
 0001:000747c0       ?SetPathName@CDocument@@UAEXPBDH@Z 004757c0 f   mfc90:mfc90.dll
 0001:000747c6       ?GetFirstViewPosition@CDocument@@UBEPAU__POSITION@@XZ 004757c6 f   mfc90:mfc90.dll
 0001:000747cc       ?GetNextView@CDocument@@UBEPAVCView@@AAPAU__POSITION@@@Z 004757cc f   mfc90:mfc90.dll
 0001:000747d2       ?OnChangedViewList@CDocument@@UAEXXZ 004757d2 f   mfc90:mfc90.dll
 0001:000747d8       ?DeleteContents@CDocument@@UAEXXZ 004757d8 f   mfc90:mfc90.dll
 0001:000747de       ?OnOpenDocument@CDocument@@UAEHPBD@Z 004757de f   mfc90:mfc90.dll
 0001:000747e4       ?OnSaveDocument@CDocument@@UAEHPBD@Z 004757e4 f   mfc90:mfc90.dll
 0001:000747ea       ?OnCloseDocument@CDocument@@UAEXXZ 004757ea f   mfc90:mfc90.dll
 0001:000747f0       ?ReportSaveLoadException@CDocument@@UAEXPBDPAVCException@@HI@Z 004757f0 f   mfc90:mfc90.dll
 0001:000747f6       ?GetFile@CDocument@@UAEPAVCFile@@PBDIPAVCFileException@@@Z 004757f6 f   mfc90:mfc90.dll
 0001:000747fc       ?ReleaseFile@CDocument@@UAEXPAVCFile@@H@Z 004757fc f   mfc90:mfc90.dll
 0001:00074802       ?CanCloseFrame@CDocument@@UAEHPAVCFrameWnd@@@Z 00475802 f   mfc90:mfc90.dll
 0001:00074808       ?SaveModified@CDocument@@UAEHXZ 00475808 f   mfc90:mfc90.dll
 0001:0007480e       ?PreCloseFrame@CDocument@@UAEXPAVCFrameWnd@@@Z 0047580e f   mfc90:mfc90.dll
 0001:00074814       ?DoSave@CDocument@@UAEHPBDH@Z 00475814 f   mfc90:mfc90.dll
 0001:0007481a       ?DoFileSave@CDocument@@UAEHXZ 0047581a f   mfc90:mfc90.dll
 0001:00074820       ?UpdateFrameCounts@CDocument@@UAEXXZ 00475820 f   mfc90:mfc90.dll
 0001:00074826       ?GetDefaultMenu@CDocument@@UAEPAUHMENU__@@XZ 00475826 f   mfc90:mfc90.dll
 0001:0007482c       ?GetDefaultAccelerator@CDocument@@UAEPAUHACCEL__@@XZ 0047582c f   mfc90:mfc90.dll
 0001:00074832       ?OnIdle@CDocument@@UAEXXZ  00475832 f   mfc90:mfc90.dll
 0001:00074838       ??1CDocument@@UAE@XZ       00475838 f   mfc90:mfc90.dll
 0001:0007483e       ?OnNewDocument@CDocument@@UAEHXZ 0047583e f   mfc90:mfc90.dll
 0001:00074844       ?GetThisClass@CFormView@@SGPAUCRuntimeClass@@XZ 00475844 f   mfc90:mfc90.dll
 0001:0007484a       ?GetThisMessageMap@CFormView@@KGPBUAFX_MSGMAP@@XZ 0047584a f   mfc90:mfc90.dll
 0001:00074850       ??1CFormView@@UAE@XZ       00475850 f   mfc90:mfc90.dll
 0001:00074856       ??0CFormView@@IAE@I@Z      00475856 f   mfc90:mfc90.dll
 0001:0007485c       ?OnCmdMsg@CView@@UAEHIHPAXPAUAFX_CMDHANDLERINFO@@@Z 0047585c f   mfc90:mfc90.dll
 0001:00074862       ?Create@CFormView@@MAEHPBD0KABUtagRECT@@PAVCWnd@@IPAUCCreateContext@@@Z 00475862 f   mfc90:mfc90.dll
 0001:00074868       ?CalcWindowRect@CScrollView@@UAEXPAUtagRECT@@I@Z 00475868 f   mfc90:mfc90.dll
 0001:0007486e       ?GetScrollBarCtrl@CView@@UBEPAVCScrollBar@@H@Z 0047586e f   mfc90:mfc90.dll
 0001:00074874       ?PostNcDestroy@CView@@MAEXXZ 00475874 f   mfc90:mfc90.dll
 0001:0007487a       ?SetOccDialogInfo@CFormView@@MAEHPAU_AFX_OCC_DIALOG_INFO@@@Z 0047587a f   mfc90:mfc90.dll
 0001:00074880       ?GetOccDialogInfo@CFormView@@MAEPAU_AFX_OCC_DIALOG_INFO@@XZ 00475880 f   mfc90:mfc90.dll
 0001:00074886       ?IsSelected@CView@@UBEHPBVCObject@@@Z 00475886 f   mfc90:mfc90.dll
 0001:0007488c       ?OnScroll@CScrollView@@UAEHIIH@Z 0047588c f   mfc90:mfc90.dll
 0001:00074892       ?OnScrollBy@CScrollView@@UAEHVCSize@@H@Z 00475892 f   mfc90:mfc90.dll
 0001:00074898       ?OnDragEnter@CView@@UAEKPAVCOleDataObject@@KVCPoint@@@Z 00475898 f   mfc90:mfc90.dll
 0001:0007489e       ?OnDragOver@CView@@UAEKPAVCOleDataObject@@KVCPoint@@@Z 0047589e f   mfc90:mfc90.dll
 0001:000748a4       ?OnDragLeave@CView@@UAEXXZ 004758a4 f   mfc90:mfc90.dll
 0001:000748aa       ?OnDrop@CView@@UAEHPAVCOleDataObject@@KVCPoint@@@Z 004758aa f   mfc90:mfc90.dll
 0001:000748b0       ?OnDropEx@CView@@UAEKPAVCOleDataObject@@KKVCPoint@@@Z 004758b0 f   mfc90:mfc90.dll
 0001:000748b6       ?OnDragScroll@CView@@UAEKKVCPoint@@@Z 004758b6 f   mfc90:mfc90.dll
 0001:000748bc       ?OnPrepareDC@CScrollView@@UAEXPAVCDC@@PAUCPrintInfo@@@Z 004758bc f   mfc90:mfc90.dll
 0001:000748c2       ?OnActivateView@CFormView@@MAEXHPAVCView@@0@Z 004758c2 f   mfc90:mfc90.dll
 0001:000748c8       ?OnActivateFrame@CFormView@@MAEXIPAVCFrameWnd@@@Z 004758c8 f   mfc90:mfc90.dll
 0001:000748ce       ?OnUpdate@CView@@MAEXPAV1@JPAVCObject@@@Z 004758ce f   mfc90:mfc90.dll
 0001:000748d4       ?OnPreparePrinting@CView@@MAEHPAUCPrintInfo@@@Z 004758d4 f   mfc90:mfc90.dll
 0001:000748da       ?OnBeginPrinting@CView@@MAEXPAVCDC@@PAUCPrintInfo@@@Z 004758da f   mfc90:mfc90.dll
 0001:000748e0       ?OnPrint@CView@@MAEXPAVCDC@@PAUCPrintInfo@@@Z 004758e0 f   mfc90:mfc90.dll
 0001:000748e6       ?OnEndPrinting@CView@@MAEXPAVCDC@@PAUCPrintInfo@@@Z 004758e6 f   mfc90:mfc90.dll
 0001:000748ec       ?OnEndPrintPreview@CView@@MAEXPAVCDC@@PAUCPrintInfo@@UtagPOINT@@PAVCPreviewView@@@Z 004758ec f   mfc90:mfc90.dll
 0001:000748f2       ?GetWheelScrollDistance@CScrollView@@UAE?AVCSize@@V2@HH@Z 004758f2 f   mfc90:mfc90.dll
 0001:000748f8       ?PreCreateWindow@CView@@MAEHAAUtagCREATESTRUCTA@@@Z 004758f8 f   mfc90:mfc90.dll
 0001:000748fe       ?GetParentFrame@CWnd@@QBEPAVCFrameWnd@@XZ 004758fe f   mfc90:mfc90.dll
 0001:00074904       ?OnInitialUpdate@CFormView@@UAEXXZ 00475904 f   mfc90:mfc90.dll
 0001:0007490a       ?MoveWindow@CWnd@@QAEXHHHHH@Z 0047590a f   mfc90:mfc90.dll
 0001:00074910       ?GetScrollPosition@CScrollView@@QBE?AVCPoint@@XZ 00475910 f   mfc90:mfc90.dll
 0001:00074916       ?OnSize@CScrollView@@QAEXIHH@Z 00475916 f   mfc90:mfc90.dll
 0001:0007491c       ?AfxBeginThread@@YGPAVCWinThread@@PAUCRuntimeClass@@HIKPAU_SECURITY_ATTRIBUTES@@@Z 0047591c f   mfc90:mfc90.dll
 0001:00074922       ?PreTranslateMessage@CFormView@@MAEHPAUtagMSG@@@Z 00475922 f   mfc90:mfc90.dll
 0001:00074928       ?GetAccessibleChild@CWnd@@QAEJUtagVARIANT@@PAPAUIDispatch@@@Z 00475928 f   mfc90:mfc90.dll
 0001:0007492e       ?GetAccessibleChildCount@CWnd@@QAEJXZ 0047592e f   mfc90:mfc90.dll
 0001:00074934       ?GetAccessibleName@CWnd@@QAEJUtagVARIANT@@PAPA_W@Z 00475934 f   mfc90:mfc90.dll
 0001:0007493a       ?GetAccessibilityLocation@CWnd@@QAEJUtagVARIANT@@PAJ111@Z 0047593a f   mfc90:mfc90.dll
 0001:00074940       ?GetAccessibilityHitTest@CWnd@@QAEJJJPAUtagVARIANT@@@Z 00475940 f   mfc90:mfc90.dll
 0001:00074946       ?FromHandle@CImageList@@SGPAV1@PAU_IMAGELIST@@@Z 00475946 f   mfc90:mfc90.dll
 0001:0007494c       ??1CMapStringToString@@UAE@XZ 0047594c f   mfc90:mfc90.dll
 0001:00074952       ?RemoveKey@CMapStringToString@@QAEHPBD@Z 00475952 f   mfc90:mfc90.dll
 0001:00074958       ?Lookup@CMapStringToString@@QBEHPBDAAV?$CStringT@DV?$StrTraitMFC_DLL@DV?$ChTraitsCRT@D@ATL@@@@@ATL@@@Z 00475958 f   mfc90:mfc90.dll
 0001:0007495e       ?InitHashTable@CMapStringToString@@QAEXIH@Z 0047595e f   mfc90:mfc90.dll
 0001:00074964       ??0CMapStringToString@@QAE@H@Z 00475964 f   mfc90:mfc90.dll
 0001:0007496a       ??ACMapStringToString@@QAEAAV?$CStringT@DV?$StrTraitMFC_DLL@DV?$ChTraitsCRT@D@ATL@@@@@ATL@@PBD@Z 0047596a f   mfc90:mfc90.dll
 0001:00074970       ?GetThisMessageMap@CListCtrl@@KGPBUAFX_MSGMAP@@XZ 00475970 f   mfc90:mfc90.dll
 0001:00074976       ?GetThisMessageMap@CFrameWndEx@@KGPBUAFX_MSGMAP@@XZ 00475976 f   mfc90:mfc90.dll
 0001:0007497c       ?OnSetFocus@CFrameWnd@@IAEXPAVCWnd@@@Z 0047597c f   mfc90:mfc90.dll
 0001:00074982       ??1CMFCRibbonStatusBar@@UAE@XZ 00475982 f   mfc90:mfc90.dll
 0001:00074988       ??1CMFCCaptionBar@@UAE@XZ  00475988 f   mfc90:mfc90.dll
 0001:0007498e       ??1CMFCShellTreeCtrl@@UAE@XZ 0047598e f   mfc90:mfc90.dll
 0001:00074994       ??1CMFCToolBarImages@@UAE@XZ 00475994 f   mfc90:mfc90.dll
 0001:0007499a       ??1CSplitterWnd@@UAE@XZ    0047599a f   mfc90:mfc90.dll
 0001:000749a0       ??1CFrameWndEx@@MAE@XZ     004759a0 f   mfc90:mfc90.dll
 0001:000749a6       ?GetInt@CWinAppEx@@QAEHPBDH@Z 004759a6 f   mfc90:mfc90.dll
 0001:000749ac       ??0CMFCRibbonStatusBar@@QAE@XZ 004759ac f   mfc90:mfc90.dll
 0001:000749b2       ??0CMFCCaptionBar@@QAE@XZ  004759b2 f   mfc90:mfc90.dll
 0001:000749b8       ??0CMFCShellTreeCtrl@@QAE@XZ 004759b8 f   mfc90:mfc90.dll
 0001:000749be       ??0CMFCToolBarImages@@QAE@XZ 004759be f   mfc90:mfc90.dll
 0001:000749c4       ??0CSplitterWnd@@QAE@XZ    004759c4 f   mfc90:mfc90.dll
 0001:000749ca       ??0CFrameWndEx@@IAE@XZ     004759ca f   mfc90:mfc90.dll
 0001:000749d0       ?OnCmdMsg@CFrameWndEx@@UAEHIHPAXPAUAFX_CMDHANDLERINFO@@@Z 004759d0 f   mfc90:mfc90.dll
 0001:000749d6       ?GetMenu@CFrameWnd@@UBEPAVCMenu@@XZ 004759d6 f   mfc90:mfc90.dll
 0001:000749dc       ?SetMenu@CFrameWnd@@UAEHPAVCMenu@@@Z 004759dc f   mfc90:mfc90.dll
 0001:000749e2       ?WinHelpA@CFrameWndEx@@UAEXKI@Z 004759e2 f   mfc90:mfc90.dll
 0001:000749e8       ?HtmlHelpA@CFrameWndEx@@MAEXKI@Z 004759e8 f   mfc90:mfc90.dll
 0001:000749ee       ?OnCommand@CFrameWndEx@@MAEHIJ@Z 004759ee f   mfc90:mfc90.dll
 0001:000749f4       ?BeginModalState@CFrameWnd@@UAEXXZ 004759f4 f   mfc90:mfc90.dll
 0001:000749fa       ?EndModalState@CFrameWnd@@UAEXXZ 004759fa f   mfc90:mfc90.dll
 0001:00074a00       ?PostNcDestroy@CFrameWnd@@MAEXXZ 00475a00 f   mfc90:mfc90.dll
 0001:00074a06       ?IsFrameWnd@CFrameWnd@@UBEHXZ 00475a06 f   mfc90:mfc90.dll
 0001:00074a0c       ?Create@CFrameWnd@@UAEHPBD0KABUtagRECT@@PAVCWnd@@0KPAUCCreateContext@@@Z 00475a0c f   mfc90:mfc90.dll
 0001:00074a12       ?LoadFrame@CFrameWndEx@@UAEHIKPAVCWnd@@PAUCCreateContext@@@Z 00475a12 f   mfc90:mfc90.dll
 0001:00074a18       ?GetActiveDocument@CFrameWnd@@UAEPAVCDocument@@XZ 00475a18 f   mfc90:mfc90.dll
 0001:00074a1e       ?GetActiveFrame@CFrameWnd@@UAEPAV1@XZ 00475a1e f   mfc90:mfc90.dll
 0001:00074a24       ?GetMessageString@CFrameWnd@@UBEXIAAV?$CStringT@DV?$StrTraitMFC_DLL@DV?$ChTraitsCRT@D@ATL@@@@@ATL@@@Z 00475a24 f   mfc90:mfc90.dll
 0001:00074a2a       ?RecalcLayout@CFrameWndEx@@UAEXH@Z 00475a2a f   mfc90:mfc90.dll
 0001:00074a30       ?ActivateFrame@CFrameWnd@@UAEXH@Z 00475a30 f   mfc90:mfc90.dll
 0001:00074a36       ?SetMenuBarVisibility@CFrameWnd@@UAEXK@Z 00475a36 f   mfc90:mfc90.dll
 0001:00074a3c       ?GetMenuBarVisibility@CFrameWnd@@UBEKXZ 00475a3c f   mfc90:mfc90.dll
 0001:00074a42       ?SetMenuBarState@CFrameWnd@@UAEHK@Z 00475a42 f   mfc90:mfc90.dll
 0001:00074a48       ?GetMenuBarState@CFrameWnd@@UBEKXZ 00475a48 f   mfc90:mfc90.dll
 0001:00074a4e       ?OnSetPreviewMode@CFrameWndEx@@UAEXHPAUCPrintPreviewState@@@Z 00475a4e f   mfc90:mfc90.dll
 0001:00074a54       ?GetMessageBar@CFrameWnd@@UAEPAVCWnd@@XZ 00475a54 f   mfc90:mfc90.dll
 0001:00074a5a       ?NegotiateBorderSpace@CFrameWndEx@@UAEHIPAUtagRECT@@@Z 00475a5a f   mfc90:mfc90.dll
 0001:00074a60       ?OnUpdateFrameTitle@CFrameWndEx@@UAEXH@Z 00475a60 f   mfc90:mfc90.dll
 0001:00074a66       ?OnUpdateFrameMenu@CFrameWndEx@@UAEXPAUHMENU__@@@Z 00475a66 f   mfc90:mfc90.dll
 0001:00074a6c       ?GetDefaultAccelerator@CFrameWnd@@UAEPAUHACCEL__@@XZ 00475a6c f   mfc90:mfc90.dll
 0001:00074a72       ?DelayUpdateFrameMenu@CFrameWndEx@@UAEXPAUHMENU__@@@Z 00475a72 f   mfc90:mfc90.dll
 0001:00074a78       ?ExitHelpMode@CFrameWnd@@UAEXXZ 00475a78 f   mfc90:mfc90.dll
 0001:00074a7e       ?OnShowMenuBar@CFrameWnd@@MAEXXZ 00475a7e f   mfc90:mfc90.dll
 0001:00074a84       ?OnHideMenuBar@CFrameWnd@@MAEXXZ 00475a84 f   mfc90:mfc90.dll
 0001:00074a8a       ?AdjustDockingLayout@CFrameWndEx@@UAEXPAX@Z 00475a8a f   mfc90:mfc90.dll
 0001:00074a90       ?OnMoveMiniFrame@CFrameWndEx@@UAEHPAVCWnd@@@Z 00475a90 f   mfc90:mfc90.dll
 0001:00074a96       ?AdjustClientArea@CFrameWndEx@@MAEXXZ 00475a96 f   mfc90:mfc90.dll
 0001:00074a9c       ?GetInPlaceActiveItem@CFrameWndEx@@MAEPAVCOleClientItem@@XZ 00475a9c f   mfc90:mfc90.dll
 0001:00074aa2       ?OnShowPopupMenu@CFrameWndEx@@UAEHPAVCMFCPopupMenu@@@Z 00475aa2 f   mfc90:mfc90.dll
 0001:00074aa8       ?OnClosePopupMenu@CFrameWndEx@@UAEXPAVCMFCPopupMenu@@@Z 00475aa8 f   mfc90:mfc90.dll
 0001:00074aae       ?OnDrawMenuImage@CFrameWndEx@@UAEHPAVCDC@@PBVCMFCToolBarMenuButton@@ABVCRect@@@Z 00475aae f   mfc90:mfc90.dll
 0001:00074ab4       ?OnShowPanes@CFrameWndEx@@UAEHH@Z 00475ab4 f   mfc90:mfc90.dll
 0001:00074aba       ??0CMFCOutlookBar@@QAE@XZ  00475aba f   mfc90:mfc90.dll
 0001:00074ac0       ?GetRuntimeClass@CMFCOutlookBar@@UBEPAUCRuntimeClass@@XZ 00475ac0 f   mfc90:mfc90.dll
 0001:00074ac6       ?Serialize@CBaseTabbedPane@@UAEXAAVCArchive@@@Z 00475ac6 f   mfc90:mfc90.dll
 0001:00074acc       ?get_accParent@CBasePane@@UAEJPAPAUIDispatch@@@Z 00475acc f   mfc90:mfc90.dll
 0001:00074ad2       ?get_accChildCount@CBasePane@@UAEJPAJ@Z 00475ad2 f   mfc90:mfc90.dll
 0001:00074ad8       ?get_accChild@CBasePane@@UAEJUtagVARIANT@@PAPAUIDispatch@@@Z 00475ad8 f   mfc90:mfc90.dll
 0001:00074ade       ?get_accName@CBasePane@@UAEJUtagVARIANT@@PAPA_W@Z 00475ade f   mfc90:mfc90.dll
 0001:00074ae4       ?get_accValue@CBasePane@@UAEJUtagVARIANT@@PAPA_W@Z 00475ae4 f   mfc90:mfc90.dll
 0001:00074aea       ?get_accDescription@CBasePane@@UAEJUtagVARIANT@@PAPA_W@Z 00475aea f   mfc90:mfc90.dll
 0001:00074af0       ?get_accRole@CBasePane@@UAEJUtagVARIANT@@PAU2@@Z 00475af0 f   mfc90:mfc90.dll
 0001:00074af6       ?get_accState@CBasePane@@UAEJUtagVARIANT@@PAU2@@Z 00475af6 f   mfc90:mfc90.dll
 0001:00074afc       ?get_accHelp@CBasePane@@UAEJUtagVARIANT@@PAPA_W@Z 00475afc f   mfc90:mfc90.dll
 0001:00074b02       ?get_accHelpTopic@CBasePane@@UAEJPAPA_WUtagVARIANT@@PAJ@Z 00475b02 f   mfc90:mfc90.dll
 0001:00074b08       ?get_accKeyboardShortcut@CBasePane@@UAEJUtagVARIANT@@PAPA_W@Z 00475b08 f   mfc90:mfc90.dll
 0001:00074b0e       ?get_accFocus@CBasePane@@UAEJPAUtagVARIANT@@@Z 00475b0e f   mfc90:mfc90.dll
 0001:00074b14       ?get_accSelection@CBasePane@@UAEJPAUtagVARIANT@@@Z 00475b14 f   mfc90:mfc90.dll
 0001:00074b1a       ?get_accDefaultAction@CBasePane@@UAEJUtagVARIANT@@PAPA_W@Z 00475b1a f   mfc90:mfc90.dll
 0001:00074b20       ?accSelect@CBasePane@@UAEJJUtagVARIANT@@@Z 00475b20 f   mfc90:mfc90.dll
 0001:00074b26       ?accLocation@CBasePane@@UAEJPAJ000UtagVARIANT@@@Z 00475b26 f   mfc90:mfc90.dll
 0001:00074b2c       ?accHitTest@CBasePane@@UAEJJJPAUtagVARIANT@@@Z 00475b2c f   mfc90:mfc90.dll
 0001:00074b32       ?PreTranslateMessage@CDockablePane@@UAEHPAUtagMSG@@@Z 00475b32 f   mfc90:mfc90.dll
 0001:00074b38       ?WindowProc@CBasePane@@MAEJIIJ@Z 00475b38 f   mfc90:mfc90.dll
 0001:00074b3e       ?IsDocked@CDockablePane@@UBEHXZ 00475b3e f   mfc90:mfc90.dll
 0001:00074b44       ?IsTabbed@CPane@@UBEHXZ    00475b44 f   mfc90:mfc90.dll
 0001:00074b4a       ?IsMDITabbed@CBasePane@@UBEHXZ 00475b4a f   mfc90:mfc90.dll
 0001:00074b50       ?IsVisible@CDockablePane@@UBEHXZ 00475b50 f   mfc90:mfc90.dll
 0001:00074b56       ?CanAcceptPane@CMFCOutlookBar@@UBEHPBVCBasePane@@@Z 00475b56 f   mfc90:mfc90.dll
 0001:00074b5c       ?CanBeTabbedDocument@CPane@@UBEHXZ 00475b5c f   mfc90:mfc90.dll
 0001:00074b62       ?GetCurrentAlignment@CBasePane@@UBEKXZ 00475b62 f   mfc90:mfc90.dll
 0001:00074b68       ?GetDockSiteFrameWnd@CBasePane@@UBEPAVCWnd@@XZ 00475b68 f   mfc90:mfc90.dll
 0001:00074b6e       ?GetCaptionHeight@CDockablePane@@UBEHXZ 00475b6e f   mfc90:mfc90.dll
 0001:00074b74       ?IsInFloatingMultiPaneFrameWnd@CDockablePane@@UBEHXZ 00475b74 f   mfc90:mfc90.dll
 0001:00074b7a       ?GetDockingMode@CBasePane@@UBE?AW4AFX_DOCK_TYPE@@XZ 00475b7a f   mfc90:mfc90.dll
 0001:00074b80       ?GetPaneIcon@CBaseTabbedPane@@UAEPAUHICON__@@H@Z 00475b80 f   mfc90:mfc90.dll
 0001:00074b86       ?CanFloat@CBaseTabbedPane@@UBEHXZ 00475b86 f   mfc90:mfc90.dll
 0001:00074b8c       ?CanAutoHide@CDockablePane@@UBEHXZ 00475b8c f   mfc90:mfc90.dll
 0001:00074b92       ?EnableGripper@CDockablePane@@UAEXH@Z 00475b92 f   mfc90:mfc90.dll
 0001:00074b98       ?DockPane@CPane@@UAEHPAVCBasePane@@PBUtagRECT@@W4AFX_DOCK_METHOD@@@Z 00475b98 f   mfc90:mfc90.dll
 0001:00074b9e       ?FloatPane@CBaseTabbedPane@@MAEHVCRect@@W4AFX_DOCK_METHOD@@_N@Z 00475b9e f   mfc90:mfc90.dll
 0001:00074ba4       ?DockToFrameWindow@CDockablePane@@UAEHKPBUtagRECT@@KPAVCBasePane@@HH@Z 00475ba4 f   mfc90:mfc90.dll
 0001:00074baa       ?RecalcLayout@CBaseTabbedPane@@UAEXXZ 00475baa f   mfc90:mfc90.dll
 0001:00074bb0       ?CreateDefaultMiniframe@CPane@@UAEPAVCPaneFrameWnd@@VCRect@@@Z 00475bb0 f   mfc90:mfc90.dll
 0001:00074bb6       ?OnBeforeChangeParent@CDockablePane@@UAEXPAVCWnd@@H@Z 00475bb6 f   mfc90:mfc90.dll
 0001:00074bbc       ?OnAfterChangeParent@CDockablePane@@UAEXPAVCWnd@@@Z 00475bbc f   mfc90:mfc90.dll
 0001:00074bc2       ?ShowPane@CDockablePane@@UAEXHHH@Z 00475bc2 f   mfc90:mfc90.dll
 0001:00074bc8       ?GetParentMiniFrame@CBasePane@@UBEPAVCPaneFrameWnd@@H@Z 00475bc8 f   mfc90:mfc90.dll
 0001:00074bce       ?LoadState@CMFCOutlookBar@@UAEHPBDHI@Z 00475bce f   mfc90:mfc90.dll
 0001:00074bd4       ?SaveState@CMFCOutlookBar@@UAEHPBDHI@Z 00475bd4 f   mfc90:mfc90.dll
 0001:00074bda       ?MoveWindow@CBasePane@@UAEPAXAAVCRect@@HPAX@Z 00475bda f   mfc90:mfc90.dll
 0001:00074be0       ?SetWindowPos@CBasePane@@UAEPAXPBVCWnd@@HHHHIPAX@Z 00475be0 f   mfc90:mfc90.dll
 0001:00074be6       ?CopyState@CBasePane@@UAEXPAV1@@Z 00475be6 f   mfc90:mfc90.dll
 0001:00074bec       ?UndockPane@CDockablePane@@UAEXH@Z 00475bec f   mfc90:mfc90.dll
 0001:00074bf2       ?OnUpdateCmdUI@CDockablePane@@UAEXPAVCFrameWnd@@H@Z 00475bf2 f   mfc90:mfc90.dll
 0001:00074bf8       ?OnPaneContextMenu@CBasePane@@UAEXPAVCWnd@@VCPoint@@@Z 00475bf8 f   mfc90:mfc90.dll
 0001:00074bfe       ?CreateEx@CBasePane@@UAEHKPBD0KABUtagRECT@@PAVCWnd@@IKPAUCCreateContext@@@Z 00475bfe f   mfc90:mfc90.dll
 0001:00074c04       ?OnSetAccData@CBasePane@@UAEHJ@Z 00475c04 f   mfc90:mfc90.dll
 0001:00074c0a       ?CalcFixedLayout@CDockablePane@@UAE?AVCSize@@HH@Z 00475c0a f   mfc90:mfc90.dll
 0001:00074c10       ?DoPaint@CBasePane@@MAEXPAVCDC@@@Z 00475c10 f   mfc90:mfc90.dll
 0001:00074c16       ?AdjustDockingLayout@CBasePane@@UAEXPAX@Z 00475c16 f   mfc90:mfc90.dll
 0001:00074c1c       ?GetMinSize@CBaseTabbedPane@@UBEXAAVCSize@@@Z 00475c1c f   mfc90:mfc90.dll
 0001:00074c22       ?GetAvailableExpandSize@CPane@@UBEHXZ 00475c22 f   mfc90:mfc90.dll
 0001:00074c28       ?GetAvailableStretchSize@CPane@@UBEHXZ 00475c28 f   mfc90:mfc90.dll
 0001:00074c2e       ?CopyState@CPane@@UAEXPAV1@@Z 00475c2e f   mfc90:mfc90.dll
 0001:00074c34       ?SetActiveInGroup@CPane@@UAEXH@Z 00475c34 f   mfc90:mfc90.dll
 0001:00074c3a       ?PrepareToDock@CPane@@UAEXPAVCDockSite@@W4AFX_DOCK_METHOD@@@Z 00475c3a f   mfc90:mfc90.dll
 0001:00074c40       ?DockByMouse@CPane@@UAEHPAVCBasePane@@@Z 00475c40 f   mfc90:mfc90.dll
 0001:00074c46       ?MovePane@CPane@@UAE?AVCSize@@VCRect@@HAAPAX@Z 00475c46 f   mfc90:mfc90.dll
 0001:00074c4c       ?StretchPaneDeferWndPos@CPane@@UAEHHAAPAX@Z 00475c4c f   mfc90:mfc90.dll
 0001:00074c52       ?DockPaneStandard@CDockablePane@@UAEPAVCPane@@AAH@Z 00475c52 f   mfc90:mfc90.dll
 0001:00074c58       ?IsChangeState@CDockablePane@@UBE?AW4AFX_CS_STATUS@@HPAPAVCBasePane@@@Z 00475c58 f   mfc90:mfc90.dll
 0001:00074c5e       ?SetDockState@CPane@@UAEXPAVCDockingManager@@@Z 00475c5e f   mfc90:mfc90.dll
 0001:00074c64       ?OnProcessDblClk@CPane@@UAEXXZ 00475c64 f   mfc90:mfc90.dll
 0001:00074c6a       ?OnBeforeFloat@CDockablePane@@UAEHAAVCRect@@W4AFX_DOCK_METHOD@@@Z 00475c6a f   mfc90:mfc90.dll
 0001:00074c70       ?OnAfterFloat@CPane@@UAEXXZ 00475c70 f   mfc90:mfc90.dll
 0001:00074c76       ?Create@CPane@@UAEHPBDKABUtagRECT@@PAVCWnd@@IKPAUCCreateContext@@@Z 00475c76 f   mfc90:mfc90.dll
 0001:00074c7c       ?CreateEx@CPane@@UAEHKPBDKABUtagRECT@@PAVCWnd@@IKPAUCCreateContext@@@Z 00475c7c f   mfc90:mfc90.dll
 0001:00074c82       ?CalcAvailableSize@CPane@@UAE?AVCSize@@VCRect@@@Z 00475c82 f   mfc90:mfc90.dll
 0001:00074c88       ?AdjustSizeImmediate@CPane@@UAEXH@Z 00475c88 f   mfc90:mfc90.dll
 0001:00074c8e       ?ToggleAutoHide@CDockablePane@@UAEXXZ 00475c8e f   mfc90:mfc90.dll
 0001:00074c94       ?OnPressCloseButton@CDockablePane@@MAEXXZ 00475c94 f   mfc90:mfc90.dll
 0001:00074c9a       ?ConvertToTabbedDocument@CBaseTabbedPane@@UAEXH@Z 00475c9a f   mfc90:mfc90.dll
 0001:00074ca0       ?OnShowControlBarMenu@CPane@@UAEHVCPoint@@@Z 00475ca0 f   mfc90:mfc90.dll
 0001:00074ca6       ?OnDrawDragRect@CDockablePane@@MAEXPBUtagRECT@@0@Z 00475ca6 f   mfc90:mfc90.dll
 0001:00074cac       ?OnBeforeDock@CPane@@MAEHPAPAVCBasePane@@PBUtagRECT@@W4AFX_DOCK_METHOD@@@Z 00475cac f   mfc90:mfc90.dll
 0001:00074cb2       ?OnAfterDock@CDockablePane@@MAEXPAVCBasePane@@PBUtagRECT@@W4AFX_DOCK_METHOD@@@Z 00475cb2 f   mfc90:mfc90.dll
 0001:00074cb8       ?RemoveFromMiniframe@CPane@@MAEXPAVCWnd@@W4AFX_DOCK_METHOD@@@Z 00475cb8 f   mfc90:mfc90.dll
 0001:00074cbe       ?SetDragMode@CPane@@MAEXH@Z 00475cbe f   mfc90:mfc90.dll
 0001:00074cc4       ?Dock@CBaseTabbedPane@@MAEHPAVCBasePane@@PBUtagRECT@@W4AFX_DOCK_METHOD@@@Z 00475cc4 f   mfc90:mfc90.dll
 0001:00074cca       ?EnterDragMode@CDockablePane@@MAEXH@Z 00475cca f   mfc90:mfc90.dll
 0001:00074cd0       ?OnRTLChanged@CPane@@MAEXH@Z 00475cd0 f   mfc90:mfc90.dll
 0001:00074cd6       ?StoreRecentDockSiteInfo@CBaseTabbedPane@@MAEXXZ 00475cd6 f   mfc90:mfc90.dll
 0001:00074cdc       ?Create@CDockablePane@@UAEHPBDPAVCWnd@@VCSize@@HIKKK@Z 00475cdc f   mfc90:mfc90.dll
 0001:00074ce2       ?Create@CDockablePane@@UAEHPBDPAVCWnd@@ABUtagRECT@@HIKKKPAUCCreateContext@@@Z 00475ce2 f   mfc90:mfc90.dll
 0001:00074ce8       ?CreateEx@CDockablePane@@UAEHKPBDPAVCWnd@@ABUtagRECT@@HIKKKPAUCCreateContext@@@Z 00475ce8 f   mfc90:mfc90.dll
 0001:00074cee       ?GetTabArea@CMFCOutlookBar@@UBEXAAVCRect@@0@Z 00475cee f   mfc90:mfc90.dll
 0001:00074cf4       ?HitTest@CDockablePane@@UAEHVCPoint@@H@Z 00475cf4 f   mfc90:mfc90.dll
 0001:00074cfa       ?CanAcceptMiniFrame@CDockablePane@@UBEHPAVCPaneFrameWnd@@@Z 00475cfa f   mfc90:mfc90.dll
 0001:00074d00       ?Slide@CDockablePane@@UAEXHH@Z 00475d00 f   mfc90:mfc90.dll
 0001:00074d06       ?GetDockingStatus@CMFCOutlookBar@@UAE?AW4AFX_CS_STATUS@@VCPoint@@H@Z 00475d06 f   mfc90:mfc90.dll
 0001:00074d0c       ?AttachToTabWnd@CDockablePane@@UAEPAV1@PAV1@W4AFX_DOCK_METHOD@@HPAPAV1@@Z 00475d0c f   mfc90:mfc90.dll
 0001:00074d12       ?CreateTabbedPane@CDockablePane@@UAEPAVCTabbedPane@@XZ 00475d12 f   mfc90:mfc90.dll
 0001:00074d18       ?DockToWindow@CDockablePane@@UAEHPAV1@KPBUtagRECT@@@Z 00475d18 f   mfc90:mfc90.dll
 0001:00074d1e       ?DockPaneContainer@CDockablePane@@UAEHAAVCPaneContainerManager@@KW4AFX_DOCK_METHOD@@@Z 00475d1e f   mfc90:mfc90.dll
 0001:00074d24       ?UnSetAutoHideMode@CDockablePane@@UAEXPAV1@@Z 00475d24 f   mfc90:mfc90.dll
 0001:00074d2a       ?SetAutoHideMode@CBaseTabbedPane@@UAEPAVCMFCAutoHideBar@@HKPAV2@H@Z 00475d2a f   mfc90:mfc90.dll
 0001:00074d30       ?CopyState@CDockablePane@@UAEXPAV1@@Z 00475d30 f   mfc90:mfc90.dll
 0001:00074d36       ?StoreRecentTabRelatedInfo@CDockablePane@@MAEXXZ 00475d36 f   mfc90:mfc90.dll
 0001:00074d3c       ?DrawCaption@CDockablePane@@MAEXPAVCDC@@VCRect@@@Z 00475d3c f   mfc90:mfc90.dll
 0001:00074d42       ?AdjustPaneToPaneContainer@CDockablePane@@MAEXPAVCPaneDivider@@@Z 00475d42 f   mfc90:mfc90.dll
 0001:00074d48       ?OnTrackCaptionButtons@CDockablePane@@MAEXVCPoint@@@Z 00475d48 f   mfc90:mfc90.dll
 0001:00074d4e       ?StopCaptionButtonsTracking@CDockablePane@@MAEXXZ 00475d4e f   mfc90:mfc90.dll
 0001:00074d54       ?SetCaptionButtons@CDockablePane@@MAEXXZ 00475d54 f   mfc90:mfc90.dll
 0001:00074d5a       ?CheckAutoHideCondition@CDockablePane@@MAEHXZ 00475d5a f   mfc90:mfc90.dll
 0001:00074d60       ?CheckStopSlideCondition@CDockablePane@@MAEHH@Z 00475d60 f   mfc90:mfc90.dll
 0001:00074d66       ?OnSlide@CDockablePane@@MAEXH@Z 00475d66 f   mfc90:mfc90.dll
 0001:00074d6c       ?AddTab@CBaseTabbedPane@@UAEHPAVCWnd@@HHH@Z 00475d6c f   mfc90:mfc90.dll
 0001:00074d72       ?FloatTab@CMFCOutlookBar@@UAEHPAVCWnd@@HW4AFX_DOCK_METHOD@@H@Z 00475d72 f   mfc90:mfc90.dll
 0001:00074d78       ?DetachPane@CBaseTabbedPane@@UAEHPAVCWnd@@H@Z 00475d78 f   mfc90:mfc90.dll
 0001:00074d7e       ?RemovePane@CBaseTabbedPane@@UAEHPAVCWnd@@@Z 00475d7e f   mfc90:mfc90.dll
 0001:00074d84       ?ShowTab@CBaseTabbedPane@@UAEHPAVCWnd@@HHH@Z 00475d84 f   mfc90:mfc90.dll
 0001:00074d8a       ?FindPaneByID@CBaseTabbedPane@@UAEPAVCWnd@@I@Z 00475d8a f   mfc90:mfc90.dll
 0001:00074d90       ?FindBarByTabNumber@CBaseTabbedPane@@UAEPAVCWnd@@HH@Z 00475d90 f   mfc90:mfc90.dll
 0001:00074d96       ?GetFirstVisibleTab@CBaseTabbedPane@@UAEPAVCWnd@@AAH@Z 00475d96 f   mfc90:mfc90.dll
 0001:00074d9c       ?ApplyRestoredTabInfo@CBaseTabbedPane@@UAEXH@Z 00475d9c f   mfc90:mfc90.dll
 0001:00074da2       ?SerializeTabWindow@CBaseTabbedPane@@UAEXAAVCArchive@@@Z 00475da2 f   mfc90:mfc90.dll
 0001:00074da8       ?SaveSiblingBarIDs@CBaseTabbedPane@@UAEXAAVCArchive@@@Z 00475da8 f   mfc90:mfc90.dll
 0001:00074dae       ?GetPaneList@CBaseTabbedPane@@UAEXAAVCObList@@PAUCRuntimeClass@@@Z 00475dae f   mfc90:mfc90.dll
 0001:00074db4       ?Create@CMFCOutlookBar@@UAEHPBDPAVCWnd@@ABUtagRECT@@IKKPAUCCreateContext@@@Z 00475db4 f   mfc90:mfc90.dll
 0001:00074dba       ??1CMFCOutlookBar@@UAE@XZ  00475dba f   mfc90:mfc90.dll
 0001:00074dc0       ?DockPane@CFrameWndEx@@QAEXPAVCBasePane@@IPBUtagRECT@@@Z 00475dc0 f   mfc90:mfc90.dll
 0001:00074dc6       ?ExtractIconA@CMFCToolBarImages@@QAEPAUHICON__@@H@Z 00475dc6 f   mfc90:mfc90.dll
 0001:00074dcc       ?Load@CMFCToolBarImages@@QAEHIPAUHINSTANCE__@@H@Z 00475dcc f   mfc90:mfc90.dll
 0001:00074dd2       ?EnableDocking@CFrameWndEx@@QAEHK@Z 00475dd2 f   mfc90:mfc90.dll
 0001:00074dd8       ?EnableAutoHidePanes@CFrameWndEx@@QAEHK@Z 00475dd8 f   mfc90:mfc90.dll
 0001:00074dde       ?SetDockingMode@CDockingManager@@SGXW4AFX_DOCK_TYPE@@@Z 00475dde f   mfc90:mfc90.dll
 0001:00074de4       ?AddExtendedElement@CMFCRibbonStatusBar@@QAEXPAVCMFCRibbonBaseElement@@PBDH@Z 00475de4 f   mfc90:mfc90.dll
 0001:00074dea       ?AddElement@CMFCRibbonStatusBar@@QAEXPAVCMFCRibbonBaseElement@@PBDH@Z 00475dea f   mfc90:mfc90.dll
 0001:00074df0       ??0CMFCRibbonStatusBarPane@@QAE@IPBDHPAUHICON__@@0@Z 00475df0 f   mfc90:mfc90.dll
 0001:00074df6       ?Create@CMFCRibbonStatusBar@@QAEHPAVCWnd@@KI@Z 00475df6 f   mfc90:mfc90.dll
 0001:00074dfc       ?Create@CMFCRibbonBar@@QAEHPAVCWnd@@KI@Z 00475dfc f   mfc90:mfc90.dll
 0001:00074e02       ?OnCreate@CFrameWndEx@@QAEHPAUtagCREATESTRUCTA@@@Z 00475e02 f   mfc90:mfc90.dll
 0001:00074e08       ?PreCreateWindow@CFrameWndEx@@MAEHAAUtagCREATESTRUCTA@@@Z 00475e08 f   mfc90:mfc90.dll
 0001:00074e0e       ?AddToTabs@CMFCRibbonBar@@QAEXPAVCMFCRibbonBaseElement@@@Z 00475e0e f   mfc90:mfc90.dll
 0001:00074e14       ??0CMFCRibbonButton@@QAE@IPBDHHH@Z 00475e14 f   mfc90:mfc90.dll
 0001:00074e1a       ?AddMainCategory@CMFCRibbonBar@@QAEPAVCMFCRibbonMainPanel@@PBDIIVCSize@@1@Z 00475e1a f   mfc90:mfc90.dll
 0001:00074e20       ?SetApplicationButton@CMFCRibbonBar@@QAEXPAVCMFCRibbonApplicationButton@@VCSize@@@Z 00475e20 f   mfc90:mfc90.dll
 0001:00074e26       ?SetImage@CMFCRibbonApplicationButton@@QAEXI@Z 00475e26 f   mfc90:mfc90.dll
 0001:00074e2c       ?Create@CTreeCtrl@@QAEHKABUtagRECT@@PAVCWnd@@I@Z 00475e2c f   mfc90:mfc90.dll
 0001:00074e32       ?WriteInt@CWinAppEx@@QAEHPBDH@Z 00475e32 f   mfc90:mfc90.dll
 0001:00074e38       ?GetThisClass@CMFCVisualManagerOffice2007@@SGPAUCRuntimeClass@@XZ 00475e38 f   mfc90:mfc90.dll
 0001:00074e3e       ?SetStyle@CMFCVisualManagerOffice2007@@SGHW4Style@1@PBD@Z 00475e3e f   mfc90:mfc90.dll
 0001:00074e44       ?GetThisClass@CMFCVisualManagerVS2005@@SGPAUCRuntimeClass@@XZ 00475e44 f   mfc90:mfc90.dll
 0001:00074e4a       ?GetThisClass@CMFCVisualManagerOffice2003@@SGPAUCRuntimeClass@@XZ 00475e4a f   mfc90:mfc90.dll
 0001:00074e50       ?GetThisClass@CMFCVisualManagerWindows@@SGPAUCRuntimeClass@@XZ 00475e50 f   mfc90:mfc90.dll
 0001:00074e56       ?GetThisClass@CMFCVisualManagerOfficeXP@@SGPAUCRuntimeClass@@XZ 00475e56 f   mfc90:mfc90.dll
 0001:00074e5c       ?SetDefaultManager@CMFCVisualManager@@SGXPAUCRuntimeClass@@@Z 00475e5c f   mfc90:mfc90.dll
 0001:00074e62       ?GetThisClass@CMFCVisualManager@@SGPAUCRuntimeClass@@XZ 00475e62 f   mfc90:mfc90.dll
 0001:00074e68       ?ShowPane@CFrameWndEx@@QAEXPAVCBasePane@@HHH@Z 00475e68 f   mfc90:mfc90.dll
 0001:00074e6e       ?SetInformation@CMFCRibbonStatusBar@@QAEXPBD@Z 00475e6e f   mfc90:mfc90.dll
 0001:00074e74       ??1CStringArray@@UAE@XZ    00475e74 f   mfc90:mfc90.dll
 0001:00074e7a       ??0CStringArray@@QAE@XZ    00475e7a f   mfc90:mfc90.dll
 0001:00074e80       ?AddPanel@CMFCRibbonCategory@@QAEPAVCMFCRibbonPanel@@PBDPAUHICON__@@PAUCRuntimeClass@@@Z 00475e80 f   mfc90:mfc90.dll
 0001:00074e86       ?AddCategory@CMFCRibbonBar@@QAEPAVCMFCRibbonCategory@@PBDIIVCSize@@1HPAUCRuntimeClass@@@Z 00475e86 f   mfc90:mfc90.dll
 0001:00074e8c       ??0CMFCRibbonCheckBox@@QAE@IPBD@Z 00475e8c f   mfc90:mfc90.dll
 0001:00074e92       ?OnClose@CFrameWndEx@@QAEXXZ 00475e92 f   mfc90:mfc90.dll
 0001:00074e98       ?OnSysCommand@CFrameWnd@@IAEXIJ@Z 00475e98 f   mfc90:mfc90.dll
 0001:00074e9e       ?PreTranslateMessage@CFrameWndEx@@UAEHPAUtagMSG@@@Z 00475e9e f   mfc90:mfc90.dll
 0001:00074ea4       ?SetWordCharFormat@CRichEditCtrl@@QAEHAAU_charformat@@@Z 00475ea4 f   mfc90:mfc90.dll
 0001:00074eaa       ?SetSel@CRichEditCtrl@@QAEXJJ@Z 00475eaa f   mfc90:mfc90.dll
 0001:00074eb0       ?GetWindowTextLengthA@CWnd@@QBEHXZ 00475eb0 f   mfc90:mfc90.dll
 0001:00074eb6       ?GetCategory@CMFCRibbonBar@@QBEPAVCMFCRibbonCategory@@H@Z 00475eb6 f   mfc90:mfc90.dll
 0001:00074ebc       ?DoModal@CPropertySheet@@UAEHXZ 00475ebc f   mfc90:mfc90.dll
 0001:00074ec2       ?EnablePageHeader@CMFCPropertySheet@@QAEXH@Z 00475ec2 f   mfc90:mfc90.dll
 0001:00074ec8       ?GetThisMessageMap@CMFCOutlookBar@@KGPBUAFX_MSGMAP@@XZ 00475ec8 f   mfc90:mfc90.dll
 0001:00074ece       ?OnRButtonDown@CDockablePane@@IAEXIVCPoint@@@Z 00475ece f   mfc90:mfc90.dll
 0001:00074ed4       ?RemoveHead@CPtrList@@QAEPAXXZ 00475ed4 f   mfc90:mfc90.dll
 0001:00074eda       ?AddTail@CPtrList@@QAEPAU__POSITION@@PAX@Z 00475eda f   mfc90:mfc90.dll
 0001:00074ee0       ?BeginWaitCursor@CCmdTarget@@QAEXXZ 00475ee0 f   mfc90:mfc90.dll
 0001:00074ee6       ?EndWaitCursor@CCmdTarget@@QAEXXZ 00475ee6 f   mfc90:mfc90.dll
 0001:00074eec       ?UpdateCount@CMFCToolBarImages@@IAEXXZ 00475eec f   mfc90:mfc90.dll
 0001:00074ef2       ?UpdateInternalImage@CMFCToolBarImages@@IAEHH@Z 00475ef2 f   mfc90:mfc90.dll
 0001:00074ef8       ??1CMFCRibbonButton@@UAE@XZ 00475ef8 f   mfc90:mfc90.dll
 0001:00074efe       ??0CMFCRibbonButton@@QAE@XZ 00475efe f   mfc90:mfc90.dll
 0001:00074f04       ?GetRuntimeClass@CMFCRibbonApplicationButton@@UBEPAUCRuntimeClass@@XZ 00475f04 f   mfc90:mfc90.dll
 0001:00074f0a       ?SetID@CMFCRibbonBaseElement@@UAEXI@Z 00475f0a f   mfc90:mfc90.dll
 0001:00074f10       ?SetText@CMFCRibbonButton@@UAEXPBD@Z 00475f10 f   mfc90:mfc90.dll
 0001:00074f16       ?SetKeys@CMFCRibbonBaseElement@@UAEXPBD0@Z 00475f16 f   mfc90:mfc90.dll
 0001:00074f1c       ?SetTextAlwaysOnRight@CMFCRibbonBaseElement@@UAEXH@Z 00475f1c f   mfc90:mfc90.dll
 0001:00074f22       ?GetToolTipText@CMFCRibbonButton@@UBE?AV?$CStringT@DV?$StrTraitMFC_DLL@DV?$ChTraitsCRT@D@ATL@@@@@ATL@@XZ 00475f22 f   mfc90:mfc90.dll
 0001:00074f28       ?GetDescription@CMFCRibbonBaseElement@@UBE?AV?$CStringT@DV?$StrTraitMFC_DLL@DV?$ChTraitsCRT@D@ATL@@@@@ATL@@XZ 00475f28 f   mfc90:mfc90.dll
 0001:00074f2e       ?SetToolTipText@CMFCRibbonBaseElement@@UAEXPBD@Z 00475f2e f   mfc90:mfc90.dll
 0001:00074f34       ?SetDescription@CMFCRibbonButton@@UAEXPBD@Z 00475f34 f   mfc90:mfc90.dll
 0001:00074f3a       ?GetRegularSize@CMFCRibbonButton@@UAE?AVCSize@@PAVCDC@@@Z 00475f3a f   mfc90:mfc90.dll
 0001:00074f40       ?GetCompactSize@CMFCRibbonButton@@UAE?AVCSize@@PAVCDC@@@Z 00475f40 f   mfc90:mfc90.dll
 0001:00074f46       ?GetIntermediateSize@CMFCRibbonButton@@UAE?AVCSize@@PAVCDC@@@Z 00475f46 f   mfc90:mfc90.dll
 0001:00074f4c       ?OnAfterChangeRect@CMFCRibbonButton@@MAEXPAVCDC@@@Z 00475f4c f   mfc90:mfc90.dll
 0001:00074f52       ?HitTest@CMFCRibbonBaseElement@@UAEPAV1@VCPoint@@@Z 00475f52 f   mfc90:mfc90.dll
 0001:00074f58       ?GetParentPanel@CMFCRibbonBaseElement@@UBEPAVCMFCRibbonPanel@@XZ 00475f58 f   mfc90:mfc90.dll
 0001:00074f5e       ?GetParentWnd@CMFCRibbonBaseElement@@UBEPAVCWnd@@XZ 00475f5e f   mfc90:mfc90.dll
 0001:00074f64       ?SetParentRibbonBar@CMFCRibbonButton@@MAEXPAVCMFCRibbonBar@@@Z 00475f64 f   mfc90:mfc90.dll
 0001:00074f6a       ?OnShowPopupMenu@CMFCRibbonButton@@MAEXXZ 00475f6a f   mfc90:mfc90.dll
 0001:00074f70       ?StretchToWholeRow@CMFCRibbonBaseElement@@UAEHPAVCDC@@H@Z 00475f70 f   mfc90:mfc90.dll
 0001:00074f76       ?SetParentCategory@CMFCRibbonButton@@UAEXPAVCMFCRibbonCategory@@@Z 00475f76 f   mfc90:mfc90.dll
 0001:00074f7c       ?CopyFrom@CMFCRibbonButton@@MAEXABVCMFCRibbonBaseElement@@@Z 00475f7c f   mfc90:mfc90.dll
 0001:00074f82       ?SetParentMenu@CMFCRibbonBaseElement@@UAEXPAVCMFCRibbonPanelMenuBar@@@Z 00475f82 f   mfc90:mfc90.dll
 0001:00074f88       ?SetOriginal@CMFCRibbonButton@@MAEXPAVCMFCRibbonBaseElement@@@Z 00475f88 f   mfc90:mfc90.dll
 0001:00074f8e       ?OnDrawOnList@CMFCRibbonButton@@MAEXPAVCDC@@V?$CStringT@DV?$StrTraitMFC_DLL@DV?$ChTraitsCRT@D@ATL@@@@@ATL@@HVCRect@@HH@Z 00475f8e f   mfc90:mfc90.dll
 0001:00074f94       ?OnDraw@CMFCRibbonButton@@UAEXPAVCDC@@@Z 00475f94 f   mfc90:mfc90.dll
 0001:00074f9a       ?OnCalcTextSize@CMFCRibbonButton@@UAEXPAVCDC@@@Z 00475f9a f   mfc90:mfc90.dll
 0001:00074fa0       ?CanBeStretched@CMFCRibbonButton@@UAEHXZ 00475fa0 f   mfc90:mfc90.dll
 0001:00074fa6       ?ClosePopupMenu@CMFCRibbonButton@@UAEXXZ 00475fa6 f   mfc90:mfc90.dll
 0001:00074fac       ?Find@CMFCRibbonBaseElement@@UAEPAV1@PBV1@@Z 00475fac f   mfc90:mfc90.dll
 0001:00074fb2       ?FindByID@CMFCRibbonButton@@MAEPAVCMFCRibbonBaseElement@@I@Z 00475fb2 f   mfc90:mfc90.dll
 0001:00074fb8       ?FindByData@CMFCRibbonButton@@MAEPAVCMFCRibbonBaseElement@@K@Z 00475fb8 f   mfc90:mfc90.dll
 0001:00074fbe       ?FindByOriginal@CMFCRibbonBaseElement@@UAEPAV1@PAV1@@Z 00475fbe f   mfc90:mfc90.dll
 0001:00074fc4       ?UpdateTooltipInfo@CMFCRibbonBaseElement@@UAEXXZ 00475fc4 f   mfc90:mfc90.dll
 0001:00074fca       ?OnAddToQAToolbar@CMFCRibbonBaseElement@@UAEHAAVCMFCRibbonQuickAccessToolBar@@@Z 00475fca f   mfc90:mfc90.dll
 0001:00074fd0       ?Redraw@CMFCRibbonBaseElement@@UAEXXZ 00475fd0 f   mfc90:mfc90.dll
 0001:00074fd6       ?GetPressed@CMFCRibbonBaseElement@@UAEPAV1@XZ 00475fd6 f   mfc90:mfc90.dll
 0001:00074fdc       ?GetDroppedDown@CMFCRibbonBaseElement@@UAEPAV1@XZ 00475fdc f   mfc90:mfc90.dll
 0001:00074fe2       ?GetHighlighted@CMFCRibbonBaseElement@@UAEPAV1@XZ 00475fe2 f   mfc90:mfc90.dll
 0001:00074fe8       ?OnDrawKeyTip@CMFCRibbonBaseElement@@UAEXPAVCDC@@ABVCRect@@H@Z 00475fe8 f   mfc90:mfc90.dll
 0001:00074fee       ?GetKeyTipSize@CMFCRibbonBaseElement@@UAE?AVCSize@@PAVCDC@@@Z 00475fee f   mfc90:mfc90.dll
 0001:00074ff4       ?GetKeyTipRect@CMFCRibbonButton@@MAE?AVCRect@@PAVCDC@@H@Z 00475ff4 f   mfc90:mfc90.dll
 0001:00074ffa       ?OnKey@CMFCRibbonApplicationButton@@MAEHH@Z 00475ffa f   mfc90:mfc90.dll
 0001:00075000       ?AddToKeyList@CMFCRibbonBaseElement@@UAEXAAV?$CArray@PAVCMFCRibbonKeyTip@@PAV1@@@@Z 00476000 f   mfc90:mfc90.dll
 0001:00075006       ?GetElementsByID@CMFCRibbonButton@@MAEXIAAV?$CArray@PAVCMFCRibbonBaseElement@@PAV1@@@@Z 00476006 f   mfc90:mfc90.dll
 0001:0007500c       ?GetElements@CMFCRibbonButton@@MAEXAAV?$CArray@PAVCMFCRibbonBaseElement@@PAV1@@@@Z 0047600c f   mfc90:mfc90.dll
 0001:00075012       ?NotifyHighlightListItem@CMFCRibbonBaseElement@@UAEXH@Z 00476012 f   mfc90:mfc90.dll
 0001:00075018       ?OnLButtonDown@CMFCRibbonApplicationButton@@MAEXVCPoint@@@Z 00476018 f   mfc90:mfc90.dll
 0001:0007501e       ?OnLButtonUp@CMFCRibbonButton@@MAEXVCPoint@@@Z 0047601e f   mfc90:mfc90.dll
 0001:00075024       ?OnMouseMove@CMFCRibbonButton@@MAEXVCPoint@@@Z 00476024 f   mfc90:mfc90.dll
 0001:0007502a       ?OnLButtonDblClk@CMFCRibbonApplicationButton@@MAEXVCPoint@@@Z 0047602a f   mfc90:mfc90.dll
 0001:00075030       ?OnUpdateCmdUI@CMFCRibbonBaseElement@@MAEXPAVCMFCRibbonCmdUI@@PAVCFrameWnd@@H@Z 00476030 f   mfc90:mfc90.dll
 0001:00075036       ?NotifyControlCommand@CMFCRibbonBaseElement@@MAEHHHIJ@Z 00476036 f   mfc90:mfc90.dll
 0001:0007503c       ?ReplaceByID@CMFCRibbonBaseElement@@MAEHIPAV1@@Z 0047603c f   mfc90:mfc90.dll
 0001:00075042       ?GetItemIDsList@CMFCRibbonBaseElement@@MBEXAAV?$CList@II@@@Z 00476042 f   mfc90:mfc90.dll
 0001:00075048       ?GetDropDownImageWidth@CMFCRibbonBaseElement@@MBEHXZ 00476048 f   mfc90:mfc90.dll
 0001:0007504e       ?DrawRibbonText@CMFCRibbonButton@@UAEHPAVCDC@@ABV?$CStringT@DV?$StrTraitMFC_DLL@DV?$ChTraitsCRT@D@ATL@@@@@ATL@@VCRect@@IK@Z 0047604e f   mfc90:mfc90.dll
 0001:00075054       ?OnClick@CMFCRibbonButton@@UAEXVCPoint@@@Z 00476054 f   mfc90:mfc90.dll
 0001:0007505a       ?OnFillBackground@CMFCRibbonButton@@UAEKPAVCDC@@@Z 0047605a f   mfc90:mfc90.dll
 0001:00075060       ?OnDrawBorder@CMFCRibbonButton@@UAEXPAVCDC@@@Z 00476060 f   mfc90:mfc90.dll
 0001:00075066       ?DrawEx@CMFCToolBarImages@@QAEHPAVCDC@@VCRect@@HW4ImageAlignHorz@1@W4ImageAlignVert@1@1E@Z 00476066 f   mfc90:mfc90.dll
 0001:0007506c       ?SetACCData@CMFCRibbonButton@@UAEHPAVCWnd@@AAVCAccessibilityData@@@Z 0047606c f   mfc90:mfc90.dll
 0001:00075072       ?AddDefaultButtonsToCustomizePane@CFrameImpl@@IAEXPAVCMFCPopupMenu@@I@Z 00476072 f   mfc90:mfc90.dll
 0001:00075078       ?Create@CAsyncSocket@@QAEHIHJPBD@Z 00476078 f   mfc90:mfc90.dll
 0001:0007507e       ??$SerializeElements@V?$CStringT@DV?$StrTraitMFC_DLL@DV?$ChTraitsCRT@D@ATL@@@@@ATL@@@@YGXAAVCArchive@@PAV?$CStringT@DV?$StrTraitMFC_DLL@DV?$ChTraitsCRT@D@ATL@@@@@ATL@@H@Z 0047607e f   mfc90:mfc90.dll
 0001:00075084       ??$HashKey@PBD@@YGIPBD@Z   00476084 f   mfc90:mfc90.dll
 0001:0007508a       ?GetThisClass@CMFCRibbonBar@@SGPAUCRuntimeClass@@XZ 0047608a f   mfc90:mfc90.dll
 0001:00075090       ??0CMFCRibbonBar@@QAE@H@Z  00476090 f   mfc90:mfc90.dll
 0001:00075096       ?Serialize@CBasePane@@UAEXAAVCArchive@@@Z 00476096 f   mfc90:mfc90.dll
 0001:0007509c       ?PreCreateWindow@CMFCRibbonBar@@MAEHAAUtagCREATESTRUCTA@@@Z 0047609c f   mfc90:mfc90.dll
 0001:000750a2       ?OnCommand@CMFCRibbonBar@@MAEHIJ@Z 004760a2 f   mfc90:mfc90.dll
 0001:000750a8       ?PreTranslateMessage@CMFCRibbonBar@@UAEHPAUtagMSG@@@Z 004760a8 f   mfc90:mfc90.dll
 0001:000750ae       ?WindowProc@CMFCRibbonBar@@MAEJIIJ@Z 004760ae f   mfc90:mfc90.dll
 0001:000750b4       ?IsDocked@CBasePane@@UBEHXZ 004760b4 f   mfc90:mfc90.dll
 0001:000750ba       ?IsVisible@CBasePane@@UBEHXZ 004760ba f   mfc90:mfc90.dll
 0001:000750c0       ?CanFloat@CBasePane@@UBEHXZ 004760c0 f   mfc90:mfc90.dll
 0001:000750c6       ?FloatPane@CPane@@UAEHVCRect@@W4AFX_DOCK_METHOD@@_N@Z 004760c6 f   mfc90:mfc90.dll
 0001:000750cc       ?RecalcLayout@CMFCRibbonBar@@UAEXXZ 004760cc f   mfc90:mfc90.dll
 0001:000750d2       ?OnBeforeChangeParent@CPane@@UAEXPAVCWnd@@H@Z 004760d2 f   mfc90:mfc90.dll
 0001:000750d8       ?OnAfterChangeParent@CPane@@UAEXPAVCWnd@@@Z 004760d8 f   mfc90:mfc90.dll
 0001:000750de       ?ShowPane@CBasePane@@UAEXHHH@Z 004760de f   mfc90:mfc90.dll
 0001:000750e4       ?LoadState@CMFCRibbonBar@@MAEHPBDHI@Z 004760e4 f   mfc90:mfc90.dll
 0001:000750ea       ?SaveState@CMFCRibbonBar@@MAEHPBDHI@Z 004760ea f   mfc90:mfc90.dll
 0001:000750f0       ?UndockPane@CPane@@UAEXH@Z 004760f0 f   mfc90:mfc90.dll
 0001:000750f6       ?OnUpdateCmdUI@CMFCRibbonBar@@MAEXPAVCFrameWnd@@H@Z 004760f6 f   mfc90:mfc90.dll
 0001:000750fc       ?OnPaneContextMenu@CMFCRibbonBar@@MAEXPAVCWnd@@VCPoint@@@Z 004760fc f   mfc90:mfc90.dll
 0001:00075102       ?OnSetAccData@CMFCRibbonBar@@UAEHJ@Z 00476102 f   mfc90:mfc90.dll
 0001:00075108       ?CalcFixedLayout@CMFCRibbonBar@@MAE?AVCSize@@HH@Z 00476108 f   mfc90:mfc90.dll
 0001:0007510e       ?GetPaneName@CPane@@UBEXAAV?$CStringT@DV?$StrTraitMFC_DLL@DV?$ChTraitsCRT@D@ATL@@@@@ATL@@@Z 0047610e f   mfc90:mfc90.dll
 0001:00075114       ?IsChangeState@CPane@@UBE?AW4AFX_CS_STATUS@@HPAPAVCBasePane@@@Z 00476114 f   mfc90:mfc90.dll
 0001:0007511a       ?OnBeforeFloat@CPane@@UAEHAAVCRect@@W4AFX_DOCK_METHOD@@@Z 0047611a f   mfc90:mfc90.dll
 0001:00075120       ?OnPressCloseButton@CPane@@UAEXXZ 00476120 f   mfc90:mfc90.dll
 0001:00075126       ?ConvertToTabbedDocument@CPane@@UAEXH@Z 00476126 f   mfc90:mfc90.dll
 0001:0007512c       ?OnContinueMoving@CPane@@MAEXXZ 0047612c f   mfc90:mfc90.dll
 0001:00075132       ?Dock@CPane@@MAEHPAVCBasePane@@PBUtagRECT@@W4AFX_DOCK_METHOD@@@Z 00476132 f   mfc90:mfc90.dll
 0001:00075138       ?EnterDragMode@CPane@@MAEXH@Z 00476138 f   mfc90:mfc90.dll
 0001:0007513e       ?OnRTLChanged@CMFCRibbonBar@@UAEXH@Z 0047613e f   mfc90:mfc90.dll
 0001:00075144       ?StoreRecentDockSiteInfo@CPane@@MAEXXZ 00476144 f   mfc90:mfc90.dll
 0001:0007514a       ?SetActiveCategory@CMFCRibbonBar@@UAEHPAVCMFCRibbonCategory@@H@Z 0047614a f   mfc90:mfc90.dll
 0001:00075150       ?HitTest@CMFCRibbonBar@@UAEPAVCMFCRibbonBaseElement@@VCPoint@@HH@Z 00476150 f   mfc90:mfc90.dll
 0001:00075156       ?GetDroppedDown@CMFCRibbonBar@@UAEPAVCMFCRibbonBaseElement@@XZ 00476156 f   mfc90:mfc90.dll
 0001:0007515c       ?OnClickButton@CMFCRibbonBar@@UAEXPAVCMFCRibbonButton@@VCPoint@@@Z 0047615c f   mfc90:mfc90.dll
 0001:00075162       ?OnEditContextMenu@CMFCRibbonBar@@UAEXPAVCMFCRibbonRichEditCtrl@@VCPoint@@@Z 00476162 f   mfc90:mfc90.dll
 0001:00075168       ?DWMCompositionChanged@CMFCRibbonBar@@UAEXXZ 00476168 f   mfc90:mfc90.dll
 0001:0007516e       ?OnShowRibbonQATMenu@CMFCRibbonBar@@UAEHPAVCWnd@@HHPAVCMFCRibbonBaseElement@@@Z 0047616e f   mfc90:mfc90.dll
 0001:00075174       ?TranslateChar@CMFCRibbonBar@@UAEHI@Z 00476174 f   mfc90:mfc90.dll
 0001:0007517a       ?OnFillBackground@CMFCRibbonBar@@MAEXPAVCDC@@VCRect@@@Z 0047617a f   mfc90:mfc90.dll
 0001:00075180       ?OnSetPrintPreviewKeys@CMFCRibbonBar@@MAEXPAVCMFCRibbonPanel@@00@Z 00476180 f   mfc90:mfc90.dll
 0001:00075186       ?OnBeforeProcessKey@CMFCRibbonBar@@MAEXAAH@Z 00476186 f   mfc90:mfc90.dll
 0001:0007518c       ??1CMFCRibbonBar@@UAE@XZ   0047618c f   mfc90:mfc90.dll
 0001:00075192       ?GetThisMessageMap@CMFCRibbonBar@@KGPBUAFX_MSGMAP@@XZ 00476192 f   mfc90:mfc90.dll
 0001:00075198       ?GetThisClass@CMFCPropertyPage@@SGPAUCRuntimeClass@@XZ 00476198 f   mfc90:mfc90.dll
 0001:0007519e       ??1CMFCPropertyPage@@UAE@XZ 0047619e f   mfc90:mfc90.dll
 0001:000751a4       ??0CMFCPropertyPage@@QAE@II@Z 004761a4 f   mfc90:mfc90.dll
 0001:000751aa       ?OnCommand@CMFCPropertyPage@@MAEHIJ@Z 004761aa f   mfc90:mfc90.dll
 0001:000751b0       ?OnNotify@CPropertyPage@@MAEHIJPAJ@Z 004761b0 f   mfc90:mfc90.dll
 0001:000751b6       ?PreTranslateMessage@CMFCPropertyPage@@UAEHPAUtagMSG@@@Z 004761b6 f   mfc90:mfc90.dll
 0001:000751bc       ?OnOK@CPropertyPage@@UAEXXZ 004761bc f   mfc90:mfc90.dll
 0001:000751c2       ?OnCancel@CPropertyPage@@UAEXXZ 004761c2 f   mfc90:mfc90.dll
 0001:000751c8       ?OnApply@CPropertyPage@@UAEHXZ 004761c8 f   mfc90:mfc90.dll
 0001:000751ce       ?OnReset@CPropertyPage@@UAEXXZ 004761ce f   mfc90:mfc90.dll
 0001:000751d4       ?OnSetActive@CMFCPropertyPage@@UAEHXZ 004761d4 f   mfc90:mfc90.dll
 0001:000751da       ?OnKillActive@CPropertyPage@@UAEHXZ 004761da f   mfc90:mfc90.dll
 0001:000751e0       ?OnQueryCancel@CPropertyPage@@UAEHXZ 004761e0 f   mfc90:mfc90.dll
 0001:000751e6       ?OnWizardBack@CPropertyPage@@UAEJXZ 004761e6 f   mfc90:mfc90.dll
 0001:000751ec       ?OnWizardNext@CPropertyPage@@UAEJXZ 004761ec f   mfc90:mfc90.dll
 0001:000751f2       ?OnWizardFinish@CPropertyPage@@UAEHXZ 004761f2 f   mfc90:mfc90.dll
 0001:000751f8       ?OnWizardFinishEx@CPropertyPage@@UAEPAUHWND__@@XZ 004761f8 f   mfc90:mfc90.dll
 0001:000751fe       ?GetThisMessageMap@CMFCPropertyPage@@KGPBUAFX_MSGMAP@@XZ 004761fe f   mfc90:mfc90.dll
 0001:00075204       ?DDX_Radio@@YGXPAVCDataExchange@@HAAH@Z 00476204 f   mfc90:mfc90.dll
 0001:0007520a       ?OnInitDialog@CMFCPropertyPage@@MAEHXZ 0047620a f   mfc90:mfc90.dll
 0001:00075210       ?GetThisClass@CMFCPropertySheet@@SGPAUCRuntimeClass@@XZ 00476210 f   mfc90:mfc90.dll
 0001:00075216       ??1CMFCPropertySheet@@UAE@XZ 00476216 f   mfc90:mfc90.dll
 0001:0007521c       ?AddPage@CMFCPropertySheet@@QAEXPAVCPropertyPage@@@Z 0047621c f   mfc90:mfc90.dll
 0001:00075222       ?SetLook@CMFCPropertySheet@@QAEXW4PropSheetLook@1@H@Z 00476222 f   mfc90:mfc90.dll
 0001:00075228       ?GetPSP@CPropertyPage@@QAEAAU_PROPSHEETPAGEA@@XZ 00476228 f   mfc90:mfc90.dll
 0001:0007522e       ??0CMFCPropertySheet@@QAE@PBDPAVCWnd@@I@Z 0047622e f   mfc90:mfc90.dll
 0001:00075234       ?OnCmdMsg@CPropertySheet@@UAEHIHPAXPAUAFX_CMDHANDLERINFO@@@Z 00476234 f   mfc90:mfc90.dll
 0001:0007523a       ?ContinueModal@CPropertySheet@@UAEHXZ 0047623a f   mfc90:mfc90.dll
 0001:00075240       ?PreTranslateMessage@CMFCPropertySheet@@UAEHPAUtagMSG@@@Z 00476240 f   mfc90:mfc90.dll
 0001:00075246       ?Create@CPropertySheet@@UAEHPAVCWnd@@KK@Z 00476246 f   mfc90:mfc90.dll
 0001:0007524c       ?BuildPropPageArray@CPropertySheet@@UAEXXZ 0047624c f   mfc90:mfc90.dll
 0001:00075252       ?OnActivatePage@CMFCPropertySheet@@UAEXPAVCPropertyPage@@@Z 00476252 f   mfc90:mfc90.dll
 0001:00075258       ?InitNavigationControl@CMFCPropertySheet@@UAEPAVCWnd@@XZ 00476258 f   mfc90:mfc90.dll
 0001:0007525e       ?OnRemoveTreePage@CMFCPropertySheet@@UAEHPAVCPropertyPage@@@Z 0047625e f   mfc90:mfc90.dll
 0001:00075264       ?GetThisMessageMap@CMFCPropertySheet@@KGPBUAFX_MSGMAP@@XZ 00476264 f   mfc90:mfc90.dll
 0001:0007526a       ??1CDrawingManager@@UAE@XZ 0047626a f   mfc90:mfc90.dll
 0001:00075270       ?DrawShadow@CDrawingManager@@QAEHVCRect@@HHHPAVCBitmap@@1KH@Z 00476270 f   mfc90:mfc90.dll
 0001:00075276       ??0CDrawingManager@@QAE@AAVCDC@@@Z 00476276 f   mfc90:mfc90.dll
 0001:0007527c       ?Draw3dRect@CDC@@QAEXPBUtagRECT@@KK@Z 0047627c f   mfc90:mfc90.dll
 0001:00075282       ?OnCommand@CPropertySheet@@UAEHIJ@Z 00476282 f   mfc90:mfc90.dll
 0001:00075288       ?OnInitDialog@CMFCPropertySheet@@UAEHXZ 00476288 f   mfc90:mfc90.dll
 0001:0007528e       ?GetRuntimeClass@CRichEditCtrl@@UBEPAUCRuntimeClass@@XZ 0047628e f   mfc90:mfc90.dll
 0001:00075294       ??1CRichEditCtrl@@UAE@XZ   00476294 f   mfc90:mfc90.dll
 0001:0007529a       ?TrackPopupMenu@CMenu@@QAEHIHHPAVCWnd@@PBUtagRECT@@@Z 0047629a f   mfc90:mfc90.dll
 0001:000752a0       ?CanPaste@CRichEditCtrl@@QBEHI@Z 004762a0 f   mfc90:mfc90.dll
 0001:000752a6       ?GetStyle@CWnd@@QBEKXZ     004762a6 f   mfc90:mfc90.dll
 0001:000752ac       ?GetItemData@CListCtrl@@QBEKH@Z 004762ac f   mfc90:mfc90.dll
 0001:000752b2       ?FromHandle@CDC@@SGPAV1@PAUHDC__@@@Z 004762b2 f   mfc90:mfc90.dll
 0001:000752b8       ?GetItemRect@CListCtrl@@QBEHHPAUtagRECT@@I@Z 004762b8 f   mfc90:mfc90.dll
 0001:000752be       ??0CBrush@@QAE@K@Z         004762be f   mfc90:mfc90.dll
 0001:000752c4       ?OnDestroy@CWnd@@IAEXXZ    004762c4 f   mfc90:mfc90.dll
 0001:000752ca       ?GetRuntimeClass@CBrush@@UBEPAUCRuntimeClass@@XZ 004762ca f   mfc90:mfc90.dll
 0001:000752d0       ?SetItem@CListCtrl@@QAEHHHIPBDHIIJ@Z 004762d0 f   mfc90:mfc90.dll
 0001:000752d6       ??1CMFCToolBar@@UAE@XZ     004762d6 f   mfc90:mfc90.dll
 0001:000752dc       ??1CDockablePane@@UAE@XZ   004762dc f   mfc90:mfc90.dll
 0001:000752e2       ??0CMFCTabCtrl@@QAE@XZ     004762e2 f   mfc90:mfc90.dll
 0001:000752e8       ??0CMFCToolBar@@QAE@XZ     004762e8 f   mfc90:mfc90.dll
 0001:000752ee       ??0CDockablePane@@QAE@XZ   004762ee f   mfc90:mfc90.dll
 0001:000752f4       ?GetRuntimeClass@CDockablePane@@UBEPAUCRuntimeClass@@XZ 004762f4 f   mfc90:mfc90.dll
 0001:000752fa       ?Serialize@CDockablePane@@UAEXAAVCArchive@@@Z 004762fa f   mfc90:mfc90.dll
 0001:00075300       ?RecalcLayout@CPane@@UAEXXZ 00476300 f   mfc90:mfc90.dll
 0001:00075306       ?LoadState@CDockablePane@@UAEHPBDHI@Z 00476306 f   mfc90:mfc90.dll
 0001:0007530c       ?SaveState@CDockablePane@@UAEHPBDHI@Z 0047630c f   mfc90:mfc90.dll
 0001:00075312       ?ConvertToTabbedDocument@CDockablePane@@UAEXH@Z 00476312 f   mfc90:mfc90.dll
 0001:00075318       ?Dock@CDockablePane@@MAEHPAVCBasePane@@PBUtagRECT@@W4AFX_DOCK_METHOD@@@Z 00476318 f   mfc90:mfc90.dll
 0001:0007531e       ?StoreRecentDockSiteInfo@CDockablePane@@MAEXXZ 0047631e f   mfc90:mfc90.dll
 0001:00075324       ?GetDockingStatus@CDockablePane@@UAE?AW4AFX_CS_STATUS@@VCPoint@@H@Z 00476324 f   mfc90:mfc90.dll
 0001:0007532a       ?SetAutoHideMode@CDockablePane@@UAEPAVCMFCAutoHideBar@@HKPAV2@H@Z 0047632a f   mfc90:mfc90.dll
 0001:00075330       ??1CMFCTabCtrl@@UAE@XZ     00476330 f   mfc90:mfc90.dll
 0001:00075336       ?GetThisMessageMap@CDockablePane@@KGPBUAFX_MSGMAP@@XZ 00476336 f   mfc90:mfc90.dll
 0001:0007533c       ?OnSetFocus@CDockablePane@@IAEXPAVCWnd@@@Z 0047633c f   mfc90:mfc90.dll
 0001:00075342       ?Create@CRichEditCtrl@@QAEHKABUtagRECT@@PAVCWnd@@I@Z 00476342 f   mfc90:mfc90.dll
 0001:00075348       ?Create@CMFCTabCtrl@@QAEHW4Style@1@ABUtagRECT@@PAVCWnd@@IW4Location@CMFCBaseTabCtrl@@H@Z 00476348 f   mfc90:mfc90.dll
 0001:0007534e       ?OnCreate@CDockablePane@@IAEHPAUtagCREATESTRUCTA@@@Z 0047634e f   mfc90:mfc90.dll
 0001:00075354       ?OnSize@CBasePane@@IAEXIHH@Z 00476354 f   mfc90:mfc90.dll
 0001:0007535a       ?GetTopLevelFrame@CWnd@@QBEPAVCFrameWnd@@XZ 0047635a f   mfc90:mfc90.dll
 0001:00075360       ?AfxDynamicDownCast@@YAPAVCObject@@PAUCRuntimeClass@@PAV1@@Z 00476360 f   mfc90:mfc90.dll
 0001:00075366       ?GetThisClass@CDockablePane@@SGPAUCRuntimeClass@@XZ 00476366 f   mfc90:mfc90.dll
 0001:0007536c       ?OnLButtonDown@CDockablePane@@IAEXIVCPoint@@@Z 0047636c f   mfc90:mfc90.dll
 0001:00075372       ?ScreenToClient@CWnd@@QBEXPAUtagRECT@@@Z 00476372 f   mfc90:mfc90.dll
 0001:00075378       ?FromHandle@CGdiObject@@SGPAV1@PAX@Z 00476378 f   mfc90:mfc90.dll
 0001:0007537e       ?DDX_Text@@YGXPAVCDataExchange@@HAAH@Z 0047637e f   mfc90:mfc90.dll
 0001:00075384       ??1CProgressCtrl@@UAE@XZ   00476384 f   mfc90:mfc90.dll
 0001:0007538a       ?GetRuntimeClass@CProgressCtrl@@UBEPAUCRuntimeClass@@XZ 0047638a f   mfc90:mfc90.dll
 0001:00075390       ?Create@CProgressCtrl@@UAEHKABUtagRECT@@PAVCWnd@@I@Z 00476390 f   mfc90:mfc90.dll
 0001:00075396       ?CreateEx@CProgressCtrl@@UAEHKKABUtagRECT@@PAVCWnd@@I@Z 00476396 f   mfc90:mfc90.dll
 0001:0007539c       ??1CTabCtrl@@UAE@XZ        0047639c f   mfc90:mfc90.dll
 0001:000753a2       ?GetNextAssoc@CMapStringToString@@QBEXAAPAU__POSITION@@AAV?$CStringT@DV?$StrTraitMFC_DLL@DV?$ChTraitsCRT@D@ATL@@@@@ATL@@1@Z 004763a2 f   mfc90:mfc90.dll
 0001:000753a8       ?GetRuntimeClass@CTabCtrl@@UBEPAUCRuntimeClass@@XZ 004763a8 f   mfc90:mfc90.dll
 0001:000753ae       ?GetMessageMap@CTabCtrl@@MBEPBUAFX_MSGMAP@@XZ 004763ae f   mfc90:mfc90.dll
 0001:000753b4       ?OnChildNotify@CTabCtrl@@MAEHIIJPAJ@Z 004763b4 f   mfc90:mfc90.dll
 0001:000753ba       ?Create@CTabCtrl@@UAEHKABUtagRECT@@PAVCWnd@@I@Z 004763ba f   mfc90:mfc90.dll
 0001:000753c0       ?CreateEx@CTabCtrl@@UAEHKKABUtagRECT@@PAVCWnd@@I@Z 004763c0 f   mfc90:mfc90.dll
 0001:000753c6       ?DrawItem@CTabCtrl@@UAEXPAUtagDRAWITEMSTRUCT@@@Z 004763c6 f   mfc90:mfc90.dll
 0001:000753cc       ?InsertItem@CTabCtrl@@QAEJIHPBDHJ@Z 004763cc f   mfc90:mfc90.dll
 0001:000753d2       ?GetThisClass@CWinThread@@SGPAUCRuntimeClass@@XZ 004763d2 f   mfc90:mfc90.dll
 0001:000753d8       ??1CWinThread@@UAE@XZ      004763d8 f   mfc90:mfc90.dll
 0001:000753de       ??0CWinThread@@QAE@XZ      004763de f   mfc90:mfc90.dll
 0001:000753e4       ?Run@CWinThread@@UAEHXZ    004763e4 f   mfc90:mfc90.dll
 0001:000753ea       ?OnIdle@CWinThread@@UAEHJ@Z 004763ea f   mfc90:mfc90.dll
 0001:000753f0       ?ProcessWndProcException@CWinThread@@UAEJPAVCException@@PBUtagMSG@@@Z 004763f0 f   mfc90:mfc90.dll
 0001:000753f6       ?ExitInstance@CWinThread@@UAEHXZ 004763f6 f   mfc90:mfc90.dll
 0001:000753fc       ?GetThisMessageMap@CCmdTarget@@KGPBUAFX_MSGMAP@@XZ 004763fc f   mfc90:mfc90.dll
 0001:00075402       ?DeleteImageList@CImageList@@QAEHXZ 00476402 f   mfc90:mfc90.dll
 0001:00075408       ?SetSize@CStringArray@@QAEXHH@Z 00476408 f   mfc90:mfc90.dll
 0001:0007540e       ?Create@CListCtrl@@QAEHKABUtagRECT@@PAVCWnd@@I@Z 0047640e f   mfc90:mfc90.dll
 0001:00075414       ?GetCheck@CListCtrl@@QBEHH@Z 00476414 f   mfc90:mfc90.dll
 0001:0007541a       ?SetCheck@CListCtrl@@QAEHHH@Z 0047641a f   mfc90:mfc90.dll
 0001:00075420       ?AfxThrowOleException@@YGXJ@Z 00476420 f   mfc90:mfc90.dll
 0001:00075426       ?Flush@CStdioFile@@UAEXXZ  00476426 f   mfc90:mfc90.dll
 0001:0007542c       ?Open@CStdioFile@@UAEHPBDIPAVCFileException@@@Z 0047642c f   mfc90:mfc90.dll
 0001:00075432       ??0CStdioFile@@QAE@XZ      00476432 f   mfc90:mfc90.dll
 0001:00075438       ?AddHead@CPtrList@@QAEPAU__POSITION@@PAX@Z 00476438 f   mfc90:mfc90.dll
 0001:0007543e       ?RemoveAt@CPtrList@@QAEXPAU__POSITION@@@Z 0047643e f   mfc90:mfc90.dll
 0001:00075444       ?ReadString@CStdioFile@@UAEHAAV?$CStringT@DV?$StrTraitMFC_DLL@DV?$ChTraitsCRT@D@ATL@@@@@ATL@@@Z 00476444 f   mfc90:mfc90.dll
 0001:0007544a       ?AfxSocketInit@@YGHPAUWSAData@@@Z 0047644a f   mfcs90:sockexp.obj
 0001:00075464       ___CxxFrameHandler3        00476464 f   msvcrt:MSVCR90.dll
 0001:0007546a       @__security_check_cookie@4 0047646a f   msvcrt:secchk.obj
 0001:00075479       ??_Etype_info@@UAEPAXI@Z   00476479 f i msvcrt:ti_inst.obj
 0001:000754c6       __CxxThrowException@8      004764c6 f   msvcrt:MSVCR90.dll
 0001:000754cc       _memset                    004764cc f   msvcrt:MSVCR90.dll
 0001:000754d2       _memcpy                    004764d2 f   msvcrt:MSVCR90.dll
 0001:000754d8       __except_handler4          004764d8 f   msvcrt:chandler4gs.obj
 0001:00075500       __chkstk                   00476500 f   msvcrt:chkstk.obj
 0001:00075500       __alloca_probe             00476500     msvcrt:chkstk.obj
 0001:0007552b       __onexit                   0047652b f   msvcrt:atonexit.obj
 0001:000755d0       _atexit                    004765d0 f   msvcrt:atonexit.obj
 0001:000755e8       ??0exception@std@@QAE@ABV01@@Z 004765e8 f   msvcrt:MSVCR90.dll
 0001:000755ee       ?what@exception@std@@UBEPBDXZ 004765ee f   msvcrt:MSVCR90.dll
 0001:000755f4       ?__ArrayUnwind@@YGXPAXIHP6EX0@Z@Z 004765f4 f   msvcrt:ehvecdtr.obj
 0001:00075652       ??_M@YGXPAXIHP6EX0@Z@Z     00476652 f   msvcrt:ehvecdtr.obj
 0001:000756b5       ??_L@YGXPAXIHP6EX0@Z1@Z    004766b5 f   msvcrt:ehvecctr.obj
 0001:00075720       __alloca_probe_16          00476720 f   msvcrt:alloca16.obj
 0001:00075736       __alloca_probe_8           00476736     msvcrt:alloca16.obj
 0001:00075750       __allmul                   00476750 f   msvcrt:llmul.obj
 0001:00075a8f       _WinMainCRTStartup         00476a8f f   msvcrt:crtexew.obj
 0001:00075aa0       __ftol2_sse                00476aa0 f   msvcrt:ftol2.obj
 0001:00075aa9       __ftol2_pentium4           00476aa9 f   msvcrt:ftol2.obj
 0001:00075abc       __ftol2_sse_excpt          00476abc f   msvcrt:ftol2.obj
 0001:00075ad6       __ftol2                    00476ad6 f   msvcrt:ftol2.obj
 0001:00075b50       __alldiv                   00476b50 f   msvcrt:lldiv.obj
 0001:00075bfa       ___report_gsfailure        00476bfa f   msvcrt:gs_report.obj
 0001:00075d00       __except_handler4_common   00476d00 f   msvcrt:MSVCR90.dll
 0001:00075d06       __unlock                   00476d06 f   msvcrt:MSVCR90.dll
 0001:00075d0c       ___dllonexit               00476d0c f   msvcrt:MSVCR90.dll
 0001:00075d12       __lock                     00476d12 f   msvcrt:MSVCR90.dll
 0001:00075d18       __SEH_prolog4              00476d18 f   msvcrt:sehprolg4.obj
 0001:00075d5d       __SEH_epilog4              00476d5d f   msvcrt:sehprolg4.obj
 0001:00075d72       ?terminate@@YAXXZ          00476d72 f   msvcrt:MSVCR90.dll
 0001:00075d78       ?__CxxUnhandledExceptionFilter@@YGJPAU_EXCEPTION_POINTERS@@@Z 00476d78 f   msvcrt:unhandld.obj
 0001:00075dba       ___CxxSetUnhandledExceptionFilter 00476dba f   msvcrt:unhandld.obj
 0001:00075dc8       __amsg_exit                00476dc8 f   msvcrt:MSVCR90.dll
 0001:00075dce       __RTC_Initialize           00476dce f   msvcrt:_initsect_.obj
 0001:00075df4       __RTC_Terminate            00476df4 f   msvcrt:_initsect_.obj
 0001:00075e1a       __XcptFilter               00476e1a f   msvcrt:MSVCR90.dll
 0001:00075e20       __ValidateImageBase        00476e20 f   msvcrt:pesect.obj
 0001:00075e60       __FindPESection            00476e60 f   msvcrt:pesect.obj
 0001:00075eb0       __IsNonwritableInCurrentImage 00476eb0 f   msvcrt:pesect.obj
 0001:00075f6e       __initterm                 00476f6e f   msvcrt:MSVCR90.dll
 0001:00075f74       __initterm_e               00476f74 f   msvcrt:MSVCR90.dll
 0001:00075f7a       __setdefaultprecision      00476f7a f   msvcrt:fp8.obj
 0001:00075fa5       __setargv                  00476fa5 f   msvcrt:dllargv.obj
 0001:00075fa5       __matherr                  00476fa5 f   msvcrt:merr.obj
 0001:00075fab       ___security_init_cookie    00476fab f   msvcrt:gs_support.obj
 0001:00076091       __get_sse2_info            00477091 f   msvcrt:cpu_disp.obj
 0001:000760f3       ___sse2_available_init     004770f3 f   msvcrt:cpu_disp.obj
 0001:00076100       __crt_debugger_hook        00477100 f   msvcrt:MSVCR90.dll
 0001:00076106       ?_type_info_dtor_internal_method@type_info@@QAEXXZ 00477106 f   msvcrt:MSVCR90.dll
 0001:00076106       ??1type_info@@UAE@XZ       00477106 f   msvcrt:MSVCR90.dll
 0001:0007610c       __invoke_watson            0047710c f   msvcrt:MSVCR90.dll
 0001:00076112       __controlfp_s              00477112 f   msvcrt:MSVCR90.dll
 0001:00076118       _Process32Next@8           00477118 f   kernel32:KERNEL32.dll
 0001:0007611e       _Process32First@8          0047711e f   kernel32:KERNEL32.dll
 0001:00076124       _CreateToolhelp32Snapshot@8 00477124 f   kernel32:KERNEL32.dll
 0001:0007612a       _GdiplusStartup@12         0047712a f   gdiplus:gdiplus.dll
 0001:00076130       _GdiplusShutdown@4         00477130 f   gdiplus:gdiplus.dll
 0001:00076140       ??1_com_error@@UAE@XZ      00477140 f i comsuppw:comraise.obj
 0001:00076180       ?_com_raise_error@@YGXJPAUIErrorInfo@@@Z 00477180 f   comsuppw:comraise.obj
 0001:000761c0       ??0_com_error@@QAE@ABV0@@Z 004771c0 f i comsuppw:comraise.obj
 0001:00076200       ??_E_com_error@@UAEPAXI@Z  00477200 f i comsuppw:comraise.obj
 0001:00076200       ??_G_com_error@@UAEPAXI@Z  00477200 f i comsuppw:comraise.obj
 0001:00076250       _ShowDllDlg                00477250 f   changeip:changeip.dll
 0001:00076256       _SetBasicInfo              00477256 f   changeip:changeip.dll
 0001:0007625c       _SetWindowTxtEx            0047725c f   changeip:changeip.dll
 0001:00076262       _SetShowPop                00477262 f   changeip:changeip.dll
 0001:00076268       _SetShowIconSet            00477268 f   changeip:changeip.dll
 0001:0007626e       _SetWindType               0047726e f   changeip:changeip.dll
 0001:00076274       _AddOneConfig              00477274 f   changeip:changeip.dll
 0001:0007627a       _SQLDisconnect@4           0047727a f   odbc32:ODBC32.dll
 0001:00076280       _SQLFreeHandle@8           00477280 f   odbc32:ODBC32.dll
 0001:00076286       _SQLColAttribute@28        00477286 f   odbc32:ODBC32.dll
 0001:0007628c       _SQLGetDiagRec@32          0047728c f   odbc32:ODBC32.dll
 0001:00076292       _SQLConnect@28             00477292 f   odbc32:ODBC32.dll
 0001:00076298       _SQLSetEnvAttr@16          00477298 f   odbc32:ODBC32.dll
 0001:0007629e       _SQLAllocHandle@12         0047729e f   odbc32:ODBC32.dll
 0001:000762a4       _SQLExecDirect@12          004772a4 f   odbc32:ODBC32.dll
 0001:000762aa       _SQLAllocStmt@8            004772aa f   odbc32:ODBC32.dll
 0001:000762b0       _SQLFreeStmt@8             004772b0 f   odbc32:ODBC32.dll
 0001:000762b6       _SQLBindCol@24             004772b6 f   odbc32:ODBC32.dll
 0001:000762bc       _SQLNumResultCols@8        004772bc f   odbc32:ODBC32.dll
 0001:000762c2       _SQLFetch@4                004772c2 f   odbc32:ODBC32.dll
 0001:000762c8       _SQLEndTran@12             004772c8 f   odbc32:ODBC32.dll
 0001:000762ce       _SQLSetConnectOption@12    004772ce f   odbc32:ODBC32.dll
 0001:000762e0       _SQLConfigDataSource@16    004772e0 f   odbccp32:funcload.obj
 0001:00076400       _StringCchCopyExA@24       00477400 f i odbccp32:dllload.obj
 0001:000769c0       _ODBC___GetSetupProc@4     004779c0 f   odbccp32:dllload.obj
 0001:00076b94       _ExRWDisk                  00477b94 f   windisk:windisk.dll
 0001:00076b9a       _ExRWDiskAbs               00477b9a f   windisk:windisk.dll
 0001:00076ba0       _ExDetectProtect           00477ba0 f   windisk:windisk.dll
 0001:00076ba6       _VerQueryValueA@16         00477ba6 f   Version:VERSION.dll
 0001:00076bac       _GetFileVersionInfoA@16    00477bac f   Version:VERSION.dll
 0001:00076bb2       _GetFileVersionInfoSizeA@8 00477bb2 f   Version:VERSION.dll
 0001:00076bb8       ?HTS_Uninit@@YGKXZ         00477bb8 f   htsapi:HTSAPI.dll
 0001:00076bbe       ?HTS_LiveStop@@YGKXZ       00477bbe f   htsapi:HTSAPI.dll
 0001:00076bc4       ?HTS_LiveStart@@YGKPAKKHHH@Z 00477bc4 f   htsapi:HTSAPI.dll
 0001:00076bca       ?HTS_Init@@YGKHKKKKPADH@Z  00477bca f   htsapi:HTSAPI.dll
 0001:00076bd0       ?HTS_SetWindowText@@YGKPAD@Z 00477bd0 f   htsapi:HTSAPI.dll
 0001:00076bd6       _GetAdaptersInfo@8         00477bd6 f   Iphlpapi:IPHLPAPI.DLL
 0001:00076bdc       ?_AfxSocketInit@@YGHPAUWSAData@@@Z 00477bdc f   mfc90:mfc90.dll
 0001:00076be2       _WinMain@16                00477be2 f   mfcs90:appmodul.obj
 0001:00076bed       ?AfxInitialize@@YGHHK@Z    00477bed f   mfcs90:appmodul.obj
 0001:00076c18       ?AfxWinMain@@YGHPAUHINSTANCE__@@0PADH@Z 00477c18 f   mfc90:mfc90.dll
 0002:00000000       __imp__RegQueryValueExA@24 00482000     advapi32:ADVAPI32.dll
 0002:00000004       __imp__RegOpenKeyExA@20    00482004     advapi32:ADVAPI32.dll
 0002:00000008       __imp__GetUserNameA@8      00482008     advapi32:ADVAPI32.dll
 0002:0000000c       __imp__RegSetValueExA@24   0048200c     advapi32:ADVAPI32.dll
 0002:00000010       __imp__AdjustTokenPrivileges@24 00482010     advapi32:ADVAPI32.dll
 0002:00000014       __imp__LookupPrivilegeValueA@12 00482014     advapi32:ADVAPI32.dll
 0002:00000018       __imp__OpenProcessToken@12 00482018     advapi32:ADVAPI32.dll
 0002:0000001c       __imp__RegDeleteKeyA@8     0048201c     advapi32:ADVAPI32.dll
 0002:00000020       __imp__RegDeleteValueA@8   00482020     advapi32:ADVAPI32.dll
 0002:00000024       __imp__RegCreateKeyExA@36  00482024     advapi32:ADVAPI32.dll
 0002:00000028       __imp__RegFlushKey@4       00482028     advapi32:ADVAPI32.dll
 0002:0000002c       __imp__RegCloseKey@4       0048202c     advapi32:ADVAPI32.dll
 0002:00000030       \177ADVAPI32_NULL_THUNK_DATA 00482030     advapi32:ADVAPI32.dll
 0002:00000034       __imp__InitCommonControlsEx@4 00482034     comctl32:COMCTL32.dll
 0002:00000038       \177COMCTL32_NULL_THUNK_DATA 00482038     comctl32:COMCTL32.dll
 0002:0000003c       __imp__GetStockObject@4    0048203c     gdi32:GDI32.dll
 0002:00000040       __imp__CreateSolidBrush@4  00482040     gdi32:GDI32.dll
 0002:00000044       __imp__DeleteObject@4      00482044     gdi32:GDI32.dll
 0002:00000048       __imp__GetTextExtentPoint32A@16 00482048     gdi32:GDI32.dll
 0002:0000004c       __imp__CreateFontA@56      0048204c     gdi32:GDI32.dll
 0002:00000050       \177GDI32_NULL_THUNK_DATA  00482050     gdi32:GDI32.dll
 0002:00000054       __imp_?HTS_LiveStop@@YGKXZ 00482054     htsapi:HTSAPI.dll
 0002:00000058       __imp_?HTS_LiveStart@@YGKPAKKHHH@Z 00482058     htsapi:HTSAPI.dll
 0002:0000005c       __imp_?HTS_Init@@YGKHKKKKPADH@Z 0048205c     htsapi:HTSAPI.dll
 0002:00000060       __imp_?HTS_SetWindowText@@YGKPAD@Z 00482060     htsapi:HTSAPI.dll
 0002:00000064       __imp_?HTS_Uninit@@YGKXZ   00482064     htsapi:HTSAPI.dll
 0002:00000068       \177HTSAPI_NULL_THUNK_DATA 00482068     htsapi:HTSAPI.dll
 0002:0000006c       __imp__GetAdaptersInfo@8   0048206c     Iphlpapi:IPHLPAPI.DLL
 0002:00000070       \177IPHLPAPI_NULL_THUNK_DATA 00482070     Iphlpapi:IPHLPAPI.DLL
 0002:00000074       __imp__SetEvent@4          00482074     kernel32:KERNEL32.dll
 0002:00000078       __imp__LoadLibraryA@4      00482078     kernel32:KERNEL32.dll
 0002:0000007c       __imp__GetModuleFileNameA@12 0048207c     kernel32:KERNEL32.dll
 0002:00000080       __imp__InitializeCriticalSection@4 00482080     kernel32:KERNEL32.dll
 0002:00000084       __imp__HeapFree@12         00482084     kernel32:KERNEL32.dll
 0002:00000088       __imp__GetProcessHeap@0    00482088     kernel32:KERNEL32.dll
 0002:0000008c       __imp__DeleteCriticalSection@4 0048208c     kernel32:KERNEL32.dll
 0002:00000090       __imp__EnterCriticalSection@4 00482090     kernel32:KERNEL32.dll
 0002:00000094       __imp__LeaveCriticalSection@4 00482094     kernel32:KERNEL32.dll
 0002:00000098       __imp__SetLastError@4      00482098     kernel32:KERNEL32.dll
 0002:0000009c       __imp__GetLastError@0      0048209c     kernel32:KERNEL32.dll
 0002:000000a0       __imp__GetModuleHandleA@4  004820a0     kernel32:KERNEL32.dll
 0002:000000a4       __imp__GetCurrentDirectoryA@8 004820a4     kernel32:KERNEL32.dll
 0002:000000a8       __imp__FindClose@4         004820a8     kernel32:KERNEL32.dll
 0002:000000ac       __imp__FindFirstFileA@8    004820ac     kernel32:KERNEL32.dll
 0002:000000b0       __imp__lstrcpyA@8          004820b0     kernel32:KERNEL32.dll
 0002:000000b4       __imp__lstrcmpA@8          004820b4     kernel32:KERNEL32.dll
 0002:000000b8       __imp__FreeLibrary@4       004820b8     kernel32:KERNEL32.dll
 0002:000000bc       __imp__lstrlenA@4          004820bc     kernel32:KERNEL32.dll
 0002:000000c0       __imp__GetVersionExA@4     004820c0     kernel32:KERNEL32.dll
 0002:000000c4       __imp__WaitForSingleObject@8 004820c4     kernel32:KERNEL32.dll
 0002:000000c8       __imp__GetTickCount@0      004820c8     kernel32:KERNEL32.dll
 0002:000000cc       __imp__CreateEventA@16     004820cc     kernel32:KERNEL32.dll
 0002:000000d0       __imp__GetLocalTime@4      004820d0     kernel32:KERNEL32.dll
 0002:000000d4       __imp__FormatMessageA@28   004820d4     kernel32:KERNEL32.dll
 0002:000000d8       __imp__ResetEvent@4        004820d8     kernel32:KERNEL32.dll
 0002:000000dc       __imp__FileTimeToSystemTime@8 004820dc     kernel32:KERNEL32.dll
 0002:000000e0       __imp__FileTimeToLocalFileTime@8 004820e0     kernel32:KERNEL32.dll
 0002:000000e4       __imp__MoveFileA@8         004820e4     kernel32:KERNEL32.dll
 0002:000000e8       __imp__CreateDirectoryA@8  004820e8     kernel32:KERNEL32.dll
 0002:000000ec       __imp__LocalUnlock@4       004820ec     kernel32:KERNEL32.dll
 0002:000000f0       __imp__LocalLock@4         004820f0     kernel32:KERNEL32.dll
 0002:000000f4       __imp__MoveFileExA@12      004820f4     kernel32:KERNEL32.dll
 0002:000000f8       __imp__GetFileSize@8       004820f8     kernel32:KERNEL32.dll
 0002:000000fc       __imp__GetSystemTimeAsFileTime@4 004820fc     kernel32:KERNEL32.dll
 0002:00000100       __imp__GetCurrentProcessId@0 00482100     kernel32:KERNEL32.dll
 0002:00000104       __imp__IsDebuggerPresent@0 00482104     kernel32:KERNEL32.dll
 0002:00000108       __imp__SetUnhandledExceptionFilter@4 00482108     kernel32:KERNEL32.dll
 0002:0000010c       __imp__UnhandledExceptionFilter@4 0048210c     kernel32:KERNEL32.dll
 0002:00000110       __imp__GetStartupInfoA@4   00482110     kernel32:KERNEL32.dll
 0002:00000114       __imp__InterlockedCompareExchange@12 00482114     kernel32:KERNEL32.dll
 0002:00000118       __imp__RaiseException@16   00482118     kernel32:KERNEL32.dll
 0002:0000011c       __imp__InterlockedExchange@8 0048211c     kernel32:KERNEL32.dll
 0002:00000120       __imp__QueryPerformanceCounter@4 00482120     kernel32:KERNEL32.dll
 0002:00000124       __imp__CreateToolhelp32Snapshot@8 00482124     kernel32:KERNEL32.dll
 0002:00000128       __imp__Process32First@8    00482128     kernel32:KERNEL32.dll
 0002:0000012c       __imp__Process32Next@8     0048212c     kernel32:KERNEL32.dll
 0002:00000130       __imp__TerminateProcess@8  00482130     kernel32:KERNEL32.dll
 0002:00000134       __imp__LocalAlloc@8        00482134     kernel32:KERNEL32.dll
 0002:00000138       __imp__LocalFree@4         00482138     kernel32:KERNEL32.dll
 0002:0000013c       __imp__GetCurrentProcess@0 0048213c     kernel32:KERNEL32.dll
 0002:00000140       __imp__CreateMutexA@12     00482140     kernel32:KERNEL32.dll
 0002:00000144       __imp__ReleaseMutex@4      00482144     kernel32:KERNEL32.dll
 0002:00000148       __imp__lstrcatA@8          00482148     kernel32:KERNEL32.dll
 0002:0000014c       __imp__MultiByteToWideChar@24 0048214c     kernel32:KERNEL32.dll
 0002:00000150       __imp__GetPrivateProfileSectionA@16 00482150     kernel32:KERNEL32.dll
 0002:00000154       __imp__CreateFileA@28      00482154     kernel32:KERNEL32.dll
 0002:00000158       __imp__DeviceIoControl@32  00482158     kernel32:KERNEL32.dll
 0002:0000015c       __imp__CancelIo@4          0048215c     kernel32:KERNEL32.dll
 0002:00000160       __imp__GetQueuedCompletionStatus@20 00482160     kernel32:KERNEL32.dll
 0002:00000164       __imp__PostQueuedCompletionStatus@16 00482164     kernel32:KERNEL32.dll
 0002:00000168       __imp__CreateIoCompletionPort@16 00482168     kernel32:KERNEL32.dll
 0002:0000016c       __imp__CreateProcessA@40   0048216c     kernel32:KERNEL32.dll
 0002:00000170       __imp__GetExitCodeProcess@8 00482170     kernel32:KERNEL32.dll
 0002:00000174       __imp__lstrcpynA@12        00482174     kernel32:KERNEL32.dll
 0002:00000178       __imp__GetSystemDirectoryA@8 00482178     kernel32:KERNEL32.dll
 0002:0000017c       __imp__GetComputerNameA@8  0048217c     kernel32:KERNEL32.dll
 0002:00000180       __imp__WaitForMultipleObjects@16 00482180     kernel32:KERNEL32.dll
 0002:00000184       __imp__GetPrivateProfileStringA@24 00482184     kernel32:KERNEL32.dll
 0002:00000188       __imp__CloseHandle@4       00482188     kernel32:KERNEL32.dll
 0002:0000018c       __imp__GetCurrentThreadId@0 0048218c     kernel32:KERNEL32.dll
 0002:00000190       __imp__Sleep@4             00482190     kernel32:KERNEL32.dll
 0002:00000194       __imp__FindNextFileA@8     00482194     kernel32:KERNEL32.dll
 0002:00000198       __imp__RemoveDirectoryA@4  00482198     kernel32:KERNEL32.dll
 0002:0000019c       __imp__GetProcAddress@8    0048219c     kernel32:KERNEL32.dll
 0002:000001a0       \177KERNEL32_NULL_THUNK_DATA 004821a0     kernel32:KERNEL32.dll
 0002:000001a4       __imp_?c_str@?$basic_string@DU?$char_traits@D@std@@V?$allocator@D@2@@std@@QBEPBDXZ 004821a4     msvcprt:MSVCP90.dll
 0002:000001a8       __imp_??0?$basic_string@DU?$char_traits@D@std@@V?$allocator@D@2@@std@@QAE@ABV01@@Z 004821a8     msvcprt:MSVCP90.dll
 0002:000001ac       __imp_??0?$basic_string@DU?$char_traits@D@std@@V?$allocator@D@2@@std@@QAE@PBD@Z 004821ac     msvcprt:MSVCP90.dll
 0002:000001b0       __imp_??1?$basic_string@DU?$char_traits@D@std@@V?$allocator@D@2@@std@@QAE@XZ 004821b0     msvcprt:MSVCP90.dll
 0002:000001b4       \177MSVCP90_NULL_THUNK_DATA 004821b4     msvcprt:MSVCP90.dll
 0002:000001b8       __imp__toupper             004821b8     msvcrt:MSVCR90.dll
 0002:000001bc       __imp__remove              004821bc     msvcrt:MSVCR90.dll
 0002:000001c0       __imp__strstr              004821c0     msvcrt:MSVCR90.dll
 0002:000001c4       __imp____CxxFrameHandler3  004821c4     msvcrt:MSVCR90.dll
 0002:000001c8       __imp__strncpy_s           004821c8     msvcrt:MSVCR90.dll
 0002:000001cc       __imp__atol                004821cc     msvcrt:MSVCR90.dll
 0002:000001d0       __imp___stricmp            004821d0     msvcrt:MSVCR90.dll
 0002:000001d4       __imp__free                004821d4     msvcrt:MSVCR90.dll
 0002:000001d8       __imp__malloc              004821d8     msvcrt:MSVCR90.dll
 0002:000001dc       __imp__sprintf             004821dc     msvcrt:MSVCR90.dll
 0002:000001e0       __imp__sscanf              004821e0     msvcrt:MSVCR90.dll
 0002:000001e4       __imp___snprintf           004821e4     msvcrt:MSVCR90.dll
 0002:000001e8       __imp__strncmp             004821e8     msvcrt:MSVCR90.dll
 0002:000001ec       __imp___ismbcdigit         004821ec     msvcrt:MSVCR90.dll
 0002:000001f0       __imp__atoi                004821f0     msvcrt:MSVCR90.dll
 0002:000001f4       __imp__strcpy_s            004821f4     msvcrt:MSVCR90.dll
 0002:000001f8       __imp__memcpy              004821f8     msvcrt:MSVCR90.dll
 0002:000001fc       __imp__memset              004821fc     msvcrt:MSVCR90.dll
 0002:00000200       __imp___setmbcp            00482200     msvcrt:MSVCR90.dll
 0002:00000204       __imp___CxxThrowException@8 00482204     msvcrt:MSVCR90.dll
 0002:00000208       __imp__strncpy             00482208     msvcrt:MSVCR90.dll
 0002:0000020c       __imp__strcat_s            0048220c     msvcrt:MSVCR90.dll
 0002:00000210       __imp___controlfp_s        00482210     msvcrt:MSVCR90.dll
 0002:00000214       __imp___invoke_watson      00482214     msvcrt:MSVCR90.dll
 0002:00000218       __imp_?_type_info_dtor_internal_method@type_info@@QAEXXZ 00482218     msvcrt:MSVCR90.dll
 0002:0000021c       __imp___crt_debugger_hook  0048221c     msvcrt:MSVCR90.dll
 0002:00000220       __imp____set_app_type      00482220     msvcrt:MSVCR90.dll
 0002:00000224       __imp____p__fmode          00482224     msvcrt:MSVCR90.dll
 0002:00000228       __imp____p__commode        00482228     msvcrt:MSVCR90.dll
 0002:0000022c       __imp___adjust_fdiv        0048222c     msvcrt:MSVCR90.dll
 0002:00000230       __imp____setusermatherr    00482230     msvcrt:MSVCR90.dll
 0002:00000234       __imp___configthreadlocale 00482234     msvcrt:MSVCR90.dll
 0002:00000238       __imp___initterm_e         00482238     msvcrt:MSVCR90.dll
 0002:0000023c       __imp___initterm           0048223c     msvcrt:MSVCR90.dll
 0002:00000240       __imp___acmdln             00482240     msvcrt:MSVCR90.dll
 0002:00000244       __imp___ismbblead          00482244     msvcrt:MSVCR90.dll
 0002:00000248       __imp___XcptFilter         00482248     msvcrt:MSVCR90.dll
 0002:0000024c       __imp___exit               0048224c     msvcrt:MSVCR90.dll
 0002:00000250       __imp___cexit              00482250     msvcrt:MSVCR90.dll
 0002:00000254       __imp____getmainargs       00482254     msvcrt:MSVCR90.dll
 0002:00000258       __imp___amsg_exit          00482258     msvcrt:MSVCR90.dll
 0002:0000025c       __imp_?terminate@@YAXXZ    0048225c     msvcrt:MSVCR90.dll
 0002:00000260       __imp___decode_pointer     00482260     msvcrt:MSVCR90.dll
 0002:00000264       __imp___onexit             00482264     msvcrt:MSVCR90.dll
 0002:00000268       __imp___lock               00482268     msvcrt:MSVCR90.dll
 0002:0000026c       __imp___encode_pointer     0048226c     msvcrt:MSVCR90.dll
 0002:00000270       __imp____dllonexit         00482270     msvcrt:MSVCR90.dll
 0002:00000274       __imp___unlock             00482274     msvcrt:MSVCR90.dll
 0002:00000278       __imp___except_handler4_common 00482278     msvcrt:MSVCR90.dll
 0002:0000027c       __imp__exit                0048227c     msvcrt:MSVCR90.dll
 0002:00000280       __imp___mbslwr             00482280     msvcrt:MSVCR90.dll
 0002:00000284       __imp___mbsrchr            00482284     msvcrt:MSVCR90.dll
 0002:00000288       __imp__fopen_s             00482288     msvcrt:MSVCR90.dll
 0002:0000028c       __imp__fclose              0048228c     msvcrt:MSVCR90.dll
 0002:00000290       __imp__memcpy_s            00482290     msvcrt:MSVCR90.dll
 0002:00000294       __imp___resetstkoflw       00482294     msvcrt:MSVCR90.dll
 0002:00000298       __imp__ceil                00482298     msvcrt:MSVCR90.dll
 0002:0000029c       __imp__strtoul             0048229c     msvcrt:MSVCR90.dll
 0002:000002a0       __imp__strtod              004822a0     msvcrt:MSVCR90.dll
 0002:000002a4       __imp__memmove_s           004822a4     msvcrt:MSVCR90.dll
 0002:000002a8       __imp__printf              004822a8     msvcrt:MSVCR90.dll
 0002:000002ac       __imp__sprintf_s           004822ac     msvcrt:MSVCR90.dll
 0002:000002b0       __imp__sscanf_s            004822b0     msvcrt:MSVCR90.dll
 0002:000002b4       __imp_??0exception@std@@QAE@ABQBD@Z 004822b4     msvcrt:MSVCR90.dll
 0002:000002b8       __imp_?what@exception@std@@UBEPBDXZ 004822b8     msvcrt:MSVCR90.dll
 0002:000002bc       __imp___invalid_parameter_noinfo 004822bc     msvcrt:MSVCR90.dll
 0002:000002c0       __imp_??0exception@std@@QAE@XZ 004822c0     msvcrt:MSVCR90.dll
 0002:000002c4       __imp_??1exception@std@@UAE@XZ 004822c4     msvcrt:MSVCR90.dll
 0002:000002c8       __imp_??0exception@std@@QAE@ABV01@@Z 004822c8     msvcrt:MSVCR90.dll
 0002:000002cc       __imp__vsprintf_s          004822cc     msvcrt:MSVCR90.dll
 0002:000002d0       \177MSVCR90_NULL_THUNK_DATA 004822d0     msvcrt:MSVCR90.dll
 0002:000002d4       __imp__SQLAllocHandle@12   004822d4     odbc32:ODBC32.dll
 0002:000002d8       __imp__SQLSetConnectOption@12 004822d8     odbc32:ODBC32.dll
 0002:000002dc       __imp__SQLEndTran@12       004822dc     odbc32:ODBC32.dll
 0002:000002e0       __imp__SQLFetch@4          004822e0     odbc32:ODBC32.dll
 0002:000002e4       __imp__SQLNumResultCols@8  004822e4     odbc32:ODBC32.dll
 0002:000002e8       __imp__SQLBindCol@24       004822e8     odbc32:ODBC32.dll
 0002:000002ec       __imp__SQLFreeStmt@8       004822ec     odbc32:ODBC32.dll
 0002:000002f0       __imp__SQLDisconnect@4     004822f0     odbc32:ODBC32.dll
 0002:000002f4       __imp__SQLFreeHandle@8     004822f4     odbc32:ODBC32.dll
 0002:000002f8       __imp__SQLColAttribute@28  004822f8     odbc32:ODBC32.dll
 0002:000002fc       __imp__SQLGetDiagRec@32    004822fc     odbc32:ODBC32.dll
 0002:00000300       __imp__SQLConnect@28       00482300     odbc32:ODBC32.dll
 0002:00000304       __imp__SQLSetEnvAttr@16    00482304     odbc32:ODBC32.dll
 0002:00000308       __imp__SQLAllocStmt@8      00482308     odbc32:ODBC32.dll
 0002:0000030c       __imp__SQLExecDirect@12    0048230c     odbc32:ODBC32.dll
 0002:00000310       \177ODBC32_NULL_THUNK_DATA 00482310     odbc32:ODBC32.dll
 0002:00000314       __imp__VariantClear@4      00482314     oleaut32:OLEAUT32.dll
 0002:00000318       __imp__VarDateFromStr@16   00482318     oleaut32:OLEAUT32.dll
 0002:0000031c       \177OLEAUT32_NULL_THUNK_DATA 0048231c     oleaut32:OLEAUT32.dll
 0002:00000320       __imp__InitLogSystem       00482320     RCLogSystem:RCLogSystem.dll
 0002:00000324       __imp__EndLogSystem        00482324     RCLogSystem:RCLogSystem.dll
 0002:00000328       __imp__ShowLogManager      00482328     RCLogSystem:RCLogSystem.dll
 0002:0000032c       __imp__AddOneLogRecord     0048232c     RCLogSystem:RCLogSystem.dll
 0002:00000330       \177RCLogSystem_NULL_THUNK_DATA 00482330     RCLogSystem:RCLogSystem.dll
 0002:00000334       __imp__SHBrowseForFolderA@4 00482334     shell32:SHELL32.dll
 0002:00000338       __imp__ShellExecuteExA@4   00482338     shell32:SHELL32.dll
 0002:0000033c       __imp__Shell_NotifyIconA@8 0048233c     shell32:SHELL32.dll
 0002:00000340       __imp__ShellExecuteA@24    00482340     shell32:SHELL32.dll
 0002:00000344       __imp__SHGetPathFromIDListA@8 00482344     shell32:SHELL32.dll
 0002:00000348       \177SHELL32_NULL_THUNK_DATA 00482348     shell32:SHELL32.dll
 0002:0000034c       __imp__SendMessageA@16     0048234c     user32:USER32.dll
 0002:00000350       __imp__FindWindowA@8       00482350     user32:USER32.dll
 0002:00000354       __imp__wsprintfA           00482354     user32:USER32.dll
 0002:00000358       __imp__MessageBoxA@16      00482358     user32:USER32.dll
 0002:0000035c       __imp__ExitWindowsEx@8     0048235c     user32:USER32.dll
 0002:00000360       __imp__GetSystemMenu@8     00482360     user32:USER32.dll
 0002:00000364       __imp__UnregisterHotKey@8  00482364     user32:USER32.dll
 0002:00000368       __imp__RegisterHotKey@16   00482368     user32:USER32.dll
 0002:0000036c       __imp__LockWindowUpdate@4  0048236c     user32:USER32.dll
 0002:00000370       __imp__CopyRect@8          00482370     user32:USER32.dll
 0002:00000374       __imp__GetSysColor@4       00482374     user32:USER32.dll
 0002:00000378       __imp__SetRectEmpty@4      00482378     user32:USER32.dll
 0002:0000037c       __imp__GetFocus@0          0048237c     user32:USER32.dll
 0002:00000380       __imp__FrameRect@12        00482380     user32:USER32.dll
 0002:00000384       __imp__AppendMenuA@16      00482384     user32:USER32.dll
 0002:00000388       __imp__CreatePopupMenu@0   00482388     user32:USER32.dll
 0002:0000038c       __imp__GetDC@4             0048238c     user32:USER32.dll
 0002:00000390       __imp__ReleaseDC@8         00482390     user32:USER32.dll
 0002:00000394       __imp__EnableWindow@8      00482394     user32:USER32.dll
 0002:00000398       __imp__RedrawWindow@16     00482398     user32:USER32.dll
 0002:0000039c       __imp__InvalidateRect@12   0048239c     user32:USER32.dll
 0002:000003a0       __imp__GetCursorPos@4      004823a0     user32:USER32.dll
 0002:000003a4       __imp__SetForegroundWindow@4 004823a4     user32:USER32.dll
 0002:000003a8       __imp__GetKeyState@4       004823a8     user32:USER32.dll
 0002:000003ac       __imp__SetWindowLongA@12   004823ac     user32:USER32.dll
 0002:000003b0       __imp__LoadImageA@24       004823b0     user32:USER32.dll
 0002:000003b4       __imp__GetWindowRect@8     004823b4     user32:USER32.dll
 0002:000003b8       __imp__GetSystemMetrics@4  004823b8     user32:USER32.dll
 0002:000003bc       __imp__LoadIconA@8         004823bc     user32:USER32.dll
 0002:000003c0       __imp__ModifyMenuA@20      004823c0     user32:USER32.dll
 0002:000003c4       __imp__GetParent@4         004823c4     user32:USER32.dll
 0002:000003c8       __imp__PostMessageA@16     004823c8     user32:USER32.dll
 0002:000003cc       __imp__LoadMenuA@8         004823cc     user32:USER32.dll
 0002:000003d0       __imp__GetSubMenu@8        004823d0     user32:USER32.dll
 0002:000003d4       __imp__EnableMenuItem@12   004823d4     user32:USER32.dll
 0002:000003d8       __imp__GetWindowLongA@8    004823d8     user32:USER32.dll
 0002:000003dc       __imp__KillTimer@8         004823dc     user32:USER32.dll
 0002:000003e0       __imp__SetTimer@16         004823e0     user32:USER32.dll
 0002:000003e4       __imp__GetClientRect@8     004823e4     user32:USER32.dll
 0002:000003e8       __imp__FillRect@12         004823e8     user32:USER32.dll
 0002:000003ec       __imp__LoadBitmapA@8       004823ec     user32:USER32.dll
 0002:000003f0       __imp__InflateRect@12      004823f0     user32:USER32.dll
 0002:000003f4       __imp__UpdateWindow@4      004823f4     user32:USER32.dll
 0002:000003f8       \177USER32_NULL_THUNK_DATA 004823f8     user32:USER32.dll
 0002:000003fc       __imp__GetFileVersionInfoA@16 004823fc     Version:VERSION.dll
 0002:00000400       __imp__VerQueryValueA@16   00482400     Version:VERSION.dll
 0002:00000404       __imp__GetFileVersionInfoSizeA@8 00482404     Version:VERSION.dll
 0002:00000408       \177VERSION_NULL_THUNK_DATA 00482408     Version:VERSION.dll
 0002:0000040c       __imp__WSASocketA@24       0048240c     WS2_32:WS2_32.dll
 0002:00000410       __imp__WSASend@28          00482410     WS2_32:WS2_32.dll
 0002:00000414       __imp__WSACloseEvent@4     00482414     WS2_32:WS2_32.dll
 0002:00000418       __imp__WSAEnumNetworkEvents@12 00482418     WS2_32:WS2_32.dll
 0002:0000041c       __imp__WSAWaitForMultipleEvents@20 0048241c     WS2_32:WS2_32.dll
 0002:00000420       __imp__WSAEventSelect@12   00482420     WS2_32:WS2_32.dll
 0002:00000424       __imp__WSACreateEvent@0    00482424     WS2_32:WS2_32.dll
 0002:00000428       __imp__WSARecv@28          00482428     WS2_32:WS2_32.dll
 0002:0000042c       \177WS2_32_NULL_THUNK_DATA 0048242c     WS2_32:WS2_32.dll
 0002:00000430       __imp__socket@12           00482430     wsock32:WSOCK32.dll
 0002:00000434       __imp__closesocket@4       00482434     wsock32:WSOCK32.dll
 0002:00000438       __imp__WSAGetLastError@0   00482438     wsock32:WSOCK32.dll
 0002:0000043c       __imp__connect@12          0048243c     wsock32:WSOCK32.dll
 0002:00000440       __imp__accept@12           00482440     wsock32:WSOCK32.dll
 0002:00000444       __imp__inet_addr@4         00482444     wsock32:WSOCK32.dll
 0002:00000448       __imp__bind@12             00482448     wsock32:WSOCK32.dll
 0002:0000044c       __imp__WSAAsyncSelect@16   0048244c     wsock32:WSOCK32.dll
 0002:00000450       __imp__inet_ntoa@4         00482450     wsock32:WSOCK32.dll
 0002:00000454       __imp__WSACleanup@0        00482454     wsock32:WSOCK32.dll
 0002:00000458       __imp__WSAStartup@8        00482458     wsock32:WSOCK32.dll
 0002:0000045c       __imp__setsockopt@20       0048245c     wsock32:WSOCK32.dll
 0002:00000460       __imp__htonl@4             00482460     wsock32:WSOCK32.dll
 0002:00000464       __imp__send@16             00482464     wsock32:WSOCK32.dll
 0002:00000468       __imp__htons@4             00482468     wsock32:WSOCK32.dll
 0002:0000046c       __imp__sendto@24           0048246c     wsock32:WSOCK32.dll
 0002:00000470       __imp__recvfrom@24         00482470     wsock32:WSOCK32.dll
 0002:00000474       __imp__recv@16             00482474     wsock32:WSOCK32.dll
 0002:00000478       __imp__select@20           00482478     wsock32:WSOCK32.dll
 0002:0000047c       __imp__listen@8            0048247c     wsock32:WSOCK32.dll
 0002:00000480       \177WSOCK32_NULL_THUNK_DATA 00482480     wsock32:WSOCK32.dll
 0002:00000484       __imp__WTSUnRegisterSessionNotification@4 00482484     WtsApi32:WTSAPI32.dll
 0002:00000488       __imp__WTSRegisterSessionNotification@8 00482488     WtsApi32:WTSAPI32.dll
 0002:0000048c       \177WTSAPI32_NULL_THUNK_DATA 0048248c     WtsApi32:WTSAPI32.dll
 0002:00000490       __imp__SetBasicInfo        00482490     changeip:changeip.dll
 0002:00000494       __imp__SetWindowTxtEx      00482494     changeip:changeip.dll
 0002:00000498       __imp__SetShowPop          00482498     changeip:changeip.dll
 0002:0000049c       __imp__SetShowIconSet      0048249c     changeip:changeip.dll
 0002:000004a0       __imp__SetWindType         004824a0     changeip:changeip.dll
 0002:000004a4       __imp__ShowDllDlg          004824a4     changeip:changeip.dll
 0002:000004a8       __imp__AddOneConfig        004824a8     changeip:changeip.dll
 0002:000004ac       \177changeip_NULL_THUNK_DATA 004824ac     changeip:changeip.dll
 0002:000004b0       __imp_?GetPartitionLetter@CDiskIO@@QAEXXZ 004824b0     diskop:diskop.dll
 0002:000004b4       __imp_??1CDiskIO@@QAE@XZ   004824b4     diskop:diskop.dll
 0002:000004b8       __imp_??0CDiskIO@@QAE@H@Z  004824b8     diskop:diskop.dll
 0002:000004bc       \177diskop_NULL_THUNK_DATA 004824bc     diskop:diskop.dll
 0002:000004c0       __imp__GdiplusShutdown@4   004824c0     gdiplus:gdiplus.dll
 0002:000004c4       __imp__GdiplusStartup@12   004824c4     gdiplus:gdiplus.dll
 0002:000004c8       \177gdiplus_NULL_THUNK_DATA 004824c8     gdiplus:gdiplus.dll
 0002:000004cc       __imp_?CalcWindowRect@CScrollView@@UAEXPAUtagRECT@@I@Z 004824cc     mfc90:mfc90.dll
 0002:000004d0       __imp_?GetScrollBarCtrl@CView@@UBEPAVCScrollBar@@H@Z 004824d0     mfc90:mfc90.dll
 0002:000004d4       __imp_?PostNcDestroy@CView@@MAEXXZ 004824d4     mfc90:mfc90.dll
 0002:000004d8       __imp_?SetOccDialogInfo@CFormView@@MAEHPAU_AFX_OCC_DIALOG_INFO@@@Z 004824d8     mfc90:mfc90.dll
 0002:000004dc       __imp_?GetOccDialogInfo@CFormView@@MAEPAU_AFX_OCC_DIALOG_INFO@@XZ 004824dc     mfc90:mfc90.dll
 0002:000004e0       __imp_?IsSelected@CView@@UBEHPBVCObject@@@Z 004824e0     mfc90:mfc90.dll
 0002:000004e4       __imp_?OnScroll@CScrollView@@UAEHIIH@Z 004824e4     mfc90:mfc90.dll
 0002:000004e8       __imp_?OnScrollBy@CScrollView@@UAEHVCSize@@H@Z 004824e8     mfc90:mfc90.dll
 0002:000004ec       __imp_?OnDragEnter@CView@@UAEKPAVCOleDataObject@@KVCPoint@@@Z 004824ec     mfc90:mfc90.dll
 0002:000004f0       __imp_?OnDragOver@CView@@UAEKPAVCOleDataObject@@KVCPoint@@@Z 004824f0     mfc90:mfc90.dll
 0002:000004f4       __imp_?OnDragLeave@CView@@UAEXXZ 004824f4     mfc90:mfc90.dll
 0002:000004f8       __imp_?OnDrop@CView@@UAEHPAVCOleDataObject@@KVCPoint@@@Z 004824f8     mfc90:mfc90.dll
 0002:000004fc       __imp_?OnDropEx@CView@@UAEKPAVCOleDataObject@@KKVCPoint@@@Z 004824fc     mfc90:mfc90.dll
 0002:00000500       __imp_?OnDragScroll@CView@@UAEKKVCPoint@@@Z 00482500     mfc90:mfc90.dll
 0002:00000504       __imp_?OnPrepareDC@CScrollView@@UAEXPAVCDC@@PAUCPrintInfo@@@Z 00482504     mfc90:mfc90.dll
 0002:00000508       __imp_?OnActivateView@CFormView@@MAEXHPAVCView@@0@Z 00482508     mfc90:mfc90.dll
 0002:0000050c       __imp_?OnActivateFrame@CFormView@@MAEXIPAVCFrameWnd@@@Z 0048250c     mfc90:mfc90.dll
 0002:00000510       __imp_?OnUpdate@CView@@MAEXPAV1@JPAVCObject@@@Z 00482510     mfc90:mfc90.dll
 0002:00000514       __imp_?OnPreparePrinting@CView@@MAEHPAUCPrintInfo@@@Z 00482514     mfc90:mfc90.dll
 0002:00000518       __imp_?OnBeginPrinting@CView@@MAEXPAVCDC@@PAUCPrintInfo@@@Z 00482518     mfc90:mfc90.dll
 0002:0000051c       __imp_?OnPrint@CView@@MAEXPAVCDC@@PAUCPrintInfo@@@Z 0048251c     mfc90:mfc90.dll
 0002:00000520       __imp_?OnEndPrinting@CView@@MAEXPAVCDC@@PAUCPrintInfo@@@Z 00482520     mfc90:mfc90.dll
 0002:00000524       __imp_?OnEndPrintPreview@CView@@MAEXPAVCDC@@PAUCPrintInfo@@UtagPOINT@@PAVCPreviewView@@@Z 00482524     mfc90:mfc90.dll
 0002:00000528       __imp_?GetWheelScrollDistance@CScrollView@@UAE?AVCSize@@V2@HH@Z 00482528     mfc90:mfc90.dll
 0002:0000052c       __imp_?PreCreateWindow@CView@@MAEHAAUtagCREATESTRUCTA@@@Z 0048252c     mfc90:mfc90.dll
 0002:00000530       __imp_?GetParentFrame@CWnd@@QBEPAVCFrameWnd@@XZ 00482530     mfc90:mfc90.dll
 0002:00000534       __imp_?OnInitialUpdate@CFormView@@UAEXXZ 00482534     mfc90:mfc90.dll
 0002:00000538       __imp_?MoveWindow@CWnd@@QAEXHHHHH@Z 00482538     mfc90:mfc90.dll
 0002:0000053c       __imp_?GetScrollPosition@CScrollView@@QBE?AVCPoint@@XZ 0048253c     mfc90:mfc90.dll
 0002:00000540       __imp_?OnSize@CScrollView@@QAEXIHH@Z 00482540     mfc90:mfc90.dll
 0002:00000544       __imp_?AfxBeginThread@@YGPAVCWinThread@@PAUCRuntimeClass@@HIKPAU_SECURITY_ATTRIBUTES@@@Z 00482544     mfc90:mfc90.dll
 0002:00000548       __imp_?PreTranslateMessage@CFormView@@MAEHPAUtagMSG@@@Z 00482548     mfc90:mfc90.dll
 0002:0000054c       __imp_?GetAccessibleChild@CWnd@@QAEJUtagVARIANT@@PAPAUIDispatch@@@Z 0048254c     mfc90:mfc90.dll
 0002:00000550       __imp_?GetAccessibleChildCount@CWnd@@QAEJXZ 00482550     mfc90:mfc90.dll
 0002:00000554       __imp_?GetAccessibleName@CWnd@@QAEJUtagVARIANT@@PAPA_W@Z 00482554     mfc90:mfc90.dll
 0002:00000558       __imp_?GetAccessibilityLocation@CWnd@@QAEJUtagVARIANT@@PAJ111@Z 00482558     mfc90:mfc90.dll
 0002:0000055c       __imp_?GetAccessibilityHitTest@CWnd@@QAEJJJPAUtagVARIANT@@@Z 0048255c     mfc90:mfc90.dll
 0002:00000560       __imp_?FromHandle@CImageList@@SGPAV1@PAU_IMAGELIST@@@Z 00482560     mfc90:mfc90.dll
 0002:00000564       __imp_??1CMapStringToString@@UAE@XZ 00482564     mfc90:mfc90.dll
 0002:00000568       __imp_?RemoveKey@CMapStringToString@@QAEHPBD@Z 00482568     mfc90:mfc90.dll
 0002:0000056c       __imp_?Lookup@CMapStringToString@@QBEHPBDAAV?$CStringT@DV?$StrTraitMFC_DLL@DV?$ChTraitsCRT@D@ATL@@@@@ATL@@@Z 0048256c     mfc90:mfc90.dll
 0002:00000570       __imp_?InitHashTable@CMapStringToString@@QAEXIH@Z 00482570     mfc90:mfc90.dll
 0002:00000574       __imp_??0CMapStringToString@@QAE@H@Z 00482574     mfc90:mfc90.dll
 0002:00000578       __imp_??ACMapStringToString@@QAEAAV?$CStringT@DV?$StrTraitMFC_DLL@DV?$ChTraitsCRT@D@ATL@@@@@ATL@@PBD@Z 00482578     mfc90:mfc90.dll
 0002:0000057c       __imp_?GetThisMessageMap@CListCtrl@@KGPBUAFX_MSGMAP@@XZ 0048257c     mfc90:mfc90.dll
 0002:00000580       __imp_??Y?$CStringT@DV?$StrTraitMFC_DLL@DV?$ChTraitsCRT@D@ATL@@@@@ATL@@QAEAAV01@E@Z 00482580     mfc90:mfc90.dll
 0002:00000584       __imp_??4?$CStringT@DV?$StrTraitMFC_DLL@DV?$ChTraitsCRT@D@ATL@@@@@ATL@@QAEAAV01@PBE@Z 00482584     mfc90:mfc90.dll
 0002:00000588       __imp_?MakeUpper@?$CStringT@DV?$StrTraitMFC_DLL@DV?$ChTraitsCRT@D@ATL@@@@@ATL@@QAEAAV12@XZ 00482588     mfc90:mfc90.dll
 0002:0000058c       __imp_?GetThisMessageMap@CFrameWndEx@@KGPBUAFX_MSGMAP@@XZ 0048258c     mfc90:mfc90.dll
 0002:00000590       __imp_?OnSetFocus@CFrameWnd@@IAEXPAVCWnd@@@Z 00482590     mfc90:mfc90.dll
 0002:00000594       __imp_??1CMFCRibbonStatusBar@@UAE@XZ 00482594     mfc90:mfc90.dll
 0002:00000598       __imp_??1CMFCCaptionBar@@UAE@XZ 00482598     mfc90:mfc90.dll
 0002:0000059c       __imp_??1CMFCShellTreeCtrl@@UAE@XZ 0048259c     mfc90:mfc90.dll
 0002:000005a0       __imp_??1CMFCToolBarImages@@UAE@XZ 004825a0     mfc90:mfc90.dll
 0002:000005a4       __imp_??1CSplitterWnd@@UAE@XZ 004825a4     mfc90:mfc90.dll
 0002:000005a8       __imp_??1CFrameWndEx@@MAE@XZ 004825a8     mfc90:mfc90.dll
 0002:000005ac       __imp_?GetInt@CWinAppEx@@QAEHPBDH@Z 004825ac     mfc90:mfc90.dll
 0002:000005b0       __imp_??0CMFCRibbonStatusBar@@QAE@XZ 004825b0     mfc90:mfc90.dll
 0002:000005b4       __imp_??0CMFCCaptionBar@@QAE@XZ 004825b4     mfc90:mfc90.dll
 0002:000005b8       __imp_??0CMFCShellTreeCtrl@@QAE@XZ 004825b8     mfc90:mfc90.dll
 0002:000005bc       __imp_??0CMFCToolBarImages@@QAE@XZ 004825bc     mfc90:mfc90.dll
 0002:000005c0       __imp_??0CSplitterWnd@@QAE@XZ 004825c0     mfc90:mfc90.dll
 0002:000005c4       __imp_??0CFrameWndEx@@IAE@XZ 004825c4     mfc90:mfc90.dll
 0002:000005c8       __imp_?OnCmdMsg@CFrameWndEx@@UAEHIHPAXPAUAFX_CMDHANDLERINFO@@@Z 004825c8     mfc90:mfc90.dll
 0002:000005cc       __imp_?GetMenu@CFrameWnd@@UBEPAVCMenu@@XZ 004825cc     mfc90:mfc90.dll
 0002:000005d0       __imp_?SetMenu@CFrameWnd@@UAEHPAVCMenu@@@Z 004825d0     mfc90:mfc90.dll
 0002:000005d4       __imp_?WinHelpA@CFrameWndEx@@UAEXKI@Z 004825d4     mfc90:mfc90.dll
 0002:000005d8       __imp_?HtmlHelpA@CFrameWndEx@@MAEXKI@Z 004825d8     mfc90:mfc90.dll
 0002:000005dc       __imp_?OnCommand@CFrameWndEx@@MAEHIJ@Z 004825dc     mfc90:mfc90.dll
 0002:000005e0       __imp_?BeginModalState@CFrameWnd@@UAEXXZ 004825e0     mfc90:mfc90.dll
 0002:000005e4       __imp_?EndModalState@CFrameWnd@@UAEXXZ 004825e4     mfc90:mfc90.dll
 0002:000005e8       __imp_?PostNcDestroy@CFrameWnd@@MAEXXZ 004825e8     mfc90:mfc90.dll
 0002:000005ec       __imp_?IsFrameWnd@CFrameWnd@@UBEHXZ 004825ec     mfc90:mfc90.dll
 0002:000005f0       __imp_?Create@CFrameWnd@@UAEHPBD0KABUtagRECT@@PAVCWnd@@0KPAUCCreateContext@@@Z 004825f0     mfc90:mfc90.dll
 0002:000005f4       __imp_?LoadFrame@CFrameWndEx@@UAEHIKPAVCWnd@@PAUCCreateContext@@@Z 004825f4     mfc90:mfc90.dll
 0002:000005f8       __imp_?GetActiveDocument@CFrameWnd@@UAEPAVCDocument@@XZ 004825f8     mfc90:mfc90.dll
 0002:000005fc       __imp_?GetActiveFrame@CFrameWnd@@UAEPAV1@XZ 004825fc     mfc90:mfc90.dll
 0002:00000600       __imp_?GetMessageString@CFrameWnd@@UBEXIAAV?$CStringT@DV?$StrTraitMFC_DLL@DV?$ChTraitsCRT@D@ATL@@@@@ATL@@@Z 00482600     mfc90:mfc90.dll
 0002:00000604       __imp_?RecalcLayout@CFrameWndEx@@UAEXH@Z 00482604     mfc90:mfc90.dll
 0002:00000608       __imp_?ActivateFrame@CFrameWnd@@UAEXH@Z 00482608     mfc90:mfc90.dll
 0002:0000060c       __imp_?SetMenuBarVisibility@CFrameWnd@@UAEXK@Z 0048260c     mfc90:mfc90.dll
 0002:00000610       __imp_?GetMenuBarVisibility@CFrameWnd@@UBEKXZ 00482610     mfc90:mfc90.dll
 0002:00000614       __imp_?SetMenuBarState@CFrameWnd@@UAEHK@Z 00482614     mfc90:mfc90.dll
 0002:00000618       __imp_?GetMenuBarState@CFrameWnd@@UBEKXZ 00482618     mfc90:mfc90.dll
 0002:0000061c       __imp_?OnSetPreviewMode@CFrameWndEx@@UAEXHPAUCPrintPreviewState@@@Z 0048261c     mfc90:mfc90.dll
 0002:00000620       __imp_?GetMessageBar@CFrameWnd@@UAEPAVCWnd@@XZ 00482620     mfc90:mfc90.dll
 0002:00000624       __imp_?NegotiateBorderSpace@CFrameWndEx@@UAEHIPAUtagRECT@@@Z 00482624     mfc90:mfc90.dll
 0002:00000628       __imp_?OnUpdateFrameTitle@CFrameWndEx@@UAEXH@Z 00482628     mfc90:mfc90.dll
 0002:0000062c       __imp_?OnUpdateFrameMenu@CFrameWndEx@@UAEXPAUHMENU__@@@Z 0048262c     mfc90:mfc90.dll
 0002:00000630       __imp_?GetDefaultAccelerator@CFrameWnd@@UAEPAUHACCEL__@@XZ 00482630     mfc90:mfc90.dll
 0002:00000634       __imp_?DelayUpdateFrameMenu@CFrameWndEx@@UAEXPAUHMENU__@@@Z 00482634     mfc90:mfc90.dll
 0002:00000638       __imp_?ExitHelpMode@CFrameWnd@@UAEXXZ 00482638     mfc90:mfc90.dll
 0002:0000063c       __imp_?OnShowMenuBar@CFrameWnd@@MAEXXZ 0048263c     mfc90:mfc90.dll
 0002:00000640       __imp_?OnHideMenuBar@CFrameWnd@@MAEXXZ 00482640     mfc90:mfc90.dll
 0002:00000644       __imp_?AdjustDockingLayout@CFrameWndEx@@UAEXPAX@Z 00482644     mfc90:mfc90.dll
 0002:00000648       __imp_?OnMoveMiniFrame@CFrameWndEx@@UAEHPAVCWnd@@@Z 00482648     mfc90:mfc90.dll
 0002:0000064c       __imp_?AdjustClientArea@CFrameWndEx@@MAEXXZ 0048264c     mfc90:mfc90.dll
 0002:00000650       __imp_?GetInPlaceActiveItem@CFrameWndEx@@MAEPAVCOleClientItem@@XZ 00482650     mfc90:mfc90.dll
 0002:00000654       __imp_?OnShowPopupMenu@CFrameWndEx@@UAEHPAVCMFCPopupMenu@@@Z 00482654     mfc90:mfc90.dll
 0002:00000658       __imp_?OnClosePopupMenu@CFrameWndEx@@UAEXPAVCMFCPopupMenu@@@Z 00482658     mfc90:mfc90.dll
 0002:0000065c       __imp_?OnDrawMenuImage@CFrameWndEx@@UAEHPAVCDC@@PBVCMFCToolBarMenuButton@@ABVCRect@@@Z 0048265c     mfc90:mfc90.dll
 0002:00000660       __imp_?OnShowPanes@CFrameWndEx@@UAEHH@Z 00482660     mfc90:mfc90.dll
 0002:00000664       __imp_??0CMFCOutlookBar@@QAE@XZ 00482664     mfc90:mfc90.dll
 0002:00000668       __imp_?GetRuntimeClass@CMFCOutlookBar@@UBEPAUCRuntimeClass@@XZ 00482668     mfc90:mfc90.dll
 0002:0000066c       __imp_?Serialize@CBaseTabbedPane@@UAEXAAVCArchive@@@Z 0048266c     mfc90:mfc90.dll
 0002:00000670       __imp_?get_accParent@CBasePane@@UAEJPAPAUIDispatch@@@Z 00482670     mfc90:mfc90.dll
 0002:00000674       __imp_?get_accChildCount@CBasePane@@UAEJPAJ@Z 00482674     mfc90:mfc90.dll
 0002:00000678       __imp_?get_accChild@CBasePane@@UAEJUtagVARIANT@@PAPAUIDispatch@@@Z 00482678     mfc90:mfc90.dll
 0002:0000067c       __imp_?get_accName@CBasePane@@UAEJUtagVARIANT@@PAPA_W@Z 0048267c     mfc90:mfc90.dll
 0002:00000680       __imp_?get_accValue@CBasePane@@UAEJUtagVARIANT@@PAPA_W@Z 00482680     mfc90:mfc90.dll
 0002:00000684       __imp_?get_accDescription@CBasePane@@UAEJUtagVARIANT@@PAPA_W@Z 00482684     mfc90:mfc90.dll
 0002:00000688       __imp_?get_accRole@CBasePane@@UAEJUtagVARIANT@@PAU2@@Z 00482688     mfc90:mfc90.dll
 0002:0000068c       __imp_?get_accState@CBasePane@@UAEJUtagVARIANT@@PAU2@@Z 0048268c     mfc90:mfc90.dll
 0002:00000690       __imp_?get_accHelp@CBasePane@@UAEJUtagVARIANT@@PAPA_W@Z 00482690     mfc90:mfc90.dll
 0002:00000694       __imp_?get_accHelpTopic@CBasePane@@UAEJPAPA_WUtagVARIANT@@PAJ@Z 00482694     mfc90:mfc90.dll
 0002:00000698       __imp_?get_accKeyboardShortcut@CBasePane@@UAEJUtagVARIANT@@PAPA_W@Z 00482698     mfc90:mfc90.dll
 0002:0000069c       __imp_?get_accFocus@CBasePane@@UAEJPAUtagVARIANT@@@Z 0048269c     mfc90:mfc90.dll
 0002:000006a0       __imp_?get_accSelection@CBasePane@@UAEJPAUtagVARIANT@@@Z 004826a0     mfc90:mfc90.dll
 0002:000006a4       __imp_?get_accDefaultAction@CBasePane@@UAEJUtagVARIANT@@PAPA_W@Z 004826a4     mfc90:mfc90.dll
 0002:000006a8       __imp_?accSelect@CBasePane@@UAEJJUtagVARIANT@@@Z 004826a8     mfc90:mfc90.dll
 0002:000006ac       __imp_?accLocation@CBasePane@@UAEJPAJ000UtagVARIANT@@@Z 004826ac     mfc90:mfc90.dll
 0002:000006b0       __imp_?accHitTest@CBasePane@@UAEJJJPAUtagVARIANT@@@Z 004826b0     mfc90:mfc90.dll
 0002:000006b4       __imp_?PreTranslateMessage@CDockablePane@@UAEHPAUtagMSG@@@Z 004826b4     mfc90:mfc90.dll
 0002:000006b8       __imp_?WindowProc@CBasePane@@MAEJIIJ@Z 004826b8     mfc90:mfc90.dll
 0002:000006bc       __imp_?IsDocked@CDockablePane@@UBEHXZ 004826bc     mfc90:mfc90.dll
 0002:000006c0       __imp_?IsTabbed@CPane@@UBEHXZ 004826c0     mfc90:mfc90.dll
 0002:000006c4       __imp_?IsMDITabbed@CBasePane@@UBEHXZ 004826c4     mfc90:mfc90.dll
 0002:000006c8       __imp_?IsVisible@CDockablePane@@UBEHXZ 004826c8     mfc90:mfc90.dll
 0002:000006cc       __imp_?CanAcceptPane@CMFCOutlookBar@@UBEHPBVCBasePane@@@Z 004826cc     mfc90:mfc90.dll
 0002:000006d0       __imp_?CanBeTabbedDocument@CPane@@UBEHXZ 004826d0     mfc90:mfc90.dll
 0002:000006d4       __imp_?GetCurrentAlignment@CBasePane@@UBEKXZ 004826d4     mfc90:mfc90.dll
 0002:000006d8       __imp_?GetDockSiteFrameWnd@CBasePane@@UBEPAVCWnd@@XZ 004826d8     mfc90:mfc90.dll
 0002:000006dc       __imp_?GetCaptionHeight@CDockablePane@@UBEHXZ 004826dc     mfc90:mfc90.dll
 0002:000006e0       __imp_?IsInFloatingMultiPaneFrameWnd@CDockablePane@@UBEHXZ 004826e0     mfc90:mfc90.dll
 0002:000006e4       __imp_?GetDockingMode@CBasePane@@UBE?AW4AFX_DOCK_TYPE@@XZ 004826e4     mfc90:mfc90.dll
 0002:000006e8       __imp_?GetPaneIcon@CBaseTabbedPane@@UAEPAUHICON__@@H@Z 004826e8     mfc90:mfc90.dll
 0002:000006ec       __imp_?CanFloat@CBaseTabbedPane@@UBEHXZ 004826ec     mfc90:mfc90.dll
 0002:000006f0       __imp_?CanAutoHide@CDockablePane@@UBEHXZ 004826f0     mfc90:mfc90.dll
 0002:000006f4       __imp_?EnableGripper@CDockablePane@@UAEXH@Z 004826f4     mfc90:mfc90.dll
 0002:000006f8       __imp_?DockPane@CPane@@UAEHPAVCBasePane@@PBUtagRECT@@W4AFX_DOCK_METHOD@@@Z 004826f8     mfc90:mfc90.dll
 0002:000006fc       __imp_?FloatPane@CBaseTabbedPane@@MAEHVCRect@@W4AFX_DOCK_METHOD@@_N@Z 004826fc     mfc90:mfc90.dll
 0002:00000700       __imp_?DockToFrameWindow@CDockablePane@@UAEHKPBUtagRECT@@KPAVCBasePane@@HH@Z 00482700     mfc90:mfc90.dll
 0002:00000704       __imp_?RecalcLayout@CBaseTabbedPane@@UAEXXZ 00482704     mfc90:mfc90.dll
 0002:00000708       __imp_?CreateDefaultMiniframe@CPane@@UAEPAVCPaneFrameWnd@@VCRect@@@Z 00482708     mfc90:mfc90.dll
 0002:0000070c       __imp_?OnBeforeChangeParent@CDockablePane@@UAEXPAVCWnd@@H@Z 0048270c     mfc90:mfc90.dll
 0002:00000710       __imp_?OnAfterChangeParent@CDockablePane@@UAEXPAVCWnd@@@Z 00482710     mfc90:mfc90.dll
 0002:00000714       __imp_?ShowPane@CDockablePane@@UAEXHHH@Z 00482714     mfc90:mfc90.dll
 0002:00000718       __imp_?GetParentMiniFrame@CBasePane@@UBEPAVCPaneFrameWnd@@H@Z 00482718     mfc90:mfc90.dll
 0002:0000071c       __imp_?LoadState@CMFCOutlookBar@@UAEHPBDHI@Z 0048271c     mfc90:mfc90.dll
 0002:00000720       __imp_?SaveState@CMFCOutlookBar@@UAEHPBDHI@Z 00482720     mfc90:mfc90.dll
 0002:00000724       __imp_?MoveWindow@CBasePane@@UAEPAXAAVCRect@@HPAX@Z 00482724     mfc90:mfc90.dll
 0002:00000728       __imp_?SetWindowPos@CBasePane@@UAEPAXPBVCWnd@@HHHHIPAX@Z 00482728     mfc90:mfc90.dll
 0002:0000072c       __imp_?CopyState@CBasePane@@UAEXPAV1@@Z 0048272c     mfc90:mfc90.dll
 0002:00000730       __imp_?UndockPane@CDockablePane@@UAEXH@Z 00482730     mfc90:mfc90.dll
 0002:00000734       __imp_?OnUpdateCmdUI@CDockablePane@@UAEXPAVCFrameWnd@@H@Z 00482734     mfc90:mfc90.dll
 0002:00000738       __imp_?OnPaneContextMenu@CBasePane@@UAEXPAVCWnd@@VCPoint@@@Z 00482738     mfc90:mfc90.dll
 0002:0000073c       __imp_?CreateEx@CBasePane@@UAEHKPBD0KABUtagRECT@@PAVCWnd@@IKPAUCCreateContext@@@Z 0048273c     mfc90:mfc90.dll
 0002:00000740       __imp_?OnSetAccData@CBasePane@@UAEHJ@Z 00482740     mfc90:mfc90.dll
 0002:00000744       __imp_?CalcFixedLayout@CDockablePane@@UAE?AVCSize@@HH@Z 00482744     mfc90:mfc90.dll
 0002:00000748       __imp_?DoPaint@CBasePane@@MAEXPAVCDC@@@Z 00482748     mfc90:mfc90.dll
 0002:0000074c       __imp_?AdjustDockingLayout@CBasePane@@UAEXPAX@Z 0048274c     mfc90:mfc90.dll
 0002:00000750       __imp_?GetMinSize@CBaseTabbedPane@@UBEXAAVCSize@@@Z 00482750     mfc90:mfc90.dll
 0002:00000754       __imp_?GetAvailableExpandSize@CPane@@UBEHXZ 00482754     mfc90:mfc90.dll
 0002:00000758       __imp_?GetAvailableStretchSize@CPane@@UBEHXZ 00482758     mfc90:mfc90.dll
 0002:0000075c       __imp_?CopyState@CPane@@UAEXPAV1@@Z 0048275c     mfc90:mfc90.dll
 0002:00000760       __imp_?SetActiveInGroup@CPane@@UAEXH@Z 00482760     mfc90:mfc90.dll
 0002:00000764       __imp_?PrepareToDock@CPane@@UAEXPAVCDockSite@@W4AFX_DOCK_METHOD@@@Z 00482764     mfc90:mfc90.dll
 0002:00000768       __imp_?DockByMouse@CPane@@UAEHPAVCBasePane@@@Z 00482768     mfc90:mfc90.dll
 0002:0000076c       __imp_?MovePane@CPane@@UAE?AVCSize@@VCRect@@HAAPAX@Z 0048276c     mfc90:mfc90.dll
 0002:00000770       __imp_?StretchPaneDeferWndPos@CPane@@UAEHHAAPAX@Z 00482770     mfc90:mfc90.dll
 0002:00000774       __imp_?DockPaneStandard@CDockablePane@@UAEPAVCPane@@AAH@Z 00482774     mfc90:mfc90.dll
 0002:00000778       __imp_?IsChangeState@CDockablePane@@UBE?AW4AFX_CS_STATUS@@HPAPAVCBasePane@@@Z 00482778     mfc90:mfc90.dll
 0002:0000077c       __imp_?SetDockState@CPane@@UAEXPAVCDockingManager@@@Z 0048277c     mfc90:mfc90.dll
 0002:00000780       __imp_?OnProcessDblClk@CPane@@UAEXXZ 00482780     mfc90:mfc90.dll
 0002:00000784       __imp_?OnBeforeFloat@CDockablePane@@UAEHAAVCRect@@W4AFX_DOCK_METHOD@@@Z 00482784     mfc90:mfc90.dll
 0002:00000788       __imp_?OnAfterFloat@CPane@@UAEXXZ 00482788     mfc90:mfc90.dll
 0002:0000078c       __imp_?Create@CPane@@UAEHPBDKABUtagRECT@@PAVCWnd@@IKPAUCCreateContext@@@Z 0048278c     mfc90:mfc90.dll
 0002:00000790       __imp_?CreateEx@CPane@@UAEHKPBDKABUtagRECT@@PAVCWnd@@IKPAUCCreateContext@@@Z 00482790     mfc90:mfc90.dll
 0002:00000794       __imp_?CalcAvailableSize@CPane@@UAE?AVCSize@@VCRect@@@Z 00482794     mfc90:mfc90.dll
 0002:00000798       __imp_?AdjustSizeImmediate@CPane@@UAEXH@Z 00482798     mfc90:mfc90.dll
 0002:0000079c       __imp_?ToggleAutoHide@CDockablePane@@UAEXXZ 0048279c     mfc90:mfc90.dll
 0002:000007a0       __imp_?OnPressCloseButton@CDockablePane@@MAEXXZ 004827a0     mfc90:mfc90.dll
 0002:000007a4       __imp_?ConvertToTabbedDocument@CBaseTabbedPane@@UAEXH@Z 004827a4     mfc90:mfc90.dll
 0002:000007a8       __imp_?OnShowControlBarMenu@CPane@@UAEHVCPoint@@@Z 004827a8     mfc90:mfc90.dll
 0002:000007ac       __imp_?OnDrawDragRect@CDockablePane@@MAEXPBUtagRECT@@0@Z 004827ac     mfc90:mfc90.dll
 0002:000007b0       __imp_?OnBeforeDock@CPane@@MAEHPAPAVCBasePane@@PBUtagRECT@@W4AFX_DOCK_METHOD@@@Z 004827b0     mfc90:mfc90.dll
 0002:000007b4       __imp_?OnAfterDock@CDockablePane@@MAEXPAVCBasePane@@PBUtagRECT@@W4AFX_DOCK_METHOD@@@Z 004827b4     mfc90:mfc90.dll
 0002:000007b8       __imp_?RemoveFromMiniframe@CPane@@MAEXPAVCWnd@@W4AFX_DOCK_METHOD@@@Z 004827b8     mfc90:mfc90.dll
 0002:000007bc       __imp_?SetDragMode@CPane@@MAEXH@Z 004827bc     mfc90:mfc90.dll
 0002:000007c0       __imp_?Dock@CBaseTabbedPane@@MAEHPAVCBasePane@@PBUtagRECT@@W4AFX_DOCK_METHOD@@@Z 004827c0     mfc90:mfc90.dll
 0002:000007c4       __imp_?EnterDragMode@CDockablePane@@MAEXH@Z 004827c4     mfc90:mfc90.dll
 0002:000007c8       __imp_?OnRTLChanged@CPane@@MAEXH@Z 004827c8     mfc90:mfc90.dll
 0002:000007cc       __imp_?StoreRecentDockSiteInfo@CBaseTabbedPane@@MAEXXZ 004827cc     mfc90:mfc90.dll
 0002:000007d0       __imp_?Create@CDockablePane@@UAEHPBDPAVCWnd@@VCSize@@HIKKK@Z 004827d0     mfc90:mfc90.dll
 0002:000007d4       __imp_?Create@CDockablePane@@UAEHPBDPAVCWnd@@ABUtagRECT@@HIKKKPAUCCreateContext@@@Z 004827d4     mfc90:mfc90.dll
 0002:000007d8       __imp_?CreateEx@CDockablePane@@UAEHKPBDPAVCWnd@@ABUtagRECT@@HIKKKPAUCCreateContext@@@Z 004827d8     mfc90:mfc90.dll
 0002:000007dc       __imp_?GetTabArea@CMFCOutlookBar@@UBEXAAVCRect@@0@Z 004827dc     mfc90:mfc90.dll
 0002:000007e0       __imp_?HitTest@CDockablePane@@UAEHVCPoint@@H@Z 004827e0     mfc90:mfc90.dll
 0002:000007e4       __imp_?CanAcceptMiniFrame@CDockablePane@@UBEHPAVCPaneFrameWnd@@@Z 004827e4     mfc90:mfc90.dll
 0002:000007e8       __imp_?Slide@CDockablePane@@UAEXHH@Z 004827e8     mfc90:mfc90.dll
 0002:000007ec       __imp_?GetDockingStatus@CMFCOutlookBar@@UAE?AW4AFX_CS_STATUS@@VCPoint@@H@Z 004827ec     mfc90:mfc90.dll
 0002:000007f0       __imp_?AttachToTabWnd@CDockablePane@@UAEPAV1@PAV1@W4AFX_DOCK_METHOD@@HPAPAV1@@Z 004827f0     mfc90:mfc90.dll
 0002:000007f4       __imp_?CreateTabbedPane@CDockablePane@@UAEPAVCTabbedPane@@XZ 004827f4     mfc90:mfc90.dll
 0002:000007f8       __imp_?DockToWindow@CDockablePane@@UAEHPAV1@KPBUtagRECT@@@Z 004827f8     mfc90:mfc90.dll
 0002:000007fc       __imp_?DockPaneContainer@CDockablePane@@UAEHAAVCPaneContainerManager@@KW4AFX_DOCK_METHOD@@@Z 004827fc     mfc90:mfc90.dll
 0002:00000800       __imp_?UnSetAutoHideMode@CDockablePane@@UAEXPAV1@@Z 00482800     mfc90:mfc90.dll
 0002:00000804       __imp_?SetAutoHideMode@CBaseTabbedPane@@UAEPAVCMFCAutoHideBar@@HKPAV2@H@Z 00482804     mfc90:mfc90.dll
 0002:00000808       __imp_?CopyState@CDockablePane@@UAEXPAV1@@Z 00482808     mfc90:mfc90.dll
 0002:0000080c       __imp_?StoreRecentTabRelatedInfo@CDockablePane@@MAEXXZ 0048280c     mfc90:mfc90.dll
 0002:00000810       __imp_?DrawCaption@CDockablePane@@MAEXPAVCDC@@VCRect@@@Z 00482810     mfc90:mfc90.dll
 0002:00000814       __imp_?AdjustPaneToPaneContainer@CDockablePane@@MAEXPAVCPaneDivider@@@Z 00482814     mfc90:mfc90.dll
 0002:00000818       __imp_?OnTrackCaptionButtons@CDockablePane@@MAEXVCPoint@@@Z 00482818     mfc90:mfc90.dll
 0002:0000081c       __imp_?StopCaptionButtonsTracking@CDockablePane@@MAEXXZ 0048281c     mfc90:mfc90.dll
 0002:00000820       __imp_?SetCaptionButtons@CDockablePane@@MAEXXZ 00482820     mfc90:mfc90.dll
 0002:00000824       __imp_?CheckAutoHideCondition@CDockablePane@@MAEHXZ 00482824     mfc90:mfc90.dll
 0002:00000828       __imp_?CheckStopSlideCondition@CDockablePane@@MAEHH@Z 00482828     mfc90:mfc90.dll
 0002:0000082c       __imp_?OnSlide@CDockablePane@@MAEXH@Z 0048282c     mfc90:mfc90.dll
 0002:00000830       __imp_?AddTab@CBaseTabbedPane@@UAEHPAVCWnd@@HHH@Z 00482830     mfc90:mfc90.dll
 0002:00000834       __imp_?FloatTab@CMFCOutlookBar@@UAEHPAVCWnd@@HW4AFX_DOCK_METHOD@@H@Z 00482834     mfc90:mfc90.dll
 0002:00000838       __imp_?DetachPane@CBaseTabbedPane@@UAEHPAVCWnd@@H@Z 00482838     mfc90:mfc90.dll
 0002:0000083c       __imp_?RemovePane@CBaseTabbedPane@@UAEHPAVCWnd@@@Z 0048283c     mfc90:mfc90.dll
 0002:00000840       __imp_?ShowTab@CBaseTabbedPane@@UAEHPAVCWnd@@HHH@Z 00482840     mfc90:mfc90.dll
 0002:00000844       __imp_?FindPaneByID@CBaseTabbedPane@@UAEPAVCWnd@@I@Z 00482844     mfc90:mfc90.dll
 0002:00000848       __imp_?FindBarByTabNumber@CBaseTabbedPane@@UAEPAVCWnd@@HH@Z 00482848     mfc90:mfc90.dll
 0002:0000084c       __imp_?GetFirstVisibleTab@CBaseTabbedPane@@UAEPAVCWnd@@AAH@Z 0048284c     mfc90:mfc90.dll
 0002:00000850       __imp_?ApplyRestoredTabInfo@CBaseTabbedPane@@UAEXH@Z 00482850     mfc90:mfc90.dll
 0002:00000854       __imp_?SerializeTabWindow@CBaseTabbedPane@@UAEXAAVCArchive@@@Z 00482854     mfc90:mfc90.dll
 0002:00000858       __imp_?SaveSiblingBarIDs@CBaseTabbedPane@@UAEXAAVCArchive@@@Z 00482858     mfc90:mfc90.dll
 0002:0000085c       __imp_?GetPaneList@CBaseTabbedPane@@UAEXAAVCObList@@PAUCRuntimeClass@@@Z 0048285c     mfc90:mfc90.dll
 0002:00000860       __imp_?Create@CMFCOutlookBar@@UAEHPBDPAVCWnd@@ABUtagRECT@@IKKPAUCCreateContext@@@Z 00482860     mfc90:mfc90.dll
 0002:00000864       __imp_??1CMFCOutlookBar@@UAE@XZ 00482864     mfc90:mfc90.dll
 0002:00000868       __imp_?DockPane@CFrameWndEx@@QAEXPAVCBasePane@@IPBUtagRECT@@@Z 00482868     mfc90:mfc90.dll
 0002:0000086c       __imp_?ExtractIconA@CMFCToolBarImages@@QAEPAUHICON__@@H@Z 0048286c     mfc90:mfc90.dll
 0002:00000870       __imp_?Load@CMFCToolBarImages@@QAEHIPAUHINSTANCE__@@H@Z 00482870     mfc90:mfc90.dll
 0002:00000874       __imp_?EnableDocking@CFrameWndEx@@QAEHK@Z 00482874     mfc90:mfc90.dll
 0002:00000878       __imp_?EnableAutoHidePanes@CFrameWndEx@@QAEHK@Z 00482878     mfc90:mfc90.dll
 0002:0000087c       __imp_?SetDockingMode@CDockingManager@@SGXW4AFX_DOCK_TYPE@@@Z 0048287c     mfc90:mfc90.dll
 0002:00000880       __imp_?AddExtendedElement@CMFCRibbonStatusBar@@QAEXPAVCMFCRibbonBaseElement@@PBDH@Z 00482880     mfc90:mfc90.dll
 0002:00000884       __imp_?AddElement@CMFCRibbonStatusBar@@QAEXPAVCMFCRibbonBaseElement@@PBDH@Z 00482884     mfc90:mfc90.dll
 0002:00000888       __imp_??0CMFCRibbonStatusBarPane@@QAE@IPBDHPAUHICON__@@0@Z 00482888     mfc90:mfc90.dll
 0002:0000088c       __imp_?Create@CMFCRibbonStatusBar@@QAEHPAVCWnd@@KI@Z 0048288c     mfc90:mfc90.dll
 0002:00000890       __imp_?Create@CMFCRibbonBar@@QAEHPAVCWnd@@KI@Z 00482890     mfc90:mfc90.dll
 0002:00000894       __imp_?OnCreate@CFrameWndEx@@QAEHPAUtagCREATESTRUCTA@@@Z 00482894     mfc90:mfc90.dll
 0002:00000898       __imp_?PreCreateWindow@CFrameWndEx@@MAEHAAUtagCREATESTRUCTA@@@Z 00482898     mfc90:mfc90.dll
 0002:0000089c       __imp_?AddToTabs@CMFCRibbonBar@@QAEXPAVCMFCRibbonBaseElement@@@Z 0048289c     mfc90:mfc90.dll
 0002:000008a0       __imp_??0CMFCRibbonButton@@QAE@IPBDHHH@Z 004828a0     mfc90:mfc90.dll
 0002:000008a4       __imp_?AddMainCategory@CMFCRibbonBar@@QAEPAVCMFCRibbonMainPanel@@PBDIIVCSize@@1@Z 004828a4     mfc90:mfc90.dll
 0002:000008a8       __imp_?SetApplicationButton@CMFCRibbonBar@@QAEXPAVCMFCRibbonApplicationButton@@VCSize@@@Z 004828a8     mfc90:mfc90.dll
 0002:000008ac       __imp_?SetImage@CMFCRibbonApplicationButton@@QAEXI@Z 004828ac     mfc90:mfc90.dll
 0002:000008b0       __imp_?Create@CTreeCtrl@@QAEHKABUtagRECT@@PAVCWnd@@I@Z 004828b0     mfc90:mfc90.dll
 0002:000008b4       __imp_?WriteInt@CWinAppEx@@QAEHPBDH@Z 004828b4     mfc90:mfc90.dll
 0002:000008b8       __imp_?GetThisClass@CMFCVisualManagerOffice2007@@SGPAUCRuntimeClass@@XZ 004828b8     mfc90:mfc90.dll
 0002:000008bc       __imp_?SetStyle@CMFCVisualManagerOffice2007@@SGHW4Style@1@PBD@Z 004828bc     mfc90:mfc90.dll
 0002:000008c0       __imp_?GetThisClass@CMFCVisualManagerVS2005@@SGPAUCRuntimeClass@@XZ 004828c0     mfc90:mfc90.dll
 0002:000008c4       __imp_?GetThisClass@CMFCVisualManagerOffice2003@@SGPAUCRuntimeClass@@XZ 004828c4     mfc90:mfc90.dll
 0002:000008c8       __imp_?GetThisClass@CMFCVisualManagerWindows@@SGPAUCRuntimeClass@@XZ 004828c8     mfc90:mfc90.dll
 0002:000008cc       __imp_?m_b3DTabsXPTheme@CMFCVisualManagerWindows@@2HA 004828cc     mfc90:mfc90.dll
 0002:000008d0       __imp_?GetThisClass@CMFCVisualManagerOfficeXP@@SGPAUCRuntimeClass@@XZ 004828d0     mfc90:mfc90.dll
 0002:000008d4       __imp_?SetDefaultManager@CMFCVisualManager@@SGXPAUCRuntimeClass@@@Z 004828d4     mfc90:mfc90.dll
 0002:000008d8       __imp_?GetThisClass@CMFCVisualManager@@SGPAUCRuntimeClass@@XZ 004828d8     mfc90:mfc90.dll
 0002:000008dc       __imp_?ShowPane@CFrameWndEx@@QAEXPAVCBasePane@@HHH@Z 004828dc     mfc90:mfc90.dll
 0002:000008e0       __imp_?SetInformation@CMFCRibbonStatusBar@@QAEXPBD@Z 004828e0     mfc90:mfc90.dll
 0002:000008e4       __imp_?Find@?$CStringT@DV?$StrTraitMFC_DLL@DV?$ChTraitsCRT@D@ATL@@@@@ATL@@QBEHDH@Z 004828e4     mfc90:mfc90.dll
 0002:000008e8       __imp_??1CStringArray@@UAE@XZ 004828e8     mfc90:mfc90.dll
 0002:000008ec       __imp_?get_accName@CWnd@@UAEJUtagVARIANT@@PAPA_W@Z 004828ec     mfc90:mfc90.dll
 0002:000008f0       __imp_?AddPanel@CMFCRibbonCategory@@QAEPAVCMFCRibbonPanel@@PBDPAUHICON__@@PAUCRuntimeClass@@@Z 004828f0     mfc90:mfc90.dll
 0002:000008f4       __imp_?AddCategory@CMFCRibbonBar@@QAEPAVCMFCRibbonCategory@@PBDIIVCSize@@1HPAUCRuntimeClass@@@Z 004828f4     mfc90:mfc90.dll
 0002:000008f8       __imp_??0CMFCRibbonCheckBox@@QAE@IPBD@Z 004828f8     mfc90:mfc90.dll
 0002:000008fc       __imp_?AfxWinMain@@YGHPAUHINSTANCE__@@0PADH@Z 004828fc     mfc90:mfc90.dll
 0002:00000900       __imp_?OnClose@CFrameWndEx@@QAEXXZ 00482900     mfc90:mfc90.dll
 0002:00000904       __imp_?OnSysCommand@CFrameWnd@@IAEXIJ@Z 00482904     mfc90:mfc90.dll
 0002:00000908       __imp_?PreTranslateMessage@CFrameWndEx@@UAEHPAUtagMSG@@@Z 00482908     mfc90:mfc90.dll
 0002:0000090c       __imp_?SetWordCharFormat@CRichEditCtrl@@QAEHAAU_charformat@@@Z 0048290c     mfc90:mfc90.dll
 0002:00000910       __imp_?SetSel@CRichEditCtrl@@QAEXJJ@Z 00482910     mfc90:mfc90.dll
 0002:00000914       __imp_?GetWindowTextLengthA@CWnd@@QBEHXZ 00482914     mfc90:mfc90.dll
 0002:00000918       __imp_?GetCategory@CMFCRibbonBar@@QBEPAVCMFCRibbonCategory@@H@Z 00482918     mfc90:mfc90.dll
 0002:0000091c       __imp_?wndTopMost@CWnd@@2V1@B 0048291c     mfc90:mfc90.dll
 0002:00000920       __imp_?DoModal@CPropertySheet@@UAEHXZ 00482920     mfc90:mfc90.dll
 0002:00000924       __imp_?EnablePageHeader@CMFCPropertySheet@@QAEXH@Z 00482924     mfc90:mfc90.dll
 0002:00000928       __imp_?GetThisMessageMap@CMFCOutlookBar@@KGPBUAFX_MSGMAP@@XZ 00482928     mfc90:mfc90.dll
 0002:0000092c       __imp_?OnRButtonDown@CDockablePane@@IAEXIVCPoint@@@Z 0048292c     mfc90:mfc90.dll
 0002:00000930       __imp_?RemoveHead@CPtrList@@QAEPAXXZ 00482930     mfc90:mfc90.dll
 0002:00000934       __imp_?AddTail@CPtrList@@QAEPAU__POSITION@@PAX@Z 00482934     mfc90:mfc90.dll
 0002:00000938       __imp_?BeginWaitCursor@CCmdTarget@@QAEXXZ 00482938     mfc90:mfc90.dll
 0002:0000093c       __imp_?EndWaitCursor@CCmdTarget@@QAEXXZ 0048293c     mfc90:mfc90.dll
 0002:00000940       __imp_?UpdateCount@CMFCToolBarImages@@IAEXXZ 00482940     mfc90:mfc90.dll
 0002:00000944       __imp_?UpdateInternalImage@CMFCToolBarImages@@IAEHH@Z 00482944     mfc90:mfc90.dll
 0002:00000948       __imp_?m_bHideInAutoHideMode@CDockablePane@@2HA 00482948     mfc90:mfc90.dll
 0002:0000094c       __imp_?OnCtlColor@CWnd@@IAEPAUHBRUSH__@@PAVCDC@@PAV1@I@Z 0048294c     mfc90:mfc90.dll
 0002:00000950       __imp_??0CMFCRibbonButton@@QAE@XZ 00482950     mfc90:mfc90.dll
 0002:00000954       __imp_?GetRuntimeClass@CMFCRibbonApplicationButton@@UBEPAUCRuntimeClass@@XZ 00482954     mfc90:mfc90.dll
 0002:00000958       __imp_?SetID@CMFCRibbonBaseElement@@UAEXI@Z 00482958     mfc90:mfc90.dll
 0002:0000095c       __imp_?SetText@CMFCRibbonButton@@UAEXPBD@Z 0048295c     mfc90:mfc90.dll
 0002:00000960       __imp_?SetKeys@CMFCRibbonBaseElement@@UAEXPBD0@Z 00482960     mfc90:mfc90.dll
 0002:00000964       __imp_?SetTextAlwaysOnRight@CMFCRibbonBaseElement@@UAEXH@Z 00482964     mfc90:mfc90.dll
 0002:00000968       __imp_?GetToolTipText@CMFCRibbonButton@@UBE?AV?$CStringT@DV?$StrTraitMFC_DLL@DV?$ChTraitsCRT@D@ATL@@@@@ATL@@XZ 00482968     mfc90:mfc90.dll
 0002:0000096c       __imp_?GetDescription@CMFCRibbonBaseElement@@UBE?AV?$CStringT@DV?$StrTraitMFC_DLL@DV?$ChTraitsCRT@D@ATL@@@@@ATL@@XZ 0048296c     mfc90:mfc90.dll
 0002:00000970       __imp_?SetToolTipText@CMFCRibbonBaseElement@@UAEXPBD@Z 00482970     mfc90:mfc90.dll
 0002:00000974       __imp_?SetDescription@CMFCRibbonButton@@UAEXPBD@Z 00482974     mfc90:mfc90.dll
 0002:00000978       __imp_?GetRegularSize@CMFCRibbonButton@@UAE?AVCSize@@PAVCDC@@@Z 00482978     mfc90:mfc90.dll
 0002:0000097c       __imp_?GetCompactSize@CMFCRibbonButton@@UAE?AVCSize@@PAVCDC@@@Z 0048297c     mfc90:mfc90.dll
 0002:00000980       __imp_?GetIntermediateSize@CMFCRibbonButton@@UAE?AVCSize@@PAVCDC@@@Z 00482980     mfc90:mfc90.dll
 0002:00000984       __imp_?OnAfterChangeRect@CMFCRibbonButton@@MAEXPAVCDC@@@Z 00482984     mfc90:mfc90.dll
 0002:00000988       __imp_?HitTest@CMFCRibbonBaseElement@@UAEPAV1@VCPoint@@@Z 00482988     mfc90:mfc90.dll
 0002:0000098c       __imp_?GetParentPanel@CMFCRibbonBaseElement@@UBEPAVCMFCRibbonPanel@@XZ 0048298c     mfc90:mfc90.dll
 0002:00000990       __imp_?GetParentWnd@CMFCRibbonBaseElement@@UBEPAVCWnd@@XZ 00482990     mfc90:mfc90.dll
 0002:00000994       __imp_?SetParentRibbonBar@CMFCRibbonButton@@MAEXPAVCMFCRibbonBar@@@Z 00482994     mfc90:mfc90.dll
 0002:00000998       __imp_?OnShowPopupMenu@CMFCRibbonButton@@MAEXXZ 00482998     mfc90:mfc90.dll
 0002:0000099c       __imp_?StretchToWholeRow@CMFCRibbonBaseElement@@UAEHPAVCDC@@H@Z 0048299c     mfc90:mfc90.dll
 0002:000009a0       __imp_?SetParentCategory@CMFCRibbonButton@@UAEXPAVCMFCRibbonCategory@@@Z 004829a0     mfc90:mfc90.dll
 0002:000009a4       __imp_?CopyFrom@CMFCRibbonButton@@MAEXABVCMFCRibbonBaseElement@@@Z 004829a4     mfc90:mfc90.dll
 0002:000009a8       __imp_?SetParentMenu@CMFCRibbonBaseElement@@UAEXPAVCMFCRibbonPanelMenuBar@@@Z 004829a8     mfc90:mfc90.dll
 0002:000009ac       __imp_?SetOriginal@CMFCRibbonButton@@MAEXPAVCMFCRibbonBaseElement@@@Z 004829ac     mfc90:mfc90.dll
 0002:000009b0       __imp_?OnDrawOnList@CMFCRibbonButton@@MAEXPAVCDC@@V?$CStringT@DV?$StrTraitMFC_DLL@DV?$ChTraitsCRT@D@ATL@@@@@ATL@@HVCRect@@HH@Z 004829b0     mfc90:mfc90.dll
 0002:000009b4       __imp_?OnDraw@CMFCRibbonButton@@UAEXPAVCDC@@@Z 004829b4     mfc90:mfc90.dll
 0002:000009b8       __imp_?OnCalcTextSize@CMFCRibbonButton@@UAEXPAVCDC@@@Z 004829b8     mfc90:mfc90.dll
 0002:000009bc       __imp_?CanBeStretched@CMFCRibbonButton@@UAEHXZ 004829bc     mfc90:mfc90.dll
 0002:000009c0       __imp_?ClosePopupMenu@CMFCRibbonButton@@UAEXXZ 004829c0     mfc90:mfc90.dll
 0002:000009c4       __imp_?Find@CMFCRibbonBaseElement@@UAEPAV1@PBV1@@Z 004829c4     mfc90:mfc90.dll
 0002:000009c8       __imp_?FindByID@CMFCRibbonButton@@MAEPAVCMFCRibbonBaseElement@@I@Z 004829c8     mfc90:mfc90.dll
 0002:000009cc       __imp_?FindByData@CMFCRibbonButton@@MAEPAVCMFCRibbonBaseElement@@K@Z 004829cc     mfc90:mfc90.dll
 0002:000009d0       __imp_?FindByOriginal@CMFCRibbonBaseElement@@UAEPAV1@PAV1@@Z 004829d0     mfc90:mfc90.dll
 0002:000009d4       __imp_?UpdateTooltipInfo@CMFCRibbonBaseElement@@UAEXXZ 004829d4     mfc90:mfc90.dll
 0002:000009d8       __imp_?OnAddToQAToolbar@CMFCRibbonBaseElement@@UAEHAAVCMFCRibbonQuickAccessToolBar@@@Z 004829d8     mfc90:mfc90.dll
 0002:000009dc       __imp_?Redraw@CMFCRibbonBaseElement@@UAEXXZ 004829dc     mfc90:mfc90.dll
 0002:000009e0       __imp_?GetPressed@CMFCRibbonBaseElement@@UAEPAV1@XZ 004829e0     mfc90:mfc90.dll
 0002:000009e4       __imp_?GetDroppedDown@CMFCRibbonBaseElement@@UAEPAV1@XZ 004829e4     mfc90:mfc90.dll
 0002:000009e8       __imp_?GetHighlighted@CMFCRibbonBaseElement@@UAEPAV1@XZ 004829e8     mfc90:mfc90.dll
 0002:000009ec       __imp_?OnDrawKeyTip@CMFCRibbonBaseElement@@UAEXPAVCDC@@ABVCRect@@H@Z 004829ec     mfc90:mfc90.dll
 0002:000009f0       __imp_?GetKeyTipSize@CMFCRibbonBaseElement@@UAE?AVCSize@@PAVCDC@@@Z 004829f0     mfc90:mfc90.dll
 0002:000009f4       __imp_?GetKeyTipRect@CMFCRibbonButton@@MAE?AVCRect@@PAVCDC@@H@Z 004829f4     mfc90:mfc90.dll
 0002:000009f8       __imp_?OnKey@CMFCRibbonApplicationButton@@MAEHH@Z 004829f8     mfc90:mfc90.dll
 0002:000009fc       __imp_?AddToKeyList@CMFCRibbonBaseElement@@UAEXAAV?$CArray@PAVCMFCRibbonKeyTip@@PAV1@@@@Z 004829fc     mfc90:mfc90.dll
 0002:00000a00       __imp_?GetElementsByID@CMFCRibbonButton@@MAEXIAAV?$CArray@PAVCMFCRibbonBaseElement@@PAV1@@@@Z 00482a00     mfc90:mfc90.dll
 0002:00000a04       __imp_?GetElements@CMFCRibbonButton@@MAEXAAV?$CArray@PAVCMFCRibbonBaseElement@@PAV1@@@@Z 00482a04     mfc90:mfc90.dll
 0002:00000a08       __imp_?NotifyHighlightListItem@CMFCRibbonBaseElement@@UAEXH@Z 00482a08     mfc90:mfc90.dll
 0002:00000a0c       __imp_?OnLButtonDown@CMFCRibbonApplicationButton@@MAEXVCPoint@@@Z 00482a0c     mfc90:mfc90.dll
 0002:00000a10       __imp_?OnLButtonUp@CMFCRibbonButton@@MAEXVCPoint@@@Z 00482a10     mfc90:mfc90.dll
 0002:00000a14       __imp_?OnMouseMove@CMFCRibbonButton@@MAEXVCPoint@@@Z 00482a14     mfc90:mfc90.dll
 0002:00000a18       __imp_?OnLButtonDblClk@CMFCRibbonApplicationButton@@MAEXVCPoint@@@Z 00482a18     mfc90:mfc90.dll
 0002:00000a1c       __imp_?OnUpdateCmdUI@CMFCRibbonBaseElement@@MAEXPAVCMFCRibbonCmdUI@@PAVCFrameWnd@@H@Z 00482a1c     mfc90:mfc90.dll
 0002:00000a20       __imp_?NotifyControlCommand@CMFCRibbonBaseElement@@MAEHHHIJ@Z 00482a20     mfc90:mfc90.dll
 0002:00000a24       __imp_?ReplaceByID@CMFCRibbonBaseElement@@MAEHIPAV1@@Z 00482a24     mfc90:mfc90.dll
 0002:00000a28       __imp_?GetItemIDsList@CMFCRibbonBaseElement@@MBEXAAV?$CList@II@@@Z 00482a28     mfc90:mfc90.dll
 0002:00000a2c       __imp_?GetDropDownImageWidth@CMFCRibbonBaseElement@@MBEHXZ 00482a2c     mfc90:mfc90.dll
 0002:00000a30       __imp_?DrawRibbonText@CMFCRibbonButton@@UAEHPAVCDC@@ABV?$CStringT@DV?$StrTraitMFC_DLL@DV?$ChTraitsCRT@D@ATL@@@@@ATL@@VCRect@@IK@Z 00482a30     mfc90:mfc90.dll
 0002:00000a34       __imp_?OnClick@CMFCRibbonButton@@UAEXVCPoint@@@Z 00482a34     mfc90:mfc90.dll
 0002:00000a38       __imp_?OnFillBackground@CMFCRibbonButton@@UAEKPAVCDC@@@Z 00482a38     mfc90:mfc90.dll
 0002:00000a3c       __imp_?OnDrawBorder@CMFCRibbonButton@@UAEXPAVCDC@@@Z 00482a3c     mfc90:mfc90.dll
 0002:00000a40       __imp_?DrawEx@CMFCToolBarImages@@QAEHPAVCDC@@VCRect@@HW4ImageAlignHorz@1@W4ImageAlignVert@1@1E@Z 00482a40     mfc90:mfc90.dll
 0002:00000a44       __imp_?SetACCData@CMFCRibbonButton@@UAEHPAVCWnd@@AAVCAccessibilityData@@@Z 00482a44     mfc90:mfc90.dll
 0002:00000a48       __imp_?AddDefaultButtonsToCustomizePane@CFrameImpl@@IAEXPAVCMFCPopupMenu@@I@Z 00482a48     mfc90:mfc90.dll
 0002:00000a4c       __imp_?Create@CAsyncSocket@@QAEHIHJPBD@Z 00482a4c     mfc90:mfc90.dll
 0002:00000a50       __imp_??$SerializeElements@V?$CStringT@DV?$StrTraitMFC_DLL@DV?$ChTraitsCRT@D@ATL@@@@@ATL@@@@YGXAAVCArchive@@PAV?$CStringT@DV?$StrTraitMFC_DLL@DV?$ChTraitsCRT@D@ATL@@@@@ATL@@H@Z 00482a50     mfc90:mfc90.dll
 0002:00000a54       __imp_??$HashKey@PBD@@YGIPBD@Z 00482a54     mfc90:mfc90.dll
 0002:00000a58       __imp_?GetThisClass@CMFCRibbonBar@@SGPAUCRuntimeClass@@XZ 00482a58     mfc90:mfc90.dll
 0002:00000a5c       __imp_??0CMFCRibbonBar@@QAE@H@Z 00482a5c     mfc90:mfc90.dll
 0002:00000a60       __imp_?Serialize@CBasePane@@UAEXAAVCArchive@@@Z 00482a60     mfc90:mfc90.dll
 0002:00000a64       __imp_?PreCreateWindow@CMFCRibbonBar@@MAEHAAUtagCREATESTRUCTA@@@Z 00482a64     mfc90:mfc90.dll
 0002:00000a68       __imp_?OnCommand@CMFCRibbonBar@@MAEHIJ@Z 00482a68     mfc90:mfc90.dll
 0002:00000a6c       __imp_?PreTranslateMessage@CMFCRibbonBar@@UAEHPAUtagMSG@@@Z 00482a6c     mfc90:mfc90.dll
 0002:00000a70       __imp_?WindowProc@CMFCRibbonBar@@MAEJIIJ@Z 00482a70     mfc90:mfc90.dll
 0002:00000a74       __imp_?IsDocked@CBasePane@@UBEHXZ 00482a74     mfc90:mfc90.dll
 0002:00000a78       __imp_?IsVisible@CBasePane@@UBEHXZ 00482a78     mfc90:mfc90.dll
 0002:00000a7c       __imp_?CanFloat@CBasePane@@UBEHXZ 00482a7c     mfc90:mfc90.dll
 0002:00000a80       __imp_?FloatPane@CPane@@UAEHVCRect@@W4AFX_DOCK_METHOD@@_N@Z 00482a80     mfc90:mfc90.dll
 0002:00000a84       __imp_?RecalcLayout@CMFCRibbonBar@@UAEXXZ 00482a84     mfc90:mfc90.dll
 0002:00000a88       __imp_?OnBeforeChangeParent@CPane@@UAEXPAVCWnd@@H@Z 00482a88     mfc90:mfc90.dll
 0002:00000a8c       __imp_?OnAfterChangeParent@CPane@@UAEXPAVCWnd@@@Z 00482a8c     mfc90:mfc90.dll
 0002:00000a90       __imp_?ShowPane@CBasePane@@UAEXHHH@Z 00482a90     mfc90:mfc90.dll
 0002:00000a94       __imp_?LoadState@CMFCRibbonBar@@MAEHPBDHI@Z 00482a94     mfc90:mfc90.dll
 0002:00000a98       __imp_?SaveState@CMFCRibbonBar@@MAEHPBDHI@Z 00482a98     mfc90:mfc90.dll
 0002:00000a9c       __imp_?UndockPane@CPane@@UAEXH@Z 00482a9c     mfc90:mfc90.dll
 0002:00000aa0       __imp_?OnUpdateCmdUI@CMFCRibbonBar@@MAEXPAVCFrameWnd@@H@Z 00482aa0     mfc90:mfc90.dll
 0002:00000aa4       __imp_?OnPaneContextMenu@CMFCRibbonBar@@MAEXPAVCWnd@@VCPoint@@@Z 00482aa4     mfc90:mfc90.dll
 0002:00000aa8       __imp_?OnSetAccData@CMFCRibbonBar@@UAEHJ@Z 00482aa8     mfc90:mfc90.dll
 0002:00000aac       __imp_?CalcFixedLayout@CMFCRibbonBar@@MAE?AVCSize@@HH@Z 00482aac     mfc90:mfc90.dll
 0002:00000ab0       __imp_?GetPaneName@CPane@@UBEXAAV?$CStringT@DV?$StrTraitMFC_DLL@DV?$ChTraitsCRT@D@ATL@@@@@ATL@@@Z 00482ab0     mfc90:mfc90.dll
 0002:00000ab4       __imp_?IsChangeState@CPane@@UBE?AW4AFX_CS_STATUS@@HPAPAVCBasePane@@@Z 00482ab4     mfc90:mfc90.dll
 0002:00000ab8       __imp_?OnBeforeFloat@CPane@@UAEHAAVCRect@@W4AFX_DOCK_METHOD@@@Z 00482ab8     mfc90:mfc90.dll
 0002:00000abc       __imp_?OnPressCloseButton@CPane@@UAEXXZ 00482abc     mfc90:mfc90.dll
 0002:00000ac0       __imp_?ConvertToTabbedDocument@CPane@@UAEXH@Z 00482ac0     mfc90:mfc90.dll
 0002:00000ac4       __imp_?OnContinueMoving@CPane@@MAEXXZ 00482ac4     mfc90:mfc90.dll
 0002:00000ac8       __imp_?Dock@CPane@@MAEHPAVCBasePane@@PBUtagRECT@@W4AFX_DOCK_METHOD@@@Z 00482ac8     mfc90:mfc90.dll
 0002:00000acc       __imp_?EnterDragMode@CPane@@MAEXH@Z 00482acc     mfc90:mfc90.dll
 0002:00000ad0       __imp_?OnRTLChanged@CMFCRibbonBar@@UAEXH@Z 00482ad0     mfc90:mfc90.dll
 0002:00000ad4       __imp_?StoreRecentDockSiteInfo@CPane@@MAEXXZ 00482ad4     mfc90:mfc90.dll
 0002:00000ad8       __imp_?SetActiveCategory@CMFCRibbonBar@@UAEHPAVCMFCRibbonCategory@@H@Z 00482ad8     mfc90:mfc90.dll
 0002:00000adc       __imp_?HitTest@CMFCRibbonBar@@UAEPAVCMFCRibbonBaseElement@@VCPoint@@HH@Z 00482adc     mfc90:mfc90.dll
 0002:00000ae0       __imp_?GetDroppedDown@CMFCRibbonBar@@UAEPAVCMFCRibbonBaseElement@@XZ 00482ae0     mfc90:mfc90.dll
 0002:00000ae4       __imp_?ReleaseBuffer@?$CSimpleStringT@D$00@ATL@@QAEXH@Z 00482ae4     mfc90:mfc90.dll
 0002:00000ae8       __imp_?InitApplication@CWinApp@@UAEHXZ 00482ae8     mfc90:mfc90.dll
 0002:00000aec       __imp_?DWMCompositionChanged@CMFCRibbonBar@@UAEXXZ 00482aec     mfc90:mfc90.dll
 0002:00000af0       __imp_?OnShowRibbonQATMenu@CMFCRibbonBar@@UAEHPAVCWnd@@HHPAVCMFCRibbonBaseElement@@@Z 00482af0     mfc90:mfc90.dll
 0002:00000af4       __imp_?TranslateChar@CMFCRibbonBar@@UAEHI@Z 00482af4     mfc90:mfc90.dll
 0002:00000af8       __imp_?OnFillBackground@CMFCRibbonBar@@MAEXPAVCDC@@VCRect@@@Z 00482af8     mfc90:mfc90.dll
 0002:00000afc       __imp_?OnSetPrintPreviewKeys@CMFCRibbonBar@@MAEXPAVCMFCRibbonPanel@@00@Z 00482afc     mfc90:mfc90.dll
 0002:00000b00       __imp_?OnBeforeProcessKey@CMFCRibbonBar@@MAEXAAH@Z 00482b00     mfc90:mfc90.dll
 0002:00000b04       __imp_??1CMFCRibbonBar@@UAE@XZ 00482b04     mfc90:mfc90.dll
 0002:00000b08       __imp_?GetThisMessageMap@CMFCRibbonBar@@KGPBUAFX_MSGMAP@@XZ 00482b08     mfc90:mfc90.dll
 0002:00000b0c       __imp_?GetThisClass@CMFCPropertyPage@@SGPAUCRuntimeClass@@XZ 00482b0c     mfc90:mfc90.dll
 0002:00000b10       __imp_??1CMFCPropertyPage@@UAE@XZ 00482b10     mfc90:mfc90.dll
 0002:00000b14       __imp_??0CMFCPropertyPage@@QAE@II@Z 00482b14     mfc90:mfc90.dll
 0002:00000b18       __imp_?OnCommand@CMFCPropertyPage@@MAEHIJ@Z 00482b18     mfc90:mfc90.dll
 0002:00000b1c       __imp_?OnNotify@CPropertyPage@@MAEHIJPAJ@Z 00482b1c     mfc90:mfc90.dll
 0002:00000b20       __imp_?PreTranslateMessage@CMFCPropertyPage@@UAEHPAUtagMSG@@@Z 00482b20     mfc90:mfc90.dll
 0002:00000b24       __imp_?OnOK@CPropertyPage@@UAEXXZ 00482b24     mfc90:mfc90.dll
 0002:00000b28       __imp_?OnCancel@CPropertyPage@@UAEXXZ 00482b28     mfc90:mfc90.dll
 0002:00000b2c       __imp_?OnApply@CPropertyPage@@UAEHXZ 00482b2c     mfc90:mfc90.dll
 0002:00000b30       __imp_?OnReset@CPropertyPage@@UAEXXZ 00482b30     mfc90:mfc90.dll
 0002:00000b34       __imp_?OnSetActive@CMFCPropertyPage@@UAEHXZ 00482b34     mfc90:mfc90.dll
 0002:00000b38       __imp_?OnKillActive@CPropertyPage@@UAEHXZ 00482b38     mfc90:mfc90.dll
 0002:00000b3c       __imp_?OnQueryCancel@CPropertyPage@@UAEHXZ 00482b3c     mfc90:mfc90.dll
 0002:00000b40       __imp_?OnWizardBack@CPropertyPage@@UAEJXZ 00482b40     mfc90:mfc90.dll
 0002:00000b44       __imp_?OnWizardNext@CPropertyPage@@UAEJXZ 00482b44     mfc90:mfc90.dll
 0002:00000b48       __imp_?OnWizardFinish@CPropertyPage@@UAEHXZ 00482b48     mfc90:mfc90.dll
 0002:00000b4c       __imp_?OnWizardFinishEx@CPropertyPage@@UAEPAUHWND__@@XZ 00482b4c     mfc90:mfc90.dll
 0002:00000b50       __imp_?GetThisMessageMap@CMFCPropertyPage@@KGPBUAFX_MSGMAP@@XZ 00482b50     mfc90:mfc90.dll
 0002:00000b54       __imp_?DDX_Radio@@YGXPAVCDataExchange@@HAAH@Z 00482b54     mfc90:mfc90.dll
 0002:00000b58       __imp_?OnInitDialog@CMFCPropertyPage@@MAEHXZ 00482b58     mfc90:mfc90.dll
 0002:00000b5c       __imp_?GetThisClass@CMFCPropertySheet@@SGPAUCRuntimeClass@@XZ 00482b5c     mfc90:mfc90.dll
 0002:00000b60       __imp_??1CMFCPropertySheet@@UAE@XZ 00482b60     mfc90:mfc90.dll
 0002:00000b64       __imp_?AddPage@CMFCPropertySheet@@QAEXPAVCPropertyPage@@@Z 00482b64     mfc90:mfc90.dll
 0002:00000b68       __imp_?Create@CFormView@@MAEHPBD0KABUtagRECT@@PAVCWnd@@IPAUCCreateContext@@@Z 00482b68     mfc90:mfc90.dll
 0002:00000b6c       __imp_?FindFile@CFileFind@@UAEHPBDK@Z 00482b6c     mfc90:mfc90.dll
 0002:00000b70       __imp_??0CMFCPropertySheet@@QAE@PBDPAVCWnd@@I@Z 00482b70     mfc90:mfc90.dll
 0002:00000b74       __imp_?OnCmdMsg@CPropertySheet@@UAEHIHPAXPAUAFX_CMDHANDLERINFO@@@Z 00482b74     mfc90:mfc90.dll
 0002:00000b78       __imp_?ContinueModal@CPropertySheet@@UAEHXZ 00482b78     mfc90:mfc90.dll
 0002:00000b7c       __imp_?PreTranslateMessage@CMFCPropertySheet@@UAEHPAUtagMSG@@@Z 00482b7c     mfc90:mfc90.dll
 0002:00000b80       __imp_?Create@CPropertySheet@@UAEHPAVCWnd@@KK@Z 00482b80     mfc90:mfc90.dll
 0002:00000b84       __imp_?BuildPropPageArray@CPropertySheet@@UAEXXZ 00482b84     mfc90:mfc90.dll
 0002:00000b88       __imp_?OnActivatePage@CMFCPropertySheet@@UAEXPAVCPropertyPage@@@Z 00482b88     mfc90:mfc90.dll
 0002:00000b8c       __imp_?InitNavigationControl@CMFCPropertySheet@@UAEPAVCWnd@@XZ 00482b8c     mfc90:mfc90.dll
 0002:00000b90       __imp_?OnRemoveTreePage@CMFCPropertySheet@@UAEHPAVCPropertyPage@@@Z 00482b90     mfc90:mfc90.dll
 0002:00000b94       __imp_?GetThisMessageMap@CMFCPropertySheet@@KGPBUAFX_MSGMAP@@XZ 00482b94     mfc90:mfc90.dll
 0002:00000b98       __imp_??1CDrawingManager@@UAE@XZ 00482b98     mfc90:mfc90.dll
 0002:00000b9c       __imp_?DrawShadow@CDrawingManager@@QAEHVCRect@@HHHPAVCBitmap@@1KH@Z 00482b9c     mfc90:mfc90.dll
 0002:00000ba0       __imp_??0CDrawingManager@@QAE@AAVCDC@@@Z 00482ba0     mfc90:mfc90.dll
 0002:00000ba4       __imp_?Draw3dRect@CDC@@QAEXPBUtagRECT@@KK@Z 00482ba4     mfc90:mfc90.dll
 0002:00000ba8       __imp_?OnCommand@CPropertySheet@@UAEHIJ@Z 00482ba8     mfc90:mfc90.dll
 0002:00000bac       __imp_?OnInitDialog@CMFCPropertySheet@@UAEHXZ 00482bac     mfc90:mfc90.dll
 0002:00000bb0       __imp_?GetRuntimeClass@CRichEditCtrl@@UBEPAUCRuntimeClass@@XZ 00482bb0     mfc90:mfc90.dll
 0002:00000bb4       __imp_??1CRichEditCtrl@@UAE@XZ 00482bb4     mfc90:mfc90.dll
 0002:00000bb8       __imp_?TrackPopupMenu@CMenu@@QAEHIHHPAVCWnd@@PBUtagRECT@@@Z 00482bb8     mfc90:mfc90.dll
 0002:00000bbc       __imp_?CanPaste@CRichEditCtrl@@QBEHI@Z 00482bbc     mfc90:mfc90.dll
 0002:00000bc0       __imp_?GetStyle@CWnd@@QBEKXZ 00482bc0     mfc90:mfc90.dll
 0002:00000bc4       __imp_?GetItemData@CListCtrl@@QBEKH@Z 00482bc4     mfc90:mfc90.dll
 0002:00000bc8       __imp_?FromHandle@CDC@@SGPAV1@PAUHDC__@@@Z 00482bc8     mfc90:mfc90.dll
 0002:00000bcc       __imp_?GetItemRect@CListCtrl@@QBEHHPAUtagRECT@@I@Z 00482bcc     mfc90:mfc90.dll
 0002:00000bd0       __imp_??0CBrush@@QAE@K@Z   00482bd0     mfc90:mfc90.dll
 0002:00000bd4       __imp_?OnDestroy@CWnd@@IAEXXZ 00482bd4     mfc90:mfc90.dll
 0002:00000bd8       __imp_?GetRuntimeClass@CBrush@@UBEPAUCRuntimeClass@@XZ 00482bd8     mfc90:mfc90.dll
 0002:00000bdc       __imp_?SetItem@CListCtrl@@QAEHHHIPBDHIIJ@Z 00482bdc     mfc90:mfc90.dll
 0002:00000be0       __imp_??1CMFCToolBar@@UAE@XZ 00482be0     mfc90:mfc90.dll
 0002:00000be4       __imp_??1CDockablePane@@UAE@XZ 00482be4     mfc90:mfc90.dll
 0002:00000be8       __imp_??0CMFCTabCtrl@@QAE@XZ 00482be8     mfc90:mfc90.dll
 0002:00000bec       __imp_??0CMFCToolBar@@QAE@XZ 00482bec     mfc90:mfc90.dll
 0002:00000bf0       __imp_??0CDockablePane@@QAE@XZ 00482bf0     mfc90:mfc90.dll
 0002:00000bf4       __imp_?GetRuntimeClass@CDockablePane@@UBEPAUCRuntimeClass@@XZ 00482bf4     mfc90:mfc90.dll
 0002:00000bf8       __imp_?Serialize@CDockablePane@@UAEXAAVCArchive@@@Z 00482bf8     mfc90:mfc90.dll
 0002:00000bfc       __imp_?RecalcLayout@CPane@@UAEXXZ 00482bfc     mfc90:mfc90.dll
 0002:00000c00       __imp_?LoadState@CDockablePane@@UAEHPBDHI@Z 00482c00     mfc90:mfc90.dll
 0002:00000c04       __imp_?SaveState@CDockablePane@@UAEHPBDHI@Z 00482c04     mfc90:mfc90.dll
 0002:00000c08       __imp_?ConvertToTabbedDocument@CDockablePane@@UAEXH@Z 00482c08     mfc90:mfc90.dll
 0002:00000c0c       __imp_?Dock@CDockablePane@@MAEHPAVCBasePane@@PBUtagRECT@@W4AFX_DOCK_METHOD@@@Z 00482c0c     mfc90:mfc90.dll
 0002:00000c10       __imp_?StoreRecentDockSiteInfo@CDockablePane@@MAEXXZ 00482c10     mfc90:mfc90.dll
 0002:00000c14       __imp_?GetDockingStatus@CDockablePane@@UAE?AW4AFX_CS_STATUS@@VCPoint@@H@Z 00482c14     mfc90:mfc90.dll
 0002:00000c18       __imp_?SetAutoHideMode@CDockablePane@@UAEPAVCMFCAutoHideBar@@HKPAV2@H@Z 00482c18     mfc90:mfc90.dll
 0002:00000c1c       __imp_??1CMFCTabCtrl@@UAE@XZ 00482c1c     mfc90:mfc90.dll
 0002:00000c20       __imp_?GetThisMessageMap@CDockablePane@@KGPBUAFX_MSGMAP@@XZ 00482c20     mfc90:mfc90.dll
 0002:00000c24       __imp_?OnSetFocus@CDockablePane@@IAEXPAVCWnd@@@Z 00482c24     mfc90:mfc90.dll
 0002:00000c28       __imp_?Create@CRichEditCtrl@@QAEHKABUtagRECT@@PAVCWnd@@I@Z 00482c28     mfc90:mfc90.dll
 0002:00000c2c       __imp_?Create@CMFCTabCtrl@@QAEHW4Style@1@ABUtagRECT@@PAVCWnd@@IW4Location@CMFCBaseTabCtrl@@H@Z 00482c2c     mfc90:mfc90.dll
 0002:00000c30       __imp_?OnCreate@CDockablePane@@IAEHPAUtagCREATESTRUCTA@@@Z 00482c30     mfc90:mfc90.dll
 0002:00000c34       __imp_?OnSize@CBasePane@@IAEXIHH@Z 00482c34     mfc90:mfc90.dll
 0002:00000c38       __imp_?GetTopLevelFrame@CWnd@@QBEPAVCFrameWnd@@XZ 00482c38     mfc90:mfc90.dll
 0002:00000c3c       __imp_?AfxDynamicDownCast@@YAPAVCObject@@PAUCRuntimeClass@@PAV1@@Z 00482c3c     mfc90:mfc90.dll
 0002:00000c40       __imp_?GetThisClass@CDockablePane@@SGPAUCRuntimeClass@@XZ 00482c40     mfc90:mfc90.dll
 0002:00000c44       __imp_?OnLButtonDown@CDockablePane@@IAEXIVCPoint@@@Z 00482c44     mfc90:mfc90.dll
 0002:00000c48       __imp_?ScreenToClient@CWnd@@QBEXPAUtagRECT@@@Z 00482c48     mfc90:mfc90.dll
 0002:00000c4c       __imp_?FromHandle@CGdiObject@@SGPAV1@PAX@Z 00482c4c     mfc90:mfc90.dll
 0002:00000c50       __imp_?DDX_Text@@YGXPAVCDataExchange@@HAAH@Z 00482c50     mfc90:mfc90.dll
 0002:00000c54       __imp_??1CProgressCtrl@@UAE@XZ 00482c54     mfc90:mfc90.dll
 0002:00000c58       __imp_?GetRuntimeClass@CProgressCtrl@@UBEPAUCRuntimeClass@@XZ 00482c58     mfc90:mfc90.dll
 0002:00000c5c       __imp_?Create@CProgressCtrl@@UAEHKABUtagRECT@@PAVCWnd@@I@Z 00482c5c     mfc90:mfc90.dll
 0002:00000c60       __imp_?CreateEx@CProgressCtrl@@UAEHKKABUtagRECT@@PAVCWnd@@I@Z 00482c60     mfc90:mfc90.dll
 0002:00000c64       __imp_??1CTabCtrl@@UAE@XZ  00482c64     mfc90:mfc90.dll
 0002:00000c68       __imp_?GetNextAssoc@CMapStringToString@@QBEXAAPAU__POSITION@@AAV?$CStringT@DV?$StrTraitMFC_DLL@DV?$ChTraitsCRT@D@ATL@@@@@ATL@@1@Z 00482c68     mfc90:mfc90.dll
 0002:00000c6c       __imp_?Replace@?$CStringT@DV?$StrTraitMFC_DLL@DV?$ChTraitsCRT@D@ATL@@@@@ATL@@QAEHPBD0@Z 00482c6c     mfc90:mfc90.dll
 0002:00000c70       __imp_?GetRuntimeClass@CTabCtrl@@UBEPAUCRuntimeClass@@XZ 00482c70     mfc90:mfc90.dll
 0002:00000c74       __imp_?GetMessageMap@CTabCtrl@@MBEPBUAFX_MSGMAP@@XZ 00482c74     mfc90:mfc90.dll
 0002:00000c78       __imp_?OnChildNotify@CTabCtrl@@MAEHIIJPAJ@Z 00482c78     mfc90:mfc90.dll
 0002:00000c7c       __imp_?Create@CTabCtrl@@UAEHKABUtagRECT@@PAVCWnd@@I@Z 00482c7c     mfc90:mfc90.dll
 0002:00000c80       __imp_?CreateEx@CTabCtrl@@UAEHKKABUtagRECT@@PAVCWnd@@I@Z 00482c80     mfc90:mfc90.dll
 0002:00000c84       __imp_?DrawItem@CTabCtrl@@UAEXPAUtagDRAWITEMSTRUCT@@@Z 00482c84     mfc90:mfc90.dll
 0002:00000c88       __imp_?InsertItem@CTabCtrl@@QAEJIHPBDHJ@Z 00482c88     mfc90:mfc90.dll
 0002:00000c8c       __imp_?GetThisClass@CWinThread@@SGPAUCRuntimeClass@@XZ 00482c8c     mfc90:mfc90.dll
 0002:00000c90       __imp_??1CWinThread@@UAE@XZ 00482c90     mfc90:mfc90.dll
 0002:00000c94       __imp_??0CWinThread@@QAE@XZ 00482c94     mfc90:mfc90.dll
 0002:00000c98       __imp_?Run@CWinThread@@UAEHXZ 00482c98     mfc90:mfc90.dll
 0002:00000c9c       __imp_?OnIdle@CWinThread@@UAEHJ@Z 00482c9c     mfc90:mfc90.dll
 0002:00000ca0       __imp_?ProcessWndProcException@CWinThread@@UAEJPAVCException@@PBUtagMSG@@@Z 00482ca0     mfc90:mfc90.dll
 0002:00000ca4       __imp_?ExitInstance@CWinThread@@UAEHXZ 00482ca4     mfc90:mfc90.dll
 0002:00000ca8       __imp_?GetThisMessageMap@CCmdTarget@@KGPBUAFX_MSGMAP@@XZ 00482ca8     mfc90:mfc90.dll
 0002:00000cac       __imp_?DeleteImageList@CImageList@@QAEHXZ 00482cac     mfc90:mfc90.dll
 0002:00000cb0       __imp_?SetSize@CStringArray@@QAEXHH@Z 00482cb0     mfc90:mfc90.dll
 0002:00000cb4       __imp_?Create@CListCtrl@@QAEHKABUtagRECT@@PAVCWnd@@I@Z 00482cb4     mfc90:mfc90.dll
 0002:00000cb8       __imp_?GetCheck@CListCtrl@@QBEHH@Z 00482cb8     mfc90:mfc90.dll
 0002:00000cbc       __imp_?SetCheck@CListCtrl@@QAEHHH@Z 00482cbc     mfc90:mfc90.dll
 0002:00000cc0       __imp_?AfxThrowOleException@@YGXJ@Z 00482cc0     mfc90:mfc90.dll
 0002:00000cc4       __imp_?CompareNoCase@?$CStringT@DV?$StrTraitMFC_DLL@DV?$ChTraitsCRT@D@ATL@@@@@ATL@@QBEHPBD@Z 00482cc4     mfc90:mfc90.dll
 0002:00000cc8       __imp_?GetBufferSetLength@?$CSimpleStringT@D$00@ATL@@QAEPADH@Z 00482cc8     mfc90:mfc90.dll
 0002:00000ccc       __imp_?Flush@CStdioFile@@UAEXXZ 00482ccc     mfc90:mfc90.dll
 0002:00000cd0       __imp_?Open@CStdioFile@@UAEHPBDIPAVCFileException@@@Z 00482cd0     mfc90:mfc90.dll
 0002:00000cd4       __imp_??0CStdioFile@@QAE@XZ 00482cd4     mfc90:mfc90.dll
 0002:00000cd8       __imp_?AddHead@CPtrList@@QAEPAU__POSITION@@PAX@Z 00482cd8     mfc90:mfc90.dll
 0002:00000cdc       __imp_?RemoveAt@CPtrList@@QAEXPAU__POSITION@@@Z 00482cdc     mfc90:mfc90.dll
 0002:00000ce0       __imp_?ReadString@CStdioFile@@UAEHAAV?$CStringT@DV?$StrTraitMFC_DLL@DV?$ChTraitsCRT@D@ATL@@@@@ATL@@@Z 00482ce0     mfc90:mfc90.dll
 0002:00000ce4       __imp_?GetDlgCtrlID@CWnd@@QBEHXZ 00482ce4     mfc90:mfc90.dll
 0002:00000ce8       __imp_?DDV_MaxChars@@YGXPAVCDataExchange@@ABV?$CStringT@DV?$StrTraitMFC_DLL@DV?$ChTraitsCRT@D@ATL@@@@@ATL@@H@Z 00482ce8     mfc90:mfc90.dll
 0002:00000cec       __imp_??1CEdit@@UAE@XZ     00482cec     mfc90:mfc90.dll
 0002:00000cf0       __imp_?Read@CArchive@@QAEIPAXI@Z 00482cf0     mfc90:mfc90.dll
 0002:00000cf4       __imp_?AfxThrowArchiveException@@YGXHPBD@Z 00482cf4     mfc90:mfc90.dll
 0002:00000cf8       __imp_?Write@CArchive@@QAEXPBXI@Z 00482cf8     mfc90:mfc90.dll
 0002:00000cfc       __imp_?Create@CPlex@@SGPAU1@AAPAU1@II@Z 00482cfc     mfc90:mfc90.dll
 0002:00000d00       __imp_?FreeDataChain@CPlex@@QAEXXZ 00482d00     mfc90:mfc90.dll
 0002:00000d04       __imp_?WriteCount@CArchive@@QAEXK@Z 00482d04     mfc90:mfc90.dll
 0002:00000d08       __imp_?ReadCount@CArchive@@QAEKXZ 00482d08     mfc90:mfc90.dll
 0002:00000d0c       __imp_?GetRuntimeClass@CObject@@UBEPAUCRuntimeClass@@XZ 00482d0c     mfc90:mfc90.dll
 0002:00000d10       __imp_?Mid@?$CStringT@DV?$StrTraitMFC_DLL@DV?$ChTraitsCRT@D@ATL@@@@@ATL@@QBE?AV12@HH@Z 00482d10     mfc90:mfc90.dll
 0002:00000d14       __imp_??0CStdioFile@@QAE@PBDI@Z 00482d14     mfc90:mfc90.dll
 0002:00000d18       __imp_?ReadString@CStdioFile@@UAEPADPADI@Z 00482d18     mfc90:mfc90.dll
 0002:00000d1c       __imp_?Find@CStringList@@QBEPAU__POSITION@@PBDPAU2@@Z 00482d1c     mfc90:mfc90.dll
 0002:00000d20       __imp_?InsertAfter@CStringList@@QAEPAU__POSITION@@PAU2@ABV?$CStringT@DV?$StrTraitMFC_DLL@DV?$ChTraitsCRT@D@ATL@@@@@ATL@@@Z 00482d20     mfc90:mfc90.dll
 0002:00000d24       __imp_?AddHead@CStringList@@QAEPAU__POSITION@@ABV?$CStringT@DV?$StrTraitMFC_DLL@DV?$ChTraitsCRT@D@ATL@@@@@ATL@@@Z 00482d24     mfc90:mfc90.dll
 0002:00000d28       __imp_?Close@CStdioFile@@UAEXXZ 00482d28     mfc90:mfc90.dll
 0002:00000d2c       __imp_??1CStdioFile@@UAE@XZ 00482d2c     mfc90:mfc90.dll
 0002:00000d30       __imp_?OnClose@CAsyncSocket@@MAEXH@Z 00482d30     mfc90:mfc90.dll
 0002:00000d34       __imp_?AfxBeginThread@@YGPAVCWinThread@@P6AIPAX@Z0HIKPAU_SECURITY_ATTRIBUTES@@@Z 00482d34     mfc90:mfc90.dll
 0002:00000d38       __imp_?OnAccept@CAsyncSocket@@MAEXH@Z 00482d38     mfc90:mfc90.dll
 0002:00000d3c       __imp_?PumpMessages@CSocket@@MAEHI@Z 00482d3c     mfc90:mfc90.dll
 0002:00000d40       __imp_?OnMessagePending@CSocket@@MAEHXZ 00482d40     mfc90:mfc90.dll
 0002:00000d44       __imp_?SendToHelper@CSocket@@MAEHPBXHPBUsockaddr@@HH@Z 00482d44     mfc90:mfc90.dll
 0002:00000d48       __imp_?ReceiveFromHelper@CSocket@@MAEHPAXHPAUsockaddr@@PAHH@Z 00482d48     mfc90:mfc90.dll
 0002:00000d4c       __imp_?ConnectHelper@CSocket@@MAEHPBUsockaddr@@H@Z 00482d4c     mfc90:mfc90.dll
 0002:00000d50       __imp_?OnConnect@CAsyncSocket@@MAEXH@Z 00482d50     mfc90:mfc90.dll
 0002:00000d54       __imp_?OnOutOfBandData@CAsyncSocket@@MAEXH@Z 00482d54     mfc90:mfc90.dll
 0002:00000d58       __imp_?OnSend@CAsyncSocket@@MAEXH@Z 00482d58     mfc90:mfc90.dll
 0002:00000d5c       __imp_?OnReceive@CAsyncSocket@@MAEXH@Z 00482d5c     mfc90:mfc90.dll
 0002:00000d60       __imp_?Send@CSocket@@UAEHPBXHH@Z 00482d60     mfc90:mfc90.dll
 0002:00000d64       __imp_?Receive@CSocket@@UAEHPAXHH@Z 00482d64     mfc90:mfc90.dll
 0002:00000d68       __imp_?Close@CSocket@@UAEXXZ 00482d68     mfc90:mfc90.dll
 0002:00000d6c       __imp_?Accept@CSocket@@UAEHAAVCAsyncSocket@@PAUsockaddr@@PAH@Z 00482d6c     mfc90:mfc90.dll
 0002:00000d70       __imp_?GetRuntimeClass@CSocket@@UBEPAUCRuntimeClass@@XZ 00482d70     mfc90:mfc90.dll
 0002:00000d74       __imp_??0CSocket@@QAE@XZ   00482d74     mfc90:mfc90.dll
 0002:00000d78       __imp_??1CSocket@@UAE@XZ   00482d78     mfc90:mfc90.dll
 0002:00000d7c       __imp_?Find@?$CStringT@DV?$StrTraitMFC_DLL@DV?$ChTraitsCRT@D@ATL@@@@@ATL@@QBEHPBDH@Z 00482d7c     mfc90:mfc90.dll
 0002:00000d80       __imp_?AddTail@CStringList@@QAEPAU__POSITION@@PBD@Z 00482d80     mfc90:mfc90.dll
 0002:00000d84       __imp_?m_pVisManager@CMFCVisualManager@@1PAV1@A 00482d84     mfc90:mfc90.dll
 0002:00000d88       __imp_?m_pRTIDefault@CMFCVisualManager@@1PAUCRuntimeClass@@A 00482d88     mfc90:mfc90.dll
 0002:00000d8c       __imp_??0CMFCVisualManager@@QAE@H@Z 00482d8c     mfc90:mfc90.dll
 0002:00000d90       __imp_?CreateObject@CRuntimeClass@@QAEPAVCObject@@XZ 00482d90     mfc90:mfc90.dll
 0002:00000d94       __imp_?Create@CMonthCalCtrl@@UAEHKABUtagRECT@@PAVCWnd@@I@Z 00482d94     mfc90:mfc90.dll
 0002:00000d98       __imp_?Create@CMonthCalCtrl@@UAEHKABUtagPOINT@@PAVCWnd@@I@Z 00482d98     mfc90:mfc90.dll
 0002:00000d9c       __imp_?GetRuntimeClass@CMonthCalCtrl@@UBEPAUCRuntimeClass@@XZ 00482d9c     mfc90:mfc90.dll
 0002:00000da0       __imp_?GetString@?$CSimpleStringT@D$00@ATL@@QBEPBDXZ 00482da0     mfc90:mfc90.dll
 0002:00000da4       __imp_?AfxActivateActCtxWrapper@@YG?AW4eActCtxResult@@PAXPAK@Z 00482da4     mfc90:mfc90.dll
 0002:00000da8       __imp_?AfxDeactivateActCtx@@YGHKK@Z 00482da8     mfc90:mfc90.dll
 0002:00000dac       __imp_?AfxGetModuleState@@YGPAVAFX_MODULE_STATE@@XZ 00482dac     mfc90:mfc90.dll
 0002:00000db0       __imp_?AfxFindResourceHandle@@YGPAUHINSTANCE__@@PBD0@Z 00482db0     mfc90:mfc90.dll
 0002:00000db4       __imp_?Attach@CGdiObject@@QAEHPAX@Z 00482db4     mfc90:mfc90.dll
 0002:00000db8       __imp_?DeleteObject@CGdiObject@@QAEHXZ 00482db8     mfc90:mfc90.dll
 0002:00000dbc       __imp_?GetRuntimeClass@CGdiObject@@UBEPAUCRuntimeClass@@XZ 00482dbc     mfc90:mfc90.dll
 0002:00000dc0       __imp_?GetRuntimeClass@CBitmap@@UBEPAUCRuntimeClass@@XZ 00482dc0     mfc90:mfc90.dll
 0002:00000dc4       __imp_??0CPaintDC@@QAE@PAVCWnd@@@Z 00482dc4     mfc90:mfc90.dll
 0002:00000dc8       __imp_?afxGlobalData@@3UAFX_GLOBAL_DATA@@A 00482dc8     mfc90:mfc90.dll
 0002:00000dcc       __imp_?SelectObject@CDC@@QAEPAVCPen@@PAV2@@Z 00482dcc     mfc90:mfc90.dll
 0002:00000dd0       __imp_?MoveTo@CDC@@QAE?AVCPoint@@HH@Z 00482dd0     mfc90:mfc90.dll
 0002:00000dd4       __imp_?LineTo@CDC@@QAEHHH@Z 00482dd4     mfc90:mfc90.dll
 0002:00000dd8       __imp_?SelectStockObject@CDC@@UAEPAVCGdiObject@@H@Z 00482dd8     mfc90:mfc90.dll
 0002:00000ddc       __imp_?SetBkMode@CDC@@QAEHH@Z 00482ddc     mfc90:mfc90.dll
 0002:00000de0       __imp_?SetTextColor@CDC@@UAEKK@Z 00482de0     mfc90:mfc90.dll
 0002:00000de4       __imp_?SelectObject@CDC@@UAEPAVCFont@@PAV2@@Z 00482de4     mfc90:mfc90.dll
 0002:00000de8       __imp_?LoadStringA@?$CStringT@DV?$StrTraitMFC_DLL@DV?$ChTraitsCRT@D@ATL@@@@@ATL@@QAEHI@Z 00482de8     mfc90:mfc90.dll
 0002:00000dec       __imp_?FillSolidRect@CDC@@QAEXPBUtagRECT@@K@Z 00482dec     mfc90:mfc90.dll
 0002:00000df0       __imp_??1CPaintDC@@UAE@XZ  00482df0     mfc90:mfc90.dll
 0002:00000df4       __imp_?SetWindowPos@CWnd@@QAEHPBV1@HHHHI@Z 00482df4     mfc90:mfc90.dll
 0002:00000df8       __imp_?Create@CImageList@@QAEHHHIHH@Z 00482df8     mfc90:mfc90.dll
 0002:00000dfc       __imp_?OnSettingChange@CWnd@@IAEXIPBD@Z 00482dfc     mfc90:mfc90.dll
 0002:00000e00       __imp_?GetThisMessageMap@CWnd@@KGPBUAFX_MSGMAP@@XZ 00482e00     mfc90:mfc90.dll
 0002:00000e04       __imp_??1CImageList@@UAE@XZ 00482e04     mfc90:mfc90.dll
 0002:00000e08       __imp_?GetRuntimeClass@CWnd@@UBEPAUCRuntimeClass@@XZ 00482e08     mfc90:mfc90.dll
 0002:00000e0c       __imp_??0CImageList@@QAE@XZ 00482e0c     mfc90:mfc90.dll
 0002:00000e10       __imp_??1CWnd@@UAE@XZ      00482e10     mfc90:mfc90.dll
 0002:00000e14       __imp_??1CMonthCalCtrl@@UAE@XZ 00482e14     mfc90:mfc90.dll
 0002:00000e18       __imp_?Default@CWnd@@IAEJXZ 00482e18     mfc90:mfc90.dll
 0002:00000e1c       __imp_?GetSafeOwner@CWnd@@SGPAV1@PAV1@PAPAUHWND__@@@Z 00482e1c     mfc90:mfc90.dll
 0002:00000e20       __imp_?IsWindowEnabled@CWnd@@QBEHXZ 00482e20     mfc90:mfc90.dll
 0002:00000e24       __imp_?IsEmpty@?$CSimpleStringT@D$00@ATL@@QBE_NXZ 00482e24     mfc90:mfc90.dll
 0002:00000e28       __imp_?GetBuffer@?$CSimpleStringT@D$00@ATL@@QAEPADH@Z 00482e28     mfc90:mfc90.dll
 0002:00000e2c       __imp_?DDX_Check@@YGXPAVCDataExchange@@HAAH@Z 00482e2c     mfc90:mfc90.dll
 0002:00000e30       __imp_?GetRuntimeClass@CCriticalSection@@UBEPAUCRuntimeClass@@XZ 00482e30     mfc90:mfc90.dll
 0002:00000e34       __imp_??0CSyncObject@@QAE@PBD@Z 00482e34     mfc90:mfc90.dll
 0002:00000e38       __imp_?AfxThrowMemoryException@@YGXXZ 00482e38     mfc90:mfc90.dll
 0002:00000e3c       __imp_??1CSyncObject@@UAE@XZ 00482e3c     mfc90:mfc90.dll
 0002:00000e40       __imp_??0CPtrList@@QAE@H@Z 00482e40     mfc90:mfc90.dll
 0002:00000e44       __imp_?GetRuntimeClass@CPtrList@@UBEPAUCRuntimeClass@@XZ 00482e44     mfc90:mfc90.dll
 0002:00000e48       __imp_??1CPtrList@@UAE@XZ  00482e48     mfc90:mfc90.dll
 0002:00000e4c       __imp_??2@YAPAXI@Z         00482e4c     mfc90:mfc90.dll
 0002:00000e50       __imp_??_V@YAXPAX@Z        00482e50     mfc90:mfc90.dll
 0002:00000e54       __imp_??_U@YAPAXI@Z        00482e54     mfc90:mfc90.dll
 0002:00000e58       __imp_?GetThisClass@CObject@@SGPAUCRuntimeClass@@XZ 00482e58     mfc90:mfc90.dll
 0002:00000e5c       __imp_?ReportError@CException@@UAEHII@Z 00482e5c     mfc90:mfc90.dll
 0002:00000e60       __imp_?GetErrorMessage@CException@@UBEHPADIPAI@Z 00482e60     mfc90:mfc90.dll
 0002:00000e64       __imp_??0CException@@QAE@XZ 00482e64     mfc90:mfc90.dll
 0002:00000e68       __imp_?GetThisClass@CException@@SGPAUCRuntimeClass@@XZ 00482e68     mfc90:mfc90.dll
 0002:00000e6c       __imp_?InsertItem@CListCtrl@@QAEHIHPBDIIHJ@Z 00482e6c     mfc90:mfc90.dll
 0002:00000e70       __imp_?DrawItem@CListCtrl@@UAEXPAUtagDRAWITEMSTRUCT@@@Z 00482e70     mfc90:mfc90.dll
 0002:00000e74       __imp_?OnChildNotify@CListCtrl@@MAEHIIJPAJ@Z 00482e74     mfc90:mfc90.dll
 0002:00000e78       __imp_?GetMessageMap@CListCtrl@@MBEPBUAFX_MSGMAP@@XZ 00482e78     mfc90:mfc90.dll
 0002:00000e7c       __imp_?GetRuntimeClass@CListCtrl@@UBEPAUCRuntimeClass@@XZ 00482e7c     mfc90:mfc90.dll
 0002:00000e80       __imp_?SetItemState@CListCtrl@@QAEHHII@Z 00482e80     mfc90:mfc90.dll
 0002:00000e84       __imp_?SetFocus@CWnd@@QAEPAV1@XZ 00482e84     mfc90:mfc90.dll
 0002:00000e88       __imp_??1CListCtrl@@UAE@XZ 00482e88     mfc90:mfc90.dll
 0002:00000e8c       __imp_?MessageBoxA@CWnd@@QAEHPBD0I@Z 00482e8c     mfc90:mfc90.dll
 0002:00000e90       __imp_?GetItemText@CListCtrl@@QBE?AV?$CStringT@DV?$StrTraitMFC_DLL@DV?$ChTraitsCRT@D@ATL@@@@@ATL@@HH@Z 00482e90     mfc90:mfc90.dll
 0002:00000e94       __imp_?Format@?$CStringT@DV?$StrTraitMFC_DLL@DV?$ChTraitsCRT@D@ATL@@@@@ATL@@QAAXPBDZZ 00482e94     mfc90:mfc90.dll
 0002:00000e98       __imp_?InsertColumn@CListCtrl@@QAEHHPBDHHH@Z 00482e98     mfc90:mfc90.dll
 0002:00000e9c       __imp_?SetItemText@CListCtrl@@QAEHHHPBD@Z 00482e9c     mfc90:mfc90.dll
 0002:00000ea0       __imp_?DeleteItem@CComboBox@@UAEXPAUtagDELETEITEMSTRUCT@@@Z 00482ea0     mfc90:mfc90.dll
 0002:00000ea4       __imp_?CompareItem@CComboBox@@UAEHPAUtagCOMPAREITEMSTRUCT@@@Z 00482ea4     mfc90:mfc90.dll
 0002:00000ea8       __imp_?MeasureItem@CComboBox@@UAEXPAUtagMEASUREITEMSTRUCT@@@Z 00482ea8     mfc90:mfc90.dll
 0002:00000eac       __imp_?DrawItem@CComboBox@@UAEXPAUtagDRAWITEMSTRUCT@@@Z 00482eac     mfc90:mfc90.dll
 0002:00000eb0       __imp_?Create@CComboBox@@UAEHKABUtagRECT@@PAVCWnd@@I@Z 00482eb0     mfc90:mfc90.dll
 0002:00000eb4       __imp_?OnChildNotify@CComboBox@@MAEHIIJPAJ@Z 00482eb4     mfc90:mfc90.dll
 0002:00000eb8       __imp_?GetRuntimeClass@CComboBox@@UBEPAUCRuntimeClass@@XZ 00482eb8     mfc90:mfc90.dll
 0002:00000ebc       __imp_?AfxThrowInvalidArgException@@YGXXZ 00482ebc     mfc90:mfc90.dll
 0002:00000ec0       __imp_?GetNextAssoc@CMapStringToPtr@@QBEXAAPAU__POSITION@@AAV?$CStringT@DV?$StrTraitMFC_DLL@DV?$ChTraitsCRT@D@ATL@@@@@ATL@@AAPAX@Z 00482ec0     mfc90:mfc90.dll
 0002:00000ec4       __imp_?FindIndex@CStringList@@QBEPAU__POSITION@@H@Z 00482ec4     mfc90:mfc90.dll
 0002:00000ec8       __imp_??0CStringList@@QAE@H@Z 00482ec8     mfc90:mfc90.dll
 0002:00000ecc       __imp_?AddTail@CStringList@@QAEPAU__POSITION@@ABV?$CStringT@DV?$StrTraitMFC_DLL@DV?$ChTraitsCRT@D@ATL@@@@@ATL@@@Z 00482ecc     mfc90:mfc90.dll
 0002:00000ed0       __imp_??1CStringList@@UAE@XZ 00482ed0     mfc90:mfc90.dll
 0002:00000ed4       __imp_?DDX_CBString@@YGXPAVCDataExchange@@HAAV?$CStringT@DV?$StrTraitMFC_DLL@DV?$ChTraitsCRT@D@ATL@@@@@ATL@@@Z 00482ed4     mfc90:mfc90.dll
 0002:00000ed8       __imp_?GetRuntimeClass@CDialog@@UBEPAUCRuntimeClass@@XZ 00482ed8     mfc90:mfc90.dll
 0002:00000edc       __imp_??1CComboBox@@UAE@XZ 00482edc     mfc90:mfc90.dll
 0002:00000ee0       __imp_?GetManager@?$CStringT@DV?$StrTraitMFC_DLL@DV?$ChTraitsCRT@D@ATL@@@@@ATL@@QBEPAUIAtlStringMgr@2@XZ 00482ee0     mfc90:mfc90.dll
 0002:00000ee4       __imp_??0?$CStringT@DV?$StrTraitMFC_DLL@DV?$ChTraitsCRT@D@ATL@@@@@ATL@@QAE@PAUIAtlStringMgr@1@@Z 00482ee4     mfc90:mfc90.dll
 0002:00000ee8       __imp_?StringLength@?$CSimpleStringT@D$00@ATL@@SAHPBD@Z 00482ee8     mfc90:mfc90.dll
 0002:00000eec       __imp_?Concatenate@?$CSimpleStringT@D$00@ATL@@KAXAAV12@PBDH1H@Z 00482eec     mfc90:mfc90.dll
 0002:00000ef0       __imp_?DrawItem@CStatic@@UAEXPAUtagDRAWITEMSTRUCT@@@Z 00482ef0     mfc90:mfc90.dll
 0002:00000ef4       __imp_?Create@CStatic@@UAEHPBDKABUtagRECT@@PAVCWnd@@I@Z 00482ef4     mfc90:mfc90.dll
 0002:00000ef8       __imp_?GetOccDialogInfo@CWnd@@MAEPAU_AFX_OCC_DIALOG_INFO@@XZ 00482ef8     mfc90:mfc90.dll
 0002:00000efc       __imp_?SetOccDialogInfo@CWnd@@MAEHPAU_AFX_OCC_DIALOG_INFO@@@Z 00482efc     mfc90:mfc90.dll
 0002:00000f00       __imp_?CheckAutoCenter@CWnd@@UAEHXZ 00482f00     mfc90:mfc90.dll
 0002:00000f04       __imp_?OnChildNotify@CStatic@@MAEHIIJPAJ@Z 00482f04     mfc90:mfc90.dll
 0002:00000f08       __imp_?PreTranslateMessage@CWnd@@UAEHPAUtagMSG@@@Z 00482f08     mfc90:mfc90.dll
 0002:00000f0c       __imp_?GetMessageMap@CWnd@@MBEPBUAFX_MSGMAP@@XZ 00482f0c     mfc90:mfc90.dll
 0002:00000f10       __imp_?OnCmdMsg@CCmdTarget@@UAEHIHPAXPAUAFX_CMDHANDLERINFO@@@Z 00482f10     mfc90:mfc90.dll
 0002:00000f14       __imp_?GetRuntimeClass@CStatic@@UBEPAUCRuntimeClass@@XZ 00482f14     mfc90:mfc90.dll
 0002:00000f18       __imp_??0CWnd@@QAE@XZ      00482f18     mfc90:mfc90.dll
 0002:00000f1c       __imp_?AfxMessageBox@@YGHPBDII@Z 00482f1c     mfc90:mfc90.dll
 0002:00000f20       __imp_?EnableWindow@CWnd@@QAEHH@Z 00482f20     mfc90:mfc90.dll
 0002:00000f24       __imp_?OnInitDialog@CDialog@@UAEHXZ 00482f24     mfc90:mfc90.dll
 0002:00000f28       __imp_??0?$CStringT@DV?$StrTraitMFC_DLL@DV?$ChTraitsCRT@D@ATL@@@@@ATL@@QAE@XZ 00482f28     mfc90:mfc90.dll
 0002:00000f2c       __imp_??4?$CStringT@DV?$StrTraitMFC_DLL@DV?$ChTraitsCRT@D@ATL@@@@@ATL@@QAEAAV01@PBD@Z 00482f2c     mfc90:mfc90.dll
 0002:00000f30       __imp_?Right@?$CStringT@DV?$StrTraitMFC_DLL@DV?$ChTraitsCRT@D@ATL@@@@@ATL@@QBE?AV12@H@Z 00482f30     mfc90:mfc90.dll
 0002:00000f34       __imp_??4?$CStringT@DV?$StrTraitMFC_DLL@DV?$ChTraitsCRT@D@ATL@@@@@ATL@@QAEAAV01@ABV01@@Z 00482f34     mfc90:mfc90.dll
 0002:00000f38       __imp_??0?$CStringT@DV?$StrTraitMFC_DLL@DV?$ChTraitsCRT@D@ATL@@@@@ATL@@QAE@ABV01@@Z 00482f38     mfc90:mfc90.dll
 0002:00000f3c       __imp_?GetLength@?$CSimpleStringT@D$00@ATL@@QBEHXZ 00482f3c     mfc90:mfc90.dll
 0002:00000f40       __imp_?Insert@?$CStringT@DV?$StrTraitMFC_DLL@DV?$ChTraitsCRT@D@ATL@@@@@ATL@@QAEHHPBD@Z 00482f40     mfc90:mfc90.dll
 0002:00000f44       __imp_??B?$CSimpleStringT@D$00@ATL@@QBEPBDXZ 00482f44     mfc90:mfc90.dll
 0002:00000f48       __imp_?SetWindowTextA@CWnd@@QAEXPBD@Z 00482f48     mfc90:mfc90.dll
 0002:00000f4c       __imp_?Compare@?$CStringT@DV?$StrTraitMFC_DLL@DV?$ChTraitsCRT@D@ATL@@@@@ATL@@QBEHPBD@Z 00482f4c     mfc90:mfc90.dll
 0002:00000f50       __imp_?GetDlgItem@CWnd@@QBEPAV1@H@Z 00482f50     mfc90:mfc90.dll
 0002:00000f54       __imp_?ShowWindow@CWnd@@QAEHH@Z 00482f54     mfc90:mfc90.dll
 0002:00000f58       __imp_?ReverseFind@?$CStringT@DV?$StrTraitMFC_DLL@DV?$ChTraitsCRT@D@ATL@@@@@ATL@@QBEHD@Z 00482f58     mfc90:mfc90.dll
 0002:00000f5c       __imp_?Delete@?$CStringT@DV?$StrTraitMFC_DLL@DV?$ChTraitsCRT@D@ATL@@@@@ATL@@QAEHHH@Z 00482f5c     mfc90:mfc90.dll
 0002:00000f60       __imp_?UpdateData@CWnd@@QAEHH@Z 00482f60     mfc90:mfc90.dll
 0002:00000f64       __imp_?GetThisMessageMap@CDialog@@KGPBUAFX_MSGMAP@@XZ 00482f64     mfc90:mfc90.dll
 0002:00000f68       __imp_?DDX_Control@@YGXPAVCDataExchange@@HAAVCWnd@@@Z 00482f68     mfc90:mfc90.dll
 0002:00000f6c       __imp_?DDX_Text@@YGXPAVCDataExchange@@HAAV?$CStringT@DV?$StrTraitMFC_DLL@DV?$ChTraitsCRT@D@ATL@@@@@ATL@@@Z 00482f6c     mfc90:mfc90.dll
 0002:00000f70       __imp_??1?$CStringT@DV?$StrTraitMFC_DLL@DV?$ChTraitsCRT@D@ATL@@@@@ATL@@QAE@XZ 00482f70     mfc90:mfc90.dll
 0002:00000f74       __imp_?PreInitDialog@CDialog@@MAEXXZ 00482f74     mfc90:mfc90.dll
 0002:00000f78       __imp_?OnCancel@CDialog@@MAEXXZ 00482f78     mfc90:mfc90.dll
 0002:00000f7c       __imp_?AddToRecentFileList@CWinApp@@UAEXPBD@Z 00482f7c     mfc90:mfc90.dll
 0002:00000f80       __imp_?OpenDocumentFile@CWinApp@@UAEPAVCDocument@@PBD@Z 00482f80     mfc90:mfc90.dll
 0002:00000f84       __imp_?Unregister@CWinApp@@UAEHXZ 00482f84     mfc90:mfc90.dll
 0002:00000f88       __imp_?Register@CWinApp@@UAEHXZ 00482f88     mfc90:mfc90.dll
 0002:00000f8c       __imp_?InitLibId@CWinApp@@UAEXXZ 00482f8c     mfc90:mfc90.dll
 0002:00000f90       __imp_?Delete@CWinThread@@UAEXXZ 00482f90     mfc90:mfc90.dll
 0002:00000f94       __imp_?GetMainWnd@CWinThread@@UAEPAVCWnd@@XZ 00482f94     mfc90:mfc90.dll
 0002:00000f98       __imp_?ProcessMessageFilter@CWinThread@@UAEHHPAUtagMSG@@@Z 00482f98     mfc90:mfc90.dll
 0002:00000f9c       __imp_?ProcessWndProcException@CWinApp@@UAEJPAVCException@@PBUtagMSG@@@Z 00482f9c     mfc90:mfc90.dll
 0002:00000fa0       __imp_?IsIdleMessage@CWinThread@@UAEHPAUtagMSG@@@Z 00482fa0     mfc90:mfc90.dll
 0002:00000fa4       __imp_?OnIdle@CWinApp@@UAEHJ@Z 00482fa4     mfc90:mfc90.dll
 0002:00000fa8       __imp_?PumpMessage@CWinThread@@UAEHXZ 00482fa8     mfc90:mfc90.dll
 0002:00000fac       __imp_?PreTranslateMessage@CWinThread@@UAEHPAUtagMSG@@@Z 00482fac     mfc90:mfc90.dll
 0002:00000fb0       __imp_?Run@CWinApp@@UAEHXZ 00482fb0     mfc90:mfc90.dll
 0002:00000fb4       __imp_?GetInterfaceMap@CCmdTarget@@MBEPBUAFX_INTERFACEMAP@@XZ 00482fb4     mfc90:mfc90.dll
 0002:00000fb8       __imp_?OnFinalRelease@CCmdTarget@@UAEXXZ 00482fb8     mfc90:mfc90.dll
 0002:00000fbc       __imp_?GetRuntimeClass@CWinAppEx@@UBEPAUCRuntimeClass@@XZ 00482fbc     mfc90:mfc90.dll
 0002:00000fc0       __imp_??0CWinAppEx@@QAE@H@Z 00482fc0     mfc90:mfc90.dll
 0002:00000fc4       __imp_?OnFileOpen@CWinApp@@IAEXXZ 00482fc4     mfc90:mfc90.dll
 0002:00000fc8       __imp_?OnFileNew@CWinApp@@IAEXXZ 00482fc8     mfc90:mfc90.dll
 0002:00000fcc       __imp_?GetThisMessageMap@CWinApp@@KGPBUAFX_MSGMAP@@XZ 00482fcc     mfc90:mfc90.dll
 0002:00000fd0       __imp_?GetNextAssoc@CMapPtrToPtr@@QBEXAAPAU__POSITION@@AAPAX1@Z 00482fd0     mfc90:mfc90.dll
 0002:00000fd4       __imp_?RemoveKey@CMapPtrToPtr@@QAEHPAX@Z 00482fd4     mfc90:mfc90.dll
 0002:00000fd8       __imp_??ACMapPtrToPtr@@QAEAAPAXPAX@Z 00482fd8     mfc90:mfc90.dll
 0002:00000fdc       __imp_?Lookup@CMapPtrToPtr@@QBEHPAXAAPAX@Z 00482fdc     mfc90:mfc90.dll
 0002:00000fe0       __imp_?GetRuntimeClass@CMapPtrToPtr@@UBEPAUCRuntimeClass@@XZ 00482fe0     mfc90:mfc90.dll
 0002:00000fe4       __imp_??0CMapPtrToPtr@@QAE@H@Z 00482fe4     mfc90:mfc90.dll
 0002:00000fe8       __imp_??1CMapPtrToPtr@@UAE@XZ 00482fe8     mfc90:mfc90.dll
 0002:00000fec       __imp_?RemoveAll@CMapPtrToPtr@@QAEXXZ 00482fec     mfc90:mfc90.dll
 0002:00000ff0       __imp_?GetMessageMap@CTreeCtrl@@MBEPBUAFX_MSGMAP@@XZ 00482ff0     mfc90:mfc90.dll
 0002:00000ff4       __imp_?Attach@CMenu@@QAEHPAUHMENU__@@@Z 00482ff4     mfc90:mfc90.dll
 0002:00000ff8       __imp_?FromHandle@CMenu@@SGPAV1@PAUHMENU__@@@Z 00482ff8     mfc90:mfc90.dll
 0002:00000ffc       __imp_?DestroyMenu@CMenu@@QAEHXZ 00482ffc     mfc90:mfc90.dll
 0002:00001000       __imp_?MeasureItem@CMenu@@UAEXPAUtagMEASUREITEMSTRUCT@@@Z 00483000     mfc90:mfc90.dll
 0002:00001004       __imp_?DrawItem@CMenu@@UAEXPAUtagDRAWITEMSTRUCT@@@Z 00483004     mfc90:mfc90.dll
 0002:00001008       __imp_?GetRuntimeClass@CMenu@@UBEPAUCRuntimeClass@@XZ 00483008     mfc90:mfc90.dll
 0002:0000100c       __imp_?AfxGetThread@@YGPAVCWinThread@@XZ 0048300c     mfc90:mfc90.dll
 0002:00001010       __imp_?Mid@?$CStringT@DV?$StrTraitMFC_DLL@DV?$ChTraitsCRT@D@ATL@@@@@ATL@@QBE?AV12@H@Z 00483010     mfc90:mfc90.dll
 0002:00001014       __imp_?GetItemRect@CTreeCtrl@@QBEHPAU_TREEITEM@@PAUtagRECT@@H@Z 00483014     mfc90:mfc90.dll
 0002:00001018       __imp_?Create@CEdit@@QAEHKABUtagRECT@@PAVCWnd@@I@Z 00483018     mfc90:mfc90.dll
 0002:0000101c       __imp_?ClientToScreen@CWnd@@QBEXPAUtagRECT@@@Z 0048301c     mfc90:mfc90.dll
 0002:00001020       __imp_?GetThisClass@CFrameWndEx@@SGPAUCRuntimeClass@@XZ 00483020     mfc90:mfc90.dll
 0002:00001024       __imp_?IsKindOf@CObject@@QBEHPBUCRuntimeClass@@@Z 00483024     mfc90:mfc90.dll
 0002:00001028       __imp_??0CMFCPopupMenu@@QAE@XZ 00483028     mfc90:mfc90.dll
 0002:0000102c       __imp_?UpdateDialogControls@CWnd@@QAEXPAVCCmdTarget@@H@Z 0048302c     mfc90:mfc90.dll
 0002:00001030       __imp_?HitTest@CTreeCtrl@@QBEPAU_TREEITEM@@VCPoint@@PAI@Z 00483030     mfc90:mfc90.dll
 0002:00001034       __imp_?GetItemText@CTreeCtrl@@QBE?AV?$CStringT@DV?$StrTraitMFC_DLL@DV?$ChTraitsCRT@D@ATL@@@@@ATL@@PAU_TREEITEM@@@Z 00483034     mfc90:mfc90.dll
 0002:00001038       __imp_?GetThisMessageMap@CTreeCtrl@@KGPBUAFX_MSGMAP@@XZ 00483038     mfc90:mfc90.dll
 0002:0000103c       __imp_??1CTreeCtrl@@UAE@XZ 0048303c     mfc90:mfc90.dll
 0002:00001040       __imp_?GetRuntimeClass@CTreeCtrl@@UBEPAUCRuntimeClass@@XZ 00483040     mfc90:mfc90.dll
 0002:00001044       __imp_?SetAt@?$CSimpleStringT@D$00@ATL@@QAEXHD@Z 00483044     mfc90:mfc90.dll
 0002:00001048       __imp_?WriteString@CStdioFile@@UAEXPBD@Z 00483048     mfc90:mfc90.dll
 0002:0000104c       __imp_??0CFile@@QAE@PBDI@Z 0048304c     mfc90:mfc90.dll
 0002:00001050       __imp_?GetRuntimeClass@CFont@@UBEPAUCRuntimeClass@@XZ 00483050     mfc90:mfc90.dll
 0002:00001054       __imp_?GetWindowTextA@CWnd@@QBEXAAV?$CStringT@DV?$StrTraitMFC_DLL@DV?$ChTraitsCRT@D@ATL@@@@@ATL@@@Z 00483054     mfc90:mfc90.dll
 0002:00001058       __imp_?Detach@CGdiObject@@QAEPAXXZ 00483058     mfc90:mfc90.dll
 0002:0000105c       __imp_?ModifyStyle@CWnd@@QAEHKKI@Z 0048305c     mfc90:mfc90.dll
 0002:00001060       __imp_?GetAt@?$CSimpleStringT@D$00@ATL@@QBEDH@Z 00483060     mfc90:mfc90.dll
 0002:00001064       __imp_?Remove@?$CStringT@DV?$StrTraitMFC_DLL@DV?$ChTraitsCRT@D@ATL@@@@@ATL@@QAEHD@Z 00483064     mfc90:mfc90.dll
 0002:00001068       __imp_??Y?$CStringT@DV?$StrTraitMFC_DLL@DV?$ChTraitsCRT@D@ATL@@@@@ATL@@QAEAAV01@D@Z 00483068     mfc90:mfc90.dll
 0002:0000106c       __imp_??0CFileDialog@@QAE@HPBD0K0PAVCWnd@@KH@Z 0048306c     mfc90:mfc90.dll
 0002:00001070       __imp_?DoModal@CFileDialog@@UAEHXZ 00483070     mfc90:mfc90.dll
 0002:00001074       __imp_?GetPathName@CFileDialog@@QBE?AV?$CStringT@DV?$StrTraitMFC_DLL@DV?$ChTraitsCRT@D@ATL@@@@@ATL@@XZ 00483074     mfc90:mfc90.dll
 0002:00001078       __imp_??1CFileDialog@@UAE@XZ 00483078     mfc90:mfc90.dll
 0002:0000107c       __imp_?Replace@?$CStringT@DV?$StrTraitMFC_DLL@DV?$ChTraitsCRT@D@ATL@@@@@ATL@@QAEHDD@Z 0048307c     mfc90:mfc90.dll
 0002:00001080       __imp_??Y?$CStringT@DV?$StrTraitMFC_DLL@DV?$ChTraitsCRT@D@ATL@@@@@ATL@@QAEAAV01@ABV?$CSimpleStringT@D$00@1@@Z 00483080     mfc90:mfc90.dll
 0002:00001084       __imp_??Y?$CStringT@DV?$StrTraitMFC_DLL@DV?$ChTraitsCRT@D@ATL@@@@@ATL@@QAEAAV01@PBD@Z 00483084     mfc90:mfc90.dll
 0002:00001088       __imp_?Left@?$CStringT@DV?$StrTraitMFC_DLL@DV?$ChTraitsCRT@D@ATL@@@@@ATL@@QBE?AV12@H@Z 00483088     mfc90:mfc90.dll
 0002:0000108c       __imp_?DrawItem@CButton@@UAEXPAUtagDRAWITEMSTRUCT@@@Z 0048308c     mfc90:mfc90.dll
 0002:00001090       __imp_?Create@CButton@@UAEHPBDKABUtagRECT@@PAVCWnd@@I@Z 00483090     mfc90:mfc90.dll
 0002:00001094       __imp_?OnChildNotify@CButton@@MAEHIIJPAJ@Z 00483094     mfc90:mfc90.dll
 0002:00001098       __imp_?GetRuntimeClass@CButton@@UBEPAUCRuntimeClass@@XZ 00483098     mfc90:mfc90.dll
 0002:0000109c       __imp_??1CButton@@UAE@XZ   0048309c     mfc90:mfc90.dll
 0002:000010a0       __imp_?CreateEx@CSpinButtonCtrl@@UAEHKKABUtagRECT@@PAVCWnd@@I@Z 004830a0     mfc90:mfc90.dll
 0002:000010a4       __imp_?Create@CSpinButtonCtrl@@UAEHKABUtagRECT@@PAVCWnd@@I@Z 004830a4     mfc90:mfc90.dll
 0002:000010a8       __imp_?GetRuntimeClass@CSpinButtonCtrl@@UBEPAUCRuntimeClass@@XZ 004830a8     mfc90:mfc90.dll
 0002:000010ac       __imp_??A?$CSimpleStringT@D$00@ATL@@QBEDH@Z 004830ac     mfc90:mfc90.dll
 0002:000010b0       __imp_?GetLBText@CComboBox@@QBEXHAAV?$CStringT@DV?$StrTraitMFC_DLL@DV?$ChTraitsCRT@D@ATL@@@@@ATL@@@Z 004830b0     mfc90:mfc90.dll
 0002:000010b4       __imp_?RemoveAll@CPtrList@@QAEXXZ 004830b4     mfc90:mfc90.dll
 0002:000010b8       __imp_??1CSpinButtonCtrl@@UAE@XZ 004830b8     mfc90:mfc90.dll
 0002:000010bc       __imp_?get_accChild@CWnd@@UAEJUtagVARIANT@@PAPAUIDispatch@@@Z 004830bc     mfc90:mfc90.dll
 0002:000010c0       __imp_?get_accChildCount@CWnd@@UAEJPAJ@Z 004830c0     mfc90:mfc90.dll
 0002:000010c4       __imp_?get_accParent@CWnd@@UAEJPAPAUIDispatch@@@Z 004830c4     mfc90:mfc90.dll
 0002:000010c8       __imp_?EnsureStdObj@CWnd@@UAEJXZ 004830c8     mfc90:mfc90.dll
 0002:000010cc       __imp_?EndModalLoop@CWnd@@UAEXH@Z 004830cc     mfc90:mfc90.dll
 0002:000010d0       __imp_?ContinueModal@CWnd@@UAEHXZ 004830d0     mfc90:mfc90.dll
 0002:000010d4       __imp_?WinHelpInternal@CWnd@@UAEXKI@Z 004830d4     mfc90:mfc90.dll
 0002:000010d8       __imp_?HtmlHelpA@CWnd@@UAEXKI@Z 004830d8     mfc90:mfc90.dll
 0002:000010dc       __imp_?WinHelpA@CWnd@@UAEXKI@Z 004830dc     mfc90:mfc90.dll
 0002:000010e0       __imp_?GetScrollBarCtrl@CWnd@@UBEPAVCScrollBar@@H@Z 004830e0     mfc90:mfc90.dll
 0002:000010e4       __imp_?OnToolHitTest@CWnd@@UBEHVCPoint@@PAUtagTOOLINFOA@@@Z 004830e4     mfc90:mfc90.dll
 0002:000010e8       __imp_?SetMenu@CWnd@@UAEHPAVCMenu@@@Z 004830e8     mfc90:mfc90.dll
 0002:000010ec       __imp_?GetMenu@CWnd@@UBEPAVCMenu@@XZ 004830ec     mfc90:mfc90.dll
 0002:000010f0       __imp_?CalcWindowRect@CWnd@@UAEXPAUtagRECT@@I@Z 004830f0     mfc90:mfc90.dll
 0002:000010f4       __imp_?PreCreateWindow@CWnd@@UAEHAAUtagCREATESTRUCTA@@@Z 004830f4     mfc90:mfc90.dll
 0002:000010f8       __imp_?DestroyWindow@CWnd@@UAEHXZ 004830f8     mfc90:mfc90.dll
 0002:000010fc       __imp_?CreateEx@CWnd@@UAEHKPBD0KHHHHPAUHWND__@@PAUHMENU__@@PAX@Z 004830fc     mfc90:mfc90.dll
 0002:00001100       __imp_?CreateEx@CWnd@@UAEHKPBD0KABUtagRECT@@PAV1@IPAX@Z 00483100     mfc90:mfc90.dll
 0002:00001104       __imp_?Create@CWnd@@UAEHPBD0KABUtagRECT@@PAV1@IPAUCCreateContext@@@Z 00483104     mfc90:mfc90.dll
 0002:00001108       __imp_?PreSubclassWindow@CWnd@@UAEXXZ 00483108     mfc90:mfc90.dll
 0002:0000110c       __imp_?GetConnectionHook@CCmdTarget@@MAEPAUIConnectionPoint@@ABU_GUID@@@Z 0048310c     mfc90:mfc90.dll
 0002:00001110       __imp_?GetExtraConnectionPoints@CCmdTarget@@MAEHPAVCPtrArray@@@Z 00483110     mfc90:mfc90.dll
 0002:00001114       __imp_?GetInterfaceHook@CCmdTarget@@UAEPAUIUnknown@@PBX@Z 00483114     mfc90:mfc90.dll
 0002:00001118       __imp_?OnCreateAggregates@CCmdTarget@@UAEHXZ 00483118     mfc90:mfc90.dll
 0002:0000111c       __imp_?GetEventSinkMap@CCmdTarget@@MBEPBUAFX_EVENTSINKMAP@@XZ 0048311c     mfc90:mfc90.dll
 0002:00001120       __imp_?GetInterfaceMap@CWnd@@MBEPBUAFX_INTERFACEMAP@@XZ 00483120     mfc90:mfc90.dll
 0002:00001124       __imp_?GetConnectionMap@CCmdTarget@@MBEPBUAFX_CONNECTIONMAP@@XZ 00483124     mfc90:mfc90.dll
 0002:00001128       __imp_?GetDispatchMap@CCmdTarget@@MBEPBUAFX_DISPMAP@@XZ 00483128     mfc90:mfc90.dll
 0002:0000112c       __imp_?GetCommandMap@CCmdTarget@@MBEPBUAFX_OLECMDMAP@@XZ 0048312c     mfc90:mfc90.dll
 0002:00001130       __imp_?GetTypeLib@CCmdTarget@@UAEJKPAPAUITypeLib@@@Z 00483130     mfc90:mfc90.dll
 0002:00001134       __imp_?GetTypeLibCache@CCmdTarget@@UAEPAVCTypeLibCache@@XZ 00483134     mfc90:mfc90.dll
 0002:00001138       __imp_?GetTypeInfoCount@CCmdTarget@@UAEIXZ 00483138     mfc90:mfc90.dll
 0002:0000113c       __imp_?GetDispatchIID@CCmdTarget@@UAEHPAU_GUID@@@Z 0048313c     mfc90:mfc90.dll
 0002:00001140       __imp_?IsInvokeAllowed@CCmdTarget@@UAEHJ@Z 00483140     mfc90:mfc90.dll
 0002:00001144       __imp_?OnFinalRelease@CWnd@@UAEXXZ 00483144     mfc90:mfc90.dll
 0002:00001148       __imp_?OnCmdMsg@CDialog@@UAEHIHPAXPAUAFX_CMDHANDLERINFO@@@Z 00483148     mfc90:mfc90.dll
 0002:0000114c       __imp_??0CDialog@@QAE@IPAVCWnd@@@Z 0048314c     mfc90:mfc90.dll
 0002:00001150       __imp_??0?$CStringT@DV?$StrTraitMFC_DLL@DV?$ChTraitsCRT@D@ATL@@@@@ATL@@QAE@PBD@Z 00483150     mfc90:mfc90.dll
 0002:00001154       __imp_??1CDialog@@UAE@XZ   00483154     mfc90:mfc90.dll
 0002:00001158       __imp_??1CStatic@@UAE@XZ   00483158     mfc90:mfc90.dll
 0002:0000115c       __imp_?GetThisClass@CDialog@@SGPAUCRuntimeClass@@XZ 0048315c     mfc90:mfc90.dll
 0002:00001160       __imp_??3@YAXPAX@Z         00483160     mfc90:mfc90.dll
 0002:00001164       __imp_?Close@CFileFind@@QAEXXZ 00483164     mfc90:mfc90.dll
 0002:00001168       __imp_??1CFileFind@@UAE@XZ 00483168     mfc90:mfc90.dll
 0002:0000116c       __imp_?GetContextMenuManager@CWinAppEx@@QAEPAVCContextMenuManager@@XZ 0048316c     mfc90:mfc90.dll
 0002:00001170       __imp_?OnCmdMsg@CView@@UAEHIHPAXPAUAFX_CMDHANDLERINFO@@@Z 00483170     mfc90:mfc90.dll
 0002:00001174       __imp_??0CFormView@@IAE@I@Z 00483174     mfc90:mfc90.dll
 0002:00001178       __imp_??1CFormView@@UAE@XZ 00483178     mfc90:mfc90.dll
 0002:0000117c       __imp_?GetThisMessageMap@CFormView@@KGPBUAFX_MSGMAP@@XZ 0048317c     mfc90:mfc90.dll
 0002:00001180       __imp_?SetItem@CTreeCtrl@@QAEHPAU_TREEITEM@@IPBDHHIIJ@Z 00483180     mfc90:mfc90.dll
 0002:00001184       __imp_?InsertItem@CTreeCtrl@@QAEPAU_TREEITEM@@IPBDHHIIJPAU2@1@Z 00483184     mfc90:mfc90.dll
 0002:00001188       __imp_?RemoveKey@CMapStringToPtr@@QAEHPBD@Z 00483188     mfc90:mfc90.dll
 0002:0000118c       __imp_??ACMapStringToPtr@@QAEAAPAXPBD@Z 0048318c     mfc90:mfc90.dll
 0002:00001190       __imp_?Lookup@CMapStringToPtr@@QBEHPBDAAPAX@Z 00483190     mfc90:mfc90.dll
 0002:00001194       __imp_?GetRuntimeClass@CMapStringToPtr@@UBEPAUCRuntimeClass@@XZ 00483194     mfc90:mfc90.dll
 0002:00001198       __imp_?InitHashTable@CMapStringToPtr@@QAEXIH@Z 00483198     mfc90:mfc90.dll
 0002:0000119c       __imp_?RemoveAll@CMapStringToPtr@@QAEXXZ 0048319c     mfc90:mfc90.dll
 0002:000011a0       __imp_??1CMapStringToPtr@@UAE@XZ 004831a0     mfc90:mfc90.dll
 0002:000011a4       __imp_?OnOK@CDialog@@MAEXXZ 004831a4     mfc90:mfc90.dll
 0002:000011a8       __imp_?OnSetFont@CDialog@@UAEXPAVCFont@@@Z 004831a8     mfc90:mfc90.dll
 0002:000011ac       __imp_?DoModal@CDialog@@UAEHXZ 004831ac     mfc90:mfc90.dll
 0002:000011b0       __imp_?CreateIndirect@CDialog@@UAEHPBUDLGTEMPLATE@@PAVCWnd@@PAX@Z 004831b0     mfc90:mfc90.dll
 0002:000011b4       __imp_?CreateIndirect@CDialog@@UAEHPAXPAVCWnd@@@Z 004831b4     mfc90:mfc90.dll
 0002:000011b8       __imp_?Create@CDialog@@UAEHPBDPAVCWnd@@@Z 004831b8     mfc90:mfc90.dll
 0002:000011bc       __imp_?GetOccDialogInfo@CDialog@@MAEPAU_AFX_OCC_DIALOG_INFO@@XZ 004831bc     mfc90:mfc90.dll
 0002:000011c0       __imp_?SetOccDialogInfo@CDialog@@MAEHPAU_AFX_OCC_DIALOG_INFO@@@Z 004831c0     mfc90:mfc90.dll
 0002:000011c4       __imp_?CreateControlSite@CWnd@@MAEHPAVCOleControlContainer@@PAPAVCOleControlSite@@IABU_GUID@@@Z 004831c4     mfc90:mfc90.dll
 0002:000011c8       __imp_?CreateControlContainer@CWnd@@MAEHPAPAVCOleControlContainer@@@Z 004831c8     mfc90:mfc90.dll
 0002:000011cc       __imp_?IsFrameWnd@CWnd@@UBEHXZ 004831cc     mfc90:mfc90.dll
 0002:000011d0       __imp_?CheckAutoCenter@CDialog@@UAEHXZ 004831d0     mfc90:mfc90.dll
 0002:000011d4       __imp_?OnChildNotify@CWnd@@MAEHIIJPAJ@Z 004831d4     mfc90:mfc90.dll
 0002:000011d8       __imp_?GetThisClass@CFormView@@SGPAUCRuntimeClass@@XZ 004831d8     mfc90:mfc90.dll
 0002:000011dc       __imp_?OnNewDocument@CDocument@@UAEHXZ 004831dc     mfc90:mfc90.dll
 0002:000011e0       __imp_??1CDocument@@UAE@XZ 004831e0     mfc90:mfc90.dll
 0002:000011e4       __imp_?OnIdle@CDocument@@UAEXXZ 004831e4     mfc90:mfc90.dll
 0002:000011e8       __imp_?GetDefaultAccelerator@CDocument@@UAEPAUHACCEL__@@XZ 004831e8     mfc90:mfc90.dll
 0002:000011ec       __imp_?GetDefaultMenu@CDocument@@UAEPAUHMENU__@@XZ 004831ec     mfc90:mfc90.dll
 0002:000011f0       __imp_?UpdateFrameCounts@CDocument@@UAEXXZ 004831f0     mfc90:mfc90.dll
 0002:000011f4       __imp_?DoFileSave@CDocument@@UAEHXZ 004831f4     mfc90:mfc90.dll
 0002:000011f8       __imp_?DoSave@CDocument@@UAEHPBDH@Z 004831f8     mfc90:mfc90.dll
 0002:000011fc       __imp_?PreCloseFrame@CDocument@@UAEXPAVCFrameWnd@@@Z 004831fc     mfc90:mfc90.dll
 0002:00001200       __imp_?SaveModified@CDocument@@UAEHXZ 00483200     mfc90:mfc90.dll
 0002:00001204       __imp_?CanCloseFrame@CDocument@@UAEHPAVCFrameWnd@@@Z 00483204     mfc90:mfc90.dll
 0002:00001208       __imp_?ReleaseFile@CDocument@@UAEXPAVCFile@@H@Z 00483208     mfc90:mfc90.dll
 0002:0000120c       __imp_?GetFile@CDocument@@UAEPAVCFile@@PBDIPAVCFileException@@@Z 0048320c     mfc90:mfc90.dll
 0002:00001210       __imp_?ReportSaveLoadException@CDocument@@UAEXPBDPAVCException@@HI@Z 00483210     mfc90:mfc90.dll
 0002:00001214       __imp_?OnCloseDocument@CDocument@@UAEXXZ 00483214     mfc90:mfc90.dll
 0002:00001218       __imp_?OnSaveDocument@CDocument@@UAEHPBD@Z 00483218     mfc90:mfc90.dll
 0002:0000121c       __imp_?OnOpenDocument@CDocument@@UAEHPBD@Z 0048321c     mfc90:mfc90.dll
 0002:00001220       __imp_?DeleteContents@CDocument@@UAEXXZ 00483220     mfc90:mfc90.dll
 0002:00001224       __imp_?OnChangedViewList@CDocument@@UAEXXZ 00483224     mfc90:mfc90.dll
 0002:00001228       __imp_?GetNextView@CDocument@@UBEPAVCView@@AAPAU__POSITION@@@Z 00483228     mfc90:mfc90.dll
 0002:0000122c       __imp_?GetFirstViewPosition@CDocument@@UBEPAU__POSITION@@XZ 0048322c     mfc90:mfc90.dll
 0002:00001230       __imp_?SetPathName@CDocument@@UAEXPBDH@Z 00483230     mfc90:mfc90.dll
 0002:00001234       __imp_?SetTitle@CDocument@@UAEXPBD@Z 00483234     mfc90:mfc90.dll
 0002:00001238       __imp_?OnFinalRelease@CDocument@@UAEXXZ 00483238     mfc90:mfc90.dll
 0002:0000123c       __imp_?OnCmdMsg@CDocument@@UAEHIHPAXPAUAFX_CMDHANDLERINFO@@@Z 0048323c     mfc90:mfc90.dll
 0002:00001240       __imp_??0CDocument@@QAE@XZ 00483240     mfc90:mfc90.dll
 0002:00001244       __imp_?GetThisMessageMap@CDocument@@KGPBUAFX_MSGMAP@@XZ 00483244     mfc90:mfc90.dll
 0002:00001248       __imp_?GetThisClass@CDocument@@SGPAUCRuntimeClass@@XZ 00483248     mfc90:mfc90.dll
 0002:0000124c       __imp_?FromHandle@CWnd@@SGPAV1@PAUHWND__@@@Z 0048324c     mfc90:mfc90.dll
 0002:00001250       __imp_?SetLook@CMFCPropertySheet@@QAEXW4PropSheetLook@1@H@Z 00483250     mfc90:mfc90.dll
 0002:00001254       __imp_??0CFileFind@@QAE@XZ 00483254     mfc90:mfc90.dll
 0002:00001258       __imp_?PostNcDestroy@CWnd@@MAEXXZ 00483258     mfc90:mfc90.dll
 0002:0000125c       __imp_?DefWindowProcA@CWnd@@MAEJIIJ@Z 0048325c     mfc90:mfc90.dll
 0002:00001260       __imp_?OnWndMsg@CWnd@@MAEHIIJPAJ@Z 00483260     mfc90:mfc90.dll
 0002:00001264       __imp_?WindowProc@CWnd@@MAEJIIJ@Z 00483264     mfc90:mfc90.dll
 0002:00001268       __imp_?OnAmbientProperty@CWnd@@UAEHPAVCOleControlSite@@JPAUtagVARIANT@@@Z 00483268     mfc90:mfc90.dll
 0002:0000126c       __imp_?AddMenu@CContextMenuManager@@QAEHPBDI@Z 0048326c     mfc90:mfc90.dll
 0002:00001270       __imp_?ExitInstance@CWinApp@@UAEHXZ 00483270     mfc90:mfc90.dll
 0002:00001274       __imp_?AfxInitRichEdit2@@YGHXZ 00483274     mfc90:mfc90.dll
 0002:00001278       __imp_?InitInstance@CWinApp@@UAEHXZ 00483278     mfc90:mfc90.dll
 0002:0000127c       __imp_?AfxOleInit@@YGHXZ   0048327c     mfc90:mfc90.dll
 0002:00001280       __imp_?AfxMessageBox@@YGHIII@Z 00483280     mfc90:mfc90.dll
 0002:00001284       __imp_?AfxEnableControlContainer@@YAXPAVCOccManager@@@Z 00483284     mfc90:mfc90.dll
 0002:00001288       __imp_?SetRegistryKey@CWinApp@@IAEXPBD@Z 00483288     mfc90:mfc90.dll
 0002:0000128c       __imp_?LoadStdProfileSettings@CWinApp@@IAEXI@Z 0048328c     mfc90:mfc90.dll
 0002:00001290       __imp_?InitContextMenuManager@CWinAppEx@@QAEHXZ 00483290     mfc90:mfc90.dll
 0002:00001294       __imp_?InitShellManager@CWinAppEx@@QAEHXZ 00483294     mfc90:mfc90.dll
 0002:00001298       __imp_?InitKeyboardManager@CWinAppEx@@QAEHXZ 00483298     mfc90:mfc90.dll
 0002:0000129c       __imp_?InitTooltipManager@CWinAppEx@@QAEHXZ 0048329c     mfc90:mfc90.dll
 0002:000012a0       __imp_?GetThisClass@CMFCToolTipCtrl@@SGPAUCRuntimeClass@@XZ 004832a0     mfc90:mfc90.dll
 0002:000012a4       __imp_?GetTooltipManager@CWinAppEx@@QAEPAVCTooltipManager@@XZ 004832a4     mfc90:mfc90.dll
 0002:000012a8       __imp_?SetTooltipParams@CTooltipManager@@QAEXIPAUCRuntimeClass@@PAVCMFCToolTipInfo@@@Z 004832a8     mfc90:mfc90.dll
 0002:000012ac       __imp_??0CSingleDocTemplate@@QAE@IPAUCRuntimeClass@@00@Z 004832ac     mfc90:mfc90.dll
 0002:000012b0       __imp_?AddDocTemplate@CWinApp@@QAEXPAVCDocTemplate@@@Z 004832b0     mfc90:mfc90.dll
 0002:000012b4       __imp_??0CCommandLineInfo@@QAE@XZ 004832b4     mfc90:mfc90.dll
 0002:000012b8       __imp_?ParseCommandLine@CWinApp@@QAEXAAVCCommandLineInfo@@@Z 004832b8     mfc90:mfc90.dll
 0002:000012bc       __imp_?ProcessShellCommand@CWinApp@@QAEHAAVCCommandLineInfo@@@Z 004832bc     mfc90:mfc90.dll
 0002:000012c0       __imp_??1CCommandLineInfo@@UAE@XZ 004832c0     mfc90:mfc90.dll
 0002:000012c4       __imp_?GetActiveView@CFrameWnd@@QBEPAVCView@@XZ 004832c4     mfc90:mfc90.dll
 0002:000012c8       __imp_??1CWinAppEx@@UAE@XZ 004832c8     mfc90:mfc90.dll
 0002:000012cc       __imp_?ReloadWindowPlacement@CWinAppEx@@MAEHPAVCFrameWnd@@@Z 004832cc     mfc90:mfc90.dll
 0002:000012d0       __imp_?StoreWindowPlacement@CWinAppEx@@MAEHABVCRect@@HH@Z 004832d0     mfc90:mfc90.dll
 0002:000012d4       __imp_?LoadWindowPlacement@CWinAppEx@@MAEHAAVCRect@@AAH1@Z 004832d4     mfc90:mfc90.dll
 0002:000012d8       __imp_?OnClosingMainFrame@CWinAppEx@@MAEXPAVCFrameImpl@@@Z 004832d8     mfc90:mfc90.dll
 0002:000012dc       __imp_?OnAppContextHelp@CWinAppEx@@UAEXPAVCWnd@@QBK@Z 004832dc     mfc90:mfc90.dll
 0002:000012e0       __imp_?ShowPopupMenu@CWinAppEx@@UAEHIABVCPoint@@PAVCWnd@@@Z 004832e0     mfc90:mfc90.dll
 0002:000012e4       __imp_?OnViewDoubleClick@CWinAppEx@@UAEHPAVCWnd@@H@Z 004832e4     mfc90:mfc90.dll
 0002:000012e8       __imp_?SaveState@CWinAppEx@@UAEHPBDPAVCFrameImpl@@@Z 004832e8     mfc90:mfc90.dll
 0002:000012ec       __imp_?CleanState@CWinAppEx@@UAEHPBD@Z 004832ec     mfc90:mfc90.dll
 0002:000012f0       __imp_?LoadState@CWinAppEx@@UAEHPBDPAVCFrameImpl@@@Z 004832f0     mfc90:mfc90.dll
 0002:000012f4       __imp_?LoadSysPolicies@CWinApp@@UAEHXZ 004832f4     mfc90:mfc90.dll
 0002:000012f8       __imp_?LoadAppLangResourceDLL@CWinApp@@UAEPAUHINSTANCE__@@XZ 004832f8     mfc90:mfc90.dll
 0002:000012fc       __imp_?WinHelpInternal@CWinApp@@UAEXKI@Z 004832fc     mfc90:mfc90.dll
 0002:00001300       __imp_?HtmlHelpA@CWinApp@@UAEXKI@Z 00483300     mfc90:mfc90.dll
 0002:00001304       __imp_?WinHelpA@CWinApp@@UAEXKI@Z 00483304     mfc90:mfc90.dll
 0002:00001308       __imp_?OnDDECommand@CWinApp@@UAEHPAD@Z 00483308     mfc90:mfc90.dll
 0002:0000130c       __imp_?DoWaitCursor@CWinApp@@UAEXH@Z 0048330c     mfc90:mfc90.dll
 0002:00001310       __imp_?DoMessageBox@CWinApp@@UAEHPBDII@Z 00483310     mfc90:mfc90.dll
 0002:00001314       __imp_?GetPSP@CPropertyPage@@QAEAAU_PROPSHEETPAGEA@@XZ 00483314     mfc90:mfc90.dll
 0002:00001318       __imp_?SaveAllModified@CWinApp@@UAEHXZ 00483318     mfc90:mfc90.dll
 0002:0000131c       __imp_?PreTranslateMessage@CDialog@@UAEHPAUtagMSG@@@Z 0048331c     mfc90:mfc90.dll
 0002:00001320       __imp_?GetSuperWndProcAddr@CWnd@@MAEPAP6GJPAUHWND__@@IIJ@ZXZ 00483320     mfc90:mfc90.dll
 0002:00001324       __imp_?OnNotify@CWnd@@MAEHIJPAJ@Z 00483324     mfc90:mfc90.dll
 0002:00001328       __imp_?OnCommand@CWnd@@MAEHIJ@Z 00483328     mfc90:mfc90.dll
 0002:0000132c       __imp_?CreateAccessibleProxy@CWnd@@UAEJIJPAJ@Z 0048332c     mfc90:mfc90.dll
 0002:00001330       __imp_?SetProxy@CWnd@@UAEJPAUIAccessibleProxy@@@Z 00483330     mfc90:mfc90.dll
 0002:00001334       __imp_?put_accValue@CWnd@@UAEJUtagVARIANT@@PA_W@Z 00483334     mfc90:mfc90.dll
 0002:00001338       __imp_?put_accName@CWnd@@UAEJUtagVARIANT@@PA_W@Z 00483338     mfc90:mfc90.dll
 0002:0000133c       __imp_?accDoDefaultAction@CWnd@@UAEJUtagVARIANT@@@Z 0048333c     mfc90:mfc90.dll
 0002:00001340       __imp_?accHitTest@CWnd@@UAEJJJPAUtagVARIANT@@@Z 00483340     mfc90:mfc90.dll
 0002:00001344       __imp_?accNavigate@CWnd@@UAEJJUtagVARIANT@@PAU2@@Z 00483344     mfc90:mfc90.dll
 0002:00001348       __imp_?accLocation@CWnd@@UAEJPAJ000UtagVARIANT@@@Z 00483348     mfc90:mfc90.dll
 0002:0000134c       __imp_?accSelect@CWnd@@UAEJJUtagVARIANT@@@Z 0048334c     mfc90:mfc90.dll
 0002:00001350       __imp_?get_accDefaultAction@CWnd@@UAEJUtagVARIANT@@PAPA_W@Z 00483350     mfc90:mfc90.dll
 0002:00001354       __imp_?get_accSelection@CWnd@@UAEJPAUtagVARIANT@@@Z 00483354     mfc90:mfc90.dll
 0002:00001358       __imp_?get_accFocus@CWnd@@UAEJPAUtagVARIANT@@@Z 00483358     mfc90:mfc90.dll
 0002:0000135c       __imp_?get_accKeyboardShortcut@CWnd@@UAEJUtagVARIANT@@PAPA_W@Z 0048335c     mfc90:mfc90.dll
 0002:00001360       __imp_?get_accHelpTopic@CWnd@@UAEJPAPA_WUtagVARIANT@@PAJ@Z 00483360     mfc90:mfc90.dll
 0002:00001364       __imp_?get_accHelp@CWnd@@UAEJUtagVARIANT@@PAPA_W@Z 00483364     mfc90:mfc90.dll
 0002:00001368       __imp_?get_accState@CWnd@@UAEJUtagVARIANT@@PAU2@@Z 00483368     mfc90:mfc90.dll
 0002:0000136c       __imp_??0CMapStringToPtr@@QAE@H@Z 0048336c     mfc90:mfc90.dll
 0002:00001370       __imp_?RemoveAt@CStringList@@QAEXPAU__POSITION@@@Z 00483370     mfc90:mfc90.dll
 0002:00001374       __imp_?OnEditContextMenu@CMFCRibbonBar@@UAEXPAVCMFCRibbonRichEditCtrl@@VCPoint@@@Z 00483374     mfc90:mfc90.dll
 0002:00001378       __imp_?Empty@?$CSimpleStringT@D$00@ATL@@QAEXXZ 00483378     mfc90:mfc90.dll
 0002:0000137c       __imp_?OnClickButton@CMFCRibbonBar@@UAEXPAVCMFCRibbonButton@@VCPoint@@@Z 0048337c     mfc90:mfc90.dll
 0002:00001380       __imp_?GetRuntimeClass@CEdit@@UBEPAUCRuntimeClass@@XZ 00483380     mfc90:mfc90.dll
 0002:00001384       __imp_?get_accRole@CWnd@@UAEJUtagVARIANT@@PAU2@@Z 00483384     mfc90:mfc90.dll
 0002:00001388       __imp_?get_accDescription@CWnd@@UAEJUtagVARIANT@@PAPA_W@Z 00483388     mfc90:mfc90.dll
 0002:0000138c       __imp_??1CMFCRibbonButton@@UAE@XZ 0048338c     mfc90:mfc90.dll
 0002:00001390       __imp_?get_accValue@CWnd@@UAEJUtagVARIANT@@PAPA_W@Z 00483390     mfc90:mfc90.dll
 0002:00001394       __imp_??0CStringArray@@QAE@XZ 00483394     mfc90:mfc90.dll
 0002:00001398       __imp_?_AfxSocketInit@@YGHPAUWSAData@@@Z 00483398     mfc90:mfc90.dll
 0002:0000139c       \177mfc90_NULL_THUNK_DATA  0048339c     mfc90:mfc90.dll
 0002:000013a0       __imp__ExRWDiskAbs         004833a0     windisk:windisk.dll
 0002:000013a4       __imp__ExDetectProtect     004833a4     windisk:windisk.dll
 0002:000013a8       __imp__ExRWDisk            004833a8     windisk:windisk.dll
 0002:000013ac       \177windisk_NULL_THUNK_DATA 004833ac     windisk:windisk.dll
 0002:000013b0       ___xc_a                    004833b0     msvcrt:cinitexe.obj
 0002:00001404       ___xc_z                    00483404     msvcrt:cinitexe.obj
 0002:00001408       ___xi_a                    00483408     msvcrt:cinitexe.obj
 0002:00001418       ___xi_z                    00483418     msvcrt:cinitexe.obj
 0002:0000163c       ?classCAboutDlg@CAboutDlg@@2UCRuntimeClass@@B 0048363c     AboutDlg.obj
 0002:0000165c       ??_7CAboutDlg@@6B@         0048365c     AboutDlg.obj
 0002:00001804       ??_7CStatic@@6B@           00483804     AboutDlg.obj
 0002:000019dc       ??_7CAddToGroup@@6B@       004839dc     AddToGroup.obj
 0002:00001b4c       ??_7CComboBox@@6B@         00483b4c     AddToGroup.obj
 0002:00001dbc       ??_7CBlackListDlg@@6B@     00483dbc     BlackListDlg.obj
 0002:00001f64       ??_7CListCtrl@@6B@         00483f64     BlackListDlg.obj
 0002:00002208       ?classCBlockingSocketException@CBlockingSocketException@@2UCRuntimeClass@@B 00484208     blocksock.obj
 0002:00002224       ?classCBlockingSocket@CBlockingSocket@@2UCRuntimeClass@@B 00484224     blocksock.obj
 0002:00002244       ??_7CBlockingSocketException@@6B@ 00484244     blocksock.obj
 0002:00002268       ??_7CBlockingSocket@@6B@   00484268     blocksock.obj
 0002:00002304       ??_7CBootModuleManager@@6B@ 00484304     BootModuleManager.obj
 0002:0000230c       ??_7?$CTypedPtrList@VCPtrList@@PAK@@6B@ 0048430c     BootModuleManager.obj
 0002:00002324       ??_7?$_CTypedPtrList@VCPtrList@@PAK@@6B@ 00484324     BootModuleManager.obj
 0002:0000233c       ??_7CCriticalSection@@6B@  0048433c     BootModuleManager.obj
 0002:000024dc       ?classCBroadIE@CBroadIE@@2UCRuntimeClass@@B 004844dc     BroadIE.obj
 0002:000024fc       ??_7CBroadIE@@6B@          004844fc     BroadIE.obj
 0002:000026fc       ?classCBroadWaitDlg@CBroadWaitDlg@@2UCRuntimeClass@@B 004846fc     BroadWaitDlg.obj
 0002:0000271c       ??_7CBroadWaitDlg@@6B@     0048471c     BroadWaitDlg.obj
 0002:000028e4       ??_7CCalendarBar@@6B@      004848e4     CalendarBar.obj
 0002:00002acc       ??_7CBitmap@@6B@           00484acc     CalendarBar.obj
 0002:00002ae4       ??_7CGdiObject@@6B@        00484ae4     CalendarBar.obj
 0002:00002af8       ??_C@_0L@LBHJMCDF@?$CFs?5?$CI?$CFs?3?$CFd?$CJ?$AA@ 00484af8     CalendarBar.obj
 0002:00002b04       ??_C@_0O@KHJMBFME@?$CFs?5?$CI?$CFs?3?$CFd?$CJ?6?$CFs?$AA@ 00484b04     CalendarBar.obj
 0002:00002b14       ??_C@_0BP@OIEOKIDM@Exception?5thrown?5in?5destructor?$AA@ 00484b14     CalendarBar.obj
 0002:00002b38       ??_C@_0EL@OJNFJNGL@H?3?2Program?5Files?2Microsoft?5Visua@ 00484b38     CalendarBar.obj
 0002:00002b84       ??_C@_0BE@MAHEJAGB@ImageList_AddMasked?$AA@ 00484b84     CalendarBar.obj
 0002:00002b98       ??_C@_0P@PHOGADFO@ImageList_Draw?$AA@ 00484b98     CalendarBar.obj
 0002:00002bac       ??_7CMonthCalCtrl@@6B@     00484bac     CalendarBar.obj
 0002:00002dac       ??_7CFtpd@@6B@             00484dac     CFtpd.obj
 0002:00002e00       ??_7?$CList@PAVCFtpdPi@@PAV1@@@6B@ 00484e00     CFtpd.obj
 0002:00002e9c       ??_7CCheckPasswordDlg@@6B@ 00484e9c     CheckPasswordDlg.obj
 0002:00003044       ??_7CEdit@@6B@             00485044     CheckPasswordDlg.obj
 0002:000037d0       ??_7CClientInfoManager@@6B@ 004857d0     ClientInfoManager.obj
 0002:000037d8       ??_7?$CTypedPtrMap@VCMapStringToPtr@@V?$CStringT@DV?$StrTraitMFC_DLL@DV?$ChTraitsCRT@D@ATL@@@@@ATL@@PAUtagCLIENTMAININFO@@@@6B@ 004857d8     ClientInfoManager.obj
 0002:000037f0       ??_7?$CTypedPtrMap@VCMapStringToPtr@@V?$CStringT@DV?$StrTraitMFC_DLL@DV?$ChTraitsCRT@D@ATL@@@@@ATL@@PAUtagBLACKLIST@@@@6B@ 004857f0     ClientInfoManager.obj
 0002:00003808       ??_7?$CTypedPtrMap@VCMapStringToPtr@@V?$CStringT@DV?$StrTraitMFC_DLL@DV?$ChTraitsCRT@D@ATL@@@@@ATL@@PAVCStringList@@@@6B@ 00485808     ClientInfoManager.obj
 0002:0000415c       ??_7CClientSettingsDlg@@6B@ 0048615c     ClientSettingsDlg.obj
 0002:0000437c       ??_7CSpinButtonCtrl@@6B@   0048637c     ClientSettingsDlg.obj
 0002:0000453c       ??_7CCmdEnquireDlg@@6B@    0048653c     CmdEnquireDlg.obj
 0002:000046e4       ??_7CButton@@6B@           004866e4     CmdEnquireDlg.obj
 0002:00004bc8       ?classCExecuteProcedure@CExecuteProcedure@@2UCRuntimeClass@@B 00486bc8     ExecuteProcedure.obj
 0002:00004bec       ??_7CExecuteProcedure@@6B@ 00486bec     ExecuteProcedure.obj
 0002:00004dc0       ??_7CFont@@6B@             00486dc0     FontStatic.obj
 0002:00004ddc       ??_7CFtpPasvSrv@@6B@       00486ddc     FtpdPasvSrv.obj
 0002:00005e44       ??_7CFtpdPi@@6B@           00487e44     FtpdPi.obj
 0002:00005fe8       ?classCGroupExt@CGroupExt@@2UCRuntimeClass@@B 00487fe8     GroupExt.obj
 0002:0000600c       ??_7CGroupExt@@6B@         0048800c     GroupExt.obj
 0002:000065bc       ??_7CGroupTree@@6B@        004885bc     GroupTree.obj
 0002:000067fc       ??_7CMenu@@6B@             004887fc     GroupTree.obj
 0002:0000681c       ??_7CTreeCtrl@@6B@         0048881c     GroupTree.obj
 0002:0000697c       ??_7CInfoPromptDlg@@6B@    0048897c     InfoPromptDlg.obj
 0002:00006da0       ??_7CIOCPImplement@@6B@    00488da0     IOCPImplement.obj
 0002:00006dc0       ??_7?$CTypedPtrMap@VCMapPtrToPtr@@PAVCClientContext@@PAUIOCP_DataRecvBuffer@@@@6B@ 00488dc0     IOCPImplement.obj
 0002:00006f34       ??_7CKiboManagerApp@@6B@   00488f34     KiboManager.obj
 0002:0000709c       ?classCKiboManagerDoc@CKiboManagerDoc@@2UCRuntimeClass@@B 0048909c     KiboManagerDoc.obj
 0002:000070c4       ??_7CKiboManagerDoc@@6B@   004890c4     KiboManagerDoc.obj
 0002:00007e04       ?classCKiboManagerView@CKiboManagerView@@2UCRuntimeClass@@B 00489e04     KiboManagerView.obj
 0002:000081a4       ??_7CKiboManagerView@@6B@  0048a1a4     KiboManagerView.obj
 0002:00008340       ??_7logic_error@std@@6B@   0048a340     KiboManagerView.obj
 0002:00008348       ??_C@_0BD@OLBABOEK@vector?$DMT?$DO?5too?5long?$AA@ 0048a348     KiboManagerView.obj
 0002:00008360       ??_7length_error@std@@6B@  0048a360     KiboManagerView.obj
 0002:0000836c       ??_7bad_alloc@std@@6B@     0048a36c     KiboManagerView.obj
 0002:00008f84       ??_7CLenPropertyODBC@@6B@  0048af84     LenPropertyODBC.obj
 0002:00009140       ?classCLoginPasswordDlg@CLoginPasswordDlg@@2UCRuntimeClass@@B 0048b140     LoginPasswordDlg.obj
 0002:00009164       ??_7CLoginPasswordDlg@@6B@ 0048b164     LoginPasswordDlg.obj
 0002:0000ff60       ?classCMainFrame@CMainFrame@@2UCRuntimeClass@@B 00491f60     MainFrm.obj
 0002:0001097c       ??_7CMainFrame@@6B@        0049297c     MainFrm.obj
 0002:00010b5c       ??_7COutlookBar@@6B@       00492b5c     MainFrm.obj
 0002:00010f80       ??_7?$CTypedPtrList@VCPtrList@@PAUtagRECVREQUEST@@@@6B@ 00492f80     MainFrm.obj
 0002:00010f98       ??_7?$CTypedPtrList@VCPtrList@@PAUPartitionTransInfo@@@@6B@ 00492f98     MainFrm.obj
 0002:00010fb0       ??_7?$CTypedPtrMap@VCMapStringToPtr@@V?$CStringT@DV?$StrTraitMFC_DLL@DV?$ChTraitsCRT@D@ATL@@@@@ATL@@PAV23@@@6B@ 00492fb0     MainFrm.obj
 0002:00010fc8       ??_7?$_CTypedPtrList@VCPtrList@@PAUtagRECVREQUEST@@@@6B@ 00492fc8     MainFrm.obj
 0002:00010fe0       ??_7?$_CTypedPtrList@VCPtrList@@PAUPartitionTransInfo@@@@6B@ 00492fe0     MainFrm.obj
 0002:00010ff8       ??_7?$CList@II@@6B@        00492ff8     MainFrm.obj
 0002:00011010       ??_7?$CList@PAVCFtpd@@PAV1@@@6B@ 00493010     MainFrm.obj
 0002:00011028       ??_C@_0EL@GPEBOPMF@H?3?2Program?5Files?2Microsoft?5Visua@ 00493028     MainFrm.obj
 0002:0001107c       ??_7CMFCRibbonApplicationButton@@6B@ 0049307c     MainFrm.obj
 0002:00011250       ??_7?$CMap@V?$CStringT@DV?$StrTraitMFC_DLL@DV?$ChTraitsCRT@D@ATL@@@@@ATL@@PBDUItemInfo@@AAU3@@@6B@ 00493250     MainFrm.obj
 0002:00011278       ?classCMFCRibbonBarNew@CMFCRibbonBarNew@@2UCRuntimeClass@@B 00493278     MFCRibbonBarNew.obj
 0002:0001129c       ??_7CMFCRibbonBarNew@@6B@  0049329c     MFCRibbonBarNew.obj
 0002:000116d4       ??_7CModifyGroup@@6B@      004936d4     ModifyGroup.obj
 0002:0001198c       ?classCMsgDlg@CMsgDlg@@2UCRuntimeClass@@B 0049398c     MsgDlg.obj
 0002:000119ac       ??_7CMsgDlg@@6B@           004939ac     MsgDlg.obj
 0002:00011bc4       ??_7CMyEdit@@6B@           00493bc4     MyEdit.obj
 0002:000120dc       ??_7CMyIOCP@@6B@           004940dc     MyIOCP.obj
 0002:00012434       ?classCMyPropertyPage1@CMyPropertyPage1@@2UCRuntimeClass@@B 00494434     MyPropertyPage1.obj
 0002:00012450       ?classCMyPropertyPage2@CMyPropertyPage2@@2UCRuntimeClass@@B 00494450     MyPropertyPage1.obj
 0002:0001246c       ?classCMyPropertyPage3@CMyPropertyPage3@@2UCRuntimeClass@@B 0049446c     MyPropertyPage1.obj
 0002:0001248c       ??_7CMyPropertyPage1@@6B@  0049448c     MyPropertyPage1.obj
 0002:0001265c       ??_7CMyPropertyPage2@@6B@  0049465c     MyPropertyPage1.obj
 0002:000127fc       ??_7CMyPropertyPage3@@6B@  004947fc     MyPropertyPage1.obj
 0002:00012a58       ?classCMyPropertySheet@CMyPropertySheet@@2UCRuntimeClass@@B 00494a58     MyPropertySheet.obj
 0002:00012a7c       ??_7CMyPropertySheet@@6B@  00494a7c     MyPropertySheet.obj
 0002:00012c7c       ??_7CMyRichEdit@@6B@       00494c7c     MyRichEdit.obj
 0002:00012e88       ??_C@_00CNPNBAHC@?$AA@     00494e88     MyRichEdit.obj
 0002:00012e94       ??_7CRichEditCtrl@@6B@     00494e94     MyRichEdit.obj
 0002:00012fe4       ??_7CNewListCtrl@@6B@      00494fe4     NewListCtrl.obj
 0002:0001319c       ??_7CBrush@@6B@            0049519c     NewListCtrl.obj
 0002:000131b0       ??_C@_0BH@KAPMGNKC@ImageList_GetImageInfo?$AA@ 004951b0     NewListCtrl.obj
 0002:000131ec       ??_7COutputWnd@@6B@        004951ec     OutputWnd.obj
 0002:00013614       ??_7COutputList@@6B@       00495614     OutputWnd.obj
 0002:00013bf4       ??_7CPartitionSettingDlg@@6B@ 00495bf4     PartitionSettingDlg.obj
 0002:00013ea0       ?classCPortChannelDlg@CPortChannelDlg@@2UCRuntimeClass@@B 00495ea0     PortChannelDlg.obj
 0002:00013ec4       ??_7CPortChannelDlg@@6B@   00495ec4     PortChannelDlg.obj
 0002:0001421c       ?classCPortCtrlDlg@CPortCtrlDlg@@2UCRuntimeClass@@B 0049621c     PortCtrlDlg.obj
 0002:0001423c       ??_7CPortCtrlDlg@@6B@      0049623c     PortCtrlDlg.obj
 0002:0001446c       ??_7CPrivateProfileFile@@6B@ 0049646c     PrivateProfileFile.obj
 0002:000144cc       ??_7CProgressDlg@@6B@      004964cc     ProgressDlg.obj
 0002:00014674       ??_7CProgressCtrl@@6B@     00496674     ProgressDlg.obj
 0002:00014fc4       ??_7CPropertyViewDlg@@6B@  00496fc4     PropertyViewDlg.obj
 0002:00015240       ??_C@_0BG@PBOJJDFO@ImageList_ReplaceIcon?$AA@ 00497240     PropertyViewDlg.obj
 0002:0001525c       ??_7CTabCtrl@@6B@          0049725c     PropertyViewDlg.obj
 0002:000153c4       ?classCPropertyViewUIThread@CPropertyViewUIThread@@2UCRuntimeClass@@B 004973c4     PropertyViewUIThread.obj
 0002:000153e4       ??_7CPropertyViewUIThread@@6B@ 004973e4     PropertyViewUIThread.obj
 0002:000154bc       ??_7CReportCtrl@@6B@       004974bc     ReportCtrl.obj
 0002:0001571c       ??_7?$CArray@KK@@6B@       0049771c     ReportCtrl.obj
 0002:00015734       ??_7?$CArray@HH@@6B@       00497734     ReportCtrl.obj
 0002:00015748       __real@bff0000000000000    00497748     ReportCtrl.obj
 0002:0001584c       ?classCSetClientchancelDLg@CSetClientchancelDLg@@2UCRuntimeClass@@B 0049784c     SetClientchancelDLg.obj
 0002:0001586c       ??_7CSetClientchancelDLg@@6B@ 0049786c     SetClientchancelDLg.obj
 0002:00015b30       ?classCSetDrfaultNICDlg@CSetDrfaultNICDlg@@2UCRuntimeClass@@B 00497b30     SetDrfaultNICDlg.obj
 0002:00015b54       ??_7CSetDrfaultNICDlg@@6B@ 00497b54     SetDrfaultNICDlg.obj
 0002:0001607c       ?classCSpecialPartitionRS@CSpecialPartitionRS@@2UCRuntimeClass@@B 0049807c     SpecialPartitionRS.obj
 0002:0001609c       ??_7CSpecialPartitionRS@@6B@ 0049809c     SpecialPartitionRS.obj
 0002:00016424       ??_7CWait@@6B@             00498424     Wait.obj
 0002:00016714       ??_7CWorkspaceBar@@6B@     00498714     WorkspaceBar.obj
 0002:00016a9c       ??_C@_0BF@GPBDCGIL@ImageList_SetBkColor?$AA@ 00498a9c     WorkspaceBar.obj
 0002:00016b6c       ??_7CWorkspaceBar2@@6B@    00498b6c     WorkspaceBar2.obj
 0002:00016f58       ??_C@_01MCMALHOG@a?$AA@    00498f58     comfunc:comfunc.obj
 0002:00016f5c       ??_C@_0BE@POPFGFGJ@SeShutdownPrivilege?$AA@ 00498f5c     comfunc:comfunc.obj
 0002:00016f70       ??_C@_04PFOHOKJK@?5?5?5?5?$AA@ 00498f70     comfunc:comfunc.obj
 0002:00016f78       ??_C@_01EEMJAFIK@?6?$AA@   00498f78     comfunc:comfunc.obj
 0002:00016f7c       ??_C@_0BN@JIAHOFFK@?$CFd?4?$CF02d?4?$CF02d?5?5?$CF02d?3?$CF02d?3?$CF02d?$AA@ 00498f7c     comfunc:comfunc.obj
 0002:00016f9c       ??_C@_0L@NCKBCEGF@runlog?4txt?$AA@ 00498f9c     comfunc:comfunc.obj
 0002:00016fa8       ??_C@_0BH@OHOHHLFP@Get?5system?5type?5error?$CB?$AA@ 00498fa8     comfunc:comfunc.obj
 0002:00016fc0       ??_C@_09EEDNEKAE@enabledbg?$AA@ 00498fc0     comfunc:comfunc.obj
 0002:00016fcc       ??_C@_0BA@FDJEPFGB@Software?2Saming?$AA@ 00498fcc     comfunc:comfunc.obj
 0002:00016fdc       ??_C@_01KICIPPFI@?2?$AA@   00498fdc     comfunc:comfunc.obj
 0002:00016fe0       ??_C@_0BJ@GKGENCBH@?$CF02X?$CF02X?$CF02X?$CF02X?$CF02X?$CF02X?$AA@ 00498fe0     helpful:helpful.obj
 0002:00016ffc       ??_C@_04LAGKFANA@ssdd?$AA@ 00498ffc     commod2:MulticastSocket.obj
 0002:00017008       ??_7?$CTypedPtrList@VCPtrList@@PAUtagUDPRECV@@@@6B@ 00499008     commod2:MulticastSocket.obj
 0002:0001701c       ??_C@_0CL@DJBNJEFG@CMulticastSocket?3?5Failed?5during?5@ 0049901c     commod2:MulticastSocket.obj
 0002:0001704c       ??_7CMulticastSocket@@6B@  0049904c     commod2:MulticastSocket.obj
 0002:00017054       ??_7CODBCSet@@6B@          00499054     dbmod2:MyODBC.obj
 0002:0001705c       ??_7CMyODBC@@6B@           0049905c     dbmod2:MyODBC.obj
 0002:00017060       ??_C@_0BD@BILABGPF@?$LC?$LL?V?$KH?$LD?V?U?b?V?V?W?$KK?$LL?$LL?9?9?$CFd?$AA@ 00499060     dbmod2:MyODBC.obj
 0002:00017074       ??_C@_0P@KLLMCBAP@?$LC?$LL?V?$KH?$LD?V?U?b?V?V?$MA?$OA?P?M?$AA@ 00499074     dbmod2:MyODBC.obj
 0002:00017084       ??_C@_0BD@CLLCBKDL@?H?$KB?A?P?P?$KB?J?$PN?$LD?$KE?$LG?H?J?$LB?J?$KH?$LA?$NM?$AA@ 00499084     dbmod2:MyODBC.obj
 0002:00017098       ??_C@_0BJ@BOBHMLK@?H?$KB?A?P?U?$PL?J?$PN?$LC?$LP?$LH?V?$LF?D?$LD?$KE?$LG?H?J?$LB?J?$KH?$LA?$NM?$AA@ 00499098     dbmod2:MyODBC.obj
 0002:000170b4       ??_C@_0P@PKNKGHKM@?H?$KB?A?P?$LD?$KE?$LG?H?J?$LB?J?$KH?$LA?$NM?$AA@ 004990b4     dbmod2:MyODBC.obj
 0002:000170c4       ??_C@_05HHFOOOHO@?$CFs?0?$CFs?$AA@ 004990c4     dbmod2:MyODBC.obj
 0002:000170cc       ??_C@_0CK@FIGMMGFF@?$LB?$KI?$LI?f?$LH?$KC?I?z?$LE?m?N?s?$LF?D?T?$KN?R?r?J?$LB?$KD?$KM?$LH?V?E?dsqlsta@ 004990cc     dbmod2:MyODBC.obj
 0002:000170f8       ??_C@_0BN@KOHBDADE@?$LL?$LJ?C?$LL?S?P?V?$KH?$LD?V?U?b?V?V?J?$PN?$LO?$NN?$MA?$OA?P?M?$LF?D?W?$KK?$LL?$LL?$AA@ 004990f8     dbmod2:MyODBC.obj
 0002:00017118       ??_C@_0BO@MNMDKANI@?$CF04u?9?$CF02u?9?$CF02u?5?$CF02u?3?$CF02u?3?$CF02u?$AA@ 00499118     dbmod2:MyODBC.obj
 0002:00017138       ??_C@_0CJ@GGAGLOLK@Microsoft?5Access?5Driver?5?$CI?$CK?4mdb?0?5@ 00499138     dbmod2:MyODBC.obj
 0002:00017164       ??_C@_0CA@PKJCKLPO@Microsoft?5Access?5Driver?5?$CI?$CK?4mdb?$CJ?$AA@ 00499164     dbmod2:MyODBC.obj
 0002:00017184       ??_C@_0CP@PAMPJGDK@FIL?$DNMS?5Access?$DLMaxBufferSize?$DN2048@ 00499184     dbmod2:MyODBC.obj
 0002:000171b4       ??_C@_01ICJEACDI@?$DL?$AA@ 004991b4     dbmod2:MyODBC.obj
 0002:000171b8       ??_C@_05LLHIMLDE@?$DLDBQ?$DN?$AA@ 004991b8     dbmod2:MyODBC.obj
 0002:000171c0       ??_C@_04FNPKLOFD@DSN?$DN?$AA@ 004991c0     dbmod2:MyODBC.obj
 0002:000171c8       ??_C@_0BA@LGDNGBOD@?A?$KM?$LN?S?J?$PN?$LO?$NN?$LP?b?J?$KH?$LA?$NM?$CB?$AA@ 004991c8     dbmod2:MyODBC.obj
 0002:000171d8       ??_C@_0BC@JNNOGHED@?$LH?V?E?d?A?$KM?$LN?S?$LO?d?$LB?z?J?$KH?$LA?$NM?$CB?$AA@ 004991d8     dbmod2:MyODBC.obj
 0002:000171ec       ??_C@_0BG@BPKLANBO@?I?h?V?Codbc?$LA?f?$LB?$LO?$LK?E?J?$LB?J?$KH?$LA?$NM?$CB?$AA@ 004991ec     dbmod2:MyODBC.obj
 0002:00017204       ??_C@_0BC@NBACFDCM@?$LH?V?E?d?$LL?$LH?$LO?$LD?$LO?d?$LB?z?J?$KH?$LA?$NM?$CB?$AA@ 00499204     dbmod2:MyODBC.obj
 0002:00017218       ??_C@_0BJ@GBNMNHDA@?V?$LE?P?Psql?S?o?$LO?d?J?$KH?$LA?$NM?0?$LC?$LL?D?$NM?V?$LE?P?P?$AA@ 00499218     dbmod2:MyODBC.obj
 0002:00017234       ??_C@_0CC@ENBFEKBI@?$LF?Z?5?$CFd?5?A?P?$LA?s?$LG?$KI?J?$KH?$LA?$NM?0?D?c?V?$LI?$LG?$KI?$LF?D?$MA?$OA?P?M?J?G?$CF@ 00499234     dbmod2:MyODBC.obj
 0002:00017258       ??_C@_0BB@MOCCFPIG@fail?3?5new?5char?$FL?$FN?$AA@ 00499258     dbmod2:MyODBC.obj
 0002:0001726c       ??_C@_0BB@LMNPGODF@?H?$KB?$MA?$OA?P?M?$LE?z?B?k?J?$LB?J?$KH?$LA?$NM?$AA@ 0049926c     dbmod2:MyODBC.obj
 0002:00017280       ??_C@_0N@GKHAMIGD@?H?$KB?A?P?C?$PL?J?$LB?J?$KH?$LA?$NM?$AA@ 00499280     dbmod2:MyODBC.obj
 0002:00017290       ??_C@_0BO@IPIHKJMO@?$LH?V?E?d?C?$LP?$LI?v?A?P?P?E?O?$KC?$LF?D?D?Z?$LE?f?$LP?U?$LM?d?J?$KH?$LA?$NM?6?$AA@ 00499290     dbmod2:MyODBC.obj
 0002:000172b0       ??_C@_0BI@MKFDIKED@?$LH?V?E?d?C?$LP?$LI?v?A?P?D?Z?$LE?f?$LP?U?$LM?d?J?$KH?$LA?$NM?6?$AA@ 004992b0     dbmod2:MyODBC.obj
 0002:000172c8       ??_C@_0BE@BDKBBOHH@?H?$KB?A?P?J?$PN?J?$KH?$LA?$NM?0?$LC?$LL?D?$NM?V?$LE?P?P?$AA@ 004992c8     dbmod2:MyODBC.obj
 0002:000172dc       ??_C@_0BA@GHDJECJK@?V?$LE?P?Psql?S?o?$LO?d?J?$KH?$LA?$NM?$AA@ 004992dc     dbmod2:MyODBC.obj
 0002:000172ec       ??_C@_0BK@ONOCIDFK@?$LH?V?E?d?S?o?$LO?d?$LO?d?$LB?z?J?$KH?$LA?$NM?0?$LC?$LL?D?$NM?V?$LE?P?P?$AA@ 004992ec     dbmod2:MyODBC.obj
 0002:00017308       ??_C@_0BO@PAOPDBPK@?C?$LL?S?P?A?$KM?$LN?S?J?$PN?$LO?$NN?$LP?b?$KD?$KM?G?k?O?H?$LN?x?P?P?A?$KK?$LN?S?$CB?$AA@ 00499308     dbmod2:MyODBC.obj
 0002:00017328       ??_C@_0BL@GJEFBMFM@?V?$LE?P?P?J?B?N?q?J?$KH?$LA?$NM?$KD?$KM?$LC?$KC?G?R?$LL?X?$LJ?v?J?$KH?$LA?$NM?$AA@ 00499328     dbmod2:MyODBC.obj
 0002:00017344       ??_C@_0BF@BGOMMHMF@?I?h?V?C?W?T?$LG?$KP?L?a?$LN?$LL?$LH?$LN?J?$LN?J?$KH?$LA?$NM?$AA@ 00499344     dbmod2:MyODBC.obj
 0002:0001735c       ??_C@_0BJ@LIOFMFLB@?V?$LE?P?P?J?B?N?q?M?j?$LD?I?$LK?s?$KD?$KM?L?a?$LN?$LL?J?$KH?$LA?$NM?$AA@ 0049935c     dbmod2:MyODBC.obj
 0002:00017378       ??_C@_0BF@JEKDNIMJ@?I?h?V?C?J?V?$LG?$KP?L?a?$LN?$LL?$LH?$LN?J?$LN?J?$KH?$LA?$NM?$AA@ 00499378     dbmod2:MyODBC.obj
 0002:00017390       ??_C@_0BH@CFIEDKAI@?A?$KM?$LN?S?$LO?d?$LB?z?N?$KK?$LP?U?$KD?$KM?$LC?$LL?D?$NM?V?$LE?P?P?$AA@ 00499390     dbmod2:MyODBC.obj
 0002:000173a8       ??_C@_0BB@CBHBLOIH@Para?5flag?5error?$CB?$AA@ 004993a8     kibokern:kibokern.obj
 0002:000173bc       ??_C@_0BM@PEOJADO@Para?5sector?5checksum?5error?$CB?$AA@ 004993bc     kibokern:kibokern.obj
 0002:000173d8       ??_C@_07NFANNNEC@UNKNOWN?$AA@ 004993d8     kibokern:kibokern.obj
 0002:000173e0       ??_C@_04NLFHDAEB@SWAP?$AA@ 004993e0     kibokern:kibokern.obj
 0002:000173e8       ??_C@_04CBLCCKIL@EXT2?$AA@ 004993e8     kibokern:kibokern.obj
 0002:000173f0       ??_C@_04HPPAIJNK@NTFS?$AA@ 004993f0     kibokern:kibokern.obj
 0002:000173f8       ??_C@_05HNJNFBJJ@FAT32?$AA@ 004993f8     kibokern:kibokern.obj
 0002:00017400       ??_C@_05BKHFEAPD@FAT16?$AA@ 00499400     kibokern:kibokern.obj
 0002:00017408       ??_C@_01JOAMLHOP@?9?$AA@   00499408     kibokern:kibokern.obj
 0002:0001740c       ??_C@_03BOCCJCAP@?$CFC?3?$AA@ 0049940c     kibokern:kibokern.obj
 0002:00017414       ??_7?$CTypedPtrList@VCPtrList@@PAUSTRUCT_PROTECTITEM@@@@6B@ 00499414     kibokern:kibokern.obj
 0002:0001742c       ??_7CKiboKern@@6B@         0049942c     kibokern:kibokern.obj
 0002:00017430       ??_C@_02JOGGLHBA@?2n?$AA@  00499430     loadres:exloadres.obj
 0002:00017434       ??_C@_0M@DEBJHILM@?2string?4ini?$AA@ 00499434     loadres:exloadres.obj
 0002:00017440       ??_C@_07GACLGDNA@novalue?$AA@ 00499440     loadres:exloadres.obj
 0002:00017448       ??_C@_0CC@EOMOIDBP@Resource?5error?3File?5?$CFs?5not?5exist@ 00499448     loadres:exloadres.obj
 0002:0001746c       ??_C@_08DALEMBDJ@?2bmp?4ini?$AA@ 0049946c     loadres:exloadres.obj
 0002:00017478       ??_C@_0BG@IADDKNOI@resource?5lib?5is?5bad2?$CB?$AA@ 00499478     loadres:exloadres.obj
 0002:00017490       ??_C@_03CAKEDOOO@bmp?$AA@  00499490     loadres:exloadres.obj
 0002:00017494       ??_C@_0BB@JBENNHDF@IDS_PRODUCT_NAME?$AA@ 00499494     loadres:exloadres.obj
 0002:000174a8       ??_C@_06ICGJLFIM@string?$AA@ 004994a8     loadres:exloadres.obj
 0002:000174b0       ??_C@_09BADPAGCD@$product$?$AA@ 004994b0     loadres:exloadres.obj
 0002:000174bc       ??_C@_0BG@ICHFBDLB@resource?5lib?5is?5bad1?$CB?$AA@ 004994bc     loadres:exloadres.obj
 0002:000174d4       ??_C@_0BE@EOONMDND@Can?8t?5find?5file?5?$CFs?$CB?$AA@ 004994d4     loadres:exloadres.obj
 0002:000174e8       ??_C@_06BGHBJFGM@reschk?$AA@ 004994e8     loadres:exloadres.obj
 0002:000174f0       ??_C@_0BM@OKCEOKKE@File?5?$CFs?0section?5?$CFs?5too?5big?$CB?$AA@ 004994f0     loadres:initwork.obj
 0002:0001750c       ??_C@_0O@BANLFAHC@?$CFCURRENT_DIR?$CF?$AA@ 0049950c     loadres:initwork.obj
 0002:0001751c       ??_C@_07CLEHDIEJ@replace?$AA@ 0049951c     loadres:initwork.obj
 0002:00017524       ??_C@_0DK@JCHLPDBB@Resource?5error?3File?5?$CFs?0section?5?$CF@ 00499524     loadres:initwork.obj
 0002:00017560       ??_C@_0CJ@OCLBFGHK@File?5?$CFs?0section?5?$CFs?0key?5?$CFs?5value?5@ 00499560     loadres:initwork.obj
 0002:00017590       __sz_dwmapi_dll            00499590     dwmapi:dwmapi.dll
 0002:0001759c       ??_C@_06JBKGCNBB@Delete?$AA@ 0049959c     mfcs90:nolib.obj
 0002:000175a4       ??_C@_08KAAPDIAN@NoRemove?$AA@ 004995a4     mfcs90:nolib.obj
 0002:000175b0       ??_C@_0M@DBGDLGLL@ForceRemove?$AA@ 004995b0     mfcs90:nolib.obj
 0002:000175bc       ??_C@_03LAIAPFCB@Val?$AA@  004995bc     mfcs90:nolib.obj
 0002:000175c0       ??_C@_01HMGJMAIH@B?$AA@    004995c0     mfcs90:nolib.obj
 0002:000175c4       ??_C@_01CKDDGHAB@D?$AA@    004995c4     mfcs90:nolib.obj
 0002:000175c8       ??_C@_01PLPBNMEI@M?$AA@    004995c8     mfcs90:nolib.obj
 0002:000175cc       ??_C@_01CPLAODJH@S?$AA@    004995cc     mfcs90:nolib.obj
 0002:00017634       ??_7type_info@@6B@         00499634     msvcrt:ti_inst.obj
 0002:00017640       ??_7_com_error@@6B@        00499640     comsuppw:comraise.obj
 0002:00017644       ??_C@_0BE@LCNCPACH@SQLConfigDataSource?$AA@ 00499644     odbccp32:funcload.obj
 0002:00017658       ??_C@_0N@JLIDKDKN@odbccp32?4dll?$AA@ 00499658     odbccp32:dllload.obj
 0002:00017668       ??_C@_0P@EGBPEC@VerQueryValueA?$AA@ 00499668     odbccp32:dllload.obj
 0002:00017678       ??_C@_0BE@JIHADGJK@GetFileVersionInfoA?$AA@ 00499678     odbccp32:dllload.obj
 0002:0001768c       ??_C@_0BI@FKDAHLLJ@GetFileVersionInfoSizeA?$AA@ 0049968c     odbccp32:dllload.obj
 0002:000176a4       ??_C@_0M@JHNIIDCD@version?4dll?$AA@ 004996a4     odbccp32:dllload.obj
 0002:000176b0       ??_C@_0O@KNNIIANP@?2odbccp32?4bad?$AA@ 004996b0     odbccp32:dllload.obj
 0002:000176c0       ??_C@_0BI@GDDJKAE@?$CJ?4?5Press?5OK?5to?5proceed?4?$AA@ 004996c0     odbccp32:dllload.obj
 0002:000176d8       ??_C@_0DL@FOLMDFBE@?5which?5is?5not?5supported?5in?5the?5l@ 004996d8     odbccp32:dllload.obj
 0002:00017714       ??_C@_0DF@PNAOPFGD@?0?5or?5one?5of?5its?5DLLs?5attempted?5t@ 00499714     odbccp32:dllload.obj
 0002:0001774c       ??_C@_0N@NKOCMOAI@The?5program?5?$AA@ 0049974c     odbccp32:dllload.obj
 0002:00017760       ??_C@_0EH@EGPNBEPO@The?5ODBC?5installer?5DLL?5?$CIODBCCP32@ 00499760     odbccp32:dllload.obj
 0002:000177a8       ??_C@_0BF@NMOIJPAJ@ODBC?5Installer?5Error?$AA@ 004997a8     odbccp32:dllload.obj
 0002:000177c0       _LIBID_WbemClient_v1       004997c0     wbemuuid:wbemcli_i.obj
 0002:000177d0       _IID_IWbemClassObject      004997d0     wbemuuid:wbemcli_i.obj
 0002:000177e0       _IID_IWbemObjectAccess     004997e0     wbemuuid:wbemcli_i.obj
 0002:000177f0       _IID_IWbemQualifierSet     004997f0     wbemuuid:wbemcli_i.obj
 0002:00017800       _IID_IWbemServices         00499800     wbemuuid:wbemcli_i.obj
 0002:00017810       _IID_IWbemLocator          00499810     wbemuuid:wbemcli_i.obj
 0002:00017820       _IID_IWbemObjectSink       00499820     wbemuuid:wbemcli_i.obj
 0002:00017830       _IID_IEnumWbemClassObject  00499830     wbemuuid:wbemcli_i.obj
 0002:00017840       _IID_IWbemCallResult       00499840     wbemuuid:wbemcli_i.obj
 0002:00017850       _IID_IWbemContext          00499850     wbemuuid:wbemcli_i.obj
 0002:00017860       _IID_IUnsecuredApartment   00499860     wbemuuid:wbemcli_i.obj
 0002:00017870       _IID_IWbemUnsecuredApartment 00499870     wbemuuid:wbemcli_i.obj
 0002:00017880       _IID_IWbemStatusCodeText   00499880     wbemuuid:wbemcli_i.obj
 0002:00017890       _IID_IWbemBackupRestore    00499890     wbemuuid:wbemcli_i.obj
 0002:000178a0       _IID_IWbemBackupRestoreEx  004998a0     wbemuuid:wbemcli_i.obj
 0002:000178b0       _IID_IWbemRefresher        004998b0     wbemuuid:wbemcli_i.obj
 0002:000178c0       _IID_IWbemHiPerfEnum       004998c0     wbemuuid:wbemcli_i.obj
 0002:000178d0       _IID_IWbemConfigureRefresher 004998d0     wbemuuid:wbemcli_i.obj
 0002:000178e0       _CLSID_WbemLocator         004998e0     wbemuuid:wbemcli_i.obj
 0002:000178f0       _CLSID_WbemContext         004998f0     wbemuuid:wbemcli_i.obj
 0002:00017900       _CLSID_UnsecuredApartment  00499900     wbemuuid:wbemcli_i.obj
 0002:00017910       _CLSID_WbemClassObject     00499910     wbemuuid:wbemcli_i.obj
 0002:00017920       _CLSID_MofCompiler         00499920     wbemuuid:wbemcli_i.obj
 0002:00017930       _CLSID_WbemStatusCodeText  00499930     wbemuuid:wbemcli_i.obj
 0002:00017940       _CLSID_WbemBackupRestore   00499940     wbemuuid:wbemcli_i.obj
 0002:00017950       _CLSID_WbemRefresher       00499950     wbemuuid:wbemcli_i.obj
 0002:00017960       _CLSID_WbemObjectTextSrc   00499960     wbemuuid:wbemcli_i.obj
 0002:00017970       _IID_IWbemShutdown         00499970     wbemuuid:wbemcli_i.obj
 0002:00017980       _IID_IWbemObjectTextSrc    00499980     wbemuuid:wbemcli_i.obj
 0002:00017990       _IID_IMofCompiler          00499990     wbemuuid:wbemcli_i.obj
 0002:000179c0       __load_config_used         004999c0     msvcrt:loadcfg.obj
 0002:00017a54       ??_R4CAboutDlg@@6B@        00499a54     AboutDlg.obj
 0002:00017a68       ??_R3CAboutDlg@@8          00499a68     AboutDlg.obj
 0002:00017a78       ??_R2CAboutDlg@@8          00499a78     AboutDlg.obj
 0002:00017a90       ??_R1A@?0A@EA@CAboutDlg@@8 00499a90     AboutDlg.obj
 0002:00017aac       ??_R1A@?0A@EA@CDialog@@8   00499aac     AboutDlg.obj
 0002:00017ac8       ??_R3CDialog@@8            00499ac8     AboutDlg.obj
 0002:00017ad8       ??_R2CDialog@@8            00499ad8     AboutDlg.obj
 0002:00017aec       ??_R1A@?0A@EA@CWnd@@8      00499aec     AboutDlg.obj
 0002:00017b08       ??_R3CWnd@@8               00499b08     AboutDlg.obj
 0002:00017b18       ??_R2CWnd@@8               00499b18     AboutDlg.obj
 0002:00017b28       ??_R1A@?0A@EA@CCmdTarget@@8 00499b28     AboutDlg.obj
 0002:00017b44       ??_R3CCmdTarget@@8         00499b44     AboutDlg.obj
 0002:00017b54       ??_R2CCmdTarget@@8         00499b54     AboutDlg.obj
 0002:00017b60       ??_R1A@?0A@EA@CObject@@8   00499b60     AboutDlg.obj
 0002:00017b7c       ??_R3CObject@@8            00499b7c     AboutDlg.obj
 0002:00017b8c       ??_R2CObject@@8            00499b8c     AboutDlg.obj
 0002:00017b94       ??_R4CStatic@@6B@          00499b94     AboutDlg.obj
 0002:00017ba8       ??_R3CStatic@@8            00499ba8     AboutDlg.obj
 0002:00017bb8       ??_R2CStatic@@8            00499bb8     AboutDlg.obj
 0002:00017bcc       ??_R1A@?0A@EA@CStatic@@8   00499bcc     AboutDlg.obj
 0002:00017be8       ??_R4CAddToGroup@@6B@      00499be8     AddToGroup.obj
 0002:00017bfc       ??_R3CAddToGroup@@8        00499bfc     AddToGroup.obj
 0002:00017c0c       ??_R2CAddToGroup@@8        00499c0c     AddToGroup.obj
 0002:00017c24       ??_R1A@?0A@EA@CAddToGroup@@8 00499c24     AddToGroup.obj
 0002:00017c40       ??_R4CComboBox@@6B@        00499c40     AddToGroup.obj
 0002:00017c54       ??_R3CComboBox@@8          00499c54     AddToGroup.obj
 0002:00017c64       ??_R2CComboBox@@8          00499c64     AddToGroup.obj
 0002:00017c78       ??_R1A@?0A@EA@CComboBox@@8 00499c78     AddToGroup.obj
 0002:00017c94       ??_R4CBlackListDlg@@6B@    00499c94     BlackListDlg.obj
 0002:00017ca8       ??_R3CBlackListDlg@@8      00499ca8     BlackListDlg.obj
 0002:00017cb8       ??_R2CBlackListDlg@@8      00499cb8     BlackListDlg.obj
 0002:00017cd0       ??_R1A@?0A@EA@CBlackListDlg@@8 00499cd0     BlackListDlg.obj
 0002:00017cec       ??_R4CListCtrl@@6B@        00499cec     BlackListDlg.obj
 0002:00017d00       ??_R3CListCtrl@@8          00499d00     BlackListDlg.obj
 0002:00017d10       ??_R2CListCtrl@@8          00499d10     BlackListDlg.obj
 0002:00017d24       ??_R1A@?0A@EA@CListCtrl@@8 00499d24     BlackListDlg.obj
 0002:00017d40       ??_R4CBlockingSocketException@@6B@ 00499d40     blocksock.obj
 0002:00017d54       ??_R3CBlockingSocketException@@8 00499d54     blocksock.obj
 0002:00017d64       ??_R2CBlockingSocketException@@8 00499d64     blocksock.obj
 0002:00017d74       ??_R1A@?0A@EA@CBlockingSocketException@@8 00499d74     blocksock.obj
 0002:00017d90       ??_R1A@?0A@EA@CException@@8 00499d90     blocksock.obj
 0002:00017dac       ??_R3CException@@8         00499dac     blocksock.obj
 0002:00017dbc       ??_R2CException@@8         00499dbc     blocksock.obj
 0002:00017dc8       ??_R1A@?0A@EA@CBlockingSocket@@8 00499dc8     blocksock.obj
 0002:00017de4       ??_R3CBlockingSocket@@8    00499de4     blocksock.obj
 0002:00017df4       ??_R2CBlockingSocket@@8    00499df4     blocksock.obj
 0002:00017e00       ??_R4CBlockingSocket@@6B@  00499e00     blocksock.obj
 0002:00017e14       ??_R4CBootModuleManager@@6B@ 00499e14     BootModuleManager.obj
 0002:00017e28       ??_R3CBootModuleManager@@8 00499e28     BootModuleManager.obj
 0002:00017e38       ??_R2CBootModuleManager@@8 00499e38     BootModuleManager.obj
 0002:00017e40       ??_R1A@?0A@EA@CBootModuleManager@@8 00499e40     BootModuleManager.obj
 0002:00017e5c       ??_R4?$CTypedPtrList@VCPtrList@@PAK@@6B@ 00499e5c     BootModuleManager.obj
 0002:00017e70       ??_R3?$CTypedPtrList@VCPtrList@@PAK@@8 00499e70     BootModuleManager.obj
 0002:00017e80       ??_R2?$CTypedPtrList@VCPtrList@@PAK@@8 00499e80     BootModuleManager.obj
 0002:00017e94       ??_R1A@?0A@EA@?$CTypedPtrList@VCPtrList@@PAK@@8 00499e94     BootModuleManager.obj
 0002:00017eb0       ??_R1A@?0A@EA@?$_CTypedPtrList@VCPtrList@@PAK@@8 00499eb0     BootModuleManager.obj
 0002:00017ecc       ??_R3?$_CTypedPtrList@VCPtrList@@PAK@@8 00499ecc     BootModuleManager.obj
 0002:00017edc       ??_R2?$_CTypedPtrList@VCPtrList@@PAK@@8 00499edc     BootModuleManager.obj
 0002:00017eec       ??_R1A@?0A@EA@CPtrList@@8  00499eec     BootModuleManager.obj
 0002:00017f08       ??_R3CPtrList@@8           00499f08     BootModuleManager.obj
 0002:00017f18       ??_R2CPtrList@@8           00499f18     BootModuleManager.obj
 0002:00017f24       ??_R4?$_CTypedPtrList@VCPtrList@@PAK@@6B@ 00499f24     BootModuleManager.obj
 0002:00017f38       ??_R4CCriticalSection@@6B@ 00499f38     BootModuleManager.obj
 0002:00017f4c       ??_R3CCriticalSection@@8   00499f4c     BootModuleManager.obj
 0002:00017f5c       ??_R2CCriticalSection@@8   00499f5c     BootModuleManager.obj
 0002:00017f6c       ??_R1A@?0A@EA@CCriticalSection@@8 00499f6c     BootModuleManager.obj
 0002:00017f88       ??_R1A@?0A@EA@CSyncObject@@8 00499f88     BootModuleManager.obj
 0002:00017fa4       ??_R3CSyncObject@@8        00499fa4     BootModuleManager.obj
 0002:00017fb4       ??_R2CSyncObject@@8        00499fb4     BootModuleManager.obj
 0002:00017fc0       ??_R4CBroadIE@@6B@         00499fc0     BroadIE.obj
 0002:00017fd4       ??_R3CBroadIE@@8           00499fd4     BroadIE.obj
 0002:00017fe4       ??_R2CBroadIE@@8           00499fe4     BroadIE.obj
 0002:00017ffc       ??_R1A@?0A@EA@CBroadIE@@8  00499ffc     BroadIE.obj
 0002:00018018       ??_R4CBroadWaitDlg@@6B@    0049a018     BroadWaitDlg.obj
 0002:0001802c       ??_R3CBroadWaitDlg@@8      0049a02c     BroadWaitDlg.obj
 0002:0001803c       ??_R2CBroadWaitDlg@@8      0049a03c     BroadWaitDlg.obj
 0002:00018054       ??_R1A@?0A@EA@CBroadWaitDlg@@8 0049a054     BroadWaitDlg.obj
 0002:00018070       ??_R4CCalendarBar@@6B@     0049a070     CalendarBar.obj
 0002:00018084       ??_R3CCalendarBar@@8       0049a084     CalendarBar.obj
 0002:00018094       ??_R2CCalendarBar@@8       0049a094     CalendarBar.obj
 0002:000180a8       ??_R1A@?0A@EA@CCalendarBar@@8 0049a0a8     CalendarBar.obj
 0002:000180c4       ??_R4CBitmap@@6B@          0049a0c4     CalendarBar.obj
 0002:000180d8       ??_R3CBitmap@@8            0049a0d8     CalendarBar.obj
 0002:000180e8       ??_R2CBitmap@@8            0049a0e8     CalendarBar.obj
 0002:000180f8       ??_R1A@?0A@EA@CBitmap@@8   0049a0f8     CalendarBar.obj
 0002:00018114       ??_R1A@?0A@EA@CGdiObject@@8 0049a114     CalendarBar.obj
 0002:00018130       ??_R3CGdiObject@@8         0049a130     CalendarBar.obj
 0002:00018140       ??_R2CGdiObject@@8         0049a140     CalendarBar.obj
 0002:0001814c       ??_R4CGdiObject@@6B@       0049a14c     CalendarBar.obj
 0002:00018160       ??_R4CMonthCalCtrl@@6B@    0049a160     CalendarBar.obj
 0002:00018174       ??_R3CMonthCalCtrl@@8      0049a174     CalendarBar.obj
 0002:00018184       ??_R2CMonthCalCtrl@@8      0049a184     CalendarBar.obj
 0002:00018198       ??_R1A@?0A@EA@CMonthCalCtrl@@8 0049a198     CalendarBar.obj
 0002:000181b4       ??_R4CFtpd@@6B@            0049a1b4     CFtpd.obj
 0002:000181c8       ??_R3CFtpd@@8              0049a1c8     CFtpd.obj
 0002:000181d8       ??_R2CFtpd@@8              0049a1d8     CFtpd.obj
 0002:000181ec       ??_R1A@?0A@EA@CFtpd@@8     0049a1ec     CFtpd.obj
 0002:00018208       ??_R1A@?0A@EA@CSocket@@8   0049a208     CFtpd.obj
 0002:00018224       ??_R3CSocket@@8            0049a224     CFtpd.obj
 0002:00018234       ??_R2CSocket@@8            0049a234     CFtpd.obj
 0002:00018244       ??_R1A@?0A@EA@CAsyncSocket@@8 0049a244     CFtpd.obj
 0002:00018260       ??_R3CAsyncSocket@@8       0049a260     CFtpd.obj
 0002:00018270       ??_R2CAsyncSocket@@8       0049a270     CFtpd.obj
 0002:0001827c       ??_R4?$CList@PAVCFtpdPi@@PAV1@@@6B@ 0049a27c     CFtpd.obj
 0002:00018290       ??_R3?$CList@PAVCFtpdPi@@PAV1@@@8 0049a290     CFtpd.obj
 0002:000182a0       ??_R2?$CList@PAVCFtpdPi@@PAV1@@@8 0049a2a0     CFtpd.obj
 0002:000182ac       ??_R1A@?0A@EA@?$CList@PAVCFtpdPi@@PAV1@@@8 0049a2ac     CFtpd.obj
 0002:000182c8       ??_R4CCheckPasswordDlg@@6B@ 0049a2c8     CheckPasswordDlg.obj
 0002:000182dc       ??_R3CCheckPasswordDlg@@8  0049a2dc     CheckPasswordDlg.obj
 0002:000182ec       ??_R2CCheckPasswordDlg@@8  0049a2ec     CheckPasswordDlg.obj
 0002:00018304       ??_R1A@?0A@EA@CCheckPasswordDlg@@8 0049a304     CheckPasswordDlg.obj
 0002:00018320       ??_R4CEdit@@6B@            0049a320     CheckPasswordDlg.obj
 0002:00018334       ??_R3CEdit@@8              0049a334     CheckPasswordDlg.obj
 0002:00018344       ??_R2CEdit@@8              0049a344     CheckPasswordDlg.obj
 0002:00018358       ??_R1A@?0A@EA@CEdit@@8     0049a358     CheckPasswordDlg.obj
 0002:00018374       ??_R4CClientInfoManager@@6B@ 0049a374     ClientInfoManager.obj
 0002:00018388       ??_R3CClientInfoManager@@8 0049a388     ClientInfoManager.obj
 0002:00018398       ??_R2CClientInfoManager@@8 0049a398     ClientInfoManager.obj
 0002:000183a0       ??_R1A@?0A@EA@CClientInfoManager@@8 0049a3a0     ClientInfoManager.obj
 0002:000183bc       ??_R4?$CTypedPtrMap@VCMapStringToPtr@@V?$CStringT@DV?$StrTraitMFC_DLL@DV?$ChTraitsCRT@D@ATL@@@@@ATL@@PAUtagCLIENTMAININFO@@@@6B@ 0049a3bc     ClientInfoManager.obj
 0002:000183d0       ??_R3?$CTypedPtrMap@VCMapStringToPtr@@V?$CStringT@DV?$StrTraitMFC_DLL@DV?$ChTraitsCRT@D@ATL@@@@@ATL@@PAUtagCLIENTMAININFO@@@@8 0049a3d0     ClientInfoManager.obj
 0002:000183e0       ??_R2?$CTypedPtrMap@VCMapStringToPtr@@V?$CStringT@DV?$StrTraitMFC_DLL@DV?$ChTraitsCRT@D@ATL@@@@@ATL@@PAUtagCLIENTMAININFO@@@@8 0049a3e0     ClientInfoManager.obj
 0002:000183f0       ??_R1A@?0A@EA@?$CTypedPtrMap@VCMapStringToPtr@@V?$CStringT@DV?$StrTraitMFC_DLL@DV?$ChTraitsCRT@D@ATL@@@@@ATL@@PAUtagCLIENTMAININFO@@@@8 0049a3f0     ClientInfoManager.obj
 0002:0001840c       ??_R1A@?0A@EA@CMapStringToPtr@@8 0049a40c     ClientInfoManager.obj
 0002:00018428       ??_R3CMapStringToPtr@@8    0049a428     ClientInfoManager.obj
 0002:00018438       ??_R2CMapStringToPtr@@8    0049a438     ClientInfoManager.obj
 0002:00018444       ??_R4?$CTypedPtrMap@VCMapStringToPtr@@V?$CStringT@DV?$StrTraitMFC_DLL@DV?$ChTraitsCRT@D@ATL@@@@@ATL@@PAUtagBLACKLIST@@@@6B@ 0049a444     ClientInfoManager.obj
 0002:00018458       ??_R3?$CTypedPtrMap@VCMapStringToPtr@@V?$CStringT@DV?$StrTraitMFC_DLL@DV?$ChTraitsCRT@D@ATL@@@@@ATL@@PAUtagBLACKLIST@@@@8 0049a458     ClientInfoManager.obj
 0002:00018468       ??_R2?$CTypedPtrMap@VCMapStringToPtr@@V?$CStringT@DV?$StrTraitMFC_DLL@DV?$ChTraitsCRT@D@ATL@@@@@ATL@@PAUtagBLACKLIST@@@@8 0049a468     ClientInfoManager.obj
 0002:00018478       ??_R1A@?0A@EA@?$CTypedPtrMap@VCMapStringToPtr@@V?$CStringT@DV?$StrTraitMFC_DLL@DV?$ChTraitsCRT@D@ATL@@@@@ATL@@PAUtagBLACKLIST@@@@8 0049a478     ClientInfoManager.obj
 0002:00018494       ??_R4?$CTypedPtrMap@VCMapStringToPtr@@V?$CStringT@DV?$StrTraitMFC_DLL@DV?$ChTraitsCRT@D@ATL@@@@@ATL@@PAVCStringList@@@@6B@ 0049a494     ClientInfoManager.obj
 0002:000184a8       ??_R3?$CTypedPtrMap@VCMapStringToPtr@@V?$CStringT@DV?$StrTraitMFC_DLL@DV?$ChTraitsCRT@D@ATL@@@@@ATL@@PAVCStringList@@@@8 0049a4a8     ClientInfoManager.obj
 0002:000184b8       ??_R2?$CTypedPtrMap@VCMapStringToPtr@@V?$CStringT@DV?$StrTraitMFC_DLL@DV?$ChTraitsCRT@D@ATL@@@@@ATL@@PAVCStringList@@@@8 0049a4b8     ClientInfoManager.obj
 0002:000184c8       ??_R1A@?0A@EA@?$CTypedPtrMap@VCMapStringToPtr@@V?$CStringT@DV?$StrTraitMFC_DLL@DV?$ChTraitsCRT@D@ATL@@@@@ATL@@PAVCStringList@@@@8 0049a4c8     ClientInfoManager.obj
 0002:000184e4       ??_R4CClientSettingsDlg@@6B@ 0049a4e4     ClientSettingsDlg.obj
 0002:000184f8       ??_R3CClientSettingsDlg@@8 0049a4f8     ClientSettingsDlg.obj
 0002:00018508       ??_R2CClientSettingsDlg@@8 0049a508     ClientSettingsDlg.obj
 0002:00018520       ??_R1A@?0A@EA@CClientSettingsDlg@@8 0049a520     ClientSettingsDlg.obj
 0002:0001853c       ??_R4CSpinButtonCtrl@@6B@  0049a53c     ClientSettingsDlg.obj
 0002:00018550       ??_R3CSpinButtonCtrl@@8    0049a550     ClientSettingsDlg.obj
 0002:00018560       ??_R2CSpinButtonCtrl@@8    0049a560     ClientSettingsDlg.obj
 0002:00018574       ??_R1A@?0A@EA@CSpinButtonCtrl@@8 0049a574     ClientSettingsDlg.obj
 0002:00018590       ??_R4CCmdEnquireDlg@@6B@   0049a590     CmdEnquireDlg.obj
 0002:000185a4       ??_R3CCmdEnquireDlg@@8     0049a5a4     CmdEnquireDlg.obj
 0002:000185b4       ??_R2CCmdEnquireDlg@@8     0049a5b4     CmdEnquireDlg.obj
 0002:000185cc       ??_R1A@?0A@EA@CCmdEnquireDlg@@8 0049a5cc     CmdEnquireDlg.obj
 0002:000185e8       ??_R4CButton@@6B@          0049a5e8     CmdEnquireDlg.obj
 0002:000185fc       ??_R3CButton@@8            0049a5fc     CmdEnquireDlg.obj
 0002:0001860c       ??_R2CButton@@8            0049a60c     CmdEnquireDlg.obj
 0002:00018620       ??_R1A@?0A@EA@CButton@@8   0049a620     CmdEnquireDlg.obj
 0002:0001863c       ??_R4CExecuteProcedure@@6B@ 0049a63c     ExecuteProcedure.obj
 0002:00018650       ??_R3CExecuteProcedure@@8  0049a650     ExecuteProcedure.obj
 0002:00018660       ??_R2CExecuteProcedure@@8  0049a660     ExecuteProcedure.obj
 0002:00018678       ??_R1A@?0A@EA@CExecuteProcedure@@8 0049a678     ExecuteProcedure.obj
 0002:00018694       ??_R4CFont@@6B@            0049a694     FontStatic.obj
 0002:000186a8       ??_R3CFont@@8              0049a6a8     FontStatic.obj
 0002:000186b8       ??_R2CFont@@8              0049a6b8     FontStatic.obj
 0002:000186c8       ??_R1A@?0A@EA@CFont@@8     0049a6c8     FontStatic.obj
 0002:000186e4       ??_R4CFtpPasvSrv@@6B@      0049a6e4     FtpdPasvSrv.obj
 0002:000186f8       ??_R3CFtpPasvSrv@@8        0049a6f8     FtpdPasvSrv.obj
 0002:00018708       ??_R2CFtpPasvSrv@@8        0049a708     FtpdPasvSrv.obj
 0002:00018718       ??_R1A@?0A@EA@CFtpPasvSrv@@8 0049a718     FtpdPasvSrv.obj
 0002:00018734       ??_R4CFtpdPi@@6B@          0049a734     FtpdPi.obj
 0002:00018748       ??_R3CFtpdPi@@8            0049a748     FtpdPi.obj
 0002:00018758       ??_R2CFtpdPi@@8            0049a758     FtpdPi.obj
 0002:0001876c       ??_R1A@?0A@EA@CFtpdPi@@8   0049a76c     FtpdPi.obj
 0002:00018788       ??_R4CGroupExt@@6B@        0049a788     GroupExt.obj
 0002:0001879c       ??_R3CGroupExt@@8          0049a79c     GroupExt.obj
 0002:000187ac       ??_R2CGroupExt@@8          0049a7ac     GroupExt.obj
 0002:000187c4       ??_R1A@?0A@EA@CGroupExt@@8 0049a7c4     GroupExt.obj
 0002:000187e0       ??_R4CGroupTree@@6B@       0049a7e0     GroupTree.obj
 0002:000187f4       ??_R3CGroupTree@@8         0049a7f4     GroupTree.obj
 0002:00018804       ??_R2CGroupTree@@8         0049a804     GroupTree.obj
 0002:0001881c       ??_R1A@?0A@EA@CGroupTree@@8 0049a81c     GroupTree.obj
 0002:00018838       ??_R1A@?0A@EA@CTreeCtrl@@8 0049a838     GroupTree.obj
 0002:00018854       ??_R3CTreeCtrl@@8          0049a854     GroupTree.obj
 0002:00018864       ??_R2CTreeCtrl@@8          0049a864     GroupTree.obj
 0002:00018878       ??_R4CMenu@@6B@            0049a878     GroupTree.obj
 0002:0001888c       ??_R3CMenu@@8              0049a88c     GroupTree.obj
 0002:0001889c       ??_R2CMenu@@8              0049a89c     GroupTree.obj
 0002:000188a8       ??_R1A@?0A@EA@CMenu@@8     0049a8a8     GroupTree.obj
 0002:000188c4       ??_R4CTreeCtrl@@6B@        0049a8c4     GroupTree.obj
 0002:000188d8       ??_R4CInfoPromptDlg@@6B@   0049a8d8     InfoPromptDlg.obj
 0002:000188ec       ??_R3CInfoPromptDlg@@8     0049a8ec     InfoPromptDlg.obj
 0002:000188fc       ??_R2CInfoPromptDlg@@8     0049a8fc     InfoPromptDlg.obj
 0002:00018914       ??_R1A@?0A@EA@CInfoPromptDlg@@8 0049a914     InfoPromptDlg.obj
 0002:00018930       ??_R4CIOCPImplement@@6B@   0049a930     IOCPImplement.obj
 0002:00018944       ??_R3CIOCPImplement@@8     0049a944     IOCPImplement.obj
 0002:00018954       ??_R2CIOCPImplement@@8     0049a954     IOCPImplement.obj
 0002:00018960       ??_R1A@?0A@EA@CIOCPImplement@@8 0049a960     IOCPImplement.obj
 0002:0001897c       ??_R1A@?0A@EA@CMyIOCP@@8   0049a97c     IOCPImplement.obj
 0002:00018998       ??_R3CMyIOCP@@8            0049a998     IOCPImplement.obj
 0002:000189a8       ??_R2CMyIOCP@@8            0049a9a8     IOCPImplement.obj
 0002:000189b0       ??_R4?$CTypedPtrMap@VCMapPtrToPtr@@PAVCClientContext@@PAUIOCP_DataRecvBuffer@@@@6B@ 0049a9b0     IOCPImplement.obj
 0002:000189c4       ??_R3?$CTypedPtrMap@VCMapPtrToPtr@@PAVCClientContext@@PAUIOCP_DataRecvBuffer@@@@8 0049a9c4     IOCPImplement.obj
 0002:000189d4       ??_R2?$CTypedPtrMap@VCMapPtrToPtr@@PAVCClientContext@@PAUIOCP_DataRecvBuffer@@@@8 0049a9d4     IOCPImplement.obj
 0002:000189e4       ??_R1A@?0A@EA@?$CTypedPtrMap@VCMapPtrToPtr@@PAVCClientContext@@PAUIOCP_DataRecvBuffer@@@@8 0049a9e4     IOCPImplement.obj
 0002:00018a00       ??_R1A@?0A@EA@CMapPtrToPtr@@8 0049aa00     IOCPImplement.obj
 0002:00018a1c       ??_R3CMapPtrToPtr@@8       0049aa1c     IOCPImplement.obj
 0002:00018a2c       ??_R2CMapPtrToPtr@@8       0049aa2c     IOCPImplement.obj
 0002:00018a38       ??_R4CKiboManagerApp@@6B@  0049aa38     KiboManager.obj
 0002:00018a4c       ??_R3CKiboManagerApp@@8    0049aa4c     KiboManager.obj
 0002:00018a5c       ??_R2CKiboManagerApp@@8    0049aa5c     KiboManager.obj
 0002:00018a78       ??_R1A@?0A@EA@CKiboManagerApp@@8 0049aa78     KiboManager.obj
 0002:00018a94       ??_R1A@?0A@EA@CWinAppEx@@8 0049aa94     KiboManager.obj
 0002:00018ab0       ??_R3CWinAppEx@@8          0049aab0     KiboManager.obj
 0002:00018ac0       ??_R2CWinAppEx@@8          0049aac0     KiboManager.obj
 0002:00018ad8       ??_R1A@?0A@EA@CWinApp@@8   0049aad8     KiboManager.obj
 0002:00018af4       ??_R3CWinApp@@8            0049aaf4     KiboManager.obj
 0002:00018b04       ??_R2CWinApp@@8            0049ab04     KiboManager.obj
 0002:00018b18       ??_R1A@?0A@EA@CWinThread@@8 0049ab18     KiboManager.obj
 0002:00018b34       ??_R3CWinThread@@8         0049ab34     KiboManager.obj
 0002:00018b44       ??_R2CWinThread@@8         0049ab44     KiboManager.obj
 0002:00018b54       ??_R4CKiboManagerDoc@@6B@  0049ab54     KiboManagerDoc.obj
 0002:00018b68       ??_R3CKiboManagerDoc@@8    0049ab68     KiboManagerDoc.obj
 0002:00018b78       ??_R2CKiboManagerDoc@@8    0049ab78     KiboManagerDoc.obj
 0002:00018b8c       ??_R1A@?0A@EA@CKiboManagerDoc@@8 0049ab8c     KiboManagerDoc.obj
 0002:00018ba8       ??_R1A@?0A@EA@CDocument@@8 0049aba8     KiboManagerDoc.obj
 0002:00018bc4       ??_R3CDocument@@8          0049abc4     KiboManagerDoc.obj
 0002:00018bd4       ??_R2CDocument@@8          0049abd4     KiboManagerDoc.obj
 0002:00018be4       ??_R4CKiboManagerView@@6B@ 0049abe4     KiboManagerView.obj
 0002:00018bf8       ??_R3CKiboManagerView@@8   0049abf8     KiboManagerView.obj
 0002:00018c08       ??_R2CKiboManagerView@@8   0049ac08     KiboManagerView.obj
 0002:00018c28       ??_R1A@?0A@EA@CKiboManagerView@@8 0049ac28     KiboManagerView.obj
 0002:00018c44       ??_R1A@?0A@EA@CFormView@@8 0049ac44     KiboManagerView.obj
 0002:00018c60       ??_R3CFormView@@8          0049ac60     KiboManagerView.obj
 0002:00018c70       ??_R2CFormView@@8          0049ac70     KiboManagerView.obj
 0002:00018c8c       ??_R1A@?0A@EA@CScrollView@@8 0049ac8c     KiboManagerView.obj
 0002:00018ca8       ??_R3CScrollView@@8        0049aca8     KiboManagerView.obj
 0002:00018cb8       ??_R2CScrollView@@8        0049acb8     KiboManagerView.obj
 0002:00018cd0       ??_R1A@?0A@EA@CView@@8     0049acd0     KiboManagerView.obj
 0002:00018cec       ??_R3CView@@8              0049acec     KiboManagerView.obj
 0002:00018cfc       ??_R2CView@@8              0049acfc     KiboManagerView.obj
 0002:00018d10       ??_R1A@?0A@EA@logic_error@std@@8 0049ad10     KiboManagerView.obj
 0002:00018d2c       ??_R3logic_error@std@@8    0049ad2c     KiboManagerView.obj
 0002:00018d3c       ??_R2logic_error@std@@8    0049ad3c     KiboManagerView.obj
 0002:00018d48       ??_R1A@?0A@EA@exception@std@@8 0049ad48     KiboManagerView.obj
 0002:00018d64       ??_R3exception@std@@8      0049ad64     KiboManagerView.obj
 0002:00018d74       ??_R2exception@std@@8      0049ad74     KiboManagerView.obj
 0002:00018d7c       ??_R4logic_error@std@@6B@  0049ad7c     KiboManagerView.obj
 0002:00018d90       ??_R4length_error@std@@6B@ 0049ad90     KiboManagerView.obj
 0002:00018da4       ??_R3length_error@std@@8   0049ada4     KiboManagerView.obj
 0002:00018db4       ??_R2length_error@std@@8   0049adb4     KiboManagerView.obj
 0002:00018dc4       ??_R1A@?0A@EA@length_error@std@@8 0049adc4     KiboManagerView.obj
 0002:00018de0       ??_R4bad_alloc@std@@6B@    0049ade0     KiboManagerView.obj
 0002:00018df4       ??_R3bad_alloc@std@@8      0049adf4     KiboManagerView.obj
 0002:00018e04       ??_R2bad_alloc@std@@8      0049ae04     KiboManagerView.obj
 0002:00018e10       ??_R1A@?0A@EA@bad_alloc@std@@8 0049ae10     KiboManagerView.obj
 0002:00018e2c       ??_R4CLenPropertyODBC@@6B@ 0049ae2c     LenPropertyODBC.obj
 0002:00018e40       ??_R3CLenPropertyODBC@@8   0049ae40     LenPropertyODBC.obj
 0002:00018e50       ??_R2CLenPropertyODBC@@8   0049ae50     LenPropertyODBC.obj
 0002:00018e5c       ??_R1A@?0A@EA@CLenPropertyODBC@@8 0049ae5c     LenPropertyODBC.obj
 0002:00018e78       ??_R1A@?0A@EA@CMyODBC@@8   0049ae78     LenPropertyODBC.obj
 0002:00018e94       ??_R3CMyODBC@@8            0049ae94     LenPropertyODBC.obj
 0002:00018ea4       ??_R2CMyODBC@@8            0049aea4     LenPropertyODBC.obj
 0002:00018eac       ??_R1A@?0A@EA@CNewListCtrl@@8 0049aeac     ListCtrlEx.obj
 0002:00018ec8       ??_R3CNewListCtrl@@8       0049aec8     ListCtrlEx.obj
 0002:00018ed8       ??_R2CNewListCtrl@@8       0049aed8     ListCtrlEx.obj
 0002:00018ef0       ??_R4CLoginPasswordDlg@@6B@ 0049aef0     LoginPasswordDlg.obj
 0002:00018f04       ??_R3CLoginPasswordDlg@@8  0049af04     LoginPasswordDlg.obj
 0002:00018f14       ??_R2CLoginPasswordDlg@@8  0049af14     LoginPasswordDlg.obj
 0002:00018f2c       ??_R1A@?0A@EA@CLoginPasswordDlg@@8 0049af2c     LoginPasswordDlg.obj
 0002:00018f48       ??_R4CMainFrame@@6B@       0049af48     MainFrm.obj
 0002:00018f5c       ??_R3CMainFrame@@8         0049af5c     MainFrm.obj
 0002:00018f6c       ??_R2CMainFrame@@8         0049af6c     MainFrm.obj
 0002:00018f88       ??_R1A@?0A@EA@CMainFrame@@8 0049af88     MainFrm.obj
 0002:00018fa4       ??_R1A@?0A@EA@CFrameWndEx@@8 0049afa4     MainFrm.obj
 0002:00018fc0       ??_R3CFrameWndEx@@8        0049afc0     MainFrm.obj
 0002:00018fd0       ??_R2CFrameWndEx@@8        0049afd0     MainFrm.obj
 0002:00018fe8       ??_R1A@?0A@EA@CFrameWnd@@8 0049afe8     MainFrm.obj
 0002:00019004       ??_R3CFrameWnd@@8          0049b004     MainFrm.obj
 0002:00019014       ??_R2CFrameWnd@@8          0049b014     MainFrm.obj
 0002:00019028       ??_R4COutlookBar@@6B@      0049b028     MainFrm.obj
 0002:0001903c       ??_R3COutlookBar@@8        0049b03c     MainFrm.obj
 0002:0001904c       ??_R2COutlookBar@@8        0049b04c     MainFrm.obj
 0002:00019074       ??_R1A@?0A@EA@COutlookBar@@8 0049b074     MainFrm.obj
 0002:00019090       ??_R1A@?0A@EA@CMFCOutlookBar@@8 0049b090     MainFrm.obj
 0002:000190ac       ??_R3CMFCOutlookBar@@8     0049b0ac     MainFrm.obj
 0002:000190bc       ??_R2CMFCOutlookBar@@8     0049b0bc     MainFrm.obj
 0002:000190e0       ??_R1A@?0A@EA@CBaseTabbedPane@@8 0049b0e0     MainFrm.obj
 0002:000190fc       ??_R3CBaseTabbedPane@@8    0049b0fc     MainFrm.obj
 0002:0001910c       ??_R2CBaseTabbedPane@@8    0049b10c     MainFrm.obj
 0002:0001912c       ??_R1A@?0A@EA@CDockablePane@@8 0049b12c     MainFrm.obj
 0002:00019148       ??_R3CDockablePane@@8      0049b148     MainFrm.obj
 0002:00019158       ??_R2CDockablePane@@8      0049b158     MainFrm.obj
 0002:00019174       ??_R1A@?0A@EA@CPane@@8     0049b174     MainFrm.obj
 0002:00019190       ??_R3CPane@@8              0049b190     MainFrm.obj
 0002:000191a0       ??_R2CPane@@8              0049b1a0     MainFrm.obj
 0002:000191b8       ??_R1A@?0A@EA@CBasePane@@8 0049b1b8     MainFrm.obj
 0002:000191d4       ??_R3CBasePane@@8          0049b1d4     MainFrm.obj
 0002:000191e4       ??_R2CBasePane@@8          0049b1e4     MainFrm.obj
 0002:000191f8       ??_R4?$CTypedPtrList@VCPtrList@@PAUtagRECVREQUEST@@@@6B@ 0049b1f8     MainFrm.obj
 0002:0001920c       ??_R3?$CTypedPtrList@VCPtrList@@PAUtagRECVREQUEST@@@@8 0049b20c     MainFrm.obj
 0002:0001921c       ??_R2?$CTypedPtrList@VCPtrList@@PAUtagRECVREQUEST@@@@8 0049b21c     MainFrm.obj
 0002:00019230       ??_R1A@?0A@EA@?$CTypedPtrList@VCPtrList@@PAUtagRECVREQUEST@@@@8 0049b230     MainFrm.obj
 0002:0001924c       ??_R1A@?0A@EA@?$_CTypedPtrList@VCPtrList@@PAUtagRECVREQUEST@@@@8 0049b24c     MainFrm.obj
 0002:00019268       ??_R3?$_CTypedPtrList@VCPtrList@@PAUtagRECVREQUEST@@@@8 0049b268     MainFrm.obj
 0002:00019278       ??_R2?$_CTypedPtrList@VCPtrList@@PAUtagRECVREQUEST@@@@8 0049b278     MainFrm.obj
 0002:00019288       ??_R4?$CTypedPtrList@VCPtrList@@PAUPartitionTransInfo@@@@6B@ 0049b288     MainFrm.obj
 0002:0001929c       ??_R3?$CTypedPtrList@VCPtrList@@PAUPartitionTransInfo@@@@8 0049b29c     MainFrm.obj
 0002:000192ac       ??_R2?$CTypedPtrList@VCPtrList@@PAUPartitionTransInfo@@@@8 0049b2ac     MainFrm.obj
 0002:000192c0       ??_R1A@?0A@EA@?$CTypedPtrList@VCPtrList@@PAUPartitionTransInfo@@@@8 0049b2c0     MainFrm.obj
 0002:000192dc       ??_R1A@?0A@EA@?$_CTypedPtrList@VCPtrList@@PAUPartitionTransInfo@@@@8 0049b2dc     MainFrm.obj
 0002:000192f8       ??_R3?$_CTypedPtrList@VCPtrList@@PAUPartitionTransInfo@@@@8 0049b2f8     MainFrm.obj
 0002:00019308       ??_R2?$_CTypedPtrList@VCPtrList@@PAUPartitionTransInfo@@@@8 0049b308     MainFrm.obj
 0002:00019318       ??_R4?$CTypedPtrMap@VCMapStringToPtr@@V?$CStringT@DV?$StrTraitMFC_DLL@DV?$ChTraitsCRT@D@ATL@@@@@ATL@@PAV23@@@6B@ 0049b318     MainFrm.obj
 0002:0001932c       ??_R3?$CTypedPtrMap@VCMapStringToPtr@@V?$CStringT@DV?$StrTraitMFC_DLL@DV?$ChTraitsCRT@D@ATL@@@@@ATL@@PAV23@@@8 0049b32c     MainFrm.obj
 0002:0001933c       ??_R2?$CTypedPtrMap@VCMapStringToPtr@@V?$CStringT@DV?$StrTraitMFC_DLL@DV?$ChTraitsCRT@D@ATL@@@@@ATL@@PAV23@@@8 0049b33c     MainFrm.obj
 0002:0001934c       ??_R1A@?0A@EA@?$CTypedPtrMap@VCMapStringToPtr@@V?$CStringT@DV?$StrTraitMFC_DLL@DV?$ChTraitsCRT@D@ATL@@@@@ATL@@PAV23@@@8 0049b34c     MainFrm.obj
 0002:00019368       ??_R4?$_CTypedPtrList@VCPtrList@@PAUtagRECVREQUEST@@@@6B@ 0049b368     MainFrm.obj
 0002:0001937c       ??_R4?$_CTypedPtrList@VCPtrList@@PAUPartitionTransInfo@@@@6B@ 0049b37c     MainFrm.obj
 0002:00019390       ??_R4?$CList@II@@6B@       0049b390     MainFrm.obj
 0002:000193a4       ??_R3?$CList@II@@8         0049b3a4     MainFrm.obj
 0002:000193b4       ??_R2?$CList@II@@8         0049b3b4     MainFrm.obj
 0002:000193c0       ??_R1A@?0A@EA@?$CList@II@@8 0049b3c0     MainFrm.obj
 0002:000193dc       ??_R4?$CList@PAVCFtpd@@PAV1@@@6B@ 0049b3dc     MainFrm.obj
 0002:000193f0       ??_R3?$CList@PAVCFtpd@@PAV1@@@8 0049b3f0     MainFrm.obj
 0002:00019400       ??_R2?$CList@PAVCFtpd@@PAV1@@@8 0049b400     MainFrm.obj
 0002:0001940c       ??_R1A@?0A@EA@?$CList@PAVCFtpd@@PAV1@@@8 0049b40c     MainFrm.obj
 0002:00019428       ??_R4CMFCRibbonApplicationButton@@6B@ 0049b428     MainFrm.obj
 0002:0001943c       ??_R3CMFCRibbonApplicationButton@@8 0049b43c     MainFrm.obj
 0002:0001944c       ??_R2CMFCRibbonApplicationButton@@8 0049b44c     MainFrm.obj
 0002:00019460       ??_R1A@?0A@EA@CMFCRibbonApplicationButton@@8 0049b460     MainFrm.obj
 0002:0001947c       ??_R1A@?0A@EA@CMFCRibbonButton@@8 0049b47c     MainFrm.obj
 0002:00019498       ??_R3CMFCRibbonButton@@8   0049b498     MainFrm.obj
 0002:000194a8       ??_R2CMFCRibbonButton@@8   0049b4a8     MainFrm.obj
 0002:000194b8       ??_R1A@?0A@EA@CMFCRibbonBaseElement@@8 0049b4b8     MainFrm.obj
 0002:000194d4       ??_R3CMFCRibbonBaseElement@@8 0049b4d4     MainFrm.obj
 0002:000194e4       ??_R2CMFCRibbonBaseElement@@8 0049b4e4     MainFrm.obj
 0002:000194f0       ??_R4?$CMap@V?$CStringT@DV?$StrTraitMFC_DLL@DV?$ChTraitsCRT@D@ATL@@@@@ATL@@PBDUItemInfo@@AAU3@@@6B@ 0049b4f0     MainFrm.obj
 0002:00019504       ??_R3?$CMap@V?$CStringT@DV?$StrTraitMFC_DLL@DV?$ChTraitsCRT@D@ATL@@@@@ATL@@PBDUItemInfo@@AAU3@@@8 0049b504     MainFrm.obj
 0002:00019514       ??_R2?$CMap@V?$CStringT@DV?$StrTraitMFC_DLL@DV?$ChTraitsCRT@D@ATL@@@@@ATL@@PBDUItemInfo@@AAU3@@@8 0049b514     MainFrm.obj
 0002:00019520       ??_R1A@?0A@EA@?$CMap@V?$CStringT@DV?$StrTraitMFC_DLL@DV?$ChTraitsCRT@D@ATL@@@@@ATL@@PBDUItemInfo@@AAU3@@@8 0049b520     MainFrm.obj
 0002:0001953c       ??_R4CMFCRibbonBarNew@@6B@ 0049b53c     MFCRibbonBarNew.obj
 0002:00019550       ??_R3CMFCRibbonBarNew@@8   0049b550     MFCRibbonBarNew.obj
 0002:00019560       ??_R2CMFCRibbonBarNew@@8   0049b560     MFCRibbonBarNew.obj
 0002:00019580       ??_R1A@?0A@EA@CMFCRibbonBarNew@@8 0049b580     MFCRibbonBarNew.obj
 0002:0001959c       ??_R1A@?0A@EA@CMFCRibbonBar@@8 0049b59c     MFCRibbonBarNew.obj
 0002:000195b8       ??_R3CMFCRibbonBar@@8      0049b5b8     MFCRibbonBarNew.obj
 0002:000195c8       ??_R2CMFCRibbonBar@@8      0049b5c8     MFCRibbonBarNew.obj
 0002:000195e4       ??_R4CModifyGroup@@6B@     0049b5e4     ModifyGroup.obj
 0002:000195f8       ??_R3CModifyGroup@@8       0049b5f8     ModifyGroup.obj
 0002:00019608       ??_R2CModifyGroup@@8       0049b608     ModifyGroup.obj
 0002:00019620       ??_R1A@?0A@EA@CModifyGroup@@8 0049b620     ModifyGroup.obj
 0002:0001963c       ??_R4CMsgDlg@@6B@          0049b63c     MsgDlg.obj
 0002:00019650       ??_R3CMsgDlg@@8            0049b650     MsgDlg.obj
 0002:00019660       ??_R2CMsgDlg@@8            0049b660     MsgDlg.obj
 0002:00019678       ??_R1A@?0A@EA@CMsgDlg@@8   0049b678     MsgDlg.obj
 0002:00019694       ??_R4CMyEdit@@6B@          0049b694     MyEdit.obj
 0002:000196a8       ??_R3CMyEdit@@8            0049b6a8     MyEdit.obj
 0002:000196b8       ??_R2CMyEdit@@8            0049b6b8     MyEdit.obj
 0002:000196d0       ??_R1A@?0A@EA@CMyEdit@@8   0049b6d0     MyEdit.obj
 0002:000196ec       ??_R4CMyIOCP@@6B@          0049b6ec     MyIOCP.obj
 0002:00019700       ??_R4CMyPropertyPage1@@6B@ 0049b700     MyPropertyPage1.obj
 0002:00019714       ??_R3CMyPropertyPage1@@8   0049b714     MyPropertyPage1.obj
 0002:00019724       ??_R2CMyPropertyPage1@@8   0049b724     MyPropertyPage1.obj
 0002:00019744       ??_R1A@?0A@EA@CMyPropertyPage1@@8 0049b744     MyPropertyPage1.obj
 0002:00019760       ??_R1A@?0A@EA@CMFCPropertyPage@@8 0049b760     MyPropertyPage1.obj
 0002:0001977c       ??_R3CMFCPropertyPage@@8   0049b77c     MyPropertyPage1.obj
 0002:0001978c       ??_R2CMFCPropertyPage@@8   0049b78c     MyPropertyPage1.obj
 0002:000197a8       ??_R1A@?0A@EA@CPropertyPage@@8 0049b7a8     MyPropertyPage1.obj
 0002:000197c4       ??_R3CPropertyPage@@8      0049b7c4     MyPropertyPage1.obj
 0002:000197d4       ??_R2CPropertyPage@@8      0049b7d4     MyPropertyPage1.obj
 0002:000197ec       ??_R4CMyPropertyPage2@@6B@ 0049b7ec     MyPropertyPage1.obj
 0002:00019800       ??_R3CMyPropertyPage2@@8   0049b800     MyPropertyPage1.obj
 0002:00019810       ??_R2CMyPropertyPage2@@8   0049b810     MyPropertyPage1.obj
 0002:00019830       ??_R1A@?0A@EA@CMyPropertyPage2@@8 0049b830     MyPropertyPage1.obj
 0002:0001984c       ??_R4CMyPropertyPage3@@6B@ 0049b84c     MyPropertyPage1.obj
 0002:00019860       ??_R3CMyPropertyPage3@@8   0049b860     MyPropertyPage1.obj
 0002:00019870       ??_R2CMyPropertyPage3@@8   0049b870     MyPropertyPage1.obj
 0002:00019890       ??_R1A@?0A@EA@CMyPropertyPage3@@8 0049b890     MyPropertyPage1.obj
 0002:000198ac       ??_R4CMyPropertySheet@@6B@ 0049b8ac     MyPropertySheet.obj
 0002:000198c0       ??_R3CMyPropertySheet@@8   0049b8c0     MyPropertySheet.obj
 0002:000198d0       ??_R2CMyPropertySheet@@8   0049b8d0     MyPropertySheet.obj
 0002:000198ec       ??_R1A@?0A@EA@CMyPropertySheet@@8 0049b8ec     MyPropertySheet.obj
 0002:00019908       ??_R1A@?0A@EA@CMFCPropertySheet@@8 0049b908     MyPropertySheet.obj
 0002:00019924       ??_R3CMFCPropertySheet@@8  0049b924     MyPropertySheet.obj
 0002:00019934       ??_R2CMFCPropertySheet@@8  0049b934     MyPropertySheet.obj
 0002:0001994c       ??_R1A@?0A@EA@CPropertySheet@@8 0049b94c     MyPropertySheet.obj
 0002:00019968       ??_R3CPropertySheet@@8     0049b968     MyPropertySheet.obj
 0002:00019978       ??_R2CPropertySheet@@8     0049b978     MyPropertySheet.obj
 0002:0001998c       ??_R4CMyRichEdit@@6B@      0049b98c     MyRichEdit.obj
 0002:000199a0       ??_R3CMyRichEdit@@8        0049b9a0     MyRichEdit.obj
 0002:000199b0       ??_R2CMyRichEdit@@8        0049b9b0     MyRichEdit.obj
 0002:000199c8       ??_R1A@?0A@EA@CMyRichEdit@@8 0049b9c8     MyRichEdit.obj
 0002:000199e4       ??_R1A@?0A@EA@CRichEditCtrl@@8 0049b9e4     MyRichEdit.obj
 0002:00019a00       ??_R3CRichEditCtrl@@8      0049ba00     MyRichEdit.obj
 0002:00019a10       ??_R2CRichEditCtrl@@8      0049ba10     MyRichEdit.obj
 0002:00019a24       ??_R4CRichEditCtrl@@6B@    0049ba24     MyRichEdit.obj
 0002:00019a38       ??_R4CNewListCtrl@@6B@     0049ba38     NewListCtrl.obj
 0002:00019a4c       ??_R4CBrush@@6B@           0049ba4c     NewListCtrl.obj
 0002:00019a60       ??_R3CBrush@@8             0049ba60     NewListCtrl.obj
 0002:00019a70       ??_R2CBrush@@8             0049ba70     NewListCtrl.obj
 0002:00019a80       ??_R1A@?0A@EA@CBrush@@8    0049ba80     NewListCtrl.obj
 0002:00019a9c       ??_R4COutputWnd@@6B@       0049ba9c     OutputWnd.obj
 0002:00019ab0       ??_R3COutputWnd@@8         0049bab0     OutputWnd.obj
 0002:00019ac0       ??_R2COutputWnd@@8         0049bac0     OutputWnd.obj
 0002:00019ae0       ??_R1A@?0A@EA@COutputWnd@@8 0049bae0     OutputWnd.obj
 0002:00019afc       ??_R4COutputList@@6B@      0049bafc     OutputWnd.obj
 0002:00019b10       ??_R3COutputList@@8        0049bb10     OutputWnd.obj
 0002:00019b20       ??_R2COutputList@@8        0049bb20     OutputWnd.obj
 0002:00019b3c       ??_R1A@?0A@EA@COutputList@@8 0049bb3c     OutputWnd.obj
 0002:00019b58       ??_R4CPartitionSettingDlg@@6B@ 0049bb58     PartitionSettingDlg.obj
 0002:00019b6c       ??_R3CPartitionSettingDlg@@8 0049bb6c     PartitionSettingDlg.obj
 0002:00019b7c       ??_R2CPartitionSettingDlg@@8 0049bb7c     PartitionSettingDlg.obj
 0002:00019b94       ??_R1A@?0A@EA@CPartitionSettingDlg@@8 0049bb94     PartitionSettingDlg.obj
 0002:00019bb0       ??_R4CPortChannelDlg@@6B@  0049bbb0     PortChannelDlg.obj
 0002:00019bc4       ??_R3CPortChannelDlg@@8    0049bbc4     PortChannelDlg.obj
 0002:00019bd4       ??_R2CPortChannelDlg@@8    0049bbd4     PortChannelDlg.obj
 0002:00019bec       ??_R1A@?0A@EA@CPortChannelDlg@@8 0049bbec     PortChannelDlg.obj
 0002:00019c08       ??_R4CPortCtrlDlg@@6B@     0049bc08     PortCtrlDlg.obj
 0002:00019c1c       ??_R3CPortCtrlDlg@@8       0049bc1c     PortCtrlDlg.obj
 0002:00019c2c       ??_R2CPortCtrlDlg@@8       0049bc2c     PortCtrlDlg.obj
 0002:00019c44       ??_R1A@?0A@EA@CPortCtrlDlg@@8 0049bc44     PortCtrlDlg.obj
 0002:00019c60       ??_R4CPrivateProfileFile@@6B@ 0049bc60     PrivateProfileFile.obj
 0002:00019c74       ??_R3CPrivateProfileFile@@8 0049bc74     PrivateProfileFile.obj
 0002:00019c84       ??_R2CPrivateProfileFile@@8 0049bc84     PrivateProfileFile.obj
 0002:00019c8c       ??_R1A@?0A@EA@CPrivateProfileFile@@8 0049bc8c     PrivateProfileFile.obj
 0002:00019ca8       ??_R4CProgressDlg@@6B@     0049bca8     ProgressDlg.obj
 0002:00019cbc       ??_R3CProgressDlg@@8       0049bcbc     ProgressDlg.obj
 0002:00019ccc       ??_R2CProgressDlg@@8       0049bccc     ProgressDlg.obj
 0002:00019ce4       ??_R1A@?0A@EA@CProgressDlg@@8 0049bce4     ProgressDlg.obj
 0002:00019d00       ??_R4CProgressCtrl@@6B@    0049bd00     ProgressDlg.obj
 0002:00019d14       ??_R3CProgressCtrl@@8      0049bd14     ProgressDlg.obj
 0002:00019d24       ??_R2CProgressCtrl@@8      0049bd24     ProgressDlg.obj
 0002:00019d38       ??_R1A@?0A@EA@CProgressCtrl@@8 0049bd38     ProgressDlg.obj
 0002:00019d54       ??_R4CPropertyViewDlg@@6B@ 0049bd54     PropertyViewDlg.obj
 0002:00019d68       ??_R3CPropertyViewDlg@@8   0049bd68     PropertyViewDlg.obj
 0002:00019d78       ??_R2CPropertyViewDlg@@8   0049bd78     PropertyViewDlg.obj
 0002:00019d90       ??_R1A@?0A@EA@CPropertyViewDlg@@8 0049bd90     PropertyViewDlg.obj
 0002:00019dac       ??_R4CTabCtrl@@6B@         0049bdac     PropertyViewDlg.obj
 0002:00019dc0       ??_R3CTabCtrl@@8           0049bdc0     PropertyViewDlg.obj
 0002:00019dd0       ??_R2CTabCtrl@@8           0049bdd0     PropertyViewDlg.obj
 0002:00019de4       ??_R1A@?0A@EA@CTabCtrl@@8  0049bde4     PropertyViewDlg.obj
 0002:00019e00       ??_R4CPropertyViewUIThread@@6B@ 0049be00     PropertyViewUIThread.obj
 0002:00019e14       ??_R3CPropertyViewUIThread@@8 0049be14     PropertyViewUIThread.obj
 0002:00019e24       ??_R2CPropertyViewUIThread@@8 0049be24     PropertyViewUIThread.obj
 0002:00019e38       ??_R1A@?0A@EA@CPropertyViewUIThread@@8 0049be38     PropertyViewUIThread.obj
 0002:00019e54       ??_R4CReportCtrl@@6B@      0049be54     ReportCtrl.obj
 0002:00019e68       ??_R3CReportCtrl@@8        0049be68     ReportCtrl.obj
 0002:00019e78       ??_R2CReportCtrl@@8        0049be78     ReportCtrl.obj
 0002:00019e90       ??_R1A@?0A@EA@CReportCtrl@@8 0049be90     ReportCtrl.obj
 0002:00019eac       ??_R4?$CArray@KK@@6B@      0049beac     ReportCtrl.obj
 0002:00019ec0       ??_R3?$CArray@KK@@8        0049bec0     ReportCtrl.obj
 0002:00019ed0       ??_R2?$CArray@KK@@8        0049bed0     ReportCtrl.obj
 0002:00019edc       ??_R1A@?0A@EA@?$CArray@KK@@8 0049bedc     ReportCtrl.obj
 0002:00019ef8       ??_R4?$CArray@HH@@6B@      0049bef8     ReportCtrl.obj
 0002:00019f0c       ??_R3?$CArray@HH@@8        0049bf0c     ReportCtrl.obj
 0002:00019f1c       ??_R2?$CArray@HH@@8        0049bf1c     ReportCtrl.obj
 0002:00019f28       ??_R1A@?0A@EA@?$CArray@HH@@8 0049bf28     ReportCtrl.obj
 0002:00019f44       ??_R4CSetClientchancelDLg@@6B@ 0049bf44     SetClientchancelDLg.obj
 0002:00019f58       ??_R3CSetClientchancelDLg@@8 0049bf58     SetClientchancelDLg.obj
 0002:00019f68       ??_R2CSetClientchancelDLg@@8 0049bf68     SetClientchancelDLg.obj
 0002:00019f80       ??_R1A@?0A@EA@CSetClientchancelDLg@@8 0049bf80     SetClientchancelDLg.obj
 0002:00019f9c       ??_R4CSetDrfaultNICDlg@@6B@ 0049bf9c     SetDrfaultNICDlg.obj
 0002:00019fb0       ??_R3CSetDrfaultNICDlg@@8  0049bfb0     SetDrfaultNICDlg.obj
 0002:00019fc0       ??_R2CSetDrfaultNICDlg@@8  0049bfc0     SetDrfaultNICDlg.obj
 0002:00019fd8       ??_R1A@?0A@EA@CSetDrfaultNICDlg@@8 0049bfd8     SetDrfaultNICDlg.obj
 0002:00019ff4       ??_R4CSpecialPartitionRS@@6B@ 0049bff4     SpecialPartitionRS.obj
 0002:0001a008       ??_R3CSpecialPartitionRS@@8 0049c008     SpecialPartitionRS.obj
 0002:0001a018       ??_R2CSpecialPartitionRS@@8 0049c018     SpecialPartitionRS.obj
 0002:0001a030       ??_R1A@?0A@EA@CSpecialPartitionRS@@8 0049c030     SpecialPartitionRS.obj
 0002:0001a04c       ??_R4CWait@@6B@            0049c04c     Wait.obj
 0002:0001a060       ??_R3CWait@@8              0049c060     Wait.obj
 0002:0001a070       ??_R2CWait@@8              0049c070     Wait.obj
 0002:0001a088       ??_R1A@?0A@EA@CWait@@8     0049c088     Wait.obj
 0002:0001a0a4       ??_R4CWorkspaceBar@@6B@    0049c0a4     WorkspaceBar.obj
 0002:0001a0b8       ??_R3CWorkspaceBar@@8      0049c0b8     WorkspaceBar.obj
 0002:0001a0c8       ??_R2CWorkspaceBar@@8      0049c0c8     WorkspaceBar.obj
 0002:0001a0e8       ??_R1A@?0A@EA@CWorkspaceBar@@8 0049c0e8     WorkspaceBar.obj
 0002:0001a104       ??_R4CWorkspaceBar2@@6B@   0049c104     WorkspaceBar2.obj
 0002:0001a118       ??_R3CWorkspaceBar2@@8     0049c118     WorkspaceBar2.obj
 0002:0001a128       ??_R2CWorkspaceBar2@@8     0049c128     WorkspaceBar2.obj
 0002:0001a148       ??_R1A@?0A@EA@CWorkspaceBar2@@8 0049c148     WorkspaceBar2.obj
 0002:0001a164       ??_R3?$_CTypedPtrList@VCPtrList@@PAUtagUDPRECV@@@@8 0049c164     commod2:MulticastSocket.obj
 0002:0001a174       ??_R2?$_CTypedPtrList@VCPtrList@@PAUtagUDPRECV@@@@8 0049c174     commod2:MulticastSocket.obj
 0002:0001a184       ??_R1A@?0A@EA@?$_CTypedPtrList@VCPtrList@@PAUtagUDPRECV@@@@8 0049c184     commod2:MulticastSocket.obj
 0002:0001a1a0       ??_R4?$CTypedPtrList@VCPtrList@@PAUtagUDPRECV@@@@6B@ 0049c1a0     commod2:MulticastSocket.obj
 0002:0001a1b4       ??_R3?$CTypedPtrList@VCPtrList@@PAUtagUDPRECV@@@@8 0049c1b4     commod2:MulticastSocket.obj
 0002:0001a1c4       ??_R2?$CTypedPtrList@VCPtrList@@PAUtagUDPRECV@@@@8 0049c1c4     commod2:MulticastSocket.obj
 0002:0001a1d8       ??_R1A@?0A@EA@?$CTypedPtrList@VCPtrList@@PAUtagUDPRECV@@@@8 0049c1d8     commod2:MulticastSocket.obj
 0002:0001a1f4       ??_R4CMulticastSocket@@6B@ 0049c1f4     commod2:MulticastSocket.obj
 0002:0001a208       ??_R3CMulticastSocket@@8   0049c208     commod2:MulticastSocket.obj
 0002:0001a218       ??_R2CMulticastSocket@@8   0049c218     commod2:MulticastSocket.obj
 0002:0001a220       ??_R1A@?0A@EA@CMulticastSocket@@8 0049c220     commod2:MulticastSocket.obj
 0002:0001a23c       ??_R4CODBCSet@@6B@         0049c23c     dbmod2:MyODBC.obj
 0002:0001a250       ??_R3CODBCSet@@8           0049c250     dbmod2:MyODBC.obj
 0002:0001a260       ??_R2CODBCSet@@8           0049c260     dbmod2:MyODBC.obj
 0002:0001a268       ??_R1A@?0A@EA@CODBCSet@@8  0049c268     dbmod2:MyODBC.obj
 0002:0001a284       ??_R4CMyODBC@@6B@          0049c284     dbmod2:MyODBC.obj
 0002:0001a298       ??_R3?$_CTypedPtrList@VCPtrList@@PAUSTRUCT_PROTECTITEM@@@@8 0049c298     kibokern:kibokern.obj
 0002:0001a2a8       ??_R2?$_CTypedPtrList@VCPtrList@@PAUSTRUCT_PROTECTITEM@@@@8 0049c2a8     kibokern:kibokern.obj
 0002:0001a2b8       ??_R1A@?0A@EA@?$_CTypedPtrList@VCPtrList@@PAUSTRUCT_PROTECTITEM@@@@8 0049c2b8     kibokern:kibokern.obj
 0002:0001a2d4       ??_R4?$CTypedPtrList@VCPtrList@@PAUSTRUCT_PROTECTITEM@@@@6B@ 0049c2d4     kibokern:kibokern.obj
 0002:0001a2e8       ??_R3?$CTypedPtrList@VCPtrList@@PAUSTRUCT_PROTECTITEM@@@@8 0049c2e8     kibokern:kibokern.obj
 0002:0001a2f8       ??_R2?$CTypedPtrList@VCPtrList@@PAUSTRUCT_PROTECTITEM@@@@8 0049c2f8     kibokern:kibokern.obj
 0002:0001a30c       ??_R1A@?0A@EA@?$CTypedPtrList@VCPtrList@@PAUSTRUCT_PROTECTITEM@@@@8 0049c30c     kibokern:kibokern.obj
 0002:0001a328       ??_R4CKiboKern@@6B@        0049c328     kibokern:kibokern.obj
 0002:0001a33c       ??_R3CKiboKern@@8          0049c33c     kibokern:kibokern.obj
 0002:0001a34c       ??_R2CKiboKern@@8          0049c34c     kibokern:kibokern.obj
 0002:0001a354       ??_R1A@?0A@EA@CKiboKern@@8 0049c354     kibokern:kibokern.obj
 0002:0001a370       ??_R4type_info@@6B@        0049c370     msvcrt:ti_inst.obj
 0002:0001a384       ??_R3type_info@@8          0049c384     msvcrt:ti_inst.obj
 0002:0001a394       ??_R2type_info@@8          0049c394     msvcrt:ti_inst.obj
 0002:0001a39c       ??_R1A@?0A@EA@type_info@@8 0049c39c     msvcrt:ti_inst.obj
 0002:0001a3c0       ___safe_se_handler_table   0049c3c0     <linker-defined>
 0002:0001a920       ___rtc_iaa                 0049c920     msvcrt:_initsect_.obj
 0002:0001a924       ___rtc_izz                 0049c924     msvcrt:_initsect_.obj
 0002:0001a928       ___rtc_taa                 0049c928     msvcrt:_initsect_.obj
 0002:0001a92c       ___rtc_tzz                 0049c92c     msvcrt:_initsect_.obj
 0002:0001aca8       __TI4PAVCBlockingSocketException@@ 0049cca8     blocksock.obj
 0002:0001ace4       __CTA4PAVCBlockingSocketException@@ 0049cce4     blocksock.obj
 0002:0001acf8       __CT??_R0PAVCBlockingSocketException@@@84 0049ccf8     blocksock.obj
 0002:0001ad14       __CT??_R0PAVCException@@@84 0049cd14     blocksock.obj
 0002:0001ad30       __CT??_R0PAVCObject@@@84   0049cd30     blocksock.obj
 0002:0001ad4c       __CT??_R0PAX@84            0049cd4c     blocksock.obj
 0002:0001d54c       __CT??_R0?AVlogic_error@std@@@8??0logic_error@std@@QAE@ABV01@@Z40 0049f54c     KiboManagerView.obj
 0002:0001d568       __CT??_R0?AVexception@std@@@8??0exception@std@@QAE@ABV01@@Z12 0049f568     KiboManagerView.obj
 0002:0001d5b0       __TI3?AVlength_error@std@@ 0049f5b0     KiboManagerView.obj
 0002:0001d5c0       __CTA3?AVlength_error@std@@ 0049f5c0     KiboManagerView.obj
 0002:0001d5d0       __CT??_R0?AVlength_error@std@@@8??0length_error@std@@QAE@ABV01@@Z40 0049f5d0     KiboManagerView.obj
 0002:0001d5ec       __TI2?AVbad_alloc@std@@    0049f5ec     KiboManagerView.obj
 0002:0001d5fc       __CTA2?AVbad_alloc@std@@   0049f5fc     KiboManagerView.obj
 0002:0001d608       __CT??_R0?AVbad_alloc@std@@@8??0bad_alloc@std@@QAE@ABV01@@Z12 0049f608     KiboManagerView.obj
 0002:00022684       __TI1?AV_com_error@@       004a4684     comsuppw:comraise.obj
 0002:00022694       __CTA1?AV_com_error@@      004a4694     comsuppw:comraise.obj
 0002:0002269c       __CT??_R0?AV_com_error@@@8??0_com_error@@QAE@ABV0@@Z16 004a469c     comsuppw:comraise.obj
 0002:000226b8       __DELAY_IMPORT_DESCRIPTOR_dwmapi_dll 004a46b8     dwmapi:dwmapi.dll
 0002:000226d8       __NULL_DELAY_IMPORT_DESCRIPTOR 004a46d8     dwmapi:dwmapi.dll
 0002:000226fc       \177dwmapi_NULL_THUNK_DATA_DLN 004a46fc     dwmapi:dwmapi.dll
 0002:00022704       \177dwmapi_NULL_THUNK_DATA_DLB 004a4704     dwmapi:dwmapi.dll
 0002:00022708       __IMPORT_DESCRIPTOR_RCLogSystem 004a4708     RCLogSystem:RCLogSystem.dll
 0002:0002271c       __IMPORT_DESCRIPTOR_diskop 004a471c     diskop:diskop.dll
 0002:00022730       __IMPORT_DESCRIPTOR_WTSAPI32 004a4730     WtsApi32:WTSAPI32.dll
 0002:00022744       __IMPORT_DESCRIPTOR_mfc90  004a4744     mfc90:mfc90.dll
 0002:00022758       __IMPORT_DESCRIPTOR_MSVCR90 004a4758     msvcrt:MSVCR90.dll
 0002:0002276c       __IMPORT_DESCRIPTOR_KERNEL32 004a476c     kernel32:KERNEL32.dll
 0002:00022780       __IMPORT_DESCRIPTOR_USER32 004a4780     user32:USER32.dll
 0002:00022794       __IMPORT_DESCRIPTOR_GDI32  004a4794     gdi32:GDI32.dll
 0002:000227a8       __IMPORT_DESCRIPTOR_ADVAPI32 004a47a8     advapi32:ADVAPI32.dll
 0002:000227bc       __IMPORT_DESCRIPTOR_SHELL32 004a47bc     shell32:SHELL32.dll
 0002:000227d0       __IMPORT_DESCRIPTOR_COMCTL32 004a47d0     comctl32:COMCTL32.dll
 0002:000227e4       __IMPORT_DESCRIPTOR_OLEAUT32 004a47e4     oleaut32:OLEAUT32.dll
 0002:000227f8       __IMPORT_DESCRIPTOR_gdiplus 004a47f8     gdiplus:gdiplus.dll
 0002:0002280c       __IMPORT_DESCRIPTOR_MSVCP90 004a480c     msvcprt:MSVCP90.dll
 0002:00022820       __IMPORT_DESCRIPTOR_WSOCK32 004a4820     wsock32:WSOCK32.dll
 0002:00022834       __IMPORT_DESCRIPTOR_WS2_32 004a4834     WS2_32:WS2_32.dll
 0002:00022848       __IMPORT_DESCRIPTOR_changeip 004a4848     changeip:changeip.dll
 0002:0002285c       __IMPORT_DESCRIPTOR_ODBC32 004a485c     odbc32:ODBC32.dll
 0002:00022870       __IMPORT_DESCRIPTOR_windisk 004a4870     windisk:windisk.dll
 0002:00022884       __IMPORT_DESCRIPTOR_VERSION 004a4884     Version:VERSION.dll
 0002:00022898       __IMPORT_DESCRIPTOR_HTSAPI 004a4898     htsapi:HTSAPI.dll
 0002:000228ac       __IMPORT_DESCRIPTOR_IPHLPAPI 004a48ac     Iphlpapi:IPHLPAPI.DLL
 0002:000228c0       __NULL_IMPORT_DESCRIPTOR   004a48c0     usbdog:usbdog.dll
 0003:00000000       ?gbtime@@3PADA             004a7000     AboutDlg.obj
 0003:00000014       ?Version@@3PADA            004a7014     AboutDlg.obj
 0003:00000028       ??_R0?AVCAboutDlg@@@8      004a7028     AboutDlg.obj
 0003:00000040       ??_R0?AVCDialog@@@8        004a7040     AboutDlg.obj
 0003:00000058       ??_R0?AVCWnd@@@8           004a7058     AboutDlg.obj
 0003:0000006c       ??_R0?AVCCmdTarget@@@8     004a706c     AboutDlg.obj
 0003:00000088       ??_R0?AVCObject@@@8        004a7088     AboutDlg.obj
 0003:000000a0       ??_R0?AVCStatic@@@8        004a70a0     AboutDlg.obj
 0003:000000b8       ??_R0?AVCAddToGroup@@@8    004a70b8     AddToGroup.obj
 0003:000000d4       ??_R0?AVCComboBox@@@8      004a70d4     AddToGroup.obj
 0003:000000ec       ??_R0?AVCBlackListDlg@@@8  004a70ec     BlackListDlg.obj
 0003:00000108       ??_R0?AVCListCtrl@@@8      004a7108     BlackListDlg.obj
 0003:00000120       ??_R0?AVCBlockingSocketException@@@8 004a7120     blocksock.obj
 0003:00000148       ??_R0?AVCException@@@8     004a7148     blocksock.obj
 0003:00000164       ??_R0PAVCBlockingSocketException@@@8 004a7164     blocksock.obj
 0003:0000018c       ??_R0PAVCException@@@8     004a718c     blocksock.obj
 0003:000001a8       ??_R0PAVCObject@@@8        004a71a8     blocksock.obj
 0003:000001c0       ??_R0PAX@8                 004a71c0     blocksock.obj
 0003:000001d0       ??_R0?AVCBlockingSocket@@@8 004a71d0     blocksock.obj
 0003:000001f0       ??_R0?AVCBootModuleManager@@@8 004a71f0     BootModuleManager.obj
 0003:00000214       ??_R0?AV?$CTypedPtrList@VCPtrList@@PAK@@@8 004a7214     BootModuleManager.obj
 0003:00000244       ??_R0?AV?$_CTypedPtrList@VCPtrList@@PAK@@@8 004a7244     BootModuleManager.obj
 0003:00000274       ??_R0?AVCPtrList@@@8       004a7274     BootModuleManager.obj
 0003:0000028c       ??_R0?AVCCriticalSection@@@8 004a728c     BootModuleManager.obj
 0003:000002ac       ??_R0?AVCSyncObject@@@8    004a72ac     BootModuleManager.obj
 0003:000002c8       ??_R0?AVCBroadIE@@@8       004a72c8     BroadIE.obj
 0003:000002e0       ??_R0?AVCBroadWaitDlg@@@8  004a72e0     BroadWaitDlg.obj
 0003:000002fc       ??_R0?AVCCalendarBar@@@8   004a72fc     CalendarBar.obj
 0003:00000318       ??_R0?AVCBitmap@@@8        004a7318     CalendarBar.obj
 0003:00000330       ??_R0?AVCGdiObject@@@8     004a7330     CalendarBar.obj
 0003:0000034c       ??_R0?AVCMonthCalCtrl@@@8  004a734c     CalendarBar.obj
 0003:00000368       ??_R0?AVCFtpd@@@8          004a7368     CFtpd.obj
 0003:0000037c       ??_R0?AVCSocket@@@8        004a737c     CFtpd.obj
 0003:00000394       ??_R0?AVCAsyncSocket@@@8   004a7394     CFtpd.obj
 0003:000003b0       ??_R0?AV?$CList@PAVCFtpdPi@@PAV1@@@@8 004a73b0     CFtpd.obj
 0003:000003d8       ??_R0?AVCCheckPasswordDlg@@@8 004a73d8     CheckPasswordDlg.obj
 0003:000003f8       ??_R0?AVCEdit@@@8          004a73f8     CheckPasswordDlg.obj
 0003:0000040c       ??_R0?AVCClientInfoManager@@@8 004a740c     ClientInfoManager.obj
 0003:00000430       ??_R0?AV?$CTypedPtrMap@VCMapStringToPtr@@V?$CStringT@DV?$StrTraitMFC_DLL@DV?$ChTraitsCRT@D@ATL@@@@@ATL@@PAUtagCLIENTMAININFO@@@@@8 004a7430     ClientInfoManager.obj
 0003:000004b8       ??_R0?AVCMapStringToPtr@@@8 004a74b8     ClientInfoManager.obj
 0003:000004d8       ??_R0?AV?$CTypedPtrMap@VCMapStringToPtr@@V?$CStringT@DV?$StrTraitMFC_DLL@DV?$ChTraitsCRT@D@ATL@@@@@ATL@@PAUtagBLACKLIST@@@@@8 004a74d8     ClientInfoManager.obj
 0003:00000558       ??_R0?AV?$CTypedPtrMap@VCMapStringToPtr@@V?$CStringT@DV?$StrTraitMFC_DLL@DV?$ChTraitsCRT@D@ATL@@@@@ATL@@PAVCStringList@@@@@8 004a7558     ClientInfoManager.obj
 0003:000005d8       ??_R0?AVCClientSettingsDlg@@@8 004a75d8     ClientSettingsDlg.obj
 0003:000005fc       ??_R0?AVCSpinButtonCtrl@@@8 004a75fc     ClientSettingsDlg.obj
 0003:0000061c       ??_R0?AVCCmdEnquireDlg@@@8 004a761c     CmdEnquireDlg.obj
 0003:0000063c       ??_R0?AVCButton@@@8        004a763c     CmdEnquireDlg.obj
 0003:00000654       ??_R0?AVCExecuteProcedure@@@8 004a7654     ExecuteProcedure.obj
 0003:00000674       ??_R0?AVCFont@@@8          004a7674     FontStatic.obj
 0003:00000688       ??_R0?AVCFtpPasvSrv@@@8    004a7688     FtpdPasvSrv.obj
 0003:000006a4       ??_R0?AVCFtpdPi@@@8        004a76a4     FtpdPi.obj
 0003:000006bc       ??_R0?AVCGroupExt@@@8      004a76bc     GroupExt.obj
 0003:000006d4       ??_R0?AVCGroupTree@@@8     004a76d4     GroupTree.obj
 0003:000006f0       ??_R0?AVCTreeCtrl@@@8      004a76f0     GroupTree.obj
 0003:00000708       ??_R0?AVCMenu@@@8          004a7708     GroupTree.obj
 0003:0000071c       ??_R0?AVCInfoPromptDlg@@@8 004a771c     InfoPromptDlg.obj
 0003:0000073c       ??_R0?AVCIOCPImplement@@@8 004a773c     IOCPImplement.obj
 0003:0000075c       ??_R0?AVCMyIOCP@@@8        004a775c     IOCPImplement.obj
 0003:00000778       ??_R0?AV?$CTypedPtrMap@VCMapPtrToPtr@@PAVCClientContext@@PAUIOCP_DataRecvBuffer@@@@@8 004a7778     IOCPImplement.obj
 0003:000007d0       ??_R0?AVCMapPtrToPtr@@@8   004a77d0     IOCPImplement.obj
 0003:000007ec       ??_R0?AVCKiboManagerApp@@@8 004a77ec     KiboManager.obj
 0003:0000080c       ??_R0?AVCWinAppEx@@@8      004a780c     KiboManager.obj
 0003:00000824       ??_R0?AVCWinApp@@@8        004a7824     KiboManager.obj
 0003:0000083c       ??_R0?AVCWinThread@@@8     004a783c     KiboManager.obj
 0003:00000858       ??_R0?AVCKiboManagerDoc@@@8 004a7858     KiboManagerDoc.obj
 0003:00000878       ??_R0?AVCDocument@@@8      004a7878     KiboManagerDoc.obj
 0003:00000890       ??_R0?AVCKiboManagerView@@@8 004a7890     KiboManagerView.obj
 0003:000008b0       ??_R0?AVCFormView@@@8      004a78b0     KiboManagerView.obj
 0003:000008c8       ??_R0?AVCScrollView@@@8    004a78c8     KiboManagerView.obj
 0003:000008e4       ??_R0?AVCView@@@8          004a78e4     KiboManagerView.obj
 0003:000008f8       ??_R0?AVlogic_error@std@@@8 004a78f8     KiboManagerView.obj
 0003:00000918       ??_R0?AVexception@std@@@8  004a7918     KiboManagerView.obj
 0003:00000934       ??_R0?AVlength_error@std@@@8 004a7934     KiboManagerView.obj
 0003:00000954       ??_R0?AVbad_alloc@std@@@8  004a7954     KiboManagerView.obj
 0003:00000970       ??_R0?AVCLenPropertyODBC@@@8 004a7970     LenPropertyODBC.obj
 0003:00000990       ??_R0?AVCMyODBC@@@8        004a7990     LenPropertyODBC.obj
 0003:000009a8       ??_R0?AVCNewListCtrl@@@8   004a79a8     ListCtrlEx.obj
 0003:000009c4       ??_R0?AVCLoginPasswordDlg@@@8 004a79c4     LoginPasswordDlg.obj
 0003:000009e4       ??_R0?AVCMainFrame@@@8     004a79e4     MainFrm.obj
 0003:00000a00       ??_R0?AVCFrameWndEx@@@8    004a7a00     MainFrm.obj
 0003:00000a1c       ??_R0?AVCFrameWnd@@@8      004a7a1c     MainFrm.obj
 0003:00000a34       ??_R0?AVCOutlookBar@@@8    004a7a34     MainFrm.obj
 0003:00000a50       ??_R0?AVCMFCOutlookBar@@@8 004a7a50     MainFrm.obj
 0003:00000a70       ??_R0?AVCBaseTabbedPane@@@8 004a7a70     MainFrm.obj
 0003:00000a90       ??_R0?AVCDockablePane@@@8  004a7a90     MainFrm.obj
 0003:00000aac       ??_R0?AVCPane@@@8          004a7aac     MainFrm.obj
 0003:00000ac0       ??_R0?AVCBasePane@@@8      004a7ac0     MainFrm.obj
 0003:00000ad8       ??_R0?AV?$CTypedPtrList@VCPtrList@@PAUtagRECVREQUEST@@@@@8 004a7ad8     MainFrm.obj
 0003:00000b18       ??_R0?AV?$_CTypedPtrList@VCPtrList@@PAUtagRECVREQUEST@@@@@8 004a7b18     MainFrm.obj
 0003:00000b58       ??_R0?AV?$CTypedPtrList@VCPtrList@@PAUPartitionTransInfo@@@@@8 004a7b58     MainFrm.obj
 0003:00000ba0       ??_R0?AV?$_CTypedPtrList@VCPtrList@@PAUPartitionTransInfo@@@@@8 004a7ba0     MainFrm.obj
 0003:00000be8       ??_R0?AV?$CTypedPtrMap@VCMapStringToPtr@@V?$CStringT@DV?$StrTraitMFC_DLL@DV?$ChTraitsCRT@D@ATL@@@@@ATL@@PAV23@@@@8 004a7be8     MainFrm.obj
 0003:00000c60       ??_R0?AV?$CList@II@@@8     004a7c60     MainFrm.obj
 0003:00000c7c       ??_R0?AV?$CList@PAVCFtpd@@PAV1@@@@8 004a7c7c     MainFrm.obj
 0003:00000ca4       ??_R0?AVCMFCRibbonApplicationButton@@@8 004a7ca4     MainFrm.obj
 0003:00000cd0       ??_R0?AVCMFCRibbonButton@@@8 004a7cd0     MainFrm.obj
 0003:00000cf0       ??_R0?AVCMFCRibbonBaseElement@@@8 004a7cf0     MainFrm.obj
 0003:00000d18       ??_R0?AV?$CMap@V?$CStringT@DV?$StrTraitMFC_DLL@DV?$ChTraitsCRT@D@ATL@@@@@ATL@@PBDUItemInfo@@AAU3@@@@8 004a7d18     MainFrm.obj
 0003:00000d80       ??_R0?AVCMFCRibbonBarNew@@@8 004a7d80     MFCRibbonBarNew.obj
 0003:00000da0       ??_R0?AVCMFCRibbonBar@@@8  004a7da0     MFCRibbonBarNew.obj
 0003:00000dbc       ??_R0?AVCModifyGroup@@@8   004a7dbc     ModifyGroup.obj
 0003:00000dd8       ??_R0?AVCMsgDlg@@@8        004a7dd8     MsgDlg.obj
 0003:00000df0       ??_R0?AVCMyEdit@@@8        004a7df0     MyEdit.obj
 0003:00000e08       ??_R0?AVCMyPropertyPage1@@@8 004a7e08     MyPropertyPage1.obj
 0003:00000e28       ??_R0?AVCMFCPropertyPage@@@8 004a7e28     MyPropertyPage1.obj
 0003:00000e48       ??_R0?AVCPropertyPage@@@8  004a7e48     MyPropertyPage1.obj
 0003:00000e64       ??_R0?AVCMyPropertyPage2@@@8 004a7e64     MyPropertyPage1.obj
 0003:00000e84       ??_R0?AVCMyPropertyPage3@@@8 004a7e84     MyPropertyPage1.obj
 0003:00000ea4       ??_R0?AVCMyPropertySheet@@@8 004a7ea4     MyPropertySheet.obj
 0003:00000ec4       ??_R0?AVCMFCPropertySheet@@@8 004a7ec4     MyPropertySheet.obj
 0003:00000ee4       ??_R0?AVCPropertySheet@@@8 004a7ee4     MyPropertySheet.obj
 0003:00000f04       ??_R0?AVCMyRichEdit@@@8    004a7f04     MyRichEdit.obj
 0003:00000f20       ??_R0?AVCRichEditCtrl@@@8  004a7f20     MyRichEdit.obj
 0003:00000f3c       ??_R0?AVCBrush@@@8         004a7f3c     NewListCtrl.obj
 0003:00000f54       ??_R0?AVCOutputWnd@@@8     004a7f54     OutputWnd.obj
 0003:00000f70       ??_R0?AVCOutputList@@@8    004a7f70     OutputWnd.obj
 0003:00000f90       ?StrArray1@@3PAPADA        004a7f90     PartitionSettingDlg.obj
 0003:00000fa0       ?StrArray2@@3PAPADA        004a7fa0     PartitionSettingDlg.obj
 0003:00001020       ?StrArray3@@3PAPADA        004a8020     PartitionSettingDlg.obj
 0003:00001030       ?StrArray4@@3PAPADA        004a8030     PartitionSettingDlg.obj
 0003:000010a8       ??_R0?AVCPartitionSettingDlg@@@8 004a80a8     PartitionSettingDlg.obj
 0003:000010cc       ??_R0?AVCPortChannelDlg@@@8 004a80cc     PortChannelDlg.obj
 0003:000010ec       ??_R0?AVCPortCtrlDlg@@@8   004a80ec     PortCtrlDlg.obj
 0003:00001108       ??_R0?AVCPrivateProfileFile@@@8 004a8108     PrivateProfileFile.obj
 0003:0000112c       ??_R0?AVCProgressDlg@@@8   004a812c     ProgressDlg.obj
 0003:00001148       ??_R0?AVCProgressCtrl@@@8  004a8148     ProgressDlg.obj
 0003:00001164       ??_R0?AVCPropertyViewDlg@@@8 004a8164     PropertyViewDlg.obj
 0003:00001184       ??_R0?AVCTabCtrl@@@8       004a8184     PropertyViewDlg.obj
 0003:0000119c       ??_R0?AVCPropertyViewUIThread@@@8 004a819c     PropertyViewUIThread.obj
 0003:000011c0       ??_R0?AVCReportCtrl@@@8    004a81c0     ReportCtrl.obj
 0003:000011dc       ??_R0?AV?$CArray@KK@@@8    004a81dc     ReportCtrl.obj
 0003:000011f8       ??_R0?AV?$CArray@HH@@@8    004a81f8     ReportCtrl.obj
 0003:00001214       ??_R0?AVCSetClientchancelDLg@@@8 004a8214     SetClientchancelDLg.obj
 0003:00001238       ??_R0?AVCSetDrfaultNICDlg@@@8 004a8238     SetDrfaultNICDlg.obj
 0003:00001258       ??_R0?AVCSpecialPartitionRS@@@8 004a8258     SpecialPartitionRS.obj
 0003:00001280       ??_R0?AVCWait@@@8          004a8280     Wait.obj
 0003:00001294       ??_R0?AVCWorkspaceBar@@@8  004a8294     WorkspaceBar.obj
 0003:000012b0       ??_R0?AVCWorkspaceBar2@@@8 004a82b0     WorkspaceBar2.obj
 0003:00001310       ??_R0?AV?$_CTypedPtrList@VCPtrList@@PAUtagUDPRECV@@@@@8 004a8310     commod2:MulticastSocket.obj
 0003:0000134c       ??_R0?AV?$CTypedPtrList@VCPtrList@@PAUtagUDPRECV@@@@@8 004a834c     commod2:MulticastSocket.obj
 0003:00001388       ??_R0?AVCMulticastSocket@@@8 004a8388     commod2:MulticastSocket.obj
 0003:000013a8       ??_R0?AVCODBCSet@@@8       004a83a8     dbmod2:MyODBC.obj
 0003:000013c0       ?encrypt_key@@3PADA        004a83c0     kibokern:kibokern.obj
 0003:000013d0       ??_R0?AV?$_CTypedPtrList@VCPtrList@@PAUSTRUCT_PROTECTITEM@@@@@8 004a83d0     kibokern:kibokern.obj
 0003:00001418       ??_R0?AV?$CTypedPtrList@VCPtrList@@PAUSTRUCT_PROTECTITEM@@@@@8 004a8418     kibokern:kibokern.obj
 0003:0000145c       ??_R0?AVCKiboKern@@@8      004a845c     kibokern:kibokern.obj
 0003:00001474       ___security_cookie         004a8474     msvcrt:gs_cookie.obj
 0003:00001478       ___security_cookie_complement 004a8478     msvcrt:gs_cookie.obj
 0003:0000147c       ??_R0?AVtype_info@@@8      004a847c     msvcrt:ti_inst.obj
 0003:000014a0       ___native_dllmain_reason   004a84a0     msvcrt:natstart.obj
 0003:000014a4       ___native_vcclrit_reason   004a84a4     msvcrt:natstart.obj
 0003:000014a8       ___globallocalestatus      004a84a8     msvcrt:xthdloc.obj
 0003:000014ac       ___defaultmatherr          004a84ac     msvcrt:merr.obj
 0003:000014b0       ?vtMissing@@3V_variant_t@@A 004a84b0     comsuppw:comutil.obj
 0003:000014c0       ?__errorPfn@@3P6GXJPAUIErrorInfo@@@ZA 004a84c0     comsuppw:comsupp.obj
 0003:000014c4       ??_R0?AV_com_error@@@8     004a84c4     comsuppw:comraise.obj
 0003:000014e4       __imp__DwmEnableComposition@4 004a84e4     dwmapi:dwmapi.dll
 0003:000014e8       \177dwmapi_NULL_THUNK_DATA_DLA 004a84e8     dwmapi:dwmapi.dll
 0003:000014f0       ?lpsockftpd@@3Usockaddr_in@@A 004a84f0     CFtpd.obj
 0003:00001500       ?lpTranslate@@3PAULANGANDCODEPAGE@@A 004a8500     CommonFunc.obj
 0003:00001504       ?istip@@3HA                004a8504     CommonFunc.obj
 0003:00001508       ?sadr@@3PADA               004a8508     FtpdPasvSrv.obj
 0003:00001528       ?sadr2@@3PADA              004a8528     FtpdPi.obj
 0003:00001548       ?bIsRButton@@3HA           004a8548     GroupTree.obj
 0003:00001550       ?g_winVer@@3KA             004a8550     KiboManager.obj
 0003:00001554       ?g_mainPwd@@3V?$CStringT@DV?$StrTraitMFC_DLL@DV?$ChTraitsCRT@D@ATL@@@@@ATL@@A 004a8554     KiboManager.obj
 0003:00001558       ?theApp@@3VCKiboManagerApp@@A 004a8558     KiboManager.obj
 0003:0000164c       ?g_pMainView@@3PAVCKiboManagerView@@A 004a864c     KiboManagerView.obj
 0003:00001650       ?chCpName@@3PADA           004a8650     KiboManagerView.obj
 0003:00001670       ?isViewPt@@3HA             004a8670     KiboManagerView.obj
 0003:00001674       ?g_nType@@3HA              004a8674     MainDlg.obj
 0003:00001678       ?g_nFirstFocus@@3HA        004a8678     MainDlg.obj
 0003:00001680       ?m_hostIpaddrbackup@@3PADA 004a8680     MainFrm.obj
 0003:00001694       ?g_hostMac@@3PADA          004a8694     MainFrm.obj
 0003:000016a4       ?g_userName@@3PADA         004a86a4     MainFrm.obj
 0003:000016d8       ?g_pMainFrm@@3PAVCMainFrame@@A 004a86d8     MainFrm.obj
 0003:000016dc       ?first@@3HA                004a86dc     MainFrm.obj
 0003:000016e0       ?isInitError@@3HA          004a86e0     MainFrm.obj
 0003:000016e4       ?m_SendPort@CMainFrame@@2GA 004a86e4     MainFrm.obj
 0003:000016e8       ?istipinfo@@3HA            004a86e8     MainFrm.obj
 0003:000016ec       ?g_strStatusBarMain@@3V?$CStringT@DV?$StrTraitMFC_DLL@DV?$ChTraitsCRT@D@ATL@@@@@ATL@@A 004a86ec     MainFrm.obj
 0003:000016f0       ?m_bootMgr@@3VCBootModuleManager@@A 004a86f0     MainFrm.obj
 0003:0000295c       ?g_arrMessage@@3VCStringArray@@A 004a995c     MainFrm.obj
 0003:00002970       ?g_sock@@3VCMulticastSocket@@A 004a9970     MainFrm.obj
 0003:000029d0       ?g_strStatusBarOther@@3V?$CStringT@DV?$StrTraitMFC_DLL@DV?$ChTraitsCRT@D@ATL@@@@@ATL@@A 004a99d0     MainFrm.obj
 0003:000029d4       ?g_ipAddr@@3V?$CStringT@DV?$StrTraitMFC_DLL@DV?$ChTraitsCRT@D@ATL@@@@@ATL@@A 004a99d4     MainFrm.obj
 0003:000029d8       ?g_macname@@3V?$CStringT@DV?$StrTraitMFC_DLL@DV?$ChTraitsCRT@D@ATL@@@@@ATL@@A 004a99d8     MainFrm.obj
 0003:000029dc       ?gVersion@@3V?$CStringT@DV?$StrTraitMFC_DLL@DV?$ChTraitsCRT@D@ATL@@@@@ATL@@A 004a99dc     MainFrm.obj
 0003:000029e0       ?g_hdserialinfo@@3V?$CMap@V?$CStringT@DV?$StrTraitMFC_DLL@DV?$ChTraitsCRT@D@ATL@@@@@ATL@@PBDUItemInfo@@AAU3@@@A 004a99e0     MainFrm.obj
 0003:000029fc       ?g_regserialinfo@@3V?$CMap@V?$CStringT@DV?$StrTraitMFC_DLL@DV?$ChTraitsCRT@D@ATL@@@@@ATL@@PBDUItemInfo@@AAU3@@@A 004a99fc     MainFrm.obj
 0003:00002a18       ?m_GroupTree@@3VCGroupTree@@A 004a9a18     MyEdit.obj
 0003:00002ab8       ?g_UpfilePage@@3PAVCMyPropertyPage1@@A 004a9ab8     MyPropertyPage1.obj
 0003:00002abc       ?g_ClassPage@@3PAVCMyPropertyPage2@@A 004a9abc     MyPropertyPage1.obj
 0003:00002ac0       ?g_BroPage@@3PAVCMyPropertyPage3@@A 004a9ac0     MyPropertyPage1.obj
 0003:00002ac4       ?gMaxOnlineNum@@3HA        004a9ac4     myPublic.obj
 0003:00002b00       ?NtQuerySystemInformation@@3P6GJIPAXKPAK@ZA 004a9b00     comfunc:comfunc.obj
 0003:00002b04       ?g_bIsNT@@3HA              004a9b04     comfunc:comfunc.obj
 0003:00002b08       ?g_enabledbg@@3HA          004a9b08     comfunc:comfunc.obj
 0003:00002b0c       ?g_CurrentPath@@3V?$CStringT@DV?$StrTraitMFC_DLL@DV?$ChTraitsCRT@D@ATL@@@@@ATL@@A 004a9b0c     comfunc:comfunc.obj
 0003:00002b10       ?g_tempstring@@3V?$CStringT@DV?$StrTraitMFC_DLL@DV?$ChTraitsCRT@D@ATL@@@@@ATL@@A 004a9b10     loadres:exloadres.obj
 0003:00002b14       ?g_BasicPath@@3V?$CStringT@DV?$StrTraitMFC_DLL@DV?$ChTraitsCRT@D@ATL@@@@@ATL@@A 004a9b14     loadres:exloadres.obj
 0003:00002b18       __hmod__dwmapi_dll         004a9b18     dwmapi:dwmapi.dll
 0003:00002b1c       ___puiHead                 004a9b1c     DelayImp:delayhlp.obj
 0003:00002b20       ___pfnDliFailureHook2      004a9b20     DelayImp:delayhk1.obj
 0003:00002b24       ___pfnDliNotifyHook2       004a9b24     DelayImp:delayhk2.obj
 0003:00002b28       __afxForceEXCLUDE          004a9b28     mfcs90:nolib.obj
 0003:00002b2c       __afxForceSTDAFX           004a9b2c     mfcs90:stdafx.obj
 0003:00002e74       __forceCRTManifestRTM      004a9e74     msvcrt:crtmanifestrtm.obj
 0003:00002e78       __dowildcard               004a9e78     msvcrt:wildcard.obj
 0003:00002e7c       __newmode                  004a9e7c     msvcrt:_newmode.obj
 0003:00002e80       __commode                  004a9e80     msvcrt:xncommod.obj
 0003:00002e84       __fmode                    004a9e84     msvcrt:xtxtmode.obj
 0003:00002e8c       ?_afxInitAppState@@3DA     004a9e8c     mfcs90:appmodul.obj
 0003:00002e90       __forceMFCManifestRTM      004a9e90     mfcs90:mfcmanifestrtm.obj
 0003:00002e94       ___sse2_available          004a9e94     <common>
 0003:00002e98       __adjust_fdiv              004a9e98     <common>
 0003:00002e9c       ___native_startup_state    004a9e9c     <common>
 0003:00002ea0       ___native_startup_lock     004a9ea0     <common>
 0003:00002ea4       ___dyn_tls_init_callback   004a9ea4     <common>
 0003:00002ea8       ___onexitend               004a9ea8     <common>
 0003:00002eac       ___onexitbegin             004a9eac     <common>

 entry point at        0001:00075a8f

 Static symbols

 0001:00004a6f       __catch$??1CGdiObject@@UAE@XZ$0 00405a6f f i CalendarBar.obj
 0001:0000571f       __catch$?thAcceptCmd@@YAIPAX@Z$0 0040671f f   CFtpd.obj
 0001:00005b2b       __catch$?OnAccept@CFtpd@@UAEXH@Z$0 00406b2b f   CFtpd.obj
 0001:00005bc8       __catch$?AddClient@CFtpd@@QAEXPAVCFtpdPi@@@Z$0 00406bc8 f   CFtpd.obj
 0001:00005cad       __catch$?RemoveClient@CFtpd@@QAEXPAVCFtpdPi@@@Z$0 00406cad f   CFtpd.obj
 0001:000126d2       __catch$?canclePasvListenSocket@@YA_NPAVCFtpPasvSrv@@@Z$0 004136d2 f   FtpdPi.obj
 0001:0001274b       __catch$?deleFtpPI@@YA_NPAVCFtpdPi@@@Z$0 0041374b f   FtpdPi.obj
 0001:00012a99       __catch$?thSendData@@YAIPAX@Z$0 00413a99 f   FtpdPi.obj
 0001:00013144       __catch$?thSendData@@YAIPAX@Z$2 00414144 f   FtpdPi.obj
 0001:00013972       __catch$?OnReceive@CFtpdPi@@UAEXH@Z$0 00414972 f   FtpdPi.obj
 0001:000147de       __catch$?ProcessMsg@CFtpdPi@@QAEXPAD@Z$0 004157de f   FtpdPi.obj
 0001:00014c10       __catch$?ProcessMsg@CFtpdPi@@QAEXPAD@Z$2 00415c10 f   FtpdPi.obj
 0001:00014fbd       __catch$?ProcessMsg@CFtpdPi@@QAEXPAD@Z$4 00415fbd f   FtpdPi.obj
 0001:000153a9       __catch$?ProcessMsg@CFtpdPi@@QAEXPAD@Z$6 004163a9 f   FtpdPi.obj
 0001:00015734       __catch$?ProcessMsg@CFtpdPi@@QAEXPAD@Z$8 00416734 f   FtpdPi.obj
 0001:00015a99       __catch$?ProcessMsg@CFtpdPi@@QAEXPAD@Z$10 00416a99 f   FtpdPi.obj
 0001:00015d56       __catch$?ProcessMsg@CFtpdPi@@QAEXPAD@Z$12 00416d56 f   FtpdPi.obj
 0001:00016a04       __catch$?ProcessMsg@CFtpdPi@@QAEXPAD@Z$14 00417a04 f   FtpdPi.obj
 0001:000176ec       __catch$?ProcessMsg@CFtpdPi@@QAEXPAD@Z$16 004186ec f   FtpdPi.obj
 0001:00017912       __catch$?RemoveLeadingSpace@CFtpdPi@@QAEPADPAD@Z$0 00418912 f   FtpdPi.obj
 0001:00018c06       __catch$?SafeSend@CFtpdPi@@QAEXPAD@Z$0 00419c06 f   FtpdPi.obj
 0001:00019b55       __catch$?ListEngine@CFtpdPi@@QAEXPAD_N@Z$0 0041ab55 f   FtpdPi.obj
 0001:00055dba       __catch$??1CWaitCursor@@QAE@XZ$0 00456dba f i MainFrm.obj
 0001:0005b13c       __catch$?_Insert_n@?$vector@PAVCClientContext@@V?$allocator@PAVCClientContext@@@std@@@std@@IAEXV?$_Vector_const_iterator@PAVCClientContext@@V?$allocator@PAVCClientContext@@@std@@@2@IABQAVCClientContext@@@Z$0 0045c13c f i MyIOCP.obj
 0001:0005b293       __catch$?_Insert_n@?$vector@PAVCClientContext@@V?$allocator@PAVCClientContext@@@std@@@std@@IAEXV?$_Vector_const_iterator@PAVCClientContext@@V?$allocator@PAVCClientContext@@@std@@@2@IABQAVCClientContext@@@Z$2 0045c293 f i MyIOCP.obj
 0001:00075784       _pre_cpp_init              00476784 f   msvcrt:crtexew.obj
 0001:000757cf       ___tmainCRTStartup         004767cf f   msvcrt:crtexew.obj
 0001:000759ae       _pre_c_init                004769ae f   msvcrt:crtexew.obj
 0001:00076041       _has_osfxsr_set            00477041 f   msvcrt:cpu_disp.obj
 0001:00076300       _StringExHandleOtherFlagsA@24 00477300 f   odbccp32:dllload.obj
 0001:00076390       _GetVersionProcs@12        00477390 f   odbccp32:dllload.obj
 0001:000765a0       _LoadProperSetupDLL@0      004775a0 f   odbccp32:dllload.obj
 0001:00076c20       __unwindfunclet$??0CAboutDlg@@QAE@PAVCWnd@@@Z$0 00477c20 f   AboutDlg.obj
 0001:00076c28       __unwindfunclet$??0CAboutDlg@@QAE@PAVCWnd@@@Z$1 00477c28 f   AboutDlg.obj
 0001:00076c33       __unwindfunclet$??0CAboutDlg@@QAE@PAVCWnd@@@Z$2 00477c33 f   AboutDlg.obj
 0001:00076c41       __unwindfunclet$??0CAboutDlg@@QAE@PAVCWnd@@@Z$3 00477c41 f   AboutDlg.obj
 0001:00076c4f       __unwindfunclet$??0CAboutDlg@@QAE@PAVCWnd@@@Z$4 00477c4f f   AboutDlg.obj
 0001:00076c5d       __ehhandler$??0CAboutDlg@@QAE@PAVCWnd@@@Z 00477c5d f   AboutDlg.obj
 0001:00076c80       __unwindfunclet$??1CAboutDlg@@UAE@XZ$0 00477c80 f   AboutDlg.obj
 0001:00076c88       __unwindfunclet$??1CAboutDlg@@UAE@XZ$1 00477c88 f   AboutDlg.obj
 0001:00076c93       __unwindfunclet$??1CAboutDlg@@UAE@XZ$2 00477c93 f   AboutDlg.obj
 0001:00076ca1       __unwindfunclet$??1CAboutDlg@@UAE@XZ$3 00477ca1 f   AboutDlg.obj
 0001:00076caf       __ehhandler$??1CAboutDlg@@UAE@XZ 00477caf f   AboutDlg.obj
 0001:00076cd0       __unwindfunclet$?OnInitDialog@CAboutDlg@@MAEHXZ$0 00477cd0 f   AboutDlg.obj
 0001:00076cd9       __unwindfunclet$?OnInitDialog@CAboutDlg@@MAEHXZ$1 00477cd9 f   AboutDlg.obj
 0001:00076ce5       __unwindfunclet$?OnInitDialog@CAboutDlg@@MAEHXZ$3 00477ce5 f   AboutDlg.obj
 0001:00076cf1       __unwindfunclet$?OnInitDialog@CAboutDlg@@MAEHXZ$4 00477cf1 f   AboutDlg.obj
 0001:00076cfd       __unwindfunclet$?OnInitDialog@CAboutDlg@@MAEHXZ$5 00477cfd f   AboutDlg.obj
 0001:00076d06       __unwindfunclet$?OnInitDialog@CAboutDlg@@MAEHXZ$6 00477d06 f   AboutDlg.obj
 0001:00076d12       __unwindfunclet$?OnInitDialog@CAboutDlg@@MAEHXZ$7 00477d12 f   AboutDlg.obj
 0001:00076d1e       __unwindfunclet$?OnInitDialog@CAboutDlg@@MAEHXZ$8 00477d1e f   AboutDlg.obj
 0001:00076d2a       __unwindfunclet$?OnInitDialog@CAboutDlg@@MAEHXZ$9 00477d2a f   AboutDlg.obj
 0001:00076d36       __unwindfunclet$?OnInitDialog@CAboutDlg@@MAEHXZ$10 00477d36 f   AboutDlg.obj
 0001:00076d42       __ehhandler$?OnInitDialog@CAboutDlg@@MAEHXZ 00477d42 f   AboutDlg.obj
 0001:00076d70       __unwindfunclet$?SetTitle@CAboutDlg@@QAEXXZ$0 00477d70 f   AboutDlg.obj
 0001:00076d70       __unwindfunclet$?SetTitle@CSpecialPartitionRS@@QAEXXZ$0 00477d70 f   AboutDlg.obj
 0001:00076d79       __unwindfunclet$?SetTitle@CSpecialPartitionRS@@QAEXXZ$1 00477d79 f   AboutDlg.obj
 0001:00076d79       __unwindfunclet$?SetTitle@CAboutDlg@@QAEXXZ$1 00477d79 f   AboutDlg.obj
 0001:00076d82       __unwindfunclet$?SetTitle@CAboutDlg@@QAEXXZ$2 00477d82 f   AboutDlg.obj
 0001:00076d82       __unwindfunclet$?SetTitle@CSpecialPartitionRS@@QAEXXZ$2 00477d82 f   AboutDlg.obj
 0001:00076d8b       __unwindfunclet$?SetTitle@CAboutDlg@@QAEXXZ$3 00477d8b f   AboutDlg.obj
 0001:00076d8b       __unwindfunclet$?SetTitle@CSpecialPartitionRS@@QAEXXZ$3 00477d8b f   AboutDlg.obj
 0001:00076d94       __ehhandler$?SetTitle@CSpecialPartitionRS@@QAEXXZ 00477d94 f   AboutDlg.obj
 0001:00076d94       __ehhandler$?SetTitle@CAboutDlg@@QAEXXZ 00477d94 f   AboutDlg.obj
 0001:00076db0       __unwindfunclet$?OnBnClickedButton1@CAboutDlg@@QAEXXZ$0 00477db0 f   AboutDlg.obj
 0001:00076db9       __unwindfunclet$?OnBnClickedButton1@CAboutDlg@@QAEXXZ$1 00477db9 f   AboutDlg.obj
 0001:00076dc2       __unwindfunclet$?OnBnClickedButton1@CAboutDlg@@QAEXXZ$2 00477dc2 f   AboutDlg.obj
 0001:00076dcb       __unwindfunclet$?OnBnClickedButton1@CAboutDlg@@QAEXXZ$3 00477dcb f   AboutDlg.obj
 0001:00076dd4       __ehhandler$?OnBnClickedButton1@CAboutDlg@@QAEXXZ 00477dd4 f   AboutDlg.obj
 0001:00076df0       __unwindfunclet$??HATL@@YA?AV?$CStringT@DV?$StrTraitMFC_DLL@DV?$ChTraitsCRT@D@ATL@@@@@0@ABV10@PBD@Z$0 00477df0 f   AboutDlg.obj
 0001:00076df0       __unwindfunclet$?OnOK@CCheckPasswordDlg@@MAEXXZ$0 00477df0 f   AboutDlg.obj
 0001:00076df0       __unwindfunclet$??HATL@@YA?AV?$CStringT@DV?$StrTraitMFC_DLL@DV?$ChTraitsCRT@D@ATL@@@@@0@PBDABV10@@Z$0 00477df0 f   AboutDlg.obj
 0001:00076df9       __ehhandler$??HATL@@YA?AV?$CStringT@DV?$StrTraitMFC_DLL@DV?$ChTraitsCRT@D@ATL@@@@@0@PBDABV10@@Z 00477df9 f   AboutDlg.obj
 0001:00076df9       __ehhandler$?OnOK@CCheckPasswordDlg@@MAEXXZ 00477df9 f   AboutDlg.obj
 0001:00076df9       __ehhandler$??HATL@@YA?AV?$CStringT@DV?$StrTraitMFC_DLL@DV?$ChTraitsCRT@D@ATL@@@@@0@ABV10@PBD@Z 00477df9 f   AboutDlg.obj
 0001:00076e20       __unwindfunclet$??1CSpecialPartitionRS@@UAE@XZ$0 00477e20 f   AddToGroup.obj
 0001:00076e20       __unwindfunclet$??0CGroupExt@@QAE@PAVCWnd@@@Z$0 00477e20 f   AddToGroup.obj
 0001:00076e20       __unwindfunclet$??1CBlackListDlg@@UAE@XZ$0 00477e20 f   AddToGroup.obj
 0001:00076e20       __unwindfunclet$??1CModifyGroup@@UAE@XZ$0 00477e20 f   AddToGroup.obj
 0001:00076e20       __unwindfunclet$??1CCheckPasswordDlg@@UAE@XZ$0 00477e20 f   AddToGroup.obj
 0001:00076e20       __unwindfunclet$??1CGroupExt@@UAE@XZ$0 00477e20 f   AddToGroup.obj
 0001:00076e20       __unwindfunclet$??1CAddToGroup@@UAE@XZ$0 00477e20 f   AddToGroup.obj
 0001:00076e20       __unwindfunclet$??1CSetDrfaultNICDlg@@UAE@XZ$0 00477e20 f   AddToGroup.obj
 0001:00076e20       __unwindfunclet$??1CBroadIE@@UAE@XZ$0 00477e20 f   AddToGroup.obj
 0001:00076e20       __unwindfunclet$??0CBlackListDlg@@QAE@PAVCWnd@@@Z$0 00477e20 f   AddToGroup.obj
 0001:00076e28       __ehhandler$??1CSetDrfaultNICDlg@@UAE@XZ 00477e28 f   AddToGroup.obj
 0001:00076e28       __ehhandler$??1CBroadIE@@UAE@XZ 00477e28 f   AddToGroup.obj
 0001:00076e28       __ehhandler$??1CSpecialPartitionRS@@UAE@XZ 00477e28 f   AddToGroup.obj
 0001:00076e28       __ehhandler$??1CBlackListDlg@@UAE@XZ 00477e28 f   AddToGroup.obj
 0001:00076e28       __ehhandler$??1CGroupExt@@UAE@XZ 00477e28 f   AddToGroup.obj
 0001:00076e28       __ehhandler$??1CAddToGroup@@UAE@XZ 00477e28 f   AddToGroup.obj
 0001:00076e28       __ehhandler$??1CCheckPasswordDlg@@UAE@XZ 00477e28 f   AddToGroup.obj
 0001:00076e28       __ehhandler$??0CBlackListDlg@@QAE@PAVCWnd@@@Z 00477e28 f   AddToGroup.obj
 0001:00076e28       __ehhandler$??1CModifyGroup@@UAE@XZ 00477e28 f   AddToGroup.obj
 0001:00076e28       __ehhandler$??0CGroupExt@@QAE@PAVCWnd@@@Z 00477e28 f   AddToGroup.obj
 0001:00076e50       __unwindfunclet$?OnInitDialog@CAddToGroup@@MAEHXZ$0 00477e50 f   AddToGroup.obj
 0001:00076e59       __unwindfunclet$?OnInitDialog@CAddToGroup@@MAEHXZ$1 00477e59 f   AddToGroup.obj
 0001:00076e62       __unwindfunclet$?OnInitDialog@CAddToGroup@@MAEHXZ$2 00477e62 f   AddToGroup.obj
 0001:00076e6b       __unwindfunclet$?OnInitDialog@CAddToGroup@@MAEHXZ$3 00477e6b f   AddToGroup.obj
 0001:00076e74       __unwindfunclet$?OnInitDialog@CAddToGroup@@MAEHXZ$4 00477e74 f   AddToGroup.obj
 0001:00076e7d       __unwindfunclet$?OnInitDialog@CAddToGroup@@MAEHXZ$5 00477e7d f   AddToGroup.obj
 0001:00076e85       __ehhandler$?OnInitDialog@CAddToGroup@@MAEHXZ 00477e85 f   AddToGroup.obj
 0001:00076ea0       __unwindfunclet$?SortGroup@CAddToGroup@@QAEHAAVCStringList@@@Z$0 00477ea0 f   AddToGroup.obj
 0001:00076ea9       __unwindfunclet$?SortGroup@CAddToGroup@@QAEHAAVCStringList@@@Z$1 00477ea9 f   AddToGroup.obj
 0001:00076eb2       __unwindfunclet$?SortGroup@CAddToGroup@@QAEHAAVCStringList@@@Z$2 00477eb2 f   AddToGroup.obj
 0001:00076ebb       __ehhandler$?SortGroup@CAddToGroup@@QAEHAAVCStringList@@@Z 00477ebb f   AddToGroup.obj
 0001:00076ee0       __unwindfunclet$?OnInitDialog@CBlackListDlg@@MAEHXZ$0 00477ee0 f   BlackListDlg.obj
 0001:00076ee9       __unwindfunclet$?OnInitDialog@CBlackListDlg@@MAEHXZ$1 00477ee9 f   BlackListDlg.obj
 0001:00076ef2       __unwindfunclet$?OnInitDialog@CBlackListDlg@@MAEHXZ$2 00477ef2 f   BlackListDlg.obj
 0001:00076efb       __unwindfunclet$?OnInitDialog@CBlackListDlg@@MAEHXZ$3 00477efb f   BlackListDlg.obj
 0001:00076f04       __unwindfunclet$?OnInitDialog@CBlackListDlg@@MAEHXZ$4 00477f04 f   BlackListDlg.obj
 0001:00076f0d       __unwindfunclet$?OnInitDialog@CBlackListDlg@@MAEHXZ$5 00477f0d f   BlackListDlg.obj
 0001:00076f16       __unwindfunclet$?OnInitDialog@CBlackListDlg@@MAEHXZ$6 00477f16 f   BlackListDlg.obj
 0001:00076f1f       __unwindfunclet$?OnInitDialog@CBlackListDlg@@MAEHXZ$7 00477f1f f   BlackListDlg.obj
 0001:00076f28       __unwindfunclet$?OnInitDialog@CBlackListDlg@@MAEHXZ$8 00477f28 f   BlackListDlg.obj
 0001:00076f31       __ehhandler$?OnInitDialog@CBlackListDlg@@MAEHXZ 00477f31 f   BlackListDlg.obj
 0001:00076f50       __unwindfunclet$?OnOK@CBlackListDlg@@MAEXXZ$0 00477f50 f   BlackListDlg.obj
 0001:00076f59       __unwindfunclet$?OnOK@CBlackListDlg@@MAEXXZ$1 00477f59 f   BlackListDlg.obj
 0001:00076f62       __unwindfunclet$?OnOK@CBlackListDlg@@MAEXXZ$2 00477f62 f   BlackListDlg.obj
 0001:00076f6b       __unwindfunclet$?OnOK@CBlackListDlg@@MAEXXZ$3 00477f6b f   BlackListDlg.obj
 0001:00076f74       __unwindfunclet$?OnOK@CBlackListDlg@@MAEXXZ$5 00477f74 f   BlackListDlg.obj
 0001:00076f7d       __unwindfunclet$?OnOK@CBlackListDlg@@MAEXXZ$6 00477f7d f   BlackListDlg.obj
 0001:00076f86       __unwindfunclet$?OnOK@CBlackListDlg@@MAEXXZ$7 00477f86 f   BlackListDlg.obj
 0001:00076f8f       __unwindfunclet$?OnOK@CBlackListDlg@@MAEXXZ$8 00477f8f f   BlackListDlg.obj
 0001:00076f98       __ehhandler$?OnOK@CBlackListDlg@@MAEXXZ 00477f98 f   BlackListDlg.obj
 0001:00076fc0       __unwindfunclet$??0CBlockingSocketException@@QAE@PAD@Z$0 00477fc0 f   blocksock.obj
 0001:00076fc8       __unwindfunclet$??0CBlockingSocketException@@QAE@PAD@Z$1 00477fc8 f   blocksock.obj
 0001:00076fd4       __ehhandler$??0CBlockingSocketException@@QAE@PAD@Z 00477fd4 f   blocksock.obj
 0001:00076ff0       __unwindfunclet$?Accept@CBlockingSocket@@QAEHAAV1@PAUsockaddr@@@Z$0 00477ff0 f   blocksock.obj
 0001:00076ffa       __ehhandler$?Accept@CBlockingSocket@@QAEHAAV1@PAUsockaddr@@@Z 00477ffa f   blocksock.obj
 0001:00077020       __unwindfunclet$?Close@CBlockingSocket@@QAEXXZ$0 00478020 f   blocksock.obj
 0001:0007702a       __ehhandler$?Close@CBlockingSocket@@QAEXXZ 0047802a f   blocksock.obj
 0001:00077050       __unwindfunclet$?Receive@CBlockingSocket@@QAEHPADHH@Z$0 00478050 f   blocksock.obj
 0001:00077050       __unwindfunclet$?Send@CBlockingSocket@@QAEHPBDHH@Z$0 00478050 f   blocksock.obj
 0001:0007705d       __unwindfunclet$?Receive@CBlockingSocket@@QAEHPADHH@Z$1 0047805d f   blocksock.obj
 0001:0007705d       __unwindfunclet$?Send@CBlockingSocket@@QAEHPBDHH@Z$1 0047805d f   blocksock.obj
 0001:0007706a       __ehhandler$?Send@CBlockingSocket@@QAEHPBDHH@Z 0047806a f   blocksock.obj
 0001:0007706a       __ehhandler$?Receive@CBlockingSocket@@QAEHPADHH@Z 0047806a f   blocksock.obj
 0001:00077090       __unwindfunclet$??1CBootModuleManager@@UAE@XZ$0 00478090 f   BootModuleManager.obj
 0001:00077090       __unwindfunclet$??0CBootModuleManager@@QAE@XZ$0 00478090 f   BootModuleManager.obj
 0001:0007709b       __unwindfunclet$??0CBootModuleManager@@QAE@XZ$1 0047809b f   BootModuleManager.obj
 0001:0007709b       __unwindfunclet$??1CBootModuleManager@@UAE@XZ$1 0047809b f   BootModuleManager.obj
 0001:000770a6       __unwindfunclet$??1CBootModuleManager@@UAE@XZ$2 004780a6 f   BootModuleManager.obj
 0001:000770a6       __unwindfunclet$??0CBootModuleManager@@QAE@XZ$2 004780a6 f   BootModuleManager.obj
 0001:000770b4       __ehhandler$??1CBootModuleManager@@UAE@XZ 004780b4 f   BootModuleManager.obj
 0001:000770b4       __ehhandler$??0CBootModuleManager@@QAE@XZ 004780b4 f   BootModuleManager.obj
 0001:000770d0       __unwindfunclet$??0CCriticalSection@@QAE@XZ$0 004780d0 f   BootModuleManager.obj
 0001:000770d8       __ehhandler$??0CCriticalSection@@QAE@XZ 004780d8 f   BootModuleManager.obj
 0001:00077100       __unwindfunclet$??0CBroadIE@@QAE@PAVCWnd@@@Z$0 00478100 f   BroadIE.obj
 0001:00077100       __unwindfunclet$??0CAddToGroup@@QAE@PAVCWnd@@@Z$0 00478100 f   BroadIE.obj
 0001:00077108       __unwindfunclet$??0CBroadIE@@QAE@PAVCWnd@@@Z$1 00478108 f   BroadIE.obj
 0001:00077108       __unwindfunclet$??0CAddToGroup@@QAE@PAVCWnd@@@Z$1 00478108 f   BroadIE.obj
 0001:00077113       __unwindfunclet$??0CAddToGroup@@QAE@PAVCWnd@@@Z$2 00478113 f   BroadIE.obj
 0001:00077113       __unwindfunclet$??0CBroadIE@@QAE@PAVCWnd@@@Z$2 00478113 f   BroadIE.obj
 0001:00077122       __ehhandler$??0CAddToGroup@@QAE@PAVCWnd@@@Z 00478122 f   BroadIE.obj
 0001:00077122       __ehhandler$??0CBroadIE@@QAE@PAVCWnd@@@Z 00478122 f   BroadIE.obj
 0001:00077140       __unwindfunclet$?OnInitDialog@CBroadIE@@MAEHXZ$0 00478140 f   BroadIE.obj
 0001:00077149       __unwindfunclet$?OnInitDialog@CBroadIE@@MAEHXZ$1 00478149 f   BroadIE.obj
 0001:00077152       __unwindfunclet$?OnInitDialog@CBroadIE@@MAEHXZ$2 00478152 f   BroadIE.obj
 0001:0007715b       __unwindfunclet$?OnInitDialog@CBroadIE@@MAEHXZ$3 0047815b f   BroadIE.obj
 0001:00077164       __unwindfunclet$?OnInitDialog@CBroadIE@@MAEHXZ$4 00478164 f   BroadIE.obj
 0001:0007716d       __unwindfunclet$?OnInitDialog@CBroadIE@@MAEHXZ$5 0047816d f   BroadIE.obj
 0001:00077176       __unwindfunclet$?OnInitDialog@CBroadIE@@MAEHXZ$6 00478176 f   BroadIE.obj
 0001:0007717e       __unwindfunclet$?OnInitDialog@CBroadIE@@MAEHXZ$9 0047817e f   BroadIE.obj
 0001:00077187       __unwindfunclet$?OnInitDialog@CBroadIE@@MAEHXZ$11 00478187 f   BroadIE.obj
 0001:00077190       __ehhandler$?OnInitDialog@CBroadIE@@MAEHXZ 00478190 f   BroadIE.obj
 0001:000771b0       __unwindfunclet$?OnBnClickedOk@CBroadIE@@QAEXXZ$0 004781b0 f   BroadIE.obj
 0001:000771b9       __unwindfunclet$?OnBnClickedOk@CBroadIE@@QAEXXZ$1 004781b9 f   BroadIE.obj
 0001:000771c5       __unwindfunclet$?OnBnClickedOk@CBroadIE@@QAEXXZ$2 004781c5 f   BroadIE.obj
 0001:000771d1       __unwindfunclet$?OnBnClickedOk@CBroadIE@@QAEXXZ$3 004781d1 f   BroadIE.obj
 0001:000771dd       __unwindfunclet$?OnBnClickedOk@CBroadIE@@QAEXXZ$4 004781dd f   BroadIE.obj
 0001:000771e9       __unwindfunclet$?OnBnClickedOk@CBroadIE@@QAEXXZ$5 004781e9 f   BroadIE.obj
 0001:000771f5       __unwindfunclet$?OnBnClickedOk@CBroadIE@@QAEXXZ$6 004781f5 f   BroadIE.obj
 0001:00077201       __unwindfunclet$?OnBnClickedOk@CBroadIE@@QAEXXZ$7 00478201 f   BroadIE.obj
 0001:0007720d       __unwindfunclet$?OnBnClickedOk@CBroadIE@@QAEXXZ$8 0047820d f   BroadIE.obj
 0001:00077219       __unwindfunclet$?OnBnClickedOk@CBroadIE@@QAEXXZ$9 00478219 f   BroadIE.obj
 0001:00077225       __unwindfunclet$?OnBnClickedOk@CBroadIE@@QAEXXZ$10 00478225 f   BroadIE.obj
 0001:00077231       __unwindfunclet$?OnBnClickedOk@CBroadIE@@QAEXXZ$12 00478231 f   BroadIE.obj
 0001:0007723a       __unwindfunclet$?OnBnClickedOk@CBroadIE@@QAEXXZ$13 0047823a f   BroadIE.obj
 0001:00077242       __unwindfunclet$?OnBnClickedOk@CBroadIE@@QAEXXZ$16 00478242 f   BroadIE.obj
 0001:0007724e       __unwindfunclet$?OnBnClickedOk@CBroadIE@@QAEXXZ$18 0047824e f   BroadIE.obj
 0001:0007725a       __unwindfunclet$?OnBnClickedOk@CBroadIE@@QAEXXZ$20 0047825a f   BroadIE.obj
 0001:00077266       __ehhandler$?OnBnClickedOk@CBroadIE@@QAEXXZ 00478266 f   BroadIE.obj
 0001:00077290       __unwindfunclet$?OnBnClickedClear@CBroadIE@@QAEXXZ$0 00478290 f   BroadIE.obj
 0001:00077298       __ehhandler$?OnBnClickedClear@CBroadIE@@QAEXXZ 00478298 f   BroadIE.obj
 0001:000772c0       __unwindfunclet$??1CBroadWaitDlg@@UAE@XZ$0 004782c0 f   BroadWaitDlg.obj
 0001:000772c8       __unwindfunclet$??1CBroadWaitDlg@@UAE@XZ$1 004782c8 f   BroadWaitDlg.obj
 0001:000772d4       __unwindfunclet$??1CBroadWaitDlg@@UAE@XZ$2 004782d4 f   BroadWaitDlg.obj
 0001:000772e3       __ehhandler$??1CBroadWaitDlg@@UAE@XZ 004782e3 f   BroadWaitDlg.obj
 0001:00077300       __unwindfunclet$?OnInitDialog@CBroadWaitDlg@@UAEHXZ$0 00478300 f   BroadWaitDlg.obj
 0001:00077300       __unwindfunclet$?GetFileSystemType@CClientSettingsDlg@@QAE?AV?$CStringT@DV?$StrTraitMFC_DLL@DV?$ChTraitsCRT@D@ATL@@@@@ATL@@E@Z$0 00478300 f   BroadWaitDlg.obj
 0001:00077300       __unwindfunclet$?OnBnClickedOk@CPortChannelDlg@@QAEXXZ$0 00478300 f   BroadWaitDlg.obj
 0001:00077300       __unwindfunclet$?OnInitDialog@CInfoPromptDlg@@MAEHXZ$0 00478300 f   BroadWaitDlg.obj
 0001:00077300       __unwindfunclet$?OnBnClickedOk@CSetClientchancelDLg@@QAEXXZ$0 00478300 f   BroadWaitDlg.obj
 0001:00077300       __unwindfunclet$?GetFileSystemType@CSpecialPartitionRS@@QAE?AV?$CStringT@DV?$StrTraitMFC_DLL@DV?$ChTraitsCRT@D@ATL@@@@@ATL@@E@Z$0 00478300 f   BroadWaitDlg.obj
 0001:00077309       __ehhandler$?OnBnClickedOk@CSetClientchancelDLg@@QAEXXZ 00478309 f   BroadWaitDlg.obj
 0001:00077309       __ehhandler$?GetFileSystemType@CSpecialPartitionRS@@QAE?AV?$CStringT@DV?$StrTraitMFC_DLL@DV?$ChTraitsCRT@D@ATL@@@@@ATL@@E@Z 00478309 f   BroadWaitDlg.obj
 0001:00077309       __ehhandler$?OnInitDialog@CBroadWaitDlg@@UAEHXZ 00478309 f   BroadWaitDlg.obj
 0001:00077309       __ehhandler$?OnBnClickedOk@CPortChannelDlg@@QAEXXZ 00478309 f   BroadWaitDlg.obj
 0001:00077309       __ehhandler$?GetFileSystemType@CClientSettingsDlg@@QAE?AV?$CStringT@DV?$StrTraitMFC_DLL@DV?$ChTraitsCRT@D@ATL@@@@@ATL@@E@Z 00478309 f   BroadWaitDlg.obj
 0001:00077309       __ehhandler$?OnInitDialog@CInfoPromptDlg@@MAEHXZ 00478309 f   BroadWaitDlg.obj
 0001:00077330       __unwindfunclet$?WaitStart@CBroadWaitDlg@@QAEHV?$CStringT@DV?$StrTraitMFC_DLL@DV?$ChTraitsCRT@D@ATL@@@@@ATL@@0HPAVCWnd@@@Z$0 00478330 f   BroadWaitDlg.obj
 0001:00077339       __unwindfunclet$?WaitStart@CBroadWaitDlg@@QAEHV?$CStringT@DV?$StrTraitMFC_DLL@DV?$ChTraitsCRT@D@ATL@@@@@ATL@@0HPAVCWnd@@@Z$1 00478339 f   BroadWaitDlg.obj
 0001:00077342       __unwindfunclet$?WaitStart@CBroadWaitDlg@@QAEHV?$CStringT@DV?$StrTraitMFC_DLL@DV?$ChTraitsCRT@D@ATL@@@@@ATL@@0HPAVCWnd@@@Z$2 00478342 f   BroadWaitDlg.obj
 0001:0007734d       __ehhandler$?WaitStart@CBroadWaitDlg@@QAEHV?$CStringT@DV?$StrTraitMFC_DLL@DV?$ChTraitsCRT@D@ATL@@@@@ATL@@0HPAVCWnd@@@Z 0047834d f   BroadWaitDlg.obj
 0001:00077370       __unwindfunclet$??1CCalendarBar@@UAE@XZ$0 00478370 f   CalendarBar.obj
 0001:00077370       __unwindfunclet$??0CCalendarBar@@QAE@XZ$0 00478370 f   CalendarBar.obj
 0001:00077378       __unwindfunclet$??1CCalendarBar@@UAE@XZ$1 00478378 f   CalendarBar.obj
 0001:00077378       __unwindfunclet$??0CCalendarBar@@QAE@XZ$1 00478378 f   CalendarBar.obj
 0001:00077383       __ehhandler$??1CCalendarBar@@UAE@XZ 00478383 f   CalendarBar.obj
 0001:00077383       __ehhandler$??0CCalendarBar@@QAE@XZ 00478383 f   CalendarBar.obj
 0001:000773a0       __unwindfunclet$?OnCreate@CCalendarBar@@IAEHPAUtagCREATESTRUCTA@@@Z$0 004783a0 f   CalendarBar.obj
 0001:000773a8       __ehhandler$?OnCreate@CCalendarBar@@IAEHPAUtagCREATESTRUCTA@@@Z 004783a8 f   CalendarBar.obj
 0001:000773d0       __unwindfunclet$?OnPaint@CCalendarBar@@IAEXXZ$0 004783d0 f   CalendarBar.obj
 0001:000773d8       __unwindfunclet$?OnPaint@CCalendarBar@@IAEXXZ$1 004783d8 f   CalendarBar.obj
 0001:000773e4       __ehhandler$?OnPaint@CCalendarBar@@IAEXXZ 004783e4 f   CalendarBar.obj
 0001:00077410       __unwindfunclet$??1CGdiObject@@UAE@XZ$2 00478410 f   CalendarBar.obj
 0001:0007741b       __unwindfunclet$??1CGdiObject@@UAE@XZ$3 0047841b f   CalendarBar.obj
 0001:00077427       __ehhandler$??1CGdiObject@@UAE@XZ 00478427 f   CalendarBar.obj
 0001:00077450       __unwindfunclet$?thAcceptCmd@@YAIPAX@Z$2 00478450 f   CFtpd.obj
 0001:00077458       __unwindfunclet$?thAcceptCmd@@YAIPAX@Z$3 00478458 f   CFtpd.obj
 0001:00077461       __unwindfunclet$?thAcceptCmd@@YAIPAX@Z$4 00478461 f   CFtpd.obj
 0001:0007746a       __ehhandler$?thAcceptCmd@@YAIPAX@Z 0047846a f   CFtpd.obj
 0001:000774a0       __unwindfunclet$??0CFtpd@@QAE@XZ$0 004784a0 f   CFtpd.obj
 0001:000774a8       __unwindfunclet$??0CFtpd@@QAE@XZ$1 004784a8 f   CFtpd.obj
 0001:000774b6       __unwindfunclet$??0CFtpd@@QAE@XZ$2 004784b6 f   CFtpd.obj
 0001:000774c5       __unwindfunclet$??0CFtpd@@QAE@XZ$3 004784c5 f   CFtpd.obj
 0001:000774d4       __unwindfunclet$??0CFtpd@@QAE@XZ$4 004784d4 f   CFtpd.obj
 0001:000774e3       __unwindfunclet$??0CFtpd@@QAE@XZ$5 004784e3 f   CFtpd.obj
 0001:000774f1       __unwindfunclet$??0CFtpd@@QAE@XZ$6 004784f1 f   CFtpd.obj
 0001:000774ff       __ehhandler$??0CFtpd@@QAE@XZ 004784ff f   CFtpd.obj
 0001:00077520       __unwindfunclet$??1CFtpd@@UAE@XZ$0 00478520 f   CFtpd.obj
 0001:00077528       __unwindfunclet$??1CFtpd@@UAE@XZ$1 00478528 f   CFtpd.obj
 0001:00077536       __unwindfunclet$??1CFtpd@@UAE@XZ$2 00478536 f   CFtpd.obj
 0001:00077545       __unwindfunclet$??1CFtpd@@UAE@XZ$3 00478545 f   CFtpd.obj
 0001:00077554       __unwindfunclet$??1CFtpd@@UAE@XZ$4 00478554 f   CFtpd.obj
 0001:00077563       __unwindfunclet$??1CFtpd@@UAE@XZ$5 00478563 f   CFtpd.obj
 0001:00077571       __unwindfunclet$??1CFtpd@@UAE@XZ$6 00478571 f   CFtpd.obj
 0001:0007757f       __ehhandler$??1CFtpd@@UAE@XZ 0047857f f   CFtpd.obj
 0001:000775a0       __unwindfunclet$?OnAccept@CFtpd@@UAEXH@Z$2 004785a0 f   CFtpd.obj
 0001:000775aa       __ehhandler$?OnAccept@CFtpd@@UAEXH@Z 004785aa f   CFtpd.obj
 0001:000775d0       __ehhandler$?AddClient@CFtpd@@QAEXPAVCFtpdPi@@@Z 004785d0 f   CFtpd.obj
 0001:000775f0       __ehhandler$?RemoveClient@CFtpd@@QAEXPAVCFtpdPi@@@Z 004785f0 f   CFtpd.obj
 0001:00077610       __unwindfunclet$?FileToCsl@@YAXPADPAVCStringList@@@Z$0 00478610 f   CFtpd.obj
 0001:00077618       __unwindfunclet$?FileToCsl@@YAXPADPAVCStringList@@@Z$1 00478618 f   CFtpd.obj
 0001:00077624       __ehhandler$?FileToCsl@@YAXPADPAVCStringList@@@Z 00478624 f   CFtpd.obj
 0001:00077650       __unwindfunclet$??0CCheckPasswordDlg@@QAE@PAVCWnd@@@Z$0 00478650 f   CheckPasswordDlg.obj
 0001:00077658       __unwindfunclet$??0CCheckPasswordDlg@@QAE@PAVCWnd@@@Z$1 00478658 f   CheckPasswordDlg.obj
 0001:00077663       __unwindfunclet$??0CCheckPasswordDlg@@QAE@PAVCWnd@@@Z$2 00478663 f   CheckPasswordDlg.obj
 0001:00077672       __unwindfunclet$??0CCheckPasswordDlg@@QAE@PAVCWnd@@@Z$3 00478672 f   CheckPasswordDlg.obj
 0001:00077681       __ehhandler$??0CCheckPasswordDlg@@QAE@PAVCWnd@@@Z 00478681 f   CheckPasswordDlg.obj
 0001:000776a0       __unwindfunclet$??0CClientInfoManager@@QAE@XZ$0 004786a0 f   ClientInfoManager.obj
 0001:000776ab       __unwindfunclet$??0CClientInfoManager@@QAE@XZ$1 004786ab f   ClientInfoManager.obj
 0001:000776b6       __unwindfunclet$??0CClientInfoManager@@QAE@XZ$2 004786b6 f   ClientInfoManager.obj
 0001:000776c1       __ehhandler$??0CClientInfoManager@@QAE@XZ 004786c1 f   ClientInfoManager.obj
 0001:000776e0       __unwindfunclet$??1CClientInfoManager@@UAE@XZ$0 004786e0 f   ClientInfoManager.obj
 0001:000776eb       __unwindfunclet$??1CClientInfoManager@@UAE@XZ$1 004786eb f   ClientInfoManager.obj
 0001:000776f6       __unwindfunclet$??1CClientInfoManager@@UAE@XZ$2 004786f6 f   ClientInfoManager.obj
 0001:00077701       __unwindfunclet$??1CClientInfoManager@@UAE@XZ$3 00478701 f   ClientInfoManager.obj
 0001:0007770c       __ehhandler$??1CClientInfoManager@@UAE@XZ 0047870c f   ClientInfoManager.obj
 0001:00077730       __unwindfunclet$?InsertNewClient@CClientInfoManager@@QAEHPAUtagLOGIN_REQ@@AAPAUtagCLIENTMAININFO@@@Z$0 00478730 f   ClientInfoManager.obj
 0001:0007773c       __ehhandler$?InsertNewClient@CClientInfoManager@@QAEHPAUtagLOGIN_REQ@@AAPAUtagCLIENTMAININFO@@@Z 0047873c f   ClientInfoManager.obj
 0001:00077770       __unwindfunclet$?RemoveOneClient@CClientInfoManager@@QAEHPBD@Z$0 00478770 f   ClientInfoManager.obj
 0001:00077778       __unwindfunclet$?RemoveOneClient@CClientInfoManager@@QAEHPBD@Z$1 00478778 f   ClientInfoManager.obj
 0001:00077781       __unwindfunclet$?RemoveOneClient@CClientInfoManager@@QAEHPBD@Z$2 00478781 f   ClientInfoManager.obj
 0001:0007778a       __unwindfunclet$?RemoveOneClient@CClientInfoManager@@QAEHPBD@Z$3 0047878a f   ClientInfoManager.obj
 0001:00077793       __unwindfunclet$?RemoveOneClient@CClientInfoManager@@QAEHPBD@Z$4 00478793 f   ClientInfoManager.obj
 0001:0007779c       __unwindfunclet$?RemoveOneClient@CClientInfoManager@@QAEHPBD@Z$5 0047879c f   ClientInfoManager.obj
 0001:000777a5       __unwindfunclet$?RemoveOneClient@CClientInfoManager@@QAEHPBD@Z$6 004787a5 f   ClientInfoManager.obj
 0001:000777ae       __unwindfunclet$?RemoveOneClient@CClientInfoManager@@QAEHPBD@Z$7 004787ae f   ClientInfoManager.obj
 0001:000777b7       __unwindfunclet$?RemoveOneClient@CClientInfoManager@@QAEHPBD@Z$8 004787b7 f   ClientInfoManager.obj
 0001:000777c0       __unwindfunclet$?RemoveOneClient@CClientInfoManager@@QAEHPBD@Z$9 004787c0 f   ClientInfoManager.obj
 0001:000777c9       __unwindfunclet$?RemoveOneClient@CClientInfoManager@@QAEHPBD@Z$12 004787c9 f   ClientInfoManager.obj
 0001:000777d2       __unwindfunclet$?RemoveOneClient@CClientInfoManager@@QAEHPBD@Z$13 004787d2 f   ClientInfoManager.obj
 0001:000777db       __unwindfunclet$?RemoveOneClient@CClientInfoManager@@QAEHPBD@Z$14 004787db f   ClientInfoManager.obj
 0001:000777e4       __unwindfunclet$?RemoveOneClient@CClientInfoManager@@QAEHPBD@Z$15 004787e4 f   ClientInfoManager.obj
 0001:000777ed       __unwindfunclet$?RemoveOneClient@CClientInfoManager@@QAEHPBD@Z$17 004787ed f   ClientInfoManager.obj
 0001:000777f6       __ehhandler$?RemoveOneClient@CClientInfoManager@@QAEHPBD@Z 004787f6 f   ClientInfoManager.obj
 0001:00077820       __unwindfunclet$?ClearAllFromClientInfoMap@CClientInfoManager@@QAEXXZ$0 00478820 f   ClientInfoManager.obj
 0001:00077820       __unwindfunclet$?ClearAllFromBlackMap@CClientInfoManager@@QAEXXZ$0 00478820 f   ClientInfoManager.obj
 0001:00077829       __ehhandler$?ClearAllFromBlackMap@CClientInfoManager@@QAEXXZ 00478829 f   ClientInfoManager.obj
 0001:00077829       __ehhandler$?ClearAllFromClientInfoMap@CClientInfoManager@@QAEXXZ 00478829 f   ClientInfoManager.obj
 0001:00077850       __unwindfunclet$?UpdateOneClientInfo@CClientInfoManager@@QAEHPAUtagLOGIN_REQ@@AAPAUtagCLIENTMAININFO@@AAH@Z$1 00478850 f   ClientInfoManager.obj
 0001:0007785c       __ehhandler$?UpdateOneClientInfo@CClientInfoManager@@QAEHPAUtagLOGIN_REQ@@AAPAUtagCLIENTMAININFO@@AAH@Z 0047885c f   ClientInfoManager.obj
 0001:00077890       __unwindfunclet$?LoadComputersToMap@CClientInfoManager@@QAEHXZ$0 00478890 f   ClientInfoManager.obj
 0001:0007789c       __unwindfunclet$?LoadComputersToMap@CClientInfoManager@@QAEHXZ$1 0047889c f   ClientInfoManager.obj
 0001:000778a7       __unwindfunclet$?LoadComputersToMap@CClientInfoManager@@QAEHXZ$2 004788a7 f   ClientInfoManager.obj
 0001:000778b3       __unwindfunclet$?LoadComputersToMap@CClientInfoManager@@QAEHXZ$3 004788b3 f   ClientInfoManager.obj
 0001:000778bf       __unwindfunclet$?LoadComputersToMap@CClientInfoManager@@QAEHXZ$4 004788bf f   ClientInfoManager.obj
 0001:000778cb       __ehhandler$?LoadComputersToMap@CClientInfoManager@@QAEHXZ 004788cb f   ClientInfoManager.obj
 0001:00077900       __unwindfunclet$?RemoveOneFromBlack@CClientInfoManager@@QAEHV?$CStringT@DV?$StrTraitMFC_DLL@DV?$ChTraitsCRT@D@ATL@@@@@ATL@@@Z$0 00478900 f   ClientInfoManager.obj
 0001:00077909       __unwindfunclet$?RemoveOneFromBlack@CClientInfoManager@@QAEHV?$CStringT@DV?$StrTraitMFC_DLL@DV?$ChTraitsCRT@D@ATL@@@@@ATL@@@Z$1 00478909 f   ClientInfoManager.obj
 0001:00077911       __unwindfunclet$?RemoveOneFromBlack@CClientInfoManager@@QAEHV?$CStringT@DV?$StrTraitMFC_DLL@DV?$ChTraitsCRT@D@ATL@@@@@ATL@@@Z$3 00478911 f   ClientInfoManager.obj
 0001:0007791a       __ehhandler$?RemoveOneFromBlack@CClientInfoManager@@QAEHV?$CStringT@DV?$StrTraitMFC_DLL@DV?$ChTraitsCRT@D@ATL@@@@@ATL@@@Z 0047891a f   ClientInfoManager.obj
 0001:00077940       __unwindfunclet$?LoadBlackListToMap@CClientInfoManager@@QAEHXZ$0 00478940 f   ClientInfoManager.obj
 0001:00077949       __unwindfunclet$?LoadBlackListToMap@CClientInfoManager@@QAEHXZ$1 00478949 f   ClientInfoManager.obj
 0001:00077951       __ehhandler$?LoadBlackListToMap@CClientInfoManager@@QAEHXZ 00478951 f   ClientInfoManager.obj
 0001:00077970       __unwindfunclet$?InsertClientToGroup@CClientInfoManager@@QAEHUtagGroupClient@@@Z$0 00478970 f   ClientInfoManager.obj
 0001:00077979       __unwindfunclet$?InsertClientToGroup@CClientInfoManager@@QAEHUtagGroupClient@@@Z$2 00478979 f   ClientInfoManager.obj
 0001:00077982       __unwindfunclet$?InsertClientToGroup@CClientInfoManager@@QAEHUtagGroupClient@@@Z$3 00478982 f   ClientInfoManager.obj
 0001:0007798b       __unwindfunclet$?InsertClientToGroup@CClientInfoManager@@QAEHUtagGroupClient@@@Z$4 0047898b f   ClientInfoManager.obj
 0001:00077995       __ehhandler$?InsertClientToGroup@CClientInfoManager@@QAEHUtagGroupClient@@@Z 00478995 f   ClientInfoManager.obj
 0001:000779b0       __unwindfunclet$?UpdateGroupInfoOfClient@CClientInfoManager@@QAEHUtagGroupClient@@@Z$0 004789b0 f   ClientInfoManager.obj
 0001:000779b9       __unwindfunclet$?UpdateGroupInfoOfClient@CClientInfoManager@@QAEHUtagGroupClient@@@Z$1 004789b9 f   ClientInfoManager.obj
 0001:000779c2       __unwindfunclet$?UpdateGroupInfoOfClient@CClientInfoManager@@QAEHUtagGroupClient@@@Z$2 004789c2 f   ClientInfoManager.obj
 0001:000779cb       __unwindfunclet$?UpdateGroupInfoOfClient@CClientInfoManager@@QAEHUtagGroupClient@@@Z$4 004789cb f   ClientInfoManager.obj
 0001:000779d4       __unwindfunclet$?UpdateGroupInfoOfClient@CClientInfoManager@@QAEHUtagGroupClient@@@Z$5 004789d4 f   ClientInfoManager.obj
 0001:000779de       __unwindfunclet$?UpdateGroupInfoOfClient@CClientInfoManager@@QAEHUtagGroupClient@@@Z$6 004789de f   ClientInfoManager.obj
 0001:000779e7       __ehhandler$?UpdateGroupInfoOfClient@CClientInfoManager@@QAEHUtagGroupClient@@@Z 004789e7 f   ClientInfoManager.obj
 0001:00077a10       __unwindfunclet$?ClearAllFromGroupMap@CClientInfoManager@@QAEXXZ$0 00478a10 f   ClientInfoManager.obj
 0001:00077a19       __ehhandler$?ClearAllFromGroupMap@CClientInfoManager@@QAEXXZ 00478a19 f   ClientInfoManager.obj
 0001:00077a40       __unwindfunclet$?InsertNewGroup@CClientInfoManager@@QAEHV?$CStringT@DV?$StrTraitMFC_DLL@DV?$ChTraitsCRT@D@ATL@@@@@ATL@@@Z$0 00478a40 f   ClientInfoManager.obj
 0001:00077a49       __unwindfunclet$?InsertNewGroup@CClientInfoManager@@QAEHV?$CStringT@DV?$StrTraitMFC_DLL@DV?$ChTraitsCRT@D@ATL@@@@@ATL@@@Z$1 00478a49 f   ClientInfoManager.obj
 0001:00077a52       __unwindfunclet$?InsertNewGroup@CClientInfoManager@@QAEHV?$CStringT@DV?$StrTraitMFC_DLL@DV?$ChTraitsCRT@D@ATL@@@@@ATL@@@Z$2 00478a52 f   ClientInfoManager.obj
 0001:00077a5b       __unwindfunclet$?InsertNewGroup@CClientInfoManager@@QAEHV?$CStringT@DV?$StrTraitMFC_DLL@DV?$ChTraitsCRT@D@ATL@@@@@ATL@@@Z$3 00478a5b f   ClientInfoManager.obj
 0001:00077a64       __unwindfunclet$?InsertNewGroup@CClientInfoManager@@QAEHV?$CStringT@DV?$StrTraitMFC_DLL@DV?$ChTraitsCRT@D@ATL@@@@@ATL@@@Z$5 00478a64 f   ClientInfoManager.obj
 0001:00077a6d       __unwindfunclet$?InsertNewGroup@CClientInfoManager@@QAEHV?$CStringT@DV?$StrTraitMFC_DLL@DV?$ChTraitsCRT@D@ATL@@@@@ATL@@@Z$6 00478a6d f   ClientInfoManager.obj
 0001:00077a77       __ehhandler$?InsertNewGroup@CClientInfoManager@@QAEHV?$CStringT@DV?$StrTraitMFC_DLL@DV?$ChTraitsCRT@D@ATL@@@@@ATL@@@Z 00478a77 f   ClientInfoManager.obj
 0001:00077aa0       __unwindfunclet$?LoadGroupClientToMap@CClientInfoManager@@QAEHXZ$0 00478aa0 f   ClientInfoManager.obj
 0001:00077aa9       __unwindfunclet$?LoadGroupClientToMap@CClientInfoManager@@QAEHXZ$1 00478aa9 f   ClientInfoManager.obj
 0001:00077ab1       __unwindfunclet$?LoadGroupClientToMap@CClientInfoManager@@QAEHXZ$2 00478ab1 f   ClientInfoManager.obj
 0001:00077aba       __unwindfunclet$?LoadGroupClientToMap@CClientInfoManager@@QAEHXZ$3 00478aba f   ClientInfoManager.obj
 0001:00077ac7       __unwindfunclet$?LoadGroupClientToMap@CClientInfoManager@@QAEHXZ$5 00478ac7 f   ClientInfoManager.obj
 0001:00077ad3       __unwindfunclet$?LoadGroupClientToMap@CClientInfoManager@@QAEHXZ$6 00478ad3 f   ClientInfoManager.obj
 0001:00077adc       __unwindfunclet$?LoadGroupClientToMap@CClientInfoManager@@QAEHXZ$8 00478adc f   ClientInfoManager.obj
 0001:00077ae5       __unwindfunclet$?LoadGroupClientToMap@CClientInfoManager@@QAEHXZ$9 00478ae5 f   ClientInfoManager.obj
 0001:00077aed       __unwindfunclet$?LoadGroupClientToMap@CClientInfoManager@@QAEHXZ$11 00478aed f   ClientInfoManager.obj
 0001:00077af9       __unwindfunclet$?LoadGroupClientToMap@CClientInfoManager@@QAEHXZ$12 00478af9 f   ClientInfoManager.obj
 0001:00077b06       __unwindfunclet$?LoadGroupClientToMap@CClientInfoManager@@QAEHXZ$13 00478b06 f   ClientInfoManager.obj
 0001:00077b12       __unwindfunclet$?LoadGroupClientToMap@CClientInfoManager@@QAEHXZ$15 00478b12 f   ClientInfoManager.obj
 0001:00077b1e       __unwindfunclet$?LoadGroupClientToMap@CClientInfoManager@@QAEHXZ$17 00478b1e f   ClientInfoManager.obj
 0001:00077b2a       __ehhandler$?LoadGroupClientToMap@CClientInfoManager@@QAEHXZ 00478b2a f   ClientInfoManager.obj
 0001:00077b60       __unwindfunclet$?UpdateGroupInfoByOldGroupName@CClientInfoManager@@QAEHV?$CStringT@DV?$StrTraitMFC_DLL@DV?$ChTraitsCRT@D@ATL@@@@@ATL@@UtagGroupClient@@@Z$0 00478b60 f   ClientInfoManager.obj
 0001:00077b69       __unwindfunclet$?UpdateGroupInfoByOldGroupName@CClientInfoManager@@QAEHV?$CStringT@DV?$StrTraitMFC_DLL@DV?$ChTraitsCRT@D@ATL@@@@@ATL@@UtagGroupClient@@@Z$2 00478b69 f   ClientInfoManager.obj
 0001:00077b72       __ehhandler$?UpdateGroupInfoByOldGroupName@CClientInfoManager@@QAEHV?$CStringT@DV?$StrTraitMFC_DLL@DV?$ChTraitsCRT@D@ATL@@@@@ATL@@UtagGroupClient@@@Z 00478b72 f   ClientInfoManager.obj
 0001:00077b90       __unwindfunclet$?UpdateGroup@CClientInfoManager@@QAEHV?$CStringT@DV?$StrTraitMFC_DLL@DV?$ChTraitsCRT@D@ATL@@@@@ATL@@0@Z$0 00478b90 f   ClientInfoManager.obj
 0001:00077b99       __unwindfunclet$?UpdateGroup@CClientInfoManager@@QAEHV?$CStringT@DV?$StrTraitMFC_DLL@DV?$ChTraitsCRT@D@ATL@@@@@ATL@@0@Z$1 00478b99 f   ClientInfoManager.obj
 0001:00077ba2       __unwindfunclet$?UpdateGroup@CClientInfoManager@@QAEHV?$CStringT@DV?$StrTraitMFC_DLL@DV?$ChTraitsCRT@D@ATL@@@@@ATL@@0@Z$2 00478ba2 f   ClientInfoManager.obj
 0001:00077bab       __unwindfunclet$?UpdateGroup@CClientInfoManager@@QAEHV?$CStringT@DV?$StrTraitMFC_DLL@DV?$ChTraitsCRT@D@ATL@@@@@ATL@@0@Z$4 00478bab f   ClientInfoManager.obj
 0001:00077bb4       __ehhandler$?UpdateGroup@CClientInfoManager@@QAEHV?$CStringT@DV?$StrTraitMFC_DLL@DV?$ChTraitsCRT@D@ATL@@@@@ATL@@0@Z 00478bb4 f   ClientInfoManager.obj
 0001:00077bd0       __unwindfunclet$?RemoveGroup@CClientInfoManager@@QAEHV?$CStringT@DV?$StrTraitMFC_DLL@DV?$ChTraitsCRT@D@ATL@@@@@ATL@@@Z$0 00478bd0 f   ClientInfoManager.obj
 0001:00077bd9       __unwindfunclet$?RemoveGroup@CClientInfoManager@@QAEHV?$CStringT@DV?$StrTraitMFC_DLL@DV?$ChTraitsCRT@D@ATL@@@@@ATL@@@Z$2 00478bd9 f   ClientInfoManager.obj
 0001:00077be2       __ehhandler$?RemoveGroup@CClientInfoManager@@QAEHV?$CStringT@DV?$StrTraitMFC_DLL@DV?$ChTraitsCRT@D@ATL@@@@@ATL@@@Z 00478be2 f   ClientInfoManager.obj
 0001:00077c00       __unwindfunclet$?UpdateOneToGroup@CClientInfoManager@@QAEHUtagGroupClient@@@Z$0 00478c00 f   ClientInfoManager.obj
 0001:00077c09       __unwindfunclet$?UpdateOneToGroup@CClientInfoManager@@QAEHUtagGroupClient@@@Z$1 00478c09 f   ClientInfoManager.obj
 0001:00077c12       __ehhandler$?UpdateOneToGroup@CClientInfoManager@@QAEHUtagGroupClient@@@Z 00478c12 f   ClientInfoManager.obj
 0001:00077c30       __unwindfunclet$?RemoveOneGroupCLient@CClientInfoManager@@QAEHV?$CStringT@DV?$StrTraitMFC_DLL@DV?$ChTraitsCRT@D@ATL@@@@@ATL@@@Z$0 00478c30 f   ClientInfoManager.obj
 0001:00077c39       __unwindfunclet$?RemoveOneGroupCLient@CClientInfoManager@@QAEHV?$CStringT@DV?$StrTraitMFC_DLL@DV?$ChTraitsCRT@D@ATL@@@@@ATL@@@Z$2 00478c39 f   ClientInfoManager.obj
 0001:00077c42       __unwindfunclet$?RemoveOneGroupCLient@CClientInfoManager@@QAEHV?$CStringT@DV?$StrTraitMFC_DLL@DV?$ChTraitsCRT@D@ATL@@@@@ATL@@@Z$3 00478c42 f   ClientInfoManager.obj
 0001:00077c4b       __ehhandler$?RemoveOneGroupCLient@CClientInfoManager@@QAEHV?$CStringT@DV?$StrTraitMFC_DLL@DV?$ChTraitsCRT@D@ATL@@@@@ATL@@@Z 00478c4b f   ClientInfoManager.obj
 0001:00077c70       __unwindfunclet$?RemoveKey@?$CTypedPtrMap@VCMapStringToPtr@@V?$CStringT@DV?$StrTraitMFC_DLL@DV?$ChTraitsCRT@D@ATL@@@@@ATL@@PAUtagCLIENTMAININFO@@@@QAEHV?$CStringT@DV?$StrTraitMFC_DLL@DV?$ChTraitsCRT@D@ATL@@@@@ATL@@@Z$0 00478c70 f   ClientInfoManager.obj
 0001:00077c70       __unwindfunclet$?RemoveKey@?$CTypedPtrMap@VCMapStringToPtr@@V?$CStringT@DV?$StrTraitMFC_DLL@DV?$ChTraitsCRT@D@ATL@@@@@ATL@@PAVCStringList@@@@QAEHV?$CStringT@DV?$StrTraitMFC_DLL@DV?$ChTraitsCRT@D@ATL@@@@@ATL@@@Z$0 00478c70 f   ClientInfoManager.obj
 0001:00077c70       __unwindfunclet$?RemoveKey@?$CTypedPtrMap@VCMapStringToPtr@@V?$CStringT@DV?$StrTraitMFC_DLL@DV?$ChTraitsCRT@D@ATL@@@@@ATL@@PAUtagBLACKLIST@@@@QAEHV?$CStringT@DV?$StrTraitMFC_DLL@DV?$ChTraitsCRT@D@ATL@@@@@ATL@@@Z$0 00478c70 f   ClientInfoManager.obj
 0001:00077c70       __unwindfunclet$?RemoveKey@?$CTypedPtrMap@VCMapStringToPtr@@V?$CStringT@DV?$StrTraitMFC_DLL@DV?$ChTraitsCRT@D@ATL@@@@@ATL@@PAV23@@@QAEHV?$CStringT@DV?$StrTraitMFC_DLL@DV?$ChTraitsCRT@D@ATL@@@@@ATL@@@Z$0 00478c70 f   ClientInfoManager.obj
 0001:00077c79       __ehhandler$?RemoveKey@?$CTypedPtrMap@VCMapStringToPtr@@V?$CStringT@DV?$StrTraitMFC_DLL@DV?$ChTraitsCRT@D@ATL@@@@@ATL@@PAVCStringList@@@@QAEHV?$CStringT@DV?$StrTraitMFC_DLL@DV?$ChTraitsCRT@D@ATL@@@@@ATL@@@Z 00478c79 f   ClientInfoManager.obj
 0001:00077c79       __ehhandler$?RemoveKey@?$CTypedPtrMap@VCMapStringToPtr@@V?$CStringT@DV?$StrTraitMFC_DLL@DV?$ChTraitsCRT@D@ATL@@@@@ATL@@PAV23@@@QAEHV?$CStringT@DV?$StrTraitMFC_DLL@DV?$ChTraitsCRT@D@ATL@@@@@ATL@@@Z 00478c79 f   ClientInfoManager.obj
 0001:00077c79       __ehhandler$?RemoveKey@?$CTypedPtrMap@VCMapStringToPtr@@V?$CStringT@DV?$StrTraitMFC_DLL@DV?$ChTraitsCRT@D@ATL@@@@@ATL@@PAUtagCLIENTMAININFO@@@@QAEHV?$CStringT@DV?$StrTraitMFC_DLL@DV?$ChTraitsCRT@D@ATL@@@@@ATL@@@Z 00478c79 f   ClientInfoManager.obj
 0001:00077c79       __ehhandler$?RemoveKey@?$CTypedPtrMap@VCMapStringToPtr@@V?$CStringT@DV?$StrTraitMFC_DLL@DV?$ChTraitsCRT@D@ATL@@@@@ATL@@PAUtagBLACKLIST@@@@QAEHV?$CStringT@DV?$StrTraitMFC_DLL@DV?$ChTraitsCRT@D@ATL@@@@@ATL@@@Z 00478c79 f   ClientInfoManager.obj
 0001:00077ca0       __unwindfunclet$??0CClientSettingsDlg@@QAE@PAVCWnd@@@Z$0 00478ca0 f   ClientSettingsDlg.obj
 0001:00077ca8       __unwindfunclet$??0CClientSettingsDlg@@QAE@PAVCWnd@@@Z$1 00478ca8 f   ClientSettingsDlg.obj
 0001:00077cb3       __unwindfunclet$??0CClientSettingsDlg@@QAE@PAVCWnd@@@Z$2 00478cb3 f   ClientSettingsDlg.obj
 0001:00077cc1       __unwindfunclet$??0CClientSettingsDlg@@QAE@PAVCWnd@@@Z$3 00478cc1 f   ClientSettingsDlg.obj
 0001:00077ccf       __unwindfunclet$??0CClientSettingsDlg@@QAE@PAVCWnd@@@Z$4 00478ccf f   ClientSettingsDlg.obj
 0001:00077cde       __unwindfunclet$??0CClientSettingsDlg@@QAE@PAVCWnd@@@Z$5 00478cde f   ClientSettingsDlg.obj
 0001:00077ced       __unwindfunclet$??0CClientSettingsDlg@@QAE@PAVCWnd@@@Z$6 00478ced f   ClientSettingsDlg.obj
 0001:00077cfc       __unwindfunclet$??0CClientSettingsDlg@@QAE@PAVCWnd@@@Z$7 00478cfc f   ClientSettingsDlg.obj
 0001:00077d0b       __unwindfunclet$??0CClientSettingsDlg@@QAE@PAVCWnd@@@Z$8 00478d0b f   ClientSettingsDlg.obj
 0001:00077d1a       __unwindfunclet$??0CClientSettingsDlg@@QAE@PAVCWnd@@@Z$9 00478d1a f   ClientSettingsDlg.obj
 0001:00077d29       __unwindfunclet$??0CClientSettingsDlg@@QAE@PAVCWnd@@@Z$10 00478d29 f   ClientSettingsDlg.obj
 0001:00077d38       __unwindfunclet$??0CClientSettingsDlg@@QAE@PAVCWnd@@@Z$11 00478d38 f   ClientSettingsDlg.obj
 0001:00077d46       __unwindfunclet$??0CClientSettingsDlg@@QAE@PAVCWnd@@@Z$12 00478d46 f   ClientSettingsDlg.obj
 0001:00077d54       __unwindfunclet$??0CClientSettingsDlg@@QAE@PAVCWnd@@@Z$13 00478d54 f   ClientSettingsDlg.obj
 0001:00077d62       __unwindfunclet$??0CClientSettingsDlg@@QAE@PAVCWnd@@@Z$14 00478d62 f   ClientSettingsDlg.obj
 0001:00077d70       __unwindfunclet$??0CClientSettingsDlg@@QAE@PAVCWnd@@@Z$15 00478d70 f   ClientSettingsDlg.obj
 0001:00077d7e       __ehhandler$??0CClientSettingsDlg@@QAE@PAVCWnd@@@Z 00478d7e f   ClientSettingsDlg.obj
 0001:00077da0       __unwindfunclet$??1CClientSettingsDlg@@UAE@XZ$0 00478da0 f   ClientSettingsDlg.obj
 0001:00077da8       __unwindfunclet$??1CClientSettingsDlg@@UAE@XZ$1 00478da8 f   ClientSettingsDlg.obj
 0001:00077db3       __unwindfunclet$??1CClientSettingsDlg@@UAE@XZ$2 00478db3 f   ClientSettingsDlg.obj
 0001:00077dc1       __unwindfunclet$??1CClientSettingsDlg@@UAE@XZ$3 00478dc1 f   ClientSettingsDlg.obj
 0001:00077dcf       __unwindfunclet$??1CClientSettingsDlg@@UAE@XZ$4 00478dcf f   ClientSettingsDlg.obj
 0001:00077dde       __unwindfunclet$??1CClientSettingsDlg@@UAE@XZ$5 00478dde f   ClientSettingsDlg.obj
 0001:00077ded       __unwindfunclet$??1CClientSettingsDlg@@UAE@XZ$6 00478ded f   ClientSettingsDlg.obj
 0001:00077dfc       __unwindfunclet$??1CClientSettingsDlg@@UAE@XZ$7 00478dfc f   ClientSettingsDlg.obj
 0001:00077e0b       __unwindfunclet$??1CClientSettingsDlg@@UAE@XZ$8 00478e0b f   ClientSettingsDlg.obj
 0001:00077e1a       __unwindfunclet$??1CClientSettingsDlg@@UAE@XZ$9 00478e1a f   ClientSettingsDlg.obj
 0001:00077e29       __unwindfunclet$??1CClientSettingsDlg@@UAE@XZ$10 00478e29 f   ClientSettingsDlg.obj
 0001:00077e38       __unwindfunclet$??1CClientSettingsDlg@@UAE@XZ$11 00478e38 f   ClientSettingsDlg.obj
 0001:00077e46       __unwindfunclet$??1CClientSettingsDlg@@UAE@XZ$12 00478e46 f   ClientSettingsDlg.obj
 0001:00077e54       __unwindfunclet$??1CClientSettingsDlg@@UAE@XZ$13 00478e54 f   ClientSettingsDlg.obj
 0001:00077e62       __unwindfunclet$??1CClientSettingsDlg@@UAE@XZ$14 00478e62 f   ClientSettingsDlg.obj
 0001:00077e70       __ehhandler$??1CClientSettingsDlg@@UAE@XZ 00478e70 f   ClientSettingsDlg.obj
 0001:00077e90       __unwindfunclet$?OnOK@CClientSettingsDlg@@MAEXXZ$4 00478e90 f   ClientSettingsDlg.obj
 0001:00077e99       __unwindfunclet$?OnOK@CClientSettingsDlg@@MAEXXZ$5 00478e99 f   ClientSettingsDlg.obj
 0001:00077ea2       __unwindfunclet$?OnOK@CClientSettingsDlg@@MAEXXZ$6 00478ea2 f   ClientSettingsDlg.obj
 0001:00077eab       __unwindfunclet$?OnOK@CClientSettingsDlg@@MAEXXZ$7 00478eab f   ClientSettingsDlg.obj
 0001:00077eb4       __unwindfunclet$?OnOK@CClientSettingsDlg@@MAEXXZ$8 00478eb4 f   ClientSettingsDlg.obj
 0001:00077ebd       __unwindfunclet$?OnOK@CClientSettingsDlg@@MAEXXZ$9 00478ebd f   ClientSettingsDlg.obj
 0001:00077ec6       __unwindfunclet$?OnOK@CClientSettingsDlg@@MAEXXZ$10 00478ec6 f   ClientSettingsDlg.obj
 0001:00077ecf       __unwindfunclet$?OnOK@CClientSettingsDlg@@MAEXXZ$11 00478ecf f   ClientSettingsDlg.obj
 0001:00077ed8       __unwindfunclet$?OnOK@CClientSettingsDlg@@MAEXXZ$12 00478ed8 f   ClientSettingsDlg.obj
 0001:00077ee1       __unwindfunclet$?OnOK@CClientSettingsDlg@@MAEXXZ$13 00478ee1 f   ClientSettingsDlg.obj
 0001:00077eea       __unwindfunclet$?OnOK@CClientSettingsDlg@@MAEXXZ$16 00478eea f   ClientSettingsDlg.obj
 0001:00077ef3       __unwindfunclet$?OnOK@CClientSettingsDlg@@MAEXXZ$20 00478ef3 f   ClientSettingsDlg.obj
 0001:00077eff       __unwindfunclet$?OnOK@CClientSettingsDlg@@MAEXXZ$21 00478eff f   ClientSettingsDlg.obj
 0001:00077f0b       __unwindfunclet$?OnOK@CClientSettingsDlg@@MAEXXZ$22 00478f0b f   ClientSettingsDlg.obj
 0001:00077f17       __unwindfunclet$?OnOK@CClientSettingsDlg@@MAEXXZ$23 00478f17 f   ClientSettingsDlg.obj
 0001:00077f23       __unwindfunclet$?OnOK@CClientSettingsDlg@@MAEXXZ$24 00478f23 f   ClientSettingsDlg.obj
 0001:00077f2f       __unwindfunclet$?OnOK@CClientSettingsDlg@@MAEXXZ$25 00478f2f f   ClientSettingsDlg.obj
 0001:00077f3b       __unwindfunclet$?OnOK@CClientSettingsDlg@@MAEXXZ$26 00478f3b f   ClientSettingsDlg.obj
 0001:00077f47       __unwindfunclet$?OnOK@CClientSettingsDlg@@MAEXXZ$27 00478f47 f   ClientSettingsDlg.obj
 0001:00077f53       __ehhandler$?OnOK@CClientSettingsDlg@@MAEXXZ 00478f53 f   ClientSettingsDlg.obj
 0001:00077f80       __unwindfunclet$?OnInitDialog@CClientSettingsDlg@@MAEHXZ$0 00478f80 f   ClientSettingsDlg.obj
 0001:00077f89       __unwindfunclet$?OnInitDialog@CClientSettingsDlg@@MAEHXZ$1 00478f89 f   ClientSettingsDlg.obj
 0001:00077f92       __unwindfunclet$?OnInitDialog@CClientSettingsDlg@@MAEHXZ$2 00478f92 f   ClientSettingsDlg.obj
 0001:00077f9b       __unwindfunclet$?OnInitDialog@CClientSettingsDlg@@MAEHXZ$3 00478f9b f   ClientSettingsDlg.obj
 0001:00077fa4       __unwindfunclet$?OnInitDialog@CClientSettingsDlg@@MAEHXZ$4 00478fa4 f   ClientSettingsDlg.obj
 0001:00077fad       __unwindfunclet$?OnInitDialog@CClientSettingsDlg@@MAEHXZ$5 00478fad f   ClientSettingsDlg.obj
 0001:00077fb6       __unwindfunclet$?OnInitDialog@CClientSettingsDlg@@MAEHXZ$6 00478fb6 f   ClientSettingsDlg.obj
 0001:00077fbf       __unwindfunclet$?OnInitDialog@CClientSettingsDlg@@MAEHXZ$7 00478fbf f   ClientSettingsDlg.obj
 0001:00077fc8       __unwindfunclet$?OnInitDialog@CClientSettingsDlg@@MAEHXZ$8 00478fc8 f   ClientSettingsDlg.obj
 0001:00077fd1       __unwindfunclet$?OnInitDialog@CClientSettingsDlg@@MAEHXZ$9 00478fd1 f   ClientSettingsDlg.obj
 0001:00077fda       __unwindfunclet$?OnInitDialog@CClientSettingsDlg@@MAEHXZ$10 00478fda f   ClientSettingsDlg.obj
 0001:00077fe3       __unwindfunclet$?OnInitDialog@CClientSettingsDlg@@MAEHXZ$11 00478fe3 f   ClientSettingsDlg.obj
 0001:00077fec       __unwindfunclet$?OnInitDialog@CClientSettingsDlg@@MAEHXZ$12 00478fec f   ClientSettingsDlg.obj
 0001:00077ff5       __unwindfunclet$?OnInitDialog@CClientSettingsDlg@@MAEHXZ$13 00478ff5 f   ClientSettingsDlg.obj
 0001:00077ffe       __unwindfunclet$?OnInitDialog@CClientSettingsDlg@@MAEHXZ$14 00478ffe f   ClientSettingsDlg.obj
 0001:00078007       __unwindfunclet$?OnInitDialog@CClientSettingsDlg@@MAEHXZ$15 00479007 f   ClientSettingsDlg.obj
 0001:00078010       __unwindfunclet$?OnInitDialog@CClientSettingsDlg@@MAEHXZ$16 00479010 f   ClientSettingsDlg.obj
 0001:00078019       __unwindfunclet$?OnInitDialog@CClientSettingsDlg@@MAEHXZ$17 00479019 f   ClientSettingsDlg.obj
 0001:00078022       __unwindfunclet$?OnInitDialog@CClientSettingsDlg@@MAEHXZ$18 00479022 f   ClientSettingsDlg.obj
 0001:0007802b       __unwindfunclet$?OnInitDialog@CClientSettingsDlg@@MAEHXZ$19 0047902b f   ClientSettingsDlg.obj
 0001:00078034       __unwindfunclet$?OnInitDialog@CClientSettingsDlg@@MAEHXZ$20 00479034 f   ClientSettingsDlg.obj
 0001:0007803d       __unwindfunclet$?OnInitDialog@CClientSettingsDlg@@MAEHXZ$21 0047903d f   ClientSettingsDlg.obj
 0001:00078046       __unwindfunclet$?OnInitDialog@CClientSettingsDlg@@MAEHXZ$22 00479046 f   ClientSettingsDlg.obj
 0001:0007804f       __unwindfunclet$?OnInitDialog@CClientSettingsDlg@@MAEHXZ$23 0047904f f   ClientSettingsDlg.obj
 0001:00078058       __unwindfunclet$?OnInitDialog@CClientSettingsDlg@@MAEHXZ$24 00479058 f   ClientSettingsDlg.obj
 0001:00078061       __unwindfunclet$?OnInitDialog@CClientSettingsDlg@@MAEHXZ$25 00479061 f   ClientSettingsDlg.obj
 0001:0007806a       __unwindfunclet$?OnInitDialog@CClientSettingsDlg@@MAEHXZ$26 0047906a f   ClientSettingsDlg.obj
 0001:00078073       __unwindfunclet$?OnInitDialog@CClientSettingsDlg@@MAEHXZ$27 00479073 f   ClientSettingsDlg.obj
 0001:0007807c       __unwindfunclet$?OnInitDialog@CClientSettingsDlg@@MAEHXZ$28 0047907c f   ClientSettingsDlg.obj
 0001:00078085       __unwindfunclet$?OnInitDialog@CClientSettingsDlg@@MAEHXZ$29 00479085 f   ClientSettingsDlg.obj
 0001:00078091       __unwindfunclet$?OnInitDialog@CClientSettingsDlg@@MAEHXZ$30 00479091 f   ClientSettingsDlg.obj
 0001:0007809d       __unwindfunclet$?OnInitDialog@CClientSettingsDlg@@MAEHXZ$31 0047909d f   ClientSettingsDlg.obj
 0001:000780a9       __unwindfunclet$?OnInitDialog@CClientSettingsDlg@@MAEHXZ$32 004790a9 f   ClientSettingsDlg.obj
 0001:000780b5       __unwindfunclet$?OnInitDialog@CClientSettingsDlg@@MAEHXZ$33 004790b5 f   ClientSettingsDlg.obj
 0001:000780c1       __unwindfunclet$?OnInitDialog@CClientSettingsDlg@@MAEHXZ$34 004790c1 f   ClientSettingsDlg.obj
 0001:000780cd       __unwindfunclet$?OnInitDialog@CClientSettingsDlg@@MAEHXZ$35 004790cd f   ClientSettingsDlg.obj
 0001:000780d9       __unwindfunclet$?OnInitDialog@CClientSettingsDlg@@MAEHXZ$36 004790d9 f   ClientSettingsDlg.obj
 0001:000780e5       __unwindfunclet$?OnInitDialog@CClientSettingsDlg@@MAEHXZ$37 004790e5 f   ClientSettingsDlg.obj
 0001:000780f1       __unwindfunclet$?OnInitDialog@CClientSettingsDlg@@MAEHXZ$38 004790f1 f   ClientSettingsDlg.obj
 0001:000780fd       __ehhandler$?OnInitDialog@CClientSettingsDlg@@MAEHXZ 004790fd f   ClientSettingsDlg.obj
 0001:00078120       __unwindfunclet$?OnDblclkPartitionList@CClientSettingsDlg@@IAEXPAUtagNMHDR@@PAJ@Z$1 00479120 f   ClientSettingsDlg.obj
 0001:0007812b       __unwindfunclet$?OnDblclkPartitionList@CClientSettingsDlg@@IAEXPAUtagNMHDR@@PAJ@Z$2 0047912b f   ClientSettingsDlg.obj
 0001:00078137       __unwindfunclet$?OnDblclkPartitionList@CClientSettingsDlg@@IAEXPAUtagNMHDR@@PAJ@Z$3 00479137 f   ClientSettingsDlg.obj
 0001:00078143       __unwindfunclet$?OnDblclkPartitionList@CClientSettingsDlg@@IAEXPAUtagNMHDR@@PAJ@Z$4 00479143 f   ClientSettingsDlg.obj
 0001:0007814f       __unwindfunclet$?OnDblclkPartitionList@CClientSettingsDlg@@IAEXPAUtagNMHDR@@PAJ@Z$5 0047914f f   ClientSettingsDlg.obj
 0001:0007815b       __unwindfunclet$?OnDblclkPartitionList@CClientSettingsDlg@@IAEXPAUtagNMHDR@@PAJ@Z$6 0047915b f   ClientSettingsDlg.obj
 0001:00078167       __unwindfunclet$?OnDblclkPartitionList@CClientSettingsDlg@@IAEXPAUtagNMHDR@@PAJ@Z$7 00479167 f   ClientSettingsDlg.obj
 0001:00078173       __unwindfunclet$?OnDblclkPartitionList@CClientSettingsDlg@@IAEXPAUtagNMHDR@@PAJ@Z$8 00479173 f   ClientSettingsDlg.obj
 0001:0007817f       __ehhandler$?OnDblclkPartitionList@CClientSettingsDlg@@IAEXPAUtagNMHDR@@PAJ@Z 0047917f f   ClientSettingsDlg.obj
 0001:000781b0       __unwindfunclet$??1CPartitionSettingDlg@@UAE@XZ$0 004791b0 f   ClientSettingsDlg.obj
 0001:000781b8       __unwindfunclet$??1CPartitionSettingDlg@@UAE@XZ$1 004791b8 f   ClientSettingsDlg.obj
 0001:000781c6       __unwindfunclet$??1CPartitionSettingDlg@@UAE@XZ$2 004791c6 f   ClientSettingsDlg.obj
 0001:000781d4       __unwindfunclet$??1CPartitionSettingDlg@@UAE@XZ$3 004791d4 f   ClientSettingsDlg.obj
 0001:000781e3       __unwindfunclet$??1CPartitionSettingDlg@@UAE@XZ$4 004791e3 f   ClientSettingsDlg.obj
 0001:000781f2       __unwindfunclet$??1CPartitionSettingDlg@@UAE@XZ$5 004791f2 f   ClientSettingsDlg.obj
 0001:00078201       __unwindfunclet$??1CPartitionSettingDlg@@UAE@XZ$6 00479201 f   ClientSettingsDlg.obj
 0001:00078210       __unwindfunclet$??1CPartitionSettingDlg@@UAE@XZ$7 00479210 f   ClientSettingsDlg.obj
 0001:0007821f       __unwindfunclet$??1CPartitionSettingDlg@@UAE@XZ$8 0047921f f   ClientSettingsDlg.obj
 0001:0007822e       __unwindfunclet$??1CPartitionSettingDlg@@UAE@XZ$9 0047922e f   ClientSettingsDlg.obj
 0001:0007823d       __ehhandler$??1CPartitionSettingDlg@@UAE@XZ 0047923d f   ClientSettingsDlg.obj
 0001:00078260       __unwindfunclet$?InitClientInfoDisplay@CClientSettingsDlg@@QAEXXZ$0 00479260 f   ClientSettingsDlg.obj
 0001:00078269       __unwindfunclet$?InitClientInfoDisplay@CClientSettingsDlg@@QAEXXZ$1 00479269 f   ClientSettingsDlg.obj
 0001:00078272       __unwindfunclet$?InitClientInfoDisplay@CClientSettingsDlg@@QAEXXZ$2 00479272 f   ClientSettingsDlg.obj
 0001:0007827b       __unwindfunclet$?InitClientInfoDisplay@CClientSettingsDlg@@QAEXXZ$3 0047927b f   ClientSettingsDlg.obj
 0001:00078284       __unwindfunclet$?InitClientInfoDisplay@CClientSettingsDlg@@QAEXXZ$4 00479284 f   ClientSettingsDlg.obj
 0001:0007828d       __unwindfunclet$?InitClientInfoDisplay@CClientSettingsDlg@@QAEXXZ$5 0047928d f   ClientSettingsDlg.obj
 0001:00078296       __unwindfunclet$?InitClientInfoDisplay@CClientSettingsDlg@@QAEXXZ$6 00479296 f   ClientSettingsDlg.obj
 0001:0007829f       __unwindfunclet$?InitClientInfoDisplay@CClientSettingsDlg@@QAEXXZ$7 0047929f f   ClientSettingsDlg.obj
 0001:000782a8       __unwindfunclet$?InitClientInfoDisplay@CClientSettingsDlg@@QAEXXZ$8 004792a8 f   ClientSettingsDlg.obj
 0001:000782b1       __unwindfunclet$?InitClientInfoDisplay@CClientSettingsDlg@@QAEXXZ$9 004792b1 f   ClientSettingsDlg.obj
 0001:000782ba       __unwindfunclet$?InitClientInfoDisplay@CClientSettingsDlg@@QAEXXZ$10 004792ba f   ClientSettingsDlg.obj
 0001:000782c3       __unwindfunclet$?InitClientInfoDisplay@CClientSettingsDlg@@QAEXXZ$11 004792c3 f   ClientSettingsDlg.obj
 0001:000782cc       __unwindfunclet$?InitClientInfoDisplay@CClientSettingsDlg@@QAEXXZ$12 004792cc f   ClientSettingsDlg.obj
 0001:000782d5       __unwindfunclet$?InitClientInfoDisplay@CClientSettingsDlg@@QAEXXZ$13 004792d5 f   ClientSettingsDlg.obj
 0001:000782de       __unwindfunclet$?InitClientInfoDisplay@CClientSettingsDlg@@QAEXXZ$14 004792de f   ClientSettingsDlg.obj
 0001:000782e7       __unwindfunclet$?InitClientInfoDisplay@CClientSettingsDlg@@QAEXXZ$15 004792e7 f   ClientSettingsDlg.obj
 0001:000782f0       __ehhandler$?InitClientInfoDisplay@CClientSettingsDlg@@QAEXXZ 004792f0 f   ClientSettingsDlg.obj
 0001:00078320       __unwindfunclet$?GetProtectTypeStr@CClientSettingsDlg@@QAE?AV?$CStringT@DV?$StrTraitMFC_DLL@DV?$ChTraitsCRT@D@ATL@@@@@ATL@@E@Z$0 00479320 f   ClientSettingsDlg.obj
 0001:00078329       __unwindfunclet$?GetProtectTypeStr@CClientSettingsDlg@@QAE?AV?$CStringT@DV?$StrTraitMFC_DLL@DV?$ChTraitsCRT@D@ATL@@@@@ATL@@E@Z$1 00479329 f   ClientSettingsDlg.obj
 0001:00078332       __unwindfunclet$?GetProtectTypeStr@CClientSettingsDlg@@QAE?AV?$CStringT@DV?$StrTraitMFC_DLL@DV?$ChTraitsCRT@D@ATL@@@@@ATL@@E@Z$2 00479332 f   ClientSettingsDlg.obj
 0001:0007833b       __unwindfunclet$?GetProtectTypeStr@CClientSettingsDlg@@QAE?AV?$CStringT@DV?$StrTraitMFC_DLL@DV?$ChTraitsCRT@D@ATL@@@@@ATL@@E@Z$3 0047933b f   ClientSettingsDlg.obj
 0001:00078344       __unwindfunclet$?GetProtectTypeStr@CClientSettingsDlg@@QAE?AV?$CStringT@DV?$StrTraitMFC_DLL@DV?$ChTraitsCRT@D@ATL@@@@@ATL@@E@Z$4 00479344 f   ClientSettingsDlg.obj
 0001:0007834d       __ehhandler$?GetProtectTypeStr@CClientSettingsDlg@@QAE?AV?$CStringT@DV?$StrTraitMFC_DLL@DV?$ChTraitsCRT@D@ATL@@@@@ATL@@E@Z 0047934d f   ClientSettingsDlg.obj
 0001:00078370       __unwindfunclet$?GetFrequenceTypeStr@CClientSettingsDlg@@QAE?AV?$CStringT@DV?$StrTraitMFC_DLL@DV?$ChTraitsCRT@D@ATL@@@@@ATL@@E@Z$0 00479370 f   ClientSettingsDlg.obj
 0001:00078379       __unwindfunclet$?GetFrequenceTypeStr@CClientSettingsDlg@@QAE?AV?$CStringT@DV?$StrTraitMFC_DLL@DV?$ChTraitsCRT@D@ATL@@@@@ATL@@E@Z$1 00479379 f   ClientSettingsDlg.obj
 0001:00078382       __unwindfunclet$?GetFrequenceTypeStr@CClientSettingsDlg@@QAE?AV?$CStringT@DV?$StrTraitMFC_DLL@DV?$ChTraitsCRT@D@ATL@@@@@ATL@@E@Z$2 00479382 f   ClientSettingsDlg.obj
 0001:0007838b       __unwindfunclet$?GetFrequenceTypeStr@CClientSettingsDlg@@QAE?AV?$CStringT@DV?$StrTraitMFC_DLL@DV?$ChTraitsCRT@D@ATL@@@@@ATL@@E@Z$3 0047938b f   ClientSettingsDlg.obj
 0001:00078394       __ehhandler$?GetFrequenceTypeStr@CClientSettingsDlg@@QAE?AV?$CStringT@DV?$StrTraitMFC_DLL@DV?$ChTraitsCRT@D@ATL@@@@@ATL@@E@Z 00479394 f   ClientSettingsDlg.obj
 0001:000783b0       __unwindfunclet$?VerifyPassword@CClientSettingsDlg@@QAE_NV?$CStringT@DV?$StrTraitMFC_DLL@DV?$ChTraitsCRT@D@ATL@@@@@ATL@@@Z$0 004793b0 f   ClientSettingsDlg.obj
 0001:000783b9       __unwindfunclet$?VerifyPassword@CClientSettingsDlg@@QAE_NV?$CStringT@DV?$StrTraitMFC_DLL@DV?$ChTraitsCRT@D@ATL@@@@@ATL@@@Z$1 004793b9 f   ClientSettingsDlg.obj
 0001:000783c2       __ehhandler$?VerifyPassword@CClientSettingsDlg@@QAE_NV?$CStringT@DV?$StrTraitMFC_DLL@DV?$ChTraitsCRT@D@ATL@@@@@ATL@@@Z 004793c2 f   ClientSettingsDlg.obj
 0001:000783e0       __unwindfunclet$??0CCmdEnquireDlg@@QAE@PAVCWnd@@@Z$0 004793e0 f   CmdEnquireDlg.obj
 0001:000783e8       __unwindfunclet$??0CCmdEnquireDlg@@QAE@PAVCWnd@@@Z$1 004793e8 f   CmdEnquireDlg.obj
 0001:000783f4       __unwindfunclet$??0CCmdEnquireDlg@@QAE@PAVCWnd@@@Z$2 004793f4 f   CmdEnquireDlg.obj
 0001:00078400       __unwindfunclet$??0CCmdEnquireDlg@@QAE@PAVCWnd@@@Z$3 00479400 f   CmdEnquireDlg.obj
 0001:0007840b       __unwindfunclet$??0CCmdEnquireDlg@@QAE@PAVCWnd@@@Z$4 0047940b f   CmdEnquireDlg.obj
 0001:00078419       __unwindfunclet$??0CCmdEnquireDlg@@QAE@PAVCWnd@@@Z$5 00479419 f   CmdEnquireDlg.obj
 0001:00078428       __unwindfunclet$??0CCmdEnquireDlg@@QAE@PAVCWnd@@@Z$6 00479428 f   CmdEnquireDlg.obj
 0001:00078431       __ehhandler$??0CCmdEnquireDlg@@QAE@PAVCWnd@@@Z 00479431 f   CmdEnquireDlg.obj
 0001:00078450       __unwindfunclet$??1CCmdEnquireDlg@@UAE@XZ$0 00479450 f   CmdEnquireDlg.obj
 0001:00078458       __unwindfunclet$??1CCmdEnquireDlg@@UAE@XZ$1 00479458 f   CmdEnquireDlg.obj
 0001:00078464       __unwindfunclet$??1CCmdEnquireDlg@@UAE@XZ$2 00479464 f   CmdEnquireDlg.obj
 0001:00078470       __unwindfunclet$??1CCmdEnquireDlg@@UAE@XZ$3 00479470 f   CmdEnquireDlg.obj
 0001:0007847b       __ehhandler$??1CCmdEnquireDlg@@UAE@XZ 0047947b f   CmdEnquireDlg.obj
 0001:000784a0       __unwindfunclet$?IsSameLanguage@@YAHPAD0@Z$0 004794a0 f   CommonFunc.obj
 0001:000784a9       __unwindfunclet$?IsSameLanguage@@YAHPAD0@Z$1 004794a9 f   CommonFunc.obj
 0001:000784b2       __unwindfunclet$?IsSameLanguage@@YAHPAD0@Z$2 004794b2 f   CommonFunc.obj
 0001:000784bb       __ehhandler$?IsSameLanguage@@YAHPAD0@Z 004794bb f   CommonFunc.obj
 0001:000784e0       __unwindfunclet$?IsPhysicalLocalMac@@YAHABV?$CStringT@DV?$StrTraitMFC_DLL@DV?$ChTraitsCRT@D@ATL@@@@@ATL@@@Z$0 004794e0 f   CommonFunc.obj
 0001:000784ec       __unwindfunclet$?IsPhysicalLocalMac@@YAHABV?$CStringT@DV?$StrTraitMFC_DLL@DV?$ChTraitsCRT@D@ATL@@@@@ATL@@@Z$1 004794ec f   CommonFunc.obj
 0001:000784f8       __ehhandler$?IsPhysicalLocalMac@@YAHABV?$CStringT@DV?$StrTraitMFC_DLL@DV?$ChTraitsCRT@D@ATL@@@@@ATL@@@Z 004794f8 f   CommonFunc.obj
 0001:00078520       __unwindfunclet$?GetLocalComputerInfo@@YAHPAD0@Z$0 00479520 f   CommonFunc.obj
 0001:00078529       __unwindfunclet$?GetLocalComputerInfo@@YAHPAD0@Z$1 00479529 f   CommonFunc.obj
 0001:00078535       __unwindfunclet$?GetLocalComputerInfo@@YAHPAD0@Z$2 00479535 f   CommonFunc.obj
 0001:00078540       __unwindfunclet$?GetLocalComputerInfo@@YAHPAD0@Z$4 00479540 f   CommonFunc.obj
 0001:0007854c       __unwindfunclet$?GetLocalComputerInfo@@YAHPAD0@Z$5 0047954c f   CommonFunc.obj
 0001:00078558       __unwindfunclet$?GetLocalComputerInfo@@YAHPAD0@Z$7 00479558 f   CommonFunc.obj
 0001:00078564       __unwindfunclet$?GetLocalComputerInfo@@YAHPAD0@Z$8 00479564 f   CommonFunc.obj
 0001:0007856f       __unwindfunclet$?GetLocalComputerInfo@@YAHPAD0@Z$10 0047956f f   CommonFunc.obj
 0001:0007857b       __unwindfunclet$?GetLocalComputerInfo@@YAHPAD0@Z$12 0047957b f   CommonFunc.obj
 0001:00078587       __unwindfunclet$?GetLocalComputerInfo@@YAHPAD0@Z$13 00479587 f   CommonFunc.obj
 0001:00078592       __unwindfunclet$?GetLocalComputerInfo@@YAHPAD0@Z$15 00479592 f   CommonFunc.obj
 0001:0007859e       __unwindfunclet$?GetLocalComputerInfo@@YAHPAD0@Z$16 0047959e f   CommonFunc.obj
 0001:000785aa       __ehhandler$?GetLocalComputerInfo@@YAHPAD0@Z 004795aa f   CommonFunc.obj
 0001:000785e0       __unwindfunclet$?NICLinknumber@@YAHXZ$0 004795e0 f   CommonFunc.obj
 0001:000785e9       __unwindfunclet$?NICLinknumber@@YAHXZ$1 004795e9 f   CommonFunc.obj
 0001:000785f5       __ehhandler$?NICLinknumber@@YAHXZ 004795f5 f   CommonFunc.obj
 0001:00078620       __unwindfunclet$?ReadParttionPara@@YAHAAUPartion_para_sector_s@@@Z$0 00479620 f   CommonFunc.obj
 0001:0007862b       __ehhandler$?ReadParttionPara@@YAHAAUPartion_para_sector_s@@@Z 0047962b f   CommonFunc.obj
 0001:00078660       __unwindfunclet$?WriteParttionPara@@YAHUPartion_para_sector_s@@H@Z$0 00479660 f   CommonFunc.obj
 0001:0007866b       __ehhandler$?WriteParttionPara@@YAHUPartion_para_sector_s@@H@Z 0047966b f   CommonFunc.obj
 0001:000786a0       __unwindfunclet$?GetfileVersion@@YAHV?$CStringT@DV?$StrTraitMFC_DLL@DV?$ChTraitsCRT@D@ATL@@@@@ATL@@AAV12@@Z$0 004796a0 f   CommonFunc.obj
 0001:000786a9       __unwindfunclet$?GetfileVersion@@YAHV?$CStringT@DV?$StrTraitMFC_DLL@DV?$ChTraitsCRT@D@ATL@@@@@ATL@@AAV12@@Z$1 004796a9 f   CommonFunc.obj
 0001:000786b2       __ehhandler$?GetfileVersion@@YAHV?$CStringT@DV?$StrTraitMFC_DLL@DV?$ChTraitsCRT@D@ATL@@@@@ATL@@AAV12@@Z 004796b2 f   CommonFunc.obj
 0001:000786d0       __unwindfunclet$?OnBtnBrowse@CExecuteProcedure@@QAEXXZ$0 004796d0 f   ExecuteProcedure.obj
 0001:000786db       __unwindfunclet$?OnBtnBrowse@CExecuteProcedure@@QAEXXZ$1 004796db f   ExecuteProcedure.obj
 0001:000786e7       __ehhandler$?OnBtnBrowse@CExecuteProcedure@@QAEXXZ 004796e7 f   ExecuteProcedure.obj
 0001:00078710       __ehhandler$?canclePasvListenSocket@@YA_NPAVCFtpPasvSrv@@@Z 00479710 f   FtpdPi.obj
 0001:00078730       __ehhandler$?deleFtpPI@@YA_NPAVCFtpdPi@@@Z 00479730 f   FtpdPi.obj
 0001:00078750       __unwindfunclet$?thSendData@@YAIPAX@Z$4 00479750 f   FtpdPi.obj
 0001:0007875d       __unwindfunclet$?thSendData@@YAIPAX@Z$5 0047975d f   FtpdPi.obj
 0001:0007876a       __ehhandler$?thSendData@@YAIPAX@Z 0047976a f   FtpdPi.obj
 0001:000787a0       __unwindfunclet$??0CFtpdPi@@QAE@XZ$0 004797a0 f   FtpdPi.obj
 0001:000787a8       __unwindfunclet$??0CFtpdPi@@QAE@XZ$1 004797a8 f   FtpdPi.obj
 0001:000787b6       __unwindfunclet$??0CFtpdPi@@QAE@XZ$2 004797b6 f   FtpdPi.obj
 0001:000787c4       __ehhandler$??0CFtpdPi@@QAE@XZ 004797c4 f   FtpdPi.obj
 0001:000787e0       __unwindfunclet$??1CFtpdPi@@UAE@XZ$0 004797e0 f   FtpdPi.obj
 0001:000787e8       __unwindfunclet$??1CFtpdPi@@UAE@XZ$1 004797e8 f   FtpdPi.obj
 0001:000787f6       __unwindfunclet$??1CFtpdPi@@UAE@XZ$2 004797f6 f   FtpdPi.obj
 0001:00078804       __ehhandler$??1CFtpdPi@@UAE@XZ 00479804 f   FtpdPi.obj
 0001:00078820       __unwindfunclet$?OnReceive@CFtpdPi@@UAEXH@Z$2 00479820 f   FtpdPi.obj
 0001:0007882b       __ehhandler$?OnReceive@CFtpdPi@@UAEXH@Z 0047982b f   FtpdPi.obj
 0001:00078860       __unwindfunclet$?ProcessMsg@CFtpdPi@@QAEXPAD@Z$18 00479860 f   FtpdPi.obj
 0001:0007886d       __unwindfunclet$?ProcessMsg@CFtpdPi@@QAEXPAD@Z$19 0047986d f   FtpdPi.obj
 0001:0007887a       __unwindfunclet$?ProcessMsg@CFtpdPi@@QAEXPAD@Z$20 0047987a f   FtpdPi.obj
 0001:00078887       __unwindfunclet$?ProcessMsg@CFtpdPi@@QAEXPAD@Z$21 00479887 f   FtpdPi.obj
 0001:00078894       __unwindfunclet$?ProcessMsg@CFtpdPi@@QAEXPAD@Z$22 00479894 f   FtpdPi.obj
 0001:000788a1       __unwindfunclet$?ProcessMsg@CFtpdPi@@QAEXPAD@Z$23 004798a1 f   FtpdPi.obj
 0001:000788ae       __unwindfunclet$?ProcessMsg@CFtpdPi@@QAEXPAD@Z$24 004798ae f   FtpdPi.obj
 0001:000788bb       __unwindfunclet$?ProcessMsg@CFtpdPi@@QAEXPAD@Z$25 004798bb f   FtpdPi.obj
 0001:000788c7       __ehhandler$?ProcessMsg@CFtpdPi@@QAEXPAD@Z 004798c7 f   FtpdPi.obj
 0001:000788f0       __ehhandler$?RemoveLeadingSpace@CFtpdPi@@QAEPADPAD@Z 004798f0 f   FtpdPi.obj
 0001:00078910       __ehhandler$?SafeSend@CFtpdPi@@QAEXPAD@Z 00479910 f   FtpdPi.obj
 0001:00078930       __unwindfunclet$?LoadIpRange@CFtpdPi@@QAEXXZ$0 00479930 f   FtpdPi.obj
 0001:00078938       __ehhandler$?LoadIpRange@CFtpdPi@@QAEXXZ 00479938 f   FtpdPi.obj
 0001:00078960       __ehhandler$?ListEngine@CFtpdPi@@QAEXPAD_N@Z 00479960 f   FtpdPi.obj
 0001:00078990       __unwindfunclet$?OnOK@CGroupExt@@UAEXXZ$0 00479990 f   GroupExt.obj
 0001:00078999       __unwindfunclet$?OnOK@CGroupExt@@UAEXXZ$1 00479999 f   GroupExt.obj
 0001:000789a2       __unwindfunclet$?OnOK@CGroupExt@@UAEXXZ$2 004799a2 f   GroupExt.obj
 0001:000789ab       __unwindfunclet$?OnOK@CGroupExt@@UAEXXZ$3 004799ab f   GroupExt.obj
 0001:000789b4       __unwindfunclet$?OnOK@CGroupExt@@UAEXXZ$4 004799b4 f   GroupExt.obj
 0001:000789bd       __unwindfunclet$?OnOK@CGroupExt@@UAEXXZ$5 004799bd f   GroupExt.obj
 0001:000789c6       __unwindfunclet$?OnOK@CGroupExt@@UAEXXZ$6 004799c6 f   GroupExt.obj
 0001:000789cf       __ehhandler$?OnOK@CGroupExt@@UAEXXZ 004799cf f   GroupExt.obj
 0001:000789f0       __unwindfunclet$?OnInitDialog@CGroupExt@@UAEHXZ$0 004799f0 f   GroupExt.obj
 0001:000789f9       __unwindfunclet$?OnInitDialog@CGroupExt@@UAEHXZ$1 004799f9 f   GroupExt.obj
 0001:00078a02       __unwindfunclet$?OnInitDialog@CGroupExt@@UAEHXZ$2 00479a02 f   GroupExt.obj
 0001:00078a0b       __unwindfunclet$?OnInitDialog@CGroupExt@@UAEHXZ$3 00479a0b f   GroupExt.obj
 0001:00078a13       __ehhandler$?OnInitDialog@CGroupExt@@UAEHXZ 00479a13 f   GroupExt.obj
 0001:00078a30       __unwindfunclet$??1CGroupTree@@UAE@XZ$0 00479a30 f   GroupTree.obj
 0001:00078a38       __unwindfunclet$??1CGroupTree@@UAE@XZ$1 00479a38 f   GroupTree.obj
 0001:00078a44       __unwindfunclet$??1CGroupTree@@UAE@XZ$2 00479a44 f   GroupTree.obj
 0001:00078a50       __unwindfunclet$??1CGroupTree@@UAE@XZ$3 00479a50 f   GroupTree.obj
 0001:00078a5f       __ehhandler$??1CGroupTree@@UAE@XZ 00479a5f f   GroupTree.obj
 0001:00078a80       __unwindfunclet$?OnLButtonDown@CGroupTree@@IAEXIVCPoint@@@Z$0 00479a80 f   GroupTree.obj
 0001:00078a89       __unwindfunclet$?OnLButtonDown@CGroupTree@@IAEXIVCPoint@@@Z$1 00479a89 f   GroupTree.obj
 0001:00078a92       __unwindfunclet$?OnLButtonDown@CGroupTree@@IAEXIVCPoint@@@Z$2 00479a92 f   GroupTree.obj
 0001:00078a9b       __ehhandler$?OnLButtonDown@CGroupTree@@IAEXIVCPoint@@@Z 00479a9b f   GroupTree.obj
 0001:00078ac0       __unwindfunclet$?OnRButtonDown@CGroupTree@@IAEXIVCPoint@@@Z$0 00479ac0 f   GroupTree.obj
 0001:00078ac9       __unwindfunclet$?OnRButtonDown@CGroupTree@@IAEXIVCPoint@@@Z$1 00479ac9 f   GroupTree.obj
 0001:00078ad1       __unwindfunclet$?OnRButtonDown@CGroupTree@@IAEXIVCPoint@@@Z$2 00479ad1 f   GroupTree.obj
 0001:00078aeb       __unwindfunclet$?OnRButtonDown@CGroupTree@@IAEXIVCPoint@@@Z$3 00479aeb f   GroupTree.obj
 0001:00078b05       __unwindfunclet$?OnRButtonDown@CGroupTree@@IAEXIVCPoint@@@Z$5 00479b05 f   GroupTree.obj
 0001:00078b0f       __ehhandler$?OnRButtonDown@CGroupTree@@IAEXIVCPoint@@@Z 00479b0f f   GroupTree.obj
 0001:00078b30       __unwindfunclet$?Rename@CGroupTree@@QAEHXZ$0 00479b30 f   GroupTree.obj
 0001:00078b3a       __unwindfunclet$?Rename@CGroupTree@@QAEHXZ$1 00479b3a f   GroupTree.obj
 0001:00078b43       __ehhandler$?Rename@CGroupTree@@QAEHXZ 00479b43 f   GroupTree.obj
 0001:00078b60       __unwindfunclet$?OnTreeAddgroup@CGroupTree@@IAEXXZ$1 00479b60 f   GroupTree.obj
 0001:00078b69       __ehhandler$?OnTreeAddgroup@CGroupTree@@IAEXXZ 00479b69 f   GroupTree.obj
 0001:00078b90       __unwindfunclet$?DelEditObj@CGroupTree@@QAEHXZ$0 00479b90 f   GroupTree.obj
 0001:00078b99       __unwindfunclet$?DelEditObj@CGroupTree@@QAEHXZ$1 00479b99 f   GroupTree.obj
 0001:00078ba2       __unwindfunclet$?DelEditObj@CGroupTree@@QAEHXZ$3 00479ba2 f   GroupTree.obj
 0001:00078bab       __unwindfunclet$?DelEditObj@CGroupTree@@QAEHXZ$5 00479bab f   GroupTree.obj
 0001:00078bb4       __unwindfunclet$?DelEditObj@CGroupTree@@QAEHXZ$7 00479bb4 f   GroupTree.obj
 0001:00078bbd       __unwindfunclet$?DelEditObj@CGroupTree@@QAEHXZ$9 00479bbd f   GroupTree.obj
 0001:00078bc6       __unwindfunclet$?DelEditObj@CGroupTree@@QAEHXZ$12 00479bc6 f   GroupTree.obj
 0001:00078bcf       __unwindfunclet$?DelEditObj@CGroupTree@@QAEHXZ$13 00479bcf f   GroupTree.obj
 0001:00078bd8       __unwindfunclet$?DelEditObj@CGroupTree@@QAEHXZ$14 00479bd8 f   GroupTree.obj
 0001:00078be1       __unwindfunclet$?DelEditObj@CGroupTree@@QAEHXZ$15 00479be1 f   GroupTree.obj
 0001:00078bea       __unwindfunclet$?DelEditObj@CGroupTree@@QAEHXZ$17 00479bea f   GroupTree.obj
 0001:00078bf6       __unwindfunclet$?DelEditObj@CGroupTree@@QAEHXZ$18 00479bf6 f   GroupTree.obj
 0001:00078c02       __unwindfunclet$?DelEditObj@CGroupTree@@QAEHXZ$19 00479c02 f   GroupTree.obj
 0001:00078c0e       __ehhandler$?DelEditObj@CGroupTree@@QAEHXZ 00479c0e f   GroupTree.obj
 0001:00078c30       __unwindfunclet$?OnTreeDelgroup@CGroupTree@@IAEXXZ$0 00479c30 f   GroupTree.obj
 0001:00078c3b       __unwindfunclet$?OnTreeDelgroup@CGroupTree@@IAEXXZ$1 00479c3b f   GroupTree.obj
 0001:00078c47       __unwindfunclet$?OnTreeDelgroup@CGroupTree@@IAEXXZ$2 00479c47 f   GroupTree.obj
 0001:00078c53       __unwindfunclet$?OnTreeDelgroup@CGroupTree@@IAEXXZ$3 00479c53 f   GroupTree.obj
 0001:00078c5f       __unwindfunclet$?OnTreeDelgroup@CGroupTree@@IAEXXZ$4 00479c5f f   GroupTree.obj
 0001:00078c6b       __unwindfunclet$?OnTreeDelgroup@CGroupTree@@IAEXXZ$5 00479c6b f   GroupTree.obj
 0001:00078c77       __unwindfunclet$?OnTreeDelgroup@CGroupTree@@IAEXXZ$6 00479c77 f   GroupTree.obj
 0001:00078c83       __ehhandler$?OnTreeDelgroup@CGroupTree@@IAEXXZ 00479c83 f   GroupTree.obj
 0001:00078cb0       __unwindfunclet$?_DelGroupThread@CGroupTree@@SAIPAX@Z$0 00479cb0 f   GroupTree.obj
 0001:00078cb9       __unwindfunclet$?_DelGroupThread@CGroupTree@@SAIPAX@Z$1 00479cb9 f   GroupTree.obj
 0001:00078cc2       __unwindfunclet$?_DelGroupThread@CGroupTree@@SAIPAX@Z$2 00479cc2 f   GroupTree.obj
 0001:00078ccb       __unwindfunclet$?_DelGroupThread@CGroupTree@@SAIPAX@Z$4 00479ccb f   GroupTree.obj
 0001:00078cd4       __unwindfunclet$?_DelGroupThread@CGroupTree@@SAIPAX@Z$5 00479cd4 f   GroupTree.obj
 0001:00078cdd       __unwindfunclet$?_DelGroupThread@CGroupTree@@SAIPAX@Z$6 00479cdd f   GroupTree.obj
 0001:00078ce6       __unwindfunclet$?_DelGroupThread@CGroupTree@@SAIPAX@Z$7 00479ce6 f   GroupTree.obj
 0001:00078cf2       __unwindfunclet$?_DelGroupThread@CGroupTree@@SAIPAX@Z$8 00479cf2 f   GroupTree.obj
 0001:00078cfe       __unwindfunclet$?_DelGroupThread@CGroupTree@@SAIPAX@Z$9 00479cfe f   GroupTree.obj
 0001:00078d0a       __ehhandler$?_DelGroupThread@CGroupTree@@SAIPAX@Z 00479d0a f   GroupTree.obj
 0001:00078d40       __unwindfunclet$?_RenameGroupThread@CGroupTree@@SAIPAX@Z$0 00479d40 f   GroupTree.obj
 0001:00078d49       __unwindfunclet$?_RenameGroupThread@CGroupTree@@SAIPAX@Z$3 00479d49 f   GroupTree.obj
 0001:00078d52       __unwindfunclet$?_RenameGroupThread@CGroupTree@@SAIPAX@Z$5 00479d52 f   GroupTree.obj
 0001:00078d5b       __unwindfunclet$?_RenameGroupThread@CGroupTree@@SAIPAX@Z$6 00479d5b f   GroupTree.obj
 0001:00078d67       __unwindfunclet$?_RenameGroupThread@CGroupTree@@SAIPAX@Z$7 00479d67 f   GroupTree.obj
 0001:00078d73       __unwindfunclet$?_RenameGroupThread@CGroupTree@@SAIPAX@Z$8 00479d73 f   GroupTree.obj
 0001:00078d7f       __unwindfunclet$?_RenameGroupThread@CGroupTree@@SAIPAX@Z$9 00479d7f f   GroupTree.obj
 0001:00078d8b       __ehhandler$?_RenameGroupThread@CGroupTree@@SAIPAX@Z 00479d8b f   GroupTree.obj
 0001:00078dc0       __unwindfunclet$?GetNewGroupName@CGroupTree@@QAE?AV?$CStringT@DV?$StrTraitMFC_DLL@DV?$ChTraitsCRT@D@ATL@@@@@ATL@@V23@@Z$0 00479dc0 f   GroupTree.obj
 0001:00078dc9       __unwindfunclet$?GetNewGroupName@CGroupTree@@QAE?AV?$CStringT@DV?$StrTraitMFC_DLL@DV?$ChTraitsCRT@D@ATL@@@@@ATL@@V23@@Z$1 00479dc9 f   GroupTree.obj
 0001:00078dd2       __unwindfunclet$?GetNewGroupName@CGroupTree@@QAE?AV?$CStringT@DV?$StrTraitMFC_DLL@DV?$ChTraitsCRT@D@ATL@@@@@ATL@@V23@@Z$2 00479dd2 f   GroupTree.obj
 0001:00078ddb       __unwindfunclet$?GetNewGroupName@CGroupTree@@QAE?AV?$CStringT@DV?$StrTraitMFC_DLL@DV?$ChTraitsCRT@D@ATL@@@@@ATL@@V23@@Z$3 00479ddb f   GroupTree.obj
 0001:00078de4       __unwindfunclet$?GetNewGroupName@CGroupTree@@QAE?AV?$CStringT@DV?$StrTraitMFC_DLL@DV?$ChTraitsCRT@D@ATL@@@@@ATL@@V23@@Z$4 00479de4 f   GroupTree.obj
 0001:00078ded       __unwindfunclet$?GetNewGroupName@CGroupTree@@QAE?AV?$CStringT@DV?$StrTraitMFC_DLL@DV?$ChTraitsCRT@D@ATL@@@@@ATL@@V23@@Z$6 00479ded f   GroupTree.obj
 0001:00078df6       __unwindfunclet$?GetNewGroupName@CGroupTree@@QAE?AV?$CStringT@DV?$StrTraitMFC_DLL@DV?$ChTraitsCRT@D@ATL@@@@@ATL@@V23@@Z$7 00479df6 f   GroupTree.obj
 0001:00078dff       __ehhandler$?GetNewGroupName@CGroupTree@@QAE?AV?$CStringT@DV?$StrTraitMFC_DLL@DV?$ChTraitsCRT@D@ATL@@@@@ATL@@V23@@Z 00479dff f   GroupTree.obj
 0001:00078e20       __unwindfunclet$??0CInfoPromptDlg@@QAE@PAVCWnd@@@Z$0 00479e20 f   InfoPromptDlg.obj
 0001:00078e28       __unwindfunclet$??0CInfoPromptDlg@@QAE@PAVCWnd@@@Z$1 00479e28 f   InfoPromptDlg.obj
 0001:00078e34       __unwindfunclet$??0CInfoPromptDlg@@QAE@PAVCWnd@@@Z$2 00479e34 f   InfoPromptDlg.obj
 0001:00078e40       __ehhandler$??0CInfoPromptDlg@@QAE@PAVCWnd@@@Z 00479e40 f   InfoPromptDlg.obj
 0001:00078e60       __unwindfunclet$??0CIOCPImplement@@QAE@XZ$0 00479e60 f   IOCPImplement.obj
 0001:00078e68       __ehhandler$??0CIOCPImplement@@QAE@XZ 00479e68 f   IOCPImplement.obj
 0001:00078e90       __unwindfunclet$??1CIOCPImplement@@UAE@XZ$0 00479e90 f   IOCPImplement.obj
 0001:00078e98       __unwindfunclet$??1CIOCPImplement@@UAE@XZ$1 00479e98 f   IOCPImplement.obj
 0001:00078ea3       __ehhandler$??1CIOCPImplement@@UAE@XZ 00479ea3 f   IOCPImplement.obj
 0001:00078ec0       __unwindfunclet$?SendAck@CIOCPImplement@@UAEHPAVCClientContext@@@Z$0 00479ec0 f   IOCPImplement.obj
 0001:00078ec9       __ehhandler$?SendAck@CIOCPImplement@@UAEHPAVCClientContext@@@Z 00479ec9 f   IOCPImplement.obj
 0001:00078f00       __unwindfunclet$?InitInstance@CKiboManagerApp@@UAEHXZ$0 00479f00 f   KiboManager.obj
 0001:00078f0c       __unwindfunclet$?InitInstance@CKiboManagerApp@@UAEHXZ$1 00479f0c f   KiboManager.obj
 0001:00078f18       __unwindfunclet$?InitInstance@CKiboManagerApp@@UAEHXZ$2 00479f18 f   KiboManager.obj
 0001:00078f23       __unwindfunclet$?InitInstance@CKiboManagerApp@@UAEHXZ$3 00479f23 f   KiboManager.obj
 0001:00078f30       __unwindfunclet$?InitInstance@CKiboManagerApp@@UAEHXZ$4 00479f30 f   KiboManager.obj
 0001:00078f3b       __unwindfunclet$?InitInstance@CKiboManagerApp@@UAEHXZ$5 00479f3b f   KiboManager.obj
 0001:00078f47       __ehhandler$?InitInstance@CKiboManagerApp@@UAEHXZ 00479f47 f   KiboManager.obj
 0001:00078f80       __unwindfunclet$?ExitInstance@CKiboManagerApp@@UAEHXZ$0 00479f80 f   KiboManager.obj
 0001:00078f80       __unwindfunclet$?OnBnClickedAdd@CPortCtrlDlg@@QAEXXZ$0 00479f80 f   KiboManager.obj
 0001:00078f80       __unwindfunclet$?OnBnClickedDel@CPortCtrlDlg@@QAEXXZ$0 00479f80 f   KiboManager.obj
 0001:00078f80       __unwindfunclet$?InsertOneClientToBlack@CLenPropertyODBC@@QAE?AV?$CStringT@DV?$StrTraitMFC_DLL@DV?$ChTraitsCRT@D@ATL@@@@@ATL@@UComputerInfo@@@Z$0 00479f80 f   KiboManager.obj
 0001:00078f89       __ehhandler$?ExitInstance@CKiboManagerApp@@UAEHXZ 00479f89 f   KiboManager.obj
 0001:00078f89       __ehhandler$?InsertOneClientToBlack@CLenPropertyODBC@@QAE?AV?$CStringT@DV?$StrTraitMFC_DLL@DV?$ChTraitsCRT@D@ATL@@@@@ATL@@UComputerInfo@@@Z 00479f89 f   KiboManager.obj
 0001:00078f89       __ehhandler$?OnBnClickedAdd@CPortCtrlDlg@@QAEXXZ 00479f89 f   KiboManager.obj
 0001:00078f89       __ehhandler$?OnBnClickedDel@CPortCtrlDlg@@QAEXXZ 00479f89 f   KiboManager.obj
 0001:00078fb0       __unwindfunclet$?OnNewDocument@CKiboManagerDoc@@UAEHXZ$0 00479fb0 f   KiboManagerDoc.obj
 0001:00078fb8       __unwindfunclet$?OnNewDocument@CKiboManagerDoc@@UAEHXZ$3 00479fb8 f   KiboManagerDoc.obj
 0001:00078fc1       __unwindfunclet$?OnNewDocument@CKiboManagerDoc@@UAEHXZ$4 00479fc1 f   KiboManagerDoc.obj
 0001:00078fca       __ehhandler$?OnNewDocument@CKiboManagerDoc@@UAEHXZ 00479fca f   KiboManagerDoc.obj
 0001:00078ff0       __unwindfunclet$?CreateObject@CMyPropertyPage3@@SGPAVCObject@@XZ$0 00479ff0 f   KiboManagerView.obj
 0001:00078ff0       __unwindfunclet$?CreateObject@CKiboManagerView@@SGPAVCObject@@XZ$0 00479ff0 f   KiboManagerView.obj
 0001:00078ff0       __unwindfunclet$?CreateObject@CKiboManagerDoc@@SGPAVCObject@@XZ$0 00479ff0 f   KiboManagerView.obj
 0001:00078ff0       __unwindfunclet$?CreateObject@CPropertyViewUIThread@@SGPAVCObject@@XZ$0 00479ff0 f   KiboManagerView.obj
 0001:00078ff0       __unwindfunclet$?CreateObject@CMyPropertyPage2@@SGPAVCObject@@XZ$0 00479ff0 f   KiboManagerView.obj
 0001:00078ff0       __unwindfunclet$?CreateObject@CMainFrame@@SGPAVCObject@@XZ$0 00479ff0 f   KiboManagerView.obj
 0001:00078ff0       __unwindfunclet$?GetInstance@CMFCVisualManager@@SGPAV1@XZ$0 00479ff0 f   KiboManagerView.obj
 0001:00078ff0       __unwindfunclet$?CreateObject@CMyPropertyPage1@@SGPAVCObject@@XZ$0 00479ff0 f   KiboManagerView.obj
 0001:00078ffa       __ehhandler$?CreateObject@CMyPropertyPage2@@SGPAVCObject@@XZ 00479ffa f   KiboManagerView.obj
 0001:00078ffa       __ehhandler$?CreateObject@CKiboManagerDoc@@SGPAVCObject@@XZ 00479ffa f   KiboManagerView.obj
 0001:00078ffa       __ehhandler$?CreateObject@CPropertyViewUIThread@@SGPAVCObject@@XZ 00479ffa f   KiboManagerView.obj
 0001:00078ffa       __ehhandler$?CreateObject@CMyPropertyPage3@@SGPAVCObject@@XZ 00479ffa f   KiboManagerView.obj
 0001:00078ffa       __ehhandler$?CreateObject@CKiboManagerView@@SGPAVCObject@@XZ 00479ffa f   KiboManagerView.obj
 0001:00078ffa       __ehhandler$?GetInstance@CMFCVisualManager@@SGPAV1@XZ 00479ffa f   KiboManagerView.obj
 0001:00078ffa       __ehhandler$?CreateObject@CMyPropertyPage1@@SGPAVCObject@@XZ 00479ffa f   KiboManagerView.obj
 0001:00078ffa       __ehhandler$?CreateObject@CMainFrame@@SGPAVCObject@@XZ 00479ffa f   KiboManagerView.obj
 0001:00079020       __unwindfunclet$??0CKiboManagerView@@IAE@XZ$0 0047a020 f   KiboManagerView.obj
 0001:00079020       __unwindfunclet$??1CKiboManagerView@@UAE@XZ$0 0047a020 f   KiboManagerView.obj
 0001:00079028       __unwindfunclet$??0CKiboManagerView@@IAE@XZ$1 0047a028 f   KiboManagerView.obj
 0001:00079028       __unwindfunclet$??1CKiboManagerView@@UAE@XZ$1 0047a028 f   KiboManagerView.obj
 0001:00079037       __unwindfunclet$??1CKiboManagerView@@UAE@XZ$2 0047a037 f   KiboManagerView.obj
 0001:00079037       __unwindfunclet$??0CKiboManagerView@@IAE@XZ$2 0047a037 f   KiboManagerView.obj
 0001:00079045       __unwindfunclet$??1CKiboManagerView@@UAE@XZ$3 0047a045 f   KiboManagerView.obj
 0001:00079045       __unwindfunclet$??0CKiboManagerView@@IAE@XZ$3 0047a045 f   KiboManagerView.obj
 0001:00079053       __unwindfunclet$??0CKiboManagerView@@IAE@XZ$4 0047a053 f   KiboManagerView.obj
 0001:00079053       __unwindfunclet$??1CKiboManagerView@@UAE@XZ$4 0047a053 f   KiboManagerView.obj
 0001:00079061       __ehhandler$??0CKiboManagerView@@IAE@XZ 0047a061 f   KiboManagerView.obj
 0001:00079061       __ehhandler$??1CKiboManagerView@@UAE@XZ 0047a061 f   KiboManagerView.obj
 0001:00079080       __unwindfunclet$?OnInitialUpdate@CKiboManagerView@@MAEXXZ$0 0047a080 f   KiboManagerView.obj
 0001:00079088       __unwindfunclet$?OnInitialUpdate@CKiboManagerView@@MAEXXZ$1 0047a088 f   KiboManagerView.obj
 0001:00079091       __unwindfunclet$?OnInitialUpdate@CKiboManagerView@@MAEXXZ$2 0047a091 f   KiboManagerView.obj
 0001:0007909a       __unwindfunclet$?OnInitialUpdate@CKiboManagerView@@MAEXXZ$3 0047a09a f   KiboManagerView.obj
 0001:000790a3       __unwindfunclet$?OnInitialUpdate@CKiboManagerView@@MAEXXZ$4 0047a0a3 f   KiboManagerView.obj
 0001:000790ac       __unwindfunclet$?OnInitialUpdate@CKiboManagerView@@MAEXXZ$5 0047a0ac f   KiboManagerView.obj
 0001:000790b5       __unwindfunclet$?OnInitialUpdate@CKiboManagerView@@MAEXXZ$6 0047a0b5 f   KiboManagerView.obj
 0001:000790be       __unwindfunclet$?OnInitialUpdate@CKiboManagerView@@MAEXXZ$7 0047a0be f   KiboManagerView.obj
 0001:000790c7       __unwindfunclet$?OnInitialUpdate@CKiboManagerView@@MAEXXZ$8 0047a0c7 f   KiboManagerView.obj
 0001:000790d0       __unwindfunclet$?OnInitialUpdate@CKiboManagerView@@MAEXXZ$9 0047a0d0 f   KiboManagerView.obj
 0001:000790d9       __unwindfunclet$?OnInitialUpdate@CKiboManagerView@@MAEXXZ$10 0047a0d9 f   KiboManagerView.obj
 0001:000790e2       __unwindfunclet$?OnInitialUpdate@CKiboManagerView@@MAEXXZ$11 0047a0e2 f   KiboManagerView.obj
 0001:000790eb       __ehhandler$?OnInitialUpdate@CKiboManagerView@@MAEXXZ 0047a0eb f   KiboManagerView.obj
 0001:00079110       __unwindfunclet$?OnContextMenu@CKiboManagerView@@IAEXPAVCWnd@@VCPoint@@@Z$1 0047a110 f   KiboManagerView.obj
 0001:00079119       __unwindfunclet$?OnContextMenu@CKiboManagerView@@IAEXPAVCWnd@@VCPoint@@@Z$2 0047a119 f   KiboManagerView.obj
 0001:00079122       __unwindfunclet$?OnContextMenu@CKiboManagerView@@IAEXPAVCWnd@@VCPoint@@@Z$3 0047a122 f   KiboManagerView.obj
 0001:0007913c       __unwindfunclet$?OnContextMenu@CKiboManagerView@@IAEXPAVCWnd@@VCPoint@@@Z$5 0047a13c f   KiboManagerView.obj
 0001:00079144       __unwindfunclet$?OnContextMenu@CKiboManagerView@@IAEXPAVCWnd@@VCPoint@@@Z$6 0047a144 f   KiboManagerView.obj
 0001:0007914d       __unwindfunclet$?OnContextMenu@CKiboManagerView@@IAEXPAVCWnd@@VCPoint@@@Z$7 0047a14d f   KiboManagerView.obj
 0001:00079156       __unwindfunclet$?OnContextMenu@CKiboManagerView@@IAEXPAVCWnd@@VCPoint@@@Z$8 0047a156 f   KiboManagerView.obj
 0001:00079160       __ehhandler$?OnContextMenu@CKiboManagerView@@IAEXPAVCWnd@@VCPoint@@@Z 0047a160 f   KiboManagerView.obj
 0001:00079180       __unwindfunclet$?CheckSelectionForCmd@CKiboManagerView@@QAEHH@Z$0 0047a180 f   KiboManagerView.obj
 0001:00079189       __unwindfunclet$?CheckSelectionForCmd@CKiboManagerView@@QAEHH@Z$1 0047a189 f   KiboManagerView.obj
 0001:00079192       __unwindfunclet$?CheckSelectionForCmd@CKiboManagerView@@QAEHH@Z$2 0047a192 f   KiboManagerView.obj
 0001:0007919b       __unwindfunclet$?CheckSelectionForCmd@CKiboManagerView@@QAEHH@Z$3 0047a19b f   KiboManagerView.obj
 0001:000791a4       __unwindfunclet$?CheckSelectionForCmd@CKiboManagerView@@QAEHH@Z$4 0047a1a4 f   KiboManagerView.obj
 0001:000791ad       __unwindfunclet$?CheckSelectionForCmd@CKiboManagerView@@QAEHH@Z$5 0047a1ad f   KiboManagerView.obj
 0001:000791b6       __unwindfunclet$?CheckSelectionForCmd@CKiboManagerView@@QAEHH@Z$6 0047a1b6 f   KiboManagerView.obj
 0001:000791bf       __unwindfunclet$?CheckSelectionForCmd@CKiboManagerView@@QAEHH@Z$7 0047a1bf f   KiboManagerView.obj
 0001:000791c8       __ehhandler$?CheckSelectionForCmd@CKiboManagerView@@QAEHH@Z 0047a1c8 f   KiboManagerView.obj
 0001:000791f0       __unwindfunclet$?CheckDriverAndStatus@CKiboManagerView@@QAEHH@Z$0 0047a1f0 f   KiboManagerView.obj
 0001:000791f9       __unwindfunclet$?CheckDriverAndStatus@CKiboManagerView@@QAEHH@Z$1 0047a1f9 f   KiboManagerView.obj
 0001:00079202       __unwindfunclet$?CheckDriverAndStatus@CKiboManagerView@@QAEHH@Z$2 0047a202 f   KiboManagerView.obj
 0001:0007920b       __unwindfunclet$?CheckDriverAndStatus@CKiboManagerView@@QAEHH@Z$3 0047a20b f   KiboManagerView.obj
 0001:00079214       __unwindfunclet$?CheckDriverAndStatus@CKiboManagerView@@QAEHH@Z$4 0047a214 f   KiboManagerView.obj
 0001:0007921d       __unwindfunclet$?CheckDriverAndStatus@CKiboManagerView@@QAEHH@Z$5 0047a21d f   KiboManagerView.obj
 0001:00079226       __unwindfunclet$?CheckDriverAndStatus@CKiboManagerView@@QAEHH@Z$6 0047a226 f   KiboManagerView.obj
 0001:0007922f       __unwindfunclet$?CheckDriverAndStatus@CKiboManagerView@@QAEHH@Z$7 0047a22f f   KiboManagerView.obj
 0001:00079238       __ehhandler$?CheckDriverAndStatus@CKiboManagerView@@QAEHH@Z 0047a238 f   KiboManagerView.obj
 0001:00079260       __unwindfunclet$?CheckAllSelOnline@CKiboManagerView@@QAEHXZ$0 0047a260 f   KiboManagerView.obj
 0001:00079260       __unwindfunclet$?CheckOnlineAndRegistered@CKiboManagerView@@QAEHXZ$0 0047a260 f   KiboManagerView.obj
 0001:00079260       __unwindfunclet$?CheckOnlineAndHasSysForCmd@CKiboManagerView@@QAEHXZ$0 0047a260 f   KiboManagerView.obj
 0001:00079269       __unwindfunclet$?CheckAllSelOnline@CKiboManagerView@@QAEHXZ$1 0047a269 f   KiboManagerView.obj
 0001:00079269       __unwindfunclet$?CheckOnlineAndRegistered@CKiboManagerView@@QAEHXZ$1 0047a269 f   KiboManagerView.obj
 0001:00079269       __unwindfunclet$?CheckOnlineAndHasSysForCmd@CKiboManagerView@@QAEHXZ$1 0047a269 f   KiboManagerView.obj
 0001:00079272       __unwindfunclet$?CheckAllSelOnline@CKiboManagerView@@QAEHXZ$2 0047a272 f   KiboManagerView.obj
 0001:00079272       __unwindfunclet$?CheckOnlineAndHasSysForCmd@CKiboManagerView@@QAEHXZ$2 0047a272 f   KiboManagerView.obj
 0001:00079272       __unwindfunclet$?CheckOnlineAndRegistered@CKiboManagerView@@QAEHXZ$2 0047a272 f   KiboManagerView.obj
 0001:0007927b       __unwindfunclet$?CheckAllSelOnline@CKiboManagerView@@QAEHXZ$3 0047a27b f   KiboManagerView.obj
 0001:0007927b       __unwindfunclet$?CheckOnlineAndRegistered@CKiboManagerView@@QAEHXZ$3 0047a27b f   KiboManagerView.obj
 0001:0007927b       __unwindfunclet$?CheckOnlineAndHasSysForCmd@CKiboManagerView@@QAEHXZ$3 0047a27b f   KiboManagerView.obj
 0001:00079284       __unwindfunclet$?CheckOnlineAndRegistered@CKiboManagerView@@QAEHXZ$4 0047a284 f   KiboManagerView.obj
 0001:00079284       __unwindfunclet$?CheckOnlineAndHasSysForCmd@CKiboManagerView@@QAEHXZ$4 0047a284 f   KiboManagerView.obj
 0001:00079284       __unwindfunclet$?CheckAllSelOnline@CKiboManagerView@@QAEHXZ$4 0047a284 f   KiboManagerView.obj
 0001:0007928d       __unwindfunclet$?CheckOnlineAndHasSysForCmd@CKiboManagerView@@QAEHXZ$5 0047a28d f   KiboManagerView.obj
 0001:0007928d       __unwindfunclet$?CheckOnlineAndRegistered@CKiboManagerView@@QAEHXZ$5 0047a28d f   KiboManagerView.obj
 0001:0007928d       __unwindfunclet$?CheckAllSelOnline@CKiboManagerView@@QAEHXZ$5 0047a28d f   KiboManagerView.obj
 0001:00079296       __ehhandler$?CheckOnlineAndHasSysForCmd@CKiboManagerView@@QAEHXZ 0047a296 f   KiboManagerView.obj
 0001:00079296       __ehhandler$?CheckAllSelOnline@CKiboManagerView@@QAEHXZ 0047a296 f   KiboManagerView.obj
 0001:00079296       __ehhandler$?CheckOnlineAndRegistered@CKiboManagerView@@QAEHXZ 0047a296 f   KiboManagerView.obj
 0001:000792c0       __unwindfunclet$?_SortListItemThread@CKiboManagerView@@SAIPAX@Z$0 0047a2c0 f   KiboManagerView.obj
 0001:000792c9       __unwindfunclet$?_SortListItemThread@CKiboManagerView@@SAIPAX@Z$1 0047a2c9 f   KiboManagerView.obj
 0001:000792d2       __ehhandler$?_SortListItemThread@CKiboManagerView@@SAIPAX@Z 0047a2d2 f   KiboManagerView.obj
 0001:000792f0       __unwindfunclet$?OnLvnItemchangedList1@CKiboManagerView@@QAEXPAUtagNMHDR@@PAJ@Z$1 0047a2f0 f   KiboManagerView.obj
 0001:000792f9       __unwindfunclet$?OnLvnItemchangedList1@CKiboManagerView@@QAEXPAUtagNMHDR@@PAJ@Z$2 0047a2f9 f   KiboManagerView.obj
 0001:00079302       __unwindfunclet$?OnLvnItemchangedList1@CKiboManagerView@@QAEXPAUtagNMHDR@@PAJ@Z$3 0047a302 f   KiboManagerView.obj
 0001:0007930b       __unwindfunclet$?OnLvnItemchangedList1@CKiboManagerView@@QAEXPAUtagNMHDR@@PAJ@Z$4 0047a30b f   KiboManagerView.obj
 0001:00079314       __unwindfunclet$?OnLvnItemchangedList1@CKiboManagerView@@QAEXPAUtagNMHDR@@PAJ@Z$5 0047a314 f   KiboManagerView.obj
 0001:0007931d       __unwindfunclet$?OnLvnItemchangedList1@CKiboManagerView@@QAEXPAUtagNMHDR@@PAJ@Z$6 0047a31d f   KiboManagerView.obj
 0001:00079326       __unwindfunclet$?OnLvnItemchangedList1@CKiboManagerView@@QAEXPAUtagNMHDR@@PAJ@Z$7 0047a326 f   KiboManagerView.obj
 0001:0007932f       __unwindfunclet$?OnLvnItemchangedList1@CKiboManagerView@@QAEXPAUtagNMHDR@@PAJ@Z$8 0047a32f f   KiboManagerView.obj
 0001:00079338       __unwindfunclet$?OnLvnItemchangedList1@CKiboManagerView@@QAEXPAUtagNMHDR@@PAJ@Z$10 0047a338 f   KiboManagerView.obj
 0001:00079341       __unwindfunclet$?OnLvnItemchangedList1@CKiboManagerView@@QAEXPAUtagNMHDR@@PAJ@Z$11 0047a341 f   KiboManagerView.obj
 0001:0007934a       __unwindfunclet$?OnLvnItemchangedList1@CKiboManagerView@@QAEXPAUtagNMHDR@@PAJ@Z$12 0047a34a f   KiboManagerView.obj
 0001:00079353       __unwindfunclet$?OnLvnItemchangedList1@CKiboManagerView@@QAEXPAUtagNMHDR@@PAJ@Z$14 0047a353 f   KiboManagerView.obj
 0001:0007935c       __ehhandler$?OnLvnItemchangedList1@CKiboManagerView@@QAEXPAUtagNMHDR@@PAJ@Z 0047a35c f   KiboManagerView.obj
 0001:00079380       __unwindfunclet$?_DeleteListItemThread@CKiboManagerView@@SAIPAX@Z$0 0047a380 f   KiboManagerView.obj
 0001:00079389       __unwindfunclet$?_DeleteListItemThread@CKiboManagerView@@SAIPAX@Z$1 0047a389 f   KiboManagerView.obj
 0001:00079395       __unwindfunclet$?_DeleteListItemThread@CKiboManagerView@@SAIPAX@Z$5 0047a395 f   KiboManagerView.obj
 0001:0007939e       __unwindfunclet$?_DeleteListItemThread@CKiboManagerView@@SAIPAX@Z$6 0047a39e f   KiboManagerView.obj
 0001:000793aa       __ehhandler$?_DeleteListItemThread@CKiboManagerView@@SAIPAX@Z 0047a3aa f   KiboManagerView.obj
 0001:000793e0       __unwindfunclet$?LoadComputerView@CKiboManagerView@@QAEXXZ$0 0047a3e0 f   KiboManagerView.obj
 0001:000793e9       __unwindfunclet$?LoadComputerView@CKiboManagerView@@QAEXXZ$1 0047a3e9 f   KiboManagerView.obj
 0001:000793f2       __unwindfunclet$?LoadComputerView@CKiboManagerView@@QAEXXZ$2 0047a3f2 f   KiboManagerView.obj
 0001:000793fb       __unwindfunclet$?LoadComputerView@CKiboManagerView@@QAEXXZ$3 0047a3fb f   KiboManagerView.obj
 0001:00079404       __unwindfunclet$?LoadComputerView@CKiboManagerView@@QAEXXZ$4 0047a404 f   KiboManagerView.obj
 0001:0007940d       __unwindfunclet$?LoadComputerView@CKiboManagerView@@QAEXXZ$5 0047a40d f   KiboManagerView.obj
 0001:00079416       __unwindfunclet$?LoadComputerView@CKiboManagerView@@QAEXXZ$6 0047a416 f   KiboManagerView.obj
 0001:0007941f       __unwindfunclet$?LoadComputerView@CKiboManagerView@@QAEXXZ$7 0047a41f f   KiboManagerView.obj
 0001:00079428       __unwindfunclet$?LoadComputerView@CKiboManagerView@@QAEXXZ$8 0047a428 f   KiboManagerView.obj
 0001:00079431       __unwindfunclet$?LoadComputerView@CKiboManagerView@@QAEXXZ$9 0047a431 f   KiboManagerView.obj
 0001:0007943a       __unwindfunclet$?LoadComputerView@CKiboManagerView@@QAEXXZ$10 0047a43a f   KiboManagerView.obj
 0001:00079443       __ehhandler$?LoadComputerView@CKiboManagerView@@QAEXXZ 0047a443 f   KiboManagerView.obj
 0001:00079470       __unwindfunclet$?LoadGroupView@CKiboManagerView@@QAEXXZ$0 0047a470 f   KiboManagerView.obj
 0001:00079479       __ehhandler$?LoadGroupView@CKiboManagerView@@QAEXXZ 0047a479 f   KiboManagerView.obj
 0001:000794a0       __unwindfunclet$?OnSetItemTextList1@CKiboManagerView@@QAEXPAUtagNMHDR@@PAJ@Z$1 0047a4a0 f   KiboManagerView.obj
 0001:000794a9       __unwindfunclet$?OnSetItemTextList1@CKiboManagerView@@QAEXPAUtagNMHDR@@PAJ@Z$2 0047a4a9 f   KiboManagerView.obj
 0001:000794b2       __unwindfunclet$?OnSetItemTextList1@CKiboManagerView@@QAEXPAUtagNMHDR@@PAJ@Z$3 0047a4b2 f   KiboManagerView.obj
 0001:000794bb       __unwindfunclet$?OnSetItemTextList1@CKiboManagerView@@QAEXPAUtagNMHDR@@PAJ@Z$4 0047a4bb f   KiboManagerView.obj
 0001:000794c4       __unwindfunclet$?OnSetItemTextList1@CKiboManagerView@@QAEXPAUtagNMHDR@@PAJ@Z$5 0047a4c4 f   KiboManagerView.obj
 0001:000794cd       __unwindfunclet$?OnSetItemTextList1@CKiboManagerView@@QAEXPAUtagNMHDR@@PAJ@Z$6 0047a4cd f   KiboManagerView.obj
 0001:000794d6       __unwindfunclet$?OnSetItemTextList1@CKiboManagerView@@QAEXPAUtagNMHDR@@PAJ@Z$7 0047a4d6 f   KiboManagerView.obj
 0001:000794df       __unwindfunclet$?OnSetItemTextList1@CKiboManagerView@@QAEXPAUtagNMHDR@@PAJ@Z$8 0047a4df f   KiboManagerView.obj
 0001:000794e8       __ehhandler$?OnSetItemTextList1@CKiboManagerView@@QAEXPAUtagNMHDR@@PAJ@Z 0047a4e8 f   KiboManagerView.obj
 0001:00079510       __unwindfunclet$?OnNMDblclkList1@CKiboManagerView@@QAEXPAUtagNMHDR@@PAJ@Z$1 0047a510 f   KiboManagerView.obj
 0001:00079510       __unwindfunclet$?InsertOneClientToBlack@CClientInfoManager@@QAEHUComputerInfo@@@Z$0 0047a510 f   KiboManagerView.obj
 0001:00079519       __ehhandler$?OnNMDblclkList1@CKiboManagerView@@QAEXPAUtagNMHDR@@PAJ@Z 0047a519 f   KiboManagerView.obj
 0001:00079519       __ehhandler$?InsertOneClientToBlack@CClientInfoManager@@QAEHUComputerInfo@@@Z 0047a519 f   KiboManagerView.obj
 0001:00079540       __unwindfunclet$?OnViewproperty@CKiboManagerView@@QAEXXZ$1 0047a540 f   KiboManagerView.obj
 0001:00079549       __unwindfunclet$?OnViewproperty@CKiboManagerView@@QAEXXZ$2 0047a549 f   KiboManagerView.obj
 0001:00079552       __unwindfunclet$?OnViewproperty@CKiboManagerView@@QAEXXZ$3 0047a552 f   KiboManagerView.obj
 0001:0007955b       __unwindfunclet$?OnViewproperty@CKiboManagerView@@QAEXXZ$4 0047a55b f   KiboManagerView.obj
 0001:00079564       __unwindfunclet$?OnViewproperty@CKiboManagerView@@QAEXXZ$5 0047a564 f   KiboManagerView.obj
 0001:0007956d       __ehhandler$?OnViewproperty@CKiboManagerView@@QAEXXZ 0047a56d f   KiboManagerView.obj
 0001:00079590       __unwindfunclet$?OnMenuDelfromgroup@CKiboManagerView@@QAEXXZ$0 0047a590 f   KiboManagerView.obj
 0001:0007959b       __unwindfunclet$?OnMenuDelfromgroup@CKiboManagerView@@QAEXXZ$1 0047a59b f   KiboManagerView.obj
 0001:000795a7       __unwindfunclet$?OnMenuDelfromgroup@CKiboManagerView@@QAEXXZ$2 0047a5a7 f   KiboManagerView.obj
 0001:000795b3       __unwindfunclet$?OnMenuDelfromgroup@CKiboManagerView@@QAEXXZ$3 0047a5b3 f   KiboManagerView.obj
 0001:000795bf       __unwindfunclet$?OnMenuDelfromgroup@CKiboManagerView@@QAEXXZ$4 0047a5bf f   KiboManagerView.obj
 0001:000795cb       __unwindfunclet$?OnMenuDelfromgroup@CKiboManagerView@@QAEXXZ$5 0047a5cb f   KiboManagerView.obj
 0001:000795d7       __unwindfunclet$?OnMenuDelfromgroup@CKiboManagerView@@QAEXXZ$6 0047a5d7 f   KiboManagerView.obj
 0001:000795e3       __ehhandler$?OnMenuDelfromgroup@CKiboManagerView@@QAEXXZ 0047a5e3 f   KiboManagerView.obj
 0001:00079610       __unwindfunclet$?_DelFromGroupThread@CKiboManagerView@@SAIPAX@Z$0 0047a610 f   KiboManagerView.obj
 0001:00079619       __unwindfunclet$?_DelFromGroupThread@CKiboManagerView@@SAIPAX@Z$1 0047a619 f   KiboManagerView.obj
 0001:00079622       __unwindfunclet$?_DelFromGroupThread@CKiboManagerView@@SAIPAX@Z$3 0047a622 f   KiboManagerView.obj
 0001:0007962b       __unwindfunclet$?_DelFromGroupThread@CKiboManagerView@@SAIPAX@Z$5 0047a62b f   KiboManagerView.obj
 0001:00079637       __unwindfunclet$?_DelFromGroupThread@CKiboManagerView@@SAIPAX@Z$8 0047a637 f   KiboManagerView.obj
 0001:00079640       __unwindfunclet$?_DelFromGroupThread@CKiboManagerView@@SAIPAX@Z$9 0047a640 f   KiboManagerView.obj
 0001:0007964c       __unwindfunclet$?_DelFromGroupThread@CKiboManagerView@@SAIPAX@Z$10 0047a64c f   KiboManagerView.obj
 0001:00079658       __unwindfunclet$?_DelFromGroupThread@CKiboManagerView@@SAIPAX@Z$11 0047a658 f   KiboManagerView.obj
 0001:00079664       __unwindfunclet$?_DelFromGroupThread@CKiboManagerView@@SAIPAX@Z$12 0047a664 f   KiboManagerView.obj
 0001:00079670       __unwindfunclet$?_DelFromGroupThread@CKiboManagerView@@SAIPAX@Z$13 0047a670 f   KiboManagerView.obj
 0001:0007967c       __ehhandler$?_DelFromGroupThread@CKiboManagerView@@SAIPAX@Z 0047a67c f   KiboManagerView.obj
 0001:000796b0       __unwindfunclet$?OnMenuAddtogroup@CKiboManagerView@@QAEXXZ$0 0047a6b0 f   KiboManagerView.obj
 0001:000796bb       __unwindfunclet$?OnMenuAddtogroup@CKiboManagerView@@QAEXXZ$1 0047a6bb f   KiboManagerView.obj
 0001:000796c7       __unwindfunclet$?OnMenuAddtogroup@CKiboManagerView@@QAEXXZ$2 0047a6c7 f   KiboManagerView.obj
 0001:000796d3       __unwindfunclet$?OnMenuAddtogroup@CKiboManagerView@@QAEXXZ$3 0047a6d3 f   KiboManagerView.obj
 0001:000796df       __unwindfunclet$?OnMenuAddtogroup@CKiboManagerView@@QAEXXZ$5 0047a6df f   KiboManagerView.obj
 0001:000796eb       __unwindfunclet$?OnMenuAddtogroup@CKiboManagerView@@QAEXXZ$6 0047a6eb f   KiboManagerView.obj
 0001:000796f7       __unwindfunclet$?OnMenuAddtogroup@CKiboManagerView@@QAEXXZ$7 0047a6f7 f   KiboManagerView.obj
 0001:00079703       __unwindfunclet$?OnMenuAddtogroup@CKiboManagerView@@QAEXXZ$8 0047a703 f   KiboManagerView.obj
 0001:0007970f       __unwindfunclet$?OnMenuAddtogroup@CKiboManagerView@@QAEXXZ$9 0047a70f f   KiboManagerView.obj
 0001:0007971b       __unwindfunclet$?OnMenuAddtogroup@CKiboManagerView@@QAEXXZ$10 0047a71b f   KiboManagerView.obj
 0001:00079727       __unwindfunclet$?OnMenuAddtogroup@CKiboManagerView@@QAEXXZ$11 0047a727 f   KiboManagerView.obj
 0001:00079733       __ehhandler$?OnMenuAddtogroup@CKiboManagerView@@QAEXXZ 0047a733 f   KiboManagerView.obj
 0001:00079760       __unwindfunclet$?_AddClientToGroupThread@CKiboManagerView@@SAIPAX@Z$0 0047a760 f   KiboManagerView.obj
 0001:00079769       __unwindfunclet$?_AddClientToGroupThread@CKiboManagerView@@SAIPAX@Z$1 0047a769 f   KiboManagerView.obj
 0001:00079772       __unwindfunclet$?_AddClientToGroupThread@CKiboManagerView@@SAIPAX@Z$3 0047a772 f   KiboManagerView.obj
 0001:0007977b       __unwindfunclet$?_AddClientToGroupThread@CKiboManagerView@@SAIPAX@Z$4 0047a77b f   KiboManagerView.obj
 0001:00079784       __unwindfunclet$?_AddClientToGroupThread@CKiboManagerView@@SAIPAX@Z$5 0047a784 f   KiboManagerView.obj
 0001:00079790       __unwindfunclet$?_AddClientToGroupThread@CKiboManagerView@@SAIPAX@Z$6 0047a790 f   KiboManagerView.obj
 0001:0007979c       __unwindfunclet$?_AddClientToGroupThread@CKiboManagerView@@SAIPAX@Z$7 0047a79c f   KiboManagerView.obj
 0001:000797a8       __unwindfunclet$?_AddClientToGroupThread@CKiboManagerView@@SAIPAX@Z$8 0047a7a8 f   KiboManagerView.obj
 0001:000797b4       __ehhandler$?_AddClientToGroupThread@CKiboManagerView@@SAIPAX@Z 0047a7b4 f   KiboManagerView.obj
 0001:000797e0       __unwindfunclet$?OnLvnGetInfoTipList1@CKiboManagerView@@QAEXPAUtagNMHDR@@PAJ@Z$0 0047a7e0 f   KiboManagerView.obj
 0001:000797e9       __unwindfunclet$?OnLvnGetInfoTipList1@CKiboManagerView@@QAEXPAUtagNMHDR@@PAJ@Z$1 0047a7e9 f   KiboManagerView.obj
 0001:000797f2       __unwindfunclet$?OnLvnGetInfoTipList1@CKiboManagerView@@QAEXPAUtagNMHDR@@PAJ@Z$2 0047a7f2 f   KiboManagerView.obj
 0001:000797fb       __unwindfunclet$?OnLvnGetInfoTipList1@CKiboManagerView@@QAEXPAUtagNMHDR@@PAJ@Z$3 0047a7fb f   KiboManagerView.obj
 0001:00079804       __unwindfunclet$?OnLvnGetInfoTipList1@CKiboManagerView@@QAEXPAUtagNMHDR@@PAJ@Z$4 0047a804 f   KiboManagerView.obj
 0001:0007980d       __unwindfunclet$?OnLvnGetInfoTipList1@CKiboManagerView@@QAEXPAUtagNMHDR@@PAJ@Z$5 0047a80d f   KiboManagerView.obj
 0001:00079816       __unwindfunclet$?OnLvnGetInfoTipList1@CKiboManagerView@@QAEXPAUtagNMHDR@@PAJ@Z$6 0047a816 f   KiboManagerView.obj
 0001:0007981f       __unwindfunclet$?OnLvnGetInfoTipList1@CKiboManagerView@@QAEXPAUtagNMHDR@@PAJ@Z$7 0047a81f f   KiboManagerView.obj
 0001:00079828       __unwindfunclet$?OnLvnGetInfoTipList1@CKiboManagerView@@QAEXPAUtagNMHDR@@PAJ@Z$8 0047a828 f   KiboManagerView.obj
 0001:00079831       __unwindfunclet$?OnLvnGetInfoTipList1@CKiboManagerView@@QAEXPAUtagNMHDR@@PAJ@Z$10 0047a831 f   KiboManagerView.obj
 0001:0007983a       __unwindfunclet$?OnLvnGetInfoTipList1@CKiboManagerView@@QAEXPAUtagNMHDR@@PAJ@Z$11 0047a83a f   KiboManagerView.obj
 0001:00079843       __ehhandler$?OnLvnGetInfoTipList1@CKiboManagerView@@QAEXPAUtagNMHDR@@PAJ@Z 0047a843 f   KiboManagerView.obj
 0001:00079870       __unwindfunclet$?CheckMode@CKiboManagerView@@QAEHH@Z$0 0047a870 f   KiboManagerView.obj
 0001:00079879       __unwindfunclet$?CheckMode@CKiboManagerView@@QAEHH@Z$1 0047a879 f   KiboManagerView.obj
 0001:00079882       __unwindfunclet$?CheckMode@CKiboManagerView@@QAEHH@Z$2 0047a882 f   KiboManagerView.obj
 0001:0007988b       __unwindfunclet$?CheckMode@CKiboManagerView@@QAEHH@Z$3 0047a88b f   KiboManagerView.obj
 0001:00079894       __unwindfunclet$?CheckMode@CKiboManagerView@@QAEHH@Z$4 0047a894 f   KiboManagerView.obj
 0001:0007989d       __unwindfunclet$?CheckMode@CKiboManagerView@@QAEHH@Z$5 0047a89d f   KiboManagerView.obj
 0001:000798a6       __unwindfunclet$?CheckMode@CKiboManagerView@@QAEHH@Z$6 0047a8a6 f   KiboManagerView.obj
 0001:000798af       __unwindfunclet$?CheckMode@CKiboManagerView@@QAEHH@Z$7 0047a8af f   KiboManagerView.obj
 0001:000798b8       __unwindfunclet$?CheckMode@CKiboManagerView@@QAEHH@Z$8 0047a8b8 f   KiboManagerView.obj
 0001:000798c1       __unwindfunclet$?CheckMode@CKiboManagerView@@QAEHH@Z$9 0047a8c1 f   KiboManagerView.obj
 0001:000798ca       __unwindfunclet$?CheckMode@CKiboManagerView@@QAEHH@Z$10 0047a8ca f   KiboManagerView.obj
 0001:000798d3       __unwindfunclet$?CheckMode@CKiboManagerView@@QAEHH@Z$11 0047a8d3 f   KiboManagerView.obj
 0001:000798dc       __unwindfunclet$?CheckMode@CKiboManagerView@@QAEHH@Z$12 0047a8dc f   KiboManagerView.obj
 0001:000798e5       __unwindfunclet$?CheckMode@CKiboManagerView@@QAEHH@Z$13 0047a8e5 f   KiboManagerView.obj
 0001:000798ee       __unwindfunclet$?CheckMode@CKiboManagerView@@QAEHH@Z$14 0047a8ee f   KiboManagerView.obj
 0001:000798f7       __unwindfunclet$?CheckMode@CKiboManagerView@@QAEHH@Z$15 0047a8f7 f   KiboManagerView.obj
 0001:00079900       __unwindfunclet$?CheckMode@CKiboManagerView@@QAEHH@Z$16 0047a900 f   KiboManagerView.obj
 0001:00079909       __unwindfunclet$?CheckMode@CKiboManagerView@@QAEHH@Z$17 0047a909 f   KiboManagerView.obj
 0001:00079915       __unwindfunclet$?CheckMode@CKiboManagerView@@QAEHH@Z$18 0047a915 f   KiboManagerView.obj
 0001:00079921       __unwindfunclet$?CheckMode@CKiboManagerView@@QAEHH@Z$19 0047a921 f   KiboManagerView.obj
 0001:0007992d       __unwindfunclet$?CheckMode@CKiboManagerView@@QAEHH@Z$20 0047a92d f   KiboManagerView.obj
 0001:00079939       __unwindfunclet$?CheckMode@CKiboManagerView@@QAEHH@Z$21 0047a939 f   KiboManagerView.obj
 0001:00079945       __ehhandler$?CheckMode@CKiboManagerView@@QAEHH@Z 0047a945 f   KiboManagerView.obj
 0001:00079970       __unwindfunclet$?CheckSelectionNum@CKiboManagerView@@QAEHHH@Z$0 0047a970 f   KiboManagerView.obj
 0001:00079979       __unwindfunclet$?CheckSelectionNum@CKiboManagerView@@QAEHHH@Z$1 0047a979 f   KiboManagerView.obj
 0001:00079982       __unwindfunclet$?CheckSelectionNum@CKiboManagerView@@QAEHHH@Z$2 0047a982 f   KiboManagerView.obj
 0001:0007998b       __unwindfunclet$?CheckSelectionNum@CKiboManagerView@@QAEHHH@Z$3 0047a98b f   KiboManagerView.obj
 0001:00079994       __unwindfunclet$?CheckSelectionNum@CKiboManagerView@@QAEHHH@Z$4 0047a994 f   KiboManagerView.obj
 0001:0007999d       __unwindfunclet$?CheckSelectionNum@CKiboManagerView@@QAEHHH@Z$5 0047a99d f   KiboManagerView.obj
 0001:000799a6       __unwindfunclet$?CheckSelectionNum@CKiboManagerView@@QAEHHH@Z$6 0047a9a6 f   KiboManagerView.obj
 0001:000799af       __unwindfunclet$?CheckSelectionNum@CKiboManagerView@@QAEHHH@Z$7 0047a9af f   KiboManagerView.obj
 0001:000799b8       __ehhandler$?CheckSelectionNum@CKiboManagerView@@QAEHHH@Z 0047a9b8 f   KiboManagerView.obj
 0001:000799e0       __unwindfunclet$?OnNMRClickList1@CKiboManagerView@@QAEXPAUtagNMHDR@@PAJ@Z$0 0047a9e0 f   KiboManagerView.obj
 0001:000799e9       __ehhandler$?OnNMRClickList1@CKiboManagerView@@QAEXPAUtagNMHDR@@PAJ@Z 0047a9e9 f   KiboManagerView.obj
 0001:00079a10       __unwindfunclet$??0logic_error@std@@QAE@ABV01@@Z$0 0047aa10 f   KiboManagerView.obj
 0001:00079a10       __unwindfunclet$??0logic_error@std@@QAE@ABV?$basic_string@DU?$char_traits@D@std@@V?$allocator@D@2@@1@@Z$0 0047aa10 f   KiboManagerView.obj
 0001:00079a19       __ehhandler$??0logic_error@std@@QAE@ABV?$basic_string@DU?$char_traits@D@std@@V?$allocator@D@2@@1@@Z 0047aa19 f   KiboManagerView.obj
 0001:00079a19       __ehhandler$??0logic_error@std@@QAE@ABV01@@Z 0047aa19 f   KiboManagerView.obj
 0001:00079a40       __unwindfunclet$?UpdateOneComputerInfo@CLenPropertyODBC@@QAE?AV?$CStringT@DV?$StrTraitMFC_DLL@DV?$ChTraitsCRT@D@ATL@@@@@ATL@@PAUComputerInfo@@@Z$0 0047aa40 f   LenPropertyODBC.obj
 0001:00079a40       __unwindfunclet$?GetAllGroup@CLenPropertyODBC@@QAE?AV?$CStringT@DV?$StrTraitMFC_DLL@DV?$ChTraitsCRT@D@ATL@@@@@ATL@@XZ$0 0047aa40 f   LenPropertyODBC.obj
 0001:00079a40       __unwindfunclet$?GetAllBlackComputer@CLenPropertyODBC@@QAE?AV?$CStringT@DV?$StrTraitMFC_DLL@DV?$ChTraitsCRT@D@ATL@@@@@ATL@@XZ$0 0047aa40 f   LenPropertyODBC.obj
 0001:00079a40       __unwindfunclet$?InsertOneComputerInfo@CLenPropertyODBC@@QAE?AV?$CStringT@DV?$StrTraitMFC_DLL@DV?$ChTraitsCRT@D@ATL@@@@@ATL@@PAUComputerInfo@@@Z$0 0047aa40 f   LenPropertyODBC.obj
 0001:00079a40       __unwindfunclet$?DeleteOneComputerInfo@CLenPropertyODBC@@QAE?AV?$CStringT@DV?$StrTraitMFC_DLL@DV?$ChTraitsCRT@D@ATL@@@@@ATL@@PBD@Z$0 0047aa40 f   LenPropertyODBC.obj
 0001:00079a40       __unwindfunclet$?GetAllComputerInfo@CLenPropertyODBC@@QAE?AV?$CStringT@DV?$StrTraitMFC_DLL@DV?$ChTraitsCRT@D@ATL@@@@@ATL@@XZ$0 0047aa40 f   LenPropertyODBC.obj
 0001:00079a40       __unwindfunclet$?PreLoadState@CKiboManagerApp@@UAEXXZ$0 0047aa40 f   LenPropertyODBC.obj
 0001:00079a49       __ehhandler$?InsertOneComputerInfo@CLenPropertyODBC@@QAE?AV?$CStringT@DV?$StrTraitMFC_DLL@DV?$ChTraitsCRT@D@ATL@@@@@ATL@@PAUComputerInfo@@@Z 0047aa49 f   LenPropertyODBC.obj
 0001:00079a49       __ehhandler$?UpdateOneComputerInfo@CLenPropertyODBC@@QAE?AV?$CStringT@DV?$StrTraitMFC_DLL@DV?$ChTraitsCRT@D@ATL@@@@@ATL@@PAUComputerInfo@@@Z 0047aa49 f   LenPropertyODBC.obj
 0001:00079a49       __ehhandler$?GetAllGroup@CLenPropertyODBC@@QAE?AV?$CStringT@DV?$StrTraitMFC_DLL@DV?$ChTraitsCRT@D@ATL@@@@@ATL@@XZ 0047aa49 f   LenPropertyODBC.obj
 0001:00079a49       __ehhandler$?GetAllComputerInfo@CLenPropertyODBC@@QAE?AV?$CStringT@DV?$StrTraitMFC_DLL@DV?$ChTraitsCRT@D@ATL@@@@@ATL@@XZ 0047aa49 f   LenPropertyODBC.obj
 0001:00079a49       __ehhandler$?PreLoadState@CKiboManagerApp@@UAEXXZ 0047aa49 f   LenPropertyODBC.obj
 0001:00079a49       __ehhandler$?DeleteOneComputerInfo@CLenPropertyODBC@@QAE?AV?$CStringT@DV?$StrTraitMFC_DLL@DV?$ChTraitsCRT@D@ATL@@@@@ATL@@PBD@Z 0047aa49 f   LenPropertyODBC.obj
 0001:00079a49       __ehhandler$?GetAllBlackComputer@CLenPropertyODBC@@QAE?AV?$CStringT@DV?$StrTraitMFC_DLL@DV?$ChTraitsCRT@D@ATL@@@@@ATL@@XZ 0047aa49 f   LenPropertyODBC.obj
 0001:00079a70       __unwindfunclet$?DeleteSoftwareInfo@CLenPropertyODBC@@QAE?AV?$CStringT@DV?$StrTraitMFC_DLL@DV?$ChTraitsCRT@D@ATL@@@@@ATL@@PBDIH@Z$0 0047aa70 f   LenPropertyODBC.obj
 0001:00079a70       __unwindfunclet$?InsertOnePropertyMainInfo@CLenPropertyODBC@@QAE?AV?$CStringT@DV?$StrTraitMFC_DLL@DV?$ChTraitsCRT@D@ATL@@@@@ATL@@PAUPropertyInfo@@H@Z$0 0047aa70 f   LenPropertyODBC.obj
 0001:00079a70       __unwindfunclet$?UpdateOnePropertyMainInfo@CLenPropertyODBC@@QAE?AV?$CStringT@DV?$StrTraitMFC_DLL@DV?$ChTraitsCRT@D@ATL@@@@@ATL@@PAUPropertyInfo@@H@Z$0 0047aa70 f   LenPropertyODBC.obj
 0001:00079a70       __unwindfunclet$?DeleteSoftwareInfo@CLenPropertyODBC@@QAE?AV?$CStringT@DV?$StrTraitMFC_DLL@DV?$ChTraitsCRT@D@ATL@@@@@ATL@@PBDH@Z$0 0047aa70 f   LenPropertyODBC.obj
 0001:00079a70       __unwindfunclet$?SortSoftwareInfo@CLenPropertyODBC@@QAE?AV?$CStringT@DV?$StrTraitMFC_DLL@DV?$ChTraitsCRT@D@ATL@@@@@ATL@@H@Z$0 0047aa70 f   LenPropertyODBC.obj
 0001:00079a70       __unwindfunclet$?InsertOneSoftwareInfo@CLenPropertyODBC@@QAE?AV?$CStringT@DV?$StrTraitMFC_DLL@DV?$ChTraitsCRT@D@ATL@@@@@ATL@@PBDI0H@Z$0 0047aa70 f   LenPropertyODBC.obj
 0001:00079a70       __unwindfunclet$?DeleteOnePropertyMainInfo@CLenPropertyODBC@@QAE?AV?$CStringT@DV?$StrTraitMFC_DLL@DV?$ChTraitsCRT@D@ATL@@@@@ATL@@PBDH@Z$0 0047aa70 f   LenPropertyODBC.obj
 0001:00079a79       __unwindfunclet$?InsertOnePropertyMainInfo@CLenPropertyODBC@@QAE?AV?$CStringT@DV?$StrTraitMFC_DLL@DV?$ChTraitsCRT@D@ATL@@@@@ATL@@PAUPropertyInfo@@H@Z$1 0047aa79 f   LenPropertyODBC.obj
 0001:00079a79       __unwindfunclet$?DeleteSoftwareInfo@CLenPropertyODBC@@QAE?AV?$CStringT@DV?$StrTraitMFC_DLL@DV?$ChTraitsCRT@D@ATL@@@@@ATL@@PBDH@Z$1 0047aa79 f   LenPropertyODBC.obj
 0001:00079a79       __unwindfunclet$?SortSoftwareInfo@CLenPropertyODBC@@QAE?AV?$CStringT@DV?$StrTraitMFC_DLL@DV?$ChTraitsCRT@D@ATL@@@@@ATL@@H@Z$1 0047aa79 f   LenPropertyODBC.obj
 0001:00079a79       __unwindfunclet$?InsertOneSoftwareInfo@CLenPropertyODBC@@QAE?AV?$CStringT@DV?$StrTraitMFC_DLL@DV?$ChTraitsCRT@D@ATL@@@@@ATL@@PBDI0H@Z$1 0047aa79 f   LenPropertyODBC.obj
 0001:00079a79       __unwindfunclet$?UpdateOnePropertyMainInfo@CLenPropertyODBC@@QAE?AV?$CStringT@DV?$StrTraitMFC_DLL@DV?$ChTraitsCRT@D@ATL@@@@@ATL@@PAUPropertyInfo@@H@Z$1 0047aa79 f   LenPropertyODBC.obj
 0001:00079a79       __unwindfunclet$?DeleteOnePropertyMainInfo@CLenPropertyODBC@@QAE?AV?$CStringT@DV?$StrTraitMFC_DLL@DV?$ChTraitsCRT@D@ATL@@@@@ATL@@PBDH@Z$1 0047aa79 f   LenPropertyODBC.obj
 0001:00079a79       __unwindfunclet$?DeleteSoftwareInfo@CLenPropertyODBC@@QAE?AV?$CStringT@DV?$StrTraitMFC_DLL@DV?$ChTraitsCRT@D@ATL@@@@@ATL@@PBDIH@Z$1 0047aa79 f   LenPropertyODBC.obj
 0001:00079a82       __ehhandler$?InsertOnePropertyMainInfo@CLenPropertyODBC@@QAE?AV?$CStringT@DV?$StrTraitMFC_DLL@DV?$ChTraitsCRT@D@ATL@@@@@ATL@@PAUPropertyInfo@@H@Z 0047aa82 f   LenPropertyODBC.obj
 0001:00079a82       __ehhandler$?InsertOneSoftwareInfo@CLenPropertyODBC@@QAE?AV?$CStringT@DV?$StrTraitMFC_DLL@DV?$ChTraitsCRT@D@ATL@@@@@ATL@@PBDI0H@Z 0047aa82 f   LenPropertyODBC.obj
 0001:00079a82       __ehhandler$?SortSoftwareInfo@CLenPropertyODBC@@QAE?AV?$CStringT@DV?$StrTraitMFC_DLL@DV?$ChTraitsCRT@D@ATL@@@@@ATL@@H@Z 0047aa82 f   LenPropertyODBC.obj
 0001:00079a82       __ehhandler$?DeleteSoftwareInfo@CLenPropertyODBC@@QAE?AV?$CStringT@DV?$StrTraitMFC_DLL@DV?$ChTraitsCRT@D@ATL@@@@@ATL@@PBDH@Z 0047aa82 f   LenPropertyODBC.obj
 0001:00079a82       __ehhandler$?DeleteOnePropertyMainInfo@CLenPropertyODBC@@QAE?AV?$CStringT@DV?$StrTraitMFC_DLL@DV?$ChTraitsCRT@D@ATL@@@@@ATL@@PBDH@Z 0047aa82 f   LenPropertyODBC.obj
 0001:00079a82       __ehhandler$?UpdateOnePropertyMainInfo@CLenPropertyODBC@@QAE?AV?$CStringT@DV?$StrTraitMFC_DLL@DV?$ChTraitsCRT@D@ATL@@@@@ATL@@PAUPropertyInfo@@H@Z 0047aa82 f   LenPropertyODBC.obj
 0001:00079a82       __ehhandler$?DeleteSoftwareInfo@CLenPropertyODBC@@QAE?AV?$CStringT@DV?$StrTraitMFC_DLL@DV?$ChTraitsCRT@D@ATL@@@@@ATL@@PBDIH@Z 0047aa82 f   LenPropertyODBC.obj
 0001:00079aa0       __unwindfunclet$?GetOnePropertyInfo@CLenPropertyODBC@@QAEHPBDIHPAUPropertyInfo@@@Z$0 0047aaa0 f   LenPropertyODBC.obj
 0001:00079aa9       __unwindfunclet$?GetOnePropertyInfo@CLenPropertyODBC@@QAEHPBDIHPAUPropertyInfo@@@Z$1 0047aaa9 f   LenPropertyODBC.obj
 0001:00079ab1       __unwindfunclet$?GetOnePropertyInfo@CLenPropertyODBC@@QAEHPBDIHPAUPropertyInfo@@@Z$2 0047aab1 f   LenPropertyODBC.obj
 0001:00079aba       __unwindfunclet$?GetOnePropertyInfo@CLenPropertyODBC@@QAEHPBDIHPAUPropertyInfo@@@Z$3 0047aaba f   LenPropertyODBC.obj
 0001:00079ac3       __ehhandler$?GetOnePropertyInfo@CLenPropertyODBC@@QAEHPBDIHPAUPropertyInfo@@@Z 0047aac3 f   LenPropertyODBC.obj
 0001:00079ae0       __unwindfunclet$?IfCurrentPropertyInfoChanged@CLenPropertyODBC@@QAEHPAUPropertyInfo@@AAV?$CStringT@DV?$StrTraitMFC_DLL@DV?$ChTraitsCRT@D@ATL@@@@@ATL@@@Z$0 0047aae0 f   LenPropertyODBC.obj
 0001:00079aeb       __unwindfunclet$?IfCurrentPropertyInfoChanged@CLenPropertyODBC@@QAEHPAUPropertyInfo@@AAV?$CStringT@DV?$StrTraitMFC_DLL@DV?$ChTraitsCRT@D@ATL@@@@@ATL@@@Z$1 0047aaeb f   LenPropertyODBC.obj
 0001:00079af7       __unwindfunclet$?IfCurrentPropertyInfoChanged@CLenPropertyODBC@@QAEHPAUPropertyInfo@@AAV?$CStringT@DV?$StrTraitMFC_DLL@DV?$ChTraitsCRT@D@ATL@@@@@ATL@@@Z$2 0047aaf7 f   LenPropertyODBC.obj
 0001:00079b03       __unwindfunclet$?IfCurrentPropertyInfoChanged@CLenPropertyODBC@@QAEHPAUPropertyInfo@@AAV?$CStringT@DV?$StrTraitMFC_DLL@DV?$ChTraitsCRT@D@ATL@@@@@ATL@@@Z$3 0047ab03 f   LenPropertyODBC.obj
 0001:00079b0f       __unwindfunclet$?IfCurrentPropertyInfoChanged@CLenPropertyODBC@@QAEHPAUPropertyInfo@@AAV?$CStringT@DV?$StrTraitMFC_DLL@DV?$ChTraitsCRT@D@ATL@@@@@ATL@@@Z$4 0047ab0f f   LenPropertyODBC.obj
 0001:00079b1b       __unwindfunclet$?IfCurrentPropertyInfoChanged@CLenPropertyODBC@@QAEHPAUPropertyInfo@@AAV?$CStringT@DV?$StrTraitMFC_DLL@DV?$ChTraitsCRT@D@ATL@@@@@ATL@@@Z$5 0047ab1b f   LenPropertyODBC.obj
 0001:00079b27       __unwindfunclet$?IfCurrentPropertyInfoChanged@CLenPropertyODBC@@QAEHPAUPropertyInfo@@AAV?$CStringT@DV?$StrTraitMFC_DLL@DV?$ChTraitsCRT@D@ATL@@@@@ATL@@@Z$6 0047ab27 f   LenPropertyODBC.obj
 0001:00079b33       __unwindfunclet$?IfCurrentPropertyInfoChanged@CLenPropertyODBC@@QAEHPAUPropertyInfo@@AAV?$CStringT@DV?$StrTraitMFC_DLL@DV?$ChTraitsCRT@D@ATL@@@@@ATL@@@Z$7 0047ab33 f   LenPropertyODBC.obj
 0001:00079b3e       __unwindfunclet$?IfCurrentPropertyInfoChanged@CLenPropertyODBC@@QAEHPAUPropertyInfo@@AAV?$CStringT@DV?$StrTraitMFC_DLL@DV?$ChTraitsCRT@D@ATL@@@@@ATL@@@Z$8 0047ab3e f   LenPropertyODBC.obj
 0001:00079b4a       __unwindfunclet$?IfCurrentPropertyInfoChanged@CLenPropertyODBC@@QAEHPAUPropertyInfo@@AAV?$CStringT@DV?$StrTraitMFC_DLL@DV?$ChTraitsCRT@D@ATL@@@@@ATL@@@Z$9 0047ab4a f   LenPropertyODBC.obj
 0001:00079b56       __unwindfunclet$?IfCurrentPropertyInfoChanged@CLenPropertyODBC@@QAEHPAUPropertyInfo@@AAV?$CStringT@DV?$StrTraitMFC_DLL@DV?$ChTraitsCRT@D@ATL@@@@@ATL@@@Z$10 0047ab56 f   LenPropertyODBC.obj
 0001:00079b62       __unwindfunclet$?IfCurrentPropertyInfoChanged@CLenPropertyODBC@@QAEHPAUPropertyInfo@@AAV?$CStringT@DV?$StrTraitMFC_DLL@DV?$ChTraitsCRT@D@ATL@@@@@ATL@@@Z$11 0047ab62 f   LenPropertyODBC.obj
 0001:00079b6e       __ehhandler$?IfCurrentPropertyInfoChanged@CLenPropertyODBC@@QAEHPAUPropertyInfo@@AAV?$CStringT@DV?$StrTraitMFC_DLL@DV?$ChTraitsCRT@D@ATL@@@@@ATL@@@Z 0047ab6e f   LenPropertyODBC.obj
 0001:00079ba0       __unwindfunclet$?CompareAndGetAbstract@CLenPropertyODBC@@QAEHPAUPropertyInfo@@0AAV?$CStringT@DV?$StrTraitMFC_DLL@DV?$ChTraitsCRT@D@ATL@@@@@ATL@@@Z$0 0047aba0 f   LenPropertyODBC.obj
 0001:00079ba9       __unwindfunclet$?CompareAndGetAbstract@CLenPropertyODBC@@QAEHPAUPropertyInfo@@0AAV?$CStringT@DV?$StrTraitMFC_DLL@DV?$ChTraitsCRT@D@ATL@@@@@ATL@@@Z$1 0047aba9 f   LenPropertyODBC.obj
 0001:00079bb2       __unwindfunclet$?CompareAndGetAbstract@CLenPropertyODBC@@QAEHPAUPropertyInfo@@0AAV?$CStringT@DV?$StrTraitMFC_DLL@DV?$ChTraitsCRT@D@ATL@@@@@ATL@@@Z$2 0047abb2 f   LenPropertyODBC.obj
 0001:00079bbb       __unwindfunclet$?CompareAndGetAbstract@CLenPropertyODBC@@QAEHPAUPropertyInfo@@0AAV?$CStringT@DV?$StrTraitMFC_DLL@DV?$ChTraitsCRT@D@ATL@@@@@ATL@@@Z$3 0047abbb f   LenPropertyODBC.obj
 0001:00079bc3       __unwindfunclet$?CompareAndGetAbstract@CLenPropertyODBC@@QAEHPAUPropertyInfo@@0AAV?$CStringT@DV?$StrTraitMFC_DLL@DV?$ChTraitsCRT@D@ATL@@@@@ATL@@@Z$4 0047abc3 f   LenPropertyODBC.obj
 0001:00079bcc       __unwindfunclet$?CompareAndGetAbstract@CLenPropertyODBC@@QAEHPAUPropertyInfo@@0AAV?$CStringT@DV?$StrTraitMFC_DLL@DV?$ChTraitsCRT@D@ATL@@@@@ATL@@@Z$5 0047abcc f   LenPropertyODBC.obj
 0001:00079bd5       __unwindfunclet$?CompareAndGetAbstract@CLenPropertyODBC@@QAEHPAUPropertyInfo@@0AAV?$CStringT@DV?$StrTraitMFC_DLL@DV?$ChTraitsCRT@D@ATL@@@@@ATL@@@Z$6 0047abd5 f   LenPropertyODBC.obj
 0001:00079bde       __unwindfunclet$?CompareAndGetAbstract@CLenPropertyODBC@@QAEHPAUPropertyInfo@@0AAV?$CStringT@DV?$StrTraitMFC_DLL@DV?$ChTraitsCRT@D@ATL@@@@@ATL@@@Z$7 0047abde f   LenPropertyODBC.obj
 0001:00079be7       __unwindfunclet$?CompareAndGetAbstract@CLenPropertyODBC@@QAEHPAUPropertyInfo@@0AAV?$CStringT@DV?$StrTraitMFC_DLL@DV?$ChTraitsCRT@D@ATL@@@@@ATL@@@Z$8 0047abe7 f   LenPropertyODBC.obj
 0001:00079bf0       __unwindfunclet$?CompareAndGetAbstract@CLenPropertyODBC@@QAEHPAUPropertyInfo@@0AAV?$CStringT@DV?$StrTraitMFC_DLL@DV?$ChTraitsCRT@D@ATL@@@@@ATL@@@Z$9 0047abf0 f   LenPropertyODBC.obj
 0001:00079bf9       __ehhandler$?CompareAndGetAbstract@CLenPropertyODBC@@QAEHPAUPropertyInfo@@0AAV?$CStringT@DV?$StrTraitMFC_DLL@DV?$ChTraitsCRT@D@ATL@@@@@ATL@@@Z 0047abf9 f   LenPropertyODBC.obj
 0001:00079c20       __unwindfunclet$?RemoveOneFromBlack@CLenPropertyODBC@@QAE?AV?$CStringT@DV?$StrTraitMFC_DLL@DV?$ChTraitsCRT@D@ATL@@@@@ATL@@V23@@Z$0 0047ac20 f   LenPropertyODBC.obj
 0001:00079c20       __unwindfunclet$?RemoveOneGroupCLient@CLenPropertyODBC@@QAE?AV?$CStringT@DV?$StrTraitMFC_DLL@DV?$ChTraitsCRT@D@ATL@@@@@ATL@@V23@@Z$0 0047ac20 f   LenPropertyODBC.obj
 0001:00079c29       __unwindfunclet$?RemoveOneFromBlack@CLenPropertyODBC@@QAE?AV?$CStringT@DV?$StrTraitMFC_DLL@DV?$ChTraitsCRT@D@ATL@@@@@ATL@@V23@@Z$1 0047ac29 f   LenPropertyODBC.obj
 0001:00079c29       __unwindfunclet$?RemoveOneGroupCLient@CLenPropertyODBC@@QAE?AV?$CStringT@DV?$StrTraitMFC_DLL@DV?$ChTraitsCRT@D@ATL@@@@@ATL@@V23@@Z$1 0047ac29 f   LenPropertyODBC.obj
 0001:00079c32       __ehhandler$?RemoveOneGroupCLient@CLenPropertyODBC@@QAE?AV?$CStringT@DV?$StrTraitMFC_DLL@DV?$ChTraitsCRT@D@ATL@@@@@ATL@@V23@@Z 0047ac32 f   LenPropertyODBC.obj
 0001:00079c32       __ehhandler$?RemoveOneFromBlack@CLenPropertyODBC@@QAE?AV?$CStringT@DV?$StrTraitMFC_DLL@DV?$ChTraitsCRT@D@ATL@@@@@ATL@@V23@@Z 0047ac32 f   LenPropertyODBC.obj
 0001:00079c50       __unwindfunclet$?UpdateGroupName@CLenPropertyODBC@@QAE?AV?$CStringT@DV?$StrTraitMFC_DLL@DV?$ChTraitsCRT@D@ATL@@@@@ATL@@V23@0@Z$0 0047ac50 f   LenPropertyODBC.obj
 0001:00079c59       __unwindfunclet$?UpdateGroupName@CLenPropertyODBC@@QAE?AV?$CStringT@DV?$StrTraitMFC_DLL@DV?$ChTraitsCRT@D@ATL@@@@@ATL@@V23@0@Z$1 0047ac59 f   LenPropertyODBC.obj
 0001:00079c62       __unwindfunclet$?UpdateGroupName@CLenPropertyODBC@@QAE?AV?$CStringT@DV?$StrTraitMFC_DLL@DV?$ChTraitsCRT@D@ATL@@@@@ATL@@V23@0@Z$3 0047ac62 f   LenPropertyODBC.obj
 0001:00079c6b       __unwindfunclet$?UpdateGroupName@CLenPropertyODBC@@QAE?AV?$CStringT@DV?$StrTraitMFC_DLL@DV?$ChTraitsCRT@D@ATL@@@@@ATL@@V23@0@Z$5 0047ac6b f   LenPropertyODBC.obj
 0001:00079c74       __unwindfunclet$?UpdateGroupName@CLenPropertyODBC@@QAE?AV?$CStringT@DV?$StrTraitMFC_DLL@DV?$ChTraitsCRT@D@ATL@@@@@ATL@@V23@0@Z$6 0047ac74 f   LenPropertyODBC.obj
 0001:00079c7d       __ehhandler$?UpdateGroupName@CLenPropertyODBC@@QAE?AV?$CStringT@DV?$StrTraitMFC_DLL@DV?$ChTraitsCRT@D@ATL@@@@@ATL@@V23@0@Z 0047ac7d f   LenPropertyODBC.obj
 0001:00079ca0       __unwindfunclet$?UpdateGroupInfoByOldGroupName@CLenPropertyODBC@@QAE?AV?$CStringT@DV?$StrTraitMFC_DLL@DV?$ChTraitsCRT@D@ATL@@@@@ATL@@V23@UtagGroupClient@@@Z$0 0047aca0 f   LenPropertyODBC.obj
 0001:00079ca9       __unwindfunclet$?UpdateGroupInfoByOldGroupName@CLenPropertyODBC@@QAE?AV?$CStringT@DV?$StrTraitMFC_DLL@DV?$ChTraitsCRT@D@ATL@@@@@ATL@@V23@UtagGroupClient@@@Z$2 0047aca9 f   LenPropertyODBC.obj
 0001:00079cb2       __unwindfunclet$?UpdateGroupInfoByOldGroupName@CLenPropertyODBC@@QAE?AV?$CStringT@DV?$StrTraitMFC_DLL@DV?$ChTraitsCRT@D@ATL@@@@@ATL@@V23@UtagGroupClient@@@Z$4 0047acb2 f   LenPropertyODBC.obj
 0001:00079cbb       __unwindfunclet$?UpdateGroupInfoByOldGroupName@CLenPropertyODBC@@QAE?AV?$CStringT@DV?$StrTraitMFC_DLL@DV?$ChTraitsCRT@D@ATL@@@@@ATL@@V23@UtagGroupClient@@@Z$5 0047acbb f   LenPropertyODBC.obj
 0001:00079cc4       __ehhandler$?UpdateGroupInfoByOldGroupName@CLenPropertyODBC@@QAE?AV?$CStringT@DV?$StrTraitMFC_DLL@DV?$ChTraitsCRT@D@ATL@@@@@ATL@@V23@UtagGroupClient@@@Z 0047acc4 f   LenPropertyODBC.obj
 0001:00079ce0       __unwindfunclet$?GetAllGroupClient@CLenPropertyODBC@@QAE?AV?$CStringT@DV?$StrTraitMFC_DLL@DV?$ChTraitsCRT@D@ATL@@@@@ATL@@V23@@Z$0 0047ace0 f   LenPropertyODBC.obj
 0001:00079ce0       __unwindfunclet$?InsertNewGroup@CLenPropertyODBC@@QAE?AV?$CStringT@DV?$StrTraitMFC_DLL@DV?$ChTraitsCRT@D@ATL@@@@@ATL@@V23@@Z$0 0047ace0 f   LenPropertyODBC.obj
 0001:00079ce0       __unwindfunclet$?RemoveGroup@CLenPropertyODBC@@QAE?AV?$CStringT@DV?$StrTraitMFC_DLL@DV?$ChTraitsCRT@D@ATL@@@@@ATL@@V23@@Z$0 0047ace0 f   LenPropertyODBC.obj
 0001:00079ce9       __unwindfunclet$?RemoveGroup@CLenPropertyODBC@@QAE?AV?$CStringT@DV?$StrTraitMFC_DLL@DV?$ChTraitsCRT@D@ATL@@@@@ATL@@V23@@Z$2 0047ace9 f   LenPropertyODBC.obj
 0001:00079ce9       __unwindfunclet$?GetAllGroupClient@CLenPropertyODBC@@QAE?AV?$CStringT@DV?$StrTraitMFC_DLL@DV?$ChTraitsCRT@D@ATL@@@@@ATL@@V23@@Z$2 0047ace9 f   LenPropertyODBC.obj
 0001:00079ce9       __unwindfunclet$?InsertNewGroup@CLenPropertyODBC@@QAE?AV?$CStringT@DV?$StrTraitMFC_DLL@DV?$ChTraitsCRT@D@ATL@@@@@ATL@@V23@@Z$2 0047ace9 f   LenPropertyODBC.obj
 0001:00079cf2       __unwindfunclet$?RemoveGroup@CLenPropertyODBC@@QAE?AV?$CStringT@DV?$StrTraitMFC_DLL@DV?$ChTraitsCRT@D@ATL@@@@@ATL@@V23@@Z$3 0047acf2 f   LenPropertyODBC.obj
 0001:00079cf2       __unwindfunclet$?GetAllGroupClient@CLenPropertyODBC@@QAE?AV?$CStringT@DV?$StrTraitMFC_DLL@DV?$ChTraitsCRT@D@ATL@@@@@ATL@@V23@@Z$3 0047acf2 f   LenPropertyODBC.obj
 0001:00079cf2       __unwindfunclet$?InsertNewGroup@CLenPropertyODBC@@QAE?AV?$CStringT@DV?$StrTraitMFC_DLL@DV?$ChTraitsCRT@D@ATL@@@@@ATL@@V23@@Z$3 0047acf2 f   LenPropertyODBC.obj
 0001:00079cfb       __ehhandler$?RemoveGroup@CLenPropertyODBC@@QAE?AV?$CStringT@DV?$StrTraitMFC_DLL@DV?$ChTraitsCRT@D@ATL@@@@@ATL@@V23@@Z 0047acfb f   LenPropertyODBC.obj
 0001:00079cfb       __ehhandler$?InsertNewGroup@CLenPropertyODBC@@QAE?AV?$CStringT@DV?$StrTraitMFC_DLL@DV?$ChTraitsCRT@D@ATL@@@@@ATL@@V23@@Z 0047acfb f   LenPropertyODBC.obj
 0001:00079cfb       __ehhandler$?GetAllGroupClient@CLenPropertyODBC@@QAE?AV?$CStringT@DV?$StrTraitMFC_DLL@DV?$ChTraitsCRT@D@ATL@@@@@ATL@@V23@@Z 0047acfb f   LenPropertyODBC.obj
 0001:00079d20       __unwindfunclet$?InsertClientToGroup@CLenPropertyODBC@@QAE?AV?$CStringT@DV?$StrTraitMFC_DLL@DV?$ChTraitsCRT@D@ATL@@@@@ATL@@UtagGroupClient@@@Z$1 0047ad20 f   LenPropertyODBC.obj
 0001:00079d20       __unwindfunclet$?UpdateGroupNameOfClient@CLenPropertyODBC@@QAE?AV?$CStringT@DV?$StrTraitMFC_DLL@DV?$ChTraitsCRT@D@ATL@@@@@ATL@@UtagGroupClient@@@Z$1 0047ad20 f   LenPropertyODBC.obj
 0001:00079d20       __unwindfunclet$?UpdateOneToGroup@CLenPropertyODBC@@QAE?AV?$CStringT@DV?$StrTraitMFC_DLL@DV?$ChTraitsCRT@D@ATL@@@@@ATL@@UtagGroupClient@@@Z$1 0047ad20 f   LenPropertyODBC.obj
 0001:00079d29       __unwindfunclet$?InsertClientToGroup@CLenPropertyODBC@@QAE?AV?$CStringT@DV?$StrTraitMFC_DLL@DV?$ChTraitsCRT@D@ATL@@@@@ATL@@UtagGroupClient@@@Z$2 0047ad29 f   LenPropertyODBC.obj
 0001:00079d29       __unwindfunclet$?UpdateOneToGroup@CLenPropertyODBC@@QAE?AV?$CStringT@DV?$StrTraitMFC_DLL@DV?$ChTraitsCRT@D@ATL@@@@@ATL@@UtagGroupClient@@@Z$2 0047ad29 f   LenPropertyODBC.obj
 0001:00079d29       __unwindfunclet$?UpdateGroupNameOfClient@CLenPropertyODBC@@QAE?AV?$CStringT@DV?$StrTraitMFC_DLL@DV?$ChTraitsCRT@D@ATL@@@@@ATL@@UtagGroupClient@@@Z$2 0047ad29 f   LenPropertyODBC.obj
 0001:00079d32       __ehhandler$?UpdateGroupNameOfClient@CLenPropertyODBC@@QAE?AV?$CStringT@DV?$StrTraitMFC_DLL@DV?$ChTraitsCRT@D@ATL@@@@@ATL@@UtagGroupClient@@@Z 0047ad32 f   LenPropertyODBC.obj
 0001:00079d32       __ehhandler$?InsertClientToGroup@CLenPropertyODBC@@QAE?AV?$CStringT@DV?$StrTraitMFC_DLL@DV?$ChTraitsCRT@D@ATL@@@@@ATL@@UtagGroupClient@@@Z 0047ad32 f   LenPropertyODBC.obj
 0001:00079d32       __ehhandler$?UpdateOneToGroup@CLenPropertyODBC@@QAE?AV?$CStringT@DV?$StrTraitMFC_DLL@DV?$ChTraitsCRT@D@ATL@@@@@ATL@@UtagGroupClient@@@Z 0047ad32 f   LenPropertyODBC.obj
 0001:00079d50       __unwindfunclet$?TranHexToString@CLenPropertyODBC@@QAE?AV?$CStringT@DV?$StrTraitMFC_DLL@DV?$ChTraitsCRT@D@ATL@@@@@ATL@@V23@H@Z$0 0047ad50 f   LenPropertyODBC.obj
 0001:00079d59       __unwindfunclet$?TranHexToString@CLenPropertyODBC@@QAE?AV?$CStringT@DV?$StrTraitMFC_DLL@DV?$ChTraitsCRT@D@ATL@@@@@ATL@@V23@H@Z$1 0047ad59 f   LenPropertyODBC.obj
 0001:00079d62       __unwindfunclet$?TranHexToString@CLenPropertyODBC@@QAE?AV?$CStringT@DV?$StrTraitMFC_DLL@DV?$ChTraitsCRT@D@ATL@@@@@ATL@@V23@H@Z$2 0047ad62 f   LenPropertyODBC.obj
 0001:00079d6b       __unwindfunclet$?TranHexToString@CLenPropertyODBC@@QAE?AV?$CStringT@DV?$StrTraitMFC_DLL@DV?$ChTraitsCRT@D@ATL@@@@@ATL@@V23@H@Z$4 0047ad6b f   LenPropertyODBC.obj
 0001:00079d74       __ehhandler$?TranHexToString@CLenPropertyODBC@@QAE?AV?$CStringT@DV?$StrTraitMFC_DLL@DV?$ChTraitsCRT@D@ATL@@@@@ATL@@V23@H@Z 0047ad74 f   LenPropertyODBC.obj
 0001:00079da0       __unwindfunclet$??0CLoginPasswordDlg@@QAE@PAVCWnd@@@Z$0 0047ada0 f   LoginPasswordDlg.obj
 0001:00079da8       __unwindfunclet$??0CLoginPasswordDlg@@QAE@PAVCWnd@@@Z$1 0047ada8 f   LoginPasswordDlg.obj
 0001:00079db4       __unwindfunclet$??0CLoginPasswordDlg@@QAE@PAVCWnd@@@Z$2 0047adb4 f   LoginPasswordDlg.obj
 0001:00079dbf       __ehhandler$??0CLoginPasswordDlg@@QAE@PAVCWnd@@@Z 0047adbf f   LoginPasswordDlg.obj
 0001:00079de0       __unwindfunclet$??1CMsgDlg@@UAE@XZ$0 0047ade0 f   LoginPasswordDlg.obj
 0001:00079de0       __unwindfunclet$??0CExecuteProcedure@@QAE@PAVCWnd@@@Z$0 0047ade0 f   LoginPasswordDlg.obj
 0001:00079de0       __unwindfunclet$??0CBroadWaitDlg@@QAE@PAVCWnd@@@Z$0 0047ade0 f   LoginPasswordDlg.obj
 0001:00079de0       __unwindfunclet$??1CLoginPasswordDlg@@UAE@XZ$0 0047ade0 f   LoginPasswordDlg.obj
 0001:00079de8       __unwindfunclet$??1CLoginPasswordDlg@@UAE@XZ$1 0047ade8 f   LoginPasswordDlg.obj
 0001:00079de8       __unwindfunclet$??0CExecuteProcedure@@QAE@PAVCWnd@@@Z$1 0047ade8 f   LoginPasswordDlg.obj
 0001:00079de8       __unwindfunclet$??0CBroadWaitDlg@@QAE@PAVCWnd@@@Z$1 0047ade8 f   LoginPasswordDlg.obj
 0001:00079de8       __unwindfunclet$??1CMsgDlg@@UAE@XZ$1 0047ade8 f   LoginPasswordDlg.obj
 0001:00079df4       __ehhandler$??1CLoginPasswordDlg@@UAE@XZ 0047adf4 f   LoginPasswordDlg.obj
 0001:00079df4       __ehhandler$??0CBroadWaitDlg@@QAE@PAVCWnd@@@Z 0047adf4 f   LoginPasswordDlg.obj
 0001:00079df4       __ehhandler$??0CExecuteProcedure@@QAE@PAVCWnd@@@Z 0047adf4 f   LoginPasswordDlg.obj
 0001:00079df4       __ehhandler$??1CMsgDlg@@UAE@XZ 0047adf4 f   LoginPasswordDlg.obj
 0001:00079e10       __unwindfunclet$?OnOK@CLoginPasswordDlg@@MAEXXZ$0 0047ae10 f   LoginPasswordDlg.obj
 0001:00079e18       __ehhandler$?OnOK@CLoginPasswordDlg@@MAEXXZ 0047ae18 f   LoginPasswordDlg.obj
 0001:00079e40       __unwindfunclet$?OnInitDialog@CLoginPasswordDlg@@MAEHXZ$0 0047ae40 f   LoginPasswordDlg.obj
 0001:00079e49       __unwindfunclet$?OnInitDialog@CLoginPasswordDlg@@MAEHXZ$1 0047ae49 f   LoginPasswordDlg.obj
 0001:00079e52       __unwindfunclet$?OnInitDialog@CLoginPasswordDlg@@MAEHXZ$2 0047ae52 f   LoginPasswordDlg.obj
 0001:00079e5b       __unwindfunclet$?OnInitDialog@CLoginPasswordDlg@@MAEHXZ$3 0047ae5b f   LoginPasswordDlg.obj
 0001:00079e64       __unwindfunclet$?OnInitDialog@CLoginPasswordDlg@@MAEHXZ$4 0047ae64 f   LoginPasswordDlg.obj
 0001:00079e6c       __unwindfunclet$?OnInitDialog@CLoginPasswordDlg@@MAEHXZ$7 0047ae6c f   LoginPasswordDlg.obj
 0001:00079e75       __unwindfunclet$?OnInitDialog@CLoginPasswordDlg@@MAEHXZ$8 0047ae75 f   LoginPasswordDlg.obj
 0001:00079e7e       __ehhandler$?OnInitDialog@CLoginPasswordDlg@@MAEHXZ 0047ae7e f   LoginPasswordDlg.obj
 0001:00079eb0       __unwindfunclet$?OnBnClickedOk@CLoginPasswordDlg@@QAEXXZ$0 0047aeb0 f   LoginPasswordDlg.obj
 0001:00079eb9       __unwindfunclet$?OnBnClickedOk@CLoginPasswordDlg@@QAEXXZ$1 0047aeb9 f   LoginPasswordDlg.obj
 0001:00079ec2       __ehhandler$?OnBnClickedOk@CLoginPasswordDlg@@QAEXXZ 0047aec2 f   LoginPasswordDlg.obj
 0001:00079ee0       __unwindfunclet$?ExtPwd@CLoginPasswordDlg@@AAE_NAAV?$CStringT@DV?$StrTraitMFC_DLL@DV?$ChTraitsCRT@D@ATL@@@@@ATL@@PAEH@Z$0 0047aee0 f   LoginPasswordDlg.obj
 0001:00079ee9       __ehhandler$?ExtPwd@CLoginPasswordDlg@@AAE_NAAV?$CStringT@DV?$StrTraitMFC_DLL@DV?$ChTraitsCRT@D@ATL@@@@@ATL@@PAEH@Z 0047aee9 f   LoginPasswordDlg.obj
 0001:00079f10       __unwindfunclet$?CompareProc@@YGHJJJ@Z$0 0047af10 f   MainFrm.obj
 0001:00079f19       __unwindfunclet$?CompareProc@@YGHJJJ@Z$1 0047af19 f   MainFrm.obj
 0001:00079f22       __unwindfunclet$?CompareProc@@YGHJJJ@Z$2 0047af22 f   MainFrm.obj
 0001:00079f2b       __unwindfunclet$?CompareProc@@YGHJJJ@Z$3 0047af2b f   MainFrm.obj
 0001:00079f34       __unwindfunclet$?CompareProc@@YGHJJJ@Z$4 0047af34 f   MainFrm.obj
 0001:00079f3d       __unwindfunclet$?CompareProc@@YGHJJJ@Z$5 0047af3d f   MainFrm.obj
 0001:00079f46       __unwindfunclet$?CompareProc@@YGHJJJ@Z$6 0047af46 f   MainFrm.obj
 0001:00079f4f       __unwindfunclet$?CompareProc@@YGHJJJ@Z$7 0047af4f f   MainFrm.obj
 0001:00079f58       __unwindfunclet$?CompareProc@@YGHJJJ@Z$8 0047af58 f   MainFrm.obj
 0001:00079f61       __unwindfunclet$?CompareProc@@YGHJJJ@Z$9 0047af61 f   MainFrm.obj
 0001:00079f6a       __unwindfunclet$?CompareProc@@YGHJJJ@Z$10 0047af6a f   MainFrm.obj
 0001:00079f73       __unwindfunclet$?CompareProc@@YGHJJJ@Z$11 0047af73 f   MainFrm.obj
 0001:00079f7c       __unwindfunclet$?CompareProc@@YGHJJJ@Z$12 0047af7c f   MainFrm.obj
 0001:00079f85       __unwindfunclet$?CompareProc@@YGHJJJ@Z$13 0047af85 f   MainFrm.obj
 0001:00079f8e       __ehhandler$?CompareProc@@YGHJJJ@Z 0047af8e f   MainFrm.obj
 0001:00079fb0       __unwindfunclet$??0CMainFrame@@IAE@XZ$0 0047afb0 f   MainFrm.obj
 0001:00079fb8       __unwindfunclet$??0CMainFrame@@IAE@XZ$1 0047afb8 f   MainFrm.obj
 0001:00079fc6       __unwindfunclet$??0CMainFrame@@IAE@XZ$2 0047afc6 f   MainFrm.obj
 0001:00079fd5       __unwindfunclet$??0CMainFrame@@IAE@XZ$3 0047afd5 f   MainFrm.obj
 0001:00079fe3       __unwindfunclet$??0CMainFrame@@IAE@XZ$4 0047afe3 f   MainFrm.obj
 0001:00079ff1       __unwindfunclet$??0CMainFrame@@IAE@XZ$5 0047aff1 f   MainFrm.obj
 0001:00079fff       __unwindfunclet$??0CMainFrame@@IAE@XZ$6 0047afff f   MainFrm.obj
 0001:0007a00d       __unwindfunclet$??0CMainFrame@@IAE@XZ$7 0047b00d f   MainFrm.obj
 0001:0007a01b       __unwindfunclet$??0CMainFrame@@IAE@XZ$8 0047b01b f   MainFrm.obj
 0001:0007a029       __unwindfunclet$??0CMainFrame@@IAE@XZ$9 0047b029 f   MainFrm.obj
 0001:0007a038       __unwindfunclet$??0CMainFrame@@IAE@XZ$10 0047b038 f   MainFrm.obj
 0001:0007a046       __unwindfunclet$??0CMainFrame@@IAE@XZ$11 0047b046 f   MainFrm.obj
 0001:0007a054       __unwindfunclet$??0CMainFrame@@IAE@XZ$12 0047b054 f   MainFrm.obj
 0001:0007a062       __unwindfunclet$??0CMainFrame@@IAE@XZ$13 0047b062 f   MainFrm.obj
 0001:0007a070       __unwindfunclet$??0CMainFrame@@IAE@XZ$14 0047b070 f   MainFrm.obj
 0001:0007a07e       __unwindfunclet$??0CMainFrame@@IAE@XZ$15 0047b07e f   MainFrm.obj
 0001:0007a08c       __unwindfunclet$??0CMainFrame@@IAE@XZ$16 0047b08c f   MainFrm.obj
 0001:0007a09a       __unwindfunclet$??0CMainFrame@@IAE@XZ$17 0047b09a f   MainFrm.obj
 0001:0007a0a8       __unwindfunclet$??0CMainFrame@@IAE@XZ$18 0047b0a8 f   MainFrm.obj
 0001:0007a0b6       __unwindfunclet$??0CMainFrame@@IAE@XZ$19 0047b0b6 f   MainFrm.obj
 0001:0007a0c4       __unwindfunclet$??0CMainFrame@@IAE@XZ$20 0047b0c4 f   MainFrm.obj
 0001:0007a0d2       __unwindfunclet$??0CMainFrame@@IAE@XZ$21 0047b0d2 f   MainFrm.obj
 0001:0007a0e0       __unwindfunclet$??0CMainFrame@@IAE@XZ$22 0047b0e0 f   MainFrm.obj
 0001:0007a0ee       __unwindfunclet$??0CMainFrame@@IAE@XZ$23 0047b0ee f   MainFrm.obj
 0001:0007a0fc       __unwindfunclet$??0CMainFrame@@IAE@XZ$24 0047b0fc f   MainFrm.obj
 0001:0007a10a       __unwindfunclet$??0CMainFrame@@IAE@XZ$25 0047b10a f   MainFrm.obj
 0001:0007a118       __unwindfunclet$??0CMainFrame@@IAE@XZ$26 0047b118 f   MainFrm.obj
 0001:0007a126       __ehhandler$??0CMainFrame@@IAE@XZ 0047b126 f   MainFrm.obj
 0001:0007a150       __unwindfunclet$??1CMainFrame@@UAE@XZ$0 0047b150 f   MainFrm.obj
 0001:0007a158       __unwindfunclet$??1CMainFrame@@UAE@XZ$1 0047b158 f   MainFrm.obj
 0001:0007a166       __unwindfunclet$??1CMainFrame@@UAE@XZ$2 0047b166 f   MainFrm.obj
 0001:0007a175       __unwindfunclet$??1CMainFrame@@UAE@XZ$3 0047b175 f   MainFrm.obj
 0001:0007a183       __unwindfunclet$??1CMainFrame@@UAE@XZ$4 0047b183 f   MainFrm.obj
 0001:0007a191       __unwindfunclet$??1CMainFrame@@UAE@XZ$5 0047b191 f   MainFrm.obj
 0001:0007a19f       __unwindfunclet$??1CMainFrame@@UAE@XZ$6 0047b19f f   MainFrm.obj
 0001:0007a1ad       __unwindfunclet$??1CMainFrame@@UAE@XZ$7 0047b1ad f   MainFrm.obj
 0001:0007a1bb       __unwindfunclet$??1CMainFrame@@UAE@XZ$8 0047b1bb f   MainFrm.obj
 0001:0007a1c9       __unwindfunclet$??1CMainFrame@@UAE@XZ$9 0047b1c9 f   MainFrm.obj
 0001:0007a1d8       __unwindfunclet$??1CMainFrame@@UAE@XZ$10 0047b1d8 f   MainFrm.obj
 0001:0007a1e6       __unwindfunclet$??1CMainFrame@@UAE@XZ$11 0047b1e6 f   MainFrm.obj
 0001:0007a1f4       __unwindfunclet$??1CMainFrame@@UAE@XZ$12 0047b1f4 f   MainFrm.obj
 0001:0007a202       __unwindfunclet$??1CMainFrame@@UAE@XZ$13 0047b202 f   MainFrm.obj
 0001:0007a210       __unwindfunclet$??1CMainFrame@@UAE@XZ$14 0047b210 f   MainFrm.obj
 0001:0007a21e       __unwindfunclet$??1CMainFrame@@UAE@XZ$15 0047b21e f   MainFrm.obj
 0001:0007a22c       __unwindfunclet$??1CMainFrame@@UAE@XZ$16 0047b22c f   MainFrm.obj
 0001:0007a23a       __unwindfunclet$??1CMainFrame@@UAE@XZ$17 0047b23a f   MainFrm.obj
 0001:0007a248       __unwindfunclet$??1CMainFrame@@UAE@XZ$18 0047b248 f   MainFrm.obj
 0001:0007a256       __unwindfunclet$??1CMainFrame@@UAE@XZ$19 0047b256 f   MainFrm.obj
 0001:0007a264       __unwindfunclet$??1CMainFrame@@UAE@XZ$20 0047b264 f   MainFrm.obj
 0001:0007a272       __unwindfunclet$??1CMainFrame@@UAE@XZ$21 0047b272 f   MainFrm.obj
 0001:0007a280       __unwindfunclet$??1CMainFrame@@UAE@XZ$22 0047b280 f   MainFrm.obj
 0001:0007a28e       __unwindfunclet$??1CMainFrame@@UAE@XZ$23 0047b28e f   MainFrm.obj
 0001:0007a29c       __unwindfunclet$??1CMainFrame@@UAE@XZ$24 0047b29c f   MainFrm.obj
 0001:0007a2aa       __unwindfunclet$??1CMainFrame@@UAE@XZ$25 0047b2aa f   MainFrm.obj
 0001:0007a2b8       __ehhandler$??1CMainFrame@@UAE@XZ 0047b2b8 f   MainFrm.obj
 0001:0007a2e0       __unwindfunclet$?OnCreate@CMainFrame@@IAEHPAUtagCREATESTRUCTA@@@Z$0 0047b2e0 f   MainFrm.obj
 0001:0007a2eb       __unwindfunclet$?OnCreate@CMainFrame@@IAEHPAUtagCREATESTRUCTA@@@Z$1 0047b2eb f   MainFrm.obj
 0001:0007a2f4       __unwindfunclet$?OnCreate@CMainFrame@@IAEHPAUtagCREATESTRUCTA@@@Z$2 0047b2f4 f   MainFrm.obj
 0001:0007a300       __unwindfunclet$?OnCreate@CMainFrame@@IAEHPAUtagCREATESTRUCTA@@@Z$3 0047b300 f   MainFrm.obj
 0001:0007a30c       __unwindfunclet$?OnCreate@CMainFrame@@IAEHPAUtagCREATESTRUCTA@@@Z$4 0047b30c f   MainFrm.obj
 0001:0007a318       __unwindfunclet$?OnCreate@CMainFrame@@IAEHPAUtagCREATESTRUCTA@@@Z$6 0047b318 f   MainFrm.obj
 0001:0007a324       __unwindfunclet$?OnCreate@CMainFrame@@IAEHPAUtagCREATESTRUCTA@@@Z$7 0047b324 f   MainFrm.obj
 0001:0007a330       __unwindfunclet$?OnCreate@CMainFrame@@IAEHPAUtagCREATESTRUCTA@@@Z$8 0047b330 f   MainFrm.obj
 0001:0007a33d       __unwindfunclet$?OnCreate@CMainFrame@@IAEHPAUtagCREATESTRUCTA@@@Z$9 0047b33d f   MainFrm.obj
 0001:0007a360       __unwindfunclet$?OnCreate@CMainFrame@@IAEHPAUtagCREATESTRUCTA@@@Z$10 0047b360 f   MainFrm.obj
 0001:0007a36d       __unwindfunclet$?OnCreate@CMainFrame@@IAEHPAUtagCREATESTRUCTA@@@Z$11 0047b36d f   MainFrm.obj
 0001:0007a378       __unwindfunclet$?OnCreate@CMainFrame@@IAEHPAUtagCREATESTRUCTA@@@Z$12 0047b378 f   MainFrm.obj
 0001:0007a384       __unwindfunclet$?OnCreate@CMainFrame@@IAEHPAUtagCREATESTRUCTA@@@Z$13 0047b384 f   MainFrm.obj
 0001:0007a390       __unwindfunclet$?OnCreate@CMainFrame@@IAEHPAUtagCREATESTRUCTA@@@Z$14 0047b390 f   MainFrm.obj
 0001:0007a39c       __unwindfunclet$?OnCreate@CMainFrame@@IAEHPAUtagCREATESTRUCTA@@@Z$15 0047b39c f   MainFrm.obj
 0001:0007a3a8       __unwindfunclet$?OnCreate@CMainFrame@@IAEHPAUtagCREATESTRUCTA@@@Z$16 0047b3a8 f   MainFrm.obj
 0001:0007a3b4       __unwindfunclet$?OnCreate@CMainFrame@@IAEHPAUtagCREATESTRUCTA@@@Z$17 0047b3b4 f   MainFrm.obj
 0001:0007a3bd       __unwindfunclet$?OnCreate@CMainFrame@@IAEHPAUtagCREATESTRUCTA@@@Z$18 0047b3bd f   MainFrm.obj
 0001:0007a3c9       __unwindfunclet$?OnCreate@CMainFrame@@IAEHPAUtagCREATESTRUCTA@@@Z$19 0047b3c9 f   MainFrm.obj
 0001:0007a3d2       __unwindfunclet$?OnCreate@CMainFrame@@IAEHPAUtagCREATESTRUCTA@@@Z$20 0047b3d2 f   MainFrm.obj
 0001:0007a3db       __unwindfunclet$?OnCreate@CMainFrame@@IAEHPAUtagCREATESTRUCTA@@@Z$21 0047b3db f   MainFrm.obj
 0001:0007a3e7       __unwindfunclet$?OnCreate@CMainFrame@@IAEHPAUtagCREATESTRUCTA@@@Z$22 0047b3e7 f   MainFrm.obj
 0001:0007a3f2       __unwindfunclet$?OnCreate@CMainFrame@@IAEHPAUtagCREATESTRUCTA@@@Z$24 0047b3f2 f   MainFrm.obj
 0001:0007a3fe       __unwindfunclet$?OnCreate@CMainFrame@@IAEHPAUtagCREATESTRUCTA@@@Z$26 0047b3fe f   MainFrm.obj
 0001:0007a40a       __unwindfunclet$?OnCreate@CMainFrame@@IAEHPAUtagCREATESTRUCTA@@@Z$27 0047b40a f   MainFrm.obj
 0001:0007a416       __unwindfunclet$?OnCreate@CMainFrame@@IAEHPAUtagCREATESTRUCTA@@@Z$29 0047b416 f   MainFrm.obj
 0001:0007a422       __unwindfunclet$?OnCreate@CMainFrame@@IAEHPAUtagCREATESTRUCTA@@@Z$30 0047b422 f   MainFrm.obj
 0001:0007a42e       __ehhandler$?OnCreate@CMainFrame@@IAEHPAUtagCREATESTRUCTA@@@Z 0047b42e f   MainFrm.obj
 0001:0007a460       __unwindfunclet$?InitializeRibbon@CMainFrame@@IAEXXZ$0 0047b460 f   MainFrm.obj
 0001:0007a469       __unwindfunclet$?InitializeRibbon@CMainFrame@@IAEXXZ$1 0047b469 f   MainFrm.obj
 0001:0007a473       __unwindfunclet$?InitializeRibbon@CMainFrame@@IAEXXZ$2 0047b473 f   MainFrm.obj
 0001:0007a47b       __unwindfunclet$?InitializeRibbon@CMainFrame@@IAEXXZ$3 0047b47b f   MainFrm.obj
 0001:0007a485       __unwindfunclet$?InitializeRibbon@CMainFrame@@IAEXXZ$4 0047b485 f   MainFrm.obj
 0001:0007a4a8       __unwindfunclet$?InitializeRibbon@CMainFrame@@IAEXXZ$5 0047b4a8 f   MainFrm.obj
 0001:0007a4b5       __unwindfunclet$?InitializeRibbon@CMainFrame@@IAEXXZ$6 0047b4b5 f   MainFrm.obj
 0001:0007a4d8       __ehhandler$?InitializeRibbon@CMainFrame@@IAEXXZ 0047b4d8 f   MainFrm.obj
 0001:0007a500       __unwindfunclet$?ProductVERCheck@CMainFrame@@QAEHXZ$0 0047b500 f   MainFrm.obj
 0001:0007a509       __unwindfunclet$?ProductVERCheck@CMainFrame@@QAEHXZ$1 0047b509 f   MainFrm.obj
 0001:0007a512       __unwindfunclet$?ProductVERCheck@CMainFrame@@QAEHXZ$2 0047b512 f   MainFrm.obj
 0001:0007a51b       __ehhandler$?ProductVERCheck@CMainFrame@@QAEHXZ 0047b51b f   MainFrm.obj
 0001:0007a540       __unwindfunclet$?CreateDockingWindows@CMainFrame@@IAEHXZ$0 0047b540 f   MainFrm.obj
 0001:0007a549       __unwindfunclet$?CreateDockingWindows@CMainFrame@@IAEHXZ$1 0047b549 f   MainFrm.obj
 0001:0007a552       __ehhandler$?CreateDockingWindows@CMainFrame@@IAEHXZ 0047b552 f   MainFrm.obj
 0001:0007a570       __unwindfunclet$?OnApplicationLook@CMainFrame@@IAEXI@Z$0 0047b570 f   MainFrm.obj
 0001:0007a578       __ehhandler$?OnApplicationLook@CMainFrame@@IAEXI@Z 0047b578 f   MainFrm.obj
 0001:0007a5a0       __unwindfunclet$?OnTimer@CMainFrame@@QAEXI@Z$0 0047b5a0 f   MainFrm.obj
 0001:0007a5ac       __unwindfunclet$?OnTimer@CMainFrame@@QAEXI@Z$2 0047b5ac f   MainFrm.obj
 0001:0007a5b8       __unwindfunclet$?OnTimer@CMainFrame@@QAEXI@Z$4 0047b5b8 f   MainFrm.obj
 0001:0007a5c4       __unwindfunclet$?OnTimer@CMainFrame@@QAEXI@Z$5 0047b5c4 f   MainFrm.obj
 0001:0007a5d0       __unwindfunclet$?OnTimer@CMainFrame@@QAEXI@Z$6 0047b5d0 f   MainFrm.obj
 0001:0007a5dc       __unwindfunclet$?OnTimer@CMainFrame@@QAEXI@Z$7 0047b5dc f   MainFrm.obj
 0001:0007a5e8       __ehhandler$?OnTimer@CMainFrame@@QAEXI@Z 0047b5e8 f   MainFrm.obj
 0001:0007a610       __unwindfunclet$?InitNetworkComponent@CMainFrame@@QAEHXZ$0 0047b610 f   MainFrm.obj
 0001:0007a619       __unwindfunclet$?InitNetworkComponent@CMainFrame@@QAEHXZ$1 0047b619 f   MainFrm.obj
 0001:0007a622       __unwindfunclet$?InitNetworkComponent@CMainFrame@@QAEHXZ$2 0047b622 f   MainFrm.obj
 0001:0007a62b       __unwindfunclet$?InitNetworkComponent@CMainFrame@@QAEHXZ$3 0047b62b f   MainFrm.obj
 0001:0007a634       __ehhandler$?InitNetworkComponent@CMainFrame@@QAEHXZ 0047b634 f   MainFrm.obj
 0001:0007a650       __unwindfunclet$?_RequestHandleThread@CMainFrame@@SAIPAX@Z$0 0047b650 f   MainFrm.obj
 0001:0007a65c       __unwindfunclet$?_RequestHandleThread@CMainFrame@@SAIPAX@Z$1 0047b65c f   MainFrm.obj
 0001:0007a668       __ehhandler$?_RequestHandleThread@CMainFrame@@SAIPAX@Z 0047b668 f   MainFrm.obj
 0001:0007a690       __unwindfunclet$?CheckClientsOnline@CMainFrame@@QAEXXZ$0 0047b690 f   MainFrm.obj
 0001:0007a699       __unwindfunclet$?CheckClientsOnline@CMainFrame@@QAEXXZ$3 0047b699 f   MainFrm.obj
 0001:0007a6a2       __unwindfunclet$?CheckClientsOnline@CMainFrame@@QAEXXZ$4 0047b6a2 f   MainFrm.obj
 0001:0007a6ab       __unwindfunclet$?CheckClientsOnline@CMainFrame@@QAEXXZ$5 0047b6ab f   MainFrm.obj
 0001:0007a6b4       __unwindfunclet$?CheckClientsOnline@CMainFrame@@QAEXXZ$6 0047b6b4 f   MainFrm.obj
 0001:0007a6bd       __unwindfunclet$?CheckClientsOnline@CMainFrame@@QAEXXZ$7 0047b6bd f   MainFrm.obj
 0001:0007a6c6       __unwindfunclet$?CheckClientsOnline@CMainFrame@@QAEXXZ$8 0047b6c6 f   MainFrm.obj
 0001:0007a6cf       __unwindfunclet$?CheckClientsOnline@CMainFrame@@QAEXXZ$9 0047b6cf f   MainFrm.obj
 0001:0007a6d8       __unwindfunclet$?CheckClientsOnline@CMainFrame@@QAEXXZ$10 0047b6d8 f   MainFrm.obj
 0001:0007a6e1       __ehhandler$?CheckClientsOnline@CMainFrame@@QAEXXZ 0047b6e1 f   MainFrm.obj
 0001:0007a700       __unwindfunclet$?HandleLoginRequest@CMainFrame@@QAEHPAUtagRECVREQUEST@@@Z$0 0047b700 f   MainFrm.obj
 0001:0007a70c       __unwindfunclet$?HandleLoginRequest@CMainFrame@@QAEHPAUtagRECVREQUEST@@@Z$2 0047b70c f   MainFrm.obj
 0001:0007a718       __unwindfunclet$?HandleLoginRequest@CMainFrame@@QAEHPAUtagRECVREQUEST@@@Z$3 0047b718 f   MainFrm.obj
 0001:0007a724       __unwindfunclet$?HandleLoginRequest@CMainFrame@@QAEHPAUtagRECVREQUEST@@@Z$4 0047b724 f   MainFrm.obj
 0001:0007a730       __unwindfunclet$?HandleLoginRequest@CMainFrame@@QAEHPAUtagRECVREQUEST@@@Z$5 0047b730 f   MainFrm.obj
 0001:0007a73c       __unwindfunclet$?HandleLoginRequest@CMainFrame@@QAEHPAUtagRECVREQUEST@@@Z$6 0047b73c f   MainFrm.obj
 0001:0007a748       __unwindfunclet$?HandleLoginRequest@CMainFrame@@QAEHPAUtagRECVREQUEST@@@Z$7 0047b748 f   MainFrm.obj
 0001:0007a754       __unwindfunclet$?HandleLoginRequest@CMainFrame@@QAEHPAUtagRECVREQUEST@@@Z$8 0047b754 f   MainFrm.obj
 0001:0007a760       __unwindfunclet$?HandleLoginRequest@CMainFrame@@QAEHPAUtagRECVREQUEST@@@Z$9 0047b760 f   MainFrm.obj
 0001:0007a76c       __unwindfunclet$?HandleLoginRequest@CMainFrame@@QAEHPAUtagRECVREQUEST@@@Z$10 0047b76c f   MainFrm.obj
 0001:0007a778       __unwindfunclet$?HandleLoginRequest@CMainFrame@@QAEHPAUtagRECVREQUEST@@@Z$11 0047b778 f   MainFrm.obj
 0001:0007a784       __unwindfunclet$?HandleLoginRequest@CMainFrame@@QAEHPAUtagRECVREQUEST@@@Z$12 0047b784 f   MainFrm.obj
 0001:0007a790       __unwindfunclet$?HandleLoginRequest@CMainFrame@@QAEHPAUtagRECVREQUEST@@@Z$13 0047b790 f   MainFrm.obj
 0001:0007a79c       __unwindfunclet$?HandleLoginRequest@CMainFrame@@QAEHPAUtagRECVREQUEST@@@Z$14 0047b79c f   MainFrm.obj
 0001:0007a7a8       __unwindfunclet$?HandleLoginRequest@CMainFrame@@QAEHPAUtagRECVREQUEST@@@Z$15 0047b7a8 f   MainFrm.obj
 0001:0007a7b4       __unwindfunclet$?HandleLoginRequest@CMainFrame@@QAEHPAUtagRECVREQUEST@@@Z$18 0047b7b4 f   MainFrm.obj
 0001:0007a7c0       __unwindfunclet$?HandleLoginRequest@CMainFrame@@QAEHPAUtagRECVREQUEST@@@Z$19 0047b7c0 f   MainFrm.obj
 0001:0007a7cc       __unwindfunclet$?HandleLoginRequest@CMainFrame@@QAEHPAUtagRECVREQUEST@@@Z$20 0047b7cc f   MainFrm.obj
 0001:0007a7d8       __unwindfunclet$?HandleLoginRequest@CMainFrame@@QAEHPAUtagRECVREQUEST@@@Z$21 0047b7d8 f   MainFrm.obj
 0001:0007a7e4       __unwindfunclet$?HandleLoginRequest@CMainFrame@@QAEHPAUtagRECVREQUEST@@@Z$22 0047b7e4 f   MainFrm.obj
 0001:0007a7f0       __unwindfunclet$?HandleLoginRequest@CMainFrame@@QAEHPAUtagRECVREQUEST@@@Z$23 0047b7f0 f   MainFrm.obj
 0001:0007a7fc       __unwindfunclet$?HandleLoginRequest@CMainFrame@@QAEHPAUtagRECVREQUEST@@@Z$25 0047b7fc f   MainFrm.obj
 0001:0007a808       __unwindfunclet$?HandleLoginRequest@CMainFrame@@QAEHPAUtagRECVREQUEST@@@Z$26 0047b808 f   MainFrm.obj
 0001:0007a814       __unwindfunclet$?HandleLoginRequest@CMainFrame@@QAEHPAUtagRECVREQUEST@@@Z$27 0047b814 f   MainFrm.obj
 0001:0007a820       __unwindfunclet$?HandleLoginRequest@CMainFrame@@QAEHPAUtagRECVREQUEST@@@Z$30 0047b820 f   MainFrm.obj
 0001:0007a82c       __unwindfunclet$?HandleLoginRequest@CMainFrame@@QAEHPAUtagRECVREQUEST@@@Z$31 0047b82c f   MainFrm.obj
 0001:0007a838       __unwindfunclet$?HandleLoginRequest@CMainFrame@@QAEHPAUtagRECVREQUEST@@@Z$32 0047b838 f   MainFrm.obj
 0001:0007a844       __unwindfunclet$?HandleLoginRequest@CMainFrame@@QAEHPAUtagRECVREQUEST@@@Z$33 0047b844 f   MainFrm.obj
 0001:0007a850       __unwindfunclet$?HandleLoginRequest@CMainFrame@@QAEHPAUtagRECVREQUEST@@@Z$34 0047b850 f   MainFrm.obj
 0001:0007a85c       __unwindfunclet$?HandleLoginRequest@CMainFrame@@QAEHPAUtagRECVREQUEST@@@Z$35 0047b85c f   MainFrm.obj
 0001:0007a868       __unwindfunclet$?HandleLoginRequest@CMainFrame@@QAEHPAUtagRECVREQUEST@@@Z$36 0047b868 f   MainFrm.obj
 0001:0007a874       __unwindfunclet$?HandleLoginRequest@CMainFrame@@QAEHPAUtagRECVREQUEST@@@Z$37 0047b874 f   MainFrm.obj
 0001:0007a880       __unwindfunclet$?HandleLoginRequest@CMainFrame@@QAEHPAUtagRECVREQUEST@@@Z$38 0047b880 f   MainFrm.obj
 0001:0007a88c       __unwindfunclet$?HandleLoginRequest@CMainFrame@@QAEHPAUtagRECVREQUEST@@@Z$39 0047b88c f   MainFrm.obj
 0001:0007a898       __unwindfunclet$?HandleLoginRequest@CMainFrame@@QAEHPAUtagRECVREQUEST@@@Z$40 0047b898 f   MainFrm.obj
 0001:0007a8a4       __unwindfunclet$?HandleLoginRequest@CMainFrame@@QAEHPAUtagRECVREQUEST@@@Z$41 0047b8a4 f   MainFrm.obj
 0001:0007a8b0       __unwindfunclet$?HandleLoginRequest@CMainFrame@@QAEHPAUtagRECVREQUEST@@@Z$42 0047b8b0 f   MainFrm.obj
 0001:0007a8bc       __unwindfunclet$?HandleLoginRequest@CMainFrame@@QAEHPAUtagRECVREQUEST@@@Z$43 0047b8bc f   MainFrm.obj
 0001:0007a8c8       __unwindfunclet$?HandleLoginRequest@CMainFrame@@QAEHPAUtagRECVREQUEST@@@Z$44 0047b8c8 f   MainFrm.obj
 0001:0007a8d4       __unwindfunclet$?HandleLoginRequest@CMainFrame@@QAEHPAUtagRECVREQUEST@@@Z$45 0047b8d4 f   MainFrm.obj
 0001:0007a8e0       __unwindfunclet$?HandleLoginRequest@CMainFrame@@QAEHPAUtagRECVREQUEST@@@Z$46 0047b8e0 f   MainFrm.obj
 0001:0007a8ec       __unwindfunclet$?HandleLoginRequest@CMainFrame@@QAEHPAUtagRECVREQUEST@@@Z$47 0047b8ec f   MainFrm.obj
 0001:0007a8f8       __unwindfunclet$?HandleLoginRequest@CMainFrame@@QAEHPAUtagRECVREQUEST@@@Z$48 0047b8f8 f   MainFrm.obj
 0001:0007a904       __unwindfunclet$?HandleLoginRequest@CMainFrame@@QAEHPAUtagRECVREQUEST@@@Z$49 0047b904 f   MainFrm.obj
 0001:0007a910       __unwindfunclet$?HandleLoginRequest@CMainFrame@@QAEHPAUtagRECVREQUEST@@@Z$55 0047b910 f   MainFrm.obj
 0001:0007a91c       __unwindfunclet$?HandleLoginRequest@CMainFrame@@QAEHPAUtagRECVREQUEST@@@Z$56 0047b91c f   MainFrm.obj
 0001:0007a928       __unwindfunclet$?HandleLoginRequest@CMainFrame@@QAEHPAUtagRECVREQUEST@@@Z$57 0047b928 f   MainFrm.obj
 0001:0007a934       __unwindfunclet$?HandleLoginRequest@CMainFrame@@QAEHPAUtagRECVREQUEST@@@Z$58 0047b934 f   MainFrm.obj
 0001:0007a940       __unwindfunclet$?HandleLoginRequest@CMainFrame@@QAEHPAUtagRECVREQUEST@@@Z$59 0047b940 f   MainFrm.obj
 0001:0007a94c       __unwindfunclet$?HandleLoginRequest@CMainFrame@@QAEHPAUtagRECVREQUEST@@@Z$60 0047b94c f   MainFrm.obj
 0001:0007a958       __unwindfunclet$?HandleLoginRequest@CMainFrame@@QAEHPAUtagRECVREQUEST@@@Z$61 0047b958 f   MainFrm.obj
 0001:0007a964       __unwindfunclet$?HandleLoginRequest@CMainFrame@@QAEHPAUtagRECVREQUEST@@@Z$62 0047b964 f   MainFrm.obj
 0001:0007a970       __unwindfunclet$?HandleLoginRequest@CMainFrame@@QAEHPAUtagRECVREQUEST@@@Z$63 0047b970 f   MainFrm.obj
 0001:0007a97c       __unwindfunclet$?HandleLoginRequest@CMainFrame@@QAEHPAUtagRECVREQUEST@@@Z$64 0047b97c f   MainFrm.obj
 0001:0007a988       __unwindfunclet$?HandleLoginRequest@CMainFrame@@QAEHPAUtagRECVREQUEST@@@Z$65 0047b988 f   MainFrm.obj
 0001:0007a994       __unwindfunclet$?HandleLoginRequest@CMainFrame@@QAEHPAUtagRECVREQUEST@@@Z$66 0047b994 f   MainFrm.obj
 0001:0007a9a0       __unwindfunclet$?HandleLoginRequest@CMainFrame@@QAEHPAUtagRECVREQUEST@@@Z$67 0047b9a0 f   MainFrm.obj
 0001:0007a9ac       __unwindfunclet$?HandleLoginRequest@CMainFrame@@QAEHPAUtagRECVREQUEST@@@Z$68 0047b9ac f   MainFrm.obj
 0001:0007a9b8       __unwindfunclet$?HandleLoginRequest@CMainFrame@@QAEHPAUtagRECVREQUEST@@@Z$69 0047b9b8 f   MainFrm.obj
 0001:0007a9c4       __unwindfunclet$?HandleLoginRequest@CMainFrame@@QAEHPAUtagRECVREQUEST@@@Z$70 0047b9c4 f   MainFrm.obj
 0001:0007a9d0       __unwindfunclet$?HandleLoginRequest@CMainFrame@@QAEHPAUtagRECVREQUEST@@@Z$71 0047b9d0 f   MainFrm.obj
 0001:0007a9dc       __unwindfunclet$?HandleLoginRequest@CMainFrame@@QAEHPAUtagRECVREQUEST@@@Z$72 0047b9dc f   MainFrm.obj
 0001:0007a9e8       __unwindfunclet$?HandleLoginRequest@CMainFrame@@QAEHPAUtagRECVREQUEST@@@Z$73 0047b9e8 f   MainFrm.obj
 0001:0007a9f4       __unwindfunclet$?HandleLoginRequest@CMainFrame@@QAEHPAUtagRECVREQUEST@@@Z$74 0047b9f4 f   MainFrm.obj
 0001:0007aa00       __unwindfunclet$?HandleLoginRequest@CMainFrame@@QAEHPAUtagRECVREQUEST@@@Z$75 0047ba00 f   MainFrm.obj
 0001:0007aa0c       __unwindfunclet$?HandleLoginRequest@CMainFrame@@QAEHPAUtagRECVREQUEST@@@Z$76 0047ba0c f   MainFrm.obj
 0001:0007aa18       __unwindfunclet$?HandleLoginRequest@CMainFrame@@QAEHPAUtagRECVREQUEST@@@Z$77 0047ba18 f   MainFrm.obj
 0001:0007aa24       __unwindfunclet$?HandleLoginRequest@CMainFrame@@QAEHPAUtagRECVREQUEST@@@Z$78 0047ba24 f   MainFrm.obj
 0001:0007aa30       __unwindfunclet$?HandleLoginRequest@CMainFrame@@QAEHPAUtagRECVREQUEST@@@Z$79 0047ba30 f   MainFrm.obj
 0001:0007aa3c       __unwindfunclet$?HandleLoginRequest@CMainFrame@@QAEHPAUtagRECVREQUEST@@@Z$80 0047ba3c f   MainFrm.obj
 0001:0007aa48       __unwindfunclet$?HandleLoginRequest@CMainFrame@@QAEHPAUtagRECVREQUEST@@@Z$81 0047ba48 f   MainFrm.obj
 0001:0007aa54       __unwindfunclet$?HandleLoginRequest@CMainFrame@@QAEHPAUtagRECVREQUEST@@@Z$82 0047ba54 f   MainFrm.obj
 0001:0007aa60       __unwindfunclet$?HandleLoginRequest@CMainFrame@@QAEHPAUtagRECVREQUEST@@@Z$84 0047ba60 f   MainFrm.obj
 0001:0007aa6c       __unwindfunclet$?HandleLoginRequest@CMainFrame@@QAEHPAUtagRECVREQUEST@@@Z$85 0047ba6c f   MainFrm.obj
 0001:0007aa78       __ehhandler$?HandleLoginRequest@CMainFrame@@QAEHPAUtagRECVREQUEST@@@Z 0047ba78 f   MainFrm.obj
 0001:0007aaa0       __unwindfunclet$?InitListCtrlDisplay@CMainFrame@@QAEXXZ$0 0047baa0 f   MainFrm.obj
 0001:0007aaa9       __unwindfunclet$?InitListCtrlDisplay@CMainFrame@@QAEXXZ$2 0047baa9 f   MainFrm.obj
 0001:0007aab2       __unwindfunclet$?InitListCtrlDisplay@CMainFrame@@QAEXXZ$4 0047bab2 f   MainFrm.obj
 0001:0007aabb       __unwindfunclet$?InitListCtrlDisplay@CMainFrame@@QAEXXZ$5 0047babb f   MainFrm.obj
 0001:0007aac4       __unwindfunclet$?InitListCtrlDisplay@CMainFrame@@QAEXXZ$6 0047bac4 f   MainFrm.obj
 0001:0007aacd       __unwindfunclet$?InitListCtrlDisplay@CMainFrame@@QAEXXZ$7 0047bacd f   MainFrm.obj
 0001:0007aad6       __unwindfunclet$?InitListCtrlDisplay@CMainFrame@@QAEXXZ$8 0047bad6 f   MainFrm.obj
 0001:0007aadf       __unwindfunclet$?InitListCtrlDisplay@CMainFrame@@QAEXXZ$9 0047badf f   MainFrm.obj
 0001:0007aae8       __unwindfunclet$?InitListCtrlDisplay@CMainFrame@@QAEXXZ$12 0047bae8 f   MainFrm.obj
 0001:0007aaf1       __unwindfunclet$?InitListCtrlDisplay@CMainFrame@@QAEXXZ$13 0047baf1 f   MainFrm.obj
 0001:0007aafa       __unwindfunclet$?InitListCtrlDisplay@CMainFrame@@QAEXXZ$14 0047bafa f   MainFrm.obj
 0001:0007ab03       __unwindfunclet$?InitListCtrlDisplay@CMainFrame@@QAEXXZ$15 0047bb03 f   MainFrm.obj
 0001:0007ab0c       __unwindfunclet$?InitListCtrlDisplay@CMainFrame@@QAEXXZ$16 0047bb0c f   MainFrm.obj
 0001:0007ab15       __unwindfunclet$?InitListCtrlDisplay@CMainFrame@@QAEXXZ$17 0047bb15 f   MainFrm.obj
 0001:0007ab21       __unwindfunclet$?InitListCtrlDisplay@CMainFrame@@QAEXXZ$18 0047bb21 f   MainFrm.obj
 0001:0007ab2d       __ehhandler$?InitListCtrlDisplay@CMainFrame@@QAEXXZ 0047bb2d f   MainFrm.obj
 0001:0007ab50       __unwindfunclet$?OnWol@CMainFrame@@QAEXXZ$1 0047bb50 f   MainFrm.obj
 0001:0007ab5c       __unwindfunclet$?OnWol@CMainFrame@@QAEXXZ$2 0047bb5c f   MainFrm.obj
 0001:0007ab68       __unwindfunclet$?OnWol@CMainFrame@@QAEXXZ$3 0047bb68 f   MainFrm.obj
 0001:0007ab73       __unwindfunclet$?OnWol@CMainFrame@@QAEXXZ$4 0047bb73 f   MainFrm.obj
 0001:0007ab7f       __unwindfunclet$?OnWol@CMainFrame@@QAEXXZ$5 0047bb7f f   MainFrm.obj
 0001:0007ab8b       __unwindfunclet$?OnWol@CMainFrame@@QAEXXZ$6 0047bb8b f   MainFrm.obj
 0001:0007ab97       __unwindfunclet$?OnWol@CMainFrame@@QAEXXZ$7 0047bb97 f   MainFrm.obj
 0001:0007aba0       __unwindfunclet$?OnWol@CMainFrame@@QAEXXZ$8 0047bba0 f   MainFrm.obj
 0001:0007aba8       __unwindfunclet$?OnWol@CMainFrame@@QAEXXZ$9 0047bba8 f   MainFrm.obj
 0001:0007abb4       __unwindfunclet$?OnWol@CMainFrame@@QAEXXZ$10 0047bbb4 f   MainFrm.obj
 0001:0007abc0       __unwindfunclet$?OnWol@CMainFrame@@QAEXXZ$11 0047bbc0 f   MainFrm.obj
 0001:0007abcc       __ehhandler$?OnWol@CMainFrame@@QAEXXZ 0047bbcc f   MainFrm.obj
 0001:0007ac00       __unwindfunclet$?OnLockmonitor@CMainFrame@@QAEXXZ$1 0047bc00 f   MainFrm.obj
 0001:0007ac00       __unwindfunclet$?OnUnlockusb@CMainFrame@@QAEXXZ$1 0047bc00 f   MainFrm.obj
 0001:0007ac00       __unwindfunclet$?OnUnlockmonitor@CMainFrame@@QAEXXZ$1 0047bc00 f   MainFrm.obj
 0001:0007ac00       __unwindfunclet$?OnLockusb@CMainFrame@@QAEXXZ$1 0047bc00 f   MainFrm.obj
 0001:0007ac0c       __unwindfunclet$?OnLockusb@CMainFrame@@QAEXXZ$2 0047bc0c f   MainFrm.obj
 0001:0007ac0c       __unwindfunclet$?OnUnlockusb@CMainFrame@@QAEXXZ$2 0047bc0c f   MainFrm.obj
 0001:0007ac0c       __unwindfunclet$?OnUnlockmonitor@CMainFrame@@QAEXXZ$2 0047bc0c f   MainFrm.obj
 0001:0007ac0c       __unwindfunclet$?OnLockmonitor@CMainFrame@@QAEXXZ$2 0047bc0c f   MainFrm.obj
 0001:0007ac18       __unwindfunclet$?OnUnlockmonitor@CMainFrame@@QAEXXZ$3 0047bc18 f   MainFrm.obj
 0001:0007ac18       __unwindfunclet$?OnLockmonitor@CMainFrame@@QAEXXZ$3 0047bc18 f   MainFrm.obj
 0001:0007ac18       __unwindfunclet$?OnLockusb@CMainFrame@@QAEXXZ$3 0047bc18 f   MainFrm.obj
 0001:0007ac18       __unwindfunclet$?OnUnlockusb@CMainFrame@@QAEXXZ$3 0047bc18 f   MainFrm.obj
 0001:0007ac21       __unwindfunclet$?OnUnlockmonitor@CMainFrame@@QAEXXZ$4 0047bc21 f   MainFrm.obj
 0001:0007ac21       __unwindfunclet$?OnLockmonitor@CMainFrame@@QAEXXZ$4 0047bc21 f   MainFrm.obj
 0001:0007ac21       __unwindfunclet$?OnLockusb@CMainFrame@@QAEXXZ$4 0047bc21 f   MainFrm.obj
 0001:0007ac21       __unwindfunclet$?OnUnlockusb@CMainFrame@@QAEXXZ$4 0047bc21 f   MainFrm.obj
 0001:0007ac2d       __unwindfunclet$?OnLockusb@CMainFrame@@QAEXXZ$5 0047bc2d f   MainFrm.obj
 0001:0007ac2d       __unwindfunclet$?OnUnlockmonitor@CMainFrame@@QAEXXZ$5 0047bc2d f   MainFrm.obj
 0001:0007ac2d       __unwindfunclet$?OnUnlockusb@CMainFrame@@QAEXXZ$5 0047bc2d f   MainFrm.obj
 0001:0007ac2d       __unwindfunclet$?OnLockmonitor@CMainFrame@@QAEXXZ$5 0047bc2d f   MainFrm.obj
 0001:0007ac39       __unwindfunclet$?OnUnlockusb@CMainFrame@@QAEXXZ$6 0047bc39 f   MainFrm.obj
 0001:0007ac39       __unwindfunclet$?OnLockusb@CMainFrame@@QAEXXZ$6 0047bc39 f   MainFrm.obj
 0001:0007ac39       __unwindfunclet$?OnUnlockmonitor@CMainFrame@@QAEXXZ$6 0047bc39 f   MainFrm.obj
 0001:0007ac39       __unwindfunclet$?OnLockmonitor@CMainFrame@@QAEXXZ$6 0047bc39 f   MainFrm.obj
 0001:0007ac45       __unwindfunclet$?OnLockusb@CMainFrame@@QAEXXZ$7 0047bc45 f   MainFrm.obj
 0001:0007ac45       __unwindfunclet$?OnUnlockmonitor@CMainFrame@@QAEXXZ$7 0047bc45 f   MainFrm.obj
 0001:0007ac45       __unwindfunclet$?OnLockmonitor@CMainFrame@@QAEXXZ$7 0047bc45 f   MainFrm.obj
 0001:0007ac45       __unwindfunclet$?OnUnlockusb@CMainFrame@@QAEXXZ$7 0047bc45 f   MainFrm.obj
 0001:0007ac51       __unwindfunclet$?OnUnlockusb@CMainFrame@@QAEXXZ$8 0047bc51 f   MainFrm.obj
 0001:0007ac51       __unwindfunclet$?OnLockmonitor@CMainFrame@@QAEXXZ$8 0047bc51 f   MainFrm.obj
 0001:0007ac51       __unwindfunclet$?OnLockusb@CMainFrame@@QAEXXZ$8 0047bc51 f   MainFrm.obj
 0001:0007ac51       __unwindfunclet$?OnUnlockmonitor@CMainFrame@@QAEXXZ$8 0047bc51 f   MainFrm.obj
 0001:0007ac5d       __unwindfunclet$?OnLockmonitor@CMainFrame@@QAEXXZ$9 0047bc5d f   MainFrm.obj
 0001:0007ac5d       __unwindfunclet$?OnUnlockusb@CMainFrame@@QAEXXZ$9 0047bc5d f   MainFrm.obj
 0001:0007ac5d       __unwindfunclet$?OnLockusb@CMainFrame@@QAEXXZ$9 0047bc5d f   MainFrm.obj
 0001:0007ac5d       __unwindfunclet$?OnUnlockmonitor@CMainFrame@@QAEXXZ$9 0047bc5d f   MainFrm.obj
 0001:0007ac69       __unwindfunclet$?OnLockmonitor@CMainFrame@@QAEXXZ$10 0047bc69 f   MainFrm.obj
 0001:0007ac69       __unwindfunclet$?OnLockusb@CMainFrame@@QAEXXZ$10 0047bc69 f   MainFrm.obj
 0001:0007ac69       __unwindfunclet$?OnUnlockmonitor@CMainFrame@@QAEXXZ$10 0047bc69 f   MainFrm.obj
 0001:0007ac69       __unwindfunclet$?OnUnlockusb@CMainFrame@@QAEXXZ$10 0047bc69 f   MainFrm.obj
 0001:0007ac75       __unwindfunclet$?OnLockmonitor@CMainFrame@@QAEXXZ$11 0047bc75 f   MainFrm.obj
 0001:0007ac75       __unwindfunclet$?OnUnlockusb@CMainFrame@@QAEXXZ$11 0047bc75 f   MainFrm.obj
 0001:0007ac75       __unwindfunclet$?OnUnlockmonitor@CMainFrame@@QAEXXZ$11 0047bc75 f   MainFrm.obj
 0001:0007ac75       __unwindfunclet$?OnLockusb@CMainFrame@@QAEXXZ$11 0047bc75 f   MainFrm.obj
 0001:0007ac81       __unwindfunclet$?OnUnlockusb@CMainFrame@@QAEXXZ$12 0047bc81 f   MainFrm.obj
 0001:0007ac81       __unwindfunclet$?OnLockmonitor@CMainFrame@@QAEXXZ$12 0047bc81 f   MainFrm.obj
 0001:0007ac81       __unwindfunclet$?OnLockusb@CMainFrame@@QAEXXZ$12 0047bc81 f   MainFrm.obj
 0001:0007ac81       __unwindfunclet$?OnUnlockmonitor@CMainFrame@@QAEXXZ$12 0047bc81 f   MainFrm.obj
 0001:0007ac8d       __unwindfunclet$?OnUnlockmonitor@CMainFrame@@QAEXXZ$13 0047bc8d f   MainFrm.obj
 0001:0007ac8d       __unwindfunclet$?OnUnlockusb@CMainFrame@@QAEXXZ$13 0047bc8d f   MainFrm.obj
 0001:0007ac8d       __unwindfunclet$?OnLockmonitor@CMainFrame@@QAEXXZ$13 0047bc8d f   MainFrm.obj
 0001:0007ac8d       __unwindfunclet$?OnLockusb@CMainFrame@@QAEXXZ$13 0047bc8d f   MainFrm.obj
 0001:0007ac99       __unwindfunclet$?OnUnlockusb@CMainFrame@@QAEXXZ$14 0047bc99 f   MainFrm.obj
 0001:0007ac99       __unwindfunclet$?OnUnlockmonitor@CMainFrame@@QAEXXZ$14 0047bc99 f   MainFrm.obj
 0001:0007ac99       __unwindfunclet$?OnLockmonitor@CMainFrame@@QAEXXZ$14 0047bc99 f   MainFrm.obj
 0001:0007ac99       __unwindfunclet$?OnLockusb@CMainFrame@@QAEXXZ$14 0047bc99 f   MainFrm.obj
 0001:0007aca5       __ehhandler$?OnLockusb@CMainFrame@@QAEXXZ 0047bca5 f   MainFrm.obj
 0001:0007aca5       __ehhandler$?OnUnlockusb@CMainFrame@@QAEXXZ 0047bca5 f   MainFrm.obj
 0001:0007aca5       __ehhandler$?OnLockmonitor@CMainFrame@@QAEXXZ 0047bca5 f   MainFrm.obj
 0001:0007aca5       __ehhandler$?OnUnlockmonitor@CMainFrame@@QAEXXZ 0047bca5 f   MainFrm.obj
 0001:0007acd0       __unwindfunclet$?OnScanclient@CMainFrame@@QAEXXZ$1 0047bcd0 f   MainFrm.obj
 0001:0007acd9       __unwindfunclet$?OnScanclient@CMainFrame@@QAEXXZ$2 0047bcd9 f   MainFrm.obj
 0001:0007ace2       __ehhandler$?OnScanclient@CMainFrame@@QAEXXZ 0047bce2 f   MainFrm.obj
 0001:0007ad00       __unwindfunclet$?_RefreshThread@CMainFrame@@SAIPAX@Z$0 0047bd00 f   MainFrm.obj
 0001:0007ad09       __unwindfunclet$?_RefreshThread@CMainFrame@@SAIPAX@Z$1 0047bd09 f   MainFrm.obj
 0001:0007ad12       __unwindfunclet$?_RefreshThread@CMainFrame@@SAIPAX@Z$2 0047bd12 f   MainFrm.obj
 0001:0007ad1b       __unwindfunclet$?_RefreshThread@CMainFrame@@SAIPAX@Z$3 0047bd1b f   MainFrm.obj
 0001:0007ad24       __unwindfunclet$?_RefreshThread@CMainFrame@@SAIPAX@Z$4 0047bd24 f   MainFrm.obj
 0001:0007ad2d       __unwindfunclet$?_RefreshThread@CMainFrame@@SAIPAX@Z$5 0047bd2d f   MainFrm.obj
 0001:0007ad36       __unwindfunclet$?_RefreshThread@CMainFrame@@SAIPAX@Z$6 0047bd36 f   MainFrm.obj
 0001:0007ad3f       __unwindfunclet$?_RefreshThread@CMainFrame@@SAIPAX@Z$7 0047bd3f f   MainFrm.obj
 0001:0007ad48       __unwindfunclet$?_RefreshThread@CMainFrame@@SAIPAX@Z$8 0047bd48 f   MainFrm.obj
 0001:0007ad51       __unwindfunclet$?_RefreshThread@CMainFrame@@SAIPAX@Z$9 0047bd51 f   MainFrm.obj
 0001:0007ad5a       __unwindfunclet$?_RefreshThread@CMainFrame@@SAIPAX@Z$10 0047bd5a f   MainFrm.obj
 0001:0007ad63       __unwindfunclet$?_RefreshThread@CMainFrame@@SAIPAX@Z$11 0047bd63 f   MainFrm.obj
 0001:0007ad6c       __unwindfunclet$?_RefreshThread@CMainFrame@@SAIPAX@Z$12 0047bd6c f   MainFrm.obj
 0001:0007ad75       __ehhandler$?_RefreshThread@CMainFrame@@SAIPAX@Z 0047bd75 f   MainFrm.obj
 0001:0007ada0       __unwindfunclet$?OnSupervise@CMainFrame@@QAEXXZ$0 0047bda0 f   MainFrm.obj
 0001:0007adac       __unwindfunclet$?OnSupervise@CMainFrame@@QAEXXZ$1 0047bdac f   MainFrm.obj
 0001:0007adb8       __unwindfunclet$?OnSupervise@CMainFrame@@QAEXXZ$3 0047bdb8 f   MainFrm.obj
 0001:0007adc4       __unwindfunclet$?OnSupervise@CMainFrame@@QAEXXZ$4 0047bdc4 f   MainFrm.obj
 0001:0007add0       __unwindfunclet$?OnSupervise@CMainFrame@@QAEXXZ$5 0047bdd0 f   MainFrm.obj
 0001:0007addc       __unwindfunclet$?OnSupervise@CMainFrame@@QAEXXZ$6 0047bddc f   MainFrm.obj
 0001:0007ade8       __unwindfunclet$?OnSupervise@CMainFrame@@QAEXXZ$7 0047bde8 f   MainFrm.obj
 0001:0007adf1       __unwindfunclet$?OnSupervise@CMainFrame@@QAEXXZ$8 0047bdf1 f   MainFrm.obj
 0001:0007adfa       __unwindfunclet$?OnSupervise@CMainFrame@@QAEXXZ$9 0047bdfa f   MainFrm.obj
 0001:0007ae06       __unwindfunclet$?OnSupervise@CMainFrame@@QAEXXZ$10 0047be06 f   MainFrm.obj
 0001:0007ae12       __unwindfunclet$?OnSupervise@CMainFrame@@QAEXXZ$11 0047be12 f   MainFrm.obj
 0001:0007ae1e       __unwindfunclet$?OnSupervise@CMainFrame@@QAEXXZ$12 0047be1e f   MainFrm.obj
 0001:0007ae2a       __unwindfunclet$?OnSupervise@CMainFrame@@QAEXXZ$13 0047be2a f   MainFrm.obj
 0001:0007ae36       __unwindfunclet$?OnSupervise@CMainFrame@@QAEXXZ$14 0047be36 f   MainFrm.obj
 0001:0007ae42       __unwindfunclet$?OnSupervise@CMainFrame@@QAEXXZ$15 0047be42 f   MainFrm.obj
 0001:0007ae4d       __unwindfunclet$?OnSupervise@CMainFrame@@QAEXXZ$18 0047be4d f   MainFrm.obj
 0001:0007ae59       __unwindfunclet$?OnSupervise@CMainFrame@@QAEXXZ$19 0047be59 f   MainFrm.obj
 0001:0007ae65       __unwindfunclet$?OnSupervise@CMainFrame@@QAEXXZ$20 0047be65 f   MainFrm.obj
 0001:0007ae71       __unwindfunclet$?OnSupervise@CMainFrame@@QAEXXZ$21 0047be71 f   MainFrm.obj
 0001:0007ae7d       __unwindfunclet$?OnSupervise@CMainFrame@@QAEXXZ$22 0047be7d f   MainFrm.obj
 0001:0007ae89       __unwindfunclet$?OnSupervise@CMainFrame@@QAEXXZ$23 0047be89 f   MainFrm.obj
 0001:0007ae95       __unwindfunclet$?OnSupervise@CMainFrame@@QAEXXZ$24 0047be95 f   MainFrm.obj
 0001:0007aea1       __unwindfunclet$?OnSupervise@CMainFrame@@QAEXXZ$25 0047bea1 f   MainFrm.obj
 0001:0007aead       __unwindfunclet$?OnSupervise@CMainFrame@@QAEXXZ$26 0047bead f   MainFrm.obj
 0001:0007aeb9       __unwindfunclet$?OnSupervise@CMainFrame@@QAEXXZ$27 0047beb9 f   MainFrm.obj
 0001:0007aec5       __unwindfunclet$?OnSupervise@CMainFrame@@QAEXXZ$28 0047bec5 f   MainFrm.obj
 0001:0007aed1       __unwindfunclet$?OnSupervise@CMainFrame@@QAEXXZ$29 0047bed1 f   MainFrm.obj
 0001:0007aedd       __unwindfunclet$?OnSupervise@CMainFrame@@QAEXXZ$30 0047bedd f   MainFrm.obj
 0001:0007aee9       __unwindfunclet$?OnSupervise@CMainFrame@@QAEXXZ$31 0047bee9 f   MainFrm.obj
 0001:0007aef4       __unwindfunclet$?OnSupervise@CMainFrame@@QAEXXZ$33 0047bef4 f   MainFrm.obj
 0001:0007af00       __unwindfunclet$?OnSupervise@CMainFrame@@QAEXXZ$35 0047bf00 f   MainFrm.obj
 0001:0007af0c       __unwindfunclet$?OnSupervise@CMainFrame@@QAEXXZ$38 0047bf0c f   MainFrm.obj
 0001:0007af18       __unwindfunclet$?OnSupervise@CMainFrame@@QAEXXZ$44 0047bf18 f   MainFrm.obj
 0001:0007af24       __unwindfunclet$?OnSupervise@CMainFrame@@QAEXXZ$45 0047bf24 f   MainFrm.obj
 0001:0007af30       __unwindfunclet$?OnSupervise@CMainFrame@@QAEXXZ$46 0047bf30 f   MainFrm.obj
 0001:0007af3c       __unwindfunclet$?OnSupervise@CMainFrame@@QAEXXZ$47 0047bf3c f   MainFrm.obj
 0001:0007af48       __ehhandler$?OnSupervise@CMainFrame@@QAEXXZ 0047bf48 f   MainFrm.obj
 0001:0007af70       __unwindfunclet$?OnRemotectrl@CMainFrame@@QAEXXZ$0 0047bf70 f   MainFrm.obj
 0001:0007af7c       __unwindfunclet$?OnRemotectrl@CMainFrame@@QAEXXZ$1 0047bf7c f   MainFrm.obj
 0001:0007af88       __unwindfunclet$?OnRemotectrl@CMainFrame@@QAEXXZ$3 0047bf88 f   MainFrm.obj
 0001:0007af94       __unwindfunclet$?OnRemotectrl@CMainFrame@@QAEXXZ$4 0047bf94 f   MainFrm.obj
 0001:0007afa0       __unwindfunclet$?OnRemotectrl@CMainFrame@@QAEXXZ$5 0047bfa0 f   MainFrm.obj
 0001:0007afac       __unwindfunclet$?OnRemotectrl@CMainFrame@@QAEXXZ$6 0047bfac f   MainFrm.obj
 0001:0007afb8       __unwindfunclet$?OnRemotectrl@CMainFrame@@QAEXXZ$7 0047bfb8 f   MainFrm.obj
 0001:0007afc1       __unwindfunclet$?OnRemotectrl@CMainFrame@@QAEXXZ$8 0047bfc1 f   MainFrm.obj
 0001:0007afca       __unwindfunclet$?OnRemotectrl@CMainFrame@@QAEXXZ$9 0047bfca f   MainFrm.obj
 0001:0007afd6       __unwindfunclet$?OnRemotectrl@CMainFrame@@QAEXXZ$10 0047bfd6 f   MainFrm.obj
 0001:0007afe2       __unwindfunclet$?OnRemotectrl@CMainFrame@@QAEXXZ$11 0047bfe2 f   MainFrm.obj
 0001:0007afee       __unwindfunclet$?OnRemotectrl@CMainFrame@@QAEXXZ$12 0047bfee f   MainFrm.obj
 0001:0007affa       __unwindfunclet$?OnRemotectrl@CMainFrame@@QAEXXZ$13 0047bffa f   MainFrm.obj
 0001:0007b006       __unwindfunclet$?OnRemotectrl@CMainFrame@@QAEXXZ$14 0047c006 f   MainFrm.obj
 0001:0007b012       __unwindfunclet$?OnRemotectrl@CMainFrame@@QAEXXZ$15 0047c012 f   MainFrm.obj
 0001:0007b01d       __unwindfunclet$?OnRemotectrl@CMainFrame@@QAEXXZ$18 0047c01d f   MainFrm.obj
 0001:0007b029       __unwindfunclet$?OnRemotectrl@CMainFrame@@QAEXXZ$19 0047c029 f   MainFrm.obj
 0001:0007b035       __unwindfunclet$?OnRemotectrl@CMainFrame@@QAEXXZ$20 0047c035 f   MainFrm.obj
 0001:0007b041       __unwindfunclet$?OnRemotectrl@CMainFrame@@QAEXXZ$21 0047c041 f   MainFrm.obj
 0001:0007b04d       __unwindfunclet$?OnRemotectrl@CMainFrame@@QAEXXZ$22 0047c04d f   MainFrm.obj
 0001:0007b059       __unwindfunclet$?OnRemotectrl@CMainFrame@@QAEXXZ$23 0047c059 f   MainFrm.obj
 0001:0007b065       __unwindfunclet$?OnRemotectrl@CMainFrame@@QAEXXZ$24 0047c065 f   MainFrm.obj
 0001:0007b071       __unwindfunclet$?OnRemotectrl@CMainFrame@@QAEXXZ$25 0047c071 f   MainFrm.obj
 0001:0007b07d       __unwindfunclet$?OnRemotectrl@CMainFrame@@QAEXXZ$26 0047c07d f   MainFrm.obj
 0001:0007b089       __unwindfunclet$?OnRemotectrl@CMainFrame@@QAEXXZ$27 0047c089 f   MainFrm.obj
 0001:0007b095       __unwindfunclet$?OnRemotectrl@CMainFrame@@QAEXXZ$28 0047c095 f   MainFrm.obj
 0001:0007b0a1       __unwindfunclet$?OnRemotectrl@CMainFrame@@QAEXXZ$29 0047c0a1 f   MainFrm.obj
 0001:0007b0ad       __unwindfunclet$?OnRemotectrl@CMainFrame@@QAEXXZ$30 0047c0ad f   MainFrm.obj
 0001:0007b0b9       __unwindfunclet$?OnRemotectrl@CMainFrame@@QAEXXZ$31 0047c0b9 f   MainFrm.obj
 0001:0007b0c4       __unwindfunclet$?OnRemotectrl@CMainFrame@@QAEXXZ$33 0047c0c4 f   MainFrm.obj
 0001:0007b0d0       __unwindfunclet$?OnRemotectrl@CMainFrame@@QAEXXZ$35 0047c0d0 f   MainFrm.obj
 0001:0007b0dc       __unwindfunclet$?OnRemotectrl@CMainFrame@@QAEXXZ$38 0047c0dc f   MainFrm.obj
 0001:0007b0e8       __unwindfunclet$?OnRemotectrl@CMainFrame@@QAEXXZ$44 0047c0e8 f   MainFrm.obj
 0001:0007b0f4       __unwindfunclet$?OnRemotectrl@CMainFrame@@QAEXXZ$45 0047c0f4 f   MainFrm.obj
 0001:0007b100       __unwindfunclet$?OnRemotectrl@CMainFrame@@QAEXXZ$46 0047c100 f   MainFrm.obj
 0001:0007b10c       __unwindfunclet$?OnRemotectrl@CMainFrame@@QAEXXZ$47 0047c10c f   MainFrm.obj
 0001:0007b118       __ehhandler$?OnRemotectrl@CMainFrame@@QAEXXZ 0047c118 f   MainFrm.obj
 0001:0007b140       __unwindfunclet$?OnQuicksave@CMainFrame@@QAEXXZ$1 0047c140 f   MainFrm.obj
 0001:0007b140       __unwindfunclet$?OnQuickrecovery@CMainFrame@@QAEXXZ$1 0047c140 f   MainFrm.obj
 0001:0007b14c       __unwindfunclet$?OnQuickrecovery@CMainFrame@@QAEXXZ$2 0047c14c f   MainFrm.obj
 0001:0007b14c       __unwindfunclet$?OnQuicksave@CMainFrame@@QAEXXZ$2 0047c14c f   MainFrm.obj
 0001:0007b158       __unwindfunclet$?OnQuicksave@CMainFrame@@QAEXXZ$3 0047c158 f   MainFrm.obj
 0001:0007b158       __unwindfunclet$?OnQuickrecovery@CMainFrame@@QAEXXZ$3 0047c158 f   MainFrm.obj
 0001:0007b163       __unwindfunclet$?OnQuicksave@CMainFrame@@QAEXXZ$4 0047c163 f   MainFrm.obj
 0001:0007b163       __unwindfunclet$?OnQuickrecovery@CMainFrame@@QAEXXZ$4 0047c163 f   MainFrm.obj
 0001:0007b16f       __unwindfunclet$?OnQuicksave@CMainFrame@@QAEXXZ$5 0047c16f f   MainFrm.obj
 0001:0007b16f       __unwindfunclet$?OnQuickrecovery@CMainFrame@@QAEXXZ$5 0047c16f f   MainFrm.obj
 0001:0007b17b       __unwindfunclet$?OnQuicksave@CMainFrame@@QAEXXZ$6 0047c17b f   MainFrm.obj
 0001:0007b17b       __unwindfunclet$?OnQuickrecovery@CMainFrame@@QAEXXZ$6 0047c17b f   MainFrm.obj
 0001:0007b187       __unwindfunclet$?OnQuickrecovery@CMainFrame@@QAEXXZ$7 0047c187 f   MainFrm.obj
 0001:0007b187       __unwindfunclet$?OnQuicksave@CMainFrame@@QAEXXZ$7 0047c187 f   MainFrm.obj
 0001:0007b193       __unwindfunclet$?OnQuickrecovery@CMainFrame@@QAEXXZ$8 0047c193 f   MainFrm.obj
 0001:0007b193       __unwindfunclet$?OnQuicksave@CMainFrame@@QAEXXZ$8 0047c193 f   MainFrm.obj
 0001:0007b19f       __unwindfunclet$?OnQuicksave@CMainFrame@@QAEXXZ$9 0047c19f f   MainFrm.obj
 0001:0007b19f       __unwindfunclet$?OnQuickrecovery@CMainFrame@@QAEXXZ$9 0047c19f f   MainFrm.obj
 0001:0007b1ab       __unwindfunclet$?OnQuickrecovery@CMainFrame@@QAEXXZ$10 0047c1ab f   MainFrm.obj
 0001:0007b1ab       __unwindfunclet$?OnQuicksave@CMainFrame@@QAEXXZ$10 0047c1ab f   MainFrm.obj
 0001:0007b1b7       __unwindfunclet$?OnQuicksave@CMainFrame@@QAEXXZ$11 0047c1b7 f   MainFrm.obj
 0001:0007b1b7       __unwindfunclet$?OnQuickrecovery@CMainFrame@@QAEXXZ$11 0047c1b7 f   MainFrm.obj
 0001:0007b1c3       __unwindfunclet$?OnQuickrecovery@CMainFrame@@QAEXXZ$12 0047c1c3 f   MainFrm.obj
 0001:0007b1c3       __unwindfunclet$?OnQuicksave@CMainFrame@@QAEXXZ$12 0047c1c3 f   MainFrm.obj
 0001:0007b1cf       __unwindfunclet$?OnQuickrecovery@CMainFrame@@QAEXXZ$13 0047c1cf f   MainFrm.obj
 0001:0007b1cf       __unwindfunclet$?OnQuicksave@CMainFrame@@QAEXXZ$13 0047c1cf f   MainFrm.obj
 0001:0007b1db       __unwindfunclet$?OnQuicksave@CMainFrame@@QAEXXZ$14 0047c1db f   MainFrm.obj
 0001:0007b1db       __unwindfunclet$?OnQuickrecovery@CMainFrame@@QAEXXZ$14 0047c1db f   MainFrm.obj
 0001:0007b1e7       __ehhandler$?OnQuicksave@CMainFrame@@QAEXXZ 0047c1e7 f   MainFrm.obj
 0001:0007b1e7       __ehhandler$?OnQuickrecovery@CMainFrame@@QAEXXZ 0047c1e7 f   MainFrm.obj
 0001:0007b220       __unwindfunclet$?OnStarttrans@CMainFrame@@QAEXXZ$1 0047c220 f   MainFrm.obj
 0001:0007b220       __unwindfunclet$?OnRestart@CMainFrame@@QAEXXZ$1 0047c220 f   MainFrm.obj
 0001:0007b220       __unwindfunclet$?OnShutdown@CMainFrame@@QAEXXZ$1 0047c220 f   MainFrm.obj
 0001:0007b22c       __unwindfunclet$?OnRestart@CMainFrame@@QAEXXZ$2 0047c22c f   MainFrm.obj
 0001:0007b22c       __unwindfunclet$?OnStarttrans@CMainFrame@@QAEXXZ$2 0047c22c f   MainFrm.obj
 0001:0007b22c       __unwindfunclet$?OnShutdown@CMainFrame@@QAEXXZ$2 0047c22c f   MainFrm.obj
 0001:0007b238       __unwindfunclet$?OnRestart@CMainFrame@@QAEXXZ$3 0047c238 f   MainFrm.obj
 0001:0007b238       __unwindfunclet$?OnShutdown@CMainFrame@@QAEXXZ$3 0047c238 f   MainFrm.obj
 0001:0007b238       __unwindfunclet$?OnStarttrans@CMainFrame@@QAEXXZ$3 0047c238 f   MainFrm.obj
 0001:0007b243       __unwindfunclet$?OnRestart@CMainFrame@@QAEXXZ$4 0047c243 f   MainFrm.obj
 0001:0007b243       __unwindfunclet$?OnStarttrans@CMainFrame@@QAEXXZ$4 0047c243 f   MainFrm.obj
 0001:0007b243       __unwindfunclet$?OnShutdown@CMainFrame@@QAEXXZ$4 0047c243 f   MainFrm.obj
 0001:0007b24f       __unwindfunclet$?OnShutdown@CMainFrame@@QAEXXZ$5 0047c24f f   MainFrm.obj
 0001:0007b24f       __unwindfunclet$?OnStarttrans@CMainFrame@@QAEXXZ$5 0047c24f f   MainFrm.obj
 0001:0007b24f       __unwindfunclet$?OnRestart@CMainFrame@@QAEXXZ$5 0047c24f f   MainFrm.obj
 0001:0007b25b       __unwindfunclet$?OnStarttrans@CMainFrame@@QAEXXZ$6 0047c25b f   MainFrm.obj
 0001:0007b25b       __unwindfunclet$?OnShutdown@CMainFrame@@QAEXXZ$6 0047c25b f   MainFrm.obj
 0001:0007b25b       __unwindfunclet$?OnRestart@CMainFrame@@QAEXXZ$6 0047c25b f   MainFrm.obj
 0001:0007b267       __unwindfunclet$?OnShutdown@CMainFrame@@QAEXXZ$7 0047c267 f   MainFrm.obj
 0001:0007b267       __unwindfunclet$?OnStarttrans@CMainFrame@@QAEXXZ$7 0047c267 f   MainFrm.obj
 0001:0007b267       __unwindfunclet$?OnRestart@CMainFrame@@QAEXXZ$7 0047c267 f   MainFrm.obj
 0001:0007b273       __unwindfunclet$?OnStarttrans@CMainFrame@@QAEXXZ$8 0047c273 f   MainFrm.obj
 0001:0007b273       __unwindfunclet$?OnRestart@CMainFrame@@QAEXXZ$8 0047c273 f   MainFrm.obj
 0001:0007b273       __unwindfunclet$?OnShutdown@CMainFrame@@QAEXXZ$8 0047c273 f   MainFrm.obj
 0001:0007b27f       __unwindfunclet$?OnRestart@CMainFrame@@QAEXXZ$9 0047c27f f   MainFrm.obj
 0001:0007b27f       __unwindfunclet$?OnShutdown@CMainFrame@@QAEXXZ$9 0047c27f f   MainFrm.obj
 0001:0007b27f       __unwindfunclet$?OnStarttrans@CMainFrame@@QAEXXZ$9 0047c27f f   MainFrm.obj
 0001:0007b28b       __unwindfunclet$?OnShutdown@CMainFrame@@QAEXXZ$10 0047c28b f   MainFrm.obj
 0001:0007b28b       __unwindfunclet$?OnRestart@CMainFrame@@QAEXXZ$10 0047c28b f   MainFrm.obj
 0001:0007b28b       __unwindfunclet$?OnStarttrans@CMainFrame@@QAEXXZ$10 0047c28b f   MainFrm.obj
 0001:0007b297       __unwindfunclet$?OnStarttrans@CMainFrame@@QAEXXZ$11 0047c297 f   MainFrm.obj
 0001:0007b297       __unwindfunclet$?OnRestart@CMainFrame@@QAEXXZ$11 0047c297 f   MainFrm.obj
 0001:0007b297       __unwindfunclet$?OnShutdown@CMainFrame@@QAEXXZ$11 0047c297 f   MainFrm.obj
 0001:0007b2a3       __unwindfunclet$?OnStarttrans@CMainFrame@@QAEXXZ$12 0047c2a3 f   MainFrm.obj
 0001:0007b2a3       __unwindfunclet$?OnRestart@CMainFrame@@QAEXXZ$12 0047c2a3 f   MainFrm.obj
 0001:0007b2a3       __unwindfunclet$?OnShutdown@CMainFrame@@QAEXXZ$12 0047c2a3 f   MainFrm.obj
 0001:0007b2af       __unwindfunclet$?OnStarttrans@CMainFrame@@QAEXXZ$13 0047c2af f   MainFrm.obj
 0001:0007b2af       __unwindfunclet$?OnShutdown@CMainFrame@@QAEXXZ$13 0047c2af f   MainFrm.obj
 0001:0007b2af       __unwindfunclet$?OnRestart@CMainFrame@@QAEXXZ$13 0047c2af f   MainFrm.obj
 0001:0007b2bb       __unwindfunclet$?OnStarttrans@CMainFrame@@QAEXXZ$14 0047c2bb f   MainFrm.obj
 0001:0007b2bb       __unwindfunclet$?OnShutdown@CMainFrame@@QAEXXZ$14 0047c2bb f   MainFrm.obj
 0001:0007b2bb       __unwindfunclet$?OnRestart@CMainFrame@@QAEXXZ$14 0047c2bb f   MainFrm.obj
 0001:0007b2c7       __ehhandler$?OnShutdown@CMainFrame@@QAEXXZ 0047c2c7 f   MainFrm.obj
 0001:0007b2c7       __ehhandler$?OnStarttrans@CMainFrame@@QAEXXZ 0047c2c7 f   MainFrm.obj
 0001:0007b2c7       __ehhandler$?OnRestart@CMainFrame@@QAEXXZ 0047c2c7 f   MainFrm.obj
 0001:0007b300       __unwindfunclet$?OnSpecialSave@CMainFrame@@QAEXXZ$1 0047c300 f   MainFrm.obj
 0001:0007b300       __unwindfunclet$?OnClientsettings@CMainFrame@@QAEXXZ$1 0047c300 f   MainFrm.obj
 0001:0007b300       __unwindfunclet$?OnSpecialRecovery@CMainFrame@@QAEXXZ$1 0047c300 f   MainFrm.obj
 0001:0007b309       __unwindfunclet$?OnSpecialSave@CMainFrame@@QAEXXZ$2 0047c309 f   MainFrm.obj
 0001:0007b309       __unwindfunclet$?OnClientsettings@CMainFrame@@QAEXXZ$2 0047c309 f   MainFrm.obj
 0001:0007b309       __unwindfunclet$?OnSpecialRecovery@CMainFrame@@QAEXXZ$2 0047c309 f   MainFrm.obj
 0001:0007b312       __unwindfunclet$?OnSpecialSave@CMainFrame@@QAEXXZ$3 0047c312 f   MainFrm.obj
 0001:0007b312       __unwindfunclet$?OnSpecialRecovery@CMainFrame@@QAEXXZ$3 0047c312 f   MainFrm.obj
 0001:0007b312       __unwindfunclet$?OnClientsettings@CMainFrame@@QAEXXZ$3 0047c312 f   MainFrm.obj
 0001:0007b31b       __ehhandler$?OnSpecialSave@CMainFrame@@QAEXXZ 0047c31b f   MainFrm.obj
 0001:0007b31b       __ehhandler$?OnSpecialRecovery@CMainFrame@@QAEXXZ 0047c31b f   MainFrm.obj
 0001:0007b31b       __ehhandler$?OnClientsettings@CMainFrame@@QAEXXZ 0047c31b f   MainFrm.obj
 0001:0007b340       __unwindfunclet$?_GetBootModuleInfoThread@CMainFrame@@SAIPAX@Z$0 0047c340 f   MainFrm.obj
 0001:0007b34c       __unwindfunclet$?_GetBootModuleInfoThread@CMainFrame@@SAIPAX@Z$1 0047c34c f   MainFrm.obj
 0001:0007b358       __unwindfunclet$?_GetBootModuleInfoThread@CMainFrame@@SAIPAX@Z$2 0047c358 f   MainFrm.obj
 0001:0007b364       __ehhandler$?_GetBootModuleInfoThread@CMainFrame@@SAIPAX@Z 0047c364 f   MainFrm.obj
 0001:0007b390       __unwindfunclet$?_WaitAllThreadExited@CMainFrame@@SAIPAX@Z$0 0047c390 f   MainFrm.obj
 0001:0007b399       __unwindfunclet$?_WaitAllThreadExited@CMainFrame@@SAIPAX@Z$3 0047c399 f   MainFrm.obj
 0001:0007b3a2       __unwindfunclet$?_WaitAllThreadExited@CMainFrame@@SAIPAX@Z$4 0047c3a2 f   MainFrm.obj
 0001:0007b3ab       __unwindfunclet$?_WaitAllThreadExited@CMainFrame@@SAIPAX@Z$9 0047c3ab f   MainFrm.obj
 0001:0007b3b4       __ehhandler$?_WaitAllThreadExited@CMainFrame@@SAIPAX@Z 0047c3b4 f   MainFrm.obj
 0001:0007b3e0       __unwindfunclet$?OnSendmsg@CMainFrame@@QAEXXZ$1 0047c3e0 f   MainFrm.obj
 0001:0007b3ec       __unwindfunclet$?OnSendmsg@CMainFrame@@QAEXXZ$2 0047c3ec f   MainFrm.obj
 0001:0007b3f8       __unwindfunclet$?OnSendmsg@CMainFrame@@QAEXXZ$3 0047c3f8 f   MainFrm.obj
 0001:0007b401       __unwindfunclet$?OnSendmsg@CMainFrame@@QAEXXZ$4 0047c401 f   MainFrm.obj
 0001:0007b40d       __unwindfunclet$?OnSendmsg@CMainFrame@@QAEXXZ$5 0047c40d f   MainFrm.obj
 0001:0007b419       __unwindfunclet$?OnSendmsg@CMainFrame@@QAEXXZ$6 0047c419 f   MainFrm.obj
 0001:0007b425       __unwindfunclet$?OnSendmsg@CMainFrame@@QAEXXZ$7 0047c425 f   MainFrm.obj
 0001:0007b431       __unwindfunclet$?OnSendmsg@CMainFrame@@QAEXXZ$8 0047c431 f   MainFrm.obj
 0001:0007b43d       __unwindfunclet$?OnSendmsg@CMainFrame@@QAEXXZ$9 0047c43d f   MainFrm.obj
 0001:0007b449       __unwindfunclet$?OnSendmsg@CMainFrame@@QAEXXZ$10 0047c449 f   MainFrm.obj
 0001:0007b455       __unwindfunclet$?OnSendmsg@CMainFrame@@QAEXXZ$11 0047c455 f   MainFrm.obj
 0001:0007b460       __unwindfunclet$?OnSendmsg@CMainFrame@@QAEXXZ$12 0047c460 f   MainFrm.obj
 0001:0007b46c       __ehhandler$?OnSendmsg@CMainFrame@@QAEXXZ 0047c46c f   MainFrm.obj
 0001:0007b490       __unwindfunclet$?OnIpsettings@CMainFrame@@QAEXXZ$1 0047c490 f   MainFrm.obj
 0001:0007b49c       __unwindfunclet$?OnIpsettings@CMainFrame@@QAEXXZ$2 0047c49c f   MainFrm.obj
 0001:0007b4a8       __unwindfunclet$?OnIpsettings@CMainFrame@@QAEXXZ$3 0047c4a8 f   MainFrm.obj
 0001:0007b4b1       __unwindfunclet$?OnIpsettings@CMainFrame@@QAEXXZ$4 0047c4b1 f   MainFrm.obj
 0001:0007b4bd       __unwindfunclet$?OnIpsettings@CMainFrame@@QAEXXZ$5 0047c4bd f   MainFrm.obj
 0001:0007b4c9       __unwindfunclet$?OnIpsettings@CMainFrame@@QAEXXZ$6 0047c4c9 f   MainFrm.obj
 0001:0007b4d5       __unwindfunclet$?OnIpsettings@CMainFrame@@QAEXXZ$7 0047c4d5 f   MainFrm.obj
 0001:0007b4e1       __unwindfunclet$?OnIpsettings@CMainFrame@@QAEXXZ$8 0047c4e1 f   MainFrm.obj
 0001:0007b4ed       __unwindfunclet$?OnIpsettings@CMainFrame@@QAEXXZ$9 0047c4ed f   MainFrm.obj
 0001:0007b4f9       __unwindfunclet$?OnIpsettings@CMainFrame@@QAEXXZ$10 0047c4f9 f   MainFrm.obj
 0001:0007b505       __unwindfunclet$?OnIpsettings@CMainFrame@@QAEXXZ$11 0047c505 f   MainFrm.obj
 0001:0007b511       __unwindfunclet$?OnIpsettings@CMainFrame@@QAEXXZ$12 0047c511 f   MainFrm.obj
 0001:0007b51d       __unwindfunclet$?OnIpsettings@CMainFrame@@QAEXXZ$14 0047c51d f   MainFrm.obj
 0001:0007b526       __unwindfunclet$?OnIpsettings@CMainFrame@@QAEXXZ$15 0047c526 f   MainFrm.obj
 0001:0007b532       __ehhandler$?OnIpsettings@CMainFrame@@QAEXXZ 0047c532 f   MainFrm.obj
 0001:0007b560       __unwindfunclet$?GetHostBasicIPInfo@CMainFrame@@QAEHAAUstruct_ipsetting_param@@@Z$0 0047c560 f   MainFrm.obj
 0001:0007b56c       __unwindfunclet$?GetHostBasicIPInfo@CMainFrame@@QAEHAAUstruct_ipsetting_param@@@Z$1 0047c56c f   MainFrm.obj
 0001:0007b578       __unwindfunclet$?GetHostBasicIPInfo@CMainFrame@@QAEHAAUstruct_ipsetting_param@@@Z$2 0047c578 f   MainFrm.obj
 0001:0007b584       __unwindfunclet$?GetHostBasicIPInfo@CMainFrame@@QAEHAAUstruct_ipsetting_param@@@Z$3 0047c584 f   MainFrm.obj
 0001:0007b58d       __unwindfunclet$?GetHostBasicIPInfo@CMainFrame@@QAEHAAUstruct_ipsetting_param@@@Z$4 0047c58d f   MainFrm.obj
 0001:0007b596       __unwindfunclet$?GetHostBasicIPInfo@CMainFrame@@QAEHAAUstruct_ipsetting_param@@@Z$5 0047c596 f   MainFrm.obj
 0001:0007b59f       __unwindfunclet$?GetHostBasicIPInfo@CMainFrame@@QAEHAAUstruct_ipsetting_param@@@Z$6 0047c59f f   MainFrm.obj
 0001:0007b5ab       __unwindfunclet$?GetHostBasicIPInfo@CMainFrame@@QAEHAAUstruct_ipsetting_param@@@Z$7 0047c5ab f   MainFrm.obj
 0001:0007b5b7       __unwindfunclet$?GetHostBasicIPInfo@CMainFrame@@QAEHAAUstruct_ipsetting_param@@@Z$8 0047c5b7 f   MainFrm.obj
 0001:0007b5c3       __unwindfunclet$?GetHostBasicIPInfo@CMainFrame@@QAEHAAUstruct_ipsetting_param@@@Z$9 0047c5c3 f   MainFrm.obj
 0001:0007b5cf       __unwindfunclet$?GetHostBasicIPInfo@CMainFrame@@QAEHAAUstruct_ipsetting_param@@@Z$10 0047c5cf f   MainFrm.obj
 0001:0007b5da       __unwindfunclet$?GetHostBasicIPInfo@CMainFrame@@QAEHAAUstruct_ipsetting_param@@@Z$11 0047c5da f   MainFrm.obj
 0001:0007b5e3       __unwindfunclet$?GetHostBasicIPInfo@CMainFrame@@QAEHAAUstruct_ipsetting_param@@@Z$12 0047c5e3 f   MainFrm.obj
 0001:0007b5ee       __unwindfunclet$?GetHostBasicIPInfo@CMainFrame@@QAEHAAUstruct_ipsetting_param@@@Z$14 0047c5ee f   MainFrm.obj
 0001:0007b5fa       __unwindfunclet$?GetHostBasicIPInfo@CMainFrame@@QAEHAAUstruct_ipsetting_param@@@Z$16 0047c5fa f   MainFrm.obj
 0001:0007b606       __unwindfunclet$?GetHostBasicIPInfo@CMainFrame@@QAEHAAUstruct_ipsetting_param@@@Z$17 0047c606 f   MainFrm.obj
 0001:0007b612       __unwindfunclet$?GetHostBasicIPInfo@CMainFrame@@QAEHAAUstruct_ipsetting_param@@@Z$18 0047c612 f   MainFrm.obj
 0001:0007b61d       __unwindfunclet$?GetHostBasicIPInfo@CMainFrame@@QAEHAAUstruct_ipsetting_param@@@Z$19 0047c61d f   MainFrm.obj
 0001:0007b629       __unwindfunclet$?GetHostBasicIPInfo@CMainFrame@@QAEHAAUstruct_ipsetting_param@@@Z$20 0047c629 f   MainFrm.obj
 0001:0007b635       __unwindfunclet$?GetHostBasicIPInfo@CMainFrame@@QAEHAAUstruct_ipsetting_param@@@Z$25 0047c635 f   MainFrm.obj
 0001:0007b641       __unwindfunclet$?GetHostBasicIPInfo@CMainFrame@@QAEHAAUstruct_ipsetting_param@@@Z$27 0047c641 f   MainFrm.obj
 0001:0007b64d       __unwindfunclet$?GetHostBasicIPInfo@CMainFrame@@QAEHAAUstruct_ipsetting_param@@@Z$28 0047c64d f   MainFrm.obj
 0001:0007b659       __unwindfunclet$?GetHostBasicIPInfo@CMainFrame@@QAEHAAUstruct_ipsetting_param@@@Z$30 0047c659 f   MainFrm.obj
 0001:0007b665       __unwindfunclet$?GetHostBasicIPInfo@CMainFrame@@QAEHAAUstruct_ipsetting_param@@@Z$31 0047c665 f   MainFrm.obj
 0001:0007b671       __unwindfunclet$?GetHostBasicIPInfo@CMainFrame@@QAEHAAUstruct_ipsetting_param@@@Z$32 0047c671 f   MainFrm.obj
 0001:0007b67d       __unwindfunclet$?GetHostBasicIPInfo@CMainFrame@@QAEHAAUstruct_ipsetting_param@@@Z$33 0047c67d f   MainFrm.obj
 0001:0007b689       __unwindfunclet$?GetHostBasicIPInfo@CMainFrame@@QAEHAAUstruct_ipsetting_param@@@Z$34 0047c689 f   MainFrm.obj
 0001:0007b695       __unwindfunclet$?GetHostBasicIPInfo@CMainFrame@@QAEHAAUstruct_ipsetting_param@@@Z$35 0047c695 f   MainFrm.obj
 0001:0007b6a1       __unwindfunclet$?GetHostBasicIPInfo@CMainFrame@@QAEHAAUstruct_ipsetting_param@@@Z$36 0047c6a1 f   MainFrm.obj
 0001:0007b6ad       __ehhandler$?GetHostBasicIPInfo@CMainFrame@@QAEHAAUstruct_ipsetting_param@@@Z 0047c6ad f   MainFrm.obj
 0001:0007b6e0       __unwindfunclet$?OnScanproperty@CMainFrame@@QAEXXZ$1 0047c6e0 f   MainFrm.obj
 0001:0007b6e9       __unwindfunclet$?OnScanproperty@CMainFrame@@QAEXXZ$2 0047c6e9 f   MainFrm.obj
 0001:0007b6f2       __unwindfunclet$?OnScanproperty@CMainFrame@@QAEXXZ$3 0047c6f2 f   MainFrm.obj
 0001:0007b6fb       __unwindfunclet$?OnScanproperty@CMainFrame@@QAEXXZ$4 0047c6fb f   MainFrm.obj
 0001:0007b704       __ehhandler$?OnScanproperty@CMainFrame@@QAEXXZ 0047c704 f   MainFrm.obj
 0001:0007b720       __unwindfunclet$?_PropertyCheckThread@CMainFrame@@SAIPAX@Z$0 0047c720 f   MainFrm.obj
 0001:0007b72c       __ehhandler$?_PropertyCheckThread@CMainFrame@@SAIPAX@Z 0047c72c f   MainFrm.obj
 0001:0007b760       __unwindfunclet$?OnUpdateproperty@CMainFrame@@QAEXXZ$1 0047c760 f   MainFrm.obj
 0001:0007b76c       __unwindfunclet$?OnUpdateproperty@CMainFrame@@QAEXXZ$2 0047c76c f   MainFrm.obj
 0001:0007b778       __unwindfunclet$?OnUpdateproperty@CMainFrame@@QAEXXZ$3 0047c778 f   MainFrm.obj
 0001:0007b784       __unwindfunclet$?OnUpdateproperty@CMainFrame@@QAEXXZ$4 0047c784 f   MainFrm.obj
 0001:0007b790       __unwindfunclet$?OnUpdateproperty@CMainFrame@@QAEXXZ$5 0047c790 f   MainFrm.obj
 0001:0007b79b       __unwindfunclet$?OnUpdateproperty@CMainFrame@@QAEXXZ$6 0047c79b f   MainFrm.obj
 0001:0007b7a7       __unwindfunclet$?OnUpdateproperty@CMainFrame@@QAEXXZ$7 0047c7a7 f   MainFrm.obj
 0001:0007b7b3       __unwindfunclet$?OnUpdateproperty@CMainFrame@@QAEXXZ$8 0047c7b3 f   MainFrm.obj
 0001:0007b7bf       __ehhandler$?OnUpdateproperty@CMainFrame@@QAEXXZ 0047c7bf f   MainFrm.obj
 0001:0007b7e0       __unwindfunclet$?_PropertyUpdateThread@CMainFrame@@SAIPAX@Z$0 0047c7e0 f   MainFrm.obj
 0001:0007b7e9       __unwindfunclet$?_PropertyUpdateThread@CMainFrame@@SAIPAX@Z$1 0047c7e9 f   MainFrm.obj
 0001:0007b7f2       __unwindfunclet$?_PropertyUpdateThread@CMainFrame@@SAIPAX@Z$3 0047c7f2 f   MainFrm.obj
 0001:0007b7fb       __ehhandler$?_PropertyUpdateThread@CMainFrame@@SAIPAX@Z 0047c7fb f   MainFrm.obj
 0001:0007b820       __unwindfunclet$?UpdateOnePropertyInfoInDatabase@CMainFrame@@QAEHV?$CStringT@DV?$StrTraitMFC_DLL@DV?$ChTraitsCRT@D@ATL@@@@@ATL@@@Z$0 0047c820 f   MainFrm.obj
 0001:0007b829       __unwindfunclet$?UpdateOnePropertyInfoInDatabase@CMainFrame@@QAEHV?$CStringT@DV?$StrTraitMFC_DLL@DV?$ChTraitsCRT@D@ATL@@@@@ATL@@@Z$1 0047c829 f   MainFrm.obj
 0001:0007b831       __unwindfunclet$?UpdateOnePropertyInfoInDatabase@CMainFrame@@QAEHV?$CStringT@DV?$StrTraitMFC_DLL@DV?$ChTraitsCRT@D@ATL@@@@@ATL@@@Z$2 0047c831 f   MainFrm.obj
 0001:0007b83d       __unwindfunclet$?UpdateOnePropertyInfoInDatabase@CMainFrame@@QAEHV?$CStringT@DV?$StrTraitMFC_DLL@DV?$ChTraitsCRT@D@ATL@@@@@ATL@@@Z$3 0047c83d f   MainFrm.obj
 0001:0007b849       __unwindfunclet$?UpdateOnePropertyInfoInDatabase@CMainFrame@@QAEHV?$CStringT@DV?$StrTraitMFC_DLL@DV?$ChTraitsCRT@D@ATL@@@@@ATL@@@Z$4 0047c849 f   MainFrm.obj
 0001:0007b852       __unwindfunclet$?UpdateOnePropertyInfoInDatabase@CMainFrame@@QAEHV?$CStringT@DV?$StrTraitMFC_DLL@DV?$ChTraitsCRT@D@ATL@@@@@ATL@@@Z$5 0047c852 f   MainFrm.obj
 0001:0007b85e       __unwindfunclet$?UpdateOnePropertyInfoInDatabase@CMainFrame@@QAEHV?$CStringT@DV?$StrTraitMFC_DLL@DV?$ChTraitsCRT@D@ATL@@@@@ATL@@@Z$7 0047c85e f   MainFrm.obj
 0001:0007b86a       __unwindfunclet$?UpdateOnePropertyInfoInDatabase@CMainFrame@@QAEHV?$CStringT@DV?$StrTraitMFC_DLL@DV?$ChTraitsCRT@D@ATL@@@@@ATL@@@Z$8 0047c86a f   MainFrm.obj
 0001:0007b876       __unwindfunclet$?UpdateOnePropertyInfoInDatabase@CMainFrame@@QAEHV?$CStringT@DV?$StrTraitMFC_DLL@DV?$ChTraitsCRT@D@ATL@@@@@ATL@@@Z$9 0047c876 f   MainFrm.obj
 0001:0007b882       __unwindfunclet$?UpdateOnePropertyInfoInDatabase@CMainFrame@@QAEHV?$CStringT@DV?$StrTraitMFC_DLL@DV?$ChTraitsCRT@D@ATL@@@@@ATL@@@Z$10 0047c882 f   MainFrm.obj
 0001:0007b88e       __unwindfunclet$?UpdateOnePropertyInfoInDatabase@CMainFrame@@QAEHV?$CStringT@DV?$StrTraitMFC_DLL@DV?$ChTraitsCRT@D@ATL@@@@@ATL@@@Z$11 0047c88e f   MainFrm.obj
 0001:0007b89a       __unwindfunclet$?UpdateOnePropertyInfoInDatabase@CMainFrame@@QAEHV?$CStringT@DV?$StrTraitMFC_DLL@DV?$ChTraitsCRT@D@ATL@@@@@ATL@@@Z$12 0047c89a f   MainFrm.obj
 0001:0007b8a6       __unwindfunclet$?UpdateOnePropertyInfoInDatabase@CMainFrame@@QAEHV?$CStringT@DV?$StrTraitMFC_DLL@DV?$ChTraitsCRT@D@ATL@@@@@ATL@@@Z$13 0047c8a6 f   MainFrm.obj
 0001:0007b8b2       __unwindfunclet$?UpdateOnePropertyInfoInDatabase@CMainFrame@@QAEHV?$CStringT@DV?$StrTraitMFC_DLL@DV?$ChTraitsCRT@D@ATL@@@@@ATL@@@Z$14 0047c8b2 f   MainFrm.obj
 0001:0007b8be       __unwindfunclet$?UpdateOnePropertyInfoInDatabase@CMainFrame@@QAEHV?$CStringT@DV?$StrTraitMFC_DLL@DV?$ChTraitsCRT@D@ATL@@@@@ATL@@@Z$15 0047c8be f   MainFrm.obj
 0001:0007b8ca       __unwindfunclet$?UpdateOnePropertyInfoInDatabase@CMainFrame@@QAEHV?$CStringT@DV?$StrTraitMFC_DLL@DV?$ChTraitsCRT@D@ATL@@@@@ATL@@@Z$16 0047c8ca f   MainFrm.obj
 0001:0007b8d6       __unwindfunclet$?UpdateOnePropertyInfoInDatabase@CMainFrame@@QAEHV?$CStringT@DV?$StrTraitMFC_DLL@DV?$ChTraitsCRT@D@ATL@@@@@ATL@@@Z$17 0047c8d6 f   MainFrm.obj
 0001:0007b8e2       __unwindfunclet$?UpdateOnePropertyInfoInDatabase@CMainFrame@@QAEHV?$CStringT@DV?$StrTraitMFC_DLL@DV?$ChTraitsCRT@D@ATL@@@@@ATL@@@Z$18 0047c8e2 f   MainFrm.obj
 0001:0007b8ee       __unwindfunclet$?UpdateOnePropertyInfoInDatabase@CMainFrame@@QAEHV?$CStringT@DV?$StrTraitMFC_DLL@DV?$ChTraitsCRT@D@ATL@@@@@ATL@@@Z$19 0047c8ee f   MainFrm.obj
 0001:0007b8fa       __unwindfunclet$?UpdateOnePropertyInfoInDatabase@CMainFrame@@QAEHV?$CStringT@DV?$StrTraitMFC_DLL@DV?$ChTraitsCRT@D@ATL@@@@@ATL@@@Z$20 0047c8fa f   MainFrm.obj
 0001:0007b906       __unwindfunclet$?UpdateOnePropertyInfoInDatabase@CMainFrame@@QAEHV?$CStringT@DV?$StrTraitMFC_DLL@DV?$ChTraitsCRT@D@ATL@@@@@ATL@@@Z$21 0047c906 f   MainFrm.obj
 0001:0007b912       __unwindfunclet$?UpdateOnePropertyInfoInDatabase@CMainFrame@@QAEHV?$CStringT@DV?$StrTraitMFC_DLL@DV?$ChTraitsCRT@D@ATL@@@@@ATL@@@Z$22 0047c912 f   MainFrm.obj
 0001:0007b91e       __unwindfunclet$?UpdateOnePropertyInfoInDatabase@CMainFrame@@QAEHV?$CStringT@DV?$StrTraitMFC_DLL@DV?$ChTraitsCRT@D@ATL@@@@@ATL@@@Z$23 0047c91e f   MainFrm.obj
 0001:0007b92a       __unwindfunclet$?UpdateOnePropertyInfoInDatabase@CMainFrame@@QAEHV?$CStringT@DV?$StrTraitMFC_DLL@DV?$ChTraitsCRT@D@ATL@@@@@ATL@@@Z$24 0047c92a f   MainFrm.obj
 0001:0007b936       __unwindfunclet$?UpdateOnePropertyInfoInDatabase@CMainFrame@@QAEHV?$CStringT@DV?$StrTraitMFC_DLL@DV?$ChTraitsCRT@D@ATL@@@@@ATL@@@Z$25 0047c936 f   MainFrm.obj
 0001:0007b942       __unwindfunclet$?UpdateOnePropertyInfoInDatabase@CMainFrame@@QAEHV?$CStringT@DV?$StrTraitMFC_DLL@DV?$ChTraitsCRT@D@ATL@@@@@ATL@@@Z$26 0047c942 f   MainFrm.obj
 0001:0007b94e       __unwindfunclet$?UpdateOnePropertyInfoInDatabase@CMainFrame@@QAEHV?$CStringT@DV?$StrTraitMFC_DLL@DV?$ChTraitsCRT@D@ATL@@@@@ATL@@@Z$27 0047c94e f   MainFrm.obj
 0001:0007b95a       __unwindfunclet$?UpdateOnePropertyInfoInDatabase@CMainFrame@@QAEHV?$CStringT@DV?$StrTraitMFC_DLL@DV?$ChTraitsCRT@D@ATL@@@@@ATL@@@Z$28 0047c95a f   MainFrm.obj
 0001:0007b966       __unwindfunclet$?UpdateOnePropertyInfoInDatabase@CMainFrame@@QAEHV?$CStringT@DV?$StrTraitMFC_DLL@DV?$ChTraitsCRT@D@ATL@@@@@ATL@@@Z$29 0047c966 f   MainFrm.obj
 0001:0007b972       __unwindfunclet$?UpdateOnePropertyInfoInDatabase@CMainFrame@@QAEHV?$CStringT@DV?$StrTraitMFC_DLL@DV?$ChTraitsCRT@D@ATL@@@@@ATL@@@Z$30 0047c972 f   MainFrm.obj
 0001:0007b97e       __unwindfunclet$?UpdateOnePropertyInfoInDatabase@CMainFrame@@QAEHV?$CStringT@DV?$StrTraitMFC_DLL@DV?$ChTraitsCRT@D@ATL@@@@@ATL@@@Z$31 0047c97e f   MainFrm.obj
 0001:0007b98a       __unwindfunclet$?UpdateOnePropertyInfoInDatabase@CMainFrame@@QAEHV?$CStringT@DV?$StrTraitMFC_DLL@DV?$ChTraitsCRT@D@ATL@@@@@ATL@@@Z$32 0047c98a f   MainFrm.obj
 0001:0007b996       __unwindfunclet$?UpdateOnePropertyInfoInDatabase@CMainFrame@@QAEHV?$CStringT@DV?$StrTraitMFC_DLL@DV?$ChTraitsCRT@D@ATL@@@@@ATL@@@Z$33 0047c996 f   MainFrm.obj
 0001:0007b9a2       __unwindfunclet$?UpdateOnePropertyInfoInDatabase@CMainFrame@@QAEHV?$CStringT@DV?$StrTraitMFC_DLL@DV?$ChTraitsCRT@D@ATL@@@@@ATL@@@Z$34 0047c9a2 f   MainFrm.obj
 0001:0007b9ae       __unwindfunclet$?UpdateOnePropertyInfoInDatabase@CMainFrame@@QAEHV?$CStringT@DV?$StrTraitMFC_DLL@DV?$ChTraitsCRT@D@ATL@@@@@ATL@@@Z$35 0047c9ae f   MainFrm.obj
 0001:0007b9ba       __unwindfunclet$?UpdateOnePropertyInfoInDatabase@CMainFrame@@QAEHV?$CStringT@DV?$StrTraitMFC_DLL@DV?$ChTraitsCRT@D@ATL@@@@@ATL@@@Z$36 0047c9ba f   MainFrm.obj
 0001:0007b9c6       __unwindfunclet$?UpdateOnePropertyInfoInDatabase@CMainFrame@@QAEHV?$CStringT@DV?$StrTraitMFC_DLL@DV?$ChTraitsCRT@D@ATL@@@@@ATL@@@Z$37 0047c9c6 f   MainFrm.obj
 0001:0007b9d2       __unwindfunclet$?UpdateOnePropertyInfoInDatabase@CMainFrame@@QAEHV?$CStringT@DV?$StrTraitMFC_DLL@DV?$ChTraitsCRT@D@ATL@@@@@ATL@@@Z$38 0047c9d2 f   MainFrm.obj
 0001:0007b9de       __unwindfunclet$?UpdateOnePropertyInfoInDatabase@CMainFrame@@QAEHV?$CStringT@DV?$StrTraitMFC_DLL@DV?$ChTraitsCRT@D@ATL@@@@@ATL@@@Z$40 0047c9de f   MainFrm.obj
 0001:0007b9ea       __unwindfunclet$?UpdateOnePropertyInfoInDatabase@CMainFrame@@QAEHV?$CStringT@DV?$StrTraitMFC_DLL@DV?$ChTraitsCRT@D@ATL@@@@@ATL@@@Z$41 0047c9ea f   MainFrm.obj
 0001:0007b9f6       __ehhandler$?UpdateOnePropertyInfoInDatabase@CMainFrame@@QAEHV?$CStringT@DV?$StrTraitMFC_DLL@DV?$ChTraitsCRT@D@ATL@@@@@ATL@@@Z 0047c9f6 f   MainFrm.obj
 0001:0007ba20       __unwindfunclet$?OnDellist@CMainFrame@@QAEXXZ$1 0047ca20 f   MainFrm.obj
 0001:0007ba2c       __unwindfunclet$?OnDellist@CMainFrame@@QAEXXZ$2 0047ca2c f   MainFrm.obj
 0001:0007ba38       __unwindfunclet$?OnDellist@CMainFrame@@QAEXXZ$3 0047ca38 f   MainFrm.obj
 0001:0007ba44       __unwindfunclet$?OnDellist@CMainFrame@@QAEXXZ$4 0047ca44 f   MainFrm.obj
 0001:0007ba50       __unwindfunclet$?OnDellist@CMainFrame@@QAEXXZ$5 0047ca50 f   MainFrm.obj
 0001:0007ba5b       __unwindfunclet$?OnDellist@CMainFrame@@QAEXXZ$6 0047ca5b f   MainFrm.obj
 0001:0007ba7e       __unwindfunclet$?OnDellist@CMainFrame@@QAEXXZ$7 0047ca7e f   MainFrm.obj
 0001:0007baa1       __unwindfunclet$?OnDellist@CMainFrame@@QAEXXZ$8 0047caa1 f   MainFrm.obj
 0001:0007baad       __unwindfunclet$?OnDellist@CMainFrame@@QAEXXZ$9 0047caad f   MainFrm.obj
 0001:0007bab9       __unwindfunclet$?OnDellist@CMainFrame@@QAEXXZ$10 0047cab9 f   MainFrm.obj
 0001:0007bac5       __unwindfunclet$?OnDellist@CMainFrame@@QAEXXZ$11 0047cac5 f   MainFrm.obj
 0001:0007bad1       __unwindfunclet$?OnDellist@CMainFrame@@QAEXXZ$12 0047cad1 f   MainFrm.obj
 0001:0007badd       __ehhandler$?OnDellist@CMainFrame@@QAEXXZ 0047cadd f   MainFrm.obj
 0001:0007bb00       __unwindfunclet$?OnBlacklist@CMainFrame@@QAEXXZ$0 0047cb00 f   MainFrm.obj
 0001:0007bb0b       __ehhandler$?OnBlacklist@CMainFrame@@QAEXXZ 0047cb0b f   MainFrm.obj
 0001:0007bb30       __unwindfunclet$?HandlePropertyInfoPacket@CMainFrame@@QAEXPAUPropertyInfo@@HK@Z$0 0047cb30 f   MainFrm.obj
 0001:0007bb39       __unwindfunclet$?HandlePropertyInfoPacket@CMainFrame@@QAEXPAUPropertyInfo@@HK@Z$1 0047cb39 f   MainFrm.obj
 0001:0007bb42       __unwindfunclet$?HandlePropertyInfoPacket@CMainFrame@@QAEXPAUPropertyInfo@@HK@Z$3 0047cb42 f   MainFrm.obj
 0001:0007bb4e       __unwindfunclet$?HandlePropertyInfoPacket@CMainFrame@@QAEXPAUPropertyInfo@@HK@Z$4 0047cb4e f   MainFrm.obj
 0001:0007bb5a       __unwindfunclet$?HandlePropertyInfoPacket@CMainFrame@@QAEXPAUPropertyInfo@@HK@Z$5 0047cb5a f   MainFrm.obj
 0001:0007bb66       __unwindfunclet$?HandlePropertyInfoPacket@CMainFrame@@QAEXPAUPropertyInfo@@HK@Z$6 0047cb66 f   MainFrm.obj
 0001:0007bb72       __unwindfunclet$?HandlePropertyInfoPacket@CMainFrame@@QAEXPAUPropertyInfo@@HK@Z$7 0047cb72 f   MainFrm.obj
 0001:0007bb7e       __unwindfunclet$?HandlePropertyInfoPacket@CMainFrame@@QAEXPAUPropertyInfo@@HK@Z$8 0047cb7e f   MainFrm.obj
 0001:0007bb8a       __unwindfunclet$?HandlePropertyInfoPacket@CMainFrame@@QAEXPAUPropertyInfo@@HK@Z$9 0047cb8a f   MainFrm.obj
 0001:0007bb96       __unwindfunclet$?HandlePropertyInfoPacket@CMainFrame@@QAEXPAUPropertyInfo@@HK@Z$10 0047cb96 f   MainFrm.obj
 0001:0007bba2       __unwindfunclet$?HandlePropertyInfoPacket@CMainFrame@@QAEXPAUPropertyInfo@@HK@Z$11 0047cba2 f   MainFrm.obj
 0001:0007bbae       __unwindfunclet$?HandlePropertyInfoPacket@CMainFrame@@QAEXPAUPropertyInfo@@HK@Z$12 0047cbae f   MainFrm.obj
 0001:0007bbba       __unwindfunclet$?HandlePropertyInfoPacket@CMainFrame@@QAEXPAUPropertyInfo@@HK@Z$13 0047cbba f   MainFrm.obj
 0001:0007bbc6       __unwindfunclet$?HandlePropertyInfoPacket@CMainFrame@@QAEXPAUPropertyInfo@@HK@Z$14 0047cbc6 f   MainFrm.obj
 0001:0007bbd2       __unwindfunclet$?HandlePropertyInfoPacket@CMainFrame@@QAEXPAUPropertyInfo@@HK@Z$15 0047cbd2 f   MainFrm.obj
 0001:0007bbde       __unwindfunclet$?HandlePropertyInfoPacket@CMainFrame@@QAEXPAUPropertyInfo@@HK@Z$16 0047cbde f   MainFrm.obj
 0001:0007bbea       __unwindfunclet$?HandlePropertyInfoPacket@CMainFrame@@QAEXPAUPropertyInfo@@HK@Z$17 0047cbea f   MainFrm.obj
 0001:0007bbf6       __unwindfunclet$?HandlePropertyInfoPacket@CMainFrame@@QAEXPAUPropertyInfo@@HK@Z$18 0047cbf6 f   MainFrm.obj
 0001:0007bc02       __unwindfunclet$?HandlePropertyInfoPacket@CMainFrame@@QAEXPAUPropertyInfo@@HK@Z$19 0047cc02 f   MainFrm.obj
 0001:0007bc0e       __unwindfunclet$?HandlePropertyInfoPacket@CMainFrame@@QAEXPAUPropertyInfo@@HK@Z$20 0047cc0e f   MainFrm.obj
 0001:0007bc1a       __unwindfunclet$?HandlePropertyInfoPacket@CMainFrame@@QAEXPAUPropertyInfo@@HK@Z$21 0047cc1a f   MainFrm.obj
 0001:0007bc26       __unwindfunclet$?HandlePropertyInfoPacket@CMainFrame@@QAEXPAUPropertyInfo@@HK@Z$22 0047cc26 f   MainFrm.obj
 0001:0007bc32       __unwindfunclet$?HandlePropertyInfoPacket@CMainFrame@@QAEXPAUPropertyInfo@@HK@Z$23 0047cc32 f   MainFrm.obj
 0001:0007bc3e       __unwindfunclet$?HandlePropertyInfoPacket@CMainFrame@@QAEXPAUPropertyInfo@@HK@Z$24 0047cc3e f   MainFrm.obj
 0001:0007bc4a       __unwindfunclet$?HandlePropertyInfoPacket@CMainFrame@@QAEXPAUPropertyInfo@@HK@Z$25 0047cc4a f   MainFrm.obj
 0001:0007bc56       __unwindfunclet$?HandlePropertyInfoPacket@CMainFrame@@QAEXPAUPropertyInfo@@HK@Z$26 0047cc56 f   MainFrm.obj
 0001:0007bc62       __unwindfunclet$?HandlePropertyInfoPacket@CMainFrame@@QAEXPAUPropertyInfo@@HK@Z$27 0047cc62 f   MainFrm.obj
 0001:0007bc6e       __unwindfunclet$?HandlePropertyInfoPacket@CMainFrame@@QAEXPAUPropertyInfo@@HK@Z$28 0047cc6e f   MainFrm.obj
 0001:0007bc7a       __unwindfunclet$?HandlePropertyInfoPacket@CMainFrame@@QAEXPAUPropertyInfo@@HK@Z$29 0047cc7a f   MainFrm.obj
 0001:0007bc86       __unwindfunclet$?HandlePropertyInfoPacket@CMainFrame@@QAEXPAUPropertyInfo@@HK@Z$30 0047cc86 f   MainFrm.obj
 0001:0007bc92       __unwindfunclet$?HandlePropertyInfoPacket@CMainFrame@@QAEXPAUPropertyInfo@@HK@Z$31 0047cc92 f   MainFrm.obj
 0001:0007bc9e       __unwindfunclet$?HandlePropertyInfoPacket@CMainFrame@@QAEXPAUPropertyInfo@@HK@Z$32 0047cc9e f   MainFrm.obj
 0001:0007bcaa       __unwindfunclet$?HandlePropertyInfoPacket@CMainFrame@@QAEXPAUPropertyInfo@@HK@Z$33 0047ccaa f   MainFrm.obj
 0001:0007bcb6       __unwindfunclet$?HandlePropertyInfoPacket@CMainFrame@@QAEXPAUPropertyInfo@@HK@Z$34 0047ccb6 f   MainFrm.obj
 0001:0007bcc2       __unwindfunclet$?HandlePropertyInfoPacket@CMainFrame@@QAEXPAUPropertyInfo@@HK@Z$35 0047ccc2 f   MainFrm.obj
 0001:0007bcce       __unwindfunclet$?HandlePropertyInfoPacket@CMainFrame@@QAEXPAUPropertyInfo@@HK@Z$36 0047ccce f   MainFrm.obj
 0001:0007bcda       __unwindfunclet$?HandlePropertyInfoPacket@CMainFrame@@QAEXPAUPropertyInfo@@HK@Z$37 0047ccda f   MainFrm.obj
 0001:0007bce6       __unwindfunclet$?HandlePropertyInfoPacket@CMainFrame@@QAEXPAUPropertyInfo@@HK@Z$38 0047cce6 f   MainFrm.obj
 0001:0007bcf2       __unwindfunclet$?HandlePropertyInfoPacket@CMainFrame@@QAEXPAUPropertyInfo@@HK@Z$41 0047ccf2 f   MainFrm.obj
 0001:0007bcfe       __unwindfunclet$?HandlePropertyInfoPacket@CMainFrame@@QAEXPAUPropertyInfo@@HK@Z$42 0047ccfe f   MainFrm.obj
 0001:0007bd0a       __unwindfunclet$?HandlePropertyInfoPacket@CMainFrame@@QAEXPAUPropertyInfo@@HK@Z$43 0047cd0a f   MainFrm.obj
 0001:0007bd16       __unwindfunclet$?HandlePropertyInfoPacket@CMainFrame@@QAEXPAUPropertyInfo@@HK@Z$44 0047cd16 f   MainFrm.obj
 0001:0007bd22       __unwindfunclet$?HandlePropertyInfoPacket@CMainFrame@@QAEXPAUPropertyInfo@@HK@Z$45 0047cd22 f   MainFrm.obj
 0001:0007bd2e       __unwindfunclet$?HandlePropertyInfoPacket@CMainFrame@@QAEXPAUPropertyInfo@@HK@Z$46 0047cd2e f   MainFrm.obj
 0001:0007bd3a       __unwindfunclet$?HandlePropertyInfoPacket@CMainFrame@@QAEXPAUPropertyInfo@@HK@Z$47 0047cd3a f   MainFrm.obj
 0001:0007bd46       __unwindfunclet$?HandlePropertyInfoPacket@CMainFrame@@QAEXPAUPropertyInfo@@HK@Z$48 0047cd46 f   MainFrm.obj
 0001:0007bd52       __unwindfunclet$?HandlePropertyInfoPacket@CMainFrame@@QAEXPAUPropertyInfo@@HK@Z$49 0047cd52 f   MainFrm.obj
 0001:0007bd5e       __unwindfunclet$?HandlePropertyInfoPacket@CMainFrame@@QAEXPAUPropertyInfo@@HK@Z$50 0047cd5e f   MainFrm.obj
 0001:0007bd6a       __unwindfunclet$?HandlePropertyInfoPacket@CMainFrame@@QAEXPAUPropertyInfo@@HK@Z$51 0047cd6a f   MainFrm.obj
 0001:0007bd76       __unwindfunclet$?HandlePropertyInfoPacket@CMainFrame@@QAEXPAUPropertyInfo@@HK@Z$52 0047cd76 f   MainFrm.obj
 0001:0007bd82       __unwindfunclet$?HandlePropertyInfoPacket@CMainFrame@@QAEXPAUPropertyInfo@@HK@Z$53 0047cd82 f   MainFrm.obj
 0001:0007bd8e       __unwindfunclet$?HandlePropertyInfoPacket@CMainFrame@@QAEXPAUPropertyInfo@@HK@Z$54 0047cd8e f   MainFrm.obj
 0001:0007bd9a       __unwindfunclet$?HandlePropertyInfoPacket@CMainFrame@@QAEXPAUPropertyInfo@@HK@Z$55 0047cd9a f   MainFrm.obj
 0001:0007bda6       __unwindfunclet$?HandlePropertyInfoPacket@CMainFrame@@QAEXPAUPropertyInfo@@HK@Z$56 0047cda6 f   MainFrm.obj
 0001:0007bdb2       __unwindfunclet$?HandlePropertyInfoPacket@CMainFrame@@QAEXPAUPropertyInfo@@HK@Z$57 0047cdb2 f   MainFrm.obj
 0001:0007bdbe       __unwindfunclet$?HandlePropertyInfoPacket@CMainFrame@@QAEXPAUPropertyInfo@@HK@Z$58 0047cdbe f   MainFrm.obj
 0001:0007bdca       __unwindfunclet$?HandlePropertyInfoPacket@CMainFrame@@QAEXPAUPropertyInfo@@HK@Z$59 0047cdca f   MainFrm.obj
 0001:0007bdd6       __unwindfunclet$?HandlePropertyInfoPacket@CMainFrame@@QAEXPAUPropertyInfo@@HK@Z$60 0047cdd6 f   MainFrm.obj
 0001:0007bde2       __unwindfunclet$?HandlePropertyInfoPacket@CMainFrame@@QAEXPAUPropertyInfo@@HK@Z$61 0047cde2 f   MainFrm.obj
 0001:0007bdee       __unwindfunclet$?HandlePropertyInfoPacket@CMainFrame@@QAEXPAUPropertyInfo@@HK@Z$62 0047cdee f   MainFrm.obj
 0001:0007bdfa       __unwindfunclet$?HandlePropertyInfoPacket@CMainFrame@@QAEXPAUPropertyInfo@@HK@Z$63 0047cdfa f   MainFrm.obj
 0001:0007be06       __unwindfunclet$?HandlePropertyInfoPacket@CMainFrame@@QAEXPAUPropertyInfo@@HK@Z$64 0047ce06 f   MainFrm.obj
 0001:0007be12       __unwindfunclet$?HandlePropertyInfoPacket@CMainFrame@@QAEXPAUPropertyInfo@@HK@Z$65 0047ce12 f   MainFrm.obj
 0001:0007be1e       __unwindfunclet$?HandlePropertyInfoPacket@CMainFrame@@QAEXPAUPropertyInfo@@HK@Z$66 0047ce1e f   MainFrm.obj
 0001:0007be2a       __unwindfunclet$?HandlePropertyInfoPacket@CMainFrame@@QAEXPAUPropertyInfo@@HK@Z$67 0047ce2a f   MainFrm.obj
 0001:0007be36       __unwindfunclet$?HandlePropertyInfoPacket@CMainFrame@@QAEXPAUPropertyInfo@@HK@Z$68 0047ce36 f   MainFrm.obj
 0001:0007be42       __unwindfunclet$?HandlePropertyInfoPacket@CMainFrame@@QAEXPAUPropertyInfo@@HK@Z$69 0047ce42 f   MainFrm.obj
 0001:0007be4e       __unwindfunclet$?HandlePropertyInfoPacket@CMainFrame@@QAEXPAUPropertyInfo@@HK@Z$70 0047ce4e f   MainFrm.obj
 0001:0007be5a       __unwindfunclet$?HandlePropertyInfoPacket@CMainFrame@@QAEXPAUPropertyInfo@@HK@Z$71 0047ce5a f   MainFrm.obj
 0001:0007be66       __unwindfunclet$?HandlePropertyInfoPacket@CMainFrame@@QAEXPAUPropertyInfo@@HK@Z$72 0047ce66 f   MainFrm.obj
 0001:0007be72       __unwindfunclet$?HandlePropertyInfoPacket@CMainFrame@@QAEXPAUPropertyInfo@@HK@Z$73 0047ce72 f   MainFrm.obj
 0001:0007be7e       __unwindfunclet$?HandlePropertyInfoPacket@CMainFrame@@QAEXPAUPropertyInfo@@HK@Z$74 0047ce7e f   MainFrm.obj
 0001:0007be8a       __unwindfunclet$?HandlePropertyInfoPacket@CMainFrame@@QAEXPAUPropertyInfo@@HK@Z$75 0047ce8a f   MainFrm.obj
 0001:0007be96       __unwindfunclet$?HandlePropertyInfoPacket@CMainFrame@@QAEXPAUPropertyInfo@@HK@Z$76 0047ce96 f   MainFrm.obj
 0001:0007bea2       __ehhandler$?HandlePropertyInfoPacket@CMainFrame@@QAEXPAUPropertyInfo@@HK@Z 0047cea2 f   MainFrm.obj
 0001:0007bec0       __unwindfunclet$?OnSetStatuBarText@CMainFrame@@QAEHH@Z$0 0047cec0 f   MainFrm.obj
 0001:0007bec9       __unwindfunclet$?OnSetStatuBarText@CMainFrame@@QAEHH@Z$1 0047cec9 f   MainFrm.obj
 0001:0007bed2       __unwindfunclet$?OnSetStatuBarText@CMainFrame@@QAEHH@Z$2 0047ced2 f   MainFrm.obj
 0001:0007bedb       __ehhandler$?OnSetStatuBarText@CMainFrame@@QAEHH@Z 0047cedb f   MainFrm.obj
 0001:0007bf00       __unwindfunclet$?UpdateGroupDisplay@CMainFrame@@QAEXV?$CStringT@DV?$StrTraitMFC_DLL@DV?$ChTraitsCRT@D@ATL@@@@@ATL@@H@Z$0 0047cf00 f   MainFrm.obj
 0001:0007bf09       __unwindfunclet$?UpdateGroupDisplay@CMainFrame@@QAEXV?$CStringT@DV?$StrTraitMFC_DLL@DV?$ChTraitsCRT@D@ATL@@@@@ATL@@H@Z$3 0047cf09 f   MainFrm.obj
 0001:0007bf12       __unwindfunclet$?UpdateGroupDisplay@CMainFrame@@QAEXV?$CStringT@DV?$StrTraitMFC_DLL@DV?$ChTraitsCRT@D@ATL@@@@@ATL@@H@Z$4 0047cf12 f   MainFrm.obj
 0001:0007bf1b       __unwindfunclet$?UpdateGroupDisplay@CMainFrame@@QAEXV?$CStringT@DV?$StrTraitMFC_DLL@DV?$ChTraitsCRT@D@ATL@@@@@ATL@@H@Z$5 0047cf1b f   MainFrm.obj
 0001:0007bf24       __unwindfunclet$?UpdateGroupDisplay@CMainFrame@@QAEXV?$CStringT@DV?$StrTraitMFC_DLL@DV?$ChTraitsCRT@D@ATL@@@@@ATL@@H@Z$7 0047cf24 f   MainFrm.obj
 0001:0007bf2d       __unwindfunclet$?UpdateGroupDisplay@CMainFrame@@QAEXV?$CStringT@DV?$StrTraitMFC_DLL@DV?$ChTraitsCRT@D@ATL@@@@@ATL@@H@Z$8 0047cf2d f   MainFrm.obj
 0001:0007bf36       __ehhandler$?UpdateGroupDisplay@CMainFrame@@QAEXV?$CStringT@DV?$StrTraitMFC_DLL@DV?$ChTraitsCRT@D@ATL@@@@@ATL@@H@Z 0047cf36 f   MainFrm.obj
 0001:0007bf60       __unwindfunclet$?DisplayGroup@CMainFrame@@QAEXXZ$0 0047cf60 f   MainFrm.obj
 0001:0007bf69       __unwindfunclet$?DisplayGroup@CMainFrame@@QAEXXZ$1 0047cf69 f   MainFrm.obj
 0001:0007bf72       __ehhandler$?DisplayGroup@CMainFrame@@QAEXXZ 0047cf72 f   MainFrm.obj
 0001:0007bf90       __unwindfunclet$?DisplayAllClient@CMainFrame@@QAEXXZ$0 0047cf90 f   MainFrm.obj
 0001:0007bf99       __unwindfunclet$?DisplayAllClient@CMainFrame@@QAEXXZ$1 0047cf99 f   MainFrm.obj
 0001:0007bfa2       __unwindfunclet$?DisplayAllClient@CMainFrame@@QAEXXZ$2 0047cfa2 f   MainFrm.obj
 0001:0007bfab       __unwindfunclet$?DisplayAllClient@CMainFrame@@QAEXXZ$3 0047cfab f   MainFrm.obj
 0001:0007bfb4       __unwindfunclet$?DisplayAllClient@CMainFrame@@QAEXXZ$4 0047cfb4 f   MainFrm.obj
 0001:0007bfbd       __unwindfunclet$?DisplayAllClient@CMainFrame@@QAEXXZ$5 0047cfbd f   MainFrm.obj
 0001:0007bfc6       __unwindfunclet$?DisplayAllClient@CMainFrame@@QAEXXZ$6 0047cfc6 f   MainFrm.obj
 0001:0007bfcf       __unwindfunclet$?DisplayAllClient@CMainFrame@@QAEXXZ$7 0047cfcf f   MainFrm.obj
 0001:0007bfd8       __unwindfunclet$?DisplayAllClient@CMainFrame@@QAEXXZ$8 0047cfd8 f   MainFrm.obj
 0001:0007bfe1       __unwindfunclet$?DisplayAllClient@CMainFrame@@QAEXXZ$9 0047cfe1 f   MainFrm.obj
 0001:0007bfea       __unwindfunclet$?DisplayAllClient@CMainFrame@@QAEXXZ$10 0047cfea f   MainFrm.obj
 0001:0007bff3       __unwindfunclet$?DisplayAllClient@CMainFrame@@QAEXXZ$11 0047cff3 f   MainFrm.obj
 0001:0007bffc       __unwindfunclet$?DisplayAllClient@CMainFrame@@QAEXXZ$12 0047cffc f   MainFrm.obj
 0001:0007c005       __ehhandler$?DisplayAllClient@CMainFrame@@QAEXXZ 0047d005 f   MainFrm.obj
 0001:0007c030       __unwindfunclet$?DisplayGroupClient@CMainFrame@@QAEXV?$CStringT@DV?$StrTraitMFC_DLL@DV?$ChTraitsCRT@D@ATL@@@@@ATL@@@Z$0 0047d030 f   MainFrm.obj
 0001:0007c039       __unwindfunclet$?DisplayGroupClient@CMainFrame@@QAEXV?$CStringT@DV?$StrTraitMFC_DLL@DV?$ChTraitsCRT@D@ATL@@@@@ATL@@@Z$1 0047d039 f   MainFrm.obj
 0001:0007c042       __unwindfunclet$?DisplayGroupClient@CMainFrame@@QAEXV?$CStringT@DV?$StrTraitMFC_DLL@DV?$ChTraitsCRT@D@ATL@@@@@ATL@@@Z$2 0047d042 f   MainFrm.obj
 0001:0007c04b       __unwindfunclet$?DisplayGroupClient@CMainFrame@@QAEXV?$CStringT@DV?$StrTraitMFC_DLL@DV?$ChTraitsCRT@D@ATL@@@@@ATL@@@Z$3 0047d04b f   MainFrm.obj
 0001:0007c054       __unwindfunclet$?DisplayGroupClient@CMainFrame@@QAEXV?$CStringT@DV?$StrTraitMFC_DLL@DV?$ChTraitsCRT@D@ATL@@@@@ATL@@@Z$4 0047d054 f   MainFrm.obj
 0001:0007c05d       __unwindfunclet$?DisplayGroupClient@CMainFrame@@QAEXV?$CStringT@DV?$StrTraitMFC_DLL@DV?$ChTraitsCRT@D@ATL@@@@@ATL@@@Z$5 0047d05d f   MainFrm.obj
 0001:0007c066       __unwindfunclet$?DisplayGroupClient@CMainFrame@@QAEXV?$CStringT@DV?$StrTraitMFC_DLL@DV?$ChTraitsCRT@D@ATL@@@@@ATL@@@Z$6 0047d066 f   MainFrm.obj
 0001:0007c06f       __unwindfunclet$?DisplayGroupClient@CMainFrame@@QAEXV?$CStringT@DV?$StrTraitMFC_DLL@DV?$ChTraitsCRT@D@ATL@@@@@ATL@@@Z$7 0047d06f f   MainFrm.obj
 0001:0007c078       __unwindfunclet$?DisplayGroupClient@CMainFrame@@QAEXV?$CStringT@DV?$StrTraitMFC_DLL@DV?$ChTraitsCRT@D@ATL@@@@@ATL@@@Z$8 0047d078 f   MainFrm.obj
 0001:0007c081       __unwindfunclet$?DisplayGroupClient@CMainFrame@@QAEXV?$CStringT@DV?$StrTraitMFC_DLL@DV?$ChTraitsCRT@D@ATL@@@@@ATL@@@Z$9 0047d081 f   MainFrm.obj
 0001:0007c08a       __unwindfunclet$?DisplayGroupClient@CMainFrame@@QAEXV?$CStringT@DV?$StrTraitMFC_DLL@DV?$ChTraitsCRT@D@ATL@@@@@ATL@@@Z$10 0047d08a f   MainFrm.obj
 0001:0007c093       __unwindfunclet$?DisplayGroupClient@CMainFrame@@QAEXV?$CStringT@DV?$StrTraitMFC_DLL@DV?$ChTraitsCRT@D@ATL@@@@@ATL@@@Z$11 0047d093 f   MainFrm.obj
 0001:0007c09c       __unwindfunclet$?DisplayGroupClient@CMainFrame@@QAEXV?$CStringT@DV?$StrTraitMFC_DLL@DV?$ChTraitsCRT@D@ATL@@@@@ATL@@@Z$12 0047d09c f   MainFrm.obj
 0001:0007c0a5       __unwindfunclet$?DisplayGroupClient@CMainFrame@@QAEXV?$CStringT@DV?$StrTraitMFC_DLL@DV?$ChTraitsCRT@D@ATL@@@@@ATL@@@Z$13 0047d0a5 f   MainFrm.obj
 0001:0007c0ae       __unwindfunclet$?DisplayGroupClient@CMainFrame@@QAEXV?$CStringT@DV?$StrTraitMFC_DLL@DV?$ChTraitsCRT@D@ATL@@@@@ATL@@@Z$14 0047d0ae f   MainFrm.obj
 0001:0007c0b7       __unwindfunclet$?DisplayGroupClient@CMainFrame@@QAEXV?$CStringT@DV?$StrTraitMFC_DLL@DV?$ChTraitsCRT@D@ATL@@@@@ATL@@@Z$15 0047d0b7 f   MainFrm.obj
 0001:0007c0c0       __ehhandler$?DisplayGroupClient@CMainFrame@@QAEXV?$CStringT@DV?$StrTraitMFC_DLL@DV?$ChTraitsCRT@D@ATL@@@@@ATL@@@Z 0047d0c0 f   MainFrm.obj
 0001:0007c0e0       __unwindfunclet$?InitializeBackupPanel@CMainFrame@@QAEXXZ$0 0047d0e0 f   MainFrm.obj
 0001:0007c0e9       __unwindfunclet$?InitializeBackupPanel@CMainFrame@@QAEXXZ$1 0047d0e9 f   MainFrm.obj
 0001:0007c0f2       __unwindfunclet$?InitializeBackupPanel@CMainFrame@@QAEXXZ$2 0047d0f2 f   MainFrm.obj
 0001:0007c0fc       __unwindfunclet$?InitializeBackupPanel@CMainFrame@@QAEXXZ$3 0047d0fc f   MainFrm.obj
 0001:0007c11c       __unwindfunclet$?InitializeBackupPanel@CMainFrame@@QAEXXZ$4 0047d11c f   MainFrm.obj
 0001:0007c126       __unwindfunclet$?InitializeBackupPanel@CMainFrame@@QAEXXZ$5 0047d126 f   MainFrm.obj
 0001:0007c146       __unwindfunclet$?InitializeBackupPanel@CMainFrame@@QAEXXZ$6 0047d146 f   MainFrm.obj
 0001:0007c150       __unwindfunclet$?InitializeBackupPanel@CMainFrame@@QAEXXZ$7 0047d150 f   MainFrm.obj
 0001:0007c170       __unwindfunclet$?InitializeBackupPanel@CMainFrame@@QAEXXZ$8 0047d170 f   MainFrm.obj
 0001:0007c17d       __unwindfunclet$?InitializeBackupPanel@CMainFrame@@QAEXXZ$9 0047d17d f   MainFrm.obj
 0001:0007c1a0       __unwindfunclet$?InitializeBackupPanel@CMainFrame@@QAEXXZ$10 0047d1a0 f   MainFrm.obj
 0001:0007c1ad       __unwindfunclet$?InitializeBackupPanel@CMainFrame@@QAEXXZ$11 0047d1ad f   MainFrm.obj
 0001:0007c1d0       __unwindfunclet$?InitializeBackupPanel@CMainFrame@@QAEXXZ$12 0047d1d0 f   MainFrm.obj
 0001:0007c1dd       __unwindfunclet$?InitializeBackupPanel@CMainFrame@@QAEXXZ$13 0047d1dd f   MainFrm.obj
 0001:0007c200       __unwindfunclet$?InitializeBackupPanel@CMainFrame@@QAEXXZ$14 0047d200 f   MainFrm.obj
 0001:0007c20d       __unwindfunclet$?InitializeBackupPanel@CMainFrame@@QAEXXZ$15 0047d20d f   MainFrm.obj
 0001:0007c230       __unwindfunclet$?InitializeBackupPanel@CMainFrame@@QAEXXZ$16 0047d230 f   MainFrm.obj
 0001:0007c23d       __unwindfunclet$?InitializeBackupPanel@CMainFrame@@QAEXXZ$17 0047d23d f   MainFrm.obj
 0001:0007c265       __unwindfunclet$?InitializeBackupPanel@CMainFrame@@QAEXXZ$18 0047d265 f   MainFrm.obj
 0001:0007c272       __unwindfunclet$?InitializeBackupPanel@CMainFrame@@QAEXXZ$19 0047d272 f   MainFrm.obj
 0001:0007c29a       __unwindfunclet$?InitializeBackupPanel@CMainFrame@@QAEXXZ$20 0047d29a f   MainFrm.obj
 0001:0007c2a7       __unwindfunclet$?InitializeBackupPanel@CMainFrame@@QAEXXZ$21 0047d2a7 f   MainFrm.obj
 0001:0007c2cf       __unwindfunclet$?InitializeBackupPanel@CMainFrame@@QAEXXZ$22 0047d2cf f   MainFrm.obj
 0001:0007c2dc       __unwindfunclet$?InitializeBackupPanel@CMainFrame@@QAEXXZ$23 0047d2dc f   MainFrm.obj
 0001:0007c304       __ehhandler$?InitializeBackupPanel@CMainFrame@@QAEXXZ 0047d304 f   MainFrm.obj
 0001:0007c330       __unwindfunclet$?InitializeRegisterPanel@CMainFrame@@QAEXXZ$0 0047d330 f   MainFrm.obj
 0001:0007c339       __unwindfunclet$?InitializeRegisterPanel@CMainFrame@@QAEXXZ$1 0047d339 f   MainFrm.obj
 0001:0007c342       __unwindfunclet$?InitializeRegisterPanel@CMainFrame@@QAEXXZ$2 0047d342 f   MainFrm.obj
 0001:0007c34c       __unwindfunclet$?InitializeRegisterPanel@CMainFrame@@QAEXXZ$3 0047d34c f   MainFrm.obj
 0001:0007c366       __unwindfunclet$?InitializeRegisterPanel@CMainFrame@@QAEXXZ$4 0047d366 f   MainFrm.obj
 0001:0007c370       __unwindfunclet$?InitializeRegisterPanel@CMainFrame@@QAEXXZ$5 0047d370 f   MainFrm.obj
 0001:0007c38a       __ehhandler$?InitializeRegisterPanel@CMainFrame@@QAEXXZ 0047d38a f   MainFrm.obj
 0001:0007c3b0       __unwindfunclet$?InitializeRemoteCtrlPanel@CMainFrame@@QAEXXZ$0 0047d3b0 f   MainFrm.obj
 0001:0007c3b9       __unwindfunclet$?InitializeRemoteCtrlPanel@CMainFrame@@QAEXXZ$1 0047d3b9 f   MainFrm.obj
 0001:0007c3c2       __unwindfunclet$?InitializeRemoteCtrlPanel@CMainFrame@@QAEXXZ$2 0047d3c2 f   MainFrm.obj
 0001:0007c3cc       __unwindfunclet$?InitializeRemoteCtrlPanel@CMainFrame@@QAEXXZ$3 0047d3cc f   MainFrm.obj
 0001:0007c3ef       __unwindfunclet$?InitializeRemoteCtrlPanel@CMainFrame@@QAEXXZ$4 0047d3ef f   MainFrm.obj
 0001:0007c3fc       __unwindfunclet$?InitializeRemoteCtrlPanel@CMainFrame@@QAEXXZ$5 0047d3fc f   MainFrm.obj
 0001:0007c41f       __unwindfunclet$?InitializeRemoteCtrlPanel@CMainFrame@@QAEXXZ$6 0047d41f f   MainFrm.obj
 0001:0007c42c       __unwindfunclet$?InitializeRemoteCtrlPanel@CMainFrame@@QAEXXZ$7 0047d42c f   MainFrm.obj
 0001:0007c44f       __unwindfunclet$?InitializeRemoteCtrlPanel@CMainFrame@@QAEXXZ$8 0047d44f f   MainFrm.obj
 0001:0007c45c       __unwindfunclet$?InitializeRemoteCtrlPanel@CMainFrame@@QAEXXZ$9 0047d45c f   MainFrm.obj
 0001:0007c47f       __unwindfunclet$?InitializeRemoteCtrlPanel@CMainFrame@@QAEXXZ$10 0047d47f f   MainFrm.obj
 0001:0007c48c       __unwindfunclet$?InitializeRemoteCtrlPanel@CMainFrame@@QAEXXZ$11 0047d48c f   MainFrm.obj
 0001:0007c4af       __unwindfunclet$?InitializeRemoteCtrlPanel@CMainFrame@@QAEXXZ$12 0047d4af f   MainFrm.obj
 0001:0007c4bc       __unwindfunclet$?InitializeRemoteCtrlPanel@CMainFrame@@QAEXXZ$13 0047d4bc f   MainFrm.obj
 0001:0007c4df       __unwindfunclet$?InitializeRemoteCtrlPanel@CMainFrame@@QAEXXZ$14 0047d4df f   MainFrm.obj
 0001:0007c4ec       __unwindfunclet$?InitializeRemoteCtrlPanel@CMainFrame@@QAEXXZ$15 0047d4ec f   MainFrm.obj
 0001:0007c50f       __unwindfunclet$?InitializeRemoteCtrlPanel@CMainFrame@@QAEXXZ$16 0047d50f f   MainFrm.obj
 0001:0007c51b       __unwindfunclet$?InitializeRemoteCtrlPanel@CMainFrame@@QAEXXZ$17 0047d51b f   MainFrm.obj
 0001:0007c528       __unwindfunclet$?InitializeRemoteCtrlPanel@CMainFrame@@QAEXXZ$18 0047d528 f   MainFrm.obj
 0001:0007c550       __unwindfunclet$?InitializeRemoteCtrlPanel@CMainFrame@@QAEXXZ$19 0047d550 f   MainFrm.obj
 0001:0007c55c       __unwindfunclet$?InitializeRemoteCtrlPanel@CMainFrame@@QAEXXZ$20 0047d55c f   MainFrm.obj
 0001:0007c569       __unwindfunclet$?InitializeRemoteCtrlPanel@CMainFrame@@QAEXXZ$21 0047d569 f   MainFrm.obj
 0001:0007c591       __unwindfunclet$?InitializeRemoteCtrlPanel@CMainFrame@@QAEXXZ$22 0047d591 f   MainFrm.obj
 0001:0007c59e       __unwindfunclet$?InitializeRemoteCtrlPanel@CMainFrame@@QAEXXZ$23 0047d59e f   MainFrm.obj
 0001:0007c5c6       __unwindfunclet$?InitializeRemoteCtrlPanel@CMainFrame@@QAEXXZ$24 0047d5c6 f   MainFrm.obj
 0001:0007c5d3       __unwindfunclet$?InitializeRemoteCtrlPanel@CMainFrame@@QAEXXZ$25 0047d5d3 f   MainFrm.obj
 0001:0007c5fb       __unwindfunclet$?InitializeRemoteCtrlPanel@CMainFrame@@QAEXXZ$26 0047d5fb f   MainFrm.obj
 0001:0007c608       __unwindfunclet$?InitializeRemoteCtrlPanel@CMainFrame@@QAEXXZ$27 0047d608 f   MainFrm.obj
 0001:0007c630       __unwindfunclet$?InitializeRemoteCtrlPanel@CMainFrame@@QAEXXZ$28 0047d630 f   MainFrm.obj
 0001:0007c63d       __unwindfunclet$?InitializeRemoteCtrlPanel@CMainFrame@@QAEXXZ$29 0047d63d f   MainFrm.obj
 0001:0007c665       __unwindfunclet$?InitializeRemoteCtrlPanel@CMainFrame@@QAEXXZ$30 0047d665 f   MainFrm.obj
 0001:0007c672       __unwindfunclet$?InitializeRemoteCtrlPanel@CMainFrame@@QAEXXZ$31 0047d672 f   MainFrm.obj
 0001:0007c69a       __unwindfunclet$?InitializeRemoteCtrlPanel@CMainFrame@@QAEXXZ$32 0047d69a f   MainFrm.obj
 0001:0007c6a7       __unwindfunclet$?InitializeRemoteCtrlPanel@CMainFrame@@QAEXXZ$33 0047d6a7 f   MainFrm.obj
 0001:0007c6cf       __unwindfunclet$?InitializeRemoteCtrlPanel@CMainFrame@@QAEXXZ$34 0047d6cf f   MainFrm.obj
 0001:0007c6dc       __unwindfunclet$?InitializeRemoteCtrlPanel@CMainFrame@@QAEXXZ$35 0047d6dc f   MainFrm.obj
 0001:0007c704       __unwindfunclet$?InitializeRemoteCtrlPanel@CMainFrame@@QAEXXZ$36 0047d704 f   MainFrm.obj
 0001:0007c711       __unwindfunclet$?InitializeRemoteCtrlPanel@CMainFrame@@QAEXXZ$37 0047d711 f   MainFrm.obj
 0001:0007c739       __ehhandler$?InitializeRemoteCtrlPanel@CMainFrame@@QAEXXZ 0047d739 f   MainFrm.obj
 0001:0007c760       __unwindfunclet$?InitializeAppPanel@CMainFrame@@QAEXXZ$0 0047d760 f   MainFrm.obj
 0001:0007c769       __unwindfunclet$?InitializeAppPanel@CMainFrame@@QAEXXZ$1 0047d769 f   MainFrm.obj
 0001:0007c772       __unwindfunclet$?InitializeAppPanel@CMainFrame@@QAEXXZ$2 0047d772 f   MainFrm.obj
 0001:0007c77c       __unwindfunclet$?InitializeAppPanel@CMainFrame@@QAEXXZ$3 0047d77c f   MainFrm.obj
 0001:0007c79c       __unwindfunclet$?InitializeAppPanel@CMainFrame@@QAEXXZ$4 0047d79c f   MainFrm.obj
 0001:0007c7a6       __unwindfunclet$?InitializeAppPanel@CMainFrame@@QAEXXZ$5 0047d7a6 f   MainFrm.obj
 0001:0007c7c6       __unwindfunclet$?InitializeAppPanel@CMainFrame@@QAEXXZ$6 0047d7c6 f   MainFrm.obj
 0001:0007c7d0       __unwindfunclet$?InitializeAppPanel@CMainFrame@@QAEXXZ$7 0047d7d0 f   MainFrm.obj
 0001:0007c7f0       __unwindfunclet$?InitializeAppPanel@CMainFrame@@QAEXXZ$8 0047d7f0 f   MainFrm.obj
 0001:0007c7f9       __unwindfunclet$?InitializeAppPanel@CMainFrame@@QAEXXZ$9 0047d7f9 f   MainFrm.obj
 0001:0007c803       __unwindfunclet$?InitializeAppPanel@CMainFrame@@QAEXXZ$10 0047d803 f   MainFrm.obj
 0001:0007c823       __unwindfunclet$?InitializeAppPanel@CMainFrame@@QAEXXZ$11 0047d823 f   MainFrm.obj
 0001:0007c82d       __unwindfunclet$?InitializeAppPanel@CMainFrame@@QAEXXZ$12 0047d82d f   MainFrm.obj
 0001:0007c84d       __unwindfunclet$?InitializeAppPanel@CMainFrame@@QAEXXZ$13 0047d84d f   MainFrm.obj
 0001:0007c85a       __unwindfunclet$?InitializeAppPanel@CMainFrame@@QAEXXZ$14 0047d85a f   MainFrm.obj
 0001:0007c87d       __unwindfunclet$?InitializeAppPanel@CMainFrame@@QAEXXZ$15 0047d87d f   MainFrm.obj
 0001:0007c88a       __unwindfunclet$?InitializeAppPanel@CMainFrame@@QAEXXZ$16 0047d88a f   MainFrm.obj
 0001:0007c8ad       __ehhandler$?InitializeAppPanel@CMainFrame@@QAEXXZ 0047d8ad f   MainFrm.obj
 0001:0007c8d0       __unwindfunclet$?InitializePropertyPanel@CMainFrame@@QAEXXZ$0 0047d8d0 f   MainFrm.obj
 0001:0007c8d0       __unwindfunclet$?InitializeOwnPanel@CMainFrame@@QAEXXZ$0 0047d8d0 f   MainFrm.obj
 0001:0007c8d9       __unwindfunclet$?InitializePropertyPanel@CMainFrame@@QAEXXZ$1 0047d8d9 f   MainFrm.obj
 0001:0007c8d9       __unwindfunclet$?InitializeOwnPanel@CMainFrame@@QAEXXZ$1 0047d8d9 f   MainFrm.obj
 0001:0007c8e2       __unwindfunclet$?InitializePropertyPanel@CMainFrame@@QAEXXZ$2 0047d8e2 f   MainFrm.obj
 0001:0007c8e2       __unwindfunclet$?InitializeOwnPanel@CMainFrame@@QAEXXZ$2 0047d8e2 f   MainFrm.obj
 0001:0007c8ec       __unwindfunclet$?InitializeOwnPanel@CMainFrame@@QAEXXZ$3 0047d8ec f   MainFrm.obj
 0001:0007c8ec       __unwindfunclet$?InitializePropertyPanel@CMainFrame@@QAEXXZ$3 0047d8ec f   MainFrm.obj
 0001:0007c906       __unwindfunclet$?InitializePropertyPanel@CMainFrame@@QAEXXZ$4 0047d906 f   MainFrm.obj
 0001:0007c906       __unwindfunclet$?InitializeOwnPanel@CMainFrame@@QAEXXZ$4 0047d906 f   MainFrm.obj
 0001:0007c910       __unwindfunclet$?InitializeOwnPanel@CMainFrame@@QAEXXZ$5 0047d910 f   MainFrm.obj
 0001:0007c910       __unwindfunclet$?InitializePropertyPanel@CMainFrame@@QAEXXZ$5 0047d910 f   MainFrm.obj
 0001:0007c92a       __unwindfunclet$?InitializeOwnPanel@CMainFrame@@QAEXXZ$6 0047d92a f   MainFrm.obj
 0001:0007c92a       __unwindfunclet$?InitializePropertyPanel@CMainFrame@@QAEXXZ$6 0047d92a f   MainFrm.obj
 0001:0007c934       __unwindfunclet$?InitializeOwnPanel@CMainFrame@@QAEXXZ$7 0047d934 f   MainFrm.obj
 0001:0007c934       __unwindfunclet$?InitializePropertyPanel@CMainFrame@@QAEXXZ$7 0047d934 f   MainFrm.obj
 0001:0007c94e       __ehhandler$?InitializeOwnPanel@CMainFrame@@QAEXXZ 0047d94e f   MainFrm.obj
 0001:0007c94e       __ehhandler$?InitializePropertyPanel@CMainFrame@@QAEXXZ 0047d94e f   MainFrm.obj
 0001:0007c970       __unwindfunclet$?OnProgressDlgClosed@CMainFrame@@QAEJIJ@Z$0 0047d970 f   MainFrm.obj
 0001:0007c97b       __unwindfunclet$?OnProgressDlgClosed@CMainFrame@@QAEJIJ@Z$1 0047d97b f   MainFrm.obj
 0001:0007c987       __unwindfunclet$?OnProgressDlgClosed@CMainFrame@@QAEJIJ@Z$2 0047d987 f   MainFrm.obj
 0001:0007c993       __unwindfunclet$?OnProgressDlgClosed@CMainFrame@@QAEJIJ@Z$3 0047d993 f   MainFrm.obj
 0001:0007c99e       __unwindfunclet$?OnProgressDlgClosed@CMainFrame@@QAEJIJ@Z$4 0047d99e f   MainFrm.obj
 0001:0007c9aa       __unwindfunclet$?OnProgressDlgClosed@CMainFrame@@QAEJIJ@Z$5 0047d9aa f   MainFrm.obj
 0001:0007c9b6       __unwindfunclet$?OnProgressDlgClosed@CMainFrame@@QAEJIJ@Z$6 0047d9b6 f   MainFrm.obj
 0001:0007c9c2       __unwindfunclet$?OnProgressDlgClosed@CMainFrame@@QAEJIJ@Z$7 0047d9c2 f   MainFrm.obj
 0001:0007c9ce       __unwindfunclet$?OnProgressDlgClosed@CMainFrame@@QAEJIJ@Z$8 0047d9ce f   MainFrm.obj
 0001:0007c9da       __unwindfunclet$?OnProgressDlgClosed@CMainFrame@@QAEJIJ@Z$9 0047d9da f   MainFrm.obj
 0001:0007c9e6       __unwindfunclet$?OnProgressDlgClosed@CMainFrame@@QAEJIJ@Z$10 0047d9e6 f   MainFrm.obj
 0001:0007c9f2       __unwindfunclet$?OnProgressDlgClosed@CMainFrame@@QAEJIJ@Z$11 0047d9f2 f   MainFrm.obj
 0001:0007c9fe       __unwindfunclet$?OnProgressDlgClosed@CMainFrame@@QAEJIJ@Z$12 0047d9fe f   MainFrm.obj
 0001:0007ca0a       __unwindfunclet$?OnProgressDlgClosed@CMainFrame@@QAEJIJ@Z$13 0047da0a f   MainFrm.obj
 0001:0007ca16       __unwindfunclet$?OnProgressDlgClosed@CMainFrame@@QAEJIJ@Z$15 0047da16 f   MainFrm.obj
 0001:0007ca22       __unwindfunclet$?OnProgressDlgClosed@CMainFrame@@QAEJIJ@Z$16 0047da22 f   MainFrm.obj
 0001:0007ca2e       __unwindfunclet$?OnProgressDlgClosed@CMainFrame@@QAEJIJ@Z$17 0047da2e f   MainFrm.obj
 0001:0007ca3a       __unwindfunclet$?OnProgressDlgClosed@CMainFrame@@QAEJIJ@Z$18 0047da3a f   MainFrm.obj
 0001:0007ca46       __unwindfunclet$?OnProgressDlgClosed@CMainFrame@@QAEJIJ@Z$19 0047da46 f   MainFrm.obj
 0001:0007ca52       __unwindfunclet$?OnProgressDlgClosed@CMainFrame@@QAEJIJ@Z$20 0047da52 f   MainFrm.obj
 0001:0007ca5e       __unwindfunclet$?OnProgressDlgClosed@CMainFrame@@QAEJIJ@Z$21 0047da5e f   MainFrm.obj
 0001:0007ca6a       __unwindfunclet$?OnProgressDlgClosed@CMainFrame@@QAEJIJ@Z$22 0047da6a f   MainFrm.obj
 0001:0007ca76       __unwindfunclet$?OnProgressDlgClosed@CMainFrame@@QAEJIJ@Z$24 0047da76 f   MainFrm.obj
 0001:0007ca82       __unwindfunclet$?OnProgressDlgClosed@CMainFrame@@QAEJIJ@Z$25 0047da82 f   MainFrm.obj
 0001:0007ca8e       __unwindfunclet$?OnProgressDlgClosed@CMainFrame@@QAEJIJ@Z$26 0047da8e f   MainFrm.obj
 0001:0007ca9a       __unwindfunclet$?OnProgressDlgClosed@CMainFrame@@QAEJIJ@Z$27 0047da9a f   MainFrm.obj
 0001:0007caa6       __unwindfunclet$?OnProgressDlgClosed@CMainFrame@@QAEJIJ@Z$28 0047daa6 f   MainFrm.obj
 0001:0007cab2       __unwindfunclet$?OnProgressDlgClosed@CMainFrame@@QAEJIJ@Z$29 0047dab2 f   MainFrm.obj
 0001:0007cabe       __unwindfunclet$?OnProgressDlgClosed@CMainFrame@@QAEJIJ@Z$30 0047dabe f   MainFrm.obj
 0001:0007caca       __unwindfunclet$?OnProgressDlgClosed@CMainFrame@@QAEJIJ@Z$31 0047daca f   MainFrm.obj
 0001:0007cad6       __unwindfunclet$?OnProgressDlgClosed@CMainFrame@@QAEJIJ@Z$33 0047dad6 f   MainFrm.obj
 0001:0007cae2       __unwindfunclet$?OnProgressDlgClosed@CMainFrame@@QAEJIJ@Z$34 0047dae2 f   MainFrm.obj
 0001:0007caee       __unwindfunclet$?OnProgressDlgClosed@CMainFrame@@QAEJIJ@Z$35 0047daee f   MainFrm.obj
 0001:0007cafa       __unwindfunclet$?OnProgressDlgClosed@CMainFrame@@QAEJIJ@Z$36 0047dafa f   MainFrm.obj
 0001:0007cb06       __unwindfunclet$?OnProgressDlgClosed@CMainFrame@@QAEJIJ@Z$37 0047db06 f   MainFrm.obj
 0001:0007cb12       __unwindfunclet$?OnProgressDlgClosed@CMainFrame@@QAEJIJ@Z$38 0047db12 f   MainFrm.obj
 0001:0007cb1e       __unwindfunclet$?OnProgressDlgClosed@CMainFrame@@QAEJIJ@Z$39 0047db1e f   MainFrm.obj
 0001:0007cb2a       __unwindfunclet$?OnProgressDlgClosed@CMainFrame@@QAEJIJ@Z$40 0047db2a f   MainFrm.obj
 0001:0007cb36       __unwindfunclet$?OnProgressDlgClosed@CMainFrame@@QAEJIJ@Z$41 0047db36 f   MainFrm.obj
 0001:0007cb42       __unwindfunclet$?OnProgressDlgClosed@CMainFrame@@QAEJIJ@Z$42 0047db42 f   MainFrm.obj
 0001:0007cb4e       __unwindfunclet$?OnProgressDlgClosed@CMainFrame@@QAEJIJ@Z$43 0047db4e f   MainFrm.obj
 0001:0007cb5a       __unwindfunclet$?OnProgressDlgClosed@CMainFrame@@QAEJIJ@Z$44 0047db5a f   MainFrm.obj
 0001:0007cb66       __unwindfunclet$?OnProgressDlgClosed@CMainFrame@@QAEJIJ@Z$45 0047db66 f   MainFrm.obj
 0001:0007cb72       __unwindfunclet$?OnProgressDlgClosed@CMainFrame@@QAEJIJ@Z$46 0047db72 f   MainFrm.obj
 0001:0007cb7e       __unwindfunclet$?OnProgressDlgClosed@CMainFrame@@QAEJIJ@Z$47 0047db7e f   MainFrm.obj
 0001:0007cb8a       __unwindfunclet$?OnProgressDlgClosed@CMainFrame@@QAEJIJ@Z$48 0047db8a f   MainFrm.obj
 0001:0007cb96       __ehhandler$?OnProgressDlgClosed@CMainFrame@@QAEJIJ@Z 0047db96 f   MainFrm.obj
 0001:0007cbd0       __unwindfunclet$?OnSysCommand@CMainFrame@@QAEXIJ@Z$0 0047dbd0 f   MainFrm.obj
 0001:0007cbd9       __ehhandler$?OnSysCommand@CMainFrame@@QAEXIJ@Z 0047dbd9 f   MainFrm.obj
 0001:0007cc00       __unwindfunclet$?OnMyMsg@CMainFrame@@QAEJIJ@Z$0 0047dc00 f   MainFrm.obj
 0001:0007cc0c       __unwindfunclet$?OnMyMsg@CMainFrame@@QAEJIJ@Z$1 0047dc0c f   MainFrm.obj
 0001:0007cc18       __unwindfunclet$?OnMyMsg@CMainFrame@@QAEJIJ@Z$2 0047dc18 f   MainFrm.obj
 0001:0007cc24       __unwindfunclet$?OnMyMsg@CMainFrame@@QAEJIJ@Z$3 0047dc24 f   MainFrm.obj
 0001:0007cc30       __ehhandler$?OnMyMsg@CMainFrame@@QAEJIJ@Z 0047dc30 f   MainFrm.obj
 0001:0007cc60       __unwindfunclet$?DriverExist@CMainFrame@@QAEHXZ$0 0047dc60 f   MainFrm.obj
 0001:0007cc6b       __unwindfunclet$?DriverExist@CMainFrame@@QAEHXZ$1 0047dc6b f   MainFrm.obj
 0001:0007cc76       __ehhandler$?DriverExist@CMainFrame@@QAEHXZ 0047dc76 f   MainFrm.obj
 0001:0007cca0       __unwindfunclet$?OnTrayBackup@CMainFrame@@QAEXXZ$0 0047dca0 f   MainFrm.obj
 0001:0007cca0       __unwindfunclet$?OnTrayRecovery@CMainFrame@@QAEXXZ$0 0047dca0 f   MainFrm.obj
 0001:0007ccac       __unwindfunclet$?OnTrayRecovery@CMainFrame@@QAEXXZ$1 0047dcac f   MainFrm.obj
 0001:0007ccac       __unwindfunclet$?OnTrayBackup@CMainFrame@@QAEXXZ$1 0047dcac f   MainFrm.obj
 0001:0007ccb8       __unwindfunclet$?OnTrayBackup@CMainFrame@@QAEXXZ$2 0047dcb8 f   MainFrm.obj
 0001:0007ccb8       __unwindfunclet$?OnTrayRecovery@CMainFrame@@QAEXXZ$2 0047dcb8 f   MainFrm.obj
 0001:0007ccc4       __unwindfunclet$?OnTrayBackup@CMainFrame@@QAEXXZ$3 0047dcc4 f   MainFrm.obj
 0001:0007ccc4       __unwindfunclet$?OnTrayRecovery@CMainFrame@@QAEXXZ$3 0047dcc4 f   MainFrm.obj
 0001:0007ccd0       __unwindfunclet$?OnTrayRecovery@CMainFrame@@QAEXXZ$4 0047dcd0 f   MainFrm.obj
 0001:0007ccd0       __unwindfunclet$?OnTrayBackup@CMainFrame@@QAEXXZ$4 0047dcd0 f   MainFrm.obj
 0001:0007ccdc       __unwindfunclet$?OnTrayBackup@CMainFrame@@QAEXXZ$5 0047dcdc f   MainFrm.obj
 0001:0007ccdc       __unwindfunclet$?OnTrayRecovery@CMainFrame@@QAEXXZ$5 0047dcdc f   MainFrm.obj
 0001:0007cce8       __unwindfunclet$?OnTrayRecovery@CMainFrame@@QAEXXZ$6 0047dce8 f   MainFrm.obj
 0001:0007cce8       __unwindfunclet$?OnTrayBackup@CMainFrame@@QAEXXZ$6 0047dce8 f   MainFrm.obj
 0001:0007ccf4       __unwindfunclet$?OnTrayRecovery@CMainFrame@@QAEXXZ$7 0047dcf4 f   MainFrm.obj
 0001:0007ccf4       __unwindfunclet$?OnTrayBackup@CMainFrame@@QAEXXZ$7 0047dcf4 f   MainFrm.obj
 0001:0007cd00       __unwindfunclet$?OnTrayBackup@CMainFrame@@QAEXXZ$8 0047dd00 f   MainFrm.obj
 0001:0007cd00       __unwindfunclet$?OnTrayRecovery@CMainFrame@@QAEXXZ$8 0047dd00 f   MainFrm.obj
 0001:0007cd0b       __unwindfunclet$?OnTrayRecovery@CMainFrame@@QAEXXZ$9 0047dd0b f   MainFrm.obj
 0001:0007cd0b       __unwindfunclet$?OnTrayBackup@CMainFrame@@QAEXXZ$9 0047dd0b f   MainFrm.obj
 0001:0007cd17       __unwindfunclet$?OnTrayRecovery@CMainFrame@@QAEXXZ$10 0047dd17 f   MainFrm.obj
 0001:0007cd17       __unwindfunclet$?OnTrayBackup@CMainFrame@@QAEXXZ$10 0047dd17 f   MainFrm.obj
 0001:0007cd22       __unwindfunclet$?OnTrayBackup@CMainFrame@@QAEXXZ$11 0047dd22 f   MainFrm.obj
 0001:0007cd22       __unwindfunclet$?OnTrayRecovery@CMainFrame@@QAEXXZ$11 0047dd22 f   MainFrm.obj
 0001:0007cd2e       __unwindfunclet$?OnTrayBackup@CMainFrame@@QAEXXZ$12 0047dd2e f   MainFrm.obj
 0001:0007cd2e       __unwindfunclet$?OnTrayRecovery@CMainFrame@@QAEXXZ$12 0047dd2e f   MainFrm.obj
 0001:0007cd3a       __unwindfunclet$?OnTrayBackup@CMainFrame@@QAEXXZ$13 0047dd3a f   MainFrm.obj
 0001:0007cd3a       __unwindfunclet$?OnTrayRecovery@CMainFrame@@QAEXXZ$13 0047dd3a f   MainFrm.obj
 0001:0007cd46       __ehhandler$?OnTrayBackup@CMainFrame@@QAEXXZ 0047dd46 f   MainFrm.obj
 0001:0007cd46       __ehhandler$?OnTrayRecovery@CMainFrame@@QAEXXZ 0047dd46 f   MainFrm.obj
 0001:0007cd70       __unwindfunclet$?OnTrayModifygroup@CMainFrame@@QAEXXZ$0 0047dd70 f   MainFrm.obj
 0001:0007cd7b       __unwindfunclet$?OnTrayModifygroup@CMainFrame@@QAEXXZ$1 0047dd7b f   MainFrm.obj
 0001:0007cd87       __unwindfunclet$?OnTrayModifygroup@CMainFrame@@QAEXXZ$2 0047dd87 f   MainFrm.obj
 0001:0007cd90       __unwindfunclet$?OnTrayModifygroup@CMainFrame@@QAEXXZ$3 0047dd90 f   MainFrm.obj
 0001:0007cd9c       __unwindfunclet$?OnTrayModifygroup@CMainFrame@@QAEXXZ$4 0047dd9c f   MainFrm.obj
 0001:0007cda8       __ehhandler$?OnTrayModifygroup@CMainFrame@@QAEXXZ 0047dda8 f   MainFrm.obj
 0001:0007cdd0       __unwindfunclet$?GetServerGroup@CMainFrame@@IAEHXZ$0 0047ddd0 f   MainFrm.obj
 0001:0007cddc       __unwindfunclet$?GetServerGroup@CMainFrame@@IAEHXZ$1 0047dddc f   MainFrm.obj
 0001:0007cde8       __unwindfunclet$?GetServerGroup@CMainFrame@@IAEHXZ$2 0047dde8 f   MainFrm.obj
 0001:0007cdf4       __ehhandler$?GetServerGroup@CMainFrame@@IAEHXZ 0047ddf4 f   MainFrm.obj
 0001:0007ce20       __unwindfunclet$?SetServerGroup@CMainFrame@@IAEHXZ$0 0047de20 f   MainFrm.obj
 0001:0007ce2c       __ehhandler$?SetServerGroup@CMainFrame@@IAEHXZ 0047de2c f   MainFrm.obj
 0001:0007ce60       __unwindfunclet$?DisplayMsg@CMainFrame@@QAEXPAXHH@Z$0 0047de60 f   MainFrm.obj
 0001:0007ce69       __unwindfunclet$?DisplayMsg@CMainFrame@@QAEXPAXHH@Z$1 0047de69 f   MainFrm.obj
 0001:0007ce72       __unwindfunclet$?DisplayMsg@CMainFrame@@QAEXPAXHH@Z$2 0047de72 f   MainFrm.obj
 0001:0007ce7a       __unwindfunclet$?DisplayMsg@CMainFrame@@QAEXPAXHH@Z$3 0047de7a f   MainFrm.obj
 0001:0007ce83       __unwindfunclet$?DisplayMsg@CMainFrame@@QAEXPAXHH@Z$4 0047de83 f   MainFrm.obj
 0001:0007ce8f       __unwindfunclet$?DisplayMsg@CMainFrame@@QAEXPAXHH@Z$5 0047de8f f   MainFrm.obj
 0001:0007ce9b       __unwindfunclet$?DisplayMsg@CMainFrame@@QAEXPAXHH@Z$6 0047de9b f   MainFrm.obj
 0001:0007cea7       __unwindfunclet$?DisplayMsg@CMainFrame@@QAEXPAXHH@Z$7 0047dea7 f   MainFrm.obj
 0001:0007ceb3       __unwindfunclet$?DisplayMsg@CMainFrame@@QAEXPAXHH@Z$8 0047deb3 f   MainFrm.obj
 0001:0007cebf       __unwindfunclet$?DisplayMsg@CMainFrame@@QAEXPAXHH@Z$9 0047debf f   MainFrm.obj
 0001:0007cecb       __unwindfunclet$?DisplayMsg@CMainFrame@@QAEXPAXHH@Z$10 0047decb f   MainFrm.obj
 0001:0007ced7       __unwindfunclet$?DisplayMsg@CMainFrame@@QAEXPAXHH@Z$11 0047ded7 f   MainFrm.obj
 0001:0007cee3       __ehhandler$?DisplayMsg@CMainFrame@@QAEXPAXHH@Z 0047dee3 f   MainFrm.obj
 0001:0007cf10       __unwindfunclet$?OnLockmouse@CMainFrame@@QAEXXZ$1 0047df10 f   MainFrm.obj
 0001:0007cf10       __unwindfunclet$?OnUnlockmouse@CMainFrame@@QAEXXZ$1 0047df10 f   MainFrm.obj
 0001:0007cf1c       __unwindfunclet$?OnUnlockmouse@CMainFrame@@QAEXXZ$2 0047df1c f   MainFrm.obj
 0001:0007cf1c       __unwindfunclet$?OnLockmouse@CMainFrame@@QAEXXZ$2 0047df1c f   MainFrm.obj
 0001:0007cf28       __unwindfunclet$?OnUnlockmouse@CMainFrame@@QAEXXZ$3 0047df28 f   MainFrm.obj
 0001:0007cf28       __unwindfunclet$?OnLockmouse@CMainFrame@@QAEXXZ$3 0047df28 f   MainFrm.obj
 0001:0007cf31       __unwindfunclet$?OnLockmouse@CMainFrame@@QAEXXZ$4 0047df31 f   MainFrm.obj
 0001:0007cf31       __unwindfunclet$?OnUnlockmouse@CMainFrame@@QAEXXZ$4 0047df31 f   MainFrm.obj
 0001:0007cf3d       __unwindfunclet$?OnLockmouse@CMainFrame@@QAEXXZ$5 0047df3d f   MainFrm.obj
 0001:0007cf3d       __unwindfunclet$?OnUnlockmouse@CMainFrame@@QAEXXZ$5 0047df3d f   MainFrm.obj
 0001:0007cf49       __unwindfunclet$?OnUnlockmouse@CMainFrame@@QAEXXZ$6 0047df49 f   MainFrm.obj
 0001:0007cf49       __unwindfunclet$?OnLockmouse@CMainFrame@@QAEXXZ$6 0047df49 f   MainFrm.obj
 0001:0007cf55       __unwindfunclet$?OnUnlockmouse@CMainFrame@@QAEXXZ$7 0047df55 f   MainFrm.obj
 0001:0007cf55       __unwindfunclet$?OnLockmouse@CMainFrame@@QAEXXZ$7 0047df55 f   MainFrm.obj
 0001:0007cf61       __unwindfunclet$?OnUnlockmouse@CMainFrame@@QAEXXZ$8 0047df61 f   MainFrm.obj
 0001:0007cf61       __unwindfunclet$?OnLockmouse@CMainFrame@@QAEXXZ$8 0047df61 f   MainFrm.obj
 0001:0007cf6d       __unwindfunclet$?OnUnlockmouse@CMainFrame@@QAEXXZ$9 0047df6d f   MainFrm.obj
 0001:0007cf6d       __unwindfunclet$?OnLockmouse@CMainFrame@@QAEXXZ$9 0047df6d f   MainFrm.obj
 0001:0007cf79       __unwindfunclet$?OnLockmouse@CMainFrame@@QAEXXZ$10 0047df79 f   MainFrm.obj
 0001:0007cf79       __unwindfunclet$?OnUnlockmouse@CMainFrame@@QAEXXZ$10 0047df79 f   MainFrm.obj
 0001:0007cf85       __ehhandler$?OnUnlockmouse@CMainFrame@@QAEXXZ 0047df85 f   MainFrm.obj
 0001:0007cf85       __ehhandler$?OnLockmouse@CMainFrame@@QAEXXZ 0047df85 f   MainFrm.obj
 0001:0007cfc0       __unwindfunclet$?OnLockkeyboard@CMainFrame@@QAEXXZ$1 0047dfc0 f   MainFrm.obj
 0001:0007cfc0       __unwindfunclet$?OnUnlockkeyboard@CMainFrame@@QAEXXZ$1 0047dfc0 f   MainFrm.obj
 0001:0007cfcc       __unwindfunclet$?OnUnlockkeyboard@CMainFrame@@QAEXXZ$2 0047dfcc f   MainFrm.obj
 0001:0007cfcc       __unwindfunclet$?OnLockkeyboard@CMainFrame@@QAEXXZ$2 0047dfcc f   MainFrm.obj
 0001:0007cfd8       __unwindfunclet$?OnUnlockkeyboard@CMainFrame@@QAEXXZ$3 0047dfd8 f   MainFrm.obj
 0001:0007cfd8       __unwindfunclet$?OnLockkeyboard@CMainFrame@@QAEXXZ$3 0047dfd8 f   MainFrm.obj
 0001:0007cfe1       __unwindfunclet$?OnLockkeyboard@CMainFrame@@QAEXXZ$4 0047dfe1 f   MainFrm.obj
 0001:0007cfe1       __unwindfunclet$?OnUnlockkeyboard@CMainFrame@@QAEXXZ$4 0047dfe1 f   MainFrm.obj
 0001:0007cfed       __unwindfunclet$?OnUnlockkeyboard@CMainFrame@@QAEXXZ$5 0047dfed f   MainFrm.obj
 0001:0007cfed       __unwindfunclet$?OnLockkeyboard@CMainFrame@@QAEXXZ$5 0047dfed f   MainFrm.obj
 0001:0007cff9       __unwindfunclet$?OnLockkeyboard@CMainFrame@@QAEXXZ$6 0047dff9 f   MainFrm.obj
 0001:0007cff9       __unwindfunclet$?OnUnlockkeyboard@CMainFrame@@QAEXXZ$6 0047dff9 f   MainFrm.obj
 0001:0007d005       __unwindfunclet$?OnLockkeyboard@CMainFrame@@QAEXXZ$7 0047e005 f   MainFrm.obj
 0001:0007d005       __unwindfunclet$?OnUnlockkeyboard@CMainFrame@@QAEXXZ$7 0047e005 f   MainFrm.obj
 0001:0007d011       __unwindfunclet$?OnUnlockkeyboard@CMainFrame@@QAEXXZ$8 0047e011 f   MainFrm.obj
 0001:0007d011       __unwindfunclet$?OnLockkeyboard@CMainFrame@@QAEXXZ$8 0047e011 f   MainFrm.obj
 0001:0007d01d       __unwindfunclet$?OnUnlockkeyboard@CMainFrame@@QAEXXZ$9 0047e01d f   MainFrm.obj
 0001:0007d01d       __unwindfunclet$?OnLockkeyboard@CMainFrame@@QAEXXZ$9 0047e01d f   MainFrm.obj
 0001:0007d029       __unwindfunclet$?OnUnlockkeyboard@CMainFrame@@QAEXXZ$10 0047e029 f   MainFrm.obj
 0001:0007d029       __unwindfunclet$?OnLockkeyboard@CMainFrame@@QAEXXZ$10 0047e029 f   MainFrm.obj
 0001:0007d035       __unwindfunclet$?OnUnlockkeyboard@CMainFrame@@QAEXXZ$11 0047e035 f   MainFrm.obj
 0001:0007d035       __unwindfunclet$?OnLockkeyboard@CMainFrame@@QAEXXZ$11 0047e035 f   MainFrm.obj
 0001:0007d041       __unwindfunclet$?OnUnlockkeyboard@CMainFrame@@QAEXXZ$12 0047e041 f   MainFrm.obj
 0001:0007d041       __unwindfunclet$?OnLockkeyboard@CMainFrame@@QAEXXZ$12 0047e041 f   MainFrm.obj
 0001:0007d04d       __ehhandler$?OnLockkeyboard@CMainFrame@@QAEXXZ 0047e04d f   MainFrm.obj
 0001:0007d04d       __ehhandler$?OnUnlockkeyboard@CMainFrame@@QAEXXZ 0047e04d f   MainFrm.obj
 0001:0007d080       __unwindfunclet$?OnSynTime@CMainFrame@@QAEXXZ$1 0047e080 f   MainFrm.obj
 0001:0007d08c       __unwindfunclet$?OnSynTime@CMainFrame@@QAEXXZ$2 0047e08c f   MainFrm.obj
 0001:0007d098       __unwindfunclet$?OnSynTime@CMainFrame@@QAEXXZ$3 0047e098 f   MainFrm.obj
 0001:0007d0a3       __unwindfunclet$?OnSynTime@CMainFrame@@QAEXXZ$4 0047e0a3 f   MainFrm.obj
 0001:0007d0af       __unwindfunclet$?OnSynTime@CMainFrame@@QAEXXZ$5 0047e0af f   MainFrm.obj
 0001:0007d0bb       __unwindfunclet$?OnSynTime@CMainFrame@@QAEXXZ$6 0047e0bb f   MainFrm.obj
 0001:0007d0c7       __unwindfunclet$?OnSynTime@CMainFrame@@QAEXXZ$7 0047e0c7 f   MainFrm.obj
 0001:0007d0d0       __unwindfunclet$?OnSynTime@CMainFrame@@QAEXXZ$8 0047e0d0 f   MainFrm.obj
 0001:0007d0dc       __unwindfunclet$?OnSynTime@CMainFrame@@QAEXXZ$9 0047e0dc f   MainFrm.obj
 0001:0007d0e8       __unwindfunclet$?OnSynTime@CMainFrame@@QAEXXZ$10 0047e0e8 f   MainFrm.obj
 0001:0007d0f4       __unwindfunclet$?OnSynTime@CMainFrame@@QAEXXZ$11 0047e0f4 f   MainFrm.obj
 0001:0007d100       __unwindfunclet$?OnSynTime@CMainFrame@@QAEXXZ$12 0047e100 f   MainFrm.obj
 0001:0007d10c       __unwindfunclet$?OnSynTime@CMainFrame@@QAEXXZ$13 0047e10c f   MainFrm.obj
 0001:0007d118       __unwindfunclet$?OnSynTime@CMainFrame@@QAEXXZ$14 0047e118 f   MainFrm.obj
 0001:0007d124       __unwindfunclet$?OnSynTime@CMainFrame@@QAEXXZ$15 0047e124 f   MainFrm.obj
 0001:0007d130       __unwindfunclet$?OnSynTime@CMainFrame@@QAEXXZ$16 0047e130 f   MainFrm.obj
 0001:0007d13c       __ehhandler$?OnSynTime@CMainFrame@@QAEXXZ 0047e13c f   MainFrm.obj
 0001:0007d170       __unwindfunclet$?HandleRemoteControlCmd@CMainFrame@@QAEXPAUtagRECVREQUEST@@@Z$0 0047e170 f   MainFrm.obj
 0001:0007d179       __unwindfunclet$?HandleRemoteControlCmd@CMainFrame@@QAEXPAUtagRECVREQUEST@@@Z$1 0047e179 f   MainFrm.obj
 0001:0007d182       __unwindfunclet$?HandleRemoteControlCmd@CMainFrame@@QAEXPAUtagRECVREQUEST@@@Z$2 0047e182 f   MainFrm.obj
 0001:0007d18e       __unwindfunclet$?HandleRemoteControlCmd@CMainFrame@@QAEXPAUtagRECVREQUEST@@@Z$3 0047e18e f   MainFrm.obj
 0001:0007d19a       __unwindfunclet$?HandleRemoteControlCmd@CMainFrame@@QAEXPAUtagRECVREQUEST@@@Z$4 0047e19a f   MainFrm.obj
 0001:0007d1a6       __unwindfunclet$?HandleRemoteControlCmd@CMainFrame@@QAEXPAUtagRECVREQUEST@@@Z$5 0047e1a6 f   MainFrm.obj
 0001:0007d1b2       __unwindfunclet$?HandleRemoteControlCmd@CMainFrame@@QAEXPAUtagRECVREQUEST@@@Z$6 0047e1b2 f   MainFrm.obj
 0001:0007d1be       __unwindfunclet$?HandleRemoteControlCmd@CMainFrame@@QAEXPAUtagRECVREQUEST@@@Z$7 0047e1be f   MainFrm.obj
 0001:0007d1ca       __ehhandler$?HandleRemoteControlCmd@CMainFrame@@QAEXPAUtagRECVREQUEST@@@Z 0047e1ca f   MainFrm.obj
 0001:0007d200       __unwindfunclet$?OnPortLock@CMainFrame@@QAEXXZ$1 0047e200 f   MainFrm.obj
 0001:0007d209       __unwindfunclet$?OnPortLock@CMainFrame@@QAEXXZ$2 0047e209 f   MainFrm.obj
 0001:0007d212       __unwindfunclet$?OnPortLock@CMainFrame@@QAEXXZ$3 0047e212 f   MainFrm.obj
 0001:0007d21b       __unwindfunclet$?OnPortLock@CMainFrame@@QAEXXZ$4 0047e21b f   MainFrm.obj
 0001:0007d224       __unwindfunclet$?OnPortLock@CMainFrame@@QAEXXZ$5 0047e224 f   MainFrm.obj
 0001:0007d22d       __unwindfunclet$?OnPortLock@CMainFrame@@QAEXXZ$6 0047e22d f   MainFrm.obj
 0001:0007d236       __unwindfunclet$?OnPortLock@CMainFrame@@QAEXXZ$7 0047e236 f   MainFrm.obj
 0001:0007d23f       __unwindfunclet$?OnPortLock@CMainFrame@@QAEXXZ$8 0047e23f f   MainFrm.obj
 0001:0007d248       __ehhandler$?OnPortLock@CMainFrame@@QAEXXZ 0047e248 f   MainFrm.obj
 0001:0007d270       __unwindfunclet$?OnSaveHistorymsg@CMainFrame@@QAEXXZ$0 0047e270 f   MainFrm.obj
 0001:0007d270       __unwindfunclet$?OnViewMaindlg@CMainFrame@@QAEXXZ$0 0047e270 f   MainFrm.obj
 0001:0007d278       __ehhandler$?OnViewMaindlg@CMainFrame@@QAEXXZ 0047e278 f   MainFrm.obj
 0001:0007d278       __ehhandler$?OnSaveHistorymsg@CMainFrame@@QAEXXZ 0047e278 f   MainFrm.obj
 0001:0007d2a0       __unwindfunclet$?_GetPortInfoThread@CMainFrame@@SAIPAX@Z$0 0047e2a0 f   MainFrm.obj
 0001:0007d2a9       __unwindfunclet$?_GetPortInfoThread@CMainFrame@@SAIPAX@Z$1 0047e2a9 f   MainFrm.obj
 0001:0007d2b5       __unwindfunclet$?_GetPortInfoThread@CMainFrame@@SAIPAX@Z$2 0047e2b5 f   MainFrm.obj
 0001:0007d2c1       __unwindfunclet$?_GetPortInfoThread@CMainFrame@@SAIPAX@Z$3 0047e2c1 f   MainFrm.obj
 0001:0007d2cd       __ehhandler$?_GetPortInfoThread@CMainFrame@@SAIPAX@Z 0047e2cd f   MainFrm.obj
 0001:0007d300       __unwindfunclet$?AddRemoveTray@CMainFrame@@QAEHH@Z$0 0047e300 f   MainFrm.obj
 0001:0007d309       __unwindfunclet$?AddRemoveTray@CMainFrame@@QAEHH@Z$1 0047e309 f   MainFrm.obj
 0001:0007d315       __unwindfunclet$?AddRemoveTray@CMainFrame@@QAEHH@Z$2 0047e315 f   MainFrm.obj
 0001:0007d321       __unwindfunclet$?AddRemoveTray@CMainFrame@@QAEHH@Z$3 0047e321 f   MainFrm.obj
 0001:0007d32d       __unwindfunclet$?AddRemoveTray@CMainFrame@@QAEHH@Z$4 0047e32d f   MainFrm.obj
 0001:0007d339       __unwindfunclet$?AddRemoveTray@CMainFrame@@QAEHH@Z$5 0047e339 f   MainFrm.obj
 0001:0007d345       __unwindfunclet$?AddRemoveTray@CMainFrame@@QAEHH@Z$6 0047e345 f   MainFrm.obj
 0001:0007d351       __ehhandler$?AddRemoveTray@CMainFrame@@QAEHH@Z 0047e351 f   MainFrm.obj
 0001:0007d380       __unwindfunclet$?DisplayMenu@CMainFrame@@QAEXXZ$0 0047e380 f   MainFrm.obj
 0001:0007d388       __unwindfunclet$?DisplayMenu@CMainFrame@@QAEXXZ$1 0047e388 f   MainFrm.obj
 0001:0007d392       __ehhandler$?DisplayMenu@CMainFrame@@QAEXXZ 0047e392 f   MainFrm.obj
 0001:0007d3b0       __unwindfunclet$?OnAppAbout@CMainFrame@@QAEXXZ$0 0047e3b0 f   MainFrm.obj
 0001:0007d3b0       __unwindfunclet$?OnRegisterLocal@CMainFrame@@QAEXXZ$0 0047e3b0 f   MainFrm.obj
 0001:0007d3bb       __ehhandler$?OnRegisterLocal@CMainFrame@@QAEXXZ 0047e3bb f   MainFrm.obj
 0001:0007d3bb       __ehhandler$?OnAppAbout@CMainFrame@@QAEXXZ 0047e3bb f   MainFrm.obj
 0001:0007d3e0       __unwindfunclet$?_InitPortThread@CPortCtrlDlg@@SAIPAX@Z$0 0047e3e0 f   MainFrm.obj
 0001:0007d3e0       __unwindfunclet$?OnHelp@CMainFrame@@QAEXXZ$0 0047e3e0 f   MainFrm.obj
 0001:0007d3e9       __ehhandler$?_InitPortThread@CPortCtrlDlg@@SAIPAX@Z 0047e3e9 f   MainFrm.obj
 0001:0007d3e9       __ehhandler$?OnHelp@CMainFrame@@QAEXXZ 0047e3e9 f   MainFrm.obj
 0001:0007d410       __unwindfunclet$?OnBroadclass@CMainFrame@@QAEXXZ$0 0047e410 f   MainFrm.obj
 0001:0007d41c       __unwindfunclet$?OnBroadclass@CMainFrame@@QAEXXZ$2 0047e41c f   MainFrm.obj
 0001:0007d428       __unwindfunclet$?OnBroadclass@CMainFrame@@QAEXXZ$3 0047e428 f   MainFrm.obj
 0001:0007d434       __unwindfunclet$?OnBroadclass@CMainFrame@@QAEXXZ$4 0047e434 f   MainFrm.obj
 0001:0007d440       __unwindfunclet$?OnBroadclass@CMainFrame@@QAEXXZ$6 0047e440 f   MainFrm.obj
 0001:0007d44b       __unwindfunclet$?OnBroadclass@CMainFrame@@QAEXXZ$7 0047e44b f   MainFrm.obj
 0001:0007d457       __unwindfunclet$?OnBroadclass@CMainFrame@@QAEXXZ$8 0047e457 f   MainFrm.obj
 0001:0007d463       __unwindfunclet$?OnBroadclass@CMainFrame@@QAEXXZ$9 0047e463 f   MainFrm.obj
 0001:0007d46f       __unwindfunclet$?OnBroadclass@CMainFrame@@QAEXXZ$10 0047e46f f   MainFrm.obj
 0001:0007d47b       __unwindfunclet$?OnBroadclass@CMainFrame@@QAEXXZ$12 0047e47b f   MainFrm.obj
 0001:0007d487       __unwindfunclet$?OnBroadclass@CMainFrame@@QAEXXZ$14 0047e487 f   MainFrm.obj
 0001:0007d490       __unwindfunclet$?OnBroadclass@CMainFrame@@QAEXXZ$15 0047e490 f   MainFrm.obj
 0001:0007d49c       __unwindfunclet$?OnBroadclass@CMainFrame@@QAEXXZ$16 0047e49c f   MainFrm.obj
 0001:0007d4a8       __unwindfunclet$?OnBroadclass@CMainFrame@@QAEXXZ$17 0047e4a8 f   MainFrm.obj
 0001:0007d4b4       __unwindfunclet$?OnBroadclass@CMainFrame@@QAEXXZ$18 0047e4b4 f   MainFrm.obj
 0001:0007d4c0       __unwindfunclet$?OnBroadclass@CMainFrame@@QAEXXZ$19 0047e4c0 f   MainFrm.obj
 0001:0007d4cc       __unwindfunclet$?OnBroadclass@CMainFrame@@QAEXXZ$20 0047e4cc f   MainFrm.obj
 0001:0007d4d8       __unwindfunclet$?OnBroadclass@CMainFrame@@QAEXXZ$21 0047e4d8 f   MainFrm.obj
 0001:0007d4e4       __unwindfunclet$?OnBroadclass@CMainFrame@@QAEXXZ$22 0047e4e4 f   MainFrm.obj
 0001:0007d4f0       __unwindfunclet$?OnBroadclass@CMainFrame@@QAEXXZ$23 0047e4f0 f   MainFrm.obj
 0001:0007d4fb       __unwindfunclet$?OnBroadclass@CMainFrame@@QAEXXZ$26 0047e4fb f   MainFrm.obj
 0001:0007d507       __unwindfunclet$?OnBroadclass@CMainFrame@@QAEXXZ$27 0047e507 f   MainFrm.obj
 0001:0007d513       __unwindfunclet$?OnBroadclass@CMainFrame@@QAEXXZ$28 0047e513 f   MainFrm.obj
 0001:0007d51f       __unwindfunclet$?OnBroadclass@CMainFrame@@QAEXXZ$30 0047e51f f   MainFrm.obj
 0001:0007d52b       __unwindfunclet$?OnBroadclass@CMainFrame@@QAEXXZ$31 0047e52b f   MainFrm.obj
 0001:0007d537       __unwindfunclet$?OnBroadclass@CMainFrame@@QAEXXZ$32 0047e537 f   MainFrm.obj
 0001:0007d543       __unwindfunclet$?OnBroadclass@CMainFrame@@QAEXXZ$34 0047e543 f   MainFrm.obj
 0001:0007d54f       __ehhandler$?OnBroadclass@CMainFrame@@QAEXXZ 0047e54f f   MainFrm.obj
 0001:0007d580       __unwindfunclet$?InitializeBroadClass@CMainFrame@@QAEXXZ$0 0047e580 f   MainFrm.obj
 0001:0007d589       __unwindfunclet$?InitializeBroadClass@CMainFrame@@QAEXXZ$1 0047e589 f   MainFrm.obj
 0001:0007d592       __unwindfunclet$?InitializeBroadClass@CMainFrame@@QAEXXZ$2 0047e592 f   MainFrm.obj
 0001:0007d59c       __unwindfunclet$?InitializeBroadClass@CMainFrame@@QAEXXZ$3 0047e59c f   MainFrm.obj
 0001:0007d5b6       __unwindfunclet$?InitializeBroadClass@CMainFrame@@QAEXXZ$4 0047e5b6 f   MainFrm.obj
 0001:0007d5bf       __unwindfunclet$?InitializeBroadClass@CMainFrame@@QAEXXZ$5 0047e5bf f   MainFrm.obj
 0001:0007d5c8       __unwindfunclet$?InitializeBroadClass@CMainFrame@@QAEXXZ$6 0047e5c8 f   MainFrm.obj
 0001:0007d5d1       __unwindfunclet$?InitializeBroadClass@CMainFrame@@QAEXXZ$7 0047e5d1 f   MainFrm.obj
 0001:0007d5db       __unwindfunclet$?InitializeBroadClass@CMainFrame@@QAEXXZ$8 0047e5db f   MainFrm.obj
 0001:0007d5f5       __unwindfunclet$?InitializeBroadClass@CMainFrame@@QAEXXZ$9 0047e5f5 f   MainFrm.obj
 0001:0007d5fe       __unwindfunclet$?InitializeBroadClass@CMainFrame@@QAEXXZ$10 0047e5fe f   MainFrm.obj
 0001:0007d607       __unwindfunclet$?InitializeBroadClass@CMainFrame@@QAEXXZ$11 0047e607 f   MainFrm.obj
 0001:0007d610       __unwindfunclet$?InitializeBroadClass@CMainFrame@@QAEXXZ$12 0047e610 f   MainFrm.obj
 0001:0007d61a       __unwindfunclet$?InitializeBroadClass@CMainFrame@@QAEXXZ$13 0047e61a f   MainFrm.obj
 0001:0007d634       __unwindfunclet$?InitializeBroadClass@CMainFrame@@QAEXXZ$14 0047e634 f   MainFrm.obj
 0001:0007d63d       __unwindfunclet$?InitializeBroadClass@CMainFrame@@QAEXXZ$15 0047e63d f   MainFrm.obj
 0001:0007d646       __unwindfunclet$?InitializeBroadClass@CMainFrame@@QAEXXZ$16 0047e646 f   MainFrm.obj
 0001:0007d64f       __ehhandler$?InitializeBroadClass@CMainFrame@@QAEXXZ 0047e64f f   MainFrm.obj
 0001:0007d670       __unwindfunclet$?OnStopbroadclass@CMainFrame@@QAEXXZ$1 0047e670 f   MainFrm.obj
 0001:0007d67c       __unwindfunclet$?OnStopbroadclass@CMainFrame@@QAEXXZ$2 0047e67c f   MainFrm.obj
 0001:0007d688       __unwindfunclet$?OnStopbroadclass@CMainFrame@@QAEXXZ$4 0047e688 f   MainFrm.obj
 0001:0007d691       __unwindfunclet$?OnStopbroadclass@CMainFrame@@QAEXXZ$5 0047e691 f   MainFrm.obj
 0001:0007d69a       __unwindfunclet$?OnStopbroadclass@CMainFrame@@QAEXXZ$6 0047e69a f   MainFrm.obj
 0001:0007d6a6       __unwindfunclet$?OnStopbroadclass@CMainFrame@@QAEXXZ$7 0047e6a6 f   MainFrm.obj
 0001:0007d6b2       __unwindfunclet$?OnStopbroadclass@CMainFrame@@QAEXXZ$8 0047e6b2 f   MainFrm.obj
 0001:0007d6be       __unwindfunclet$?OnStopbroadclass@CMainFrame@@QAEXXZ$9 0047e6be f   MainFrm.obj
 0001:0007d6ca       __unwindfunclet$?OnStopbroadclass@CMainFrame@@QAEXXZ$10 0047e6ca f   MainFrm.obj
 0001:0007d6d6       __unwindfunclet$?OnStopbroadclass@CMainFrame@@QAEXXZ$11 0047e6d6 f   MainFrm.obj
 0001:0007d6e2       __unwindfunclet$?OnStopbroadclass@CMainFrame@@QAEXXZ$12 0047e6e2 f   MainFrm.obj
 0001:0007d6ee       __ehhandler$?OnStopbroadclass@CMainFrame@@QAEXXZ 0047e6ee f   MainFrm.obj
 0001:0007d720       __unwindfunclet$?OnStudentdemo@CMainFrame@@QAEXXZ$0 0047e720 f   MainFrm.obj
 0001:0007d72c       __unwindfunclet$?OnStudentdemo@CMainFrame@@QAEXXZ$1 0047e72c f   MainFrm.obj
 0001:0007d735       __unwindfunclet$?OnStudentdemo@CMainFrame@@QAEXXZ$2 0047e735 f   MainFrm.obj
 0001:0007d73e       __unwindfunclet$?OnStudentdemo@CMainFrame@@QAEXXZ$4 0047e73e f   MainFrm.obj
 0001:0007d74a       __unwindfunclet$?OnStudentdemo@CMainFrame@@QAEXXZ$5 0047e74a f   MainFrm.obj
 0001:0007d756       __unwindfunclet$?OnStudentdemo@CMainFrame@@QAEXXZ$6 0047e756 f   MainFrm.obj
 0001:0007d762       __unwindfunclet$?OnStudentdemo@CMainFrame@@QAEXXZ$7 0047e762 f   MainFrm.obj
 0001:0007d76e       __unwindfunclet$?OnStudentdemo@CMainFrame@@QAEXXZ$8 0047e76e f   MainFrm.obj
 0001:0007d77a       __unwindfunclet$?OnStudentdemo@CMainFrame@@QAEXXZ$9 0047e77a f   MainFrm.obj
 0001:0007d786       __unwindfunclet$?OnStudentdemo@CMainFrame@@QAEXXZ$10 0047e786 f   MainFrm.obj
 0001:0007d792       __unwindfunclet$?OnStudentdemo@CMainFrame@@QAEXXZ$12 0047e792 f   MainFrm.obj
 0001:0007d79d       __unwindfunclet$?OnStudentdemo@CMainFrame@@QAEXXZ$13 0047e79d f   MainFrm.obj
 0001:0007d7a9       __unwindfunclet$?OnStudentdemo@CMainFrame@@QAEXXZ$14 0047e7a9 f   MainFrm.obj
 0001:0007d7b5       __unwindfunclet$?OnStudentdemo@CMainFrame@@QAEXXZ$15 0047e7b5 f   MainFrm.obj
 0001:0007d7c1       __unwindfunclet$?OnStudentdemo@CMainFrame@@QAEXXZ$16 0047e7c1 f   MainFrm.obj
 0001:0007d7cd       __unwindfunclet$?OnStudentdemo@CMainFrame@@QAEXXZ$18 0047e7cd f   MainFrm.obj
 0001:0007d7d9       __unwindfunclet$?OnStudentdemo@CMainFrame@@QAEXXZ$20 0047e7d9 f   MainFrm.obj
 0001:0007d7e5       __unwindfunclet$?OnStudentdemo@CMainFrame@@QAEXXZ$21 0047e7e5 f   MainFrm.obj
 0001:0007d7f1       __unwindfunclet$?OnStudentdemo@CMainFrame@@QAEXXZ$22 0047e7f1 f   MainFrm.obj
 0001:0007d7fd       __unwindfunclet$?OnStudentdemo@CMainFrame@@QAEXXZ$23 0047e7fd f   MainFrm.obj
 0001:0007d809       __unwindfunclet$?OnStudentdemo@CMainFrame@@QAEXXZ$24 0047e809 f   MainFrm.obj
 0001:0007d815       __unwindfunclet$?OnStudentdemo@CMainFrame@@QAEXXZ$25 0047e815 f   MainFrm.obj
 0001:0007d821       __unwindfunclet$?OnStudentdemo@CMainFrame@@QAEXXZ$26 0047e821 f   MainFrm.obj
 0001:0007d82d       __unwindfunclet$?OnStudentdemo@CMainFrame@@QAEXXZ$27 0047e82d f   MainFrm.obj
 0001:0007d839       __unwindfunclet$?OnStudentdemo@CMainFrame@@QAEXXZ$28 0047e839 f   MainFrm.obj
 0001:0007d845       __unwindfunclet$?OnStudentdemo@CMainFrame@@QAEXXZ$29 0047e845 f   MainFrm.obj
 0001:0007d851       __unwindfunclet$?OnStudentdemo@CMainFrame@@QAEXXZ$30 0047e851 f   MainFrm.obj
 0001:0007d85d       __unwindfunclet$?OnStudentdemo@CMainFrame@@QAEXXZ$31 0047e85d f   MainFrm.obj
 0001:0007d869       __unwindfunclet$?OnStudentdemo@CMainFrame@@QAEXXZ$32 0047e869 f   MainFrm.obj
 0001:0007d875       __unwindfunclet$?OnStudentdemo@CMainFrame@@QAEXXZ$34 0047e875 f   MainFrm.obj
 0001:0007d881       __unwindfunclet$?OnStudentdemo@CMainFrame@@QAEXXZ$35 0047e881 f   MainFrm.obj
 0001:0007d88d       __unwindfunclet$?OnStudentdemo@CMainFrame@@QAEXXZ$36 0047e88d f   MainFrm.obj
 0001:0007d899       __unwindfunclet$?OnStudentdemo@CMainFrame@@QAEXXZ$38 0047e899 f   MainFrm.obj
 0001:0007d8a5       __unwindfunclet$?OnStudentdemo@CMainFrame@@QAEXXZ$39 0047e8a5 f   MainFrm.obj
 0001:0007d8b1       __ehhandler$?OnStudentdemo@CMainFrame@@QAEXXZ 0047e8b1 f   MainFrm.obj
 0001:0007d8e0       __unwindfunclet$?OnStopstudentdemo@CMainFrame@@QAEXXZ$1 0047e8e0 f   MainFrm.obj
 0001:0007d8ec       __unwindfunclet$?OnStopstudentdemo@CMainFrame@@QAEXXZ$2 0047e8ec f   MainFrm.obj
 0001:0007d8f8       __unwindfunclet$?OnStopstudentdemo@CMainFrame@@QAEXXZ$3 0047e8f8 f   MainFrm.obj
 0001:0007d901       __unwindfunclet$?OnStopstudentdemo@CMainFrame@@QAEXXZ$4 0047e901 f   MainFrm.obj
 0001:0007d90a       __unwindfunclet$?OnStopstudentdemo@CMainFrame@@QAEXXZ$5 0047e90a f   MainFrm.obj
 0001:0007d916       __unwindfunclet$?OnStopstudentdemo@CMainFrame@@QAEXXZ$6 0047e916 f   MainFrm.obj
 0001:0007d922       __unwindfunclet$?OnStopstudentdemo@CMainFrame@@QAEXXZ$7 0047e922 f   MainFrm.obj
 0001:0007d92e       __unwindfunclet$?OnStopstudentdemo@CMainFrame@@QAEXXZ$8 0047e92e f   MainFrm.obj
 0001:0007d93a       __ehhandler$?OnStopstudentdemo@CMainFrame@@QAEXXZ 0047e93a f   MainFrm.obj
 0001:0007d970       __unwindfunclet$?OnUpdateStudentdemo@CMainFrame@@QAEXPAVCCmdUI@@@Z$0 0047e970 f   MainFrm.obj
 0001:0007d970       __unwindfunclet$?OnUpdateBroadclass@CMainFrame@@QAEXPAVCCmdUI@@@Z$0 0047e970 f   MainFrm.obj
 0001:0007d979       __unwindfunclet$?OnUpdateStudentdemo@CMainFrame@@QAEXPAVCCmdUI@@@Z$1 0047e979 f   MainFrm.obj
 0001:0007d979       __unwindfunclet$?OnUpdateBroadclass@CMainFrame@@QAEXPAVCCmdUI@@@Z$1 0047e979 f   MainFrm.obj
 0001:0007d982       __ehhandler$?OnUpdateStudentdemo@CMainFrame@@QAEXPAVCCmdUI@@@Z 0047e982 f   MainFrm.obj
 0001:0007d982       __ehhandler$?OnUpdateBroadclass@CMainFrame@@QAEXPAVCCmdUI@@@Z 0047e982 f   MainFrm.obj
 0001:0007d9a0       __unwindfunclet$?OnProtectmode@CMainFrame@@QAEXXZ$1 0047e9a0 f   MainFrm.obj
 0001:0007d9a0       __unwindfunclet$?OnExammode@CMainFrame@@QAEXXZ$1 0047e9a0 f   MainFrm.obj
 0001:0007d9a0       __unwindfunclet$?OnOpenmode@CMainFrame@@QAEXXZ$1 0047e9a0 f   MainFrm.obj
 0001:0007d9ac       __unwindfunclet$?OnExammode@CMainFrame@@QAEXXZ$2 0047e9ac f   MainFrm.obj
 0001:0007d9ac       __unwindfunclet$?OnOpenmode@CMainFrame@@QAEXXZ$2 0047e9ac f   MainFrm.obj
 0001:0007d9ac       __unwindfunclet$?OnProtectmode@CMainFrame@@QAEXXZ$2 0047e9ac f   MainFrm.obj
 0001:0007d9b8       __unwindfunclet$?OnOpenmode@CMainFrame@@QAEXXZ$3 0047e9b8 f   MainFrm.obj
 0001:0007d9b8       __unwindfunclet$?OnExammode@CMainFrame@@QAEXXZ$3 0047e9b8 f   MainFrm.obj
 0001:0007d9b8       __unwindfunclet$?OnProtectmode@CMainFrame@@QAEXXZ$3 0047e9b8 f   MainFrm.obj
 0001:0007d9c1       __unwindfunclet$?OnExammode@CMainFrame@@QAEXXZ$4 0047e9c1 f   MainFrm.obj
 0001:0007d9c1       __unwindfunclet$?OnProtectmode@CMainFrame@@QAEXXZ$4 0047e9c1 f   MainFrm.obj
 0001:0007d9c1       __unwindfunclet$?OnOpenmode@CMainFrame@@QAEXXZ$4 0047e9c1 f   MainFrm.obj
 0001:0007d9cd       __unwindfunclet$?OnProtectmode@CMainFrame@@QAEXXZ$5 0047e9cd f   MainFrm.obj
 0001:0007d9cd       __unwindfunclet$?OnOpenmode@CMainFrame@@QAEXXZ$5 0047e9cd f   MainFrm.obj
 0001:0007d9cd       __unwindfunclet$?OnExammode@CMainFrame@@QAEXXZ$5 0047e9cd f   MainFrm.obj
 0001:0007d9d9       __unwindfunclet$?OnOpenmode@CMainFrame@@QAEXXZ$6 0047e9d9 f   MainFrm.obj
 0001:0007d9d9       __unwindfunclet$?OnProtectmode@CMainFrame@@QAEXXZ$6 0047e9d9 f   MainFrm.obj
 0001:0007d9d9       __unwindfunclet$?OnExammode@CMainFrame@@QAEXXZ$6 0047e9d9 f   MainFrm.obj
 0001:0007d9e5       __unwindfunclet$?OnOpenmode@CMainFrame@@QAEXXZ$7 0047e9e5 f   MainFrm.obj
 0001:0007d9e5       __unwindfunclet$?OnProtectmode@CMainFrame@@QAEXXZ$7 0047e9e5 f   MainFrm.obj
 0001:0007d9e5       __unwindfunclet$?OnExammode@CMainFrame@@QAEXXZ$7 0047e9e5 f   MainFrm.obj
 0001:0007d9f1       __unwindfunclet$?OnExammode@CMainFrame@@QAEXXZ$8 0047e9f1 f   MainFrm.obj
 0001:0007d9f1       __unwindfunclet$?OnProtectmode@CMainFrame@@QAEXXZ$8 0047e9f1 f   MainFrm.obj
 0001:0007d9f1       __unwindfunclet$?OnOpenmode@CMainFrame@@QAEXXZ$8 0047e9f1 f   MainFrm.obj
 0001:0007d9fd       __unwindfunclet$?OnExammode@CMainFrame@@QAEXXZ$9 0047e9fd f   MainFrm.obj
 0001:0007d9fd       __unwindfunclet$?OnOpenmode@CMainFrame@@QAEXXZ$9 0047e9fd f   MainFrm.obj
 0001:0007d9fd       __unwindfunclet$?OnProtectmode@CMainFrame@@QAEXXZ$9 0047e9fd f   MainFrm.obj
 0001:0007da09       __unwindfunclet$?OnProtectmode@CMainFrame@@QAEXXZ$10 0047ea09 f   MainFrm.obj
 0001:0007da09       __unwindfunclet$?OnOpenmode@CMainFrame@@QAEXXZ$10 0047ea09 f   MainFrm.obj
 0001:0007da09       __unwindfunclet$?OnExammode@CMainFrame@@QAEXXZ$10 0047ea09 f   MainFrm.obj
 0001:0007da15       __ehhandler$?OnExammode@CMainFrame@@QAEXXZ 0047ea15 f   MainFrm.obj
 0001:0007da15       __ehhandler$?OnProtectmode@CMainFrame@@QAEXXZ 0047ea15 f   MainFrm.obj
 0001:0007da15       __ehhandler$?OnOpenmode@CMainFrame@@QAEXXZ 0047ea15 f   MainFrm.obj
 0001:0007da40       __unwindfunclet$?OnNetvideo@CMainFrame@@QAEXXZ$1 0047ea40 f   MainFrm.obj
 0001:0007da40       __unwindfunclet$?OnTransfile@CMainFrame@@QAEXXZ$1 0047ea40 f   MainFrm.obj
 0001:0007da4c       __unwindfunclet$?OnNetvideo@CMainFrame@@QAEXXZ$2 0047ea4c f   MainFrm.obj
 0001:0007da4c       __unwindfunclet$?OnTransfile@CMainFrame@@QAEXXZ$2 0047ea4c f   MainFrm.obj
 0001:0007da58       __unwindfunclet$?OnNetvideo@CMainFrame@@QAEXXZ$3 0047ea58 f   MainFrm.obj
 0001:0007da58       __unwindfunclet$?OnTransfile@CMainFrame@@QAEXXZ$3 0047ea58 f   MainFrm.obj
 0001:0007da64       __unwindfunclet$?OnTransfile@CMainFrame@@QAEXXZ$4 0047ea64 f   MainFrm.obj
 0001:0007da64       __unwindfunclet$?OnNetvideo@CMainFrame@@QAEXXZ$4 0047ea64 f   MainFrm.obj
 0001:0007da70       __unwindfunclet$?OnTransfile@CMainFrame@@QAEXXZ$5 0047ea70 f   MainFrm.obj
 0001:0007da70       __unwindfunclet$?OnNetvideo@CMainFrame@@QAEXXZ$5 0047ea70 f   MainFrm.obj
 0001:0007da7c       __unwindfunclet$?OnNetvideo@CMainFrame@@QAEXXZ$6 0047ea7c f   MainFrm.obj
 0001:0007da7c       __unwindfunclet$?OnTransfile@CMainFrame@@QAEXXZ$6 0047ea7c f   MainFrm.obj
 0001:0007da88       __unwindfunclet$?OnTransfile@CMainFrame@@QAEXXZ$7 0047ea88 f   MainFrm.obj
 0001:0007da88       __unwindfunclet$?OnNetvideo@CMainFrame@@QAEXXZ$7 0047ea88 f   MainFrm.obj
 0001:0007da94       __unwindfunclet$?OnNetvideo@CMainFrame@@QAEXXZ$8 0047ea94 f   MainFrm.obj
 0001:0007da94       __unwindfunclet$?OnTransfile@CMainFrame@@QAEXXZ$8 0047ea94 f   MainFrm.obj
 0001:0007daa0       __unwindfunclet$?OnNetvideo@CMainFrame@@QAEXXZ$9 0047eaa0 f   MainFrm.obj
 0001:0007daa0       __unwindfunclet$?OnTransfile@CMainFrame@@QAEXXZ$9 0047eaa0 f   MainFrm.obj
 0001:0007daac       __unwindfunclet$?OnTransfile@CMainFrame@@QAEXXZ$10 0047eaac f   MainFrm.obj
 0001:0007daac       __unwindfunclet$?OnNetvideo@CMainFrame@@QAEXXZ$10 0047eaac f   MainFrm.obj
 0001:0007dab8       __unwindfunclet$?OnTransfile@CMainFrame@@QAEXXZ$11 0047eab8 f   MainFrm.obj
 0001:0007dab8       __unwindfunclet$?OnNetvideo@CMainFrame@@QAEXXZ$11 0047eab8 f   MainFrm.obj
 0001:0007dac4       __unwindfunclet$?OnTransfile@CMainFrame@@QAEXXZ$12 0047eac4 f   MainFrm.obj
 0001:0007dac4       __unwindfunclet$?OnNetvideo@CMainFrame@@QAEXXZ$12 0047eac4 f   MainFrm.obj
 0001:0007dad0       __ehhandler$?OnNetvideo@CMainFrame@@QAEXXZ 0047ead0 f   MainFrm.obj
 0001:0007dad0       __ehhandler$?OnTransfile@CMainFrame@@QAEXXZ 0047ead0 f   MainFrm.obj
 0001:0007db00       __unwindfunclet$?OnMenuRemovehand@CMainFrame@@QAEXXZ$1 0047eb00 f   MainFrm.obj
 0001:0007db0c       __unwindfunclet$?OnMenuRemovehand@CMainFrame@@QAEXXZ$2 0047eb0c f   MainFrm.obj
 0001:0007db18       __unwindfunclet$?OnMenuRemovehand@CMainFrame@@QAEXXZ$3 0047eb18 f   MainFrm.obj
 0001:0007db21       __unwindfunclet$?OnMenuRemovehand@CMainFrame@@QAEXXZ$4 0047eb21 f   MainFrm.obj
 0001:0007db2d       __unwindfunclet$?OnMenuRemovehand@CMainFrame@@QAEXXZ$5 0047eb2d f   MainFrm.obj
 0001:0007db39       __unwindfunclet$?OnMenuRemovehand@CMainFrame@@QAEXXZ$6 0047eb39 f   MainFrm.obj
 0001:0007db45       __ehhandler$?OnMenuRemovehand@CMainFrame@@QAEXXZ 0047eb45 f   MainFrm.obj
 0001:0007db70       __unwindfunclet$?OnBroadIE@CMainFrame@@QAEXXZ$1 0047eb70 f   MainFrm.obj
 0001:0007db7c       __unwindfunclet$?OnBroadIE@CMainFrame@@QAEXXZ$2 0047eb7c f   MainFrm.obj
 0001:0007db88       __unwindfunclet$?OnBroadIE@CMainFrame@@QAEXXZ$3 0047eb88 f   MainFrm.obj
 0001:0007db91       __unwindfunclet$?OnBroadIE@CMainFrame@@QAEXXZ$4 0047eb91 f   MainFrm.obj
 0001:0007db9d       __unwindfunclet$?OnBroadIE@CMainFrame@@QAEXXZ$5 0047eb9d f   MainFrm.obj
 0001:0007dba9       __unwindfunclet$?OnBroadIE@CMainFrame@@QAEXXZ$6 0047eba9 f   MainFrm.obj
 0001:0007dbb5       __unwindfunclet$?OnBroadIE@CMainFrame@@QAEXXZ$7 0047ebb5 f   MainFrm.obj
 0001:0007dbc1       __unwindfunclet$?OnBroadIE@CMainFrame@@QAEXXZ$8 0047ebc1 f   MainFrm.obj
 0001:0007dbcd       __unwindfunclet$?OnBroadIE@CMainFrame@@QAEXXZ$9 0047ebcd f   MainFrm.obj
 0001:0007dbd9       __unwindfunclet$?OnBroadIE@CMainFrame@@QAEXXZ$10 0047ebd9 f   MainFrm.obj
 0001:0007dbe5       __unwindfunclet$?OnBroadIE@CMainFrame@@QAEXXZ$11 0047ebe5 f   MainFrm.obj
 0001:0007dbf0       __ehhandler$?OnBroadIE@CMainFrame@@QAEXXZ 0047ebf0 f   MainFrm.obj
 0001:0007dc10       __unwindfunclet$?InitFtpServer@CMainFrame@@QAE_NV?$CStringT@DV?$StrTraitMFC_DLL@DV?$ChTraitsCRT@D@ATL@@@@@ATL@@00I@Z$0 0047ec10 f   MainFrm.obj
 0001:0007dc19       __unwindfunclet$?InitFtpServer@CMainFrame@@QAE_NV?$CStringT@DV?$StrTraitMFC_DLL@DV?$ChTraitsCRT@D@ATL@@@@@ATL@@00I@Z$1 0047ec19 f   MainFrm.obj
 0001:0007dc22       __unwindfunclet$?InitFtpServer@CMainFrame@@QAE_NV?$CStringT@DV?$StrTraitMFC_DLL@DV?$ChTraitsCRT@D@ATL@@@@@ATL@@00I@Z$2 0047ec22 f   MainFrm.obj
 0001:0007dc2b       __unwindfunclet$?InitFtpServer@CMainFrame@@QAE_NV?$CStringT@DV?$StrTraitMFC_DLL@DV?$ChTraitsCRT@D@ATL@@@@@ATL@@00I@Z$3 0047ec2b f   MainFrm.obj
 0001:0007dc36       __unwindfunclet$?InitFtpServer@CMainFrame@@QAE_NV?$CStringT@DV?$StrTraitMFC_DLL@DV?$ChTraitsCRT@D@ATL@@@@@ATL@@00I@Z$4 0047ec36 f   MainFrm.obj
 0001:0007dc43       __ehhandler$?InitFtpServer@CMainFrame@@QAE_NV?$CStringT@DV?$StrTraitMFC_DLL@DV?$ChTraitsCRT@D@ATL@@@@@ATL@@00I@Z 0047ec43 f   MainFrm.obj
 0001:0007dc70       __unwindfunclet$?OnServersetting@CMainFrame@@QAEXXZ$0 0047ec70 f   MainFrm.obj
 0001:0007dc7b       __ehhandler$?OnServersetting@CMainFrame@@QAEXXZ 0047ec7b f   MainFrm.obj
 0001:0007dca0       __unwindfunclet$?InitializeCommonPanel@CMainFrame@@QAEXXZ$0 0047eca0 f   MainFrm.obj
 0001:0007dca9       __unwindfunclet$?InitializeCommonPanel@CMainFrame@@QAEXXZ$1 0047eca9 f   MainFrm.obj
 0001:0007dcb2       __unwindfunclet$?InitializeCommonPanel@CMainFrame@@QAEXXZ$2 0047ecb2 f   MainFrm.obj
 0001:0007dcbc       __unwindfunclet$?InitializeCommonPanel@CMainFrame@@QAEXXZ$3 0047ecbc f   MainFrm.obj
 0001:0007dcd6       __unwindfunclet$?InitializeCommonPanel@CMainFrame@@QAEXXZ$4 0047ecd6 f   MainFrm.obj
 0001:0007dce0       __unwindfunclet$?InitializeCommonPanel@CMainFrame@@QAEXXZ$5 0047ece0 f   MainFrm.obj
 0001:0007dcfa       __unwindfunclet$?InitializeCommonPanel@CMainFrame@@QAEXXZ$6 0047ecfa f   MainFrm.obj
 0001:0007dd04       __unwindfunclet$?InitializeCommonPanel@CMainFrame@@QAEXXZ$7 0047ed04 f   MainFrm.obj
 0001:0007dd1e       __unwindfunclet$?InitializeCommonPanel@CMainFrame@@QAEXXZ$8 0047ed1e f   MainFrm.obj
 0001:0007dd28       __unwindfunclet$?InitializeCommonPanel@CMainFrame@@QAEXXZ$9 0047ed28 f   MainFrm.obj
 0001:0007dd42       __ehhandler$?InitializeCommonPanel@CMainFrame@@QAEXXZ 0047ed42 f   MainFrm.obj
 0001:0007dd60       __unwindfunclet$?_CallRegisterProcess@CMainFrame@@SAIPAX@Z$0 0047ed60 f   MainFrm.obj
 0001:0007dd6c       __unwindfunclet$?_CallRegisterProcess@CMainFrame@@SAIPAX@Z$1 0047ed6c f   MainFrm.obj
 0001:0007dd78       __ehhandler$?_CallRegisterProcess@CMainFrame@@SAIPAX@Z 0047ed78 f   MainFrm.obj
 0001:0007dda0       __unwindfunclet$?CheckGroupRegister@CMainFrame@@QAEHV?$CStringT@DV?$StrTraitMFC_DLL@DV?$ChTraitsCRT@D@ATL@@@@@ATL@@AAH1@Z$0 0047eda0 f   MainFrm.obj
 0001:0007dda9       __unwindfunclet$?CheckGroupRegister@CMainFrame@@QAEHV?$CStringT@DV?$StrTraitMFC_DLL@DV?$ChTraitsCRT@D@ATL@@@@@ATL@@AAH1@Z$2 0047eda9 f   MainFrm.obj
 0001:0007ddb2       __ehhandler$?CheckGroupRegister@CMainFrame@@QAEHV?$CStringT@DV?$StrTraitMFC_DLL@DV?$ChTraitsCRT@D@ATL@@@@@ATL@@AAH1@Z 0047edb2 f   MainFrm.obj
 0001:0007ddd0       __unwindfunclet$?OnSetPort@CMainFrame@@QAEXXZ$0 0047edd0 f   MainFrm.obj
 0001:0007dddb       __unwindfunclet$?OnSetPort@CMainFrame@@QAEXXZ$2 0047eddb f   MainFrm.obj
 0001:0007dde6       __ehhandler$?OnSetPort@CMainFrame@@QAEXXZ 0047ede6 f   MainFrm.obj
 0001:0007de10       __unwindfunclet$?OnSetclientPort@CMainFrame@@QAEXXZ$0 0047ee10 f   MainFrm.obj
 0001:0007de1b       __unwindfunclet$?OnSetclientPort@CMainFrame@@QAEXXZ$3 0047ee1b f   MainFrm.obj
 0001:0007de27       __unwindfunclet$?OnSetclientPort@CMainFrame@@QAEXXZ$4 0047ee27 f   MainFrm.obj
 0001:0007de33       __unwindfunclet$?OnSetclientPort@CMainFrame@@QAEXXZ$5 0047ee33 f   MainFrm.obj
 0001:0007de3e       __unwindfunclet$?OnSetclientPort@CMainFrame@@QAEXXZ$6 0047ee3e f   MainFrm.obj
 0001:0007de47       __unwindfunclet$?OnSetclientPort@CMainFrame@@QAEXXZ$8 0047ee47 f   MainFrm.obj
 0001:0007de53       __unwindfunclet$?OnSetclientPort@CMainFrame@@QAEXXZ$9 0047ee53 f   MainFrm.obj
 0001:0007de5f       __unwindfunclet$?OnSetclientPort@CMainFrame@@QAEXXZ$10 0047ee5f f   MainFrm.obj
 0001:0007de6b       __unwindfunclet$?OnSetclientPort@CMainFrame@@QAEXXZ$11 0047ee6b f   MainFrm.obj
 0001:0007de77       __ehhandler$?OnSetclientPort@CMainFrame@@QAEXXZ 0047ee77 f   MainFrm.obj
 0001:0007deb0       __unwindfunclet$?OnNetworkSet@CMainFrame@@QAEXXZ$0 0047eeb0 f   MainFrm.obj
 0001:0007debb       __ehhandler$?OnNetworkSet@CMainFrame@@QAEXXZ 0047eebb f   MainFrm.obj
 0001:0007dee0       __unwindfunclet$?ReInitNetwrokComponent@CMainFrame@@QAEXXZ$2 0047eee0 f   MainFrm.obj
 0001:0007deec       __ehhandler$?ReInitNetwrokComponent@CMainFrame@@QAEXXZ 0047eeec f   MainFrm.obj
 0001:0007df20       __unwindfunclet$?CheckGUID@CMainFrame@@QAEHPADH0@Z$0 0047ef20 f   MainFrm.obj
 0001:0007df29       __unwindfunclet$?CheckGUID@CMainFrame@@QAEHPADH0@Z$2 0047ef29 f   MainFrm.obj
 0001:0007df32       __ehhandler$?CheckGUID@CMainFrame@@QAEHPADH0@Z 0047ef32 f   MainFrm.obj
 0001:0007df60       __unwindfunclet$?OnDisablecdrom@CMainFrame@@QAEHI@Z$1 0047ef60 f   MainFrm.obj
 0001:0007df6c       __unwindfunclet$?OnDisablecdrom@CMainFrame@@QAEHI@Z$2 0047ef6c f   MainFrm.obj
 0001:0007df78       __unwindfunclet$?OnDisablecdrom@CMainFrame@@QAEHI@Z$3 0047ef78 f   MainFrm.obj
 0001:0007df81       __unwindfunclet$?OnDisablecdrom@CMainFrame@@QAEHI@Z$4 0047ef81 f   MainFrm.obj
 0001:0007df8d       __unwindfunclet$?OnDisablecdrom@CMainFrame@@QAEHI@Z$5 0047ef8d f   MainFrm.obj
 0001:0007df99       __unwindfunclet$?OnDisablecdrom@CMainFrame@@QAEHI@Z$6 0047ef99 f   MainFrm.obj
 0001:0007dfa5       __unwindfunclet$?OnDisablecdrom@CMainFrame@@QAEHI@Z$7 0047efa5 f   MainFrm.obj
 0001:0007dfb1       __unwindfunclet$?OnDisablecdrom@CMainFrame@@QAEHI@Z$8 0047efb1 f   MainFrm.obj
 0001:0007dfbd       __unwindfunclet$?OnDisablecdrom@CMainFrame@@QAEHI@Z$9 0047efbd f   MainFrm.obj
 0001:0007dfc9       __unwindfunclet$?OnDisablecdrom@CMainFrame@@QAEHI@Z$10 0047efc9 f   MainFrm.obj
 0001:0007dfd5       __ehhandler$?OnDisablecdrom@CMainFrame@@QAEHI@Z 0047efd5 f   MainFrm.obj
 0001:0007e000       __unwindfunclet$?OnGroupset@CMainFrame@@QAEXXZ$1 0047f000 f   MainFrm.obj
 0001:0007e00c       __unwindfunclet$?OnGroupset@CMainFrame@@QAEXXZ$2 0047f00c f   MainFrm.obj
 0001:0007e018       __unwindfunclet$?OnGroupset@CMainFrame@@QAEXXZ$3 0047f018 f   MainFrm.obj
 0001:0007e023       __unwindfunclet$?OnGroupset@CMainFrame@@QAEXXZ$4 0047f023 f   MainFrm.obj
 0001:0007e02f       __unwindfunclet$?OnGroupset@CMainFrame@@QAEXXZ$5 0047f02f f   MainFrm.obj
 0001:0007e03b       __unwindfunclet$?OnGroupset@CMainFrame@@QAEXXZ$6 0047f03b f   MainFrm.obj
 0001:0007e047       __ehhandler$?OnGroupset@CMainFrame@@QAEXXZ 0047f047 f   MainFrm.obj
 0001:0007e070       __unwindfunclet$?OnRemoteRunprocedure@CMainFrame@@QAEXXZ$1 0047f070 f   MainFrm.obj
 0001:0007e07b       __unwindfunclet$?OnRemoteRunprocedure@CMainFrame@@QAEXXZ$2 0047f07b f   MainFrm.obj
 0001:0007e087       __unwindfunclet$?OnRemoteRunprocedure@CMainFrame@@QAEXXZ$3 0047f087 f   MainFrm.obj
 0001:0007e093       __unwindfunclet$?OnRemoteRunprocedure@CMainFrame@@QAEXXZ$5 0047f093 f   MainFrm.obj
 0001:0007e09f       __unwindfunclet$?OnRemoteRunprocedure@CMainFrame@@QAEXXZ$6 0047f09f f   MainFrm.obj
 0001:0007e0aa       __unwindfunclet$?OnRemoteRunprocedure@CMainFrame@@QAEXXZ$7 0047f0aa f   MainFrm.obj
 0001:0007e0b5       __unwindfunclet$?OnRemoteRunprocedure@CMainFrame@@QAEXXZ$8 0047f0b5 f   MainFrm.obj
 0001:0007e0c1       __unwindfunclet$?OnRemoteRunprocedure@CMainFrame@@QAEXXZ$9 0047f0c1 f   MainFrm.obj
 0001:0007e0cd       __ehhandler$?OnRemoteRunprocedure@CMainFrame@@QAEXXZ 0047f0cd f   MainFrm.obj
 0001:0007e100       __unwindfunclet$??1CWaitCursor@@QAE@XZ$2 0047f100 f   MainFrm.obj
 0001:0007e10c       __ehhandler$??1CWaitCursor@@QAE@XZ 0047f10c f   MainFrm.obj
 0001:0007e140       __unwindfunclet$??1CMFCRibbonApplicationButton@@UAE@XZ$0 0047f140 f   MainFrm.obj
 0001:0007e140       __unwindfunclet$??0CMFCRibbonApplicationButton@@QAE@XZ$0 0047f140 f   MainFrm.obj
 0001:0007e148       __ehhandler$??0CMFCRibbonApplicationButton@@QAE@XZ 0047f148 f   MainFrm.obj
 0001:0007e148       __ehhandler$??1CMFCRibbonApplicationButton@@UAE@XZ 0047f148 f   MainFrm.obj
 0001:0007e170       __unwindfunclet$?Serialize@?$CMap@V?$CStringT@DV?$StrTraitMFC_DLL@DV?$ChTraitsCRT@D@ATL@@@@@ATL@@PBDUItemInfo@@AAU3@@@UAEXAAVCArchive@@@Z$0 0047f170 f   MainFrm.obj
 0001:0007e184       __unwindfunclet$?Serialize@?$CMap@V?$CStringT@DV?$StrTraitMFC_DLL@DV?$ChTraitsCRT@D@ATL@@@@@ATL@@PBDUItemInfo@@AAU3@@@UAEXAAVCArchive@@@Z$1 0047f184 f   MainFrm.obj
 0001:0007e197       __ehhandler$?Serialize@?$CMap@V?$CStringT@DV?$StrTraitMFC_DLL@DV?$ChTraitsCRT@D@ATL@@@@@ATL@@PBDUItemInfo@@AAU3@@@UAEXAAVCArchive@@@Z 0047f197 f   MainFrm.obj
 0001:0007e1c0       __unwindfunclet$??1CMenu@@UAE@XZ$0 0047f1c0 f   MainFrm.obj
 0001:0007e1c0       __unwindfunclet$??1?$CList@PAVCFtpd@@PAV1@@@UAE@XZ$0 0047f1c0 f   MainFrm.obj
 0001:0007e1c0       __unwindfunclet$??1?$_Container_base_aux_alloc_real@V?$allocator@PAVCClientContext@@@std@@@std@@IAE@XZ$0 0047f1c0 f   MainFrm.obj
 0001:0007e1c0       __unwindfunclet$??1?$CMap@V?$CStringT@DV?$StrTraitMFC_DLL@DV?$ChTraitsCRT@D@ATL@@@@@ATL@@PBDUItemInfo@@AAU3@@@UAE@XZ$0 0047f1c0 f   MainFrm.obj
 0001:0007e1c0       __unwindfunclet$??1?$CList@PAVCFtpdPi@@PAV1@@@UAE@XZ$0 0047f1c0 f   MainFrm.obj
 0001:0007e1c0       __unwindfunclet$??1?$CList@II@@UAE@XZ$0 0047f1c0 f   MainFrm.obj
 0001:0007e1c8       __ehhandler$??1?$CList@PAVCFtpd@@PAV1@@@UAE@XZ 0047f1c8 f   MainFrm.obj
 0001:0007e1c8       __ehhandler$??1CMenu@@UAE@XZ 0047f1c8 f   MainFrm.obj
 0001:0007e1c8       __ehhandler$??1?$CList@PAVCFtpdPi@@PAV1@@@UAE@XZ 0047f1c8 f   MainFrm.obj
 0001:0007e1c8       __ehhandler$??1?$CList@II@@UAE@XZ 0047f1c8 f   MainFrm.obj
 0001:0007e1c8       __ehhandler$??1?$CMap@V?$CStringT@DV?$StrTraitMFC_DLL@DV?$ChTraitsCRT@D@ATL@@@@@ATL@@PBDUItemInfo@@AAU3@@@UAE@XZ 0047f1c8 f   MainFrm.obj
 0001:0007e1c8       __ehhandler$??1?$_Container_base_aux_alloc_real@V?$allocator@PAVCClientContext@@@std@@@std@@IAE@XZ 0047f1c8 f   MainFrm.obj
 0001:0007e1f0       __unwindfunclet$?NewAssoc@?$CMap@V?$CStringT@DV?$StrTraitMFC_DLL@DV?$ChTraitsCRT@D@ATL@@@@@ATL@@PBDUItemInfo@@AAU3@@@IAEPAVCAssoc@1@PBD@Z$0 0047f1f0 f   MainFrm.obj
 0001:0007e201       __ehhandler$?NewAssoc@?$CMap@V?$CStringT@DV?$StrTraitMFC_DLL@DV?$ChTraitsCRT@D@ATL@@@@@ATL@@PBDUItemInfo@@AAU3@@@IAEPAVCAssoc@1@PBD@Z 0047f201 f   MainFrm.obj
 0001:0007e220       __unwindfunclet$??0CModifyGroup@@QAE@PAVCWnd@@@Z$0 0047f220 f   ModifyGroup.obj
 0001:0007e228       __unwindfunclet$??0CModifyGroup@@QAE@PAVCWnd@@@Z$1 0047f228 f   ModifyGroup.obj
 0001:0007e233       __ehhandler$??0CModifyGroup@@QAE@PAVCWnd@@@Z 0047f233 f   ModifyGroup.obj
 0001:0007e250       __unwindfunclet$?OnInitDialog@CCheckPasswordDlg@@MAEHXZ$0 0047f250 f   ModifyGroup.obj
 0001:0007e250       __unwindfunclet$?OnInitDialog@CModifyGroup@@MAEHXZ$0 0047f250 f   ModifyGroup.obj
 0001:0007e250       __unwindfunclet$?SetTitle@CPortChannelDlg@@QAEXXZ$0 0047f250 f   ModifyGroup.obj
 0001:0007e259       __unwindfunclet$?OnInitDialog@CCheckPasswordDlg@@MAEHXZ$1 0047f259 f   ModifyGroup.obj
 0001:0007e259       __unwindfunclet$?SetTitle@CPortChannelDlg@@QAEXXZ$1 0047f259 f   ModifyGroup.obj
 0001:0007e259       __unwindfunclet$?OnInitDialog@CModifyGroup@@MAEHXZ$1 0047f259 f   ModifyGroup.obj
 0001:0007e262       __unwindfunclet$?OnInitDialog@CCheckPasswordDlg@@MAEHXZ$2 0047f262 f   ModifyGroup.obj
 0001:0007e262       __unwindfunclet$?OnInitDialog@CModifyGroup@@MAEHXZ$2 0047f262 f   ModifyGroup.obj
 0001:0007e262       __unwindfunclet$?SetTitle@CPortChannelDlg@@QAEXXZ$2 0047f262 f   ModifyGroup.obj
 0001:0007e26b       __unwindfunclet$?OnInitDialog@CCheckPasswordDlg@@MAEHXZ$3 0047f26b f   ModifyGroup.obj
 0001:0007e26b       __unwindfunclet$?OnInitDialog@CModifyGroup@@MAEHXZ$3 0047f26b f   ModifyGroup.obj
 0001:0007e26b       __unwindfunclet$?SetTitle@CPortChannelDlg@@QAEXXZ$3 0047f26b f   ModifyGroup.obj
 0001:0007e274       __unwindfunclet$?OnInitDialog@CCheckPasswordDlg@@MAEHXZ$4 0047f274 f   ModifyGroup.obj
 0001:0007e274       __unwindfunclet$?OnInitDialog@CModifyGroup@@MAEHXZ$4 0047f274 f   ModifyGroup.obj
 0001:0007e274       __unwindfunclet$?SetTitle@CPortChannelDlg@@QAEXXZ$4 0047f274 f   ModifyGroup.obj
 0001:0007e27d       __ehhandler$?OnInitDialog@CModifyGroup@@MAEHXZ 0047f27d f   ModifyGroup.obj
 0001:0007e27d       __ehhandler$?SetTitle@CPortChannelDlg@@QAEXXZ 0047f27d f   ModifyGroup.obj
 0001:0007e27d       __ehhandler$?OnInitDialog@CCheckPasswordDlg@@MAEHXZ 0047f27d f   ModifyGroup.obj
 0001:0007e2a0       __unwindfunclet$?CheckValid@CModifyGroup@@QAEHV?$CStringT@DV?$StrTraitMFC_DLL@DV?$ChTraitsCRT@D@ATL@@@@@ATL@@@Z$0 0047f2a0 f   ModifyGroup.obj
 0001:0007e2a9       __unwindfunclet$?CheckValid@CModifyGroup@@QAEHV?$CStringT@DV?$StrTraitMFC_DLL@DV?$ChTraitsCRT@D@ATL@@@@@ATL@@@Z$1 0047f2a9 f   ModifyGroup.obj
 0001:0007e2b2       __unwindfunclet$?CheckValid@CModifyGroup@@QAEHV?$CStringT@DV?$StrTraitMFC_DLL@DV?$ChTraitsCRT@D@ATL@@@@@ATL@@@Z$2 0047f2b2 f   ModifyGroup.obj
 0001:0007e2bb       __unwindfunclet$?CheckValid@CModifyGroup@@QAEHV?$CStringT@DV?$StrTraitMFC_DLL@DV?$ChTraitsCRT@D@ATL@@@@@ATL@@@Z$3 0047f2bb f   ModifyGroup.obj
 0001:0007e2c4       __unwindfunclet$?CheckValid@CModifyGroup@@QAEHV?$CStringT@DV?$StrTraitMFC_DLL@DV?$ChTraitsCRT@D@ATL@@@@@ATL@@@Z$4 0047f2c4 f   ModifyGroup.obj
 0001:0007e2cd       __ehhandler$?CheckValid@CModifyGroup@@QAEHV?$CStringT@DV?$StrTraitMFC_DLL@DV?$ChTraitsCRT@D@ATL@@@@@ATL@@@Z 0047f2cd f   ModifyGroup.obj
 0001:0007e2f0       __unwindfunclet$??0CMsgDlg@@QAE@PAVCWnd@@@Z$0 0047f2f0 f   MsgDlg.obj
 0001:0007e2f8       __unwindfunclet$??0CMsgDlg@@QAE@PAVCWnd@@@Z$1 0047f2f8 f   MsgDlg.obj
 0001:0007e304       __unwindfunclet$??0CMsgDlg@@QAE@PAVCWnd@@@Z$2 0047f304 f   MsgDlg.obj
 0001:0007e30f       __unwindfunclet$??0CMsgDlg@@QAE@PAVCWnd@@@Z$3 0047f30f f   MsgDlg.obj
 0001:0007e318       __ehhandler$??0CMsgDlg@@QAE@PAVCWnd@@@Z 0047f318 f   MsgDlg.obj
 0001:0007e340       __unwindfunclet$?OnInitDialog@CMsgDlg@@MAEHXZ$0 0047f340 f   MsgDlg.obj
 0001:0007e349       __unwindfunclet$?OnInitDialog@CMsgDlg@@MAEHXZ$1 0047f349 f   MsgDlg.obj
 0001:0007e352       __unwindfunclet$?OnInitDialog@CMsgDlg@@MAEHXZ$2 0047f352 f   MsgDlg.obj
 0001:0007e35b       __unwindfunclet$?OnInitDialog@CMsgDlg@@MAEHXZ$3 0047f35b f   MsgDlg.obj
 0001:0007e364       __ehhandler$?OnInitDialog@CMsgDlg@@MAEHXZ 0047f364 f   MsgDlg.obj
 0001:0007e390       __unwindfunclet$?OnBnClickedOk@CMsgDlg@@QAEXXZ$0 0047f390 f   MsgDlg.obj
 0001:0007e399       __unwindfunclet$?OnBnClickedOk@CMsgDlg@@QAEXXZ$1 0047f399 f   MsgDlg.obj
 0001:0007e3a5       __unwindfunclet$?OnBnClickedOk@CMsgDlg@@QAEXXZ$2 0047f3a5 f   MsgDlg.obj
 0001:0007e3b1       __unwindfunclet$?OnBnClickedOk@CMsgDlg@@QAEXXZ$3 0047f3b1 f   MsgDlg.obj
 0001:0007e3bd       __unwindfunclet$?OnBnClickedOk@CMsgDlg@@QAEXXZ$4 0047f3bd f   MsgDlg.obj
 0001:0007e3c9       __unwindfunclet$?OnBnClickedOk@CMsgDlg@@QAEXXZ$5 0047f3c9 f   MsgDlg.obj
 0001:0007e3d5       __unwindfunclet$?OnBnClickedOk@CMsgDlg@@QAEXXZ$6 0047f3d5 f   MsgDlg.obj
 0001:0007e3e1       __unwindfunclet$?OnBnClickedOk@CMsgDlg@@QAEXXZ$7 0047f3e1 f   MsgDlg.obj
 0001:0007e3ed       __unwindfunclet$?OnBnClickedOk@CMsgDlg@@QAEXXZ$8 0047f3ed f   MsgDlg.obj
 0001:0007e3f9       __unwindfunclet$?OnBnClickedOk@CMsgDlg@@QAEXXZ$10 0047f3f9 f   MsgDlg.obj
 0001:0007e405       __unwindfunclet$?OnBnClickedOk@CMsgDlg@@QAEXXZ$11 0047f405 f   MsgDlg.obj
 0001:0007e411       __unwindfunclet$?OnBnClickedOk@CMsgDlg@@QAEXXZ$12 0047f411 f   MsgDlg.obj
 0001:0007e41d       __unwindfunclet$?OnBnClickedOk@CMsgDlg@@QAEXXZ$13 0047f41d f   MsgDlg.obj
 0001:0007e429       __unwindfunclet$?OnBnClickedOk@CMsgDlg@@QAEXXZ$14 0047f429 f   MsgDlg.obj
 0001:0007e435       __unwindfunclet$?OnBnClickedOk@CMsgDlg@@QAEXXZ$15 0047f435 f   MsgDlg.obj
 0001:0007e441       __unwindfunclet$?OnBnClickedOk@CMsgDlg@@QAEXXZ$16 0047f441 f   MsgDlg.obj
 0001:0007e44d       __unwindfunclet$?OnBnClickedOk@CMsgDlg@@QAEXXZ$17 0047f44d f   MsgDlg.obj
 0001:0007e459       __unwindfunclet$?OnBnClickedOk@CMsgDlg@@QAEXXZ$19 0047f459 f   MsgDlg.obj
 0001:0007e465       __ehhandler$?OnBnClickedOk@CMsgDlg@@QAEXXZ 0047f465 f   MsgDlg.obj
 0001:0007e490       __unwindfunclet$?OnChar@CMyEdit@@IAEXIII@Z$0 0047f490 f   MyEdit.obj
 0001:0007e499       __unwindfunclet$?OnChar@CMyEdit@@IAEXIII@Z$2 0047f499 f   MyEdit.obj
 0001:0007e4a2       __ehhandler$?OnChar@CMyEdit@@IAEXIII@Z 0047f4a2 f   MyEdit.obj
 0001:0007e4c0       __unwindfunclet$?ChangeRectSize@CMyEdit@@QAEXUtagRECT@@0V?$CStringT@DV?$StrTraitMFC_DLL@DV?$ChTraitsCRT@D@ATL@@@@@ATL@@@Z$0 0047f4c0 f   MyEdit.obj
 0001:0007e4c9       __ehhandler$?ChangeRectSize@CMyEdit@@QAEXUtagRECT@@0V?$CStringT@DV?$StrTraitMFC_DLL@DV?$ChTraitsCRT@D@ATL@@@@@ATL@@@Z 0047f4c9 f   MyEdit.obj
 0001:0007e4f0       __unwindfunclet$?MyEidtBox@CMyEdit@@QAEXV?$CStringT@DV?$StrTraitMFC_DLL@DV?$ChTraitsCRT@D@ATL@@@@@ATL@@0IAAH@Z$0 0047f4f0 f   MyEdit.obj
 0001:0007e4f9       __unwindfunclet$?MyEidtBox@CMyEdit@@QAEXV?$CStringT@DV?$StrTraitMFC_DLL@DV?$ChTraitsCRT@D@ATL@@@@@ATL@@0IAAH@Z$1 0047f4f9 f   MyEdit.obj
 0001:0007e502       __ehhandler$?MyEidtBox@CMyEdit@@QAEXV?$CStringT@DV?$StrTraitMFC_DLL@DV?$ChTraitsCRT@D@ATL@@@@@ATL@@0IAAH@Z 0047f502 f   MyEdit.obj
 0001:0007e520       __unwindfunclet$?AcceptConnection@CMyIOCP@@QAEXI@Z$0 0047f520 f   MyIOCP.obj
 0001:0007e52e       __ehhandler$?AcceptConnection@CMyIOCP@@QAEXI@Z 0047f52e f   MyIOCP.obj
 0001:0007e560       __unwindfunclet$??0?$vector@PAVCClientContext@@V?$allocator@PAVCClientContext@@@std@@@std@@QAE@XZ$0 0047f560 f   MyIOCP.obj
 0001:0007e568       __ehhandler$??0?$vector@PAVCClientContext@@V?$allocator@PAVCClientContext@@@std@@@std@@QAE@XZ 0047f568 f   MyIOCP.obj
 0001:0007e590       __unwindfunclet$??1?$vector@PAVCClientContext@@V?$allocator@PAVCClientContext@@@std@@@std@@QAE@XZ$0 0047f590 f   MyIOCP.obj
 0001:0007e598       __ehhandler$??1?$vector@PAVCClientContext@@V?$allocator@PAVCClientContext@@@std@@@std@@QAE@XZ 0047f598 f   MyIOCP.obj
 0001:0007e5c0       __ehhandler$?_Insert_n@?$vector@PAVCClientContext@@V?$allocator@PAVCClientContext@@@std@@@std@@IAEXV?$_Vector_const_iterator@PAVCClientContext@@V?$allocator@PAVCClientContext@@@std@@@2@IABQAVCClientContext@@@Z 0047f5c0 f   MyIOCP.obj
 0001:0007e5e0       __unwindfunclet$?_Xlen@?$vector@PAVCClientContext@@V?$allocator@PAVCClientContext@@@std@@@std@@KAXXZ$0 0047f5e0 f   MyIOCP.obj
 0001:0007e5e9       __ehhandler$?_Xlen@?$vector@PAVCClientContext@@V?$allocator@PAVCClientContext@@@std@@@std@@KAXXZ 0047f5e9 f   MyIOCP.obj
 0001:0007e610       __unwindfunclet$??0?$_Container_base_aux_alloc_real@V?$allocator@PAVCClientContext@@@std@@@std@@IAE@V?$allocator@PAVCClientContext@@@1@@Z$0 0047f610 f   MyIOCP.obj
 0001:0007e618       __unwindfunclet$??0?$_Container_base_aux_alloc_real@V?$allocator@PAVCClientContext@@@std@@@std@@IAE@V?$allocator@PAVCClientContext@@@1@@Z$1 0047f618 f   MyIOCP.obj
 0001:0007e629       __ehhandler$??0?$_Container_base_aux_alloc_real@V?$allocator@PAVCClientContext@@@std@@@std@@IAE@V?$allocator@PAVCClientContext@@@1@@Z 0047f629 f   MyIOCP.obj
 0001:0007e650       __unwindfunclet$??0CMyPropertyPage1@@QAE@XZ$0 0047f650 f   MyPropertyPage1.obj
 0001:0007e658       __ehhandler$??0CMyPropertyPage1@@QAE@XZ 0047f658 f   MyPropertyPage1.obj
 0001:0007e680       __unwindfunclet$?OnUpfileSet@CMyPropertyPage1@@QAE_NXZ$0 0047f680 f   MyPropertyPage1.obj
 0001:0007e689       __unwindfunclet$?OnUpfileSet@CMyPropertyPage1@@QAE_NXZ$1 0047f689 f   MyPropertyPage1.obj
 0001:0007e692       __unwindfunclet$?OnUpfileSet@CMyPropertyPage1@@QAE_NXZ$2 0047f692 f   MyPropertyPage1.obj
 0001:0007e69b       __unwindfunclet$?OnUpfileSet@CMyPropertyPage1@@QAE_NXZ$3 0047f69b f   MyPropertyPage1.obj
 0001:0007e6a7       __unwindfunclet$?OnUpfileSet@CMyPropertyPage1@@QAE_NXZ$5 0047f6a7 f   MyPropertyPage1.obj
 0001:0007e6b3       __unwindfunclet$?OnUpfileSet@CMyPropertyPage1@@QAE_NXZ$6 0047f6b3 f   MyPropertyPage1.obj
 0001:0007e6bf       __unwindfunclet$?OnUpfileSet@CMyPropertyPage1@@QAE_NXZ$7 0047f6bf f   MyPropertyPage1.obj
 0001:0007e6cb       __unwindfunclet$?OnUpfileSet@CMyPropertyPage1@@QAE_NXZ$8 0047f6cb f   MyPropertyPage1.obj
 0001:0007e6d7       __unwindfunclet$?OnUpfileSet@CMyPropertyPage1@@QAE_NXZ$9 0047f6d7 f   MyPropertyPage1.obj
 0001:0007e6e3       __unwindfunclet$?OnUpfileSet@CMyPropertyPage1@@QAE_NXZ$10 0047f6e3 f   MyPropertyPage1.obj
 0001:0007e6ef       __unwindfunclet$?OnUpfileSet@CMyPropertyPage1@@QAE_NXZ$12 0047f6ef f   MyPropertyPage1.obj
 0001:0007e6fb       __unwindfunclet$?OnUpfileSet@CMyPropertyPage1@@QAE_NXZ$13 0047f6fb f   MyPropertyPage1.obj
 0001:0007e706       __unwindfunclet$?OnUpfileSet@CMyPropertyPage1@@QAE_NXZ$15 0047f706 f   MyPropertyPage1.obj
 0001:0007e712       __ehhandler$?OnUpfileSet@CMyPropertyPage1@@QAE_NXZ 0047f712 f   MyPropertyPage1.obj
 0001:0007e740       __unwindfunclet$?OnInitDialog@CMyPropertyPage1@@UAEHXZ$0 0047f740 f   MyPropertyPage1.obj
 0001:0007e74c       __unwindfunclet$?OnInitDialog@CMyPropertyPage1@@UAEHXZ$1 0047f74c f   MyPropertyPage1.obj
 0001:0007e758       __unwindfunclet$?OnInitDialog@CMyPropertyPage1@@UAEHXZ$2 0047f758 f   MyPropertyPage1.obj
 0001:0007e764       __unwindfunclet$?OnInitDialog@CMyPropertyPage1@@UAEHXZ$3 0047f764 f   MyPropertyPage1.obj
 0001:0007e76d       __unwindfunclet$?OnInitDialog@CMyPropertyPage1@@UAEHXZ$4 0047f76d f   MyPropertyPage1.obj
 0001:0007e776       __unwindfunclet$?OnInitDialog@CMyPropertyPage1@@UAEHXZ$5 0047f776 f   MyPropertyPage1.obj
 0001:0007e782       __unwindfunclet$?OnInitDialog@CMyPropertyPage1@@UAEHXZ$6 0047f782 f   MyPropertyPage1.obj
 0001:0007e78a       __unwindfunclet$?OnInitDialog@CMyPropertyPage1@@UAEHXZ$8 0047f78a f   MyPropertyPage1.obj
 0001:0007e796       __unwindfunclet$?OnInitDialog@CMyPropertyPage1@@UAEHXZ$10 0047f796 f   MyPropertyPage1.obj
 0001:0007e7a2       __unwindfunclet$?OnInitDialog@CMyPropertyPage1@@UAEHXZ$11 0047f7a2 f   MyPropertyPage1.obj
 0001:0007e7ae       __ehhandler$?OnInitDialog@CMyPropertyPage1@@UAEHXZ 0047f7ae f   MyPropertyPage1.obj
 0001:0007e7e0       __unwindfunclet$?OnInitDialog@CMyPropertyPage2@@UAEHXZ$0 0047f7e0 f   MyPropertyPage1.obj
 0001:0007e7e9       __unwindfunclet$?OnInitDialog@CMyPropertyPage2@@UAEHXZ$1 0047f7e9 f   MyPropertyPage1.obj
 0001:0007e7f2       __unwindfunclet$?OnInitDialog@CMyPropertyPage2@@UAEHXZ$2 0047f7f2 f   MyPropertyPage1.obj
 0001:0007e7fa       __ehhandler$?OnInitDialog@CMyPropertyPage2@@UAEHXZ 0047f7fa f   MyPropertyPage1.obj
 0001:0007e820       __unwindfunclet$?EClassSet@CMyPropertyPage2@@QAE_NXZ$0 0047f820 f   MyPropertyPage1.obj
 0001:0007e828       __ehhandler$?EClassSet@CMyPropertyPage2@@QAE_NXZ 0047f828 f   MyPropertyPage1.obj
 0001:0007e850       __unwindfunclet$?OnInitDialog@CMyPropertyPage3@@UAEHXZ$0 0047f850 f   MyPropertyPage1.obj
 0001:0007e859       __unwindfunclet$?OnInitDialog@CMyPropertyPage3@@UAEHXZ$1 0047f859 f   MyPropertyPage1.obj
 0001:0007e862       __unwindfunclet$?OnInitDialog@CMyPropertyPage3@@UAEHXZ$2 0047f862 f   MyPropertyPage1.obj
 0001:0007e86b       __unwindfunclet$?OnInitDialog@CMyPropertyPage3@@UAEHXZ$3 0047f86b f   MyPropertyPage1.obj
 0001:0007e873       __ehhandler$?OnInitDialog@CMyPropertyPage3@@UAEHXZ 0047f873 f   MyPropertyPage1.obj
 0001:0007e890       __unwindfunclet$?BroTypeSel@CMyPropertyPage3@@QAE_NXZ$0 0047f890 f   MyPropertyPage1.obj
 0001:0007e898       __ehhandler$?BroTypeSel@CMyPropertyPage3@@QAE_NXZ 0047f898 f   MyPropertyPage1.obj
 0001:0007e8c0       __unwindfunclet$??0CMyPropertySheet@@QAE@W4PropSheetLook@CMFCPropertySheet@@IH@Z$0 0047f8c0 f   MyPropertySheet.obj
 0001:0007e8c9       __unwindfunclet$??0CMyPropertySheet@@QAE@W4PropSheetLook@CMFCPropertySheet@@IH@Z$1 0047f8c9 f   MyPropertySheet.obj
 0001:0007e8d1       __unwindfunclet$??0CMyPropertySheet@@QAE@W4PropSheetLook@CMFCPropertySheet@@IH@Z$2 0047f8d1 f   MyPropertySheet.obj
 0001:0007e8df       __unwindfunclet$??0CMyPropertySheet@@QAE@W4PropSheetLook@CMFCPropertySheet@@IH@Z$3 0047f8df f   MyPropertySheet.obj
 0001:0007e8ed       __unwindfunclet$??0CMyPropertySheet@@QAE@W4PropSheetLook@CMFCPropertySheet@@IH@Z$4 0047f8ed f   MyPropertySheet.obj
 0001:0007e8fb       __ehhandler$??0CMyPropertySheet@@QAE@W4PropSheetLook@CMFCPropertySheet@@IH@Z 0047f8fb f   MyPropertySheet.obj
 0001:0007e920       __unwindfunclet$??1CMyPropertySheet@@UAE@XZ$0 0047f920 f   MyPropertySheet.obj
 0001:0007e928       __unwindfunclet$??1CMyPropertySheet@@UAE@XZ$1 0047f928 f   MyPropertySheet.obj
 0001:0007e936       __unwindfunclet$??1CMyPropertySheet@@UAE@XZ$2 0047f936 f   MyPropertySheet.obj
 0001:0007e944       __ehhandler$??1CMyPropertySheet@@UAE@XZ 0047f944 f   MyPropertySheet.obj
 0001:0007e960       __unwindfunclet$?OnDrawPageHeader@CMyPropertySheet@@UAEXPAVCDC@@HVCRect@@@Z$0 0047f960 f   MyPropertySheet.obj
 0001:0007e968       __unwindfunclet$?OnDrawPageHeader@CMyPropertySheet@@UAEXPAVCDC@@HVCRect@@@Z$1 0047f968 f   MyPropertySheet.obj
 0001:0007e971       __ehhandler$?OnDrawPageHeader@CMyPropertySheet@@UAEXPAVCDC@@HVCRect@@@Z 0047f971 f   MyPropertySheet.obj
 0001:0007e990       __unwindfunclet$?OnInitDialog@CMyPropertySheet@@UAEHXZ$0 0047f990 f   MyPropertySheet.obj
 0001:0007e999       __unwindfunclet$?OnInitDialog@CMyPropertySheet@@UAEHXZ$1 0047f999 f   MyPropertySheet.obj
 0001:0007e9a2       __ehhandler$?OnInitDialog@CMyPropertySheet@@UAEHXZ 0047f9a2 f   MyPropertySheet.obj
 0001:0007e9c0       __unwindfunclet$?OnRButtonDown@CMyRichEdit@@IAEXIVCPoint@@@Z$0 0047f9c0 f   MyRichEdit.obj
 0001:0007e9c8       __unwindfunclet$?OnRButtonDown@CMyRichEdit@@IAEXIVCPoint@@@Z$1 0047f9c8 f   MyRichEdit.obj
 0001:0007e9d1       __unwindfunclet$?OnRButtonDown@CMyRichEdit@@IAEXIVCPoint@@@Z$2 0047f9d1 f   MyRichEdit.obj
 0001:0007e9da       __unwindfunclet$?OnRButtonDown@CMyRichEdit@@IAEXIVCPoint@@@Z$3 0047f9da f   MyRichEdit.obj
 0001:0007e9e3       __unwindfunclet$?OnRButtonDown@CMyRichEdit@@IAEXIVCPoint@@@Z$4 0047f9e3 f   MyRichEdit.obj
 0001:0007e9ec       __unwindfunclet$?OnRButtonDown@CMyRichEdit@@IAEXIVCPoint@@@Z$5 0047f9ec f   MyRichEdit.obj
 0001:0007e9f5       __unwindfunclet$?OnRButtonDown@CMyRichEdit@@IAEXIVCPoint@@@Z$6 0047f9f5 f   MyRichEdit.obj
 0001:0007e9fe       __ehhandler$?OnRButtonDown@CMyRichEdit@@IAEXIVCPoint@@@Z 0047f9fe f   MyRichEdit.obj
 0001:0007ea20       __unwindfunclet$?OnEraseBkgnd@CNewListCtrl@@IAEHPAVCDC@@@Z$0 0047fa20 f   NewListCtrl.obj
 0001:0007ea28       __unwindfunclet$?OnEraseBkgnd@CNewListCtrl@@IAEHPAVCDC@@@Z$1 0047fa28 f   NewListCtrl.obj
 0001:0007ea30       __ehhandler$?OnEraseBkgnd@CNewListCtrl@@IAEHPAVCDC@@@Z 0047fa30 f   NewListCtrl.obj
 0001:0007ea50       __unwindfunclet$?NameCompare@CNewListCtrl@@QAEHPBD0@Z$0 0047fa50 f   NewListCtrl.obj
 0001:0007ea59       __unwindfunclet$?NameCompare@CNewListCtrl@@QAEHPBD0@Z$1 0047fa59 f   NewListCtrl.obj
 0001:0007ea62       __unwindfunclet$?NameCompare@CNewListCtrl@@QAEHPBD0@Z$2 0047fa62 f   NewListCtrl.obj
 0001:0007ea6b       __unwindfunclet$?NameCompare@CNewListCtrl@@QAEHPBD0@Z$3 0047fa6b f   NewListCtrl.obj
 0001:0007ea74       __unwindfunclet$?NameCompare@CNewListCtrl@@QAEHPBD0@Z$4 0047fa74 f   NewListCtrl.obj
 0001:0007ea7d       __unwindfunclet$?NameCompare@CNewListCtrl@@QAEHPBD0@Z$5 0047fa7d f   NewListCtrl.obj
 0001:0007ea86       __unwindfunclet$?NameCompare@CNewListCtrl@@QAEHPBD0@Z$6 0047fa86 f   NewListCtrl.obj
 0001:0007ea8f       __unwindfunclet$?NameCompare@CNewListCtrl@@QAEHPBD0@Z$7 0047fa8f f   NewListCtrl.obj
 0001:0007ea98       __unwindfunclet$?NameCompare@CNewListCtrl@@QAEHPBD0@Z$8 0047fa98 f   NewListCtrl.obj
 0001:0007eaa1       __unwindfunclet$?NameCompare@CNewListCtrl@@QAEHPBD0@Z$9 0047faa1 f   NewListCtrl.obj
 0001:0007eaaa       __unwindfunclet$?NameCompare@CNewListCtrl@@QAEHPBD0@Z$10 0047faaa f   NewListCtrl.obj
 0001:0007eab3       __unwindfunclet$?NameCompare@CNewListCtrl@@QAEHPBD0@Z$11 0047fab3 f   NewListCtrl.obj
 0001:0007eabc       __ehhandler$?NameCompare@CNewListCtrl@@QAEHPBD0@Z 0047fabc f   NewListCtrl.obj
 0001:0007eae0       __unwindfunclet$??1COutputWnd@@UAE@XZ$0 0047fae0 f   OutputWnd.obj
 0001:0007eae0       __unwindfunclet$??0COutputWnd@@QAE@XZ$0 0047fae0 f   OutputWnd.obj
 0001:0007eae8       __unwindfunclet$??1COutputWnd@@UAE@XZ$1 0047fae8 f   OutputWnd.obj
 0001:0007eae8       __unwindfunclet$??0COutputWnd@@QAE@XZ$1 0047fae8 f   OutputWnd.obj
 0001:0007eaf6       __unwindfunclet$??1COutputWnd@@UAE@XZ$2 0047faf6 f   OutputWnd.obj
 0001:0007eaf6       __unwindfunclet$??0COutputWnd@@QAE@XZ$2 0047faf6 f   OutputWnd.obj
 0001:0007eb04       __unwindfunclet$??0COutputWnd@@QAE@XZ$3 0047fb04 f   OutputWnd.obj
 0001:0007eb04       __unwindfunclet$??1COutputWnd@@UAE@XZ$3 0047fb04 f   OutputWnd.obj
 0001:0007eb12       __unwindfunclet$??0COutputWnd@@QAE@XZ$4 0047fb12 f   OutputWnd.obj
 0001:0007eb12       __unwindfunclet$??1COutputWnd@@UAE@XZ$4 0047fb12 f   OutputWnd.obj
 0001:0007eb20       __unwindfunclet$??0COutputWnd@@QAE@XZ$5 0047fb20 f   OutputWnd.obj
 0001:0007eb20       __unwindfunclet$??1COutputWnd@@UAE@XZ$5 0047fb20 f   OutputWnd.obj
 0001:0007eb2e       __ehhandler$??0COutputWnd@@QAE@XZ 0047fb2e f   OutputWnd.obj
 0001:0007eb2e       __ehhandler$??1COutputWnd@@UAE@XZ 0047fb2e f   OutputWnd.obj
 0001:0007eb50       __unwindfunclet$?OnCreate@COutputWnd@@IAEHPAUtagCREATESTRUCTA@@@Z$0 0047fb50 f   OutputWnd.obj
 0001:0007eb59       __ehhandler$?OnCreate@COutputWnd@@IAEHPAUtagCREATESTRUCTA@@@Z 0047fb59 f   OutputWnd.obj
 0001:0007eb80       __unwindfunclet$?OnContextMenu@COutputList@@IAEXPAVCWnd@@VCPoint@@@Z$0 0047fb80 f   OutputWnd.obj
 0001:0007eb88       __unwindfunclet$?OnContextMenu@COutputList@@IAEXPAVCWnd@@VCPoint@@@Z$1 0047fb88 f   OutputWnd.obj
 0001:0007eb92       __ehhandler$?OnContextMenu@COutputList@@IAEXPAVCWnd@@VCPoint@@@Z 0047fb92 f   OutputWnd.obj
 0001:0007ebb0       __unwindfunclet$??0CPartitionSettingDlg@@QAE@PAVCWnd@@@Z$0 0047fbb0 f   PartitionSettingDlg.obj
 0001:0007ebb8       __unwindfunclet$??0CPartitionSettingDlg@@QAE@PAVCWnd@@@Z$1 0047fbb8 f   PartitionSettingDlg.obj
 0001:0007ebc6       __unwindfunclet$??0CPartitionSettingDlg@@QAE@PAVCWnd@@@Z$2 0047fbc6 f   PartitionSettingDlg.obj
 0001:0007ebd4       __unwindfunclet$??0CPartitionSettingDlg@@QAE@PAVCWnd@@@Z$3 0047fbd4 f   PartitionSettingDlg.obj
 0001:0007ebe3       __unwindfunclet$??0CPartitionSettingDlg@@QAE@PAVCWnd@@@Z$4 0047fbe3 f   PartitionSettingDlg.obj
 0001:0007ebf2       __unwindfunclet$??0CPartitionSettingDlg@@QAE@PAVCWnd@@@Z$5 0047fbf2 f   PartitionSettingDlg.obj
 0001:0007ec01       __unwindfunclet$??0CPartitionSettingDlg@@QAE@PAVCWnd@@@Z$6 0047fc01 f   PartitionSettingDlg.obj
 0001:0007ec10       __unwindfunclet$??0CPartitionSettingDlg@@QAE@PAVCWnd@@@Z$7 0047fc10 f   PartitionSettingDlg.obj
 0001:0007ec1f       __unwindfunclet$??0CPartitionSettingDlg@@QAE@PAVCWnd@@@Z$8 0047fc1f f   PartitionSettingDlg.obj
 0001:0007ec2e       __unwindfunclet$??0CPartitionSettingDlg@@QAE@PAVCWnd@@@Z$9 0047fc2e f   PartitionSettingDlg.obj
 0001:0007ec3d       __unwindfunclet$??0CPartitionSettingDlg@@QAE@PAVCWnd@@@Z$10 0047fc3d f   PartitionSettingDlg.obj
 0001:0007ec4b       __unwindfunclet$??0CPartitionSettingDlg@@QAE@PAVCWnd@@@Z$11 0047fc4b f   PartitionSettingDlg.obj
 0001:0007ec5a       __ehhandler$??0CPartitionSettingDlg@@QAE@PAVCWnd@@@Z 0047fc5a f   PartitionSettingDlg.obj
 0001:0007ec80       __unwindfunclet$?OnInitDialog@CPartitionSettingDlg@@MAEHXZ$0 0047fc80 f   PartitionSettingDlg.obj
 0001:0007ec89       __unwindfunclet$?OnInitDialog@CPartitionSettingDlg@@MAEHXZ$1 0047fc89 f   PartitionSettingDlg.obj
 0001:0007ec92       __ehhandler$?OnInitDialog@CPartitionSettingDlg@@MAEHXZ 0047fc92 f   PartitionSettingDlg.obj
 0001:0007ecb0       __unwindfunclet$?OnOK@CPartitionSettingDlg@@MAEXXZ$0 0047fcb0 f   PartitionSettingDlg.obj
 0001:0007ecb9       __unwindfunclet$?OnOK@CPartitionSettingDlg@@MAEXXZ$1 0047fcb9 f   PartitionSettingDlg.obj
 0001:0007ecc2       __unwindfunclet$?OnOK@CPartitionSettingDlg@@MAEXXZ$2 0047fcc2 f   PartitionSettingDlg.obj
 0001:0007eccb       __ehhandler$?OnOK@CPartitionSettingDlg@@MAEXXZ 0047fccb f   PartitionSettingDlg.obj
 0001:0007ecf0       __unwindfunclet$?OnInitDialog@CPortChannelDlg@@UAEHXZ$0 0047fcf0 f   PortChannelDlg.obj
 0001:0007ecf0       __unwindfunclet$?InitPortAndCode@CMainFrame@@QAEXXZ$0 0047fcf0 f   PortChannelDlg.obj
 0001:0007ecf8       __ehhandler$?InitPortAndCode@CMainFrame@@QAEXXZ 0047fcf8 f   PortChannelDlg.obj
 0001:0007ecf8       __ehhandler$?OnInitDialog@CPortChannelDlg@@UAEHXZ 0047fcf8 f   PortChannelDlg.obj
 0001:0007ed20       __unwindfunclet$??1CPortCtrlDlg@@UAE@XZ$0 0047fd20 f   PortCtrlDlg.obj
 0001:0007ed20       __unwindfunclet$??0CPortCtrlDlg@@QAE@PAVCWnd@@@Z$0 0047fd20 f   PortCtrlDlg.obj
 0001:0007ed28       __unwindfunclet$??1CPortCtrlDlg@@UAE@XZ$1 0047fd28 f   PortCtrlDlg.obj
 0001:0007ed28       __unwindfunclet$??0CPortCtrlDlg@@QAE@PAVCWnd@@@Z$1 0047fd28 f   PortCtrlDlg.obj
 0001:0007ed36       __ehhandler$??1CPortCtrlDlg@@UAE@XZ 0047fd36 f   PortCtrlDlg.obj
 0001:0007ed36       __ehhandler$??0CPortCtrlDlg@@QAE@PAVCWnd@@@Z 0047fd36 f   PortCtrlDlg.obj
 0001:0007ed60       __unwindfunclet$?OnInitDialog@CPortCtrlDlg@@MAEHXZ$0 0047fd60 f   PortCtrlDlg.obj
 0001:0007ed69       __unwindfunclet$?OnInitDialog@CPortCtrlDlg@@MAEHXZ$1 0047fd69 f   PortCtrlDlg.obj
 0001:0007ed72       __unwindfunclet$?OnInitDialog@CPortCtrlDlg@@MAEHXZ$2 0047fd72 f   PortCtrlDlg.obj
 0001:0007ed7b       __unwindfunclet$?OnInitDialog@CPortCtrlDlg@@MAEHXZ$3 0047fd7b f   PortCtrlDlg.obj
 0001:0007ed84       __unwindfunclet$?OnInitDialog@CPortCtrlDlg@@MAEHXZ$4 0047fd84 f   PortCtrlDlg.obj
 0001:0007ed8d       __unwindfunclet$?OnInitDialog@CPortCtrlDlg@@MAEHXZ$5 0047fd8d f   PortCtrlDlg.obj
 0001:0007ed96       __unwindfunclet$?OnInitDialog@CPortCtrlDlg@@MAEHXZ$6 0047fd96 f   PortCtrlDlg.obj
 0001:0007ed9f       __unwindfunclet$?OnInitDialog@CPortCtrlDlg@@MAEHXZ$7 0047fd9f f   PortCtrlDlg.obj
 0001:0007eda8       __unwindfunclet$?OnInitDialog@CPortCtrlDlg@@MAEHXZ$8 0047fda8 f   PortCtrlDlg.obj
 0001:0007edb1       __unwindfunclet$?OnInitDialog@CPortCtrlDlg@@MAEHXZ$9 0047fdb1 f   PortCtrlDlg.obj
 0001:0007edba       __unwindfunclet$?OnInitDialog@CPortCtrlDlg@@MAEHXZ$10 0047fdba f   PortCtrlDlg.obj
 0001:0007edc3       __unwindfunclet$?OnInitDialog@CPortCtrlDlg@@MAEHXZ$11 0047fdc3 f   PortCtrlDlg.obj
 0001:0007edcc       __unwindfunclet$?OnInitDialog@CPortCtrlDlg@@MAEHXZ$12 0047fdcc f   PortCtrlDlg.obj
 0001:0007edd5       __ehhandler$?OnInitDialog@CPortCtrlDlg@@MAEHXZ 0047fdd5 f   PortCtrlDlg.obj
 0001:0007ee00       __unwindfunclet$?OnBnClickedOk@CPortCtrlDlg@@QAEXXZ$0 0047fe00 f   PortCtrlDlg.obj
 0001:0007ee09       __unwindfunclet$?OnBnClickedOk@CPortCtrlDlg@@QAEXXZ$1 0047fe09 f   PortCtrlDlg.obj
 0001:0007ee12       __ehhandler$?OnBnClickedOk@CPortCtrlDlg@@QAEXXZ 0047fe12 f   PortCtrlDlg.obj
 0001:0007ee30       __unwindfunclet$?GetKeyValue@CPrivateProfileFile@@QAEHV?$CStringT@DV?$StrTraitMFC_DLL@DV?$ChTraitsCRT@D@ATL@@@@@ATL@@0AAV23@@Z$0 0047fe30 f   PrivateProfileFile.obj
 0001:0007ee39       __unwindfunclet$?GetKeyValue@CPrivateProfileFile@@QAEHV?$CStringT@DV?$StrTraitMFC_DLL@DV?$ChTraitsCRT@D@ATL@@@@@ATL@@0AAV23@@Z$1 0047fe39 f   PrivateProfileFile.obj
 0001:0007ee42       __unwindfunclet$?GetKeyValue@CPrivateProfileFile@@QAEHV?$CStringT@DV?$StrTraitMFC_DLL@DV?$ChTraitsCRT@D@ATL@@@@@ATL@@0AAV23@@Z$2 0047fe42 f   PrivateProfileFile.obj
 0001:0007ee4a       __ehhandler$?GetKeyValue@CPrivateProfileFile@@QAEHV?$CStringT@DV?$StrTraitMFC_DLL@DV?$ChTraitsCRT@D@ATL@@@@@ATL@@0AAV23@@Z 0047fe4a f   PrivateProfileFile.obj
 0001:0007ee80       __unwindfunclet$??0CProgressDlg@@QAE@PAVCWnd@@@Z$0 0047fe80 f   ProgressDlg.obj
 0001:0007ee80       __unwindfunclet$??1CProgressDlg@@UAE@XZ$0 0047fe80 f   ProgressDlg.obj
 0001:0007ee88       __unwindfunclet$??1CProgressDlg@@UAE@XZ$1 0047fe88 f   ProgressDlg.obj
 0001:0007ee88       __unwindfunclet$??0CProgressDlg@@QAE@PAVCWnd@@@Z$1 0047fe88 f   ProgressDlg.obj
 0001:0007ee93       __unwindfunclet$??1CProgressDlg@@UAE@XZ$2 0047fe93 f   ProgressDlg.obj
 0001:0007ee93       __unwindfunclet$??0CProgressDlg@@QAE@PAVCWnd@@@Z$2 0047fe93 f   ProgressDlg.obj
 0001:0007eea1       __unwindfunclet$??0CProgressDlg@@QAE@PAVCWnd@@@Z$3 0047fea1 f   ProgressDlg.obj
 0001:0007eea1       __unwindfunclet$??1CProgressDlg@@UAE@XZ$3 0047fea1 f   ProgressDlg.obj
 0001:0007eeb0       __unwindfunclet$??1CProgressDlg@@UAE@XZ$4 0047feb0 f   ProgressDlg.obj
 0001:0007eeb0       __unwindfunclet$??0CProgressDlg@@QAE@PAVCWnd@@@Z$4 0047feb0 f   ProgressDlg.obj
 0001:0007eebf       __ehhandler$??0CProgressDlg@@QAE@PAVCWnd@@@Z 0047febf f   ProgressDlg.obj
 0001:0007eebf       __ehhandler$??1CProgressDlg@@UAE@XZ 0047febf f   ProgressDlg.obj
 0001:0007eee0       __unwindfunclet$?OnInitDialog@CProgressDlg@@MAEHXZ$0 0047fee0 f   ProgressDlg.obj
 0001:0007eee0       __unwindfunclet$?OnInitDialog@CCmdEnquireDlg@@MAEHXZ$0 0047fee0 f   ProgressDlg.obj
 0001:0007eee9       __unwindfunclet$?OnInitDialog@CProgressDlg@@MAEHXZ$1 0047fee9 f   ProgressDlg.obj
 0001:0007eee9       __unwindfunclet$?OnInitDialog@CCmdEnquireDlg@@MAEHXZ$1 0047fee9 f   ProgressDlg.obj
 0001:0007eef2       __unwindfunclet$?OnInitDialog@CCmdEnquireDlg@@MAEHXZ$2 0047fef2 f   ProgressDlg.obj
 0001:0007eef2       __unwindfunclet$?OnInitDialog@CProgressDlg@@MAEHXZ$2 0047fef2 f   ProgressDlg.obj
 0001:0007eefb       __ehhandler$?OnInitDialog@CProgressDlg@@MAEHXZ 0047fefb f   ProgressDlg.obj
 0001:0007eefb       __ehhandler$?OnInitDialog@CCmdEnquireDlg@@MAEHXZ 0047fefb f   ProgressDlg.obj
 0001:0007ef20       __unwindfunclet$?WaitStart@CProgressDlg@@QAEHV?$CStringT@DV?$StrTraitMFC_DLL@DV?$ChTraitsCRT@D@ATL@@@@@ATL@@0PAVCWnd@@@Z$0 0047ff20 f   ProgressDlg.obj
 0001:0007ef29       __unwindfunclet$?WaitStart@CProgressDlg@@QAEHV?$CStringT@DV?$StrTraitMFC_DLL@DV?$ChTraitsCRT@D@ATL@@@@@ATL@@0PAVCWnd@@@Z$1 0047ff29 f   ProgressDlg.obj
 0001:0007ef32       __unwindfunclet$?WaitStart@CProgressDlg@@QAEHV?$CStringT@DV?$StrTraitMFC_DLL@DV?$ChTraitsCRT@D@ATL@@@@@ATL@@0PAVCWnd@@@Z$2 0047ff32 f   ProgressDlg.obj
 0001:0007ef3d       __ehhandler$?WaitStart@CProgressDlg@@QAEHV?$CStringT@DV?$StrTraitMFC_DLL@DV?$ChTraitsCRT@D@ATL@@@@@ATL@@0PAVCWnd@@@Z 0047ff3d f   ProgressDlg.obj
 0001:0007ef60       __unwindfunclet$??1CPropertyViewDlg@@UAE@XZ$0 0047ff60 f   PropertyViewDlg.obj
 0001:0007ef60       __unwindfunclet$??0CPropertyViewDlg@@QAE@PAVCWnd@@@Z$0 0047ff60 f   PropertyViewDlg.obj
 0001:0007ef68       __unwindfunclet$??1CPropertyViewDlg@@UAE@XZ$1 0047ff68 f   PropertyViewDlg.obj
 0001:0007ef68       __unwindfunclet$??0CPropertyViewDlg@@QAE@PAVCWnd@@@Z$1 0047ff68 f   PropertyViewDlg.obj
 0001:0007ef73       __unwindfunclet$??1CPropertyViewDlg@@UAE@XZ$2 0047ff73 f   PropertyViewDlg.obj
 0001:0007ef73       __unwindfunclet$??0CPropertyViewDlg@@QAE@PAVCWnd@@@Z$2 0047ff73 f   PropertyViewDlg.obj
 0001:0007ef81       __unwindfunclet$??1CPropertyViewDlg@@UAE@XZ$3 0047ff81 f   PropertyViewDlg.obj
 0001:0007ef81       __unwindfunclet$??0CPropertyViewDlg@@QAE@PAVCWnd@@@Z$3 0047ff81 f   PropertyViewDlg.obj
 0001:0007ef8f       __unwindfunclet$??1CPropertyViewDlg@@UAE@XZ$4 0047ff8f f   PropertyViewDlg.obj
 0001:0007ef8f       __unwindfunclet$??0CPropertyViewDlg@@QAE@PAVCWnd@@@Z$4 0047ff8f f   PropertyViewDlg.obj
 0001:0007ef9d       __unwindfunclet$??0CPropertyViewDlg@@QAE@PAVCWnd@@@Z$5 0047ff9d f   PropertyViewDlg.obj
 0001:0007ef9d       __unwindfunclet$??1CPropertyViewDlg@@UAE@XZ$5 0047ff9d f   PropertyViewDlg.obj
 0001:0007efab       __unwindfunclet$??0CPropertyViewDlg@@QAE@PAVCWnd@@@Z$6 0047ffab f   PropertyViewDlg.obj
 0001:0007efab       __unwindfunclet$??1CPropertyViewDlg@@UAE@XZ$6 0047ffab f   PropertyViewDlg.obj
 0001:0007efb9       __unwindfunclet$??0CPropertyViewDlg@@QAE@PAVCWnd@@@Z$7 0047ffb9 f   PropertyViewDlg.obj
 0001:0007efb9       __unwindfunclet$??1CPropertyViewDlg@@UAE@XZ$7 0047ffb9 f   PropertyViewDlg.obj
 0001:0007efc8       __unwindfunclet$??0CPropertyViewDlg@@QAE@PAVCWnd@@@Z$8 0047ffc8 f   PropertyViewDlg.obj
 0001:0007efc8       __unwindfunclet$??1CPropertyViewDlg@@UAE@XZ$8 0047ffc8 f   PropertyViewDlg.obj
 0001:0007efd6       __ehhandler$??0CPropertyViewDlg@@QAE@PAVCWnd@@@Z 0047ffd6 f   PropertyViewDlg.obj
 0001:0007efd6       __ehhandler$??1CPropertyViewDlg@@UAE@XZ 0047ffd6 f   PropertyViewDlg.obj
 0001:0007f000       __unwindfunclet$?OnBtnUpdate@CPropertyViewDlg@@IAEXXZ$1 00480000 f   PropertyViewDlg.obj
 0001:0007f00b       __unwindfunclet$?OnBtnUpdate@CPropertyViewDlg@@IAEXXZ$2 0048000b f   PropertyViewDlg.obj
 0001:0007f017       __unwindfunclet$?OnBtnUpdate@CPropertyViewDlg@@IAEXXZ$3 00480017 f   PropertyViewDlg.obj
 0001:0007f023       __unwindfunclet$?OnBtnUpdate@CPropertyViewDlg@@IAEXXZ$4 00480023 f   PropertyViewDlg.obj
 0001:0007f02e       __unwindfunclet$?OnBtnUpdate@CPropertyViewDlg@@IAEXXZ$5 0048002e f   PropertyViewDlg.obj
 0001:0007f03a       __unwindfunclet$?OnBtnUpdate@CPropertyViewDlg@@IAEXXZ$6 0048003a f   PropertyViewDlg.obj
 0001:0007f046       __ehhandler$?OnBtnUpdate@CPropertyViewDlg@@IAEXXZ 00480046 f   PropertyViewDlg.obj
 0001:0007f070       __unwindfunclet$?OnInitDialog@CPropertyViewDlg@@MAEHXZ$0 00480070 f   PropertyViewDlg.obj
 0001:0007f079       __unwindfunclet$?OnInitDialog@CPropertyViewDlg@@MAEHXZ$1 00480079 f   PropertyViewDlg.obj
 0001:0007f082       __unwindfunclet$?OnInitDialog@CPropertyViewDlg@@MAEHXZ$2 00480082 f   PropertyViewDlg.obj
 0001:0007f08b       __unwindfunclet$?OnInitDialog@CPropertyViewDlg@@MAEHXZ$3 0048008b f   PropertyViewDlg.obj
 0001:0007f094       __unwindfunclet$?OnInitDialog@CPropertyViewDlg@@MAEHXZ$4 00480094 f   PropertyViewDlg.obj
 0001:0007f09d       __unwindfunclet$?OnInitDialog@CPropertyViewDlg@@MAEHXZ$5 0048009d f   PropertyViewDlg.obj
 0001:0007f0a6       __unwindfunclet$?OnInitDialog@CPropertyViewDlg@@MAEHXZ$6 004800a6 f   PropertyViewDlg.obj
 0001:0007f0af       __unwindfunclet$?OnInitDialog@CPropertyViewDlg@@MAEHXZ$7 004800af f   PropertyViewDlg.obj
 0001:0007f0b8       __unwindfunclet$?OnInitDialog@CPropertyViewDlg@@MAEHXZ$8 004800b8 f   PropertyViewDlg.obj
 0001:0007f0c1       __unwindfunclet$?OnInitDialog@CPropertyViewDlg@@MAEHXZ$9 004800c1 f   PropertyViewDlg.obj
 0001:0007f0ca       __unwindfunclet$?OnInitDialog@CPropertyViewDlg@@MAEHXZ$10 004800ca f   PropertyViewDlg.obj
 0001:0007f0d3       __ehhandler$?OnInitDialog@CPropertyViewDlg@@MAEHXZ 004800d3 f   PropertyViewDlg.obj
 0001:0007f100       __unwindfunclet$?InitListInfoDisplay1@CPropertyViewDlg@@QAEXXZ$0 00480100 f   PropertyViewDlg.obj
 0001:0007f109       __unwindfunclet$?InitListInfoDisplay1@CPropertyViewDlg@@QAEXXZ$1 00480109 f   PropertyViewDlg.obj
 0001:0007f112       __unwindfunclet$?InitListInfoDisplay1@CPropertyViewDlg@@QAEXXZ$2 00480112 f   PropertyViewDlg.obj
 0001:0007f11b       __unwindfunclet$?InitListInfoDisplay1@CPropertyViewDlg@@QAEXXZ$3 0048011b f   PropertyViewDlg.obj
 0001:0007f124       __unwindfunclet$?InitListInfoDisplay1@CPropertyViewDlg@@QAEXXZ$5 00480124 f   PropertyViewDlg.obj
 0001:0007f12d       __unwindfunclet$?InitListInfoDisplay1@CPropertyViewDlg@@QAEXXZ$6 0048012d f   PropertyViewDlg.obj
 0001:0007f136       __unwindfunclet$?InitListInfoDisplay1@CPropertyViewDlg@@QAEXXZ$7 00480136 f   PropertyViewDlg.obj
 0001:0007f13f       __unwindfunclet$?InitListInfoDisplay1@CPropertyViewDlg@@QAEXXZ$8 0048013f f   PropertyViewDlg.obj
 0001:0007f148       __unwindfunclet$?InitListInfoDisplay1@CPropertyViewDlg@@QAEXXZ$9 00480148 f   PropertyViewDlg.obj
 0001:0007f151       __unwindfunclet$?InitListInfoDisplay1@CPropertyViewDlg@@QAEXXZ$10 00480151 f   PropertyViewDlg.obj
 0001:0007f15a       __unwindfunclet$?InitListInfoDisplay1@CPropertyViewDlg@@QAEXXZ$11 0048015a f   PropertyViewDlg.obj
 0001:0007f163       __unwindfunclet$?InitListInfoDisplay1@CPropertyViewDlg@@QAEXXZ$12 00480163 f   PropertyViewDlg.obj
 0001:0007f16c       __unwindfunclet$?InitListInfoDisplay1@CPropertyViewDlg@@QAEXXZ$13 0048016c f   PropertyViewDlg.obj
 0001:0007f178       __unwindfunclet$?InitListInfoDisplay1@CPropertyViewDlg@@QAEXXZ$14 00480178 f   PropertyViewDlg.obj
 0001:0007f184       __unwindfunclet$?InitListInfoDisplay1@CPropertyViewDlg@@QAEXXZ$15 00480184 f   PropertyViewDlg.obj
 0001:0007f18c       __unwindfunclet$?InitListInfoDisplay1@CPropertyViewDlg@@QAEXXZ$16 0048018c f   PropertyViewDlg.obj
 0001:0007f195       __unwindfunclet$?InitListInfoDisplay1@CPropertyViewDlg@@QAEXXZ$17 00480195 f   PropertyViewDlg.obj
 0001:0007f19e       __ehhandler$?InitListInfoDisplay1@CPropertyViewDlg@@QAEXXZ 0048019e f   PropertyViewDlg.obj
 0001:0007f1c0       __unwindfunclet$?InitListInfoDisplay@CPropertyViewDlg@@QAEXXZ$0 004801c0 f   PropertyViewDlg.obj
 0001:0007f1c9       __unwindfunclet$?InitListInfoDisplay@CPropertyViewDlg@@QAEXXZ$1 004801c9 f   PropertyViewDlg.obj
 0001:0007f1d2       __unwindfunclet$?InitListInfoDisplay@CPropertyViewDlg@@QAEXXZ$2 004801d2 f   PropertyViewDlg.obj
 0001:0007f1db       __unwindfunclet$?InitListInfoDisplay@CPropertyViewDlg@@QAEXXZ$3 004801db f   PropertyViewDlg.obj
 0001:0007f1e4       __unwindfunclet$?InitListInfoDisplay@CPropertyViewDlg@@QAEXXZ$4 004801e4 f   PropertyViewDlg.obj
 0001:0007f1ed       __unwindfunclet$?InitListInfoDisplay@CPropertyViewDlg@@QAEXXZ$5 004801ed f   PropertyViewDlg.obj
 0001:0007f1f6       __unwindfunclet$?InitListInfoDisplay@CPropertyViewDlg@@QAEXXZ$6 004801f6 f   PropertyViewDlg.obj
 0001:0007f1ff       __unwindfunclet$?InitListInfoDisplay@CPropertyViewDlg@@QAEXXZ$7 004801ff f   PropertyViewDlg.obj
 0001:0007f208       __unwindfunclet$?InitListInfoDisplay@CPropertyViewDlg@@QAEXXZ$8 00480208 f   PropertyViewDlg.obj
 0001:0007f211       __unwindfunclet$?InitListInfoDisplay@CPropertyViewDlg@@QAEXXZ$9 00480211 f   PropertyViewDlg.obj
 0001:0007f21a       __unwindfunclet$?InitListInfoDisplay@CPropertyViewDlg@@QAEXXZ$10 0048021a f   PropertyViewDlg.obj
 0001:0007f223       __unwindfunclet$?InitListInfoDisplay@CPropertyViewDlg@@QAEXXZ$11 00480223 f   PropertyViewDlg.obj
 0001:0007f22c       __unwindfunclet$?InitListInfoDisplay@CPropertyViewDlg@@QAEXXZ$12 0048022c f   PropertyViewDlg.obj
 0001:0007f235       __unwindfunclet$?InitListInfoDisplay@CPropertyViewDlg@@QAEXXZ$13 00480235 f   PropertyViewDlg.obj
 0001:0007f23d       __unwindfunclet$?InitListInfoDisplay@CPropertyViewDlg@@QAEXXZ$14 0048023d f   PropertyViewDlg.obj
 0001:0007f246       __unwindfunclet$?InitListInfoDisplay@CPropertyViewDlg@@QAEXXZ$15 00480246 f   PropertyViewDlg.obj
 0001:0007f24f       __ehhandler$?InitListInfoDisplay@CPropertyViewDlg@@QAEXXZ 0048024f f   PropertyViewDlg.obj
 0001:0007f270       __unwindfunclet$?RefreshPropertyInfo@CPropertyViewDlg@@QAEHXZ$0 00480270 f   PropertyViewDlg.obj
 0001:0007f279       __unwindfunclet$?RefreshPropertyInfo@CPropertyViewDlg@@QAEHXZ$1 00480279 f   PropertyViewDlg.obj
 0001:0007f282       __unwindfunclet$?RefreshPropertyInfo@CPropertyViewDlg@@QAEHXZ$2 00480282 f   PropertyViewDlg.obj
 0001:0007f28b       __ehhandler$?RefreshPropertyInfo@CPropertyViewDlg@@QAEHXZ 0048028b f   PropertyViewDlg.obj
 0001:0007f2b0       __unwindfunclet$?InsertHardwareListItem@CPropertyViewDlg@@QAEHHPBD00H@Z$0 004802b0 f   PropertyViewDlg.obj
 0001:0007f2b9       __unwindfunclet$?InsertHardwareListItem@CPropertyViewDlg@@QAEHHPBD00H@Z$1 004802b9 f   PropertyViewDlg.obj
 0001:0007f2c2       __unwindfunclet$?InsertHardwareListItem@CPropertyViewDlg@@QAEHHPBD00H@Z$2 004802c2 f   PropertyViewDlg.obj
 0001:0007f2cb       __unwindfunclet$?InsertHardwareListItem@CPropertyViewDlg@@QAEHHPBD00H@Z$3 004802cb f   PropertyViewDlg.obj
 0001:0007f2d4       __unwindfunclet$?InsertHardwareListItem@CPropertyViewDlg@@QAEHHPBD00H@Z$4 004802d4 f   PropertyViewDlg.obj
 0001:0007f2dd       __ehhandler$?InsertHardwareListItem@CPropertyViewDlg@@QAEHHPBD00H@Z 004802dd f   PropertyViewDlg.obj
 0001:0007f300       __unwindfunclet$?InsertSoftwareListItem@CPropertyViewDlg@@QAEHHPADH@Z$0 00480300 f   PropertyViewDlg.obj
 0001:0007f309       __unwindfunclet$?InsertSoftwareListItem@CPropertyViewDlg@@QAEHHPADH@Z$1 00480309 f   PropertyViewDlg.obj
 0001:0007f312       __unwindfunclet$?InsertSoftwareListItem@CPropertyViewDlg@@QAEHHPADH@Z$2 00480312 f   PropertyViewDlg.obj
 0001:0007f31b       __unwindfunclet$?InsertSoftwareListItem@CPropertyViewDlg@@QAEHHPADH@Z$3 0048031b f   PropertyViewDlg.obj
 0001:0007f324       __unwindfunclet$?InsertSoftwareListItem@CPropertyViewDlg@@QAEHHPADH@Z$4 00480324 f   PropertyViewDlg.obj
 0001:0007f32d       __ehhandler$?InsertSoftwareListItem@CPropertyViewDlg@@QAEHHPADH@Z 0048032d f   PropertyViewDlg.obj
 0001:0007f350       __unwindfunclet$??1CPropertyViewUIThread@@MAE@XZ$0 00480350 f   PropertyViewUIThread.obj
 0001:0007f350       __unwindfunclet$??0CPropertyViewUIThread@@IAE@XZ$0 00480350 f   PropertyViewUIThread.obj
 0001:0007f358       __ehhandler$??1CPropertyViewUIThread@@MAE@XZ 00480358 f   PropertyViewUIThread.obj
 0001:0007f358       __ehhandler$??0CPropertyViewUIThread@@IAE@XZ 00480358 f   PropertyViewUIThread.obj
 0001:0007f380       __unwindfunclet$??0CReportCtrl@@QAE@XZ$0 00480380 f   ReportCtrl.obj
 0001:0007f388       __unwindfunclet$??0CReportCtrl@@QAE@XZ$1 00480388 f   ReportCtrl.obj
 0001:0007f393       __unwindfunclet$??0CReportCtrl@@QAE@XZ$2 00480393 f   ReportCtrl.obj
 0001:0007f39e       __unwindfunclet$??0CReportCtrl@@QAE@XZ$3 0048039e f   ReportCtrl.obj
 0001:0007f3a8       __ehhandler$??0CReportCtrl@@QAE@XZ 004803a8 f   ReportCtrl.obj
 0001:0007f3d0       __unwindfunclet$??1CReportCtrl@@UAE@XZ$0 004803d0 f   ReportCtrl.obj
 0001:0007f3d8       __unwindfunclet$??1CReportCtrl@@UAE@XZ$1 004803d8 f   ReportCtrl.obj
 0001:0007f3e3       __unwindfunclet$??1CReportCtrl@@UAE@XZ$2 004803e3 f   ReportCtrl.obj
 0001:0007f3ee       __ehhandler$??1CReportCtrl@@UAE@XZ 004803ee f   ReportCtrl.obj
 0001:0007f410       __unwindfunclet$?StartEdit@CReportCtrl@@QAEHHH@Z$0 00480410 f   ReportCtrl.obj
 0001:0007f419       __ehhandler$?StartEdit@CReportCtrl@@QAEHHH@Z 00480419 f   ReportCtrl.obj
 0001:0007f440       __unwindfunclet$?EndEdit@CReportCtrl@@QAEHH@Z$0 00480440 f   ReportCtrl.obj
 0001:0007f449       __unwindfunclet$?EndEdit@CReportCtrl@@QAEHH@Z$1 00480449 f   ReportCtrl.obj
 0001:0007f463       __ehhandler$?EndEdit@CReportCtrl@@QAEHH@Z 00480463 f   ReportCtrl.obj
 0001:0007f480       __unwindfunclet$?_AllocItemMemory@CReportCtrl@@IAEXH@Z$0 00480480 f   ReportCtrl.obj
 0001:0007f48b       __ehhandler$?_AllocItemMemory@CReportCtrl@@IAEXH@Z 0048048b f   ReportCtrl.obj
 0001:0007f4b0       __unwindfunclet$??1CItemData@@QAE@XZ$0 004804b0 f   ReportCtrl.obj
 0001:0007f4b0       __unwindfunclet$??0CItemData@@QAE@XZ$0 004804b0 f   ReportCtrl.obj
 0001:0007f4bb       __ehhandler$??1CItemData@@QAE@XZ 004804bb f   ReportCtrl.obj
 0001:0007f4bb       __ehhandler$??0CItemData@@QAE@XZ 004804bb f   ReportCtrl.obj
 0001:0007f4e0       __unwindfunclet$?_PartialSort@CReportCtrl@@IAEHHH@Z$0 004804e0 f   ReportCtrl.obj
 0001:0007f4eb       __unwindfunclet$?_PartialSort@CReportCtrl@@IAEHHH@Z$1 004804eb f   ReportCtrl.obj
 0001:0007f4f4       __ehhandler$?_PartialSort@CReportCtrl@@IAEHHH@Z 004804f4 f   ReportCtrl.obj
 0001:0007f510       __unwindfunclet$??0ROWINFO@@QAE@XZ$0 00480510 f   ReportCtrl.obj
 0001:0007f510       __unwindfunclet$??1ROWINFO@@QAE@XZ$0 00480510 f   ReportCtrl.obj
 0001:0007f51b       __ehhandler$??1ROWINFO@@QAE@XZ 0048051b f   ReportCtrl.obj
 0001:0007f51b       __ehhandler$??0ROWINFO@@QAE@XZ 0048051b f   ReportCtrl.obj
 0001:0007f540       __unwindfunclet$?_CompareItems@CReportCtrl@@IAEHHH@Z$0 00480540 f   ReportCtrl.obj
 0001:0007f549       __unwindfunclet$?_CompareItems@CReportCtrl@@IAEHHH@Z$1 00480549 f   ReportCtrl.obj
 0001:0007f552       __ehhandler$?_CompareItems@CReportCtrl@@IAEHHH@Z 00480552 f   ReportCtrl.obj
 0001:0007f570       __unwindfunclet$?OnInitDialog@CSetClientchancelDLg@@UAEHXZ$0 00480570 f   SetClientchancelDLg.obj
 0001:0007f578       __ehhandler$?OnInitDialog@CSetClientchancelDLg@@UAEHXZ 00480578 f   SetClientchancelDLg.obj
 0001:0007f5a0       __unwindfunclet$??0CSetDrfaultNICDlg@@QAE@PAVCWnd@@@Z$0 004805a0 f   SetDrfaultNICDlg.obj
 0001:0007f5a8       __unwindfunclet$??0CSetDrfaultNICDlg@@QAE@PAVCWnd@@@Z$1 004805a8 f   SetDrfaultNICDlg.obj
 0001:0007f5b3       __ehhandler$??0CSetDrfaultNICDlg@@QAE@PAVCWnd@@@Z 004805b3 f   SetDrfaultNICDlg.obj
 0001:0007f5d0       __unwindfunclet$?OnBnClickedOk@CSetDrfaultNICDlg@@QAEXXZ$0 004805d0 f   SetDrfaultNICDlg.obj
 0001:0007f5d8       __unwindfunclet$?OnBnClickedOk@CSetDrfaultNICDlg@@QAEXXZ$2 004805d8 f   SetDrfaultNICDlg.obj
 0001:0007f5e1       __ehhandler$?OnBnClickedOk@CSetDrfaultNICDlg@@QAEXXZ 004805e1 f   SetDrfaultNICDlg.obj
 0001:0007f610       __unwindfunclet$?OnInitDialog@CSetDrfaultNICDlg@@UAEHXZ$0 00480610 f   SetDrfaultNICDlg.obj
 0001:0007f61b       __unwindfunclet$?OnInitDialog@CSetDrfaultNICDlg@@UAEHXZ$2 0048061b f   SetDrfaultNICDlg.obj
 0001:0007f627       __unwindfunclet$?OnInitDialog@CSetDrfaultNICDlg@@UAEHXZ$4 00480627 f   SetDrfaultNICDlg.obj
 0001:0007f633       __ehhandler$?OnInitDialog@CSetDrfaultNICDlg@@UAEHXZ 00480633 f   SetDrfaultNICDlg.obj
 0001:0007f660       __unwindfunclet$?GetLocalComputerInfo@CSetDrfaultNICDlg@@QAEHXZ$0 00480660 f   SetDrfaultNICDlg.obj
 0001:0007f66c       __ehhandler$?GetLocalComputerInfo@CSetDrfaultNICDlg@@QAEHXZ 0048066c f   SetDrfaultNICDlg.obj
 0001:0007f6a0       __unwindfunclet$?SetTitle@CSetDrfaultNICDlg@@QAEXXZ$0 004806a0 f   SetDrfaultNICDlg.obj
 0001:0007f6a9       __unwindfunclet$?SetTitle@CSetDrfaultNICDlg@@QAEXXZ$1 004806a9 f   SetDrfaultNICDlg.obj
 0001:0007f6b2       __unwindfunclet$?SetTitle@CSetDrfaultNICDlg@@QAEXXZ$2 004806b2 f   SetDrfaultNICDlg.obj
 0001:0007f6bb       __unwindfunclet$?SetTitle@CSetDrfaultNICDlg@@QAEXXZ$3 004806bb f   SetDrfaultNICDlg.obj
 0001:0007f6c4       __unwindfunclet$?SetTitle@CSetDrfaultNICDlg@@QAEXXZ$4 004806c4 f   SetDrfaultNICDlg.obj
 0001:0007f6cd       __unwindfunclet$?SetTitle@CSetDrfaultNICDlg@@QAEXXZ$5 004806cd f   SetDrfaultNICDlg.obj
 0001:0007f6d6       __ehhandler$?SetTitle@CSetDrfaultNICDlg@@QAEXXZ 004806d6 f   SetDrfaultNICDlg.obj
 0001:0007f700       __unwindfunclet$??0CSpecialPartitionRS@@QAE@PAVCWnd@@@Z$0 00480700 f   SpecialPartitionRS.obj
 0001:0007f708       __unwindfunclet$??0CSpecialPartitionRS@@QAE@PAVCWnd@@@Z$1 00480708 f   SpecialPartitionRS.obj
 0001:0007f713       __unwindfunclet$??0CSpecialPartitionRS@@QAE@PAVCWnd@@@Z$2 00480713 f   SpecialPartitionRS.obj
 0001:0007f722       __ehhandler$??0CSpecialPartitionRS@@QAE@PAVCWnd@@@Z 00480722 f   SpecialPartitionRS.obj
 0001:0007f740       __unwindfunclet$?OnInitDialog@CSpecialPartitionRS@@MAEHXZ$0 00480740 f   SpecialPartitionRS.obj
 0001:0007f749       __unwindfunclet$?OnInitDialog@CSpecialPartitionRS@@MAEHXZ$1 00480749 f   SpecialPartitionRS.obj
 0001:0007f752       __unwindfunclet$?OnInitDialog@CSpecialPartitionRS@@MAEHXZ$2 00480752 f   SpecialPartitionRS.obj
 0001:0007f75b       __unwindfunclet$?OnInitDialog@CSpecialPartitionRS@@MAEHXZ$3 0048075b f   SpecialPartitionRS.obj
 0001:0007f764       __unwindfunclet$?OnInitDialog@CSpecialPartitionRS@@MAEHXZ$4 00480764 f   SpecialPartitionRS.obj
 0001:0007f76d       __unwindfunclet$?OnInitDialog@CSpecialPartitionRS@@MAEHXZ$5 0048076d f   SpecialPartitionRS.obj
 0001:0007f776       __unwindfunclet$?OnInitDialog@CSpecialPartitionRS@@MAEHXZ$6 00480776 f   SpecialPartitionRS.obj
 0001:0007f77f       __unwindfunclet$?OnInitDialog@CSpecialPartitionRS@@MAEHXZ$7 0048077f f   SpecialPartitionRS.obj
 0001:0007f788       __unwindfunclet$?OnInitDialog@CSpecialPartitionRS@@MAEHXZ$8 00480788 f   SpecialPartitionRS.obj
 0001:0007f791       __ehhandler$?OnInitDialog@CSpecialPartitionRS@@MAEHXZ 00480791 f   SpecialPartitionRS.obj
 0001:0007f7b0       __unwindfunclet$?IntiListCtrl@CSpecialPartitionRS@@QAEXXZ$0 004807b0 f   SpecialPartitionRS.obj
 0001:0007f7b9       __unwindfunclet$?IntiListCtrl@CSpecialPartitionRS@@QAEXXZ$1 004807b9 f   SpecialPartitionRS.obj
 0001:0007f7c2       __unwindfunclet$?IntiListCtrl@CSpecialPartitionRS@@QAEXXZ$2 004807c2 f   SpecialPartitionRS.obj
 0001:0007f7dc       __unwindfunclet$?IntiListCtrl@CSpecialPartitionRS@@QAEXXZ$3 004807dc f   SpecialPartitionRS.obj
 0001:0007f7f6       __unwindfunclet$?IntiListCtrl@CSpecialPartitionRS@@QAEXXZ$4 004807f6 f   SpecialPartitionRS.obj
 0001:0007f7ff       __ehhandler$?IntiListCtrl@CSpecialPartitionRS@@QAEXXZ 004807ff f   SpecialPartitionRS.obj
 0001:0007f820       __unwindfunclet$?OnDblclkPartitionList@CSpecialPartitionRS@@IAEXPAUtagNMHDR@@PAJ@Z$0 00480820 f   SpecialPartitionRS.obj
 0001:0007f829       __unwindfunclet$?OnDblclkPartitionList@CSpecialPartitionRS@@IAEXPAUtagNMHDR@@PAJ@Z$1 00480829 f   SpecialPartitionRS.obj
 0001:0007f832       __unwindfunclet$?OnDblclkPartitionList@CSpecialPartitionRS@@IAEXPAUtagNMHDR@@PAJ@Z$2 00480832 f   SpecialPartitionRS.obj
 0001:0007f83b       __unwindfunclet$?OnDblclkPartitionList@CSpecialPartitionRS@@IAEXPAUtagNMHDR@@PAJ@Z$3 0048083b f   SpecialPartitionRS.obj
 0001:0007f844       __unwindfunclet$?OnDblclkPartitionList@CSpecialPartitionRS@@IAEXPAUtagNMHDR@@PAJ@Z$4 00480844 f   SpecialPartitionRS.obj
 0001:0007f84d       __unwindfunclet$?OnDblclkPartitionList@CSpecialPartitionRS@@IAEXPAUtagNMHDR@@PAJ@Z$5 0048084d f   SpecialPartitionRS.obj
 0001:0007f856       __ehhandler$?OnDblclkPartitionList@CSpecialPartitionRS@@IAEXPAUtagNMHDR@@PAJ@Z 00480856 f   SpecialPartitionRS.obj
 0001:0007f880       __unwindfunclet$?OnOK@CSpecialPartitionRS@@MAEXXZ$0 00480880 f   SpecialPartitionRS.obj
 0001:0007f889       __unwindfunclet$?OnOK@CSpecialPartitionRS@@MAEXXZ$4 00480889 f   SpecialPartitionRS.obj
 0001:0007f892       __unwindfunclet$?OnOK@CSpecialPartitionRS@@MAEXXZ$5 00480892 f   SpecialPartitionRS.obj
 0001:0007f89b       __unwindfunclet$?OnOK@CSpecialPartitionRS@@MAEXXZ$6 0048089b f   SpecialPartitionRS.obj
 0001:0007f8a4       __unwindfunclet$?OnOK@CSpecialPartitionRS@@MAEXXZ$7 004808a4 f   SpecialPartitionRS.obj
 0001:0007f8ad       __unwindfunclet$?OnOK@CSpecialPartitionRS@@MAEXXZ$8 004808ad f   SpecialPartitionRS.obj
 0001:0007f8b6       __unwindfunclet$?OnOK@CSpecialPartitionRS@@MAEXXZ$9 004808b6 f   SpecialPartitionRS.obj
 0001:0007f8bf       __ehhandler$?OnOK@CSpecialPartitionRS@@MAEXXZ 004808bf f   SpecialPartitionRS.obj
 0001:0007f8e0       __unwindfunclet$??1CWait@@UAE@XZ$0 004808e0 f   Wait.obj
 0001:0007f8e0       __unwindfunclet$??0CWait@@QAE@PAVCWnd@@@Z$0 004808e0 f   Wait.obj
 0001:0007f8e8       __unwindfunclet$??1CWait@@UAE@XZ$1 004808e8 f   Wait.obj
 0001:0007f8e8       __unwindfunclet$??0CWait@@QAE@PAVCWnd@@@Z$1 004808e8 f   Wait.obj
 0001:0007f8f4       __unwindfunclet$??1CWait@@UAE@XZ$2 004808f4 f   Wait.obj
 0001:0007f8f4       __unwindfunclet$??0CWait@@QAE@PAVCWnd@@@Z$2 004808f4 f   Wait.obj
 0001:0007f903       __unwindfunclet$??0CWait@@QAE@PAVCWnd@@@Z$3 00480903 f   Wait.obj
 0001:0007f903       __unwindfunclet$??1CWait@@UAE@XZ$3 00480903 f   Wait.obj
 0001:0007f912       __ehhandler$??0CWait@@QAE@PAVCWnd@@@Z 00480912 f   Wait.obj
 0001:0007f912       __ehhandler$??1CWait@@UAE@XZ 00480912 f   Wait.obj
 0001:0007f930       __unwindfunclet$?OnInitDialog@CWait@@MAEHXZ$0 00480930 f   Wait.obj
 0001:0007f939       __unwindfunclet$?OnInitDialog@CWait@@MAEHXZ$1 00480939 f   Wait.obj
 0001:0007f942       __ehhandler$?OnInitDialog@CWait@@MAEHXZ 00480942 f   Wait.obj
 0001:0007f960       __unwindfunclet$?OnTimer@CWait@@IAEXI@Z$0 00480960 f   Wait.obj
 0001:0007f969       __unwindfunclet$?OnTimer@CWait@@IAEXI@Z$1 00480969 f   Wait.obj
 0001:0007f972       __ehhandler$?OnTimer@CWait@@IAEXI@Z 00480972 f   Wait.obj
 0001:0007f990       __unwindfunclet$??0CWorkspaceBar2@@QAE@XZ$0 00480990 f   WorkspaceBar.obj
 0001:0007f990       __unwindfunclet$??1CWorkspaceBar@@UAE@XZ$0 00480990 f   WorkspaceBar.obj
 0001:0007f990       __unwindfunclet$??0CWorkspaceBar@@QAE@XZ$0 00480990 f   WorkspaceBar.obj
 0001:0007f990       __unwindfunclet$??1CWorkspaceBar2@@UAE@XZ$0 00480990 f   WorkspaceBar.obj
 0001:0007f998       __ehhandler$??1CWorkspaceBar@@UAE@XZ 00480998 f   WorkspaceBar.obj
 0001:0007f998       __ehhandler$??0CWorkspaceBar2@@QAE@XZ 00480998 f   WorkspaceBar.obj
 0001:0007f998       __ehhandler$??1CWorkspaceBar2@@UAE@XZ 00480998 f   WorkspaceBar.obj
 0001:0007f998       __ehhandler$??0CWorkspaceBar@@QAE@XZ 00480998 f   WorkspaceBar.obj
 0001:0007f9c0       __unwindfunclet$?OnCreate@CWorkspaceBar@@IAEHPAUtagCREATESTRUCTA@@@Z$0 004809c0 f   WorkspaceBar.obj
 0001:0007f9ca       __unwindfunclet$?OnCreate@CWorkspaceBar@@IAEHPAUtagCREATESTRUCTA@@@Z$1 004809ca f   WorkspaceBar.obj
 0001:0007f9d3       __unwindfunclet$?OnCreate@CWorkspaceBar@@IAEHPAUtagCREATESTRUCTA@@@Z$2 004809d3 f   WorkspaceBar.obj
 0001:0007f9dc       __unwindfunclet$?OnCreate@CWorkspaceBar@@IAEHPAUtagCREATESTRUCTA@@@Z$3 004809dc f   WorkspaceBar.obj
 0001:0007f9e5       __ehhandler$?OnCreate@CWorkspaceBar@@IAEHPAUtagCREATESTRUCTA@@@Z 004809e5 f   WorkspaceBar.obj
 0001:0007fa00       __unwindfunclet$?OnPaint@CWorkspaceBar@@IAEXXZ$0 00480a00 f   WorkspaceBar.obj
 0001:0007fa00       __unwindfunclet$?OnPaint@CWorkspaceBar2@@IAEXXZ$0 00480a00 f   WorkspaceBar.obj
 0001:0007fa08       __ehhandler$?OnPaint@CWorkspaceBar@@IAEXXZ 00480a08 f   WorkspaceBar.obj
 0001:0007fa08       __ehhandler$?OnPaint@CWorkspaceBar2@@IAEXXZ 00480a08 f   WorkspaceBar.obj
 0001:0007fa30       __unwindfunclet$?GetCurrentPath@@YAHXZ$0 00480a30 f   comfunc:comfunc.obj
 0001:0007fa3c       __ehhandler$?GetCurrentPath@@YAHXZ 00480a3c f   comfunc:comfunc.obj
 0001:0007fa70       __unwindfunclet$?SetKey@CRegistry@@QAEHV?$CStringT@DV?$StrTraitMFC_DLL@DV?$ChTraitsCRT@D@ATL@@@@@ATL@@H@Z$0 00480a70 f   comfunc:Registry.obj
 0001:0007fa79       __ehhandler$?SetKey@CRegistry@@QAEHV?$CStringT@DV?$StrTraitMFC_DLL@DV?$ChTraitsCRT@D@ATL@@@@@ATL@@H@Z 00480a79 f   comfunc:Registry.obj
 0001:0007faa0       __unwindfunclet$?ReadString@CRegistry@@QAE?AV?$CStringT@DV?$StrTraitMFC_DLL@DV?$ChTraitsCRT@D@ATL@@@@@ATL@@V23@0@Z$0 00480aa0 f   comfunc:Registry.obj
 0001:0007faa9       __unwindfunclet$?ReadString@CRegistry@@QAE?AV?$CStringT@DV?$StrTraitMFC_DLL@DV?$ChTraitsCRT@D@ATL@@@@@ATL@@V23@0@Z$1 00480aa9 f   comfunc:Registry.obj
 0001:0007fab2       __ehhandler$?ReadString@CRegistry@@QAE?AV?$CStringT@DV?$StrTraitMFC_DLL@DV?$ChTraitsCRT@D@ATL@@@@@ATL@@V23@0@Z 00480ab2 f   comfunc:Registry.obj
 0001:0007fae0       __unwindfunclet$?ReadMSZString@CRegistry@@QAEHV?$CStringT@DV?$StrTraitMFC_DLL@DV?$ChTraitsCRT@D@ATL@@@@@ATL@@PAD@Z$0 00480ae0 f   comfunc:Registry.obj
 0001:0007fae9       __ehhandler$?ReadMSZString@CRegistry@@QAEHV?$CStringT@DV?$StrTraitMFC_DLL@DV?$ChTraitsCRT@D@ATL@@@@@ATL@@PAD@Z 00480ae9 f   comfunc:Registry.obj
 0001:0007fb20       __unwindfunclet$?DeleteKey@CRegistry@@QAEHV?$CStringT@DV?$StrTraitMFC_DLL@DV?$ChTraitsCRT@D@ATL@@@@@ATL@@@Z$0 00480b20 f   comfunc:Registry.obj
 0001:0007fb29       __ehhandler$?DeleteKey@CRegistry@@QAEHV?$CStringT@DV?$StrTraitMFC_DLL@DV?$ChTraitsCRT@D@ATL@@@@@ATL@@@Z 00480b29 f   comfunc:Registry.obj
 0001:0007fb50       __unwindfunclet$?TranStrToNode@@YAHPAE0@Z$0 00480b50 f   helpful:helpful.obj
 0001:0007fb59       __unwindfunclet$?TranStrToNode@@YAHPAE0@Z$1 00480b59 f   helpful:helpful.obj
 0001:0007fb62       __ehhandler$?TranStrToNode@@YAHPAE0@Z 00480b62 f   helpful:helpful.obj
 0001:0007fb80       __unwindfunclet$?Initial@CMulticastSocket@@QAEHPAVCWnd@@V?$CStringT@DV?$StrTraitMFC_DLL@DV?$ChTraitsCRT@D@ATL@@@@@ATL@@GPBDIHH@Z$0 00480b80 f   commod2:MulticastSocket.obj
 0001:0007fb89       __ehhandler$?Initial@CMulticastSocket@@QAEHPAVCWnd@@V?$CStringT@DV?$StrTraitMFC_DLL@DV?$ChTraitsCRT@D@ATL@@@@@ATL@@GPBDIHH@Z 00480b89 f   commod2:MulticastSocket.obj
 0001:0007fbb0       __unwindfunclet$??0CMulticastSocket@@QAE@XZ$0 00480bb0 f   commod2:MulticastSocket.obj
 0001:0007fbbe       __ehhandler$??0CMulticastSocket@@QAE@XZ 00480bbe f   commod2:MulticastSocket.obj
 0001:0007fbf0       __unwindfunclet$??1CMulticastSocket@@UAE@XZ$0 00480bf0 f   commod2:MulticastSocket.obj
 0001:0007fbfb       __ehhandler$??1CMulticastSocket@@UAE@XZ 00480bfb f   commod2:MulticastSocket.obj
 0001:0007fc20       __unwindfunclet$?GetDefaultCType@CMyODBC@@QAEFJ@Z$0 00480c20 f   dbmod2:MyODBC.obj
 0001:0007fc29       __ehhandler$?GetDefaultCType@CMyODBC@@QAEFJ@Z 00480c29 f   dbmod2:MyODBC.obj
 0001:0007fc50       __unwindfunclet$?ReportError@CMyODBC@@QAEXAAPAXHV?$CStringT@DV?$StrTraitMFC_DLL@DV?$ChTraitsCRT@D@ATL@@@@@ATL@@@Z$0 00480c50 f   dbmod2:MyODBC.obj
 0001:0007fc59       __unwindfunclet$?ReportError@CMyODBC@@QAEXAAPAXHV?$CStringT@DV?$StrTraitMFC_DLL@DV?$ChTraitsCRT@D@ATL@@@@@ATL@@@Z$1 00480c59 f   dbmod2:MyODBC.obj
 0001:0007fc65       __ehhandler$?ReportError@CMyODBC@@QAEXAAPAXHV?$CStringT@DV?$StrTraitMFC_DLL@DV?$ChTraitsCRT@D@ATL@@@@@ATL@@@Z 00480c65 f   dbmod2:MyODBC.obj
 0001:0007fca0       __unwindfunclet$?SetODBCSource@CMyODBC@@QAEHPAD0@Z$0 00480ca0 f   dbmod2:MyODBC.obj
 0001:0007fca9       __unwindfunclet$?SetODBCSource@CMyODBC@@QAEHPAD0@Z$1 00480ca9 f   dbmod2:MyODBC.obj
 0001:0007fcb2       __ehhandler$?SetODBCSource@CMyODBC@@QAEHPAD0@Z 00480cb2 f   dbmod2:MyODBC.obj
 0001:0007fcd0       __unwindfunclet$?PrepareSql@CMyODBC@@QAEHPBDAAVCODBCSet@@@Z$0 00480cd0 f   dbmod2:MyODBC.obj
 0001:0007fcdc       __unwindfunclet$?PrepareSql@CMyODBC@@QAEHPBDAAVCODBCSet@@@Z$1 00480cdc f   dbmod2:MyODBC.obj
 0001:0007fce8       __ehhandler$?PrepareSql@CMyODBC@@QAEHPBDAAVCODBCSet@@@Z 00480ce8 f   dbmod2:MyODBC.obj
 0001:0007fd20       __unwindfunclet$?ExecTrans@CMyODBC@@QAEHAAVCStringList@@@Z$1 00480d20 f   dbmod2:MyODBC.obj
 0001:0007fd29       __ehhandler$?ExecTrans@CMyODBC@@QAEHAAVCStringList@@@Z 00480d29 f   dbmod2:MyODBC.obj
 0001:0007fd50       __unwindfunclet$?InitKern@CKiboKern@@QAEHXZ$0 00480d50 f   kibokern:kibokern.obj
 0001:0007fd5c       __ehhandler$?InitKern@CKiboKern@@QAEHXZ 00480d5c f   kibokern:kibokern.obj
 0001:0007fd80       __unwindfunclet$??1CKiboKern@@UAE@XZ$0 00480d80 f   kibokern:kibokern.obj
 0001:0007fd8b       __ehhandler$??1CKiboKern@@UAE@XZ 00480d8b f   kibokern:kibokern.obj
 0001:0007fdb0       __unwindfunclet$?ExGetResString@@YA?AV?$CStringT@DV?$StrTraitMFC_DLL@DV?$ChTraitsCRT@D@ATL@@@@@ATL@@PAD0@Z$0 00480db0 f   loadres:exloadres.obj
 0001:0007fdb9       __unwindfunclet$?ExGetResString@@YA?AV?$CStringT@DV?$StrTraitMFC_DLL@DV?$ChTraitsCRT@D@ATL@@@@@ATL@@PAD0@Z$1 00480db9 f   loadres:exloadres.obj
 0001:0007fdc2       __ehhandler$?ExGetResString@@YA?AV?$CStringT@DV?$StrTraitMFC_DLL@DV?$ChTraitsCRT@D@ATL@@@@@ATL@@PAD0@Z 00480dc2 f   loadres:exloadres.obj
 0001:0007fde0       __unwindfunclet$?ExGetResBmp@@YA?AV?$CStringT@DV?$StrTraitMFC_DLL@DV?$ChTraitsCRT@D@ATL@@@@@ATL@@PAD0@Z$0 00480de0 f   loadres:exloadres.obj
 0001:0007fde9       __unwindfunclet$?ExGetResBmp@@YA?AV?$CStringT@DV?$StrTraitMFC_DLL@DV?$ChTraitsCRT@D@ATL@@@@@ATL@@PAD0@Z$1 00480de9 f   loadres:exloadres.obj
 0001:0007fdf2       __unwindfunclet$?ExGetResBmp@@YA?AV?$CStringT@DV?$StrTraitMFC_DLL@DV?$ChTraitsCRT@D@ATL@@@@@ATL@@PAD0@Z$2 00480df2 f   loadres:exloadres.obj
 0001:0007fdfa       __unwindfunclet$?ExGetResBmp@@YA?AV?$CStringT@DV?$StrTraitMFC_DLL@DV?$ChTraitsCRT@D@ATL@@@@@ATL@@PAD0@Z$3 00480dfa f   loadres:exloadres.obj
 0001:0007fe03       __unwindfunclet$?ExGetResBmp@@YA?AV?$CStringT@DV?$StrTraitMFC_DLL@DV?$ChTraitsCRT@D@ATL@@@@@ATL@@PAD0@Z$4 00480e03 f   loadres:exloadres.obj
 0001:0007fe1d       __ehhandler$?ExGetResBmp@@YA?AV?$CStringT@DV?$StrTraitMFC_DLL@DV?$ChTraitsCRT@D@ATL@@@@@ATL@@PAD0@Z 00480e1d f   loadres:exloadres.obj
 0001:0007fe40       __unwindfunclet$?ExCheckAllRes@@YAHPBD@Z$0 00480e40 f   loadres:exloadres.obj
 0001:0007fe4b       __unwindfunclet$?ExCheckAllRes@@YAHPBD@Z$1 00480e4b f   loadres:exloadres.obj
 0001:0007fe57       __unwindfunclet$?ExCheckAllRes@@YAHPBD@Z$2 00480e57 f   loadres:exloadres.obj
 0001:0007fe63       __unwindfunclet$?ExCheckAllRes@@YAHPBD@Z$3 00480e63 f   loadres:exloadres.obj
 0001:0007fe6f       __unwindfunclet$?ExCheckAllRes@@YAHPBD@Z$4 00480e6f f   loadres:exloadres.obj
 0001:0007fe7a       __unwindfunclet$?ExCheckAllRes@@YAHPBD@Z$5 00480e7a f   loadres:exloadres.obj
 0001:0007fe86       __unwindfunclet$?ExCheckAllRes@@YAHPBD@Z$6 00480e86 f   loadres:exloadres.obj
 0001:0007fe92       __unwindfunclet$?ExCheckAllRes@@YAHPBD@Z$7 00480e92 f   loadres:exloadres.obj
 0001:0007fe9e       __unwindfunclet$?ExCheckAllRes@@YAHPBD@Z$8 00480e9e f   loadres:exloadres.obj
 0001:0007feaa       __unwindfunclet$?ExCheckAllRes@@YAHPBD@Z$9 00480eaa f   loadres:exloadres.obj
 0001:0007feb6       __unwindfunclet$?ExCheckAllRes@@YAHPBD@Z$10 00480eb6 f   loadres:exloadres.obj
 0001:0007fec2       __unwindfunclet$?ExCheckAllRes@@YAHPBD@Z$11 00480ec2 f   loadres:exloadres.obj
 0001:0007fece       __ehhandler$?ExCheckAllRes@@YAHPBD@Z 00480ece f   loadres:exloadres.obj
 0001:0007fef0       __unwindfunclet$?addsection@CIniStruct@@QAEHPAD@Z$0 00480ef0 f   loadres:initwork.obj
 0001:0007fef9       __ehhandler$?addsection@CIniStruct@@QAEHPAD@Z 00480ef9 f   loadres:initwork.obj
 0001:0007ff20       __unwindfunclet$?ReadProfileSection@@YAKPBD0AAVCIniStruct@@@Z$0 00480f20 f   loadres:initwork.obj
 0001:0007ff2c       __ehhandler$?ReadProfileSection@@YAKPBD0AAVCIniStruct@@@Z 00480f2c f   loadres:initwork.obj
 0001:0007ff60       __unwindfunclet$??HATL@@YA?AV?$CStringT@DV?$StrTraitMFC_DLL@DV?$ChTraitsCRT@D@ATL@@@@@0@ABV10@0@Z$0 00480f60 f   loadres:initwork.obj
 0001:0007ff7a       __ehhandler$??HATL@@YA?AV?$CStringT@DV?$StrTraitMFC_DLL@DV?$ChTraitsCRT@D@ATL@@@@@0@ABV10@0@Z 00480f7a f   loadres:initwork.obj
 0001:0007ffa0       __unwindfunclet$?replacestr@@YAXPAD00@Z$0 00480fa0 f   loadres:initwork.obj
 0001:0007ffa9       __unwindfunclet$?replacestr@@YAXPAD00@Z$1 00480fa9 f   loadres:initwork.obj
 0001:0007ffb2       __unwindfunclet$?replacestr@@YAXPAD00@Z$2 00480fb2 f   loadres:initwork.obj
 0001:0007ffbb       __unwindfunclet$?replacestr@@YAXPAD00@Z$3 00480fbb f   loadres:initwork.obj
 0001:0007ffc4       __unwindfunclet$?replacestr@@YAXPAD00@Z$4 00480fc4 f   loadres:initwork.obj
 0001:0007ffcd       __unwindfunclet$?replacestr@@YAXPAD00@Z$5 00480fcd f   loadres:initwork.obj
 0001:0007ffd6       __ehhandler$?replacestr@@YAXPAD00@Z 00480fd6 f   loadres:initwork.obj
 0001:00080000       __unwindfunclet$?ReadIniFileKey@@YAAAV?$CStringT@DV?$StrTraitMFC_DLL@DV?$ChTraitsCRT@D@ATL@@@@@ATL@@PBD0PADAAV12@@Z$0 00481000 f   loadres:initwork.obj
 0001:0008000b       __unwindfunclet$?ReadIniFileKey@@YAAAV?$CStringT@DV?$StrTraitMFC_DLL@DV?$ChTraitsCRT@D@ATL@@@@@ATL@@PBD0PADAAV12@@Z$1 0048100b f   loadres:initwork.obj
 0001:00080017       __unwindfunclet$?ReadIniFileKey@@YAAAV?$CStringT@DV?$StrTraitMFC_DLL@DV?$ChTraitsCRT@D@ATL@@@@@ATL@@PBD0PADAAV12@@Z$2 00481017 f   loadres:initwork.obj
 0001:00080023       __ehhandler$?ReadIniFileKey@@YAAAV?$CStringT@DV?$StrTraitMFC_DLL@DV?$ChTraitsCRT@D@ATL@@@@@ATL@@PBD0PADAAV12@@Z 00481023 f   loadres:initwork.obj
 0001:00080060       ??__Eg_mainPwd@@YAXXZ      00481060 f   KiboManager.obj
 0001:00080080       ??__EtheApp@@YAXXZ         00481080 f   KiboManager.obj
 0001:000800a0       ??__Em_bootMgr@@YAXXZ      004810a0 f   MainFrm.obj
 0001:000800c0       ??__Eg_sock@@YAXXZ         004810c0 f   MainFrm.obj
 0001:000800e0       ??__Eg_strStatusBarMain@@YAXXZ 004810e0 f   MainFrm.obj
 0001:00080100       ??__Eg_arrMessage@@YAXXZ   00481100 f   MainFrm.obj
 0001:00080120       ??__Eg_strStatusBarOther@@YAXXZ 00481120 f   MainFrm.obj
 0001:00080140       ??__Eg_ipAddr@@YAXXZ       00481140 f   MainFrm.obj
 0001:00080160       ??__Eg_macname@@YAXXZ      00481160 f   MainFrm.obj
 0001:00080180       ??__EgVersion@@YAXXZ       00481180 f   MainFrm.obj
 0001:000801a0       ??__Eg_hdserialinfo@@YAXXZ 004811a0 f   MainFrm.obj
 0001:000801c0       ??__Eg_regserialinfo@@YAXXZ 004811c0 f   MainFrm.obj
 0001:000801e0       ??__Em_GroupTree@@YAXXZ    004811e0 f   MyEdit.obj
 0001:00080200       ??__E_afxDefaultAcceleratorDelimiter@@YAXXZ 00481200 f   stdafx.obj
 0001:00080230       ??__Eg_CurrentPath@@YAXXZ  00481230 f   comfunc:comfunc.obj
 0001:00080250       ??__Eg_tempstring@@YAXXZ   00481250 f   loadres:exloadres.obj
 0001:00080270       ??__Eg_BasicPath@@YAXXZ    00481270 f   loadres:exloadres.obj
 0001:00080290       ??__EvtMissing@@YAXXZ      00481290 f   comsuppw:comutil.obj
 0001:0008029c       ??__E_afxInitAppState@@YAXXZ 0048129c f   mfcs90:appmodul.obj
 0001:000802b0       ??__Fg_mainPwd@@YAXXZ      004812b0 f   KiboManager.obj
 0001:000802c0       ??__FtheApp@@YAXXZ         004812c0 f   KiboManager.obj
 0001:000802d0       ??__Fm_bootMgr@@YAXXZ      004812d0 f   MainFrm.obj
 0001:000802e0       ??__Fg_sock@@YAXXZ         004812e0 f   MainFrm.obj
 0001:000802f0       ??__Fg_strStatusBarMain@@YAXXZ 004812f0 f   MainFrm.obj
 0001:00080300       ??__Fg_arrMessage@@YAXXZ   00481300 f   MainFrm.obj
 0001:00080310       ??__Fg_strStatusBarOther@@YAXXZ 00481310 f   MainFrm.obj
 0001:00080320       ??__Fg_ipAddr@@YAXXZ       00481320 f   MainFrm.obj
 0001:00080330       ??__Fg_macname@@YAXXZ      00481330 f   MainFrm.obj
 0001:00080340       ??__FgVersion@@YAXXZ       00481340 f   MainFrm.obj
 0001:00080350       ??__Fg_hdserialinfo@@YAXXZ 00481350 f   MainFrm.obj
 0001:00080360       ??__Fg_regserialinfo@@YAXXZ 00481360 f   MainFrm.obj
 0001:00080370       ??__Fm_GroupTree@@YAXXZ    00481370 f   MyEdit.obj
 0001:00080380       ??__F_afxDefaultAcceleratorDelimiter@@YAXXZ 00481380 f   stdafx.obj
 0001:00080390       ??__Fg_CurrentPath@@YAXXZ  00481390 f   comfunc:comfunc.obj
 0001:000803a0       ??__Fg_tempstring@@YAXXZ   004813a0 f   loadres:exloadres.obj
 0001:000803b0       ??__Fg_BasicPath@@YAXXZ    004813b0 f   loadres:exloadres.obj
 0001:000803c0       ??__FvtMissing@@YAXXZ      004813c0 f   comsuppw:comutil.obj
